 VV3

 Timestamp is 482a46ab (Tue May 13 18:55:55 2008)

 Preferred load address is 00400000

 Start         Length     Name                   Class
 0001:00000000 000f320eH .text                   CODE
 0001:000f3210 000025d5H .text$x                 CODE
 0001:000f57f0 00012e85H .text$yc                CODE
 0001:00108680 000000e9H .text$yd                CODE
 0002:00000000 00000434H .idata$5                DATA
 0002:00000440 0002aab8H .rdata                  DATA
 0002:0002aef8 00000044H .rdata$r                DATA
 0002:0002af3c 00000004H .rtc$IAA                DATA
 0002:0002af40 00000004H .rtc$IZZ                DATA
 0002:0002af44 00000004H .rtc$TAA                DATA
 0002:0002af48 00000004H .rtc$TZZ                DATA
 0002:0002af50 00003038H .xdata$x                DATA
 0002:0002df88 00000000H ATL$__a                 DATA
 0002:0002df88 00000000H ATL$__z                 DATA
 0002:0002df88 000000dcH .idata$2                DATA
 0002:0002e064 00000014H .idata$3                DATA
 0002:0002e078 00000434H .idata$4                DATA
 0002:0002e4ac 00001210H .idata$6                DATA
 0002:0002f6bc 00000000H .edata                  DATA
 0003:00000000 00000004H .CRT$XCA                DATA
 0003:00000004 00000004H .CRT$XCAA               DATA
 0003:00000008 00000004H .CRT$XCL                DATA
 0003:0000000c 000022d4H .CRT$XCU                DATA
 0003:000022e0 00000004H .CRT$XCZ                DATA
 0003:000022e4 00000004H .CRT$XIA                DATA
 0003:000022e8 00000010H .CRT$XIC                DATA
 0003:000022f8 00000004H .CRT$XIY                DATA
 0003:000022fc 00000004H .CRT$XIZ                DATA
 0003:00002300 00000004H .CRT$XPA                DATA
 0003:00002304 00000004H .CRT$XPX                DATA
 0003:00002308 00000004H .CRT$XPZ                DATA
 0003:0000230c 00000004H .CRT$XTA                DATA
 0003:00002310 00000004H .CRT$XTB                DATA
 0003:00002314 00000004H .CRT$XTZ                DATA
 0003:00002320 0000ec60H .data                   DATA
 0003:00010f80 001affd8H .bss                    DATA
 0004:00000000 00000004H .shr                    DATA
 0005:00000000 00000354H .rsrc$01                DATA
 0005:00000360 0002b700H .rsrc$02                DATA

  Address         Publics by Value              Rva+Base     Lib:Object

 0000:00000000       ___safe_se_handler_table   00000000     <absolute>
 0000:00000000       __except_list              00000000     <absolute>
 0000:00000000       ___safe_se_handler_count   00000000     <absolute>
 0000:00000000       ___ImageBase               00400000     <linker-defined>
 0001:00000000       ??_H@YGXPAXIHP6EPAX0@Z@Z   00401000 f i ldwButton.obj
 0001:00000030       ??0ldwButton@@QAE@HPBDUldwPoint@@PAVldwScene@@_N@Z 00401030 f   ldwButton.obj
 0001:000000e0       ??0ldwButton@@QAE@HPAVldwImageStrip@@UldwPoint@@PAVldwScene@@_N@Z 004010e0 f   ldwButton.obj
 0001:00000190       ??1ldwButton@@UAE@XZ       00401190 f   ldwButton.obj
 0001:00000210       ?SetPos@ldwButton@@UAEXHH@Z 00401210 f   ldwButton.obj
 0001:00000230       ?GetWidth@ldwButton@@UAEHXZ 00401230 f   ldwButton.obj
 0001:00000250       ?GetHeight@ldwButton@@UAEHXZ 00401250 f   ldwButton.obj
 0001:00000270       ?SetActive@ldwButton@@UAEX_N@Z 00401270 f   ldwButton.obj
 0001:00000290       ?Draw@ldwButton@@UAEXXZ    00401290 f   ldwButton.obj
 0001:000002f0       ?GetBounds@ldwButton@@UAEXAAUldwRect@@@Z 004012f0 f   ldwButton.obj
 0001:00000370       ?SetText@ldwButton@@QAEXPBDPAVldwFont@@@Z 00401370 f   ldwButton.obj
 0001:00000390       ?SetText@ldwButton@@QAEXPBGPAVldwFont@@@Z 00401390 f   ldwButton.obj
 0001:000003b0       ?SetText@ldwButton@@QAEXPBDUldwColor@@11PAVldwFont@@@Z 004013b0 f   ldwButton.obj
 0001:00000400       ?SetText@ldwButton@@QAEXPBGUldwColor@@11PAVldwFont@@@Z 00401400 f   ldwButton.obj
 0001:00000450       ?SetSoundFx@ldwButton@@QAEXPAVldwSoundFx@@0@Z 00401450 f   ldwButton.obj
 0001:00000470       ?Enable@ldwButton@@QAEX_N@Z 00401470 f   ldwButton.obj
 0001:00000490       ?SetDisabledTint@ldwButton@@QAEXUldwColor@@@Z 00401490 f   ldwButton.obj
 0001:000004b0       ?DrawDownState@ldwButton@@MAEXXZ 004014b0 f   ldwButton.obj
 0001:000004d0       ?DrawUpState@ldwButton@@MAEXXZ 004014d0 f   ldwButton.obj
 0001:000004f0       ?DrawOverState@ldwButton@@MAEXXZ 004014f0 f   ldwButton.obj
 0001:00000510       ?GetFont@ldwButton@@IAEPAVldwFont@@XZ 00401510 f   ldwButton.obj
 0001:00000530       ??0ldwButtonImpl@@QAE@HPBDUldwPoint@@PAVldwScene@@PAVldwHintControl@@_N@Z 00401530 f i ldwButton.obj
 0001:000006c0       ??0ldwPoint@@QAE@XZ        004016c0 f i ldwButton.obj
 0001:000006f0       ?SetPos@ldwButtonImpl@@QAEXHH@Z 004016f0 f i ldwButton.obj
 0001:00000760       ??0ldwRect@@QAE@XZ         00401760 f i ldwButton.obj
 0001:000007a0       ?HandleMouse@ldwButtonImpl@@UAE_NHUldwPoint@@@Z 004017a0 f i ldwButton.obj
 0001:000009f0       ??0ldwColor@@QAE@XZ        004019f0 f i ldwButton.obj
 0001:00000a20       ??_GldwButtonImpl@@UAEPAXI@Z 00401a20 f i ldwButton.obj
 0001:00000a20       ??_EldwButtonImpl@@UAEPAXI@Z 00401a20 f i ldwButton.obj
 0001:00000a50       ??1ldwButtonImpl@@UAE@XZ   00401a50 f i ldwButton.obj
 0001:00000b20       ??_EldwButton@@UAEPAXI@Z   00401b20 f i ldwButton.obj
 0001:00000b20       ??_GldwButton@@UAEPAXI@Z   00401b20 f i ldwButton.obj
 0001:00000b50       ??0ldwButtonImpl@@QAE@HPAVldwImageStrip@@UldwPoint@@PAVldwScene@@PAVldwHintControl@@_N@Z 00401b50 f i ldwButton.obj
 0001:00000ca0       ?GetWidth@ldwButtonImpl@@QAEHXZ 00401ca0 f i ldwButton.obj
 0001:00000ce0       ?Width@ldwRect@@QAEHXZ     00401ce0 f i ldwButton.obj
 0001:00000d00       ?GetHeight@ldwButtonImpl@@QAEHXZ 00401d00 f i ldwButton.obj
 0001:00000d40       ?Height@ldwRect@@QAEHXZ    00401d40 f i ldwButton.obj
 0001:00000d60       ?SetActive@ldwButtonImpl@@QAEX_N@Z 00401d60 f i ldwButton.obj
 0001:00000dc0       ??1ldwEventHandler@@UAE@XZ 00401dc0 f i ldwButton.obj
 0001:00000de0       ?HandleKey@ldwEventHandler@@UAE_NHHH@Z 00401de0 f i ldwButton.obj
 0001:00000de0       ?HandleMouse@ldwEventHandler@@UAE_NHUldwPoint@@@Z 00401de0 f i ldwButton.obj
 0001:00000df0       ?HandleMessage@ldwEventHandler@@UAE_NHJ@Z 00401df0 f i ldwButton.obj
 0001:00000df0       ?Load@ldwFontImpl@@QAE_NPBDPAUFontTable@ldwFont@@@Z 00401df0 f i ldwFont.obj
 0001:00000e00       ??0ldwEventHandler@@IAE@XZ 00401e00 f i ldwButton.obj
 0001:00000e20       ??_GldwEventHandler@@UAEPAXI@Z 00401e20 f i ldwButton.obj
 0001:00000e20       ??_EldwEventHandler@@UAEPAXI@Z 00401e20 f i ldwButton.obj
 0001:00000e50       ?SetText@ldwButtonImpl@@QAEXPBDPAVldwFont@@@Z 00401e50 f i ldwButton.obj
 0001:00000f40       ?Inset@ldwRect@@QAEXH@Z    00401f40 f i ldwButton.obj
 0001:00000f90       ?SetText@ldwButtonImpl@@QAEXPBGPAVldwFont@@@Z 00401f90 f i ldwButton.obj
 0001:000010a0       ?SetSoundFx@ldwButtonImpl@@QAEXPAVldwSoundFx@@0@Z 004020a0 f i ldwButton.obj
 0001:000010c0       ?Enable@ldwButtonImpl@@QAEX_N@Z 004020c0 f i ldwButton.obj
 0001:000010f0       ?SetDisabledTint@ldwButtonImpl@@QAEXUldwColor@@@Z 004020f0 f i ldwButton.obj
 0001:00001110       ?Draw@ldwButtonImpl@@QAEXH@Z 00402110 f i ldwButton.obj
 0001:000013b0       ??0ldwColor@@QAE@EEEE@Z    004023b0 f i ldwButton.obj
 0001:000013f0       ??0ldwDialog@@QAE@XZ       004023f0 f   ldwDialog.obj
 0001:00001420       ??1ldwDialog@@UAE@XZ       00402420 f   ldwDialog.obj
 0001:00001480       ?DoModal@ldwDialog@@QAEHPAVldwScene@@_N@Z 00402480 f   ldwDialog.obj
 0001:00001530       ?SetSize@ldwDialog@@IAEXHH@Z 00402530 f   ldwDialog.obj
 0001:000015b0       ?SetPos@ldwDialog@@IAEXHH@Z 004025b0 f   ldwDialog.obj
 0001:00001630       ?Update@ldwDialog@@UAEXXZ  00402630 f   ldwDialog.obj
 0001:00001670       ?Draw@ldwDialog@@UAEXXZ    00402670 f   ldwDialog.obj
 0001:00001710       ??_EldwDialog@@UAEPAXI@Z   00402710 f i ldwDialog.obj
 0001:00001710       ??_GldwDialog@@UAEPAXI@Z   00402710 f i ldwDialog.obj
 0001:00001740       ??0ldwRect@@QAE@HHHH@Z     00402740 f i ldwDialog.obj
 0001:00001780       ?Get@ldwEventManager@@SAPAV1@XZ 00402780 f   ldwEventManager.obj
 0001:00001800       ?Destroy@ldwEventManager@@SAXXZ 00402800 f   ldwEventManager.obj
 0001:00001840       ?Subscribe@ldwEventManager@@QAEXPAVldwEventHandler@@H_N@Z 00402840 f   ldwEventManager.obj
 0001:00001870       ?Unsubscribe@ldwEventManager@@QAEXPAVldwEventHandler@@H@Z 00402870 f   ldwEventManager.obj
 0001:00001890       ?SetModal@ldwEventManager@@QAEXPAVldwEventHandler@@@Z 00402890 f   ldwEventManager.obj
 0001:000018b0       ?HandleMouse@ldwEventManager@@QAEXHUldwPoint@@@Z 004028b0 f   ldwEventManager.obj
 0001:000018e0       ?HandleKey@ldwEventManager@@QAEXHHH@Z 004028e0 f   ldwEventManager.obj
 0001:00001910       ?HandleMessage@ldwEventManager@@QAEXHJ@Z 00402910 f   ldwEventManager.obj
 0001:00001930       ?PostAMessage@ldwEventManager@@QAEXHJ@Z 00402930 f   ldwEventManager.obj
 0001:00001950       ?CaptureMouse@ldwEventManager@@QAEXPAVldwEventHandler@@@Z 00402950 f   ldwEventManager.obj
 0001:00001970       ?ReleaseMouse@ldwEventManager@@QAEXXZ 00402970 f   ldwEventManager.obj
 0001:00001990       ?GetMousePosition@ldwEventManager@@SA?AUldwPoint@@XZ 00402990 f   ldwEventManager.obj
 0001:000019b0       ?GetLeftButtonDown@ldwEventManager@@SA_NXZ 004029b0 f   ldwEventManager.obj
 0001:000019d0       ?GetMilliseconds@ldwEventManager@@SAKXZ 004029d0 f   ldwEventManager.obj
 0001:000019e0       ?Get100thSeconds@ldwEventManager@@SAKXZ 004029e0 f   ldwEventManager.obj
 0001:00001a00       ?GetMillisecondsFromNow@ldwEventManager@@SAKK@Z 00402a00 f   ldwEventManager.obj
 0001:00001a10       ?GetSeconds@ldwEventManager@@SAKXZ 00402a10 f   ldwEventManager.obj
 0001:00001a30       ?GetSecondsFromNow@ldwEventManager@@SAKK@Z 00402a30 f   ldwEventManager.obj
 0001:00001a40       ?Sleep@ldwEventManager@@SAXH@Z 00402a40 f   ldwEventManager.obj
 0001:00001a50       ??0ldwEventManager@@AAE@XZ 00402a50 f   ldwEventManager.obj
 0001:00001ad0       ??1ldwEventManager@@AAE@XZ 00402ad0 f   ldwEventManager.obj
 0001:00001b10       ??_GldwEventManager@@AAEPAXI@Z 00402b10 f i ldwEventManager.obj
 0001:00001b40       ?Subscribe@ldwEventManagerImpl@@QAEXPAVldwEventHandler@@H_N@Z 00402b40 f i ldwEventManager.obj
 0001:00001be0       ?Unsubscribe@ldwEventManagerImpl@@QAEXPAVldwEventHandler@@H@Z 00402be0 f i ldwEventManager.obj
 0001:00001c60       ??0handlerNode@ldwEventManagerImpl@@QAE@PAVldwEventHandler@@H_NPAV01@@Z 00402c60 f i ldwEventManager.obj
 0001:00001ca0       ?SetModal@ldwEventManagerImpl@@QAEXPAVldwEventHandler@@@Z 00402ca0 f i ldwEventManager.obj
 0001:00001ce0       ?HandleMouse@ldwEventManagerImpl@@QAEXHUldwPoint@@@Z 00402ce0 f i ldwEventManager.obj
 0001:00001dd0       ?HandleKey@ldwEventManagerImpl@@QAEXHHH@Z 00402dd0 f i ldwEventManager.obj
 0001:00001e50       ?HandleMessage@ldwEventManagerImpl@@QAEXHJ@Z 00402e50 f i ldwEventManager.obj
 0001:00001ed0       ?ReleaseMouse@ldwEventManagerImpl@@QAEXXZ 00402ed0 f i ldwEventManager.obj
 0001:00001ef0       ??0ldwEventManagerImpl@@QAE@XZ 00402ef0 f i ldwEventManager.obj
 0001:00001f20       ??_GldwEventManagerImpl@@QAEPAXI@Z 00402f20 f i ldwEventManager.obj
 0001:00001f50       ??1ldwEventManagerImpl@@QAE@XZ 00402f50 f i ldwEventManager.obj
 0001:00001f90       ??0ldwFont@@QAE@XZ         00402f90 f   ldwFont.obj
 0001:00002010       ??1ldwFont@@UAE@XZ         00403010 f   ldwFont.obj
 0001:00002060       ?Load@ldwFont@@IAE_NPBDPAUFontTable@1@@Z 00403060 f   ldwFont.obj
 0001:00002080       ?Load@ldwFont@@IAE_NPBDPAUFontTableEx@1@H@Z 00403080 f   ldwFont.obj
 0001:000020b0       ?GetWidth@ldwFont@@QAEHPBD@Z 004030b0 f   ldwFont.obj
 0001:000020d0       ?GetWidth@ldwFont@@QAEHPBG@Z 004030d0 f   ldwFont.obj
 0001:000020f0       ?GetWidth@ldwFont@@QAEHH@Z 004030f0 f   ldwFont.obj
 0001:00002110       ?GetHeight@ldwFont@@QAEHPBD@Z 00403110 f   ldwFont.obj
 0001:00002130       ?GetJustifiedHeight@ldwFont@@QAEHPBDH@Z 00403130 f   ldwFont.obj
 0001:00002150       ?GetNextJustifiedLine@ldwFont@@QAEPADPAD0HHAA_N@Z 00403150 f   ldwFont.obj
 0001:00002180       ?GetHeight@ldwFont@@QAEHPBG@Z 00403180 f   ldwFont.obj
 0001:000021a0       ?GetJustifiedHeight@ldwFont@@QAEHPBGH@Z 004031a0 f   ldwFont.obj
 0001:000021c0       ?GetNextJustifiedLine@ldwFont@@QAEPAGPAG0HHAA_N@Z 004031c0 f   ldwFont.obj
 0001:000021f0       ?SetColor@ldwFont@@QAEXMMMM@Z 004031f0 f   ldwFont.obj
 0001:00002220       ?SetColor@ldwFont@@QAEXUldwColor@@@Z 00403220 f   ldwFont.obj
 0001:00002240       ?SetExtraKerning@ldwFont@@QAEXH@Z 00403240 f   ldwFont.obj
 0001:00002260       ??_EldwFont@@UAEPAXI@Z     00403260 f i ldwFont.obj
 0001:00002260       ??_GldwFont@@UAEPAXI@Z     00403260 f i ldwFont.obj
 0001:00002290       ??_GldwFontImpl@@QAEPAXI@Z 00403290 f i ldwFont.obj
 0001:000022c0       ??0ldwFontImpl@@QAE@XZ     004032c0 f   ldwFontImpl.obj
 0001:00002320       ??1ldwFontImpl@@QAE@XZ     00403320 f   ldwFontImpl.obj
 0001:000023c0       ?GetWidth@ldwFontImpl@@QAEHPBD@Z 004033c0 f   ldwFontImpl.obj
 0001:00002490       ?GetWidth@ldwFontImpl@@QAEHPBG@Z 00403490 f   ldwFontImpl.obj
 0001:00002560       ?GetWidth@ldwFontImpl@@QAEHH@Z 00403560 f   ldwFontImpl.obj
 0001:00002590       ?GetHeight@ldwFontImpl@@QAEHPBD@Z 00403590 f   ldwFontImpl.obj
 0001:000025f0       ?GetHeight@ldwFontImpl@@QAEHPBG@Z 004035f0 f   ldwFontImpl.obj
 0001:00002650       ?GetJustifiedHeight@ldwFontImpl@@QAEHPBDH@Z 00403650 f   ldwFontImpl.obj
 0001:000026f0       ?GetJustifiedHeight@ldwFontImpl@@QAEHPBGH@Z 004036f0 f   ldwFontImpl.obj
 0001:00002790       ?GetNextJustifiedLine@ldwFontImpl@@QAEPADPAD0HHAA_N@Z 00403790 f   ldwFontImpl.obj
 0001:00002920       ?GetNextJustifiedLine@ldwFontImpl@@QAEPAGPAG0HHAA_N@Z 00403920 f   ldwFontImpl.obj
 0001:00002ab0       ?SetColor@ldwFontImpl@@QAEXMMMM@Z 00403ab0 f   ldwFontImpl.obj
 0001:00002ac0       ?SetColor@ldwFontImpl@@QAEXUldwColor@@@Z 00403ac0 f   ldwFontImpl.obj
 0001:00002ad0       ?Load@ldwFontImpl@@QAE_NPBDPAUFontTableEx@ldwFont@@H@Z 00403ad0 f   ldwFontImpl.obj
 0001:00002ec0       ?GetImage@ldwFontImpl@@QAEPAVCGapiRGBASurface@@UldwColor@@@Z 00403ec0 f   ldwFontImpl.obj
 0001:00003140       ?GetCharSourceRect@ldwFontImpl@@QAEXHAAUldwRect@@@Z 00404140 f   ldwFontImpl.obj
 0001:000031d0       ??_GldwImageImpl@@QAEPAXI@Z 004041d0 f i ldwFontImpl.obj
 0001:00003200       ??0fontImageNode@ldwFontImpl@@QAE@UldwColor@@PAVCGapiRGBASurface@@PAV01@@Z 00404200 f i ldwFontImpl.obj
 0001:00003230       ??0ldwGame@@QAE@XZ         00404230 f   ldwGame.obj
 0001:000032f0       ??1ldwGame@@UAE@XZ         004042f0 f   ldwGame.obj
 0001:00003350       ?Run@ldwGame@@UAEXXZ       00404350 f   ldwGame.obj
 0001:000033a0       ?LaunchURL@ldwGame@@SAXPBD@Z 004043a0 f   ldwGame.obj
 0001:000033c0       ??_EldwGame@@UAEPAXI@Z     004043c0 f i ldwGame.obj
 0001:000033c0       ??_GldwGame@@UAEPAXI@Z     004043c0 f i ldwGame.obj
 0001:000033f0       ?GetConfigPath@ldwGameState@@SAXPADH@Z 004043f0 f   ldwGameState.obj
 0001:00003450       ?GetConfigValue@ldwGameState@@SAHPBDH0@Z 00404450 f   ldwGameState.obj
 0001:000034d0       ?GetConfigString@ldwGameState@@SAXPADHPBD11@Z 004044d0 f   ldwGameState.obj
 0001:00003570       ?Get@ldwGameState@@SAPAV1@XZ 00404570 f   ldwGameState.obj
 0001:00003580       ??0ldwGameState@@IAE@XZ    00404580 f   ldwGameState.obj
 0001:000035d0       ??1ldwGameState@@MAE@XZ    004045d0 f   ldwGameState.obj
 0001:000035f0       ?MakePath@ldwGameState@@SAPBDPBD_N@Z 004045f0 f   ldwGameState.obj
 0001:00003750       ?MakeDesktopPath@ldwGameState@@SAPBDPBD@Z 00404750 f   ldwGameState.obj
 0001:000037b0       ?MakeImagePath@ldwGameState@@UAEPBDPBD@Z 004047b0 f   ldwGameState.obj
 0001:000038c0       ?MakeSoundPath@ldwGameState@@UAEPBDPBD@Z 004048c0 f   ldwGameState.obj
 0001:000039c0       ?MakeAssetsPath@ldwGameState@@UAEPBDPBD@Z 004049c0 f   ldwGameState.obj
 0001:00003ad0       ?MakeGameStatePath@ldwGameState@@UAEPBDH@Z 00404ad0 f   ldwGameState.obj
 0001:00003b20       ?GetRandom@ldwGameState@@SAHH@Z 00404b20 f   ldwGameState.obj
 0001:00003b40       ?GetSecondsFromGameStart@ldwGameState@@QAEKXZ 00404b40 f   ldwGameState.obj
 0001:00003ba0       ?SetImageResourceFile@ldwGameState@@QAEXPBD@Z 00404ba0 f   ldwGameState.obj
 0001:00003bb0       ?Save@ldwGameState@@IAE_NPAXKH@Z 00404bb0 f   ldwGameState.obj
 0001:00003c50       ?Load@ldwGameState@@IAE_NPAXKH@Z 00404c50 f   ldwGameState.obj
 0001:00003d40       ?RemoveFile@ldwGameState@@IAEXH@Z 00404d40 f   ldwGameState.obj
 0001:00003d70       ??_GldwGameState@@MAEPAXI@Z 00404d70 f i ldwGameState.obj
 0001:00003d70       ??_EldwGameState@@MAEPAXI@Z 00404d70 f i ldwGameState.obj
 0001:00003da0       ?GetFrameRate@ldwGameState@@UAEHXZ 00404da0 f i ldwGameState.obj
 0001:00003db0       ?Create@ldwGameWindow@@SAPAV1@HHPBD_NH@Z 00404db0 f   ldwGameWindow.obj
 0001:00003e40       ?Get@ldwGameWindow@@SAPAV1@XZ 00404e40 f   ldwGameWindow.obj
 0001:00003e50       ?Destroy@ldwGameWindow@@SAXXZ 00404e50 f   ldwGameWindow.obj
 0001:00003e90       ??0ldwGameWindow@@AAE@HHPBD_NH@Z 00404e90 f   ldwGameWindow.obj
 0001:00003f20       ??1ldwGameWindow@@AAE@XZ   00404f20 f   ldwGameWindow.obj
 0001:00003f80       ?Close@ldwGameWindow@@QAEXXZ 00404f80 f   ldwGameWindow.obj
 0001:00003fa0       ?GetFormat@ldwGameWindow@@QAE?AW4ELdwGraphicsFormat@@XZ 00404fa0 f   ldwGameWindow.obj
 0001:00003fb0       ?SetFrameRate@ldwGameWindow@@QAEXH@Z 00404fb0 f   ldwGameWindow.obj
 0001:00003fd0       ?GetPixel@ldwGameWindow@@QAE?AUldwColor@@HH@Z 00404fd0 f   ldwGameWindow.obj
 0001:00004000       ?SetPixel@ldwGameWindow@@QAEXHHUldwColor@@@Z 00405000 f   ldwGameWindow.obj
 0001:00004030       ?Draw@ldwGameWindow@@QAEXPAVldwImage@@@Z 00405030 f   ldwGameWindow.obj
 0001:00004050       ?Draw@ldwGameWindow@@QAEXPAVldwImage@@HH@Z 00405050 f   ldwGameWindow.obj
 0001:00004080       ?Draw@ldwGameWindow@@QAEXPAVldwImage@@HHM@Z 00405080 f   ldwGameWindow.obj
 0001:000040b0       ?Draw@ldwGameWindow@@QAEXPAVldwImage@@HHAAUldwRect@@@Z 004050b0 f   ldwGameWindow.obj
 0001:00004100       ?Draw@ldwGameWindow@@QAEXPAVldwImage@@HHAAUldwRect@@M@Z 00405100 f   ldwGameWindow.obj
 0001:00004150       ?Draw@ldwGameWindow@@QAEXPAVldwImageStrip@@HHH@Z 00405150 f   ldwGameWindow.obj
 0001:00004180       ?Draw@ldwGameWindow@@QAEXPAVldwImageGrid@@HHHH@Z 00405180 f   ldwGameWindow.obj
 0001:000041b0       ?Draw@ldwGameWindow@@QAEXPAVldwImageGrid@@HHH@Z 004051b0 f   ldwGameWindow.obj
 0001:000041e0       ?Draw@ldwGameWindow@@QAEXPAVldwImageGrid@@HHHM@Z 004051e0 f   ldwGameWindow.obj
 0001:00004210       ?DrawAdditive@ldwGameWindow@@QAEXPAVldwImage@@HH@Z 00405210 f   ldwGameWindow.obj
 0001:00004240       ?DrawAdditive@ldwGameWindow@@QAEXPAVldwImage@@HHM@Z 00405240 f   ldwGameWindow.obj
 0001:00004270       ?DrawAdditive@ldwGameWindow@@QAEXPAVldwImageGrid@@HHHH@Z 00405270 f   ldwGameWindow.obj
 0001:000042a0       ?DrawAdditive@ldwGameWindow@@QAEXPAVldwImageGrid@@HHH@Z 004052a0 f   ldwGameWindow.obj
 0001:000042d0       ?DrawAdditive@ldwGameWindow@@QAEXPAVldwImageGrid@@HHHM@Z 004052d0 f   ldwGameWindow.obj
 0001:00004300       ?DrawScaled@ldwGameWindow@@QAEXPAVldwImage@@HHH_N@Z 00405300 f   ldwGameWindow.obj
 0001:00004330       ?DrawScaled@ldwGameWindow@@QAEXPAVldwImage@@HHAAUldwRect@@H_N@Z 00405330 f   ldwGameWindow.obj
 0001:00004360       ?DrawScaled@ldwGameWindow@@QAEXPAVldwImage@@HHAAUldwRect@@MH_N@Z 00405360 f   ldwGameWindow.obj
 0001:000043a0       ?DrawScaled@ldwGameWindow@@QAEXPAVldwImage@@HHMH_N@Z 004053a0 f   ldwGameWindow.obj
 0001:000043d0       ?DrawScaled@ldwGameWindow@@QAEXPAVldwImageGrid@@HHHHH_N@Z 004053d0 f   ldwGameWindow.obj
 0001:00004410       ?DrawScaled@ldwGameWindow@@QAEXPAVldwImageGrid@@HHHH_N@Z 00405410 f   ldwGameWindow.obj
 0001:00004440       ?DrawScaled@ldwGameWindow@@QAEXPAVldwImageGrid@@HHHMH_N@Z 00405440 f   ldwGameWindow.obj
 0001:00004480       ?DrawRaw@ldwGameWindow@@QAEXHHHHW4ELdwGraphicsFormat@@PAXH@Z 00405480 f   ldwGameWindow.obj
 0001:000044c0       ?DrawTinted@ldwGameWindow@@QAEXPAVldwImageStrip@@HHHUldwColor@@@Z 004054c0 f   ldwGameWindow.obj
 0001:00004520       ?DrawTinted@ldwGameWindow@@QAEXPAVldwImageGrid@@HHHUldwColor@@@Z 00405520 f   ldwGameWindow.obj
 0001:00004580       ?FillRect@ldwGameWindow@@QAEXAAUldwRect@@UldwColor@@@Z 00405580 f   ldwGameWindow.obj
 0001:000045d0       ?FillRect@ldwGameWindow@@QAEXAAUldwRect@@MMMM@Z 004055d0 f   ldwGameWindow.obj
 0001:00004600       ?FrameRect@ldwGameWindow@@QAEXAAUldwRect@@UldwColor@@@Z 00405600 f   ldwGameWindow.obj
 0001:00004710       ?FrameRect@ldwGameWindow@@QAEXAAUldwRect@@MMMM@Z 00405710 f   ldwGameWindow.obj
 0001:000047f0       ?DrawLine@ldwGameWindow@@QAEXHHHHUldwColor@@@Z 004057f0 f   ldwGameWindow.obj
 0001:00004850       ?DrawLine@ldwGameWindow@@QAEXHHHHMMMM@Z 00405850 f   ldwGameWindow.obj
 0001:00004890       ?DrawLine@ldwGameWindow@@QAEXHHHHUldwColor@@MM@Z 00405890 f   ldwGameWindow.obj
 0001:000048d0       ?DrawString@ldwGameWindow@@QAEXPBDHHUldwColor@@PAVldwFont@@@Z 004058d0 f   ldwGameWindow.obj
 0001:00004900       ?DrawString@ldwGameWindow@@QAEXPBGHHUldwColor@@PAVldwFont@@@Z 00405900 f   ldwGameWindow.obj
 0001:00004930       ?DrawStringRight@ldwGameWindow@@QAEXPBDHHUldwColor@@PAVldwFont@@@Z 00405930 f   ldwGameWindow.obj
 0001:00004960       ?DrawStringRight@ldwGameWindow@@QAEXPBGHHUldwColor@@PAVldwFont@@@Z 00405960 f   ldwGameWindow.obj
 0001:00004990       ?DrawStringCentered@ldwGameWindow@@QAEXPBDHHUldwColor@@PAVldwFont@@@Z 00405990 f   ldwGameWindow.obj
 0001:000049c0       ?DrawStringCentered@ldwGameWindow@@QAEXPBGHHUldwColor@@PAVldwFont@@@Z 004059c0 f   ldwGameWindow.obj
 0001:000049f0       ?DrawStringCentered@ldwGameWindow@@QAEXPBDHHHUldwColor@@PAVldwFont@@@Z 004059f0 f   ldwGameWindow.obj
 0001:00004a20       ?DrawStringCentered@ldwGameWindow@@QAEXPBGHHHUldwColor@@PAVldwFont@@@Z 00405a20 f   ldwGameWindow.obj
 0001:00004a50       ?DrawChars@ldwGameWindow@@QAEHPBDHHHUldwColor@@PAVldwFont@@_N@Z 00405a50 f   ldwGameWindow.obj
 0001:00004a90       ?DrawStringJustified@ldwGameWindow@@QAEHPBDHHHUldwColor@@PAVldwFont@@_N@Z 00405a90 f   ldwGameWindow.obj
 0001:00005100       ?Update@ldwGameWindow@@QAEXXZ 00406100 f   ldwGameWindow.obj
 0001:00005120       ?GetWidth@ldwGameWindow@@QAEHXZ 00406120 f   ldwGameWindow.obj
 0001:00005140       ?GetHeight@ldwGameWindow@@QAEHXZ 00406140 f   ldwGameWindow.obj
 0001:00005160       ?IsWindowed@ldwGameWindow@@QAE_NXZ 00406160 f   ldwGameWindow.obj
 0001:00005180       ?IsFullScreen@ldwGameWindow@@QAE_NXZ 00406180 f   ldwGameWindow.obj
 0001:000051a0       ?CanMakeWindowed@ldwGameWindow@@QAE_NXZ 004061a0 f   ldwGameWindow.obj
 0001:000051c0       ?MakeWindowed@ldwGameWindow@@QAEXXZ 004061c0 f   ldwGameWindow.obj
 0001:000051e0       ?MakeFullScreen@ldwGameWindow@@QAEXXZ 004061e0 f   ldwGameWindow.obj
 0001:00005200       ?HasClosed@ldwGameWindow@@QAE_NXZ 00406200 f   ldwGameWindow.obj
 0001:00005220       ?IsActive@ldwGameWindow@@QAE_NXZ 00406220 f   ldwGameWindow.obj
 0001:00005240       ?SetCursor@ldwGameWindow@@QAEXPAVldwImage@@HH@Z 00406240 f   ldwGameWindow.obj
 0001:00005270       ?ShowCursor@ldwGameWindow@@QAEX_N@Z 00406270 f   ldwGameWindow.obj
 0001:00005290       ?GetCursorPos@ldwGameWindow@@QAE?AUldwPoint@@XZ 00406290 f   ldwGameWindow.obj
 0001:000052b0       ?GetSnapShot@ldwGameWindow@@QAEPAVldwImage@@XZ 004062b0 f   ldwGameWindow.obj
 0001:000052d0       ?SaveScreenShot@ldwGameWindow@@QAE_NPBD@Z 004062d0 f   ldwGameWindow.obj
 0001:000052f0       ?SaveScreenRect@ldwGameWindow@@QAE_NPBDAAUldwRect@@@Z 004062f0 f   ldwGameWindow.obj
 0001:00005390       ?ResetView@ldwGameWindow@@QAEXXZ 00406390 f   ldwGameWindow.obj
 0001:000053b0       ?SetFont@ldwGameWindow@@QAEXPAVldwFont@@@Z 004063b0 f   ldwGameWindow.obj
 0001:000053d0       ?GetFont@ldwGameWindow@@QAEPAVldwFont@@XZ 004063d0 f   ldwGameWindow.obj
 0001:000053f0       ?SetClipping@ldwGameWindow@@QAEXUldwRect@@@Z 004063f0 f   ldwGameWindow.obj
 0001:00005430       ?ResetClipping@ldwGameWindow@@QAEXXZ 00406430 f   ldwGameWindow.obj
 0001:00005450       ?UseSleep@ldwGameWindow@@QAEXH@Z 00406450 f   ldwGameWindow.obj
 0001:00005470       ?IsLagging@ldwGameWindow@@QAE_NXZ 00406470 f   ldwGameWindow.obj
 0001:00005490       ??_GldwGameWindow@@AAEPAXI@Z 00406490 f i ldwGameWindow.obj
 0001:000054c0       ??0ldwGameWindowImpl@@QAE@HHHPBD_N@Z 004064c0 f i ldwGameWindow.obj
 0001:00005690       ??0ldwGapiApp@@QAE@ABU_GDAPPCONFIG@@@Z 00406690 f i ldwGameWindow.obj
 0001:000056f0       ?OnMinimize@ldwGapiApp@@MAEJXZ 004066f0 f i ldwGameWindow.obj
 0001:00005710       ?OnRestore@ldwGapiApp@@MAEJXZ 00406710 f i ldwGameWindow.obj
 0001:00005730       ?KeyDown@ldwGapiApp@@MAEJKAAU_GDKEYLIST@@@Z 00406730 f i ldwGameWindow.obj
 0001:00005750       ?KeyUp@ldwGapiApp@@MAEJKAAU_GDKEYLIST@@@Z 00406750 f i ldwGameWindow.obj
 0001:00005770       ?StylusDown@ldwGapiApp@@MAEJUtagPOINT@@@Z 00406770 f i ldwGameWindow.obj
 0001:000057a0       ?StylusUp@ldwGapiApp@@MAEJUtagPOINT@@@Z 004067a0 f i ldwGameWindow.obj
 0001:000057d0       ?KeyDown@CGapiApplication@@MAEJKAAU_GDKEYLIST@@@Z 004067d0 f i ldwGapiApplication.obj
 0001:000057d0       ?StylusUp@CGapiApplication@@MAEJUtagPOINT@@@Z 004067d0 f i ldwGapiApplication.obj
 0001:000057d0       ?KeyUp@CGapiApplication@@MAEJKAAU_GDKEYLIST@@@Z 004067d0 f i ldwGapiApplication.obj
 0001:000057d0       ?StylusMove@CGapiApplication@@MAEJUtagPOINT@@@Z 004067d0 f i ldwGapiApplication.obj
 0001:000057d0       ?StylusDblClk@ldwGapiApp@@MAEJUtagPOINT@@@Z 004067d0 f i ldwGameWindow.obj
 0001:000057d0       ?StylusDown@CGapiApplication@@MAEJUtagPOINT@@@Z 004067d0 f i ldwGapiApplication.obj
 0001:000057d0       ?StylusDblClk@CGapiApplication@@MAEJUtagPOINT@@@Z 004067d0 f i ldwGapiApplication.obj
 0001:000057e0       ?StylusMove@ldwGapiApp@@MAEJUtagPOINT@@@Z 004067e0 f i ldwGameWindow.obj
 0001:00005810       ?KeyChar@ldwGapiApp@@MAEXH@Z 00406810 f i ldwGameWindow.obj
 0001:00005840       ?HandleKey@ldwGapiApp@@IAEXHH@Z 00406840 f i ldwGameWindow.obj
 0001:00005ad0       ?HandleMouse@ldwGapiApp@@IAEXHUtagPOINT@@@Z 00406ad0 f i ldwGameWindow.obj
 0001:00005b20       ??_GldwGapiApp@@UAEPAXI@Z  00406b20 f i ldwGameWindow.obj
 0001:00005b20       ??_EldwGapiApp@@UAEPAXI@Z  00406b20 f i ldwGameWindow.obj
 0001:00005b50       ??1ldwGapiApp@@UAE@XZ      00406b50 f i ldwGameWindow.obj
 0001:00005b70       ?Close@ldwGameWindowImpl@@QAEXXZ 00406b70 f i ldwGameWindow.obj
 0001:00005b90       ?Close@CGapiApplication@@QAEXXZ 00406b90 f i ldwGameWindow.obj
 0001:00005bb0       ?HasClosed@ldwGameWindowImpl@@QAE_NXZ 00406bb0 f i ldwGameWindow.obj
 0001:00005bd0       ?isQuit@CGapiApplication@@QAE_NXZ 00406bd0 f i ldwGameWindow.obj
 0001:00005bf0       ??_GldwGameWindowImpl@@QAEPAXI@Z 00406bf0 f i ldwGameWindow.obj
 0001:00005c20       ??1ldwGameWindowImpl@@QAE@XZ 00406c20 f i ldwGameWindow.obj
 0001:00005c60       ?GetPixel@ldwGameWindowImpl@@QAE?AUldwColor@@HH@Z 00406c60 f i ldwGameWindow.obj
 0001:00005cc0       ?SetPixel@ldwGameWindowImpl@@QAEXHHUldwColor@@@Z 00406cc0 f i ldwGameWindow.obj
 0001:00005d00       ?Draw@ldwGameWindowImpl@@QAEXPAVldwImage@@@Z 00406d00 f i ldwGameWindow.obj
 0001:00005d20       ?Draw@ldwGameWindowImpl@@QAEXPAVldwImage@@HH@Z 00406d20 f i ldwGameWindow.obj
 0001:00005de0       ?BlitRect@ldwGameWindowImpl@@AAEXPAVCGapiSurface@@HHHHHH@Z 00406de0 f i ldwGameWindow.obj
 0001:00005e30       ?BlitRectTransparent@ldwGameWindowImpl@@AAEXPAVCGapiRGBASurface@@HHHHHH@Z 00406e30 f i ldwGameWindow.obj
 0001:00005e80       ?ClipRect@ldwGameWindowImpl@@AAE_NAAUldwRect@@AAH1@Z 00406e80 f i ldwGameWindow.obj
 0001:00005fa0       ?Draw@ldwGameWindowImpl@@QAEXPAVldwImage@@HHM@Z 00406fa0 f i ldwGameWindow.obj
 0001:00006020       ?BlitRectWithAlpha@ldwGameWindowImpl@@AAEXPAVldwImageImpl@@HHHHHHMM_N@Z 00407020 f i ldwGameWindow.obj
 0001:00006390       ?Draw@ldwGameWindowImpl@@QAEXPAVldwImage@@HHUldwRect@@@Z 00407390 f i ldwGameWindow.obj
 0001:00006430       ?Draw@ldwGameWindowImpl@@QAEXPAVldwImage@@HHUldwRect@@M@Z 00407430 f i ldwGameWindow.obj
 0001:00006470       ?Draw@ldwGameWindowImpl@@QAEXPAVldwImageStrip@@HHH@Z 00407470 f i ldwGameWindow.obj
 0001:000064d0       ?Draw@ldwGameWindowImpl@@QAEXPAVldwImageGrid@@HHHH@Z 004074d0 f i ldwGameWindow.obj
 0001:00006530       ?Draw@ldwGameWindowImpl@@QAEXPAVldwImageGrid@@HHH@Z 00407530 f i ldwGameWindow.obj
 0001:000065b0       ?Draw@ldwGameWindowImpl@@QAEXPAVldwImageGrid@@HHHM@Z 004075b0 f i ldwGameWindow.obj
 0001:00006650       ?DrawAdditive@ldwGameWindowImpl@@QAEXPAVldwImage@@HH@Z 00407650 f i ldwGameWindow.obj
 0001:00006680       ?DrawAdditive@ldwGameWindowImpl@@QAEXPAVldwImage@@HHM@Z 00407680 f i ldwGameWindow.obj
 0001:000066b0       ?DrawAdditive@ldwGameWindowImpl@@QAEXPAVldwImageGrid@@HHHH@Z 004076b0 f i ldwGameWindow.obj
 0001:000066e0       ?DrawAdditive@ldwGameWindowImpl@@QAEXPAVldwImageGrid@@HHH@Z 004076e0 f i ldwGameWindow.obj
 0001:00006710       ?DrawAdditive@ldwGameWindowImpl@@QAEXPAVldwImageGrid@@HHHM@Z 00407710 f i ldwGameWindow.obj
 0001:00006740       ?DrawScaled@ldwGameWindowImpl@@QAEXPAVldwImage@@HHH_N@Z 00407740 f i ldwGameWindow.obj
 0001:000067b0       ?DrawScaled@ldwGameWindowImpl@@QAEXPAVldwImage@@HHAAUldwRect@@H_N@Z 004077b0 f i ldwGameWindow.obj
 0001:00006810       ?DrawScaled@ldwGameWindowImpl@@QAEXPAVldwImage@@HHAAUldwRect@@MH_N@Z 00407810 f i ldwGameWindow.obj
 0001:00006870       ?DrawScaled@ldwGameWindowImpl@@QAEXPAVldwImage@@HHMH_N@Z 00407870 f i ldwGameWindow.obj
 0001:000068e0       ?DrawScaled@ldwGameWindowImpl@@QAEXPAVldwImageGrid@@HHHHH_N@Z 004078e0 f i ldwGameWindow.obj
 0001:00006950       ?DrawScaled@ldwGameWindowImpl@@QAEXPAVldwImageGrid@@HHHH_N@Z 00407950 f i ldwGameWindow.obj
 0001:000069e0       ?DrawScaled@ldwGameWindowImpl@@QAEXPAVldwImageGrid@@HHHMH_N@Z 004079e0 f i ldwGameWindow.obj
 0001:00006a70       ?DrawRaw@ldwGameWindowImpl@@QAEXHHHHW4ELdwGraphicsFormat@@PAXH@Z 00407a70 f i ldwGameWindow.obj
 0001:00006b80       ?PtInRect@ldwRect@@QAE_NHH@Z 00407b80 f i ldwGameWindow.obj
 0001:00006b80       ?PtInRect@ldwRect@@QAE_NUldwPoint@@@Z 00407b80 f i ldwButton.obj
 0001:00006bd0       ?DrawTinted@ldwGameWindowImpl@@QAEXPAVldwImage@@HHUldwRect@@UldwColor@@@Z 00407bd0 f i ldwGameWindow.obj
 0001:00006f80       ?Offset@ldwRect@@QAEXHH@Z  00407f80 f i ldwGameWindow.obj
 0001:00006fd0       ?RedF@ldwColor@@QAEMXZ     00407fd0 f i ldwGameWindow.obj
 0001:00006ff0       ?BlueF@ldwColor@@QAEMXZ    00407ff0 f i ldwGameWindow.obj
 0001:00007010       ?GreenF@ldwColor@@QAEMXZ   00408010 f i ldwGameWindow.obj
 0001:00007030       ?AlphaF@ldwColor@@QAEMXZ   00408030 f i ldwGameWindow.obj
 0001:00007050       ?FillRect@ldwGameWindowImpl@@QAEXAAUldwRect@@MMMM@Z 00408050 f i ldwGameWindow.obj
 0001:000070f0       ?DrawLine@ldwGameWindowImpl@@QAEXHHHHMMMM@Z 004080f0 f i ldwGameWindow.obj
 0001:000071b0       ?DrawLine@ldwGameWindowImpl@@QAEXHHHHUldwColor@@MM@Z 004081b0 f i ldwGameWindow.obj
 0001:00007890       ?DrawString@ldwGameWindowImpl@@QAEXPBDHHUldwColor@@PAVldwFont@@@Z 00408890 f i ldwGameWindow.obj
 0001:00007a10       ?DrawString@ldwGameWindowImpl@@QAEXPBGHHUldwColor@@PAVldwFont@@@Z 00408a10 f i ldwGameWindow.obj
 0001:00007b90       ?DrawStringRight@ldwGameWindowImpl@@QAEXPBDHHUldwColor@@PAVldwFont@@@Z 00408b90 f i ldwGameWindow.obj
 0001:00007c00       ?DrawStringRight@ldwGameWindowImpl@@QAEXPBGHHUldwColor@@PAVldwFont@@@Z 00408c00 f i ldwGameWindow.obj
 0001:00007c70       ?DrawStringCentered@ldwGameWindowImpl@@QAEXPBDHHUldwColor@@PAVldwFont@@@Z 00408c70 f i ldwGameWindow.obj
 0001:00007ce0       ?DrawStringCentered@ldwGameWindowImpl@@QAEXPBGHHUldwColor@@PAVldwFont@@@Z 00408ce0 f i ldwGameWindow.obj
 0001:00007d50       ?DrawStringCentered@ldwGameWindowImpl@@QAEXPBDHHHUldwColor@@PAVldwFont@@@Z 00408d50 f i ldwGameWindow.obj
 0001:00007dd0       ?DrawStringCentered@ldwGameWindowImpl@@QAEXPBGHHHUldwColor@@PAVldwFont@@@Z 00408dd0 f i ldwGameWindow.obj
 0001:00007e50       ?DrawChars@ldwGameWindowImpl@@QAEHPBDHHH_NUldwColor@@PAVldwFont@@@Z 00408e50 f i ldwGameWindow.obj
 0001:00008000       ?Update@ldwGameWindowImpl@@QAEXXZ 00409000 f i ldwGameWindow.obj
 0001:00008110       ?GetCursorPos@ldwGapiApp@@QAE?AUldwPoint@@XZ 00409110 f i ldwGameWindow.obj
 0001:00008130       ?IsWindowed@ldwGameWindowImpl@@QAE_NXZ 00409130 f i ldwGameWindow.obj
 0001:00008150       ?IsFullScreen@ldwGameWindowImpl@@QAE_NXZ 00409150 f i ldwGameWindow.obj
 0001:00008170       ?MakeWindowed@ldwGameWindowImpl@@QAEXXZ 00409170 f i ldwGameWindow.obj
 0001:000081a0       ?MakeFullScreen@ldwGameWindowImpl@@QAEXXZ 004091a0 f i ldwGameWindow.obj
 0001:000081d0       ?IsActive@ldwGameWindowImpl@@QAE_NXZ 004091d0 f i ldwGameWindow.obj
 0001:000081f0       ?SetCursor@ldwGameWindowImpl@@QAEXPAVldwImage@@HH@Z 004091f0 f i ldwGameWindow.obj
 0001:00008240       ?ShowCursor@ldwGameWindowImpl@@QAEX_N@Z 00409240 f i ldwGameWindow.obj
 0001:00008280       ?GetCursorPos@ldwGameWindowImpl@@QAE?AUldwPoint@@XZ 00409280 f i ldwGameWindow.obj
 0001:000082a0       ?GetSnapShot@ldwGameWindowImpl@@QAEPAVldwImage@@XZ 004092a0 f i ldwGameWindow.obj
 0001:00008320       ?SaveScreenShot@ldwGameWindowImpl@@QAE_NPBD@Z 00409320 f i ldwGameWindow.obj
 0001:00008380       ?SaveScreenRect@ldwGameWindowImpl@@QAE_NPBDAAUldwRect@@@Z 00409380 f i ldwGameWindow.obj
 0001:00008520       ?SetFont@ldwGameWindowImpl@@QAEXPAVldwFont@@@Z 00409520 f i ldwGameWindow.obj
 0001:00008520       ?SetBabies@CVillagerState@@QAEXH@Z 00409520 f i Villager.obj
 0001:00008540       ?SetClipping@ldwGameWindowImpl@@QAEXUldwRect@@@Z 00409540 f i ldwGameWindow.obj
 0001:00008570       ?ResetClipping@ldwGameWindowImpl@@QAEXXZ 00409570 f i ldwGameWindow.obj
 0001:000085b0       ?UseSleep@ldwGameWindowImpl@@QAEXH@Z 004095b0 f i ldwGameWindow.obj
 0001:000085b0       ?SetLink@ldwRadioButtonImpl@@QAEXPAVldwRadioButton@@@Z 004095b0 f i ldwRadioButton.obj
 0001:000085b0       ?SetAgesChecked@CVillagerState@@QAEXH@Z 004095b0 f i IslandEvents.obj
 0001:000085d0       ?IsLagging@ldwGameWindowImpl@@QAE_NXZ 004095d0 f i ldwGameWindow.obj
 0001:000085f0       ??0CGapiApplication@@QAE@ABU_GDAPPCONFIG@@@Z 004095f0 f   ldwGapiApplication.obj
 0001:000089b0       ??1CGapiApplication@@UAE@XZ 004099b0 f   ldwGapiApplication.obj
 0001:00008ab0       ?Update@CGapiApplication@@QAEPAVCGapiSurface@@_N@Z 00409ab0 f   ldwGapiApplication.obj
 0001:00008b60       ?IsFullscreen@CGapiApplication@@QAEHXZ 00409b60 f   ldwGapiApplication.obj
 0001:00008b80       ?Minimize@CGapiApplication@@UAEJXZ 00409b80 f   ldwGapiApplication.obj
 0001:00008ba0       ?Pause@CGapiApplication@@UAEJK@Z 00409ba0 f   ldwGapiApplication.obj
 0001:00008bd0       ?ChangeFPS@CGapiApplication@@UAEJK@Z 00409bd0 f   ldwGapiApplication.obj
 0001:00008c50       ?Shutdown@CGapiApplication@@UAEJXZ 00409c50 f   ldwGapiApplication.obj
 0001:00008c70       ?SetError@CGapiApplication@@UAEJPBDJ@Z 00409c70 f   ldwGapiApplication.obj
 0001:00008d30       ?CreateMainWindow@CGapiApplication@@IAEJXZ 00409d30 f   ldwGapiApplication.obj
 0001:00008f60       ?DestroyMainWindow@CGapiApplication@@IAEJXZ 00409f60 f   ldwGapiApplication.obj
 0001:00008fc0       ?OpenDisplay@CGapiApplication@@IAEJXZ 00409fc0 f   ldwGapiApplication.obj
 0001:000090e0       ?CloseDisplay@CGapiApplication@@IAEJXZ 0040a0e0 f   ldwGapiApplication.obj
 0001:00009100       ?SetDisplayMode@CGapiApplication@@UAEJK@Z 0040a100 f   ldwGapiApplication.obj
 0001:00009130       ?GetGlobal@CGapiApplication@@QAEPAVCGapiDraw@@XZ 0040a130 f   ldwGapiApplication.obj
 0001:00009140       ?GetDisplay@CGapiApplication@@QAEPAVCGapiDisplay@@XZ 0040a140 f   ldwGapiApplication.obj
 0001:00009160       ?GetBackBuffer@CGapiApplication@@QAEPAVCGapiSurface@@XZ 0040a160 f   ldwGapiApplication.obj
 0001:00009180       ?GetInput@CGapiApplication@@QAEPAVCGapiInput@@XZ 0040a180 f   ldwGapiApplication.obj
 0001:000091a0       ?GetTimer@CGapiApplication@@QAEPAVCGapiTimer@@XZ 0040a1a0 f   ldwGapiApplication.obj
 0001:000091c0       ?WindowProc@CGapiApplication@@MAEJPAUHWND__@@IIJ@Z 0040a1c0 f   ldwGapiApplication.obj
 0001:00009700       ?MsgRouter@CGapiApplication@@KGJPAUHWND__@@IIJ@Z 0040a700 f   ldwGapiApplication.obj
 0001:00009770       ?MainLoopPart1@CGapiApplication@@IAEJXZ 0040a770 f   ldwGapiApplication.obj
 0001:00009890       ?MainLoopPart2@CGapiApplication@@IAEJXZ 0040a890 f   ldwGapiApplication.obj
 0001:000099e0       ?ToggleFullScreen@CGapiApplication@@QAEJ_N@Z 0040a9e0 f   ldwGapiApplication.obj
 0001:00009c10       ?GetCursorPos@CGapiApplication@@QAE?AUldwPoint@@XZ 0040ac10 f   ldwGapiApplication.obj
 0001:00009c50       ?IsLagging@CGapiApplication@@QAE_NXZ 0040ac50 f   ldwGapiApplication.obj
 0001:00009c70       ??_ECGapiApplication@@UAEPAXI@Z 0040ac70 f i ldwGapiApplication.obj
 0001:00009c70       ??_GCGapiApplication@@UAEPAXI@Z 0040ac70 f i ldwGapiApplication.obj
 0001:00009ca0       ??0controlNode@ldwSceneImpl@@QAE@PAVldwControl@@PAV01@@Z 0040aca0 f i ldwScene.obj
 0001:00009ca0       ??0ldwPoint@@QAE@HH@Z      0040aca0 f i ldwGapiApplication.obj
 0001:00009ca0       ??0SRefuseData@@QAE@W4StringId@@H@Z 0040aca0 f i HotSpot.obj
 0001:00009cd0       ?SetBackground@ldwHintControl@@SAXPAVldwBackground@@@Z 0040acd0 f   ldwHintControl.obj
 0001:00009ce0       ?SetBackgroundColors@ldwHintControl@@SAXUldwColor@@0@Z 0040ace0 f   ldwHintControl.obj
 0001:00009d00       ?SetTextProperties@ldwHintControl@@SAXUldwColor@@PAVldwFont@@@Z 0040ad00 f   ldwHintControl.obj
 0001:00009d20       ?SetWait@ldwHintControl@@SAXK@Z 0040ad20 f   ldwHintControl.obj
 0001:00009d30       ?SetOffsets@ldwHintControl@@SAXHH@Z 0040ad30 f   ldwHintControl.obj
 0001:00009d50       ?EnableHints@ldwHintControl@@SAX_N@Z 0040ad50 f   ldwHintControl.obj
 0001:00009d60       ??0ldwHintControl@@QAE@H@Z 0040ad60 f   ldwHintControl.obj
 0001:00009e20       ??0ldwHintControl@@QAE@HAAUldwRect@@PAVldwScene@@PBDUldwColor@@PAVldwFont@@PAVldwBackground@@@Z 0040ae20 f   ldwHintControl.obj
 0001:00009f00       ??0ldwHintControl@@QAE@HAAUldwRect@@PAVldwScene@@PAGUldwColor@@PAVldwFont@@PAVldwBackground@@@Z 0040af00 f   ldwHintControl.obj
 0001:00009fe0       ??1ldwHintControl@@UAE@XZ  0040afe0 f   ldwHintControl.obj
 0001:0000a060       ?SetPos@ldwHintControl@@UAEXHH@Z 0040b060 f   ldwHintControl.obj
 0001:0000a080       ?GetWidth@ldwHintControl@@UAEHXZ 0040b080 f   ldwHintControl.obj
 0001:0000a0a0       ?GetHeight@ldwHintControl@@UAEHXZ 0040b0a0 f   ldwHintControl.obj
 0001:0000a0c0       ?SetActive@ldwHintControl@@UAEX_N@Z 0040b0c0 f   ldwHintControl.obj
 0001:0000a0e0       ?DrawHint@ldwHintControl@@UAEXXZ 0040b0e0 f   ldwHintControl.obj
 0001:0000a100       ?GetBounds@ldwHintControl@@MAEXAAUldwRect@@@Z 0040b100 f   ldwHintControl.obj
 0001:0000a180       ?SetHint@ldwHintControl@@QAEXPBDUldwColor@@PAVldwFont@@PAVldwBackground@@@Z 0040b180 f   ldwHintControl.obj
 0001:0000a1b0       ?SetHint@ldwHintControl@@QAEXPBGUldwColor@@PAVldwFont@@PAVldwBackground@@@Z 0040b1b0 f   ldwHintControl.obj
 0001:0000a1f0       ?SetHintWait@ldwHintControl@@QAEXK@Z 0040b1f0 f   ldwHintControl.obj
 0001:0000a210       ?EnableHint@ldwHintControl@@QAEX_N@Z 0040b210 f   ldwHintControl.obj
 0001:0000a230       ?OnHintArea@ldwHintControl@@QAEXUldwPoint@@@Z 0040b230 f   ldwHintControl.obj
 0001:0000a250       ?OffHintArea@ldwHintControl@@QAEXXZ 0040b250 f   ldwHintControl.obj
 0001:0000a270       ??0ldwHintControlImpl@@QAE@HUldwRect@@PAVldwScene@@@Z 0040b270 f i ldwHintControl.obj
 0001:0000a3d0       ?HandleMouse@ldwHintControlImpl@@UAE_NHUldwPoint@@@Z 0040b3d0 f i ldwHintControl.obj
 0001:0000a460       ?OnHintArea@ldwHintControlImpl@@QAEXUldwPoint@@@Z 0040b460 f i ldwHintControl.obj
 0001:0000a4d0       ?OffHintArea@ldwHintControlImpl@@QAEXXZ 0040b4d0 f i ldwHintControl.obj
 0001:0000a4f0       ??_GldwHintControlImpl@@UAEPAXI@Z 0040b4f0 f i ldwHintControl.obj
 0001:0000a4f0       ??_EldwHintControlImpl@@UAEPAXI@Z 0040b4f0 f i ldwHintControl.obj
 0001:0000a520       ??1ldwHintControlImpl@@UAE@XZ 0040b520 f i ldwHintControl.obj
 0001:0000a5c0       ??_GldwHintControl@@UAEPAXI@Z 0040b5c0 f i ldwHintControl.obj
 0001:0000a5c0       ??_EldwHintControl@@UAEPAXI@Z 0040b5c0 f i ldwHintControl.obj
 0001:0000a5f0       ?SetText@ldwHintControlImpl@@QAEXPBDPAVldwFont@@UldwColor@@PAVldwBackground@@@Z 0040b5f0 f i ldwHintControl.obj
 0001:0000a6e0       ?SetText@ldwHintControlImpl@@QAEXPBGPAVldwFont@@UldwColor@@PAVldwBackground@@@Z 0040b6e0 f i ldwHintControl.obj
 0001:0000a7e0       ?SetPos@ldwHintControlImpl@@QAEXHH@Z 0040b7e0 f i ldwHintControl.obj
 0001:0000a850       ?GetWidth@ldwHintControlImpl@@QAEHXZ 0040b850 f i ldwHintControl.obj
 0001:0000a870       ?GetHeight@ldwHintControlImpl@@QAEHXZ 0040b870 f i ldwHintControl.obj
 0001:0000a890       ?SetActive@ldwHintControlImpl@@QAEX_N@Z 0040b890 f i ldwHintControl.obj
 0001:0000a8e0       ??0ldwControl@@QAE@H@Z     0040b8e0 f i ldwHintControl.obj
 0001:0000a910       ?Draw@ldwHintControlImpl@@QAEXXZ 0040b910 f i ldwHintControl.obj
 0001:0000ab80       ?FitToWindow@ldwHintControlImpl@@QAEXPAVldwGameWindow@@AAUldwRect@@@Z 0040bb80 f i ldwHintControl.obj
 0001:0000ac20       ?Inset@ldwRect@@QAEXHH@Z   0040bc20 f i ldwHintControl.obj
 0001:0000ac70       ??1ldwControl@@UAE@XZ      0040bc70 f i ldwHintControl.obj
 0001:0000ac90       ?InternalFinalConstructRelease@CComObjectRootBase@ATL@@QAEXXZ 0040bc90 f i FlashPlayer.obj
 0001:0000ac90       ?InternalFinalConstructAddRef@CComObjectRootBase@ATL@@QAEXXZ 0040bc90 f i FlashPlayer.obj
 0001:0000ac90       ?Update@IPuzzle@@UAEXXZ    0040bc90 f i AlchemyLab.obj
 0001:0000ac90       ?FinalRelease@CComObjectRootBase@ATL@@QAEXXZ 0040bc90 f i FlashPlayer.obj
 0001:0000ac90       ?Draw@IPuzzle@@UBEXXZ      0040bc90 f i AlchemyLab.obj
 0001:0000ac90       ?FadeImageSkipped@IPage@@UAEXXZ 0040bc90 f i Pages.obj
 0001:0000ac90       ?ResetView@ldwGameWindowImpl@@QAEXXZ 0040bc90 f i ldwGameWindow.obj
 0001:0000ac90       ?ReleaseAssets@IPuzzle@@UAEXXZ 0040bc90 f i AlchemyLab.obj
 0001:0000ac90       ?DrawSceneFinal@ldwScene@@MAEXXZ 0040bc90 f i ldwDialog.obj
 0001:0000ac90       ?LoadAssets@IPuzzle@@UAEXXZ 0040bc90 f i AlchemyLab.obj
 0001:0000ac90       ?Shutdown@IFlashPlayer@@UAEXXZ 0040bc90 f i FlashPlayer.obj
 0001:0000ac90       ?Enter@IPage@@UAEXXZ       0040bc90 f i Pages.obj
 0001:0000ac90       ?ImpactGame@CIslandEvent@@UAEXXZ 0040bc90 f i IslandEvents.obj
 0001:0000ac90       ?Update@IPage@@UAEXXZ      0040bc90 f i Pages.obj
 0001:0000ac90       ?Refresh@IPuzzle@@UAEXXZ   0040bc90 f i AlchemyLab.obj
 0001:0000ac90       ?ImpactGame@CEventTheReflectionInTheWater@@UAEXXZ 0040bc90 f i IslandEvents.obj
 0001:0000ac90       ?CalcAward@CIslandEvent@@UAEXXZ 0040bc90 f i IslandEvents.obj
 0001:0000ac90       ?UpdateScene@ldwScene@@MAEXXZ 0040bc90 f i ldwDialog.obj
 0001:0000ac90       ?Exit@IPage@@UAEXXZ        0040bc90 f i Pages.obj
 0001:0000ac90       ?Draw@ldwHintControl@@UAEXXZ 0040bc90 f i ldwHintControl.obj
 0001:0000ac90       ?Complete@IPuzzle@@UAEXXZ  0040bc90 f i AlchemyLab.obj
 0001:0000ac90       ?DrawHint@ldwControl@@UAEXXZ 0040bc90 f i ldwHintControl.obj
 0001:0000aca0       ??_GldwControl@@UAEPAXI@Z  0040bca0 f i ldwHintControl.obj
 0001:0000aca0       ??_EldwControl@@UAEPAXI@Z  0040bca0 f i ldwHintControl.obj
 0001:0000acd0       ?SetWait@ldwHintControlImpl@@QAEXK@Z 0040bcd0 f i ldwHintControl.obj
 0001:0000acf0       ?Enable@ldwHintControlImpl@@QAEX_N@Z 0040bcf0 f i ldwHintControl.obj
 0001:0000ad10       ??0ldwImage@@QAE@PBD@Z     0040bd10 f   ldwImage.obj
 0001:0000ada0       ??0ldwImage@@IAE@XZ        0040bda0 f   ldwImage.obj
 0001:0000add0       ??1ldwImage@@UAE@XZ        0040bdd0 f   ldwImage.obj
 0001:0000ae20       ?GetWidth@ldwImage@@QAEHXZ 0040be20 f   ldwImage.obj
 0001:0000ae50       ?GetHeight@ldwImage@@QAEHXZ 0040be50 f   ldwImage.obj
 0001:0000ae80       ?SetTransparentColor@ldwImage@@QAEXUldwColor@@@Z 0040be80 f   ldwImage.obj
 0001:0000aeb0       ?HasTransparency@ldwImage@@QAE_NXZ 0040beb0 f   ldwImage.obj
 0001:0000aee0       ?PixelIsVisible@ldwImage@@QAE_NHH@Z 0040bee0 f   ldwImage.obj
 0001:0000af20       ??0ldwImageStrip@@QAE@PBDH@Z 0040bf20 f   ldwImage.obj
 0001:0000af90       ?GetColumnCount@ldwImageStrip@@QAEHXZ 0040bf90 f   ldwImage.obj
 0001:0000afb0       ?GetCellRect@ldwImageStrip@@QAEXHAAUldwRect@@@Z 0040bfb0 f   ldwImage.obj
 0001:0000b010       ??0ldwImageGrid@@QAE@PBDHH@Z 0040c010 f   ldwImage.obj
 0001:0000b0b0       ??0ldwImageGrid@@QAE@PBD0HHHH@Z 0040c0b0 f   ldwImage.obj
 0001:0000b360       ??1ldwImageGrid@@UAE@XZ    0040c360 f   ldwImage.obj
 0001:0000b440       ?GetColumnCount@ldwImageGrid@@QAEHXZ 0040c440 f   ldwImage.obj
 0001:0000b460       ?GetRowCount@ldwImageGrid@@QAEHXZ 0040c460 f   ldwImage.obj
 0001:0000b480       ?GetCellRect@ldwImageGrid@@QAEXHAAUldwRect@@@Z 0040c480 f   ldwImage.obj
 0001:0000b4c0       ?GetCellRect@ldwImageGrid@@QAEXHHAAUldwRect@@@Z 0040c4c0 f   ldwImage.obj
 0001:0000b5c0       ??_GldwImage@@UAEPAXI@Z    0040c5c0 f i ldwImage.obj
 0001:0000b5c0       ??_EldwImage@@UAEPAXI@Z    0040c5c0 f i ldwImage.obj
 0001:0000b5f0       ??_GldwImageStrip@@UAEPAXI@Z 0040c5f0 f i ldwImage.obj
 0001:0000b5f0       ??_EldwImageStrip@@UAEPAXI@Z 0040c5f0 f i ldwImage.obj
 0001:0000b620       ??1ldwImageStrip@@UAE@XZ   0040c620 f i ldwImage.obj
 0001:0000b640       ??_GldwImageGrid@@UAEPAXI@Z 0040c640 f i ldwImage.obj
 0001:0000b640       ??_EldwImageGrid@@UAEPAXI@Z 0040c640 f i ldwImage.obj
 0001:0000b670       ?Exists@ldwImage@@SA_NPBD@Z 0040c670 f   ldwImageImpl.obj
 0001:0000b840       ?UseImageArchive@ldwImage@@SA_NPBD0@Z 0040c840 f   ldwImageImpl.obj
 0001:0000b8d0       ??0ldwImageImpl@@QAE@PBD@Z 0040c8d0 f   ldwImageImpl.obj
 0001:0000be00       ??1ldwImageImpl@@QAE@XZ    0040ce00 f   ldwImageImpl.obj
 0001:0000be70       ?GetWidth@ldwImageImpl@@QAEHXZ 0040ce70 f   ldwImageImpl.obj
 0001:0000bec0       ?GetHeight@ldwImageImpl@@QAEHXZ 0040cec0 f   ldwImageImpl.obj
 0001:0000bf10       ?SetTransparentColor@ldwImageImpl@@QAEXUldwColor@@@Z 0040cf10 f   ldwImageImpl.obj
 0001:0000bf30       ?HasTransparency@ldwImageImpl@@QAE_NXZ 0040cf30 f   ldwImageImpl.obj
 0001:0000bf50       ?PixelIsVisible@ldwImageImpl@@QAE_NHH@Z 0040cf50 f   ldwImageImpl.obj
 0001:0000bff0       ?GetGraphic@ldwImageImpl@@QAEPAVCGapiSurface@@XZ 0040cff0 f   ldwImageImpl.obj
 0001:0000c000       ?GetGraphicRGBA@ldwImageImpl@@QAEPAVCGapiRGBASurface@@XZ 0040d000 f   ldwImageImpl.obj
 0001:0000c020       ?Create@ldwLog@@SAPAV1@PBD_N@Z 0040d020 f   ldwLog.obj
 0001:0000c0c0       ?Get@ldwLog@@SAPAV1@XZ     0040d0c0 f   ldwLog.obj
 0001:0000c140       ?Destroy@ldwLog@@SAXXZ     0040d140 f   ldwLog.obj
 0001:0000c180       ?SetLogFilePath@ldwLog@@QAEXPBD@Z 0040d180 f   ldwLog.obj
 0001:0000c1a0       ?NewLine@ldwLog@@QAEXXZ    0040d1a0 f   ldwLog.obj
 0001:0000c1f0       ?WriteLine@ldwLog@@QAAXPBDZZ 0040d1f0 f   ldwLog.obj
 0001:0000c270       ?Write@ldwLog@@QAAXPBDZZ   0040d270 f   ldwLog.obj
 0001:0000c2d0       ?TimeStampOn@ldwLog@@QAEX_N@Z 0040d2d0 f   ldwLog.obj
 0001:0000c2f0       ?Open@ldwLog@@QAEXXZ       0040d2f0 f   ldwLog.obj
 0001:0000c310       ?Flush@ldwLog@@QAEXXZ      0040d310 f   ldwLog.obj
 0001:0000c330       ?Close@ldwLog@@QAEXXZ      0040d330 f   ldwLog.obj
 0001:0000c350       ??0ldwLog@@AAE@PBD_N@Z     0040d350 f   ldwLog.obj
 0001:0000c3e0       ??0ldwLog@@AAE@XZ          0040d3e0 f   ldwLog.obj
 0001:0000c460       ??1ldwLog@@AAE@XZ          0040d460 f   ldwLog.obj
 0001:0000c4a0       ??_GldwLog@@AAEPAXI@Z      0040d4a0 f i ldwLog.obj
 0001:0000c4d0       ?SetLogFilePath@ldwLogImpl@@QAEXPBD@Z 0040d4d0 f i ldwLog.obj
 0001:0000c530       ?Close@ldwLogImpl@@QAEXXZ  0040d530 f i ldwLog.obj
 0001:0000c560       ?Open@ldwLogImpl@@QAEXXZ   0040d560 f i ldwLog.obj
 0001:0000c5c0       ?IsOpen@ldwLogImpl@@QAE_NXZ 0040d5c0 f i ldwLog.obj
 0001:0000c5e0       ?WriteTimeStamp@ldwLogImpl@@QAEXXZ 0040d5e0 f i ldwLog.obj
 0001:0000c670       ?Flush@ldwLogImpl@@QAEXXZ  0040d670 f i ldwLog.obj
 0001:0000c6a0       ??0ldwLogImpl@@QAE@XZ      0040d6a0 f i ldwLog.obj
 0001:0000c6d0       ??_GldwLogImpl@@QAEPAXI@Z  0040d6d0 f i ldwLog.obj
 0001:0000c700       ??1ldwLogImpl@@QAE@XZ      0040d700 f i ldwLog.obj
 0001:0000c730       ??0ldwRadioButton@@QAE@HPAVldwImageStrip@@UldwPoint@@PAVldwScene@@PBDUldwColor@@PAVldwFont@@@Z 0040d730 f   ldwRadioButton.obj
 0001:0000c7f0       ??1ldwRadioButton@@UAE@XZ  0040d7f0 f   ldwRadioButton.obj
 0001:0000c870       ?SetPos@ldwRadioButton@@UAEXHH@Z 0040d870 f   ldwRadioButton.obj
 0001:0000c890       ?SetLink@ldwRadioButton@@QAEXPAV1@@Z 0040d890 f   ldwRadioButton.obj
 0001:0000c8b0       ?GetLink@ldwRadioButton@@QAEPAV1@XZ 0040d8b0 f   ldwRadioButton.obj
 0001:0000c8d0       ?SetCheck@ldwRadioButton@@QAEX_N@Z 0040d8d0 f   ldwRadioButton.obj
 0001:0000c8f0       ?IsChecked@ldwRadioButton@@QAE_NXZ 0040d8f0 f   ldwRadioButton.obj
 0001:0000c910       ?GetWidth@ldwRadioButton@@UAEHXZ 0040d910 f   ldwRadioButton.obj
 0001:0000c930       ?GetHeight@ldwRadioButton@@UAEHXZ 0040d930 f   ldwRadioButton.obj
 0001:0000c950       ?SetActive@ldwRadioButton@@UAEX_N@Z 0040d950 f   ldwRadioButton.obj
 0001:0000c970       ?Draw@ldwRadioButton@@UAEXXZ 0040d970 f   ldwRadioButton.obj
 0001:0000c990       ?GetBounds@ldwRadioButton@@UAEXAAUldwRect@@@Z 0040d990 f   ldwRadioButton.obj
 0001:0000ca10       ?SetSoundFx@ldwRadioButton@@QAEXPAVldwSoundFx@@0@Z 0040da10 f   ldwRadioButton.obj
 0001:0000ca30       ??0ldwRadioButtonImpl@@QAE@PAVldwRadioButton@@HPAVldwImageStrip@@UldwPoint@@PAVldwScene@@PBDUldwColor@@PAVldwFont@@PAVldwHintControl@@@Z 0040da30 f i ldwRadioButton.obj
 0001:0000cb90       ?SetPos@ldwRadioButtonImpl@@QAEXHH@Z 0040db90 f i ldwRadioButton.obj
 0001:0000cc00       ?SetText@ldwRadioButtonImpl@@QAEXPBDPAVldwFont@@@Z 0040dc00 f i ldwRadioButton.obj
 0001:0000cc70       ?HandleMouse@ldwRadioButtonImpl@@UAE_NHUldwPoint@@@Z 0040dc70 f i ldwRadioButton.obj
 0001:0000ce70       ??_GldwRadioButtonImpl@@UAEPAXI@Z 0040de70 f i ldwRadioButton.obj
 0001:0000ce70       ??_EldwRadioButtonImpl@@UAEPAXI@Z 0040de70 f i ldwRadioButton.obj
 0001:0000cea0       ??1ldwRadioButtonImpl@@UAE@XZ 0040dea0 f i ldwRadioButton.obj
 0001:0000cf60       ??_GldwRadioButton@@UAEPAXI@Z 0040df60 f i ldwRadioButton.obj
 0001:0000cf60       ??_EldwRadioButton@@UAEPAXI@Z 0040df60 f i ldwRadioButton.obj
 0001:0000cf90       ?SetCheck@ldwRadioButtonImpl@@QAEX_N@Z 0040df90 f i ldwRadioButton.obj
 0001:0000cfb0       ?IsChecked@ldwRadioButtonImpl@@QAE_NXZ 0040dfb0 f i ldwRadioButton.obj
 0001:0000cfd0       ?GetWidth@ldwRadioButtonImpl@@QAEHXZ 0040dfd0 f i ldwRadioButton.obj
 0001:0000d050       ?GetHeight@ldwRadioButtonImpl@@QAEHXZ 0040e050 f i ldwRadioButton.obj
 0001:0000d080       ?SetActive@ldwRadioButtonImpl@@QAEX_N@Z 0040e080 f i ldwRadioButton.obj
 0001:0000d0e0       ?Draw@ldwRadioButtonImpl@@QAEXXZ 0040e0e0 f i ldwRadioButton.obj
 0001:0000d290       ?SetSoundFx@ldwRadioButtonImpl@@QAEXPAVldwSoundFx@@0@Z 0040e290 f i ldwRadioButton.obj
 0001:0000d2b0       ??0ldwScene@@QAE@XZ        0040e2b0 f   ldwScene.obj
 0001:0000d340       ??1ldwScene@@UAE@XZ        0040e340 f   ldwScene.obj
 0001:0000d3e0       ?SetActive@ldwScene@@QAEX_N@Z 0040e3e0 f   ldwScene.obj
 0001:0000d450       ?IsActive@ldwScene@@QAE_NXZ 0040e450 f   ldwScene.obj
 0001:0000d470       ?GetBounds@ldwScene@@QAEXAAUldwRect@@@Z 0040e470 f   ldwScene.obj
 0001:0000d4a0       ?Update@ldwScene@@UAEXXZ   0040e4a0 f   ldwScene.obj
 0001:0000d4d0       ?Draw@ldwScene@@UAEXXZ     0040e4d0 f   ldwScene.obj
 0001:0000d520       ?SetBounds@ldwScene@@IAEXUldwRect@@@Z 0040e520 f   ldwScene.obj
 0001:0000d550       ?AddControl@ldwScene@@IAEXPAVldwControl@@@Z 0040e550 f   ldwScene.obj
 0001:0000d5f0       ?GetControl@ldwScene@@IAEPAVldwControl@@H@Z 0040e5f0 f   ldwScene.obj
 0001:0000d640       ?RemoveControl@ldwScene@@IAEXPAVldwControl@@@Z 0040e640 f   ldwScene.obj
 0001:0000d6d0       ?ActivateControls@ldwScene@@IAEX_N@Z 0040e6d0 f   ldwScene.obj
 0001:0000d710       ?DrawControls@ldwScene@@IAEXXZ 0040e710 f   ldwScene.obj
 0001:0000d750       ?DrawHints@ldwScene@@IAEXXZ 0040e750 f   ldwScene.obj
 0001:0000d790       ?DeleteControls@ldwScene@@IAEXXZ 0040e790 f   ldwScene.obj
 0001:0000d810       ??0ldwSceneImpl@@QAE@XZ    0040e810 f i ldwScene.obj
 0001:0000d880       ??_GldwScene@@UAEPAXI@Z    0040e880 f i ldwScene.obj
 0001:0000d880       ??_EldwScene@@UAEPAXI@Z    0040e880 f i ldwScene.obj
 0001:0000d8b0       ??_GldwSceneImpl@@QAEPAXI@Z 0040e8b0 f i ldwScene.obj
 0001:0000d8e0       ??1ldwSceneImpl@@QAE@XZ    0040e8e0 f i ldwScene.obj
 0001:0000d930       ??0ldwSoundFx@@QAE@PBD@Z   0040e930 f   ldwSound.obj
 0001:0000d9b0       ??1ldwSoundFx@@QAE@XZ      0040e9b0 f   ldwSound.obj
 0001:0000da00       ?Play@ldwSoundFx@@QAEX_N@Z 0040ea00 f   ldwSound.obj
 0001:0000da20       ?StopAll@ldwSoundFx@@SAXXZ 0040ea20 f   ldwSound.obj
 0001:0000da30       ?SetSoundFxOff@ldwSoundFx@@SAX_N@Z 0040ea30 f   ldwSound.obj
 0001:0000da50       ?MuteVolume@ldwSoundFx@@SAX_N@Z 0040ea50 f   ldwSound.obj
 0001:0000dab0       ?SetGlobalVolume@ldwSoundFx@@SAXM@Z 0040eab0 f   ldwSound.obj
 0001:0000daf0       ?StopPlaying@ldwSoundFx@@QAEXXZ 0040eaf0 f   ldwSound.obj
 0001:0000db10       ?IsPlaying@ldwSoundFx@@QAE_NXZ 0040eb10 f   ldwSound.obj
 0001:0000db30       ?SetVolume@ldwSoundFx@@QAEXM@Z 0040eb30 f   ldwSound.obj
 0001:0000db50       ??0ldwSoundTrack@@QAE@PBD@Z 0040eb50 f   ldwSound.obj
 0001:0000dbd0       ??1ldwSoundTrack@@QAE@XZ   0040ebd0 f   ldwSound.obj
 0001:0000dc20       ?Play@ldwSoundTrack@@QAEX_N@Z 0040ec20 f   ldwSound.obj
 0001:0000dc40       ?StopAll@ldwSoundTrack@@SAXXZ 0040ec40 f   ldwSound.obj
 0001:0000dc50       ?SetSoundTracksOff@ldwSoundTrack@@SAX_N@Z 0040ec50 f   ldwSound.obj
 0001:0000dc70       ?StopPlaying@ldwSoundTrack@@QAEXXZ 0040ec70 f   ldwSound.obj
 0001:0000dc90       ?IsPlaying@ldwSoundTrack@@QAE_NXZ 0040ec90 f   ldwSound.obj
 0001:0000dcb0       ?SetVolume@ldwSoundTrack@@QAEXM@Z 0040ecb0 f   ldwSound.obj
 0001:0000dcd0       ?GetTimePlaying@ldwSoundTrack@@QAEKXZ 0040ecd0 f   ldwSound.obj
 0001:0000dcf0       ?MuteVolume@ldwSoundTrack@@SAX_N@Z 0040ecf0 f   ldwSound.obj
 0001:0000dd50       ??0ldwSoundFxImpl@@QAE@PBD@Z 0040ed50 f i ldwSound.obj
 0001:0000ddd0       ?IncrementSoundCount@ldwSoundManager@@QAEXXZ 0040edd0 f i ldwSound.obj
 0001:0000de10       ??_GldwSoundFxImpl@@QAEPAXI@Z 0040ee10 f i ldwSound.obj
 0001:0000de40       ??1ldwSoundFxImpl@@QAE@XZ  0040ee40 f i ldwSound.obj
 0001:0000de70       ?DecrementSoundCount@ldwSoundManager@@QAEXXZ 0040ee70 f i ldwSound.obj
 0001:0000dec0       ?Play@ldwSoundFxImpl@@QAEX_N@Z 0040eec0 f i ldwSound.obj
 0001:0000df30       ?StopPlaying@ldwSoundFxImpl@@QAEXXZ 0040ef30 f i ldwSound.obj
 0001:0000df70       ?IsPlaying@ldwSoundFxImpl@@QAE_NXZ 0040ef70 f i ldwSound.obj
 0001:0000dfb0       ?SetVolume@ldwSoundFxImpl@@QAEXM@Z 0040efb0 f i ldwSound.obj
 0001:0000e000       ??0ldwSoundTrackImpl@@QAE@PBD@Z 0040f000 f i ldwSound.obj
 0001:0000e1b0       ?HandleMessage@ldwSoundTrackImpl@@UAE_NHJ@Z 0040f1b0 f i ldwSound.obj
 0001:0000e220       ?SetVolume@ldwSoundTrackImpl@@QAEXM@Z 0040f220 f i ldwSound.obj
 0001:0000e260       ?lowLevelSetVolume@ldwSoundTrackImpl@@QAEXM@Z 0040f260 f i ldwSound.obj
 0001:0000e2d0       ??_GldwSoundTrackImpl@@UAEPAXI@Z 0040f2d0 f i ldwSound.obj
 0001:0000e2d0       ??_EldwSoundTrackImpl@@UAEPAXI@Z 0040f2d0 f i ldwSound.obj
 0001:0000e300       ??1ldwSoundTrackImpl@@UAE@XZ 0040f300 f i ldwSound.obj
 0001:0000e3a0       ?Play@ldwSoundTrackImpl@@QAEX_N@Z 0040f3a0 f i ldwSound.obj
 0001:0000e440       ?StopPlaying@ldwSoundTrackImpl@@QAEXXZ 0040f440 f i ldwSound.obj
 0001:0000e490       ?IsPlaying@ldwSoundTrackImpl@@QAE_NXZ 0040f490 f i ldwSound.obj
 0001:0000e510       ?GetTimePlaying@ldwSoundTrackImpl@@QAEKXZ 0040f510 f i ldwSound.obj
 0001:0000e560       ??0ldwSoundManager@@QAE@XZ 0040f560 f i ldwSound.obj
 0001:0000e580       ??0ldwTextControl@@QAE@PAVldwScene@@UldwPoint@@PBDHPAVldwFont@@@Z 0040f580 f   ldwTextControl.obj
 0001:0000e640       ??0ldwTextControl@@QAE@PAVldwScene@@HUldwPoint@@PBDPAVldwFont@@H_N@Z 0040f640 f   ldwTextControl.obj
 0001:0000e700       ??0ldwTextControl@@QAE@PAVldwScene@@UldwPoint@@PBGHPAVldwFont@@@Z 0040f700 f   ldwTextControl.obj
 0001:0000e7c0       ??0ldwTextControl@@QAE@PAVldwScene@@HUldwPoint@@PBGPAVldwFont@@H_N@Z 0040f7c0 f   ldwTextControl.obj
 0001:0000e880       ??1ldwTextControl@@UAE@XZ  0040f880 f   ldwTextControl.obj
 0001:0000e900       ?SetBoundsFromText@ldwTextControl@@QAEXHHHH@Z 0040f900 f   ldwTextControl.obj
 0001:0000e930       ?SetBounds@ldwTextControl@@QAEXAAUldwRect@@@Z 0040f930 f   ldwTextControl.obj
 0001:0000e950       ?SetPos@ldwTextControl@@UAEXHH@Z 0040f950 f   ldwTextControl.obj
 0001:0000e970       ?GetBounds@ldwTextControl@@UAEXAAUldwRect@@@Z 0040f970 f   ldwTextControl.obj
 0001:0000e9d0       ?GetWidth@ldwTextControl@@UAEHXZ 0040f9d0 f   ldwTextControl.obj
 0001:0000ea00       ?GetHeight@ldwTextControl@@UAEHXZ 0040fa00 f   ldwTextControl.obj
 0001:0000ea30       ?SetActive@ldwTextControl@@UAEX_N@Z 0040fa30 f   ldwTextControl.obj
 0001:0000ea50       ?Draw@ldwTextControl@@UAEXXZ 0040fa50 f   ldwTextControl.obj
 0001:0000ea80       ?SetJustify@ldwTextControl@@QAEXH@Z 0040fa80 f   ldwTextControl.obj
 0001:0000eaa0       ?SetColors@ldwTextControl@@QAEXUldwColor@@0@Z 0040faa0 f   ldwTextControl.obj
 0001:0000eac0       ?SetCursorColor@ldwTextControl@@QAEXUldwColor@@@Z 0040fac0 f   ldwTextControl.obj
 0001:0000eae0       ?SetFont@ldwTextControl@@QAEXPAVldwFont@@@Z 0040fae0 f   ldwTextControl.obj
 0001:0000eb00       ?SetCanEdit@ldwTextControl@@QAEX_NH@Z 0040fb00 f   ldwTextControl.obj
 0001:0000eb20       ?SetText@ldwTextControl@@QAEXPBD@Z 0040fb20 f   ldwTextControl.obj
 0001:0000eb40       ?SetText@ldwTextControl@@QAEXPBG@Z 0040fb40 f   ldwTextControl.obj
 0001:0000eb60       ?SetIsNumber@ldwTextControl@@QAEX_NH@Z 0040fb60 f   ldwTextControl.obj
 0001:0000eb80       ?SetCursorChar@ldwTextControl@@QAEXD@Z 0040fb80 f   ldwTextControl.obj
 0001:0000eba0       ?GetTextLength@ldwTextControl@@QAEHXZ 0040fba0 f   ldwTextControl.obj
 0001:0000ebc0       ?GetText@ldwTextControl@@QAEXPADH@Z 0040fbc0 f   ldwTextControl.obj
 0001:0000ebe0       ?GetText@ldwTextControl@@QAEXPAGH@Z 0040fbe0 f   ldwTextControl.obj
 0001:0000ec00       ?GetValue@ldwTextControl@@QAEHXZ 0040fc00 f   ldwTextControl.obj
 0001:0000ec20       ?StartEdit@ldwTextControl@@QAEXXZ 0040fc20 f   ldwTextControl.obj
 0001:0000ec40       ?EndEdit@ldwTextControl@@QAEXXZ 0040fc40 f   ldwTextControl.obj
 0001:0000ec60       ??0ldwTextControlImpl@@QAE@HUldwPoint@@PAVldwScene@@PBDPAVldwFont@@H_NPAVldwHintControl@@@Z 0040fc60 f i ldwTextControl.obj
 0001:0000edd0       ?SetBoundsFromText@ldwTextControlImpl@@QAEXHHHH@Z 0040fdd0 f i ldwTextControl.obj
 0001:0000ef50       ?SetText@ldwTextControlImpl@@QAEXPBD@Z 0040ff50 f i ldwTextControl.obj
 0001:0000efa0       ?HandleMouse@ldwTextControlImpl@@UAE_NHUldwPoint@@@Z 0040ffa0 f i ldwTextControl.obj
 0001:0000f0d0       ?StartEdit@ldwTextControlImpl@@QAEXXZ 004100d0 f i ldwTextControl.obj
 0001:0000f130       ?EndEdit@ldwTextControlImpl@@QAEXXZ 00410130 f i ldwTextControl.obj
 0001:0000f180       ?HandleKey@ldwTextControlImpl@@UAE_NHHH@Z 00410180 f i ldwTextControl.obj
 0001:0000f320       ?HandleMessage@ldwTextControlImpl@@UAE_NHJ@Z 00410320 f i ldwTextControl.obj
 0001:0000f360       ??_GldwTextControlImpl@@UAEPAXI@Z 00410360 f i ldwTextControl.obj
 0001:0000f360       ??_EldwTextControlImpl@@UAEPAXI@Z 00410360 f i ldwTextControl.obj
 0001:0000f390       ??1ldwTextControlImpl@@UAE@XZ 00410390 f i ldwTextControl.obj
 0001:0000f410       ??_GldwTextControl@@UAEPAXI@Z 00410410 f i ldwTextControl.obj
 0001:0000f410       ??_EldwTextControl@@UAEPAXI@Z 00410410 f i ldwTextControl.obj
 0001:0000f440       ??0ldwTextControlImpl@@QAE@HUldwPoint@@PAVldwScene@@PBGPAVldwFont@@H_NPAVldwHintControl@@@Z 00410440 f i ldwTextControl.obj
 0001:0000f5b0       ?SetText@ldwTextControlImpl@@QAEXPBG@Z 004105b0 f i ldwTextControl.obj
 0001:0000f650       ?SetBounds@ldwTextControlImpl@@QAEXAAUldwRect@@@Z 00410650 f i ldwTextControl.obj
 0001:0000f680       ?SetPos@ldwTextControlImpl@@QAEXHH@Z 00410680 f i ldwTextControl.obj
 0001:0000f6d0       ?GetBounds@ldwTextControlImpl@@QAEXAAUldwRect@@@Z 004106d0 f i ldwTextControl.obj
 0001:0000f700       ?SetActive@ldwTextControlImpl@@QAEX_N@Z 00410700 f i ldwTextControl.obj
 0001:0000f760       ?Draw@ldwTextControlImpl@@QAEXXZ 00410760 f i ldwTextControl.obj
 0001:0000fae0       ?SetJustify@ldwTextControlImpl@@QAEXH@Z 00410ae0 f i ldwTextControl.obj
 0001:0000fb00       ?SetColors@ldwTextControlImpl@@QAEXUldwColor@@0@Z 00410b00 f i ldwTextControl.obj
 0001:0000fb30       ?SetCursorColor@ldwTextControlImpl@@QAEXUldwColor@@@Z 00410b30 f i ldwTextControl.obj
 0001:0000fb50       ?SetFont@ldwTextControlImpl@@QAEXPAVldwFont@@@Z 00410b50 f i ldwTextControl.obj
 0001:0000fb70       ?SetCanEdit@ldwTextControlImpl@@QAEX_NH@Z 00410b70 f i ldwTextControl.obj
 0001:0000fc00       ?SetIsNumber@ldwTextControlImpl@@QAEX_NH@Z 00410c00 f i ldwTextControl.obj
 0001:0000fc40       ?SetCursorChar@ldwTextControlImpl@@QAEXD@Z 00410c40 f i ldwTextControl.obj
 0001:0000fc60       ?GetTextLength@ldwTextControlImpl@@QAEHXZ 00410c60 f i ldwTextControl.obj
 0001:0000fcc0       ?GetText@ldwTextControlImpl@@QAEXPADH@Z 00410cc0 f i ldwTextControl.obj
 0001:0000fd40       ?GetText@ldwTextControlImpl@@QAEXPAGH@Z 00410d40 f i ldwTextControl.obj
 0001:0000fda0       ?GetValue@ldwTextControlImpl@@QAEHXZ 00410da0 f i ldwTextControl.obj
 0001:0000fde0       ??0ldwTiledBackground@@QAE@PAVldwImageGrid@@HH@Z 00410de0 f   ldwTiledBackground.obj
 0001:0000fe60       ??1ldwTiledBackground@@UAE@XZ 00410e60 f   ldwTiledBackground.obj
 0001:0000fe80       ?SetInteriorSize@ldwTiledBackground@@UAEXHH@Z 00410e80 f   ldwTiledBackground.obj
 0001:0000fef0       ?GetWidth@ldwTiledBackground@@UAEHXZ 00410ef0 f   ldwTiledBackground.obj
 0001:0000ff10       ?GetHeight@ldwTiledBackground@@UAEHXZ 00410f10 f   ldwTiledBackground.obj
 0001:0000ff30       ?Draw@ldwTiledBackground@@UAEXUldwPoint@@M@Z 00410f30 f   ldwTiledBackground.obj
 0001:00010170       ??_EldwTiledBackground@@UAEPAXI@Z 00411170 f i ldwTiledBackground.obj
 0001:00010170       ??_GldwTiledBackground@@UAEPAXI@Z 00411170 f i ldwTiledBackground.obj
 0001:000101a0       ??0ldwBackground@@QAE@XZ   004111a0 f i ldwTiledBackground.obj
 0001:000101c0       ??0ldwTiledDialog@@QAE@_N@Z 004111c0 f   ldwTiledDialog.obj
 0001:00010280       ??1ldwTiledDialog@@UAE@XZ  00411280 f   ldwTiledDialog.obj
 0001:00010300       ?SetTiling@ldwTiledDialog@@IAEXPAVldwImageGrid@@HH@Z 00411300 f   ldwTiledDialog.obj
 0001:000103e0       ?Activate@ldwTiledDialog@@MAEX_N@Z 004113e0 f   ldwTiledDialog.obj
 0001:00010410       ?UpdateScene@ldwTiledDialog@@MAEXXZ 00411410 f   ldwTiledDialog.obj
 0001:00010520       ?DrawScene@ldwTiledDialog@@MAEXXZ 00411520 f   ldwTiledDialog.obj
 0001:00010630       ?EndDialog@ldwTiledDialog@@IAEXXZ 00411630 f   ldwTiledDialog.obj
 0001:00010660       ?SetPos@ldwTiledDialog@@IAEXHH@Z 00411660 f   ldwTiledDialog.obj
 0001:00010690       ?SetBounds@ldwTiledDialog@@IAEXUldwRect@@@Z 00411690 f   ldwTiledDialog.obj
 0001:000106e0       ?SetClipping@ldwTiledDialog@@IAEXUldwRect@@@Z 004116e0 f   ldwTiledDialog.obj
 0001:00010720       ??_EldwTiledDialog@@UAEPAXI@Z 00411720 f i ldwTiledDialog.obj
 0001:00010720       ??_GldwTiledDialog@@UAEPAXI@Z 00411720 f i ldwTiledDialog.obj
 0001:00010750       ?Finished@ldwTiledDialog@@UAE_NXZ 00411750 f i ldwTiledDialog.obj
 0001:00010770       ?Copy@ldwWString@@SAXPAGPBGH@Z 00411770 f   ldwWString.obj
 0001:000107e0       ?Copy@ldwWString@@SAXPAGPBDH@Z 004117e0 f   ldwWString.obj
 0001:00010860       ?Concat@ldwWString@@SAXPAGPBGH@Z 00411860 f   ldwWString.obj
 0001:000108f0       ?Concat@ldwWString@@SAXPAGPBDH@Z 004118f0 f   ldwWString.obj
 0001:00010990       ?GetLength@ldwWString@@SAHPBG@Z 00411990 f   ldwWString.obj
 0001:000109c0       ?Compare@ldwWString@@SAHPBG0@Z 004119c0 f   ldwWString.obj
 0001:00010a10       ?FindChar@ldwWString@@SAPAGPAGD@Z 00411a10 f   ldwWString.obj
 0001:00010a50       ?inflate_flush@@YAHPAUinflate_blocks_state@@PAUz_stream_s@@H@Z 00411a50 f   unzip.obj
 0001:00010c30       ?inflate_codes_new@@YAPAUinflate_codes_state@@IIPBUinflate_huft_s@@0PAUz_stream_s@@@Z 00411c30 f   unzip.obj
 0001:00010c90       ?inflate_codes@@YAHPAUinflate_blocks_state@@PAUz_stream_s@@H@Z 00411c90 f   unzip.obj
 0001:00011990       ?inflate_codes_free@@YAXPAUinflate_codes_state@@PAUz_stream_s@@@Z 00412990 f   unzip.obj
 0001:000119b0       ?inflate_blocks_reset@@YAXPAUinflate_blocks_state@@PAUz_stream_s@@PAK@Z 004129b0 f   unzip.obj
 0001:00011a70       ?inflate_blocks_new@@YAPAUinflate_blocks_state@@PAUz_stream_s@@P6AKKPBEI@ZI@Z 00412a70 f   unzip.obj
 0001:00011b70       ?inflate_blocks@@YAHPAUinflate_blocks_state@@PAUz_stream_s@@H@Z 00412b70 f   unzip.obj
 0001:00012eb0       ?inflate_blocks_free@@YAHPAUinflate_blocks_state@@PAUz_stream_s@@@Z 00413eb0 f   unzip.obj
 0001:00012f10       ?huft_build@@YAHPAIIIPBI1PAPAUinflate_huft_s@@0PAU1@00@Z 00413f10 f   unzip.obj
 0001:00013730       ?inflate_trees_bits@@YAHPAI0PAPAUinflate_huft_s@@PAU1@PAUz_stream_s@@@Z 00414730 f   unzip.obj
 0001:000137e0       ?inflate_trees_dynamic@@YAHIIPAI00PAPAUinflate_huft_s@@1PAU1@PAUz_stream_s@@@Z 004147e0 f   unzip.obj
 0001:00013970       ?inflate_trees_fixed@@YAHPAI0PAPBUinflate_huft_s@@1PAUz_stream_s@@@Z 00414970 f   unzip.obj
 0001:000139a0       ?inflate_fast@@YAHIIPBUinflate_huft_s@@0PAUinflate_blocks_state@@PAUz_stream_s@@@Z 004149a0 f   unzip.obj
 0001:000140e0       ?get_crc_table@@YAPBKXZ    004150e0 f   unzip.obj
 0001:000140f0       ?ucrc32@@YAKKPBEI@Z        004150f0 f   unzip.obj
 0001:000142a0       ?Uupdate_keys@@YAXPAKD@Z   004152a0 f   unzip.obj
 0001:00014320       ?Udecrypt_byte@@YADPAK@Z   00415320 f   unzip.obj
 0001:00014350       ?zdecode@@YADPAKD@Z        00415350 f   unzip.obj
 0001:00014380       ?adler32@@YAKKPBEI@Z       00415380 f   unzip.obj
 0001:000145c0       ?zlibVersion@@YAPBDXZ      004155c0 f   unzip.obj
 0001:000145d0       ?zError@@YAPBDH@Z          004155d0 f   unzip.obj
 0001:000145f0       ?zcalloc@@YAPAXPAXII@Z     004155f0 f   unzip.obj
 0001:00014620       ?zcfree@@YAXPAX0@Z         00415620 f   unzip.obj
 0001:00014640       ?inflateReset@@YAHPAUz_stream_s@@@Z 00415640 f   unzip.obj
 0001:000146b0       ?inflateEnd@@YAHPAUz_stream_s@@@Z 004156b0 f   unzip.obj
 0001:00014720       ?inflateInit2@@YAHPAUz_stream_s@@@Z 00415720 f   unzip.obj
 0001:000148b0       ?inflate@@YAHPAUz_stream_s@@H@Z 004158b0 f   unzip.obj
 0001:00014f60       ?lufopen@@YAPAULUFILE@@PAXIKPAK@Z 00415f60 f   unzip.obj
 0001:000150e0       ?lufclose@@YAHPAULUFILE@@@Z 004160e0 f   unzip.obj
 0001:00015120       ?luferror@@YAHPAULUFILE@@@Z 00416120 f   unzip.obj
 0001:00015150       ?luftell@@YAJPAULUFILE@@@Z 00416150 f   unzip.obj
 0001:000151a0       ?lufseek@@YAHPAULUFILE@@JH@Z 004161a0 f   unzip.obj
 0001:00015280       ?lufread@@YAIPAXIIPAULUFILE@@@Z 00416280 f   unzip.obj
 0001:00015340       ?unzlocal_getByte@@YAHPAULUFILE@@PAH@Z 00416340 f   unzip.obj
 0001:00015390       ?unzlocal_getShort@@YAHPAULUFILE@@PAK@Z 00416390 f   unzip.obj
 0001:00015400       ?unzlocal_getLong@@YAHPAULUFILE@@PAK@Z 00416400 f   unzip.obj
 0001:000154b0       ?strcmpcasenosensitive_internal@@YAHPBD0@Z 004164b0 f   unzip.obj
 0001:00015560       ?unzStringFileNameCompare@@YAHPBD0H@Z 00416560 f   unzip.obj
 0001:00015590       ?unzlocal_SearchCentralDir@@YAKPAULUFILE@@@Z 00416590 f   unzip.obj
 0001:00015720       ?unzOpenInternal@@YAPAUunz_s@@PAULUFILE@@@Z 00416720 f   unzip.obj
 0001:00015980       ?unzClose@@YAHPAUunz_s@@@Z 00416980 f   unzip.obj
 0001:000159e0       ?unzGetGlobalInfo@@YAHPAUunz_s@@PAUunz_global_info_s@@@Z 004169e0 f   unzip.obj
 0001:00015a10       ?unzlocal_DosDateToTmuDate@@YAXKPAUtm_unz_s@@@Z 00416a10 f   unzip.obj
 0001:00015a90       ?unzlocal_GetCurrentFileInfoInternal@@YAHPAUunz_s@@PAUunz_file_info_s@@PAUunz_file_info_internal_s@@PADKPAXK3K@Z 00416a90 f   unzip.obj
 0001:00015ea0       ?unzGetCurrentFileInfo@@YAHPAUunz_s@@PAUunz_file_info_s@@PADKPAXK2K@Z 00416ea0 f   unzip.obj
 0001:00015ed0       ?unzGoToFirstFile@@YAHPAUunz_s@@@Z 00416ed0 f   unzip.obj
 0001:00015f40       ?unzGoToNextFile@@YAHPAUunz_s@@@Z 00416f40 f   unzip.obj
 0001:00016000       ?unzLocateFile@@YAHPAUunz_s@@PBDH@Z 00417000 f   unzip.obj
 0001:000160f0       ?unzlocal_CheckCurrentFileCoherencyHeader@@YAHPAUunz_s@@PAIPAK1@Z 004170f0 f   unzip.obj
 0001:00016370       ?unzOpenCurrentFile@@YAHPAUunz_s@@PBD@Z 00417370 f   unzip.obj
 0001:00016600       ?unzReadCurrentFile@@YAHPAUunz_s@@PAXIPA_N@Z 00417600 f   unzip.obj
 0001:00016a20       ?unztell@@YAJPAUunz_s@@@Z  00417a20 f   unzip.obj
 0001:00016a60       ?unzeof@@YAHPAUunz_s@@@Z   00417a60 f   unzip.obj
 0001:00016ab0       ?unzGetLocalExtrafield@@YAHPAUunz_s@@PAXI@Z 00417ab0 f   unzip.obj
 0001:00016b70       ?unzCloseCurrentFile@@YAHPAUunz_s@@@Z 00417b70 f   unzip.obj
 0001:00016c40       ?unzGetGlobalComment@@YAHPAUunz_s@@PADK@Z 00417c40 f   unzip.obj
 0001:00016cf0       ?timet2filetime@@YA?AU_FILETIME@@I@Z 00417cf0 f   unzip.obj
 0001:00016d30       ?dosdatetime2filetime@@YA?AU_FILETIME@@GG@Z 00417d30 f   unzip.obj
 0001:00016db0       ?Open@TUnzip@@QAEKPAXIK@Z  00417db0 f   unzip.obj
 0001:00016ec0       ?SetUnzipBaseDir@TUnzip@@QAEKPBD@Z 00417ec0 f   unzip.obj
 0001:00016f30       ?Get@TUnzip@@QAEKHPAUZIPENTRY@@@Z 00417f30 f   unzip.obj
 0001:000177f0       ?Find@TUnzip@@QAEKPBD_NPAHPAUZIPENTRY@@@Z 004187f0 f   unzip.obj
 0001:00017900       ?EnsureDirectory@@YAXPBD0@Z 00418900 f   unzip.obj
 0001:00017a40       ?Unzip@TUnzip@@QAEKHPAXIK@Z 00418a40 f   unzip.obj
 0001:00018080       ?Close@TUnzip@@QAEKXZ      00419080 f   unzip.obj
 0001:000180d0       ?FormatZipMessageU@@YAIKPADI@Z 004190d0 f   unzip.obj
 0001:000183b0       ?OpenZipInternal@@YAPAUHZIP__@@PAXIKPBD@Z 004193b0 f   unzip.obj
 0001:000184a0       ?OpenZipHandle@@YAPAUHZIP__@@PAXPBD@Z 004194a0 f   unzip.obj
 0001:000184c0       ?OpenZip@@YAPAUHZIP__@@PBD0@Z 004194c0 f   unzip.obj
 0001:000184e0       ?OpenZip@@YAPAUHZIP__@@PAXIPBD@Z 004194e0 f   unzip.obj
 0001:00018500       ?GetZipItem@@YAKPAUHZIP__@@HPAUZIPENTRY@@@Z 00419500 f   unzip.obj
 0001:00018580       ?FindZipItem@@YAKPAUHZIP__@@PBD_NPAHPAUZIPENTRY@@@Z 00419580 f   unzip.obj
 0001:000185f0       ?UnzipItemInternal@@YAKPAUHZIP__@@HPAXIK@Z 004195f0 f   unzip.obj
 0001:00018660       ?UnzipItemHandle@@YAKPAUHZIP__@@HPAX@Z 00419660 f   unzip.obj
 0001:00018680       ?UnzipItem@@YAKPAUHZIP__@@HPBD@Z 00419680 f   unzip.obj
 0001:000186a0       ?UnzipItem@@YAKPAUHZIP__@@HPAXI@Z 004196a0 f   unzip.obj
 0001:000186c0       ?SetUnzipBaseDir@@YAKPAUHZIP__@@PBD@Z 004196c0 f   unzip.obj
 0001:00018720       ?CloseZipU@@YAKPAUHZIP__@@@Z 00419720 f   unzip.obj
 0001:000187c0       ?IsZipHandleU@@YA_NPAUHZIP__@@@Z 004197c0 f   unzip.obj
 0001:000187f0       __tcsstr                   004197f0 f i unzip.obj
 0001:00018810       __tcsncpy                  00419810 f i unzip.obj
 0001:00018830       ??0TUnzip@@QAE@PBD@Z       00419830 f i unzip.obj
 0001:000188c0       ??_GTUnzip@@QAEPAXI@Z      004198c0 f i unzip.obj
 0001:000188f0       ??1TUnzip@@QAE@XZ          004198f0 f i unzip.obj
 0001:00018960       ??0CAnimControl@@QAE@XZ    00419960 f   AnimControl.obj
 0001:00018980       ?Reset@CAnimControl@@QAEXXZ 00419980 f   AnimControl.obj
 0001:000189a0       ?Update@CAnimControl@@QAEXAAW4EAnimFrame@@AAW4EHeadDirection@@AAW4EDirection@@@Z 004199a0 f   AnimControl.obj
 0001:00018a30       ?Play@CAnimControl@@QAEXW4EAnim@@_NM@Z 00419a30 f   AnimControl.obj
 0001:00018ab0       ?Stop@CAnimControl@@QAEXXZ 00419ab0 f   AnimControl.obj
 0001:00018ad0       ?SetSpeed@CAnimControl@@QAEXM@Z 00419ad0 f   AnimControl.obj
 0001:00018b10       ??0CAnimManager@@QAE@XZ    00419b10 f   AnimManager.obj
 0001:00019310       ?GetFrame@CAnimManager@@QBEXW4EAnim@@H_N1AAW4EAnimFrame@@AAW4EHeadDirection@@AAW4EDirection@@@Z 0041a310 f   AnimManager.obj
 0001:00019550       ?GetSpeed@CAnimManager@@QBE?BMW4EAnim@@@Z 0041a550 f   AnimManager.obj
 0001:00019570       ?RandomWalkFrame@CAnimManager@@QBE?BW4EAnimFrame@@XZ 0041a570 f   AnimManager.obj
 0001:00019590       ?RandomHeadDirection@CAnimManager@@QBE?BW4EHeadDirection@@W4EDirection@@_N@Z 0041a590 f   AnimManager.obj
 0001:000196e0       ?RandomNorthHeadDirection@CAnimManager@@ABE?BW4EHeadDirection@@XZ 0041a6e0 f   AnimManager.obj
 0001:00019700       ?RandomEastHeadDirection@CAnimManager@@ABE?BW4EHeadDirection@@XZ 0041a700 f   AnimManager.obj
 0001:00019720       ?RandomSouthHeadDirection@CAnimManager@@ABE?BW4EHeadDirection@@XZ 0041a720 f   AnimManager.obj
 0001:00019740       ?RandomWestHeadDirection@CAnimManager@@ABE?BW4EHeadDirection@@XZ 0041a740 f   AnimManager.obj
 0001:00019760       ?RandomDirection@CAnimManager@@QBE?BW4EDirection@@XZ 0041a760 f   AnimManager.obj
 0001:00019780       ?IsValidHeadDirection@CAnimManager@@QBE?B_NW4EHeadDirection@@W4EDirection@@@Z 0041a780 f   AnimManager.obj
 0001:000197f0       ?Initialize@SAnim@CAnimManager@@QAEXW4EAnimEffect@@M@Z 0041a7f0 f   AnimManager.obj
 0001:00019830       ?AddFrame@SAnim@CAnimManager@@QAEXW4EAnimFrame@@W4EHeadDirection@@W4EDirection@@@Z 0041a830 f   AnimManager.obj
 0001:000198a0       ??0CBehavior@@QAE@XZ       0041a8a0 f   Behavior.obj
 0001:0001a570       ?BeginNewBehavior@CBehavior@@IBE?B_NAAVCVillager@@W4EBehavior@@ABUSBehaviorData@@@Z 0041b570 f   Behavior.obj
 0001:0001a5d0       ?SetMacro@CBehavior@@QAEXW4EBehavior@@Q6AXAAVCVillager@@@Z@Z 0041b5d0 f   Behavior.obj
 0001:0001a600       ?SetMacro@CBehavior@@QAEXW4EBehavior@@Q6AXAAVCVillager@@ABUSBehaviorData@@@Z@Z 0041b600 f   Behavior.obj
 0001:0001a630       ?FailAtChief@CBehavior@@CAXAAVCVillager@@@Z 0041b630 f   Behavior.obj
 0001:0001a670       ?StudyMedicine@CBehavior@@CAXAAVCVillager@@@Z 0041b670 f   Behavior.obj
 0001:0001a880       ?GettingOutOfRain@CBehavior@@CAXAAVCVillager@@@Z 0041b880 f   Behavior.obj
 0001:0001aab0       ?BecomeChief@CBehavior@@CAXAAVCVillager@@@Z 0041bab0 f   Behavior.obj
 0001:0001ab30       ?NotBecomeChief@CBehavior@@CAXAAVCVillager@@@Z 0041bb30 f   Behavior.obj
 0001:0001ac30       ?WorryAboutFood@CBehavior@@CAXAAVCVillager@@@Z 0041bc30 f   Behavior.obj
 0001:0001aed0       ?ChiefInspectingFood@CBehavior@@CAXAAVCVillager@@@Z 0041bed0 f   Behavior.obj
 0001:0001b040       ?ChiefLookingGloriousAtFire@CBehavior@@CAXAAVCVillager@@@Z 0041c040 f   Behavior.obj
 0001:0001b080       ?ChiefWeatherDance@CBehavior@@CAXAAVCVillager@@@Z 0041c080 f   Behavior.obj
 0001:0001b3e0       ?ChiefDramaticPathStanding@CBehavior@@CAXAAVCVillager@@@Z 0041c3e0 f   Behavior.obj
 0001:0001b510       ?ChiefThinkingInAmp@CBehavior@@CAXAAVCVillager@@@Z 0041c510 f   Behavior.obj
 0001:0001b640       ?ChiefConcernedAboutSick@CBehavior@@CAXAAVCVillager@@@Z 0041c640 f   Behavior.obj
 0001:0001b720       ?ChiefMassiveCure@CBehavior@@CAXAAVCVillager@@@Z 0041c720 f   Behavior.obj
 0001:0001b830       ?ChiefGrantFood@CBehavior@@CAXAAVCVillager@@@Z 0041c830 f   Behavior.obj
 0001:0001bbd0       ?ChiefSpawnRare@CBehavior@@CAXAAVCVillager@@@Z 0041cbd0 f   Behavior.obj
 0001:0001bcf0       ?ChiefInspectingScience@CBehavior@@CAXAAVCVillager@@@Z 0041ccf0 f   Behavior.obj
 0001:0001bd30       ?Idle@CBehavior@@CAXAAVCVillager@@@Z 0041cd30 f   Behavior.obj
 0001:0001bea0       ?PaceSoCent@CBehavior@@CAXAAVCVillager@@@Z 0041cea0 f   Behavior.obj
 0001:0001bf90       ?WalkCircle@CBehavior@@CAXAAVCVillager@@@Z 0041cf90 f   Behavior.obj
 0001:0001c1c0       ?GoToSchoolPopLow@CBehavior@@CAXAAVCVillager@@@Z 0041d1c0 f   Behavior.obj
 0001:0001c350       ?GoToSchoolPopHigh@CBehavior@@CAXAAVCVillager@@@Z 0041d350 f   Behavior.obj
 0001:0001c8d0       ?Lecture@CBehavior@@CAXAAVCVillager@@@Z 0041d8d0 f   Behavior.obj
 0001:0001cab0       ?Coffee@CBehavior@@CAXAAVCVillager@@@Z 0041dab0 f   Behavior.obj
 0001:0001d330       ?SciFair@CBehavior@@CAXAAVCVillager@@@Z 0041e330 f   Behavior.obj
 0001:0001db80       ?NotFeelingWell3@CBehavior@@CAXAAVCVillager@@@Z 0041eb80 f   Behavior.obj
 0001:0001df20       ?NotFeelingWell4@CBehavior@@CAXAAVCVillager@@@Z 0041ef20 f   Behavior.obj
 0001:0001dfb0       ?DrinkingRain@CBehavior@@CAXAAVCVillager@@@Z 0041efb0 f   Behavior.obj
 0001:0001e170       ?DoingLaundry@CBehavior@@CAXAAVCVillager@@@Z 0041f170 f   Behavior.obj
 0001:0001e610       ?EvilTwin@CBehavior@@CAXAAVCVillager@@@Z 0041f610 f   Behavior.obj
 0001:0001e700       ?BlessingsDayDance@CBehavior@@CAXAAVCVillager@@@Z 0041f700 f   Behavior.obj
 0001:0001ea10       ?BlessingsDayDanceII@CBehavior@@CAXAAVCVillager@@@Z 0041fa10 f   Behavior.obj
 0001:0001ec50       ?DayOfTheDeadDance@CBehavior@@CAXAAVCVillager@@@Z 0041fc50 f   Behavior.obj
 0001:0001ee90       ?IsolaDayDance@CBehavior@@CAXAAVCVillager@@@Z 0041fe90 f   Behavior.obj
 0001:0001f2b0       ?PlayWithOtters@CBehavior@@CAXAAVCVillager@@@Z 004202b0 f   Behavior.obj
 0001:0001f610       ?MagicDance@CBehavior@@CAXAAVCVillager@@@Z 00420610 f   Behavior.obj
 0001:0001f700       ?HideInHut@CBehavior@@CAXAAVCVillager@@@Z 00420700 f   Behavior.obj
 0001:0001f780       ?BringBackFoodPrize@CBehavior@@CAXAAVCVillager@@@Z 00420780 f   Behavior.obj
 0001:0001f890       ?BringBackFoodPrizeSlow@CBehavior@@CAXAAVCVillager@@@Z 00420890 f   Behavior.obj
 0001:0001f9c0       ?RescueCrowdToBeach@CBehavior@@CAXAAVCVillager@@@Z 004209c0 f   Behavior.obj
 0001:0001fbc0       ?StompAnts@CBehavior@@CAXAAVCVillager@@@Z 00420bc0 f   Behavior.obj
 0001:0001fce0       ?PortableFrenzy@CBehavior@@CAXAAVCVillager@@HH@Z 00420ce0 f   Behavior.obj
 0001:0001fe00       ?JellyfishPanic@CBehavior@@CAXAAVCVillager@@@Z 00420e00 f   Behavior.obj
 0001:000201e0       ?WashFaceInSpring@CBehavior@@CAXAAVCVillager@@@Z 004211e0 f   Behavior.obj
 0001:00020350       ?WashHandsInSpring@CBehavior@@CAXAAVCVillager@@@Z 00421350 f   Behavior.obj
 0001:000204b0       ?BatheInSpring@CBehavior@@CAXAAVCVillager@@@Z 004214b0 f   Behavior.obj
 0001:00020670       ?GetADrink@CBehavior@@CAXAAVCVillager@@@Z 00421670 f   Behavior.obj
 0001:00020780       ?PointingAtReef@CBehavior@@CAXAAVCVillager@@@Z 00421780 f   Behavior.obj
 0001:00020b70       ?LookForMushrooms@CBehavior@@CAXAAVCVillager@@@Z 00421b70 f   Behavior.obj
 0001:00020ff0       ?Stumbling@CBehavior@@CAXAAVCVillager@@@Z 00421ff0 f   Behavior.obj
 0001:00021420       ?DoingExercise@CBehavior@@CAXAAVCVillager@@@Z 00422420 f   Behavior.obj
 0001:00021820       ?SwimmingWithFish@CBehavior@@CAXAAVCVillager@@@Z 00422820 f   Behavior.obj
 0001:00021f50       ?Worry@CBehavior@@CAXAAVCVillager@@@Z 00422f50 f   Behavior.obj
 0001:00022120       ?Bored@CBehavior@@CAXAAVCVillager@@@Z 00423120 f   Behavior.obj
 0001:00022310       ?CuriousRobe@CBehavior@@CAXAAVCVillager@@@Z 00423310 f   Behavior.obj
 0001:00022470       ?CuriousStatue@CBehavior@@CAXAAVCVillager@@@Z 00423470 f   Behavior.obj
 0001:00022630       ?CuriousDoor@CBehavior@@CAXAAVCVillager@@@Z 00423630 f   Behavior.obj
 0001:000228b0       ?CuriousClam@CBehavior@@CAXAAVCVillager@@@Z 004238b0 f   Behavior.obj
 0001:00022a20       ?CuriousHive@CBehavior@@CAXAAVCVillager@@@Z 00423a20 f   Behavior.obj
 0001:00022bf0       ?CuriousLift@CBehavior@@CAXAAVCVillager@@@Z 00423bf0 f   Behavior.obj
 0001:00022f60       ?CuriousRuins@CBehavior@@CAXAAVCVillager@@@Z 00423f60 f   Behavior.obj
 0001:000230c0       ?CuriousBath@CBehavior@@CAXAAVCVillager@@@Z 004240c0 f   Behavior.obj
 0001:000232a0       ?CuriousAlchLab@CBehavior@@CAXAAVCVillager@@@Z 004242a0 f   Behavior.obj
 0001:000233e0       ?CuriousFire@CBehavior@@CAXAAVCVillager@@@Z 004243e0 f   Behavior.obj
 0001:000235d0       ?CuriousHangingKey@CBehavior@@CAXAAVCVillager@@@Z 004245d0 f   Behavior.obj
 0001:00023770       ?CuriousOrchard@CBehavior@@CAXAAVCVillager@@@Z 00424770 f   Behavior.obj
 0001:000239b0       ?CuriousHerb1@CBehavior@@CAXAAVCVillager@@@Z 004249b0 f   Behavior.obj
 0001:00023ac0       ?CuriousHerb2@CBehavior@@CAXAAVCVillager@@@Z 00424ac0 f   Behavior.obj
 0001:00023bd0       ?CuriousHerb3@CBehavior@@CAXAAVCVillager@@@Z 00424bd0 f   Behavior.obj
 0001:00023ce0       ?CuriousHerb4@CBehavior@@CAXAAVCVillager@@@Z 00424ce0 f   Behavior.obj
 0001:00023df0       ?CuriousHerb5@CBehavior@@CAXAAVCVillager@@@Z 00424df0 f   Behavior.obj
 0001:00023f00       ?CuriousDryGrass@CBehavior@@CAXAAVCVillager@@@Z 00424f00 f   Behavior.obj
 0001:00024020       ?CuriousRoster@CBehavior@@CAXAAVCVillager@@@Z 00425020 f   Behavior.obj
 0001:00024160       ?TellStory@CBehavior@@CAXAAVCVillager@@@Z 00425160 f   Behavior.obj
 0001:000242b0       ?ListenStory@CBehavior@@CAXAAVCVillager@@@Z 004252b0 f   Behavior.obj
 0001:00024340       ?Dance@CBehavior@@CAXAAVCVillager@@@Z 00425340 f   Behavior.obj
 0001:000246d0       ?Sit@CBehavior@@CAXAAVCVillager@@@Z 004256d0 f   Behavior.obj
 0001:00024720       ?Fishing@CBehavior@@CAXAAVCVillager@@@Z 00425720 f   Behavior.obj
 0001:000249a0       ?GetHoney@CBehavior@@CAXAAVCVillager@@@Z 004259a0 f   Behavior.obj
 0001:00024b30       ?RepairBath@CBehavior@@CAXAAVCVillager@@@Z 00425b30 f   Behavior.obj
 0001:00024cf0       ?LeaveOcean@CBehavior@@CAXAAVCVillager@@@Z 00425cf0 f   Behavior.obj
 0001:00024d60       ?Eat@CBehavior@@CAXAAVCVillager@@@Z 00425d60 f   Behavior.obj
 0001:00024e50       ?HangOutPool@CBehavior@@CAXAAVCVillager@@@Z 00425e50 f   Behavior.obj
 0001:00025020       ?HangOutBeach@CBehavior@@CAXAAVCVillager@@@Z 00426020 f   Behavior.obj
 0001:000251c0       ?WanderCemetery@CBehavior@@CAXAAVCVillager@@@Z 004261c0 f   Behavior.obj
 0001:000251d0       ?GoInHouse@CBehavior@@CAXAAVCVillager@@@Z 004261d0 f   Behavior.obj
 0001:00025260       ?StrollingBeach@CBehavior@@CAXAAVCVillager@@@Z 00426260 f   Behavior.obj
 0001:000253a0       ?CircleDance@CBehavior@@CAXAAVCVillager@@@Z 004263a0 f   Behavior.obj
 0001:00025720       ?WashFeet2@CBehavior@@CAXAAVCVillager@@@Z 00426720 f   Behavior.obj
 0001:00025930       ?GenericWarming@CBehavior@@CAXAAVCVillager@@@Z 00426930 f   Behavior.obj
 0001:00025a20       ?GenericSlowWander@CBehavior@@CAXAAVCVillager@@@Z 00426a20 f   Behavior.obj
 0001:00025ad0       ?School@CBehavior@@CAXAAVCVillager@@@Z 00426ad0 f   Behavior.obj
 0001:00025ae0       ?Blessings@CBehavior@@CAXAAVCVillager@@@Z 00426ae0 f   Behavior.obj
 0001:00025af0       ?SwimInBath@CBehavior@@CAXAAVCVillager@@@Z 00426af0 f   Behavior.obj
 0001:00025ca0       ?SwimLagoon@CBehavior@@CAXAAVCVillager@@@Z 00426ca0 f   Behavior.obj
 0001:00025f40       ?Confused@CBehavior@@CAXAAVCVillager@@ABUSStringData@@@Z 00426f40 f   Behavior.obj
 0001:00026090       ?HonorTheDead@CBehavior@@CAXAAVCVillager@@@Z 00427090 f   Behavior.obj
 0001:000262a0       ?Danceparty@CBehavior@@CAXAAVCVillager@@@Z 004272a0 f   Behavior.obj
 0001:00026350       ?Relaxing@CBehavior@@CAXAAVCVillager@@@Z 00427350 f   Behavior.obj
 0001:00026520       ?RainDance@CBehavior@@CAXAAVCVillager@@@Z 00427520 f   Behavior.obj
 0001:000265b0       ?Interact@CBehavior@@CAXAAVCVillager@@@Z 004275b0 f   Behavior.obj
 0001:000267a0       ?NotFeelingWell@CBehavior@@CAXAAVCVillager@@@Z 004277a0 f   Behavior.obj
 0001:00026900       ?KidSpaz@CBehavior@@CAXAAVCVillager@@@Z 00427900 f   Behavior.obj
 0001:00026a90       ?KidPlayTag@CBehavior@@CAXAAVCVillager@@@Z 00427a90 f   Behavior.obj
 0001:00026aa0       ?KidPlaySeeSaw@CBehavior@@CAXAAVCVillager@@@Z 00427aa0 f   Behavior.obj
 0001:00026c30       ?Construct@CBehavior@@CAXAAVCVillager@@ABUSConstructionData@@@Z 00427c30 f   Behavior.obj
 0001:00026f30       ?InspectingHut@CBehavior@@CAXAAVCVillager@@ABUSConstructionData@@@Z 00427f30 f   Behavior.obj
 0001:00027030       ?RepairHut@CBehavior@@CAXAAVCVillager@@ABUSConstructionData@@@Z 00428030 f   Behavior.obj
 0001:00027170       ?RepairLoveshack@CBehavior@@CAXAAVCVillager@@@Z 00428170 f   Behavior.obj
 0001:00027180       ?DoResearch@CBehavior@@CAXAAVCVillager@@@Z 00428180 f   Behavior.obj
 0001:000274d0       ?AssembleAtTable@CBehavior@@CAXAAVCVillager@@@Z 004284d0 f   Behavior.obj
 0001:00027550       ?Sneezing@CBehavior@@CAXAAVCVillager@@@Z 00428550 f   Behavior.obj
 0001:00027610       ?GatherKindling@CBehavior@@CAXAAVCVillager@@@Z 00428610 f   Behavior.obj
 0001:000276d0       ?GatherFirewood@CBehavior@@CAXAAVCVillager@@@Z 004286d0 f   Behavior.obj
 0001:000277a0       ?StartFire@CBehavior@@CAXAAVCVillager@@@Z 004287a0 f   Behavior.obj
 0001:00027800       ?RunAway@CBehavior@@CAXAAVCVillager@@ABUSStringData@@@Z 00428800 f   Behavior.obj
 0001:000279b0       ?StudyTigerLily@CBehavior@@CAXAAVCVillager@@@Z 004289b0 f   Behavior.obj
 0001:00027b00       ?StudyPitcherPlant@CBehavior@@CAXAAVCVillager@@@Z 00428b00 f   Behavior.obj
 0001:00027bc0       ?StudyBlueRose@CBehavior@@CAXAAVCVillager@@@Z 00428bc0 f   Behavior.obj
 0001:00027c90       ?StudyBlackOrchid@CBehavior@@CAXAAVCVillager@@@Z 00428c90 f   Behavior.obj
 0001:00027da0       ?StudyPurpleDaisy@CBehavior@@CAXAAVCVillager@@@Z 00428da0 f   Behavior.obj
 0001:00027e60       ?StudyWaxPlant@CBehavior@@CAXAAVCVillager@@@Z 00428e60 f   Behavior.obj
 0001:00027f30       ?BuryDead@CBehavior@@CAXAAVCVillager@@@Z 00428f30 f   Behavior.obj
 0001:00028110       ?HonorTheStatue@CBehavior@@CAXAAVCVillager@@@Z 00429110 f   Behavior.obj
 0001:00028120       ?CelebrateEvent@CBehavior@@CAXAAVCVillager@@ABUSEventData@@@Z 00429120 f   Behavior.obj
 0001:00028760       ?UncoverMosaic@CBehavior@@CAXAAVCVillager@@@Z 00429760 f   Behavior.obj
 0001:00028770       ?PickShroom@CBehavior@@CAXAAVCVillager@@ABUSPickUpData@@@Z 00429770 f   Behavior.obj
 0001:000288c0       ?PickCollectable@CBehavior@@CAXAAVCVillager@@ABUSPickUpData@@@Z 004298c0 f   Behavior.obj
 0001:00028a90       ?ShakeHead@CBehavior@@CAXAAVCVillager@@@Z 00429a90 f   Behavior.obj
 0001:00028d30       ?SwimSW@CBehavior@@CAXAAVCVillager@@@Z 00429d30 f   Behavior.obj
 0001:00028e80       ?RestInHospital@CBehavior@@CAXAAVCVillager@@@Z 00429e80 f   Behavior.obj
 0001:000291e0       ?NotFeelingWell2@CBehavior@@CAXAAVCVillager@@@Z 0042a1e0 f   Behavior.obj
 0001:00029640       ?Dive@CBehavior@@CAXAAVCVillager@@@Z 0042a640 f   Behavior.obj
 0001:00029720       ?NatureCalls@CBehavior@@CAXAAVCVillager@@@Z 0042a720 f   Behavior.obj
 0001:00029830       ?Lonely@CBehavior@@CAXAAVCVillager@@@Z 0042a830 f   Behavior.obj
 0001:00029940       ?ChangeClothes@CBehavior@@CAXAAVCVillager@@@Z 0042a940 f   Behavior.obj
 0001:00029a10       ?WaitForContact@CBehavior@@CAXAAVCVillager@@@Z 0042aa10 f   Behavior.obj
 0001:00029a60       ?HugSprite@CBehavior@@CAXAAVCVillager@@@Z 0042aa60 f   Behavior.obj
 0001:00029ab0       ?HealSprite@CBehavior@@CAXAAVCVillager@@@Z 0042aab0 f   Behavior.obj
 0001:00029b60       ?ShowBaby@CBehavior@@CAXAAVCVillager@@@Z 0042ab60 f   Behavior.obj
 0001:00029eb0       ?WashBaby@CBehavior@@CAXAAVCVillager@@@Z 0042aeb0 f   Behavior.obj
 0001:0002a040       ?ChangeBaby@CBehavior@@CAXAAVCVillager@@@Z 0042b040 f   Behavior.obj
 0001:0002a100       ?ObserveAdults@CBehavior@@CAXAAVCVillager@@@Z 0042b100 f   Behavior.obj
 0001:0002aa00       ?RepairRainLift@CBehavior@@CAXAAVCVillager@@@Z 0042ba00 f   Behavior.obj
 0001:0002abc0       ?UseRainLift@CBehavior@@CAXAAVCVillager@@@Z 0042bbc0 f   Behavior.obj
 0001:0002ac20       ?DoAlchemy@CBehavior@@CAXAAVCVillager@@@Z 0042bc20 f   Behavior.obj
 0001:0002ad10       ?EmptyPot@CBehavior@@CAXAAVCVillager@@@Z 0042bd10 f   Behavior.obj
 0001:0002ade0       ?DrinkPotion@CBehavior@@CAXAAVCVillager@@@Z 0042bde0 f   Behavior.obj
 0001:0002ae70       ?ChiefSupervise@CBehavior@@CAXAAVCVillager@@@Z 0042be70 f   Behavior.obj
 0001:0002b810       ?Refuse@CBehavior@@CAXAAVCVillager@@ABUSRefuseData@@@Z 0042c810 f   Behavior.obj
 0001:0002b940       ?GatherHerbs@CBehavior@@CAXAAVCVillager@@ABUSGatherHerbsData@@@Z 0042c940 f   Behavior.obj
 0001:0002b9b0       ?ConstructStatueScaffolding@CBehavior@@CAXAAVCVillager@@@Z 0042c9b0 f   Behavior.obj
 0001:0002ba50       ?PushStatue@CBehavior@@CAXAAVCVillager@@@Z 0042ca50 f   Behavior.obj
 0001:0002bb20       ?PlantTree@CBehavior@@CAXAAVCVillager@@ABUSPlantTreeData@@@Z 0042cb20 f   Behavior.obj
 0001:0002bb90       ?HarvestFruit@CBehavior@@CAXAAVCVillager@@ABUSHarvestFruitData@@@Z 0042cb90 f   Behavior.obj
 0001:0002bc20       ?SmokeBees@CBehavior@@CAXAAVCVillager@@@Z 0042cc20 f   Behavior.obj
 0001:0002bca0       ?ClearRubble@CBehavior@@CAXAAVCVillager@@@Z 0042cca0 f   Behavior.obj
 0001:0002bd60       ?ClearLeaves@CBehavior@@CAXAAVCVillager@@@Z 0042cd60 f   Behavior.obj
 0001:0002be50       ?JumpForKey@CBehavior@@CAXAAVCVillager@@@Z 0042ce50 f   Behavior.obj
 0001:0002bf40       ?Faint@CBehavior@@CAXAAVCVillager@@@Z 0042cf40 f   Behavior.obj
 0001:0002c120       ?TooHot@CBehavior@@CAXAAVCVillager@@@Z 0042d120 f   Behavior.obj
 0001:0002c650       ?TooCold@CBehavior@@CAXAAVCVillager@@@Z 0042d650 f   Behavior.obj
 0001:0002c870       ?Itchy@CBehavior@@CAXAAVCVillager@@@Z 0042d870 f   Behavior.obj
 0001:0002cc80       ?Paralyzed@CBehavior@@CAXAAVCVillager@@@Z 0042dc80 f   Behavior.obj
 0001:0002cd80       ?GarlicBreath@CBehavior@@CAXAAVCVillager@@@Z 0042dd80 f   Behavior.obj
 0001:0002d150       ?BubbleBreath@CBehavior@@CAXAAVCVillager@@@Z 0042e150 f   Behavior.obj
 0001:0002d520       ?Hiccup@CBehavior@@CAXAAVCVillager@@@Z 0042e520 f   Behavior.obj
 0001:0002d8e0       ?HiccupInCenter@CBehavior@@CAXAAVCVillager@@@Z 0042e8e0 f   Behavior.obj
 0001:0002d9a0       ?GarlicInCenter@CBehavior@@CAXAAVCVillager@@@Z 0042e9a0 f   Behavior.obj
 0001:0002da60       ?BubblesInCenter@CBehavior@@CAXAAVCVillager@@@Z 0042ea60 f   Behavior.obj
 0001:0002db20       ?PlayInDirt@CBehavior@@CAXAAVCVillager@@@Z 0042eb20 f   Behavior.obj
 0001:0002dd70       ?GoneCrazy@CBehavior@@CAXAAVCVillager@@@Z 0042ed70 f   Behavior.obj
 0001:0002df50       ?GatherForSweetDrink@CBehavior@@CAXAAVCVillager@@@Z 0042ef50 f   Behavior.obj
 0001:0002dfd0       ?Blind@CBehavior@@CAXAAVCVillager@@@Z 0042efd0 f   Behavior.obj
 0001:0002e190       ?MomTeachingTalk@CBehavior@@CAXAAVCVillager@@@Z 0042f190 f   Behavior.obj
 0001:0002e310       ?PlayingInSand@CBehavior@@CAXAAVCVillager@@@Z 0042f310 f   Behavior.obj
 0001:0002e5c0       ?CleaningAfterStorm@CBehavior@@CAXAAVCVillager@@@Z 0042f5c0 f   Behavior.obj
 0001:0002e890       ?BadDancing@CBehavior@@CAXAAVCVillager@@@Z 0042f890 f   Behavior.obj
 0001:0002eaa0       ?LayDown@CBehavior@@CAXAAVCVillager@@@Z 0042faa0 f   Behavior.obj
 0001:0002eb90       ?SitDown@CBehavior@@CAXAAVCVillager@@@Z 0042fb90 f   Behavior.obj
 0001:0002eca0       ?Spirituality@CBehavior@@CAXAAVCVillager@@@Z 0042fca0 f   Behavior.obj
 0001:0002edc0       ?Trance@CBehavior@@CAXAAVCVillager@@@Z 0042fdc0 f   Behavior.obj
 0001:0002f0c0       ?DropVialInOcean@CBehavior@@CAXAAVCVillager@@@Z 004300c0 f   Behavior.obj
 0001:0002f130       ?LookingForAGrownUp@CBehavior@@CAXAAVCVillager@@@Z 00430130 f   Behavior.obj
 0001:0002f990       ?LookingForAGrownUp2@CBehavior@@CAXAAVCVillager@@@Z 00430990 f   Behavior.obj
 0001:00030730       ?ChildrenPlayInPuddles@CBehavior@@CAXAAVCVillager@@@Z 00431730 f   Behavior.obj
 0001:00030b20       ?ShowBabyBees@CBehavior@@CAXAAVCVillager@@@Z 00431b20 f   Behavior.obj
 0001:00030c10       ?ExamineAHut@CBehavior@@CAXAAVCVillager@@@Z 00431c10 f   Behavior.obj
 0001:000315f0       ?ShowBabyHerbs@CBehavior@@CAXAAVCVillager@@@Z 004325f0 f   Behavior.obj
 0001:00031840       ?HidingSomething@CBehavior@@CAXAAVCVillager@@@Z 00432840 f   Behavior.obj
 0001:00031b10       ?SpringCleaning@CBehavior@@CAXAAVCVillager@@@Z 00432b10 f   Behavior.obj
 0001:00031cc0       ?ShowBabyOrchard@CBehavior@@CAXAAVCVillager@@@Z 00432cc0 f   Behavior.obj
 0001:000320e0       ?ShowBabyAmphetheater@CBehavior@@CAXAAVCVillager@@@Z 004330e0 f   Behavior.obj
 0001:00032740       ?SunningChildByBeach@CBehavior@@CAXAAVCVillager@@@Z 00433740 f   Behavior.obj
 0001:000329b0       ?SecretlyPracticing@CBehavior@@CAXAAVCVillager@@@Z 004339b0 f   Behavior.obj
 0001:00032d70       ?HuddleAroundFire@CBehavior@@CAXAAVCVillager@@@Z 00433d70 f   Behavior.obj
 0001:00032dd0       ?DrawPlans@CBehavior@@CAXAAVCVillager@@@Z 00433dd0 f   Behavior.obj
 0001:00032e40       ?DoAromatherapy@CBehavior@@CAXAAVCVillager@@@Z 00433e40 f   Behavior.obj
 0001:00032f40       ?LightBurners@CBehavior@@CAXAAVCVillager@@@Z 00433f40 f   Behavior.obj
 0001:00033020       ?SwapPearlForKey@CBehavior@@CAXAAVCVillager@@@Z 00434020 f   Behavior.obj
 0001:00033090       ?DepositInFoodBin@CBehavior@@CAXAAVCVillager@@@Z 00434090 f   Behavior.obj
 0001:000330e0       ?QuelchFire@CBehavior@@CAXAAVCVillager@@@Z 004340e0 f   Behavior.obj
 0001:00033140       ?ShapePearlForKey@CBehavior@@CAXAAVCVillager@@@Z 00434140 f   Behavior.obj
 0001:000331d0       ?PolishPearlForKey@CBehavior@@CAXAAVCVillager@@@Z 004341d0 f   Behavior.obj
 0001:00033260       ?SetMacro@CBehavior@@QAEXW4EBehavior@@Q6AXAAVCVillager@@ABUSHarvestFruitData@@@Z@Z 00434260 f i Behavior.obj
 0001:00033260       ?SetMacro@CBehavior@@QAEXW4EBehavior@@Q6AXAAVCVillager@@ABUSEventData@@@Z@Z 00434260 f i Behavior.obj
 0001:00033260       ?SetMacro@CBehavior@@QAEXW4EBehavior@@Q6AXAAVCVillager@@ABUSPickUpData@@@Z@Z 00434260 f i Behavior.obj
 0001:00033260       ?SetMacro@CBehavior@@QAEXW4EBehavior@@Q6AXAAVCVillager@@ABUSRefuseData@@@Z@Z 00434260 f i Behavior.obj
 0001:00033260       ?SetMacro@CBehavior@@QAEXW4EBehavior@@Q6AXAAVCVillager@@ABUSGatherHerbsData@@@Z@Z 00434260 f i Behavior.obj
 0001:00033260       ?SetMacro@CBehavior@@QAEXW4EBehavior@@Q6AXAAVCVillager@@ABUSConstructionData@@@Z@Z 00434260 f i Behavior.obj
 0001:00033260       ?SetMacro@CBehavior@@QAEXW4EBehavior@@Q6AXAAVCVillager@@ABUSPlantTreeData@@@Z@Z 00434260 f i Behavior.obj
 0001:00033260       ?SetMacro@CBehavior@@QAEXW4EBehavior@@Q6AXAAVCVillager@@ABUSStringData@@@Z@Z 00434260 f i Behavior.obj
 0001:00033280       ?IsFemale@CVillagerBio@@QBE?B_NXZ 00434280 f i Behavior.obj
 0001:000332a0       ?IsAdeptAt@CVillagerSkills@@QBE?B_NW4ESkill@@@Z 004342a0 f i Behavior.obj
 0001:000332c0       ?IsChief@CVillagerState@@QBE?B_NXZ 004342c0 f i Behavior.obj
 0001:000332e0       ?IsCaringForBaby@CVillagerState@@QBE?B_NXZ 004342e0 f i Behavior.obj
 0001:00033300       ?StartNewBehavior@CVillager@@QAEXXZ 00434300 f i Behavior.obj
 0001:00033320       ?IsChild@CVillagerBio@@QBE?B_NXZ 00434320 f i Behavior.obj
 0001:00033340       ?Dislikes@CVillager@@QAE?B_NW4ELike@@@Z 00434340 f i Behavior.obj
 0001:00033360       ?SetBehaviorLabel@CVillager@@QAEXPAD@Z 00434360 f i Behavior.obj
 0001:00033390       ?ForgetPlans@CVillager@@QAEXXZ 00434390 f i Behavior.obj
 0001:000333b0       ?IsLow@CFoodStore@@QBE?B_NXZ 004343b0 f i Behavior.obj
 0001:000333d0       ?XPos@CVillager@@QBE?BHXZ  004343d0 f i Behavior.obj
 0001:000333f0       ?YPos@CVillager@@QBE?BHXZ  004343f0 f i Behavior.obj
 0001:00033410       ?SetBehaviorLabel@CVillager@@QAEXW4StringId@@@Z 00434410 f i Behavior.obj
 0001:00033450       ?Likes@CVillager@@QAE?B_NW4ELike@@@Z 00434450 f i Behavior.obj
 0001:00033470       ?HowLong@CBehavior@@QAEHXZ 00434470 f i Behavior.obj
 0001:00033490       ?IsMasterOf@CVillagerSkills@@QBE?B_NW4ESkill@@@Z 00434490 f i Behavior.obj
 0001:000334b0       ?SetPreDisposition@CVillagerState@@QAEXH@Z 004344b0 f i Behavior.obj
 0001:000334d0       ?HasDisease@CVillagerState@@QBE?B_NXZ 004344d0 f i Behavior.obj
 0001:000334f0       ?HasFocus@CVillager@@QBE?B_NXZ 004344f0 f i Behavior.obj
 0001:00033510       ?IsMale@CVillagerBio@@QBE?B_NXZ 00434510 f i Behavior.obj
 0001:00033530       ?WhichTarget@CBehavior@@QAEHXZ 00434530 f i Behavior.obj
 0001:00033550       ?IsAdult@CVillagerBio@@QBE?B_NXZ 00434550 f i Behavior.obj
 0001:00033570       ??HldwPoint@@QBE?AU0@ABU0@@Z 00434570 f i Behavior.obj
 0001:000335a0       ??GldwPoint@@QBE?AU0@ABU0@@Z 004345a0 f i Behavior.obj
 0001:000335d0       ?Exists@CVillager@@QBE?B_NXZ 004345d0 f i Behavior.obj
 0001:000335f0       ?CurrentBehavior@CVillager@@QBE?BW4EBehavior@@XZ 004345f0 f i Behavior.obj
 0001:00033610       ?GetIngredient@CAlchemyTable@@QBE?BW4ECarrying@@H@Z 00434610 f i Behavior.obj
 0001:00033630       ?PreDisposition@CVillagerState@@QBE?BHXZ 00434630 f i Behavior.obj
 0001:00033650       ??8ldwPoint@@QAE?B_NABU0@@Z 00434650 f i Behavior.obj
 0001:00033690       ?Ref@CVillager@@QBE?BHXZ   00434690 f i Behavior.obj
 0001:000336b0       ??0CDislikeList@@QAE@XZ    004346b0 f   DislikeList.obj
 0001:000336d0       ?Reset@CDislikeList@@QAEXXZ 004346d0 f   DislikeList.obj
 0001:00033710       ?Initialize@CDislikeList@@QAEXAAVCLikeList@@@Z 00434710 f   DislikeList.obj
 0001:000337c0       ?Add@CDislikeList@@QAE?B_NW4ELike@@@Z 004347c0 f   DislikeList.obj
 0001:00033820       ?Remove@CDislikeList@@QAE?B_NW4ELike@@@Z 00434820 f   DislikeList.obj
 0001:00033870       ?Contains@CDislikeList@@QBE?B_NW4ELike@@@Z 00434870 f   DislikeList.obj
 0001:000338b0       ?GetListAsString@CDislikeList@@QBEPBDXZ 004348b0 f   DislikeList.obj
 0001:000339f0       ??0CGraveyard@@QAE@XZ      004349f0 f   Graveyard.obj
 0001:00033a10       ?LoadState@CGraveyard@@QAE?B_NABUSSaveState@1@@Z 00434a10 f   Graveyard.obj
 0001:00033c50       ?SaveState@CGraveyard@@QBE?B_NAAUSSaveState@1@@Z 00434c50 f   Graveyard.obj
 0001:00033d20       ?Reset@CGraveyard@@QAEXXZ  00434d20 f   Graveyard.obj
 0001:00033df0       ?Update@CGraveyard@@QAEXXZ 00434df0 f   Graveyard.obj
 0001:00033ec0       ?Draw@CGraveyard@@QAEXXZ   00434ec0 f   Graveyard.obj
 0001:00033f50       ?Draw@CGraveyard@@QAEXH_N@Z 00434f50 f   Graveyard.obj
 0001:00034100       ?Bury@CGraveyard@@QAE?B_NABVCVillager@@H@Z 00435100 f   Graveyard.obj
 0001:00034420       ?GetGraveAtPos@CGraveyard@@QBEPBUSGrave@1@UldwPoint@@@Z 00435420 f   Graveyard.obj
 0001:00034560       ?GetTombAtPos@CGraveyard@@QBEPBUSTomb@1@UldwPoint@@@Z 00435560 f   Graveyard.obj
 0001:00034570       ?GetDeathRecord@CGraveyard@@QAEPAUSDeathRecord@1@H@Z 00435570 f   Graveyard.obj
 0001:000345b0       ?GetNumGraves@CGraveyard@@QBE?BHXZ 004355b0 f   Graveyard.obj
 0001:00034600       ?GetNumTombs@CGraveyard@@QBE?BHXZ 00435600 f   Graveyard.obj
 0001:00034650       ?GetNumDead@CGraveyard@@QBE?BHXZ 00435650 f   Graveyard.obj
 0001:00034710       ??YldwPoint@@QAEAAU0@ABU0@@Z 00435710 f i Graveyard.obj
 0001:00034750       ??ZldwPoint@@QAEAAU0@ABU0@@Z 00435750 f i Graveyard.obj
 0001:00034790       ?IsFertile@CVillagerBio@@QBE?B_NXZ 00435790 f i Graveyard.obj
 0001:000347b0       ?FirstName@CVillagerBio@@QBEPBDXZ 004357b0 f i Graveyard.obj
 0001:000347d0       ?IsDead@CVillagerState@@QBE?B_NXZ 004357d0 f i Graveyard.obj
 0001:000347f0       ?Carrying@CVillager@@QBE?BW4ECarrying@@XZ 004357f0 f i Graveyard.obj
 0001:00034810       ?Pos@CWorldView@@QBE?BUldwPoint@@XZ 00435810 f i Graveyard.obj
 0001:00034830       ??0CLikeList@@QAE@XZ       00435830 f   LikeList.obj
 0001:00034850       ?Reset@CLikeList@@QAEXXZ   00435850 f   LikeList.obj
 0001:00034890       ?Initialize@CLikeList@@QAEXXZ 00435890 f   LikeList.obj
 0001:00034930       ?Add@CLikeList@@QAE?B_NW4ELike@@@Z 00435930 f   LikeList.obj
 0001:00034990       ?Remove@CLikeList@@QAE?B_NW4ELike@@@Z 00435990 f   LikeList.obj
 0001:000349e0       ?Contains@CLikeList@@QBE?B_NW4ELike@@@Z 004359e0 f   LikeList.obj
 0001:00034a20       ?GetListAsString@CLikeList@@QBEPBDXZ 00435a20 f   LikeList.obj
 0001:00034b60       ??0CVillager@@QAE@XZ       00435b60 f   Villager.obj
 0001:00034bf0       ?Reset@CVillager@@QAEXXZ   00435bf0 f   Villager.obj
 0001:00034da0       ?Init@CVillager@@QAEXHW4ESkill@@HW4EGender@@HPBD2HHHHHH_N@Z 00435da0 f   Villager.obj
 0001:00035550       ?InitTwin@CVillager@@QAEXAAV1@@Z 00436550 f   Villager.obj
 0001:00035720       ?SaveState@CVillager@@QAE?B_NAAUSSaveState@1@@Z 00436720 f   Villager.obj
 0001:00035800       ?LoadState@CVillager@@QAE?B_NAAUSSaveState@1@@Z 00436800 f   Villager.obj
 0001:000358f0       ?DrawDetailVillager@CVillager@@QAEXXZ 004368f0 f   Villager.obj
 0001:00035d40       ?DrawDetailVillagerParents@CVillager@@QAEXXZ 00436d40 f   Villager.obj
 0001:00035e60       ?DrawEventVillager@CVillager@@QAEXHHW4EBodyPosition@@@Z 00436e60 f   Villager.obj
 0001:00036270       ?SelectDirectionBasedOnVelocity@CVillager@@AAEXXZ 00437270 f   Villager.obj
 0001:00036340       ?Update@CVillager@@QAEXXZ  00437340 f   Villager.obj
 0001:00036740       ?NewBehavior@CVillager@@QAEXW4EBehavior@@ABUSBehaviorData@@@Z 00437740 f   Villager.obj
 0001:00036770       ?StartWaiting@CVillager@@IAEXW4EBodyPosition@@W4EDirection@@W4EHeadDirection@@@Z 00437770 f   Villager.obj
 0001:00036860       ?StartBending@CVillager@@IAEXXZ 00437860 f   Villager.obj
 0001:000368a0       ?StartCheering@CVillager@@IAEXXZ 004378a0 f   Villager.obj
 0001:000368e0       ?StartTwirlingCW@CVillager@@IAEXXZ 004378e0 f   Villager.obj
 0001:00036920       ?StartTwirlingCCW@CVillager@@IAEXXZ 00437920 f   Villager.obj
 0001:00036960       ?StartDiscoing@CVillager@@IAEXXZ 00437960 f   Villager.obj
 0001:000369a0       ?StartDoingTheMonkey@CVillager@@IAEXXZ 004379a0 f   Villager.obj
 0001:000369e0       ?StartReveling@CVillager@@IAEXXZ 004379e0 f   Villager.obj
 0001:00036a20       ?StartLyingDown@CVillager@@IAEXXZ 00437a20 f   Villager.obj
 0001:00036a60       ?StartScrubbing@CVillager@@IAEXXZ 00437a60 f   Villager.obj
 0001:00036aa0       ?StartExorcisting@CVillager@@IAEXXZ 00437aa0 f   Villager.obj
 0001:00036ae0       ?StartJoyTwirlingCW@CVillager@@IAEXXZ 00437ae0 f   Villager.obj
 0001:00036b20       ?StartClimbing@CVillager@@IAEXUSClimbData@CVillagerPlans@@@Z 00437b20 f   Villager.obj
 0001:00036ba0       ?StartDancing@CVillager@@IAEXXZ 00437ba0 f   Villager.obj
 0001:00036c10       ?StartEmbrace@CVillager@@IAEXXZ 00437c10 f   Villager.obj
 0001:00036fb0       ?StartDiving@CVillager@@IAEXAAUSDiveData@CVillagerPlans@@@Z 00437fb0 f   Villager.obj
 0001:00037050       ?StartGoing@CVillager@@IAEXAAUSGoingData@CVillagerPlans@@@Z 00438050 f   Villager.obj
 0001:00037140       ?StartHiding@CVillager@@IAEXXZ 00438140 f   Villager.obj
 0001:00037190       ?StartHealing@CVillager@@IAEXXZ 00438190 f   Villager.obj
 0001:00037370       ?StartJumping@CVillager@@IAEXAAUSJumpData@CVillagerPlans@@@Z 00438370 f   Villager.obj
 0001:00037400       ?StartNothing@CVillager@@IAEXXZ 00438400 f   Villager.obj
 0001:00037450       ?StartSwimming@CVillager@@IAEXUSSwimData@CVillagerPlans@@@Z 00438450 f   Villager.obj
 0001:00037530       ?StartWandering@CVillager@@IAEXAAUSWanderingData@CVillagerPlans@@@Z 00438530 f   Villager.obj
 0001:00037630       ?StartWorking@CVillager@@IAEXXZ 00438630 f   Villager.obj
 0001:00037670       ?StartDoingPushups@CVillager@@IAEXXZ 00438670 f   Villager.obj
 0001:000376b0       ?ProcessClimbing@CVillager@@IAEXUSClimbData@CVillagerPlans@@@Z 004386b0 f   Villager.obj
 0001:00037760       ?ProcessDancing@CVillager@@IAEXXZ 00438760 f   Villager.obj
 0001:00037780       ?ProcessDiving@CVillager@@IAEXAAUSDiveData@CVillagerPlans@@@Z 00438780 f   Villager.obj
 0001:00037970       ?ProcessEmbrace@CVillager@@IAEXXZ 00438970 f   Villager.obj
 0001:000379d0       ?ProcessFollowPath@CVillager@@IAEXAAUSGoingData@CVillagerPlans@@@Z 004389d0 f   Villager.obj
 0001:00037d00       ?ProcessGoing@CVillager@@IAEXAAUSGoingData@CVillagerPlans@@@Z 00438d00 f   Villager.obj
 0001:000381e0       ?ProcessJumping@CVillager@@IAEXUSJumpData@CVillagerPlans@@@Z 004391e0 f   Villager.obj
 0001:000382d0       ?ProcessSwimming@CVillager@@IAEXXZ 004392d0 f   Villager.obj
 0001:00038500       ?ProcessWaiting@CVillager@@IAEXXZ 00439500 f   Villager.obj
 0001:00038560       ?ProcessWandering@CVillager@@IAEXAAUSWanderingData@CVillagerPlans@@@Z 00439560 f   Villager.obj
 0001:00038a60       ?AddFootprints@CVillager@@AAEXXZ 00439a60 f   Villager.obj
 0001:00038cc0       ?AddDust@CVillager@@AAEXXZ 00439cc0 f   Villager.obj
 0001:00038da0       ?ResetToNeutralBodyPosition@CVillager@@IAEXXZ 00439da0 f   Villager.obj
 0001:00038e70       ?DropVillager@CVillager@@QAEXXZ 00439e70 f   Villager.obj
 0001:00038f10       ?NormVel@CVillager@@QAEXH@Z 00439f10 f   Villager.obj
 0001:00038fb0       ?Stop@CVillager@@QAEXXZ    00439fb0 f   Villager.obj
 0001:00039000       ?ConceiveChildWith@CVillager@@QAEXPAV1@_N@Z 0043a000 f   Villager.obj
 0001:00039120       ?Impregnate@CVillager@@QAEXHW4ESkill@@HPBDHH_N@Z 0043a120 f   Villager.obj
 0001:00039330       ?SetVillagerInHand@CVillager@@QAEXXZ 0043a330 f   Villager.obj
 0001:00039390       ?ChanceOfDisease@CVillager@@QAE?BHXZ 0043a390 f   Villager.obj
 0001:000395c0       ?Attach@CVillager@@QAE?B_NAAVIVillagerAttachment@@HUldwPoint@@H@Z 0043a5c0 f   Villager.obj
 0001:00039700       ?Detach@CVillager@@QAEXAAVIVillagerAttachment@@AAH@Z 0043a700 f   Villager.obj
 0001:00039820       ?DetachAll@CVillager@@QAEXXZ 0043a820 f   Villager.obj
 0001:00039870       ?HasAttachment@CVillager@@QBE?B_NAAVIVillagerAttachment@@H@Z 0043a870 f   Villager.obj
 0001:000398e0       ?Scale@CVillager@@QBE?BMXZ 0043a8e0 f   Villager.obj
 0001:00039940       ?Dimensions@CVillager@@QBE?BUldwPoint@@XZ 0043a940 f   Villager.obj
 0001:00039980       ?SetFeetPos@CVillager@@QAEXUldwPoint@@@Z 0043a980 f   Villager.obj
 0001:000399e0       ?FeetPos@CVillager@@QBE?BUldwPoint@@XZ 0043a9e0 f   Villager.obj
 0001:00039a40       ?SetCarrying@CVillager@@QAEXW4ECarrying@@@Z 0043aa40 f   Villager.obj
 0001:00039aa0       ?ForceCarrying@CVillager@@QAEXW4ECarrying@@@Z 0043aaa0 f   Villager.obj
 0001:00039ac0       ?SayOh@CVillager@@QAEXXZ   0043aac0 f   Villager.obj
 0001:00039b80       ??0CVillagerAI@@QAE@XZ     0043ab80 f i Villager.obj
 0001:00039ba0       ??0CVillagerPlans@@QAE@XZ  0043aba0 f i Villager.obj
 0001:00039bc0       ??DldwPoint@@QBE?AU0@ABM@Z 0043abc0 f i Villager.obj
 0001:00039c00       ?SetHowLong@CBehavior@@QAEXH@Z 0043ac00 f i Villager.obj
 0001:00039c20       ?SetSkill@CVillagerSkills@@QAEXW4ESkill@@H@Z 0043ac20 f i Villager.obj
 0001:00039c70       ?Skill@CVillagerSkills@@QBE?BHW4ESkill@@@Z 0043ac70 f i Villager.obj
 0001:00039c90       ?SetPreferredSkill@CVillagerSkills@@QAEXW4ESkill@@@Z 0043ac90 f i Villager.obj
 0001:00039cb0       ?IsElderly@CVillagerBio@@QBE?B_NXZ 0043acb0 f i Villager.obj
 0001:00039cd0       ?HasGreyHair@CVillagerBio@@QBE?B_NXZ 0043acd0 f i Villager.obj
 0001:00039cf0       ?IsNotFertile@CVillagerBio@@QBE?B_NXZ 0043acf0 f i Villager.obj
 0001:00039d10       ?SetLastTimeChecked@CVillagerState@@QAEXK@Z 0043ad10 f i VillagerManager.obj
 0001:00039d10       ?CaptureMouse@ldwEventManagerImpl@@QAEXPAVldwEventHandler@@@Z 0043ad10 f i ldwEventManager.obj
 0001:00039d10       ?SetGender@CVillagerBio@@QAEXW4EGender@@@Z 0043ad10 f i Villager.obj
 0001:00039d10       ?SetExtraKerning@ldwFontImpl@@QAEXH@Z 0043ad10 f i ldwFont.obj
 0001:00039d30       ?SetGameStartTime@CGameStats@@QAEXI@Z 0043ad30 f i StoryScene.obj
 0001:00039d30       ?SetAge@CVillagerBio@@QAEXH@Z 0043ad30 f i Villager.obj
 0001:00039d30       ?SetSecondsAccumulated@CVillagerState@@QAEXK@Z 0043ad30 f i VillagerManager.obj
 0001:00039d30       ?Attach@CRegKey@ATL@@QAEXPAUHKEY__@@@Z 0043ad30 f i FlashPlayer.obj
 0001:00039d50       ?SetTotemY@CVillagerState@@QAEXH@Z 0043ad50 f i Villager.obj
 0001:00039d50       ?SetBodyType@CVillagerBio@@QAEXH@Z 0043ad50 f i Villager.obj
 0001:00039d70       ?BodyType@CVillagerBio@@QBE?BHXZ 0043ad70 f i Villager.obj
 0001:00039d70       ?TotemY@CVillagerState@@QBE?BHXZ 0043ad70 f i Villager.obj
 0001:00039d90       ?SetHeadType@CVillagerBio@@QAEXH@Z 0043ad90 f i Villager.obj
 0001:00039dd0       ?SetMotherName@CVillagerBio@@QAEXPBD@Z 0043add0 f i Villager.obj
 0001:00039e00       ?MotherName@CVillagerBio@@QBEPBDXZ 0043ae00 f i Villager.obj
 0001:00039e20       ?SetFatherName@CVillagerBio@@QAEXPBD@Z 0043ae20 f i Villager.obj
 0001:00039e50       ?FatherName@CVillagerBio@@QBEPBDXZ 0043ae50 f i Villager.obj
 0001:00039e70       ?SetFatherBodyType@CVillagerBio@@QAEXH@Z 0043ae70 f i Villager.obj
 0001:00039e90       ?FatherBodyType@CVillagerBio@@QBE?BHXZ 0043ae90 f i Villager.obj
 0001:00039eb0       ?SetMotherBodyType@CVillagerBio@@QAEXH@Z 0043aeb0 f i Villager.obj
 0001:00039ed0       ?MotherBodyType@CVillagerBio@@QBE?BHXZ 0043aed0 f i Villager.obj
 0001:00039ef0       ?SetFatherHeadType@CVillagerBio@@QAEXH@Z 0043aef0 f i Villager.obj
 0001:00039f10       ?FatherHeadType@CVillagerBio@@QBE?BHXZ 0043af10 f i Villager.obj
 0001:00039f30       ?SetMotherHeadType@CVillagerBio@@QAEXH@Z 0043af30 f i Villager.obj
 0001:00039f50       ?MotherHeadType@CVillagerBio@@QBE?BHXZ 0043af50 f i Villager.obj
 0001:00039f70       ?IsTotem@CVillagerState@@QBE?B_NXZ 0043af70 f i Villager.obj
 0001:00039f90       ?SetChiefFlag@CVillagerState@@QAEX_N@Z 0043af90 f i Villager.obj
 0001:00039fc0       ?SetChosenOne@CVillagerState@@QAEX_N@Z 0043afc0 f i Villager.obj
 0001:00039fe0       ?SetDisease@CVillagerState@@QAEXH@Z 0043afe0 f i Villager.obj
 0001:0003a000       ?IsHealthy@CVillagerState@@QBE?B_NXZ 0043b000 f i Villager.obj
 0001:0003a020       ?JumpHeight@CVillagerState@@QBE?BHXZ 0043b020 f i Villager.obj
 0001:0003a040       ??0SActionPlan@CVillagerPlans@@QAE@XZ 0043b040 f i Villager.obj
 0001:0003a070       ?NextPlan@CVillager@@QAEXXZ 0043b070 f i Villager.obj
 0001:0003a090       ?Pos@CVillager@@QBE?BUldwPoint@@XZ 0043b090 f i Villager.obj
 0001:0003a0c0       ?SetTotemX@CVillagerState@@QAEXH@Z 0043b0c0 f i Villager.obj
 0001:0003a0e0       ?SetHeadDirection@CVillager@@QAEXW4EHeadDirection@@@Z 0043b0e0 f i Villager.obj
 0001:0003a120       ?SetBodyPosition@CVillager@@IAEXW4EBodyPosition@@@Z 0043b120 f i Villager.obj
 0001:0003a140       ?AdjustSkill@CVillagerSkills@@QAEXW4ESkill@@H@Z 0043b140 f i Villager.obj
 0001:0003a1a0       ?SetFatherLName@CVillagerBio@@QAEXH@Z 0043b1a0 f i Villager.obj
 0001:0003a1c0       ?SetFatherSkillType@CVillagerBio@@QAEXW4ESkill@@@Z 0043b1c0 f i Villager.obj
 0001:0003a1e0       ?SetFatherSkillValue@CVillagerBio@@QAEXH@Z 0043b1e0 f i Villager.obj
 0001:0003a200       ?SetHusbandName@CVillagerBio@@QAEXPBD@Z 0043b200 f i Villager.obj
 0001:0003a230       ?SetHusbandBodyType@CVillagerBio@@QAEXH@Z 0043b230 f i Villager.obj
 0001:0003a250       ?SetHusbandHeadType@CVillagerBio@@QAEXH@Z 0043b250 f i Villager.obj
 0001:0003a270       ?IncrementBabiesMade@CGameStats@@QAEXH@Z 0043b270 f i Villager.obj
 0001:0003a270       ?AdjustAgesChecked@CVillagerState@@QAEXH@Z 0043b270 f i VillagerManager.obj
 0001:0003a290       ?IncrementVillagersCured@CGameStats@@QAEXH@Z 0043b290 f i Villager.obj
 0001:0003a2b0       ?IncrementTwins@CGameStats@@QAEXH@Z 0043b2b0 f i Villager.obj
 0001:0003a2d0       ?IncrementTriplets@CGameStats@@QAEXH@Z 0043b2d0 f i Villager.obj
 0001:0003a2f0       ?Reset@CVillagerAI@@QAEXAAVCVillager@@@Z 0043b2f0 f   VillagerAI.obj
 0001:0003a320       ?Update@CVillagerAI@@QAEXAAVCVillager@@@Z 0043b320 f   VillagerAI.obj
 0001:0003a440       ?DecideWhatToDo@CVillagerAI@@AAEXAAVCVillager@@@Z 0043b440 f   VillagerAI.obj
 0001:0003a930       ?DecideOnChildBehavior@CVillagerAI@@QAE?B_NAAVCVillager@@@Z 0043b930 f   VillagerAI.obj
 0001:0003ad70       ?DecideOnStormyBehavior@CVillagerAI@@AAE?B_NAAVCVillager@@@Z 0043bd70 f   VillagerAI.obj
 0001:0003ae30       ?DecideOnPregnantBehavior@CVillagerAI@@AAE?B_NAAVCVillager@@@Z 0043be30 f   VillagerAI.obj
 0001:0003b010       ?DecideOnWorkSkill@CVillagerAI@@QAE?BW4ESkill@@AAVCVillager@@@Z 0043c010 f   VillagerAI.obj
 0001:0003b280       ?DecideOnIdleBehavior@CVillagerAI@@AAE?B_NAAVCVillager@@@Z 0043c280 f   VillagerAI.obj
 0001:0003b2c0       ?DecideOnDayToDayBehavior@CVillagerAI@@AAE?B_NAAVCVillager@@@Z 0043c2c0 f   VillagerAI.obj
 0001:0003b500       ?DecideOnRecreation@CVillagerAI@@AAE?B_NAAVCVillager@@@Z 0043c500 f   VillagerAI.obj
 0001:0003b720       ?DecideOnCuriousBehavior@CVillagerAI@@AAE?B_NAAVCVillager@@@Z 0043c720 f   VillagerAI.obj
 0001:0003ba40       ?DecideOnEnlightenment@CVillagerAI@@AAE?B_NAAVCVillager@@@Z 0043ca40 f   VillagerAI.obj
 0001:0003bb70       ?DecideOnExoticBehavior@CVillagerAI@@AAE?B_NAAVCVillager@@@Z 0043cb70 f   VillagerAI.obj
 0001:0003bc00       ?DecideOnChiefBehavior@CVillagerAI@@AAE?B_NAAVCVillager@@@Z 0043cc00 f   VillagerAI.obj
 0001:0003bd80       ?DecideOnSickBehavior@CVillagerAI@@AAE?B_NAAVCVillager@@@Z 0043cd80 f   VillagerAI.obj
 0001:0003be00       ?AttemptSkill@CVillagerAI@@QAE?B_NAAVCVillager@@W4ESkill@@USSkillData@@@Z 0043ce00 f   VillagerAI.obj
 0001:0003c950       ?InitiatePredisposition@CVillagerAI@@AAE?B_NAAVCVillager@@@Z 0043d950 f   VillagerAI.obj
 0001:0003cfd0       ?InitiateChiefPredisposition@CVillagerAI@@AAE?B_NAAVCVillager@@@Z 0043dfd0 f   VillagerAI.obj
 0001:0003d2c0       ?InitiateWorkPlan@CVillagerAI@@QAE?B_NAAVCVillager@@W4ESkill@@@Z 0043e2c0 f   VillagerAI.obj
 0001:0003dce0       ?RealtimeWorkDone@CVillagerAI@@QAEXAAVCVillager@@@Z 0043ece0 f   VillagerAI.obj
 0001:0003de70       ?AdvanceState@CVillagerAI@@IAEXAAVCVillager@@H@Z 0043ee70 f   VillagerAI.obj
 0001:0003e870       ?DoBevMacInstantly@CVillagerAI@@QAEXAAVCVillager@@@Z 0043f870 f   VillagerAI.obj
 0001:0003ec90       ?AcquireTarget@CVillagerAI@@QAEXAAVCVillager@@HHW4ESpeed@@@Z 0043fc90 f   VillagerAI.obj
 0001:0003ece0       ?TakePosition@CVillagerAI@@QAEXAAVCVillager@@@Z 0043fce0 f   VillagerAI.obj
 0001:0003ee00       ?SetWhichTarget@CBehavior@@QAEXH@Z 0043fe00 f i VillagerAI.obj
 0001:0003ee20       ?IsTraineeOf@CVillagerSkills@@QBE?B_NW4ESkill@@@Z 0043fe20 f i VillagerAI.obj
 0001:0003ee40       ?SetNeedsPositioning@CBehavior@@QAEX_N@Z 0043fe40 f i VillagerAI.obj
 0001:0003ee60       ?IsIdling@CVillagerPlans@@QBE?B_NXZ 0043fe60 f i VillagerAI.obj
 0001:0003ee80       ?IsInexperiencedAt@CVillagerSkills@@QBE?B_NW4ESkill@@@Z 0043fe80 f i VillagerAI.obj
 0001:0003eea0       ?SetBusy@CVillager@@QAEX_N@Z 0043fea0 f i VillagerAI.obj
 0001:0003eec0       ?IsBusy@CVillager@@QBE?B_NXZ 0043fec0 f i VillagerAI.obj
 0001:0003eee0       ?IsAbundant@CFoodStore@@QBE?B_NXZ 0043fee0 f i VillagerAI.obj
 0001:0003ef00       ?EnoughHoneyToHarvest@CBeeHive@@QAE_NXZ 0043ff00 f i VillagerAI.obj
 0001:0003ef20       ?SetXVel@CVillager@@IAEXH@Z 0043ff20 f i VillagerAI.obj
 0001:0003ef40       ?SetYVel@CVillager@@IAEXH@Z 0043ff40 f i VillagerAI.obj
 0001:0003ef60       ??0CVillagerBio@@QAE@XZ    0043ff60 f   VillagerBio.obj
 0001:0003ef70       ?Copy@CVillagerBio@@QAEXAAV1@@Z 0043ff70 f   VillagerBio.obj
 0001:0003ef90       ?Reset@CVillagerBio@@QAEXXZ 0043ff90 f   VillagerBio.obj
 0001:0003f0d0       ?SetRandomName@CVillagerBio@@QAEXH@Z 004400d0 f   VillagerBio.obj
 0001:0003f250       ?IsOld@CVillagerBio@@QBE?B_NXZ 00440250 f   VillagerBio.obj
 0001:0003f280       ?IsNotOld@CVillagerBio@@QBE?B_NXZ 00440280 f   VillagerBio.obj
 0001:0003f2b0       ?IncrementAge@CVillagerBio@@QAEXH@Z 004402b0 f   VillagerBio.obj
 0001:0003f2f0       ??0CVillagerManager@@QAE@XZ 004402f0 f   VillagerManager.obj
 0001:0003f330       ?Reset@CVillagerManager@@QAEXXZ 00440330 f   VillagerManager.obj
 0001:0003f3c0       ?LoadAssets@CVillagerManager@@QAEXXZ 004403c0 f   VillagerManager.obj
 0001:0003f500       ?ReleaseAssets@CVillagerManager@@QAEXXZ 00440500 f   VillagerManager.obj
 0001:0003f510       ?GetVillager@CVillagerManager@@QAEAAVCVillager@@H@Z 00440510 f   VillagerManager.obj
 0001:0003f530       ?GetVillagerInFocus@CVillagerManager@@QAEPAVCVillager@@XZ 00440530 f   VillagerManager.obj
 0001:0003f590       ?GetChief@CVillagerManager@@QAEPAVCVillager@@XZ 00440590 f   VillagerManager.obj
 0001:0003f630       ?SaveState@CVillagerManager@@QAE?B_NAAUSSaveState@CVillager@@@Z 00440630 f   VillagerManager.obj
 0001:0003f6f0       ?LoadState@CVillagerManager@@QAE?B_NAAUSSaveState@CVillager@@@Z 004406f0 f   VillagerManager.obj
 0001:0003f790       ?Debug@CVillagerManager@@UAEXXZ 00440790 f   VillagerManager.obj
 0001:0003f890       ?InitStartingPositions@CVillagerManager@@QAEXXZ 00440890 f   VillagerManager.obj
 0001:0003f8d0       ?SpawnSpecificPeep@CVillagerManager@@QAE?BHHW4ESkill@@HW4EGender@@H@Z 004408d0 f   VillagerManager.obj
 0001:0003f910       ?SpawnSpecificPeep@CVillagerManager@@QAE?BHHW4ESkill@@HW4EGender@@HPBD2HHHH@Z 00440910 f   VillagerManager.obj
 0001:0003f960       ?SpawnSpecificPeep@CVillagerManager@@QAE?BHHW4ESkill@@HW4EGender@@HPBD2HHHHHH_N@Z 00440960 f   VillagerManager.obj
 0001:0003fa10       ?SpawnSpecificPeep@CVillagerManager@@QAE?BHAAVCVillager@@@Z 00440a10 f   VillagerManager.obj
 0001:0003fac0       ?SpawnSpecificPeep@CVillagerManager@@QAE?BHPAVCVillager@@@Z 00440ac0 f   VillagerManager.obj
 0001:0003fb40       ?IterateAllVillagers@CVillagerManager@@QAEXXZ 00440b40 f   VillagerManager.obj
 0001:0003fba0       ?AllVillagersTimeflowUpkeep@CVillagerManager@@QAEXXZ 00440ba0 f   VillagerManager.obj
 0001:00040170       ?AllVillagersRealtimePhysiologyAndProductivityUpkeep@CVillagerManager@@QAEXXZ 00441170 f   VillagerManager.obj
 0001:00040ec0       ?DrawVillagers@CVillagerManager@@QAEXXZ 00441ec0 f   VillagerManager.obj
 0001:00041060       ?DrawVillager@CVillagerManager@@QAEXH@Z 00442060 f   VillagerManager.obj
 0001:00041a10       ?DrawCarriedItems@CVillagerManager@@AAEXABVCVillager@@UldwPoint@@@Z 00442a10 f   VillagerManager.obj
 0001:00041b30       ?CheckForVillagerClick@CVillagerManager@@QAE?BHUldwPoint@@@Z 00442b30 f   VillagerManager.obj
 0001:00041c90       ?GetVillagerAt@CVillagerManager@@QAEPAVCVillager@@UldwPoint@@H_N@Z 00442c90 f   VillagerManager.obj
 0001:00041e10       ?GetVillagerWaitingAt@CVillagerManager@@QAEPAVCVillager@@UldwPoint@@PBV2@@Z 00442e10 f   VillagerManager.obj
 0001:00041f70       ?CheckForOtherWaitingVillagerAtPoint@CVillagerManager@@QAEPAVCVillager@@PBV2@UldwPoint@@@Z 00442f70 f   VillagerManager.obj
 0001:000420a0       ?HasAnyVillagerScaredBirds@CVillagerManager@@QAE?B_NXZ 004430a0 f   VillagerManager.obj
 0001:00042140       ?SelectChosenOne@CVillagerManager@@QAE?B_NXZ 00443140 f   VillagerManager.obj
 0001:000422d0       ?SetChief@CVillagerManager@@QAEXAAVCVillager@@@Z 004432d0 f   VillagerManager.obj
 0001:00042320       ?ChiefExists@CVillagerManager@@QAE?B_NXZ 00443320 f   VillagerManager.obj
 0001:00042340       ?ChiefPredisposition@CVillagerManager@@QAE?BHXZ 00443340 f   VillagerManager.obj
 0001:000423e0       ?ChanceOfChiefBoost@CVillagerManager@@QAE?B_NH@Z 004433e0 f   VillagerManager.obj
 0001:00042470       ?SetNoFocus@CVillagerManager@@QAEXXZ 00443470 f   VillagerManager.obj
 0001:000424e0       ?InvokeCelebration@CVillagerManager@@QAEXH@Z 004434e0 f   VillagerManager.obj
 0001:00042650       ?MakeInFocus@CVillagerManager@@QAEXH@Z 00443650 f   VillagerManager.obj
 0001:00042680       ?MakeInFocus@CVillagerManager@@QAEXPBVCVillager@@@Z 00443680 f   VillagerManager.obj
 0001:00042700       ?FindCorpse@CVillagerManager@@QAE?BHXZ 00443700 f   VillagerManager.obj
 0001:00042790       ?TakePositions@CVillagerManager@@QAEXXZ 00443790 f   VillagerManager.obj
 0001:00042820       ?SelectRandomLivingVillager@CVillagerManager@@QAE?BH_N@Z 00443820 f   VillagerManager.obj
 0001:00042900       ?SelectRandomLivingVillager@CVillagerManager@@QAE?BH_NH@Z 00443900 f   VillagerManager.obj
 0001:00042a00       ?SelectRandomLivingVillager@CVillagerManager@@QAE?BHHH@Z 00443a00 f   VillagerManager.obj
 0001:00042b00       ?SelectOtherAvailableMatingVillager@CVillagerManager@@QAE?BHAAVCVillager@@@Z 00443b00 f   VillagerManager.obj
 0001:00042d90       ?SelectPlayMateFor@CVillagerManager@@QAE?BHAAVCVillager@@@Z 00443d90 f   VillagerManager.obj
 0001:00042ea0       ?SelectOtherSickVillager@CVillagerManager@@QAE?BHAAVCVillager@@@Z 00443ea0 f   VillagerManager.obj
 0001:00042fd0       ?SelectRandomLivingChild@CVillagerManager@@QAE?BHXZ 00443fd0 f   VillagerManager.obj
 0001:000430a0       ?GetRandomVillager@CVillagerManager@@QAEPAVCVillager@@W4EAgeSelecter@@W4EGender@@_NPAH@Z 004440a0 f   VillagerManager.obj
 0001:000432a0       ?MakeRandomVillagersSick@CVillagerManager@@QAEXH_NH@Z 004442a0 f   VillagerManager.obj
 0001:000433c0       ?CureAllVillagers@CVillagerManager@@QAEXXZ 004443c0 f   VillagerManager.obj
 0001:00043460       ?MakeAllVillagersForgetWhatToDo@CVillagerManager@@QAEX_N@Z 00444460 f   VillagerManager.obj
 0001:00043500       ?MakeRandomVillagersInjured@CVillagerManager@@QAEXHHH@Z 00444500 f   VillagerManager.obj
 0001:00043600       ?MakeRandomVillagersDead@CVillagerManager@@QAEXHW4EGender@@@Z 00444600 f   VillagerManager.obj
 0001:00043700       ?MakeRandomVillagersVanish@CVillagerManager@@QAEXHW4EGender@@@Z 00444700 f   VillagerManager.obj
 0001:000437f0       ?AddRandomVillagerLike@CVillagerManager@@QAEXHW4ELike@@@Z 004447f0 f   VillagerManager.obj
 0001:00043880       ?AddRandomVillagerDislike@CVillagerManager@@QAEXHW4ELike@@@Z 00444880 f   VillagerManager.obj
 0001:00043910       ?RandomSkillPenalty@CVillagerManager@@QAEXPAVCVillager@@HH@Z 00444910 f   VillagerManager.obj
 0001:000439d0       ?RandomSkillBonus@CVillagerManager@@QAEXPAVCVillager@@HH@Z 004449d0 f   VillagerManager.obj
 0001:00043a90       ?ImproveRandomVillagersSkill@CVillagerManager@@QAEXHW4ESkill@@HH_N@Z 00444a90 f   VillagerManager.obj
 0001:00043b80       ?MakeSomeVillagersDo@CVillagerManager@@QAEXW4EBehavior@@HW4EAgeSelecter@@W4EGender@@_N@Z 00444b80 f   VillagerManager.obj
 0001:00043d90       ?ChangeRandomVillagersClothes@CVillagerManager@@QAEXH_N@Z 00444d90 f   VillagerManager.obj
 0001:00043ed0       ?MakeAllVillagersDo@CVillagerManager@@QAEXW4EBehavior@@W4EAgeSelecter@@W4EGender@@_NPAH@Z 00444ed0 f   VillagerManager.obj
 0001:00044120       ?MakeAllVillagersDo@CVillagerManager@@QAEXW4EBehavior@@W4EAgeSelecter@@W4EGender@@_N@Z 00445120 f   VillagerManager.obj
 0001:00044150       ?MakeAllVillagersDo@CVillagerManager@@QAEXW4EBehavior@@HW4EGender@@_NPAH@Z 00445150 f   VillagerManager.obj
 0001:000443d0       ?MakeAllVillagersDo@CVillagerManager@@QAEXW4EBehavior@@HW4EGender@@_N@Z 004453d0 f   VillagerManager.obj
 0001:00044400       ?TeleportAllVillagersTo@CVillagerManager@@QAEXHHW4EAgeSelecter@@W4EGender@@_N@Z 00445400 f   VillagerManager.obj
 0001:00044430       ?TeleportAllVillagersTo@CVillagerManager@@QAEXHHW4EAgeSelecter@@W4EGender@@_NPAH@Z 00445430 f   VillagerManager.obj
 0001:00044630       ?TeleportAllVillagersTo@CVillagerManager@@QAEXHHHHW4EAgeSelecter@@W4EGender@@_NPAH@Z 00445630 f   VillagerManager.obj
 0001:00044850       ?GetRandomVillagerWithSkill@CVillagerManager@@QAEPAVCVillager@@W4ESkill@@HW4EAgeSelecter@@W4EGender@@_NPAH@Z 00445850 f   VillagerManager.obj
 0001:00044a20       ?ExtremeLimitGenderCorrect@CVillagerManager@@QAE?BW4EGender@@XZ 00445a20 f   VillagerManager.obj
 0001:00044a70       ?IsRoomToPopulate@CVillagerManager@@QAE?B_NXZ 00445a70 f   VillagerManager.obj
 0001:00044bf0       ?Population@CVillagerManager@@QAE?BHXZ 00445bf0 f   VillagerManager.obj
 0001:00044cb0       ?Totems@CVillagerManager@@QAE?BHXZ 00445cb0 f   VillagerManager.obj
 0001:00044d30       ?GenderCounts@CVillagerManager@@QAE?BHAAH0@Z 00445d30 f   VillagerManager.obj
 0001:00044e00       ?MothersCaringForBabies@CVillagerManager@@QAE?BHXZ 00445e00 f   VillagerManager.obj
 0001:00044ec0       ?GatherChildrenForStory@CVillagerManager@@QAEXXZ 00445ec0 f   VillagerManager.obj
 0001:00044fd0       ?IsAnyoneCarrying@CVillagerManager@@QBE?B_NW4ECarrying@@@Z 00445fd0 f   VillagerManager.obj
 0001:00045040       ?ChangeAllBehavior@CVillagerManager@@QAEXW4EBehavior@@0@Z 00446040 f   VillagerManager.obj
 0001:00045160       ?GetVillagerDoing@CVillagerManager@@QAEPAVCVillager@@W4EBehavior@@@Z 00446160 f   VillagerManager.obj
 0001:00045190       ?GetVillagerDoing@CVillagerManager@@QAEPAVCVillager@@W4EBehavior@@_NPAH@Z 00446190 f   VillagerManager.obj
 0001:000452e0       ?VillagerExists@CVillagerManager@@QAE_NH@Z 004462e0 f   VillagerManager.obj
 0001:00045320       ??0IDebugger@@QAE@XZ       00446320 f i VillagerManager.obj
 0001:00045340       ?FatherSkillType@CVillagerBio@@QBE?BW4ESkill@@XZ 00446340 f i VillagerManager.obj
 0001:00045360       ?FatherSkillValue@CVillagerBio@@QBE?BHXZ 00446360 f i VillagerManager.obj
 0001:00045380       ?HusbandName@CVillagerBio@@QBEPBDXZ 00446380 f i VillagerManager.obj
 0001:000453a0       ?HusbandBodyType@CVillagerBio@@QBE?BHXZ 004463a0 f i VillagerManager.obj
 0001:000453c0       ?HusbandHeadType@CVillagerBio@@QBE?BHXZ 004463c0 f i VillagerManager.obj
 0001:000453e0       ?IsAlive@CVillagerState@@QBE?B_NXZ 004463e0 f i VillagerManager.obj
 0001:00045400       ?IncrementSecondsAccumulated@CVillagerState@@QAEXK@Z 00446400 f i VillagerManager.obj
 0001:00045420       ?Scale@CSceneManager@@QBE?BMXZ 00446420 f i VillagerManager.obj
 0001:00045440       ?IsWaiting@CVillagerPlans@@QBE?B_NXZ 00446440 f i VillagerManager.obj
 0001:00045460       ?TotemX@CVillagerState@@QBE?BHXZ 00446460 f i Villager.obj
 0001:00045460       ?HeadType@CVillagerBio@@QBE?BHXZ 00446460 f i Villager.obj
 0001:00045460       ?NextAction@CVillagerPlans@@QBE?BW4EAction@@XZ 00446460 f i VillagerManager.obj
 0001:00045480       ?IsChosenOne@CVillagerState@@QBE?B_NXZ 00446480 f i VillagerManager.obj
 0001:000454a0       ?SetExists@CVillager@@QAEX_N@Z 004464a0 f i VillagerManager.obj
 0001:000454c0       ?RemoveDislike@CVillager@@QAEXW4ELike@@@Z 004464c0 f i VillagerManager.obj
 0001:000454e0       ?SetRef@CVillager@@QAEXH@Z 004464e0 f i VillagerManager.obj
 0001:00045500       ?SetFocus@CVillager@@QAEX_N@Z 00446500 f i VillagerManager.obj
 0001:00045520       ?IsInHand@CVillager@@QBE?B_NXZ 00446520 f i VillagerManager.obj
 0001:00045540       ?SetInHand@CVillager@@QAEX_N@Z 00446540 f i VillagerManager.obj
 0001:00045560       ??0SEventData@@QAE@H_N@Z   00446560 f i VillagerManager.obj
 0001:00045590       ?AnimFrame@CVillager@@QBE?BW4EAnimFrame@@XZ 00446590 f i VillagerManager.obj
 0001:000455b0       ?DisplacementFrame@CVillager@@QBE?BHXZ 004465b0 f i VillagerManager.obj
 0001:000455d0       ?ScenePriority@CVillager@@QAE?BW4EScenePriority@@XZ 004465d0 f i VillagerManager.obj
 0001:000455f0       ?Direction@CVillager@@QBE?BW4EDirection@@XZ 004465f0 f i VillagerManager.obj
 0001:00045610       ?HeadDirection@CVillager@@QBE?BW4EHeadDirection@@XZ 00446610 f i VillagerManager.obj
 0001:00045630       ?BodyPosition@CVillager@@QBE?BW4EBodyPosition@@XZ 00446630 f i VillagerManager.obj
 0001:00045650       ?IsNotElderly@CVillagerBio@@QBE?B_NXZ 00446650 f i VillagerManager.obj
 0001:00045670       ?SetPregnancyStartTime@CVillagerState@@QAEXH@Z 00446670 f i Villager.obj
 0001:00045670       ?SetOldestVillager@CGameStats@@QAEXH@Z 00446670 f i VillagerManager.obj
 0001:00045690       ?OldestVillager@CGameStats@@QBE?BHXZ 00446690 f i VillagerManager.obj
 0001:00045690       ?PregnancyStartTime@CVillagerState@@QBE?BHXZ 00446690 f i VillagerManager.obj
 0001:000456b0       ?AddLike@CVillager@@QAEXW4ELike@@@Z 004466b0 f i VillagerManager.obj
 0001:000456f0       ?IsInView@CWorldView@@QBE?B_NUldwPoint@@@Z 004466f0 f i VillagerManager.obj
 0001:00045750       ?AddDislike@CVillager@@QAEXW4ELike@@@Z 00446750 f i VillagerManager.obj
 0001:00045790       ?SetXPos@CVillager@@QAEXH@Z 00446790 f i VillagerManager.obj
 0001:000457b0       ?SetYPos@CVillager@@QAEXH@Z 004467b0 f i VillagerManager.obj
 0001:000457d0       ?AddPlan@CVillagerPlans@@AAEXUSActionPlan@1@W4EPriority@@@Z 004467d0 f   VillagerPlans.obj
 0001:00045870       ?AdvanceCurrentPlan@CVillagerPlans@@QAEXAAVCVillager@@@Z 00446870 f   VillagerPlans.obj
 0001:000458e0       ?NextPlan@CVillagerPlans@@QAEXAAVCVillager@@_N@Z 004468e0 f   VillagerPlans.obj
 0001:00045970       ?ForgetPlans@CVillagerPlans@@QAEXAAVCVillager@@@Z 00446970 f   VillagerPlans.obj
 0001:00045a10       ?StartNewBehavior@CVillagerPlans@@QAEXAAVCVillager@@@Z 00446a10 f   VillagerPlans.obj
 0001:00045e80       ?ProcessCurrentPlan@CVillagerPlans@@QAEXAAVCVillager@@@Z 00446e80 f   VillagerPlans.obj
 0001:00046350       ?PlanToWander@CVillagerPlans@@QAEXHW4ESpeed@@@Z 00447350 f   VillagerPlans.obj
 0001:000463a0       ?PlanToWait@CVillagerPlans@@QAEXHW4EBodyPosition@@W4EDirection@@W4EHeadDirection@@@Z 004473a0 f   VillagerPlans.obj
 0001:00046400       ?PlanToWait@CVillagerPlans@@QAEXHW4EBodyPosition@@W4EHeadDirection@@@Z 00447400 f   VillagerPlans.obj
 0001:00046460       ?PlanToWait@CVillagerPlans@@QAEXHW4EBodyPosition@@@Z 00447460 f   VillagerPlans.obj
 0001:000464c0       ?PlanToGo@CVillagerPlans@@QAEXW4EObject@CContentMap@@W4ESpeed@@W4EPriority@@@Z 004474c0 f   VillagerPlans.obj
 0001:00046530       ?PlanToGo@CVillagerPlans@@QAEXW4EWaypoint@@W4ESpeed@@W4EPriority@@@Z 00447530 f   VillagerPlans.obj
 0001:000465a0       ?PlanToGo@CVillagerPlans@@QAEXW4EWaypoint@@UldwPoint@@W4ESpeed@@W4EPriority@@@Z 004475a0 f   VillagerPlans.obj
 0001:00046610       ?PlanToGo@CVillagerPlans@@QAEXUldwPoint@@W4ESpeed@@W4EPriority@@@Z 00447610 f   VillagerPlans.obj
 0001:00046660       ?PlanToGo@CVillagerPlans@@QAEXHHW4ESpeed@@W4EPriority@@@Z 00447660 f   VillagerPlans.obj
 0001:000466b0       ?PlanToSwim@CVillagerPlans@@QAEXH_N@Z 004476b0 f   VillagerPlans.obj
 0001:00046700       ?PlanToDance@CVillagerPlans@@QAEXH@Z 00447700 f   VillagerPlans.obj
 0001:00046750       ?PlanToLearn@CVillagerPlans@@QAEXW4ESkill@@@Z 00447750 f   VillagerPlans.obj
 0001:000467a0       ?PlanToWork@CVillagerPlans@@QAEXH@Z 004477a0 f   VillagerPlans.obj
 0001:000467f0       ?PlanToClimb@CVillagerPlans@@QAEXH@Z 004477f0 f   VillagerPlans.obj
 0001:00046840       ?PlanToDive@CVillagerPlans@@QAEXW4EAnim@@HW4EDirection@@H@Z 00447840 f   VillagerPlans.obj
 0001:000468a0       ?PlanToJump@CVillagerPlans@@QAEXH@Z 004478a0 f   VillagerPlans.obj
 0001:000468f0       ?PlanToBend@CVillagerPlans@@QAEXH@Z 004478f0 f   VillagerPlans.obj
 0001:00046940       ?PlanToCheer@CVillagerPlans@@QAEXH@Z 00447940 f   VillagerPlans.obj
 0001:00046990       ?PlanToTwirlCW@CVillagerPlans@@QAEXH@Z 00447990 f   VillagerPlans.obj
 0001:000469e0       ?PlanToTwirlCCW@CVillagerPlans@@QAEXH@Z 004479e0 f   VillagerPlans.obj
 0001:00046a30       ?PlanToDisco@CVillagerPlans@@QAEXH@Z 00447a30 f   VillagerPlans.obj
 0001:00046a80       ?PlanToDoTheMonkey@CVillagerPlans@@QAEXH@Z 00447a80 f   VillagerPlans.obj
 0001:00046ad0       ?PlanToRevel@CVillagerPlans@@QAEXH@Z 00447ad0 f   VillagerPlans.obj
 0001:00046b20       ?PlanToLieDown@CVillagerPlans@@QAEXH@Z 00447b20 f   VillagerPlans.obj
 0001:00046b70       ?PlanToScrub@CVillagerPlans@@QAEXH@Z 00447b70 f   VillagerPlans.obj
 0001:00046bc0       ?PlanToExorcist@CVillagerPlans@@QAEXH@Z 00447bc0 f   VillagerPlans.obj
 0001:00046c10       ?PlanToJoyTwirlCW@CVillagerPlans@@QAEXH@Z 00447c10 f   VillagerPlans.obj
 0001:00046c60       ?PlanToDoPushups@CVillagerPlans@@QAEXH@Z 00447c60 f   VillagerPlans.obj
 0001:00046cb0       ?PlanToEmbrace@CVillagerPlans@@QAEXXZ 00447cb0 f   VillagerPlans.obj
 0001:00046cf0       ?PlanToHide@CVillagerPlans@@QAEXH@Z 00447cf0 f   VillagerPlans.obj
 0001:00046d40       ?PlanToCarry@CVillagerPlans@@QAEXW4ECarrying@@@Z 00447d40 f   VillagerPlans.obj
 0001:00046d90       ?PlanToDrop@CVillagerPlans@@QAEXXZ 00447d90 f   VillagerPlans.obj
 0001:00046dd0       ?PlanToAdvanceState@CVillagerPlans@@QAEXW4EWorldState@@@Z 00447dd0 f   VillagerPlans.obj
 0001:00046e20       ?PlanToSpawnAnim@CVillagerPlans@@QAEXW4EFloatingAnim@@HH@Z 00447e20 f   VillagerPlans.obj
 0001:00046e70       ?PlanToSpawnAnimAtVillager@CVillagerPlans@@QAEXW4EFloatingAnim@@HH@Z 00447e70 f   VillagerPlans.obj
 0001:00046ec0       ?PlanToSpawnRareCollectible@CVillagerPlans@@QAEXXZ 00447ec0 f   VillagerPlans.obj
 0001:00046f00       ?PlanToAdvancePuzzle@CVillagerPlans@@QAEXW4EPuzzle@@H@Z 00447f00 f   VillagerPlans.obj
 0001:00046f50       ?PlanToResetPuzzle@CVillagerPlans@@QAEXW4EPuzzle@@@Z 00447f50 f   VillagerPlans.obj
 0001:00046fa0       ?PlanToShakeHead@CVillagerPlans@@QAEXHW4EBodyPosition@@@Z 00447fa0 f   VillagerPlans.obj
 0001:00046ff0       ?PlanToHeal@CVillagerPlans@@QAEXW4EPriority@@@Z 00447ff0 f   VillagerPlans.obj
 0001:00047030       ?PlanToPlaySound@CVillagerPlans@@QAEXW4ESound@@MW4ESoundType@@@Z 00448030 f   VillagerPlans.obj
 0001:00047080       ?PlanToStopSound@CVillagerPlans@@QAEXXZ 00448080 f   VillagerPlans.obj
 0001:000470c0       ?PlanToTakeCorpse@CVillagerPlans@@QAEXH@Z 004480c0 f   VillagerPlans.obj
 0001:00047100       ?PlanToSay@CVillagerPlans@@QAEXW4StringId@@@Z 00448100 f   VillagerPlans.obj
 0001:00047150       ?PlanToFollowPath@CVillagerPlans@@QAEXHHW4ESpeed@@@Z 00448150 f   VillagerPlans.obj
 0001:000471a0       ?PlanToPlayAnim@CVillagerPlans@@QAEXHW4EAnim@@_NM@Z 004481a0 f   VillagerPlans.obj
 0001:00047200       ?PlanNewBehavior@CVillagerPlans@@QAEXW4EBehavior@@ABUSBehaviorData@@@Z 00448200 f   VillagerPlans.obj
 0001:00047260       ?HasCurrentPlanExpired@CVillagerPlans@@QBE?B_NXZ 00448260 f   VillagerPlans.obj
 0001:000472a0       ?Get@CWaypoint@@QBE?BUldwPoint@@W4EWaypoint@@@Z 004482a0 f i VillagerPlans.obj
 0001:000472d0       ??0CVillagerSkills@@QAE@XZ 004482d0 f   VillagerSkills.obj
 0001:000472e0       ?Copy@CVillagerSkills@@QAEXAAV1@@Z 004482e0 f   VillagerSkills.obj
 0001:00047320       ?Reset@CVillagerSkills@@QAEXXZ 00448320 f   VillagerSkills.obj
 0001:00047360       ?Update@CVillagerSkills@@QAEXAAVCVillager@@@Z 00448360 f   VillagerSkills.obj
 0001:00047420       ?BestSkill@CVillagerSkills@@QBE?BW4ESkill@@PAH@Z 00448420 f   VillagerSkills.obj
 0001:00047490       ?IsEsteemedElder@CVillagerSkills@@QBE?B_NXZ 00448490 f   VillagerSkills.obj
 0001:00047530       ?TotalSkill@CVillagerSkills@@QBE?BHXZ 00448530 f   VillagerSkills.obj
 0001:00047570       ?SkillsMastered@CVillagerSkills@@QBE?BHXZ 00448570 f   VillagerSkills.obj
 0001:000475c0       ?IsMasterOfAny@CVillagerSkills@@QBE?B_NXZ 004485c0 f   VillagerSkills.obj
 0001:00047600       ??0CVillagerState@@QAE@XZ  00448600 f   VillagerState.obj
 0001:00047610       ?Copy@CVillagerState@@QAEXAAV1@@Z 00448610 f   VillagerState.obj
 0001:00047630       ?Reset@CVillagerState@@QAEXH@Z 00448630 f   VillagerState.obj
 0001:000476e0       ?Update@CVillagerState@@QAEXAAVCVillager@@@Z 004486e0 f   VillagerState.obj
 0001:00047720       ?SetHealth@CVillagerState@@QAEXHW4ECauseOfDeath@@@Z 00448720 f   VillagerState.obj
 0001:00047780       ?AdjustHealth@CVillagerState@@QAEXHW4ECauseOfDeath@@@Z 00448780 f   VillagerState.obj
 0001:000477e0       ??0CCollectionScene@@AAE@XZ 004487e0 f   CollectionScene.obj
 0001:00048220       ??1CCollectionScene@@EAE@XZ 00449220 f   CollectionScene.obj
 0001:00048410       ?Get@CCollectionScene@@SAPAV1@XZ 00449410 f   CollectionScene.obj
 0001:00048490       ?Ref@CCollectionScene@@SAAAV1@XZ 00449490 f   CollectionScene.obj
 0001:00048510       ?Destroy@CCollectionScene@@SAXXZ 00449510 f   CollectionScene.obj
 0001:00048550       ?Activate@CCollectionScene@@MAEX_N@Z 00449550 f   CollectionScene.obj
 0001:00048700       ?UpdateScene@CCollectionScene@@MAEXXZ 00449700 f   CollectionScene.obj
 0001:00048740       ?DrawScene@CCollectionScene@@MAEXXZ 00449740 f   CollectionScene.obj
 0001:00048890       ?HandleKey@CCollectionScene@@UAE_NHHH@Z 00449890 f   CollectionScene.obj
 0001:000488e0       ?HandleMouse@CCollectionScene@@UAE_NHUldwPoint@@@Z 004498e0 f   CollectionScene.obj
 0001:00048b40       ?HandleMessage@CCollectionScene@@UAE_NHJ@Z 00449b40 f   CollectionScene.obj
 0001:00048b90       ??_ECCollectionScene@@EAEPAXI@Z 00449b90 f i CollectionScene.obj
 0001:00048b90       ??_GCCollectionScene@@EAEPAXI@Z 00449b90 f i CollectionScene.obj
 0001:00048bc0       ?SetCurrentGameScene@theGameState@@QAEXW4EGameScene@@@Z 00449bc0 f i CollectionScene.obj
 0001:00048be0       ??0CProgressScene@@AAE@XZ  00449be0 f   ProgressScene.obj
 0001:00049610       ??1CProgressScene@@EAE@XZ  0044a610 f   ProgressScene.obj
 0001:00049950       ?Get@CProgressScene@@SAPAV1@XZ 0044a950 f   ProgressScene.obj
 0001:000499d0       ?Ref@CProgressScene@@SAAAV1@XZ 0044a9d0 f   ProgressScene.obj
 0001:00049a50       ?Destroy@CProgressScene@@SAXXZ 0044aa50 f   ProgressScene.obj
 0001:00049a90       ?Activate@CProgressScene@@MAEX_N@Z 0044aa90 f   ProgressScene.obj
 0001:00049ab0       ?UpdateScene@CProgressScene@@MAEXXZ 0044aab0 f   ProgressScene.obj
 0001:00049ae0       ?DrawScene@CProgressScene@@MAEXXZ 0044aae0 f   ProgressScene.obj
 0001:00049c60       ?DrawSceneFinal@CProgressScene@@MAEXXZ 0044ac60 f   ProgressScene.obj
 0001:00049c70       ?DrawPuzzleIcons@CProgressScene@@ABEX_N@Z 0044ac70 f   ProgressScene.obj
 0001:00049d40       ?RefreshTab@CProgressScene@@AAEXXZ 0044ad40 f   ProgressScene.obj
 0001:00049fb0       ?RefreshGlobalStats@CProgressScene@@AAEXXZ 0044afb0 f   ProgressScene.obj
 0001:0004a0c0       ?HandleKey@CProgressScene@@UAE_NHHH@Z 0044b0c0 f   ProgressScene.obj
 0001:0004a110       ?HandleMouse@CProgressScene@@UAE_NHUldwPoint@@@Z 0044b110 f   ProgressScene.obj
 0001:0004a3b0       ?HandleMessage@CProgressScene@@UAE_NHJ@Z 0044b3b0 f   ProgressScene.obj
 0001:0004a440       ??_ECProgressScene@@EAEPAXI@Z 0044b440 f i ProgressScene.obj
 0001:0004a440       ??_GCProgressScene@@EAEPAXI@Z 0044b440 f i ProgressScene.obj
 0001:0004a470       ?GlobalRankings@CGameStats@@QBEABUSGameStats@1@XZ 0044b470 f i ProgressScene.obj
 0001:0004a490       ??0CStoryScene@@AAE@XZ     0044b490 f   StoryScene.obj
 0001:0004a750       ??1CStoryScene@@EAE@XZ     0044b750 f   StoryScene.obj
 0001:0004a830       ?Get@CStoryScene@@SAPAV1@XZ 0044b830 f   StoryScene.obj
 0001:0004a8b0       ?Ref@CStoryScene@@SAAAV1@XZ 0044b8b0 f   StoryScene.obj
 0001:0004a930       ?Destroy@CStoryScene@@SAXXZ 0044b930 f   StoryScene.obj
 0001:0004a970       ?Activate@CStoryScene@@UAEX_N@Z 0044b970 f   StoryScene.obj
 0001:0004aa20       ?DrawScene@CStoryScene@@UAEXXZ 0044ba20 f   StoryScene.obj
 0001:0004aa40       ?UpdateScene@CStoryScene@@UAEXXZ 0044ba40 f   StoryScene.obj
 0001:0004aa60       ?HandleMessage@CStoryScene@@UAE_NHJ@Z 0044ba60 f   StoryScene.obj
 0001:0004ab80       ?HandleMouse@CStoryScene@@UAE_NHUldwPoint@@@Z 0044bb80 f   StoryScene.obj
 0001:0004abb0       ?AddTutorialTipButtons@CStoryScene@@QAEXXZ 0044bbb0 f   StoryScene.obj
 0001:0004abf0       ?RemoveSkipButton@CStoryScene@@QAEXXZ 0044bbf0 f   StoryScene.obj
 0001:0004ac10       ?DisplayClickLabel@CStoryScene@@QAEXXZ 0044bc10 f   StoryScene.obj
 0001:0004ac30       ?RemoveClickLabel@CStoryScene@@QAEXXZ 0044bc30 f   StoryScene.obj
 0001:0004ac50       ??_ECStoryScene@@EAEPAXI@Z 0044bc50 f i StoryScene.obj
 0001:0004ac50       ??_GCStoryScene@@EAEPAXI@Z 0044bc50 f i StoryScene.obj
 0001:0004ac80       ?Story@CStory@@QBE?BW4EStory@1@XZ 0044bc80 f i StoryScene.obj
 0001:0004aca0       ??0CTechScene@@AAE@XZ      0044bca0 f   TechScene.obj
 0001:0004b5f0       ??1CTechScene@@EAE@XZ      0044c5f0 f   TechScene.obj
 0001:0004b790       ?Get@CTechScene@@SAPAV1@XZ 0044c790 f   TechScene.obj
 0001:0004b810       ?Ref@CTechScene@@SAAAV1@XZ 0044c810 f   TechScene.obj
 0001:0004b890       ?Destroy@CTechScene@@SAXXZ 0044c890 f   TechScene.obj
 0001:0004b8d0       ?Activate@CTechScene@@MAEX_N@Z 0044c8d0 f   TechScene.obj
 0001:0004b9f0       ?UpdateScene@CTechScene@@MAEXXZ 0044c9f0 f   TechScene.obj
 0001:0004bb70       ?DrawScene@CTechScene@@MAEXXZ 0044cb70 f   TechScene.obj
 0001:0004bf00       ?ShowTechInfo@CTechScene@@AAEXW4ETech@@@Z 0044cf00 f   TechScene.obj
 0001:0004c060       ?HandleKey@CTechScene@@UAE_NHHH@Z 0044d060 f   TechScene.obj
 0001:0004c0b0       ?HandleMouse@CTechScene@@UAE_NHUldwPoint@@@Z 0044d0b0 f   TechScene.obj
 0001:0004c2d0       ?HandleMessage@CTechScene@@UAE_NHJ@Z 0044d2d0 f   TechScene.obj
 0001:0004c550       ??_ECTechScene@@EAEPAXI@Z  0044d550 f i TechScene.obj
 0001:0004c550       ??_GCTechScene@@EAEPAXI@Z  0044d550 f i TechScene.obj
 0001:0004c580       ?RandomChance@@YA?B_NH@Z   0044d580 f i TechScene.obj
 0001:0004c5a0       ??0theHelpScene@@QAE@XZ    0044d5a0 f   theHelpScene.obj
 0001:0004c950       ??1theHelpScene@@UAE@XZ    0044d950 f   theHelpScene.obj
 0001:0004c9e0       ?UpdateScene@theHelpScene@@MAEXXZ 0044d9e0 f   theHelpScene.obj
 0001:0004caa0       ?DrawScene@theHelpScene@@MAEXXZ 0044daa0 f   theHelpScene.obj
 0001:0004cb70       ?ForwardWaitingMessage@theHelpScene@@QAE_NW4StringId@@@Z 0044db70 f   theHelpScene.obj
 0001:0004cb80       ?HandleKey@theHelpScene@@UAE_NHHH@Z 0044db80 f   theHelpScene.obj
 0001:0004cbc0       ?HandleMouse@theHelpScene@@UAE_NHUldwPoint@@@Z 0044dbc0 f   theHelpScene.obj
 0001:0004cbe0       ?HandleMessage@theHelpScene@@UAE_NHJ@Z 0044dbe0 f   theHelpScene.obj
 0001:0004cd40       ??_GtheHelpScene@@UAEPAXI@Z 0044dd40 f i theHelpScene.obj
 0001:0004cd40       ??_EtheHelpScene@@UAEPAXI@Z 0044dd40 f i theHelpScene.obj
 0001:0004cd70       ??0theLoadingScene@@QAE@XZ 0044dd70 f   theLoadingScene.obj
 0001:0004cf70       ??1theLoadingScene@@UAE@XZ 0044df70 f   theLoadingScene.obj
 0001:0004cfd0       ?SetMeter@theLoadingScene@@QAEXH@Z 0044dfd0 f   theLoadingScene.obj
 0001:0004cff0       ?UpdateScene@theLoadingScene@@MAEXXZ 0044dff0 f   theLoadingScene.obj
 0001:0004d080       ?SetTimer@theLoadingScene@@QAEXXZ 0044e080 f   theLoadingScene.obj
 0001:0004d0a0       ?DrawScene@theLoadingScene@@MAEXXZ 0044e0a0 f   theLoadingScene.obj
 0001:0004d170       ?HandleKey@theLoadingScene@@UAE_NHHH@Z 0044e170 f   theLoadingScene.obj
 0001:0004d180       ?HandleMouse@theLoadingScene@@UAE_NHUldwPoint@@@Z 0044e180 f   theLoadingScene.obj
 0001:0004d190       ?HandleMessage@theLoadingScene@@UAE_NHJ@Z 0044e190 f   theLoadingScene.obj
 0001:0004d1a0       ??_GtheLoadingScene@@UAEPAXI@Z 0044e1a0 f i theLoadingScene.obj
 0001:0004d1a0       ??_EtheLoadingScene@@UAEPAXI@Z 0044e1a0 f i theLoadingScene.obj
 0001:0004d1d0       ??0theMainScene@@AAE@XZ    0044e1d0 f   theMainScene.obj
 0001:0004e730       ??1theMainScene@@EAE@XZ    0044f730 f   theMainScene.obj
 0001:0004e7d0       ?Get@theMainScene@@SAPAV1@XZ 0044f7d0 f   theMainScene.obj
 0001:0004e850       ?Ref@theMainScene@@SAAAV1@XZ 0044f850 f   theMainScene.obj
 0001:0004e8d0       ?Destroy@theMainScene@@SAXXZ 0044f8d0 f   theMainScene.obj
 0001:0004e910       ?Activate@theMainScene@@MAEX_N@Z 0044f910 f   theMainScene.obj
 0001:0004ea70       ?UpdateScene@theMainScene@@MAEXXZ 0044fa70 f   theMainScene.obj
 0001:0004f750       ?Debug@theMainScene@@MAEXXZ 00450750 f   theMainScene.obj
 0001:0004f760       ?DrawScene@theMainScene@@MAEXXZ 00450760 f   theMainScene.obj
 0001:0004f8d0       ?DrawUI@theMainScene@@IAEXXZ 004508d0 f   theMainScene.obj
 0001:0004fe60       ?HandleKeyCharacter@theMainScene@@QAE?B_ND@Z 00450e60 f   theMainScene.obj
 0001:00050270       ?HandleKeyDown@theMainScene@@QAE?B_NH@Z 00451270 f   theMainScene.obj
 0001:00050310       ?HandleKeyUp@theMainScene@@QAE?B_NH@Z 00451310 f   theMainScene.obj
 0001:00050320       ?HandleMouseDown@theMainScene@@QAE?B_NUldwPoint@@@Z 00451320 f   theMainScene.obj
 0001:00050660       ?HandleMouseUp@theMainScene@@QAE?B_NUldwPoint@@@Z 00451660 f   theMainScene.obj
 0001:000506d0       ?HandleMouseMove@theMainScene@@QAE?B_NUldwPoint@@@Z 004516d0 f   theMainScene.obj
 0001:00050c80       ?HandleKey@theMainScene@@UAE_NHHH@Z 00451c80 f   theMainScene.obj
 0001:00050cf0       ?HandleMouse@theMainScene@@UAE_NHUldwPoint@@@Z 00451cf0 f   theMainScene.obj
 0001:00050d90       ?HandleMessage@theMainScene@@UAE_NHJ@Z 00451d90 f   theMainScene.obj
 0001:00050e80       ?HandleMenuButton@theMainScene@@QAEXXZ 00451e80 f   theMainScene.obj
 0001:00050ee0       ?HandleVillagerDetailsButton@theMainScene@@QAEXXZ 00451ee0 f   theMainScene.obj
 0001:000510c0       ?HandleTechButton@theMainScene@@QAEXXZ 004520c0 f   theMainScene.obj
 0001:00051140       ?HandleOverviewButton@theMainScene@@QAEXXZ 00452140 f   theMainScene.obj
 0001:000511e0       ?HandleCollectionButton@theMainScene@@QAEXXZ 004521e0 f   theMainScene.obj
 0001:00051260       ?HandlePuzzlesButton@theMainScene@@QAEXXZ 00452260 f   theMainScene.obj
 0001:000512e0       ?HandleLastTipButton@theMainScene@@QAEXXZ 004522e0 f   theMainScene.obj
 0001:00051320       ?HandleMapClick@theMainScene@@QAEXUldwPoint@@@Z 00452320 f   theMainScene.obj
 0001:000513d0       ?HandleDropOnHotSpot@theMainScene@@QAE?B_NAAVCVillager@@@Z 004523d0 f   theMainScene.obj
 0001:00051530       ?HandleDropOnVillager@theMainScene@@QAEXAAVCVillager@@@Z 00452530 f   theMainScene.obj
 0001:000518a0       ?DropVillager@theMainScene@@QAEXXZ 004528a0 f   theMainScene.obj
 0001:00051c50       ?MapClickFeedback@theMainScene@@QAEXUldwPoint@@@Z 00452c50 f   theMainScene.obj
 0001:000525f0       ?SayCurrentContent@theMainScene@@QAEXUldwPoint@@@Z 004535f0 f   theMainScene.obj
 0001:000537b0       ??_EtheMainScene@@EAEPAXI@Z 004547b0 f i theMainScene.obj
 0001:000537b0       ??_GtheMainScene@@EAEPAXI@Z 004547b0 f i theMainScene.obj
 0001:000537e0       ?IsTraineeLevel@CVillagerSkills@@QBE?B_NH@Z 004547e0 f i theMainScene.obj
 0001:00053800       ?IsAdeptLevel@CVillagerSkills@@QBE?B_NH@Z 00454800 f i theMainScene.obj
 0001:00053820       ?IsMasterLevel@CVillagerSkills@@QBE?B_NH@Z 00454820 f i theMainScene.obj
 0001:00053840       ?BehaviorLabel@CVillager@@QBEPBDXZ 00454840 f i theMainScene.obj
 0001:00053860       ?SetPos@CVillager@@QAEXUldwPoint@@@Z 00454860 f i theMainScene.obj
 0001:00053890       ?IncrementCrisis@CGameStats@@QAEXH@Z 00454890 f i theMainScene.obj
 0001:000538b0       ?Babies@CVillagerState@@QBE?BHXZ 004548b0 f i Villager.obj
 0001:000538b0       ?Crisis@CGameStats@@QBE?BHXZ 004548b0 f i theMainScene.obj
 0001:000538b0       ?GetFont@ldwGameWindowImpl@@QAEPAVldwFont@@XZ 004548b0 f i ldwGameWindow.obj
 0001:000538d0       ?GetVillagerPosition@CVillagerManager@@QAE?BUldwPoint@@H@Z 004548d0 f i theMainScene.obj
 0001:00053920       ?Rect@CWorldView@@QBE?BUldwRect@@XZ 00454920 f i theMainScene.obj
 0001:00053960       ?ContainsKindling@CFirePit@@QBE?B_NXZ 00454960 f i HotSpot.obj
 0001:00053960       ?IsFastScrolling@CWorldView@@QBE?B_NXZ 00454960 f i theMainScene.obj
 0001:00053980       ?Honey@CBeeHive@@QAEHXZ    00454980 f i theMainScene.obj
 0001:00053980       ?VillagersCured@CGameStats@@QBE?BHXZ 00454980 f i Villager.obj
 0001:00053980       ?CauseOfDeath@CVillagerState@@QBE?BW4ECauseOfDeath@@XZ 00454980 f i Graveyard.obj
 0001:000539a0       ?IsRepaired@CPrincessStatue@@QBE?B_NXZ 004549a0 f i theMainScene.obj
 0001:000539c0       ??0theMenuScene@@QAE@XZ    004549c0 f   theMenuScene.obj
 0001:00054b90       ??1theMenuScene@@UAE@XZ    00455b90 f   theMenuScene.obj
 0001:00054c70       ?Activate@theMenuScene@@MAEX_N@Z 00455c70 f   theMenuScene.obj
 0001:00054cb0       ?UpdateScene@theMenuScene@@MAEXXZ 00455cb0 f   theMenuScene.obj
 0001:00055080       ?DrawScene@theMenuScene@@MAEXXZ 00456080 f   theMenuScene.obj
 0001:000550f0       ?DrawSceneFinal@theMenuScene@@MAEXXZ 004560f0 f   theMenuScene.obj
 0001:00055160       ?HandleKey@theMenuScene@@UAE_NHHH@Z 00456160 f   theMenuScene.obj
 0001:00055170       ?HandleMouse@theMenuScene@@UAE_NHUldwPoint@@@Z 00456170 f   theMenuScene.obj
 0001:000553e0       ?HandleMessage@theMenuScene@@UAE_NHJ@Z 004563e0 f   theMenuScene.obj
 0001:00055740       ?UpdateShowPlayer@theMenuScene@@IAEXXZ 00456740 f   theMenuScene.obj
 0001:00055800       ??_GtheMenuScene@@UAEPAXI@Z 00456800 f i theMenuScene.obj
 0001:00055800       ??_EtheMenuScene@@UAEPAXI@Z 00456800 f i theMenuScene.obj
 0001:00055830       ??0theOverviewScene@@QAE@XZ 00456830 f   theOverviewScene.obj
 0001:00056190       ??1theOverviewScene@@UAE@XZ 00457190 f   theOverviewScene.obj
 0001:000561f0       ?Activate@theOverviewScene@@MAEX_N@Z 004571f0 f   theOverviewScene.obj
 0001:00056210       ?UpdateScene@theOverviewScene@@MAEXXZ 00457210 f   theOverviewScene.obj
 0001:00056630       ?DrawScene@theOverviewScene@@MAEXXZ 00457630 f   theOverviewScene.obj
 0001:000567b0       ?DrawUI@theOverviewScene@@IAEXXZ 004577b0 f   theOverviewScene.obj
 0001:000567c0       ?HandleKey@theOverviewScene@@UAE_NHHH@Z 004577c0 f   theOverviewScene.obj
 0001:00056810       ?HandleMouse@theOverviewScene@@UAE_NHUldwPoint@@@Z 00457810 f   theOverviewScene.obj
 0001:00056940       ?HandleMessage@theOverviewScene@@UAE_NHJ@Z 00457940 f   theOverviewScene.obj
 0001:000569c0       ??_GtheOverviewScene@@UAEPAXI@Z 004579c0 f i theOverviewScene.obj
 0001:000569c0       ??_EtheOverviewScene@@UAEPAXI@Z 004579c0 f i theOverviewScene.obj
 0001:000569f0       ??0SKey@CDoorKey@@QAE@XZ   004579f0 f i DoorKey.obj
 0001:000569f0       ??0SPuzzleIcon@CProgressScene@@QAE@XZ 004579f0 f i ProgressScene.obj
 0001:000569f0       ??0SCloud@theOverviewScene@@QAE@XZ 004579f0 f i theOverviewScene.obj
 0001:000569f0       ??0PathGradient@CWorldPath@@QAE@XZ 004579f0 f i WorldPath.obj
 0001:000569f0       ??0SSunBeam@CSunBeam@@QAE@XZ 004579f0 f i SunBeam.obj
 0001:000569f0       ??0STree@COrchard@@QAE@XZ  004579f0 f i Orchard.obj
 0001:00056a10       ??0theSplashScene@@QAE@XZ  00457a10 f   theSplashScene.obj
 0001:00056c60       ??1theSplashScene@@UAE@XZ  00457c60 f   theSplashScene.obj
 0001:00056d00       ?UpdateScene@theSplashScene@@MAEXXZ 00457d00 f   theSplashScene.obj
 0001:00056e60       ?SetTimer@theSplashScene@@QAEXXZ 00457e60 f   theSplashScene.obj
 0001:00056e80       ?DrawScene@theSplashScene@@MAEXXZ 00457e80 f   theSplashScene.obj
 0001:00056ef0       ?HandleKey@theSplashScene@@UAE_NHHH@Z 00457ef0 f   theSplashScene.obj
 0001:00057000       ?HandleMouse@theSplashScene@@UAE_NHUldwPoint@@@Z 00458000 f   theSplashScene.obj
 0001:000570e0       ?HandleMessage@theSplashScene@@UAE_NHJ@Z 004580e0 f   theSplashScene.obj
 0001:000570f0       ?Activate@theSplashScene@@UAEX_N@Z 004580f0 f   theSplashScene.obj
 0001:00057220       ??_EtheSplashScene@@UAEPAXI@Z 00458220 f i theSplashScene.obj
 0001:00057220       ??_GtheSplashScene@@UAEPAXI@Z 00458220 f i theSplashScene.obj
 0001:00057250       ?SetVolume@CSoundTrack@@QAEXM@Z 00458250 f i theSplashScene.obj
 0001:00057280       ??0theVillagerScene@@QAE@XZ 00458280 f   theVillagerScene.obj
 0001:00058b30       ??1theVillagerScene@@UAE@XZ 00459b30 f   theVillagerScene.obj
 0001:00058b90       ?UpdateScene@theVillagerScene@@MAEXXZ 00459b90 f   theVillagerScene.obj
 0001:00058f60       ?DrawScene@theVillagerScene@@MAEXXZ 00459f60 f   theVillagerScene.obj
 0001:00059230       ?HandleKey@theVillagerScene@@UAE_NHHH@Z 0045a230 f   theVillagerScene.obj
 0001:00059280       ?HandleMouse@theVillagerScene@@UAE_NHUldwPoint@@@Z 0045a280 f   theVillagerScene.obj
 0001:00059850       ?HandleMessage@theVillagerScene@@UAE_NHJ@Z 0045a850 f   theVillagerScene.obj
 0001:000599b0       ?UpdateSelection@theVillagerScene@@QAEXH@Z 0045a9b0 f   theVillagerScene.obj
 0001:00059a90       ?PopulateVillagerList@theVillagerScene@@QAEXXZ 0045aa90 f   theVillagerScene.obj
 0001:00059b40       ?SortVillagers@theVillagerScene@@QAEXXZ 0045ab40 f   theVillagerScene.obj
 0001:00059be0       ?SortTest@theVillagerScene@@QAE?B_NHH@Z 0045abe0 f   theVillagerScene.obj
 0001:00059ce0       ?FindVillager@theVillagerScene@@QAE?BHH@Z 0045ace0 f   theVillagerScene.obj
 0001:00059d30       ?Activate@theVillagerScene@@UAEX_N@Z 0045ad30 f   theVillagerScene.obj
 0001:00059d90       ??_EtheVillagerScene@@UAEPAXI@Z 0045ad90 f i theVillagerScene.obj
 0001:00059d90       ??_GtheVillagerScene@@UAEPAXI@Z 0045ad90 f i theVillagerScene.obj
 0001:00059dc0       ?SetFirstName@CVillagerBio@@QAEXPBD@Z 0045adc0 f i theVillagerScene.obj
 0001:00059df0       ?GetLikesAsString@CVillager@@QAEPBDXZ 0045adf0 f i theVillagerScene.obj
 0001:00059e10       ?GetDislikesAsString@CVillager@@QAEPBDXZ 0045ae10 f i theVillagerScene.obj
 0001:00059e30       ??0CIslandEventDialog@@QAE@PAVCIslandEvent@@@Z 0045ae30 f   IslandEvents.obj
 0001:0005aa90       ??1CIslandEventDialog@@UAE@XZ 0045ba90 f   IslandEvents.obj
 0001:0005abc0       ?DrawNoFadeScene@CIslandEventDialog@@MAEXXZ 0045bbc0 f   IslandEvents.obj
 0001:0005ac90       ?HandleMessage@CIslandEventDialog@@UAE_NHJ@Z 0045bc90 f   IslandEvents.obj
 0001:0005adb0       ?ComposeStringFromTemplate@CIslandEventDialog@@AAEXW4StringId@@@Z 0045bdb0 f   IslandEvents.obj
 0001:0005aec0       ?EventScalor@CIslandEventDialog@@QAEHH@Z 0045bec0 f   IslandEvents.obj
 0001:0005af00       ?Get@CIslandEvents@@SAPAV1@XZ 0045bf00 f   IslandEvents.obj
 0001:0005af80       ?Ref@CIslandEvents@@SAAAV1@XZ 0045bf80 f   IslandEvents.obj
 0001:0005af90       ?Destroy@CIslandEvents@@SAXXZ 0045bf90 f   IslandEvents.obj
 0001:0005afd0       ??0CIslandEvents@@AAE@XZ   0045bfd0 f   IslandEvents.obj
 0001:0005c410       ??1CIslandEvents@@QAE@XZ   0045d410 f   IslandEvents.obj
 0001:0005c480       ?FireEvent@CIslandEvents@@QAE_NPAVldwScene@@@Z 0045d480 f   IslandEvents.obj
 0001:0005c650       ?ShowAll@CIslandEvents@@QAEXPAVldwScene@@@Z 0045d650 f   IslandEvents.obj
 0001:0005c690       ?ForceEvent@CIslandEvents@@QAE_NPAVldwScene@@W4IslandEventId@@@Z 0045d690 f   IslandEvents.obj
 0001:0005c780       ?PercentOfResource@CIslandEvents@@QAEHHW4EventResourceId@@@Z 0045d780 f   IslandEvents.obj
 0001:0005c820       ?EventScalor@CIslandEvents@@QAEHH@Z 0045d820 f   IslandEvents.obj
 0001:0005c860       ??_ECIslandEventDialog@@UAEPAXI@Z 0045d860 f i IslandEvents.obj
 0001:0005c860       ??_GCIslandEventDialog@@UAEPAXI@Z 0045d860 f i IslandEvents.obj
 0001:0005c890       ??_GCIslandEvents@@QAEPAXI@Z 0045d890 f i IslandEvents.obj
 0001:0005c8c0       ??0CEventTsunami@@QAE@XZ   0045d8c0 f i IslandEvents.obj
 0001:0005c8e0       ??0CIslandEvent@@QAE@XZ    0045d8e0 f i IslandEvents.obj
 0001:0005c910       ?HasChoices@CIslandEvent@@UAE_NXZ 0045d910 f i IslandEvents.obj
 0001:0005c920       ?GetChoiceAText@CIslandEvent@@UAE?AW4StringId@@XZ 0045d920 f i IslandEvents.obj
 0001:0005c920       ?GetChoiceBText@CIslandEvent@@UAE?AW4StringId@@XZ 0045d920 f i IslandEvents.obj
 0001:0005c930       ?GetResultDescription@CIslandEvent@@UAE?AW4StringId@@H@Z 0045d930 f i IslandEvents.obj
 0001:0005c940       ?AgesChecked@CVillagerState@@QBE?BHXZ 0045d940 f i Villager.obj
 0001:0005c940       ?GetSize@?$CSimpleMap@PADPAGVCExpansionVectorEqualHelper@ATL@@@ATL@@QBEHXZ 0045d940 f i FlashPlayer.obj
 0001:0005c940       ?GetAwardAmount@CIslandEvent@@UAEHXZ 0045d940 f i IslandEvents.obj
 0001:0005c940       ?GetLink@ldwRadioButtonImpl@@QAEPAVldwRadioButton@@XZ 0045d940 f i ldwRadioButton.obj
 0001:0005c940       ?FName@CVillagerBio@@QBE?BHXZ 0045d940 f i Behavior.obj
 0001:0005c940       ?GetLockCount@CAtlModule@ATL@@UAEJXZ 0045d940 f i FlashPlayer.obj
 0001:0005c960       ??_ECIslandEvent@@UAEPAXI@Z 0045d960 f i IslandEvents.obj
 0001:0005c960       ??_GCIslandEvent@@UAEPAXI@Z 0045d960 f i IslandEvents.obj
 0001:0005c990       ??1CIslandEvent@@UAE@XZ    0045d990 f i IslandEvents.obj
 0001:0005c9b0       ?GetTitle@CEventTsunami@@UAE?AW4StringId@@XZ 0045d9b0 f i IslandEvents.obj
 0001:0005c9c0       ?GetDescription@CEventTsunami@@UAE?AW4StringId@@XZ 0045d9c0 f i IslandEvents.obj
 0001:0005c9d0       ?CanFire@CEventTsunami@@UAE_NXZ 0045d9d0 f i IslandEvents.obj
 0001:0005ca40       ?ImpactGame@CEventTsunami@@UAEXXZ 0045da40 f i IslandEvents.obj
 0001:0005ca70       ??_ECEventTsunami@@UAEPAXI@Z 0045da70 f i IslandEvents.obj
 0001:0005ca70       ??_GCEventTsunami@@UAEPAXI@Z 0045da70 f i IslandEvents.obj
 0001:0005caa0       ??1CEventTsunami@@UAE@XZ   0045daa0 f i IslandEvents.obj
 0001:0005cac0       ??0CEventPlagueOfAnts@@QAE@XZ 0045dac0 f i IslandEvents.obj
 0001:0005cae0       ?GetTitle@CEventPlagueOfAnts@@UAE?AW4StringId@@XZ 0045dae0 f i IslandEvents.obj
 0001:0005caf0       ?GetDescription@CEventPlagueOfAnts@@UAE?AW4StringId@@XZ 0045daf0 f i IslandEvents.obj
 0001:0005cb00       ?CalcAward@CEventPlagueOfAnts@@UAEXXZ 0045db00 f i IslandEvents.obj
 0001:0005cb50       ?EventScalor@CIslandEvent@@QAEHH@Z 0045db50 f i IslandEvents.obj
 0001:0005cb90       ?ImpactGame@CEventPlagueOfAnts@@UAEXXZ 0045db90 f i IslandEvents.obj
 0001:0005cbc0       ??_ECEventPlagueOfAnts@@UAEPAXI@Z 0045dbc0 f i IslandEvents.obj
 0001:0005cbc0       ??_GCEventPlagueOfAnts@@UAEPAXI@Z 0045dbc0 f i IslandEvents.obj
 0001:0005cbf0       ??1CEventPlagueOfAnts@@UAE@XZ 0045dbf0 f i IslandEvents.obj
 0001:0005cc10       ??0CEventScienceFair@@QAE@XZ 0045dc10 f i IslandEvents.obj
 0001:0005cc30       ?GetTitle@CEventScienceFair@@UAE?AW4StringId@@XZ 0045dc30 f i IslandEvents.obj
 0001:0005cc40       ?GetDescription@CEventScienceFair@@UAE?AW4StringId@@XZ 0045dc40 f i IslandEvents.obj
 0001:0005cc50       ?CanFire@CEventScienceFair@@UAE_NXZ 0045dc50 f i IslandEvents.obj
 0001:0005cc90       ?ImpactGame@CEventScienceFair@@UAEXXZ 0045dc90 f i IslandEvents.obj
 0001:0005ccd0       ??_ECEventScienceFair@@UAEPAXI@Z 0045dcd0 f i IslandEvents.obj
 0001:0005ccd0       ??_GCEventScienceFair@@UAEPAXI@Z 0045dcd0 f i IslandEvents.obj
 0001:0005cd00       ??1CEventScienceFair@@UAE@XZ 0045dd00 f i IslandEvents.obj
 0001:0005cd20       ??0CEventAllergySeason@@QAE@XZ 0045dd20 f i IslandEvents.obj
 0001:0005cd40       ?GetTitle@CEventAllergySeason@@UAE?AW4StringId@@XZ 0045dd40 f i IslandEvents.obj
 0001:0005cd50       ?GetDescription@CEventAllergySeason@@UAE?AW4StringId@@XZ 0045dd50 f i IslandEvents.obj
 0001:0005cd60       ?ImpactGame@CEventAllergySeason@@UAEXXZ 0045dd60 f i IslandEvents.obj
 0001:0005cd90       ??_GCEventAllergySeason@@UAEPAXI@Z 0045dd90 f i IslandEvents.obj
 0001:0005cd90       ??_ECEventAllergySeason@@UAEPAXI@Z 0045dd90 f i IslandEvents.obj
 0001:0005cdc0       ??1CEventAllergySeason@@UAE@XZ 0045ddc0 f i IslandEvents.obj
 0001:0005cde0       ??0CEventIsolaDay@@QAE@XZ  0045dde0 f i IslandEvents.obj
 0001:0005ce00       ?GetTitle@CEventIsolaDay@@UAE?AW4StringId@@XZ 0045de00 f i IslandEvents.obj
 0001:0005ce10       ?GetDescription@CEventIsolaDay@@UAE?AW4StringId@@XZ 0045de10 f i IslandEvents.obj
 0001:0005ce20       ?ImpactGame@CEventIsolaDay@@UAEXXZ 0045de20 f i IslandEvents.obj
 0001:0005ce90       ??_ECEventIsolaDay@@UAEPAXI@Z 0045de90 f i IslandEvents.obj
 0001:0005ce90       ??_GCEventIsolaDay@@UAEPAXI@Z 0045de90 f i IslandEvents.obj
 0001:0005cec0       ??1CEventIsolaDay@@UAE@XZ  0045dec0 f i IslandEvents.obj
 0001:0005cee0       ??0CEventBlessingsDay@@QAE@XZ 0045dee0 f i IslandEvents.obj
 0001:0005cf00       ?GetTitle@CEventBlessingsDay@@UAE?AW4StringId@@XZ 0045df00 f i IslandEvents.obj
 0001:0005cf10       ?GetDescription@CEventBlessingsDay@@UAE?AW4StringId@@XZ 0045df10 f i IslandEvents.obj
 0001:0005cf20       ?ImpactGame@CEventBlessingsDay@@UAEXXZ 0045df20 f i IslandEvents.obj
 0001:0005cf80       ??_ECEventBlessingsDay@@UAEPAXI@Z 0045df80 f i IslandEvents.obj
 0001:0005cf80       ??_GCEventBlessingsDay@@UAEPAXI@Z 0045df80 f i IslandEvents.obj
 0001:0005cfb0       ??1CEventBlessingsDay@@UAE@XZ 0045dfb0 f i IslandEvents.obj
 0001:0005cfd0       ??0CEventCanoeFromOtherSide@@QAE@XZ 0045dfd0 f i IslandEvents.obj
 0001:0005cff0       ?GetTitle@CEventCanoeFromOtherSide@@UAE?AW4StringId@@XZ 0045dff0 f i IslandEvents.obj
 0001:0005d000       ?GetDescription@CEventCanoeFromOtherSide@@UAE?AW4StringId@@XZ 0045e000 f i IslandEvents.obj
 0001:0005d010       ?CanFire@CEventCanoeFromOtherSide@@UAE_NXZ 0045e010 f i IslandEvents.obj
 0001:0005d040       ?ImpactGame@CEventCanoeFromOtherSide@@UAEXXZ 0045e040 f i IslandEvents.obj
 0001:0005d0b0       ??_GCEventCanoeFromOtherSide@@UAEPAXI@Z 0045e0b0 f i IslandEvents.obj
 0001:0005d0b0       ??_ECEventCanoeFromOtherSide@@UAEPAXI@Z 0045e0b0 f i IslandEvents.obj
 0001:0005d0e0       ??1CEventCanoeFromOtherSide@@UAE@XZ 0045e0e0 f i IslandEvents.obj
 0001:0005d100       ??0CEventMysteriousFogFoodBonus@@QAE@XZ 0045e100 f i IslandEvents.obj
 0001:0005d120       ?GetTitle@CEventMysteriousFogFoodBonus@@UAE?AW4StringId@@XZ 0045e120 f i IslandEvents.obj
 0001:0005d130       ?GetDescription@CEventMysteriousFogFoodBonus@@UAE?AW4StringId@@XZ 0045e130 f i IslandEvents.obj
 0001:0005d140       ?CalcAward@CEventMysteriousFogFoodBonus@@UAEXXZ 0045e140 f i IslandEvents.obj
 0001:0005d160       ?ImpactGame@CEventMysteriousFogFoodBonus@@UAEXXZ 0045e160 f i IslandEvents.obj
 0001:0005d1a0       ??_ECEventMysteriousFogFoodBonus@@UAEPAXI@Z 0045e1a0 f i IslandEvents.obj
 0001:0005d1a0       ??_GCEventMysteriousFogFoodBonus@@UAEPAXI@Z 0045e1a0 f i IslandEvents.obj
 0001:0005d1d0       ??1CEventMysteriousFogFoodBonus@@UAE@XZ 0045e1d0 f i IslandEvents.obj
 0001:0005d1f0       ??0CEventMysteriousFogFoodPenalty@@QAE@XZ 0045e1f0 f i IslandEvents.obj
 0001:0005d210       ?GetTitle@CEventMysteriousFogFoodPenalty@@UAE?AW4StringId@@XZ 0045e210 f i IslandEvents.obj
 0001:0005d220       ?GetDescription@CEventMysteriousFogFoodPenalty@@UAE?AW4StringId@@XZ 0045e220 f i IslandEvents.obj
 0001:0005d230       ?CalcAward@CEventMysteriousFogFoodPenalty@@UAEXXZ 0045e230 f i IslandEvents.obj
 0001:0005d290       ?ImpactGame@CEventMysteriousFogFoodPenalty@@UAEXXZ 0045e290 f i IslandEvents.obj
 0001:0005d2d0       ??_GCEventMysteriousFogFoodPenalty@@UAEPAXI@Z 0045e2d0 f i IslandEvents.obj
 0001:0005d2d0       ??_ECEventMysteriousFogFoodPenalty@@UAEPAXI@Z 0045e2d0 f i IslandEvents.obj
 0001:0005d300       ??1CEventMysteriousFogFoodPenalty@@UAE@XZ 0045e300 f i IslandEvents.obj
 0001:0005d320       ??0CEventMysteriousFogTechBonus@@QAE@XZ 0045e320 f i IslandEvents.obj
 0001:0005d340       ?GetTitle@CEventMysteriousFogTechBonus@@UAE?AW4StringId@@XZ 0045e340 f i IslandEvents.obj
 0001:0005d350       ?GetDescription@CEventMysteriousFogTechBonus@@UAE?AW4StringId@@XZ 0045e350 f i IslandEvents.obj
 0001:0005d360       ?CalcAward@CEventMysteriousFogTechBonus@@UAEXXZ 0045e360 f i IslandEvents.obj
 0001:0005d380       ?ImpactGame@CEventMysteriousFogTechBonus@@UAEXXZ 0045e380 f i IslandEvents.obj
 0001:0005d3c0       ??_GCEventMysteriousFogTechBonus@@UAEPAXI@Z 0045e3c0 f i IslandEvents.obj
 0001:0005d3c0       ??_ECEventMysteriousFogTechBonus@@UAEPAXI@Z 0045e3c0 f i IslandEvents.obj
 0001:0005d3f0       ??1CEventMysteriousFogTechBonus@@UAE@XZ 0045e3f0 f i IslandEvents.obj
 0001:0005d410       ??0CEventMysteriousFogTechPenalty@@QAE@XZ 0045e410 f i IslandEvents.obj
 0001:0005d430       ?GetTitle@CEventMysteriousFogTechPenalty@@UAE?AW4StringId@@XZ 0045e430 f i IslandEvents.obj
 0001:0005d440       ?GetDescription@CEventMysteriousFogTechPenalty@@UAE?AW4StringId@@XZ 0045e440 f i IslandEvents.obj
 0001:0005d450       ?CalcAward@CEventMysteriousFogTechPenalty@@UAEXXZ 0045e450 f i IslandEvents.obj
 0001:0005d4b0       ?ImpactGame@CEventMysteriousFogTechPenalty@@UAEXXZ 0045e4b0 f i IslandEvents.obj
 0001:0005d4f0       ??_ECEventMysteriousFogTechPenalty@@UAEPAXI@Z 0045e4f0 f i IslandEvents.obj
 0001:0005d4f0       ??_GCEventMysteriousFogTechPenalty@@UAEPAXI@Z 0045e4f0 f i IslandEvents.obj
 0001:0005d520       ??1CEventMysteriousFogTechPenalty@@UAE@XZ 0045e520 f i IslandEvents.obj
 0001:0005d540       ??0CEventDayOfHonor@@QAE@XZ 0045e540 f i IslandEvents.obj
 0001:0005d560       ?GetTitle@CEventDayOfHonor@@UAE?AW4StringId@@XZ 0045e560 f i IslandEvents.obj
 0001:0005d570       ?GetDescription@CEventDayOfHonor@@UAE?AW4StringId@@XZ 0045e570 f i IslandEvents.obj
 0001:0005d580       ?CanFire@CEventDayOfHonor@@UAE_NXZ 0045e580 f i IslandEvents.obj
 0001:0005d5a0       ?ImpactGame@CEventDayOfHonor@@UAEXXZ 0045e5a0 f i IslandEvents.obj
 0001:0005d5d0       ??_ECEventDayOfHonor@@UAEPAXI@Z 0045e5d0 f i IslandEvents.obj
 0001:0005d5d0       ??_GCEventDayOfHonor@@UAEPAXI@Z 0045e5d0 f i IslandEvents.obj
 0001:0005d600       ??1CEventDayOfHonor@@UAE@XZ 0045e600 f i IslandEvents.obj
 0001:0005d620       ??0CEventMiraculousBloom@@QAE@XZ 0045e620 f i IslandEvents.obj
 0001:0005d640       ?GetTitle@CEventMiraculousBloom@@UAE?AW4StringId@@XZ 0045e640 f i IslandEvents.obj
 0001:0005d650       ?GetDescription@CEventMiraculousBloom@@UAE?AW4StringId@@XZ 0045e650 f i IslandEvents.obj
 0001:0005d660       ?CanFire@CEventMiraculousBloom@@UAE_NXZ 0045e660 f i IslandEvents.obj
 0001:0005d690       ?ImpactGame@CEventMiraculousBloom@@UAEXXZ 0045e690 f i IslandEvents.obj
 0001:0005d6b0       ??_ECEventMiraculousBloom@@UAEPAXI@Z 0045e6b0 f i IslandEvents.obj
 0001:0005d6b0       ??_GCEventMiraculousBloom@@UAEPAXI@Z 0045e6b0 f i IslandEvents.obj
 0001:0005d6e0       ??1CEventMiraculousBloom@@UAE@XZ 0045e6e0 f i IslandEvents.obj
 0001:0005d700       ??0CEventTheReflectionInTheWater@@QAE@XZ 0045e700 f i IslandEvents.obj
 0001:0005d720       ?GetTitle@CEventTheReflectionInTheWater@@UAE?AW4StringId@@XZ 0045e720 f i IslandEvents.obj
 0001:0005d730       ?GetDescription@CEventTheReflectionInTheWater@@UAE?AW4StringId@@XZ 0045e730 f i IslandEvents.obj
 0001:0005d740       ?FadeImage@IPage@@UAE?B_NXZ 0045e740 f i Pages.obj
 0001:0005d740       ?CanFire@CEventTheRainySeason@@UAE_NXZ 0045e740 f i IslandEvents.obj
 0001:0005d740       ?CanFire@CEventAllergySeason@@UAE_NXZ 0045e740 f i IslandEvents.obj
 0001:0005d740       ?CanFire@CEventTheReflectionInTheWater@@UAE_NXZ 0045e740 f i IslandEvents.obj
 0001:0005d740       ?CanFire@CEventTheSaltyAir@@UAE_NXZ 0045e740 f i IslandEvents.obj
 0001:0005d740       ?CanFire@CEventMysteriousFogTechBonus@@UAE_NXZ 0045e740 f i IslandEvents.obj
 0001:0005d740       ?CanFire@CEventIsolaDay@@UAE_NXZ 0045e740 f i IslandEvents.obj
 0001:0005d740       ?CanFire@CEventTheYellowGeckos@@UAE_NXZ 0045e740 f i IslandEvents.obj
 0001:0005d740       ?FadeOut@IPage@@UAE?B_NXZ  0045e740 f i Pages.obj
 0001:0005d740       ?CanFire@CEventMysteriousFogTechPenalty@@UAE_NXZ 0045e740 f i IslandEvents.obj
 0001:0005d740       ?CanFire@CEventTheOppressiveHumidity@@UAE_NXZ 0045e740 f i IslandEvents.obj
 0001:0005d740       ?SoundEnabled@ldwGameState@@UAE_NXZ 0045e740 f i ldwGameState.obj
 0001:0005d740       ?CanFire@CEventBlessingsDay@@UAE_NXZ 0045e740 f i IslandEvents.obj
 0001:0005d740       ?CanFire@CEventTheStingingJellyfish@@UAE_NXZ 0045e740 f i IslandEvents.obj
 0001:0005d740       ?CanFire@CEventMysteriousFogFoodBonus@@UAE_NXZ 0045e740 f i IslandEvents.obj
 0001:0005d740       ?HasChoices@CIslandEventChoiceAB@@UAE_NXZ 0045e740 f i IslandEvents.obj
 0001:0005d740       ?CanFire@CEventFoggyHeaded@@UAE_NXZ 0045e740 f i IslandEvents.obj
 0001:0005d740       ?CanFire@CEventPlagueOfAnts@@UAE_NXZ 0045e740 f i IslandEvents.obj
 0001:0005d740       ?CanMakeWindowed@ldwGameWindowImpl@@QAE_NXZ 0045e740 f i ldwGameWindow.obj
 0001:0005d740       ?CanFire@CEventMysteriousFogFoodPenalty@@UAE_NXZ 0045e740 f i IslandEvents.obj
 0001:0005d750       ??_GCEventTheReflectionInTheWater@@UAEPAXI@Z 0045e750 f i IslandEvents.obj
 0001:0005d750       ??_ECEventTheReflectionInTheWater@@UAEPAXI@Z 0045e750 f i IslandEvents.obj
 0001:0005d780       ??1CEventTheReflectionInTheWater@@UAE@XZ 0045e780 f i IslandEvents.obj
 0001:0005d7a0       ??0CEventTheChiefsAddress@@QAE@XZ 0045e7a0 f i IslandEvents.obj
 0001:0005d7c0       ?GetTitle@CEventTheChiefsAddress@@UAE?AW4StringId@@XZ 0045e7c0 f i IslandEvents.obj
 0001:0005d7d0       ?GetDescription@CEventTheChiefsAddress@@UAE?AW4StringId@@XZ 0045e7d0 f i IslandEvents.obj
 0001:0005d7e0       ?CanFire@CEventTheChiefsAddress@@UAE_NXZ 0045e7e0 f i IslandEvents.obj
 0001:0005d810       ?ImpactGame@CEventTheChiefsAddress@@UAEXXZ 0045e810 f i IslandEvents.obj
 0001:0005d8a0       ??_ECEventTheChiefsAddress@@UAEPAXI@Z 0045e8a0 f i IslandEvents.obj
 0001:0005d8a0       ??_GCEventTheChiefsAddress@@UAEPAXI@Z 0045e8a0 f i IslandEvents.obj
 0001:0005d8d0       ??1CEventTheChiefsAddress@@UAE@XZ 0045e8d0 f i IslandEvents.obj
 0001:0005d8f0       ??0CEventTheRainySeason@@QAE@XZ 0045e8f0 f i IslandEvents.obj
 0001:0005d910       ?GetTitle@CEventTheRainySeason@@UAE?AW4StringId@@XZ 0045e910 f i IslandEvents.obj
 0001:0005d920       ?GetDescription@CEventTheRainySeason@@UAE?AW4StringId@@XZ 0045e920 f i IslandEvents.obj
 0001:0005d930       ?ImpactGame@CEventTheRainySeason@@UAEXXZ 0045e930 f i IslandEvents.obj
 0001:0005d950       ??_ECEventTheRainySeason@@UAEPAXI@Z 0045e950 f i IslandEvents.obj
 0001:0005d950       ??_GCEventTheRainySeason@@UAEPAXI@Z 0045e950 f i IslandEvents.obj
 0001:0005d980       ??1CEventTheRainySeason@@UAE@XZ 0045e980 f i IslandEvents.obj
 0001:0005d9a0       ??0CEventTheColdSnap@@QAE@XZ 0045e9a0 f i IslandEvents.obj
 0001:0005d9c0       ?GetTitle@CEventTheColdSnap@@UAE?AW4StringId@@XZ 0045e9c0 f i IslandEvents.obj
 0001:0005d9d0       ?GetDescription@CEventTheColdSnap@@UAE?AW4StringId@@XZ 0045e9d0 f i IslandEvents.obj
 0001:0005d9e0       ?CanFire@CEventTheColdSnap@@UAE_NXZ 0045e9e0 f i IslandEvents.obj
 0001:0005da10       ?ImpactGame@CEventTheColdSnap@@UAEXXZ 0045ea10 f i IslandEvents.obj
 0001:0005da40       ??_ECEventTheColdSnap@@UAEPAXI@Z 0045ea40 f i IslandEvents.obj
 0001:0005da40       ??_GCEventTheColdSnap@@UAEPAXI@Z 0045ea40 f i IslandEvents.obj
 0001:0005da70       ??1CEventTheColdSnap@@UAE@XZ 0045ea70 f i IslandEvents.obj
 0001:0005da90       ??0CEventTheSaltyAir@@QAE@XZ 0045ea90 f i IslandEvents.obj
 0001:0005dab0       ?GetTitle@CEventTheSaltyAir@@UAE?AW4StringId@@XZ 0045eab0 f i IslandEvents.obj
 0001:0005dac0       ?GetDescription@CEventTheSaltyAir@@UAE?AW4StringId@@XZ 0045eac0 f i IslandEvents.obj
 0001:0005dad0       ?ImpactGame@CEventTheSaltyAir@@UAEXXZ 0045ead0 f i IslandEvents.obj
 0001:0005daf0       ??_GCEventTheSaltyAir@@UAEPAXI@Z 0045eaf0 f i IslandEvents.obj
 0001:0005daf0       ??_ECEventTheSaltyAir@@UAEPAXI@Z 0045eaf0 f i IslandEvents.obj
 0001:0005db20       ??1CEventTheSaltyAir@@UAE@XZ 0045eb20 f i IslandEvents.obj
 0001:0005db40       ??0CEventTheOppressiveHumidity@@QAE@XZ 0045eb40 f i IslandEvents.obj
 0001:0005db60       ?GetTitle@CEventTheOppressiveHumidity@@UAE?AW4StringId@@XZ 0045eb60 f i IslandEvents.obj
 0001:0005db70       ?GetDescription@CEventTheOppressiveHumidity@@UAE?AW4StringId@@XZ 0045eb70 f i IslandEvents.obj
 0001:0005db80       ?ImpactGame@CEventTheOppressiveHumidity@@UAEXXZ 0045eb80 f i IslandEvents.obj
 0001:0005dbb0       ??_GCEventTheOppressiveHumidity@@UAEPAXI@Z 0045ebb0 f i IslandEvents.obj
 0001:0005dbb0       ??_ECEventTheOppressiveHumidity@@UAEPAXI@Z 0045ebb0 f i IslandEvents.obj
 0001:0005dbe0       ??1CEventTheOppressiveHumidity@@UAE@XZ 0045ebe0 f i IslandEvents.obj
 0001:0005dc00       ??0CEventFoggyHeaded@@QAE@XZ 0045ec00 f i IslandEvents.obj
 0001:0005dc20       ?GetTitle@CEventFoggyHeaded@@UAE?AW4StringId@@XZ 0045ec20 f i IslandEvents.obj
 0001:0005dc30       ?GetDescription@CEventFoggyHeaded@@UAE?AW4StringId@@XZ 0045ec30 f i IslandEvents.obj
 0001:0005dc40       ?ImpactGame@CEventFoggyHeaded@@UAEXXZ 0045ec40 f i IslandEvents.obj
 0001:0005dc70       ??_GCEventFoggyHeaded@@UAEPAXI@Z 0045ec70 f i IslandEvents.obj
 0001:0005dc70       ??_ECEventFoggyHeaded@@UAEPAXI@Z 0045ec70 f i IslandEvents.obj
 0001:0005dca0       ??1CEventFoggyHeaded@@UAE@XZ 0045eca0 f i IslandEvents.obj
 0001:0005dcc0       ??0CEventTheStingingJellyfish@@QAE@XZ 0045ecc0 f i IslandEvents.obj
 0001:0005dce0       ?GetTitle@CEventTheStingingJellyfish@@UAE?AW4StringId@@XZ 0045ece0 f i IslandEvents.obj
 0001:0005dcf0       ?GetDescription@CEventTheStingingJellyfish@@UAE?AW4StringId@@XZ 0045ecf0 f i IslandEvents.obj
 0001:0005dd00       ?ImpactGame@CEventTheStingingJellyfish@@UAEXXZ 0045ed00 f i IslandEvents.obj
 0001:0005dd60       ??_ECEventTheStingingJellyfish@@UAEPAXI@Z 0045ed60 f i IslandEvents.obj
 0001:0005dd60       ??_GCEventTheStingingJellyfish@@UAEPAXI@Z 0045ed60 f i IslandEvents.obj
 0001:0005dd90       ??1CEventTheStingingJellyfish@@UAE@XZ 0045ed90 f i IslandEvents.obj
 0001:0005ddb0       ??0CEventTheMushroomCelebration@@QAE@XZ 0045edb0 f i IslandEvents.obj
 0001:0005ddd0       ?GetTitle@CEventTheMushroomCelebration@@UAE?AW4StringId@@XZ 0045edd0 f i IslandEvents.obj
 0001:0005dde0       ?GetDescription@CEventTheMushroomCelebration@@UAE?AW4StringId@@XZ 0045ede0 f i IslandEvents.obj
 0001:0005ddf0       ?CanFire@CEventTheMushroomCelebration@@UAE_NXZ 0045edf0 f i IslandEvents.obj
 0001:0005de20       ?Wetness@CWeather@@QBE?BHXZ 0045ee20 f i VillagerAI.obj
 0001:0005de20       ?PreferredSkill@CVillagerSkills@@QBE?BW4ESkill@@XZ 0045ee20 f i VillagerAI.obj
 0001:0005de20       ?ItemsFound@CGameStats@@QBE?BHXZ 0045ee20 f i IslandEvents.obj
 0001:0005de40       ?ImpactGame@CEventTheMushroomCelebration@@UAEXXZ 0045ee40 f i IslandEvents.obj
 0001:0005de60       ??_GCEventTheMushroomCelebration@@UAEPAXI@Z 0045ee60 f i IslandEvents.obj
 0001:0005de60       ??_ECEventTheMushroomCelebration@@UAEPAXI@Z 0045ee60 f i IslandEvents.obj
 0001:0005de90       ??1CEventTheMushroomCelebration@@UAE@XZ 0045ee90 f i IslandEvents.obj
 0001:0005deb0       ??0CEventTheYellowGeckos@@QAE@XZ 0045eeb0 f i IslandEvents.obj
 0001:0005ded0       ?GetTitle@CEventTheYellowGeckos@@UAE?AW4StringId@@XZ 0045eed0 f i IslandEvents.obj
 0001:0005dee0       ?GetDescription@CEventTheYellowGeckos@@UAE?AW4StringId@@XZ 0045eee0 f i IslandEvents.obj
 0001:0005def0       ?ImpactGame@CEventTheYellowGeckos@@UAEXXZ 0045eef0 f i IslandEvents.obj
 0001:0005df10       ??_ECEventTheYellowGeckos@@UAEPAXI@Z 0045ef10 f i IslandEvents.obj
 0001:0005df10       ??_GCEventTheYellowGeckos@@UAEPAXI@Z 0045ef10 f i IslandEvents.obj
 0001:0005df40       ??1CEventTheYellowGeckos@@UAE@XZ 0045ef40 f i IslandEvents.obj
 0001:0005df60       ??0CEventAnotherBarrelOBabies@@QAE@XZ 0045ef60 f i IslandEvents.obj
 0001:0005df80       ?GetTitle@CEventAnotherBarrelOBabies@@UAE?AW4StringId@@XZ 0045ef80 f i IslandEvents.obj
 0001:0005df90       ?GetDescription@CEventAnotherBarrelOBabies@@UAE?AW4StringId@@XZ 0045ef90 f i IslandEvents.obj
 0001:0005dfa0       ?CanFire@CEventAnotherBarrelOBabies@@UAE_NXZ 0045efa0 f i IslandEvents.obj
 0001:0005dfc0       ?ImpactGame@CEventAnotherBarrelOBabies@@UAEXXZ 0045efc0 f i IslandEvents.obj
 0001:0005e090       ??_ECEventAnotherBarrelOBabies@@UAEPAXI@Z 0045f090 f i IslandEvents.obj
 0001:0005e090       ??_GCEventAnotherBarrelOBabies@@UAEPAXI@Z 0045f090 f i IslandEvents.obj
 0001:0005e0c0       ??1CEventAnotherBarrelOBabies@@UAE@XZ 0045f0c0 f i IslandEvents.obj
 0001:0005e0e0       ??0CEventDaredevil@@QAE@XZ 0045f0e0 f i IslandEvents.obj
 0001:0005e100       ??0CIslandEventChoiceAB@@QAE@XZ 0045f100 f i IslandEvents.obj
 0001:0005e140       ?GetTargetVillager@CIslandEventChoiceAB@@UAEPAVCVillager@@XZ 0045f140 f i IslandEvents.obj
 0001:0005e170       ?Health@CVillagerState@@QBE?BHXZ 0045f170 f i Villager.obj
 0001:0005e170       ?GetTargetVillager2@CIslandEventChoiceAB@@UAEPAVCVillager@@XZ 0045f170 f i IslandEvents.obj
 0001:0005e170       ?LName@CVillagerBio@@QBE?BHXZ 0045f170 f i Behavior.obj
 0001:0005e190       ??_ECIslandEventChoiceAB@@UAEPAXI@Z 0045f190 f i IslandEvents.obj
 0001:0005e190       ??_GCIslandEventChoiceAB@@UAEPAXI@Z 0045f190 f i IslandEvents.obj
 0001:0005e1c0       ??1CIslandEventChoiceAB@@UAE@XZ 0045f1c0 f i IslandEvents.obj
 0001:0005e1e0       ?GetTitle@CEventDaredevil@@UAE?AW4StringId@@XZ 0045f1e0 f i IslandEvents.obj
 0001:0005e1f0       ?GetDescription@CEventDaredevil@@UAE?AW4StringId@@XZ 0045f1f0 f i IslandEvents.obj
 0001:0005e200       ?GetChoiceAText@CEventDaredevil@@UAE?AW4StringId@@XZ 0045f200 f i IslandEvents.obj
 0001:0005e210       ?GetChoiceBText@CEventDaredevil@@UAE?AW4StringId@@XZ 0045f210 f i IslandEvents.obj
 0001:0005e220       ?CanFire@CEventDaredevil@@UAE_NXZ 0045f220 f i IslandEvents.obj
 0001:0005e280       ?GetResultDescription@CEventDaredevil@@UAE?AW4StringId@@H@Z 0045f280 f i IslandEvents.obj
 0001:0005e2d0       ?ImpactGame@CEventDaredevil@@UAEXH@Z 0045f2d0 f i IslandEvents.obj
 0001:0005e3d0       ??_GCEventDaredevil@@UAEPAXI@Z 0045f3d0 f i IslandEvents.obj
 0001:0005e3d0       ??_ECEventDaredevil@@UAEPAXI@Z 0045f3d0 f i IslandEvents.obj
 0001:0005e400       ??1CEventDaredevil@@UAE@XZ 0045f400 f i IslandEvents.obj
 0001:0005e420       ??0CEventGhostlyNatureDream@@QAE@XZ 0045f420 f i IslandEvents.obj
 0001:0005e440       ?GetTitle@CEventGhostlyNatureDream@@UAE?AW4StringId@@XZ 0045f440 f i IslandEvents.obj
 0001:0005e450       ?GetDescription@CEventGhostlyNatureDream@@UAE?AW4StringId@@XZ 0045f450 f i IslandEvents.obj
 0001:0005e460       ?GetChoiceAText@CEventGhostlyNatureDream@@UAE?AW4StringId@@XZ 0045f460 f i IslandEvents.obj
 0001:0005e470       ?GetChoiceBText@CEventGhostlyNatureDream@@UAE?AW4StringId@@XZ 0045f470 f i IslandEvents.obj
 0001:0005e480       ?CanFire@CEventGhostlyNatureDream@@UAE_NXZ 0045f480 f i IslandEvents.obj
 0001:0005e4d0       ?GetVillagerPose@CEventGhostlyNatureDream@@UAE?AW4EBodyPosition@@XZ 0045f4d0 f i IslandEvents.obj
 0001:0005e4d0       ?GetVillagerPose@CEventTheAntInTheBed@@UAE?AW4EBodyPosition@@XZ 0045f4d0 f i IslandEvents.obj
 0001:0005e4d0       ?GetVillagerPose@CEventGhostlyMagicDream@@UAE?AW4EBodyPosition@@XZ 0045f4d0 f i IslandEvents.obj
 0001:0005e4e0       ?GetResultDescription@CEventGhostlyNatureDream@@UAE?AW4StringId@@H@Z 0045f4e0 f i IslandEvents.obj
 0001:0005e500       ?ImpactGame@CEventGhostlyNatureDream@@UAEXH@Z 0045f500 f i IslandEvents.obj
 0001:0005e570       ??_GCEventGhostlyNatureDream@@UAEPAXI@Z 0045f570 f i IslandEvents.obj
 0001:0005e570       ??_ECEventGhostlyNatureDream@@UAEPAXI@Z 0045f570 f i IslandEvents.obj
 0001:0005e5a0       ??1CEventGhostlyNatureDream@@UAE@XZ 0045f5a0 f i IslandEvents.obj
 0001:0005e5c0       ??0CEventGhostlyMagicDream@@QAE@XZ 0045f5c0 f i IslandEvents.obj
 0001:0005e5e0       ?GetTitle@CEventGhostlyMagicDream@@UAE?AW4StringId@@XZ 0045f5e0 f i IslandEvents.obj
 0001:0005e5f0       ?GetDescription@CEventGhostlyMagicDream@@UAE?AW4StringId@@XZ 0045f5f0 f i IslandEvents.obj
 0001:0005e600       ?GetChoiceAText@CEventGhostlyMagicDream@@UAE?AW4StringId@@XZ 0045f600 f i IslandEvents.obj
 0001:0005e610       ?GetChoiceBText@CEventGhostlyMagicDream@@UAE?AW4StringId@@XZ 0045f610 f i IslandEvents.obj
 0001:0005e620       ?CanFire@CEventGhostlyMagicDream@@UAE_NXZ 0045f620 f i IslandEvents.obj
 0001:0005e670       ?GetResultDescription@CEventGhostlyMagicDream@@UAE?AW4StringId@@H@Z 0045f670 f i IslandEvents.obj
 0001:0005e690       ?ImpactGame@CEventGhostlyMagicDream@@UAEXH@Z 0045f690 f i IslandEvents.obj
 0001:0005e6e0       ??_ECEventGhostlyMagicDream@@UAEPAXI@Z 0045f6e0 f i IslandEvents.obj
 0001:0005e6e0       ??_GCEventGhostlyMagicDream@@UAEPAXI@Z 0045f6e0 f i IslandEvents.obj
 0001:0005e710       ??1CEventGhostlyMagicDream@@UAE@XZ 0045f710 f i IslandEvents.obj
 0001:0005e730       ??0CEventXtalOfReflections@@QAE@XZ 0045f730 f i IslandEvents.obj
 0001:0005e750       ?GetTitle@CEventXtalOfReflections@@UAE?AW4StringId@@XZ 0045f750 f i IslandEvents.obj
 0001:0005e760       ?GetDescription@CEventXtalOfReflections@@UAE?AW4StringId@@XZ 0045f760 f i IslandEvents.obj
 0001:0005e770       ?GetChoiceAText@CEventXtalOfReflections@@UAE?AW4StringId@@XZ 0045f770 f i IslandEvents.obj
 0001:0005e780       ?GetChoiceBText@CEventXtalOfReflections@@UAE?AW4StringId@@XZ 0045f780 f i IslandEvents.obj
 0001:0005e790       ?CanFire@CEventXtalOfReflections@@UAE_NXZ 0045f790 f i IslandEvents.obj
 0001:0005e7d0       ?GetResultDescription@CEventXtalOfReflections@@UAE?AW4StringId@@H@Z 0045f7d0 f i IslandEvents.obj
 0001:0005e7f0       ?ImpactGame@CEventXtalOfReflections@@UAEXH@Z 0045f7f0 f i IslandEvents.obj
 0001:0005e8d0       ??_GCEventXtalOfReflections@@UAEPAXI@Z 0045f8d0 f i IslandEvents.obj
 0001:0005e8d0       ??_ECEventXtalOfReflections@@UAEPAXI@Z 0045f8d0 f i IslandEvents.obj
 0001:0005e900       ??1CEventXtalOfReflections@@UAE@XZ 0045f900 f i IslandEvents.obj
 0001:0005e920       ??0CEventBitterBrownBeansScience1@@QAE@XZ 0045f920 f i IslandEvents.obj
 0001:0005e940       ?GetTitle@CEventBitterBrownBeansScience1@@UAE?AW4StringId@@XZ 0045f940 f i IslandEvents.obj
 0001:0005e950       ?GetDescription@CEventBitterBrownBeansScience1@@UAE?AW4StringId@@XZ 0045f950 f i IslandEvents.obj
 0001:0005e960       ?GetChoiceAText@CEventBitterBrownBeansScience1@@UAE?AW4StringId@@XZ 0045f960 f i IslandEvents.obj
 0001:0005e970       ?GetChoiceBText@CEventBitterBrownBeansScience1@@UAE?AW4StringId@@XZ 0045f970 f i IslandEvents.obj
 0001:0005e980       ?GetResultDescription@CEventBitterBrownBeansScience1@@UAE?AW4StringId@@H@Z 0045f980 f i IslandEvents.obj
 0001:0005e9a0       ?ImpactGame@CEventBitterBrownBeansScience1@@UAEXH@Z 0045f9a0 f i IslandEvents.obj
 0001:0005eac0       ??_ECEventBitterBrownBeansScience1@@UAEPAXI@Z 0045fac0 f i IslandEvents.obj
 0001:0005eac0       ??_GCEventBitterBrownBeansScience1@@UAEPAXI@Z 0045fac0 f i IslandEvents.obj
 0001:0005eaf0       ??1CEventBitterBrownBeansScience1@@UAE@XZ 0045faf0 f i IslandEvents.obj
 0001:0005eb10       ??0CEventBitterBrownBeansScience2@@QAE@XZ 0045fb10 f i IslandEvents.obj
 0001:0005eb30       ?GetTitle@CEventBitterBrownBeansScience2@@UAE?AW4StringId@@XZ 0045fb30 f i IslandEvents.obj
 0001:0005eb40       ?GetDescription@CEventBitterBrownBeansScience2@@UAE?AW4StringId@@XZ 0045fb40 f i IslandEvents.obj
 0001:0005eb50       ?GetChoiceAText@CEventBitterBrownBeansScience2@@UAE?AW4StringId@@XZ 0045fb50 f i IslandEvents.obj
 0001:0005eb60       ?GetChoiceBText@CEventBitterBrownBeansScience2@@UAE?AW4StringId@@XZ 0045fb60 f i IslandEvents.obj
 0001:0005eb70       ?CanFire@CEventBitterBrownBeansScience2@@UAE_NXZ 0045fb70 f i IslandEvents.obj
 0001:0005ebc0       ?GetResultDescription@CEventBitterBrownBeansScience2@@UAE?AW4StringId@@H@Z 0045fbc0 f i IslandEvents.obj
 0001:0005ebe0       ?ImpactGame@CEventBitterBrownBeansScience2@@UAEXH@Z 0045fbe0 f i IslandEvents.obj
 0001:0005eca0       ??_ECEventBitterBrownBeansScience2@@UAEPAXI@Z 0045fca0 f i IslandEvents.obj
 0001:0005eca0       ??_GCEventBitterBrownBeansScience2@@UAEPAXI@Z 0045fca0 f i IslandEvents.obj
 0001:0005ecd0       ??1CEventBitterBrownBeansScience2@@UAE@XZ 0045fcd0 f i IslandEvents.obj
 0001:0005ecf0       ??0CEventAncientTabletScience1@@QAE@XZ 0045fcf0 f i IslandEvents.obj
 0001:0005ed10       ?GetTitle@CEventAncientTabletScience1@@UAE?AW4StringId@@XZ 0045fd10 f i IslandEvents.obj
 0001:0005ed20       ?GetDescription@CEventAncientTabletScience1@@UAE?AW4StringId@@XZ 0045fd20 f i IslandEvents.obj
 0001:0005ed30       ?GetChoiceAText@CEventAncientTabletScience1@@UAE?AW4StringId@@XZ 0045fd30 f i IslandEvents.obj
 0001:0005ed40       ?GetChoiceBText@CEventAncientTabletScience1@@UAE?AW4StringId@@XZ 0045fd40 f i IslandEvents.obj
 0001:0005ed50       ?CanFire@CEventAncientTabletScience1@@UAE_NXZ 0045fd50 f i IslandEvents.obj
 0001:0005ed50       ?CanFire@CEventBitterBrownBeansScience1@@UAE_NXZ 0045fd50 f i IslandEvents.obj
 0001:0005eda0       ?GetResultDescription@CEventAncientTabletScience1@@UAE?AW4StringId@@H@Z 0045fda0 f i IslandEvents.obj
 0001:0005edc0       ?ImpactGame@CEventAncientTabletScience1@@UAEXH@Z 0045fdc0 f i IslandEvents.obj
 0001:0005ee40       ??_ECEventAncientTabletScience1@@UAEPAXI@Z 0045fe40 f i IslandEvents.obj
 0001:0005ee40       ??_GCEventAncientTabletScience1@@UAEPAXI@Z 0045fe40 f i IslandEvents.obj
 0001:0005ee70       ??1CEventAncientTabletScience1@@UAE@XZ 0045fe70 f i IslandEvents.obj
 0001:0005ee90       ??0CEventAncientTabletScience2@@QAE@XZ 0045fe90 f i IslandEvents.obj
 0001:0005eeb0       ?GetTitle@CEventAncientTabletScience2@@UAE?AW4StringId@@XZ 0045feb0 f i IslandEvents.obj
 0001:0005eec0       ?GetDescription@CEventAncientTabletScience2@@UAE?AW4StringId@@XZ 0045fec0 f i IslandEvents.obj
 0001:0005eed0       ?GetChoiceAText@CEventAncientTabletScience2@@UAE?AW4StringId@@XZ 0045fed0 f i IslandEvents.obj
 0001:0005eee0       ?GetChoiceBText@CEventAncientTabletScience2@@UAE?AW4StringId@@XZ 0045fee0 f i IslandEvents.obj
 0001:0005eef0       ?CanFire@CEventAncientTabletScience2@@UAE_NXZ 0045fef0 f i IslandEvents.obj
 0001:0005ef50       ?GetResultDescription@CEventAncientTabletScience2@@UAE?AW4StringId@@H@Z 0045ff50 f i IslandEvents.obj
 0001:0005ef70       ?CalcAward@CEventAncientTabletScience2@@UAEXH@Z 0045ff70 f i IslandEvents.obj
 0001:0005efc0       ?ImpactGame@CEventAncientTabletScience2@@UAEXH@Z 0045ffc0 f i IslandEvents.obj
 0001:0005f020       ??_GCEventAncientTabletScience2@@UAEPAXI@Z 00460020 f i IslandEvents.obj
 0001:0005f020       ??_ECEventAncientTabletScience2@@UAEPAXI@Z 00460020 f i IslandEvents.obj
 0001:0005f050       ??1CEventAncientTabletScience2@@UAE@XZ 00460050 f i IslandEvents.obj
 0001:0005f070       ??0CEventTheLowTide@@QAE@XZ 00460070 f i IslandEvents.obj
 0001:0005f090       ?GetTitle@CEventTheLowTide@@UAE?AW4StringId@@XZ 00460090 f i IslandEvents.obj
 0001:0005f0a0       ?GetDescription@CEventTheLowTide@@UAE?AW4StringId@@XZ 004600a0 f i IslandEvents.obj
 0001:0005f0b0       ?GetChoiceAText@CEventTheLowTide@@UAE?AW4StringId@@XZ 004600b0 f i IslandEvents.obj
 0001:0005f0c0       ?GetChoiceBText@CEventTheLowTide@@UAE?AW4StringId@@XZ 004600c0 f i IslandEvents.obj
 0001:0005f0d0       ?CanFire@CEventTheLowTide@@UAE_NXZ 004600d0 f i IslandEvents.obj
 0001:0005f130       ?GetResultDescription@CEventTheLowTide@@UAE?AW4StringId@@H@Z 00460130 f i IslandEvents.obj
 0001:0005f160       ?CalcAward@CEventTheLowTide@@UAEXH@Z 00460160 f i IslandEvents.obj
 0001:0005f180       ?ImpactGame@CEventTheLowTide@@UAEXH@Z 00460180 f i IslandEvents.obj
 0001:0005f230       ??_GCEventTheLowTide@@UAEPAXI@Z 00460230 f i IslandEvents.obj
 0001:0005f230       ??_ECEventTheLowTide@@UAEPAXI@Z 00460230 f i IslandEvents.obj
 0001:0005f260       ??1CEventTheLowTide@@UAE@XZ 00460260 f i IslandEvents.obj
 0001:0005f280       ??0CEventAntsAndGranary@@QAE@XZ 00460280 f i IslandEvents.obj
 0001:0005f2a0       ?GetTitle@CEventAntsAndGranary@@UAE?AW4StringId@@XZ 004602a0 f i IslandEvents.obj
 0001:0005f2b0       ?GetDescription@CEventAntsAndGranary@@UAE?AW4StringId@@XZ 004602b0 f i IslandEvents.obj
 0001:0005f2c0       ?GetChoiceAText@CEventAntsAndGranary@@UAE?AW4StringId@@XZ 004602c0 f i IslandEvents.obj
 0001:0005f2d0       ?GetChoiceBText@CEventAntsAndGranary@@UAE?AW4StringId@@XZ 004602d0 f i IslandEvents.obj
 0001:0005f2e0       ?GetResultDescription@CEventAntsAndGranary@@UAE?AW4StringId@@H@Z 004602e0 f i IslandEvents.obj
 0001:0005f300       ?CalcAward@CEventAntsAndGranary@@UAEXH@Z 00460300 f i IslandEvents.obj
 0001:0005f390       ?ImpactGame@CEventAntsAndGranary@@UAEXH@Z 00460390 f i IslandEvents.obj
 0001:0005f450       ??_ECEventAntsAndGranary@@UAEPAXI@Z 00460450 f i IslandEvents.obj
 0001:0005f450       ??_GCEventAntsAndGranary@@UAEPAXI@Z 00460450 f i IslandEvents.obj
 0001:0005f480       ??1CEventAntsAndGranary@@UAE@XZ 00460480 f i IslandEvents.obj
 0001:0005f4a0       ??0CEventTheGreenPearl@@QAE@XZ 004604a0 f i IslandEvents.obj
 0001:0005f4c0       ?GetTitle@CEventTheGreenPearl@@UAE?AW4StringId@@XZ 004604c0 f i IslandEvents.obj
 0001:0005f4d0       ?GetDescription@CEventTheGreenPearl@@UAE?AW4StringId@@XZ 004604d0 f i IslandEvents.obj
 0001:0005f4e0       ?GetChoiceAText@CEventTheGreenPearl@@UAE?AW4StringId@@XZ 004604e0 f i IslandEvents.obj
 0001:0005f4f0       ?GetChoiceBText@CEventTheGreenPearl@@UAE?AW4StringId@@XZ 004604f0 f i IslandEvents.obj
 0001:0005f500       ?GetResultDescription@CEventTheGreenPearl@@UAE?AW4StringId@@H@Z 00460500 f i IslandEvents.obj
 0001:0005f520       ?ImpactGame@CEventTheGreenPearl@@UAEXH@Z 00460520 f i IslandEvents.obj
 0001:0005f5e0       ??_ECEventTheGreenPearl@@UAEPAXI@Z 004605e0 f i IslandEvents.obj
 0001:0005f5e0       ??_GCEventTheGreenPearl@@UAEPAXI@Z 004605e0 f i IslandEvents.obj
 0001:0005f610       ??1CEventTheGreenPearl@@UAE@XZ 00460610 f i IslandEvents.obj
 0001:0005f630       ??0CEventTheBluePearl@@QAE@XZ 00460630 f i IslandEvents.obj
 0001:0005f650       ?GetTitle@CEventTheBluePearl@@UAE?AW4StringId@@XZ 00460650 f i IslandEvents.obj
 0001:0005f660       ?GetDescription@CEventTheBluePearl@@UAE?AW4StringId@@XZ 00460660 f i IslandEvents.obj
 0001:0005f670       ?GetChoiceAText@CEventTheBluePearl@@UAE?AW4StringId@@XZ 00460670 f i IslandEvents.obj
 0001:0005f680       ?GetChoiceBText@CEventTheBluePearl@@UAE?AW4StringId@@XZ 00460680 f i IslandEvents.obj
 0001:0005f690       ?CanFire@CEventTheBluePearl@@UAE_NXZ 00460690 f i IslandEvents.obj
 0001:0005f6e0       ?GetResultDescription@CEventTheBluePearl@@UAE?AW4StringId@@H@Z 004606e0 f i IslandEvents.obj
 0001:0005f700       ?ImpactGame@CEventTheBluePearl@@UAEXH@Z 00460700 f i IslandEvents.obj
 0001:0005f7a0       ??_ECEventTheBluePearl@@UAEPAXI@Z 004607a0 f i IslandEvents.obj
 0001:0005f7a0       ??_GCEventTheBluePearl@@UAEPAXI@Z 004607a0 f i IslandEvents.obj
 0001:0005f7d0       ??1CEventTheBluePearl@@UAE@XZ 004607d0 f i IslandEvents.obj
 0001:0005f7f0       ??0CEventTheLazyApprentice@@QAE@XZ 004607f0 f i IslandEvents.obj
 0001:0005f810       ?GetTitle@CEventTheLazyApprentice@@UAE?AW4StringId@@XZ 00460810 f i IslandEvents.obj
 0001:0005f820       ?GetDescription@CEventTheLazyApprentice@@UAE?AW4StringId@@XZ 00460820 f i IslandEvents.obj
 0001:0005f830       ?GetChoiceAText@CEventTheLazyApprentice@@UAE?AW4StringId@@XZ 00460830 f i IslandEvents.obj
 0001:0005f840       ?GetChoiceBText@CEventTheLazyApprentice@@UAE?AW4StringId@@XZ 00460840 f i IslandEvents.obj
 0001:0005f850       ?CanFire@CEventTheLazyApprentice@@UAE_NXZ 00460850 f i IslandEvents.obj
 0001:0005f8b0       ?GetVillagerPose@CEventTheReturnOfBiggles@@UAE?AW4EBodyPosition@@XZ 004608b0 f i IslandEvents.obj
 0001:0005f8b0       ?GetVillagerPose@CEventTheGreenPearl@@UAE?AW4EBodyPosition@@XZ 004608b0 f i IslandEvents.obj
 0001:0005f8b0       ?GetVillagerPose@CEventTheShootingStar@@UAE?AW4EBodyPosition@@XZ 004608b0 f i IslandEvents.obj
 0001:0005f8b0       ?GetVillagerPose@CEventTheLazyApprentice@@UAE?AW4EBodyPosition@@XZ 004608b0 f i IslandEvents.obj
 0001:0005f8b0       ?GetVillagerPose@CEventTheLoversMale@@UAE?AW4EBodyPosition@@XZ 004608b0 f i IslandEvents.obj
 0001:0005f8b0       ?GetVillagerPose@CEventTheNoisyBird@@UAE?AW4EBodyPosition@@XZ 004608b0 f i IslandEvents.obj
 0001:0005f8b0       ?GetVillagerPose@CEventTheHoleInTheHut@@UAE?AW4EBodyPosition@@XZ 004608b0 f i IslandEvents.obj
 0001:0005f8b0       ?GetVillagerPose@CEventTheLoversFemale@@UAE?AW4EBodyPosition@@XZ 004608b0 f i IslandEvents.obj
 0001:0005f8b0       ?GetVillagerPose@CEventTheBee@@UAE?AW4EBodyPosition@@XZ 004608b0 f i IslandEvents.obj
 0001:0005f8b0       ?GetVillagerPose@CEventTheAntHill@@UAE?AW4EBodyPosition@@XZ 004608b0 f i IslandEvents.obj
 0001:0005f8b0       ?GetVillagerPose@CEventTheMedicalEmergency@@UAE?AW4EBodyPosition@@XZ 004608b0 f i IslandEvents.obj
 0001:0005f8b0       ?GetVillagerPose@CEventTheRoyalJelly@@UAE?AW4EBodyPosition@@XZ 004608b0 f i IslandEvents.obj
 0001:0005f8b0       ?GetVillagerPose@CEventTheRedStarfish@@UAE?AW4EBodyPosition@@XZ 004608b0 f i IslandEvents.obj
 0001:0005f8b0       ?GetVillagerPose@CEventThePlayfulOtters@@UAE?AW4EBodyPosition@@XZ 004608b0 f i IslandEvents.obj
 0001:0005f8b0       ?GetVillagerPose@CEventTheBlueStarfish@@UAE?AW4EBodyPosition@@XZ 004608b0 f i IslandEvents.obj
 0001:0005f8b0       ?GetVillagerPose@CEventTheBluePearl@@UAE?AW4EBodyPosition@@XZ 004608b0 f i IslandEvents.obj
 0001:0005f8c0       ?GetResultDescription@CEventTheLazyApprentice@@UAE?AW4StringId@@H@Z 004608c0 f i IslandEvents.obj
 0001:0005f8e0       ?ImpactGame@CEventTheLazyApprentice@@UAEXH@Z 004608e0 f i IslandEvents.obj
 0001:0005f990       ??_ECEventTheLazyApprentice@@UAEPAXI@Z 00460990 f i IslandEvents.obj
 0001:0005f990       ??_GCEventTheLazyApprentice@@UAEPAXI@Z 00460990 f i IslandEvents.obj
 0001:0005f9c0       ??1CEventTheLazyApprentice@@UAE@XZ 004609c0 f i IslandEvents.obj
 0001:0005f9e0       ??0CEventTheOmenInTheClouds@@QAE@XZ 004609e0 f i IslandEvents.obj
 0001:0005fa00       ?GetTitle@CEventTheOmenInTheClouds@@UAE?AW4StringId@@XZ 00460a00 f i IslandEvents.obj
 0001:0005fa10       ?GetDescription@CEventTheOmenInTheClouds@@UAE?AW4StringId@@XZ 00460a10 f i IslandEvents.obj
 0001:0005fa20       ?GetChoiceAText@CEventTheOmenInTheClouds@@UAE?AW4StringId@@XZ 00460a20 f i IslandEvents.obj
 0001:0005fa30       ?GetChoiceBText@CEventTheOmenInTheClouds@@UAE?AW4StringId@@XZ 00460a30 f i IslandEvents.obj
 0001:0005fa40       ?CanFire@CEventTheOmenInTheClouds@@UAE_NXZ 00460a40 f i IslandEvents.obj
 0001:0005fa90       ?GetResultDescription@CEventTheOmenInTheClouds@@UAE?AW4StringId@@H@Z 00460a90 f i IslandEvents.obj
 0001:0005fae0       ?CalcAward@CEventTheOmenInTheClouds@@UAEXH@Z 00460ae0 f i IslandEvents.obj
 0001:0005fba0       ?ImpactGame@CEventTheOmenInTheClouds@@UAEXH@Z 00460ba0 f i IslandEvents.obj
 0001:0005fd20       ??_ECEventTheOmenInTheClouds@@UAEPAXI@Z 00460d20 f i IslandEvents.obj
 0001:0005fd20       ??_GCEventTheOmenInTheClouds@@UAEPAXI@Z 00460d20 f i IslandEvents.obj
 0001:0005fd50       ??1CEventTheOmenInTheClouds@@UAE@XZ 00460d50 f i IslandEvents.obj
 0001:0005fd70       ??0CEventThePlayfulOtters@@QAE@XZ 00460d70 f i IslandEvents.obj
 0001:0005fd90       ?GetTitle@CEventThePlayfulOtters@@UAE?AW4StringId@@XZ 00460d90 f i IslandEvents.obj
 0001:0005fda0       ?GetDescription@CEventThePlayfulOtters@@UAE?AW4StringId@@XZ 00460da0 f i IslandEvents.obj
 0001:0005fdb0       ?GetChoiceAText@CEventThePlayfulOtters@@UAE?AW4StringId@@XZ 00460db0 f i IslandEvents.obj
 0001:0005fdc0       ?GetChoiceBText@CEventThePlayfulOtters@@UAE?AW4StringId@@XZ 00460dc0 f i IslandEvents.obj
 0001:0005fdd0       ?GetResultDescription@CEventThePlayfulOtters@@UAE?AW4StringId@@H@Z 00460dd0 f i IslandEvents.obj
 0001:0005fdf0       ?CalcAward@CEventThePlayfulOtters@@UAEXH@Z 00460df0 f i IslandEvents.obj
 0001:0005fe50       ?ImpactGame@CEventThePlayfulOtters@@UAEXH@Z 00460e50 f i IslandEvents.obj
 0001:0005ff30       ??_GCEventThePlayfulOtters@@UAEPAXI@Z 00460f30 f i IslandEvents.obj
 0001:0005ff30       ??_ECEventThePlayfulOtters@@UAEPAXI@Z 00460f30 f i IslandEvents.obj
 0001:0005ff60       ??1CEventThePlayfulOtters@@UAE@XZ 00460f60 f i IslandEvents.obj
 0001:0005ff80       ??0CEventTheAntHill@@QAE@XZ 00460f80 f i IslandEvents.obj
 0001:0005ffa0       ?GetTitle@CEventTheAntHill@@UAE?AW4StringId@@XZ 00460fa0 f i IslandEvents.obj
 0001:0005ffb0       ?GetDescription@CEventTheAntHill@@UAE?AW4StringId@@XZ 00460fb0 f i IslandEvents.obj
 0001:0005ffc0       ?GetChoiceAText@CEventTheAntHill@@UAE?AW4StringId@@XZ 00460fc0 f i IslandEvents.obj
 0001:0005ffd0       ?GetChoiceBText@CEventTheAntHill@@UAE?AW4StringId@@XZ 00460fd0 f i IslandEvents.obj
 0001:0005ffe0       ?GetResultDescription@CEventTheAntHill@@UAE?AW4StringId@@H@Z 00460fe0 f i IslandEvents.obj
 0001:00060000       ?CalcAward@CEventTheAntHill@@UAEXH@Z 00461000 f i IslandEvents.obj
 0001:00060060       ?ImpactGame@CEventTheAntHill@@UAEXH@Z 00461060 f i IslandEvents.obj
 0001:00060140       ??_ECEventTheAntHill@@UAEPAXI@Z 00461140 f i IslandEvents.obj
 0001:00060140       ??_GCEventTheAntHill@@UAEPAXI@Z 00461140 f i IslandEvents.obj
 0001:00060170       ??1CEventTheAntHill@@UAE@XZ 00461170 f i IslandEvents.obj
 0001:00060190       ??0CEventTheRedStarfish@@QAE@XZ 00461190 f i IslandEvents.obj
 0001:000601b0       ?GetTitle@CEventTheRedStarfish@@UAE?AW4StringId@@XZ 004611b0 f i IslandEvents.obj
 0001:000601c0       ?GetDescription@CEventTheRedStarfish@@UAE?AW4StringId@@XZ 004611c0 f i IslandEvents.obj
 0001:000601d0       ?GetChoiceAText@CEventTheRedStarfish@@UAE?AW4StringId@@XZ 004611d0 f i IslandEvents.obj
 0001:000601e0       ?GetChoiceBText@CEventTheRedStarfish@@UAE?AW4StringId@@XZ 004611e0 f i IslandEvents.obj
 0001:000601f0       ?CanFire@CEventTheRedStarfish@@UAE_NXZ 004611f0 f i IslandEvents.obj
 0001:000601f0       ?CanFire@CEventTheGreenPearl@@UAE_NXZ 004611f0 f i IslandEvents.obj
 0001:000601f0       ?CanFire@CEventTheBlueStarfish@@UAE_NXZ 004611f0 f i IslandEvents.obj
 0001:000601f0       ?CanFire@CEventTheRoyalJelly@@UAE_NXZ 004611f0 f i IslandEvents.obj
 0001:000601f0       ?CanFire@CEventTheAntInTheBed@@UAE_NXZ 004611f0 f i IslandEvents.obj
 0001:00060230       ?GetResultDescription@CEventTheRedStarfish@@UAE?AW4StringId@@H@Z 00461230 f i IslandEvents.obj
 0001:00060250       ?ImpactGame@CEventTheRedStarfish@@UAEXH@Z 00461250 f i IslandEvents.obj
 0001:000602e0       ??_GCEventTheRedStarfish@@UAEPAXI@Z 004612e0 f i IslandEvents.obj
 0001:000602e0       ??_ECEventTheRedStarfish@@UAEPAXI@Z 004612e0 f i IslandEvents.obj
 0001:00060310       ??1CEventTheRedStarfish@@UAE@XZ 00461310 f i IslandEvents.obj
 0001:00060330       ??0CEventTheBlueStarfish@@QAE@XZ 00461330 f i IslandEvents.obj
 0001:00060350       ?GetTitle@CEventTheBlueStarfish@@UAE?AW4StringId@@XZ 00461350 f i IslandEvents.obj
 0001:00060360       ?GetDescription@CEventTheBlueStarfish@@UAE?AW4StringId@@XZ 00461360 f i IslandEvents.obj
 0001:00060370       ?GetChoiceAText@CEventTheBlueStarfish@@UAE?AW4StringId@@XZ 00461370 f i IslandEvents.obj
 0001:00060380       ?GetChoiceBText@CEventTheBlueStarfish@@UAE?AW4StringId@@XZ 00461380 f i IslandEvents.obj
 0001:00060390       ?GetResultDescription@CEventTheBlueStarfish@@UAE?AW4StringId@@H@Z 00461390 f i IslandEvents.obj
 0001:000603b0       ?ImpactGame@CEventTheBlueStarfish@@UAEXH@Z 004613b0 f i IslandEvents.obj
 0001:00060440       ??_GCEventTheBlueStarfish@@UAEPAXI@Z 00461440 f i IslandEvents.obj
 0001:00060440       ??_ECEventTheBlueStarfish@@UAEPAXI@Z 00461440 f i IslandEvents.obj
 0001:00060470       ??1CEventTheBlueStarfish@@UAE@XZ 00461470 f i IslandEvents.obj
 0001:00060490       ??0CEventTheAntInTheBed@@QAE@XZ 00461490 f i IslandEvents.obj
 0001:000604b0       ?GetTitle@CEventTheAntInTheBed@@UAE?AW4StringId@@XZ 004614b0 f i IslandEvents.obj
 0001:000604c0       ?GetDescription@CEventTheAntInTheBed@@UAE?AW4StringId@@XZ 004614c0 f i IslandEvents.obj
 0001:000604d0       ?GetChoiceAText@CEventTheAntInTheBed@@UAE?AW4StringId@@XZ 004614d0 f i IslandEvents.obj
 0001:000604e0       ?GetChoiceBText@CEventTheAntInTheBed@@UAE?AW4StringId@@XZ 004614e0 f i IslandEvents.obj
 0001:000604f0       ?GetResultDescription@CEventTheAntInTheBed@@UAE?AW4StringId@@H@Z 004614f0 f i IslandEvents.obj
 0001:00060510       ?ImpactGame@CEventTheAntInTheBed@@UAEXH@Z 00461510 f i IslandEvents.obj
 0001:000605c0       ??_ECEventTheAntInTheBed@@UAEPAXI@Z 004615c0 f i IslandEvents.obj
 0001:000605c0       ??_GCEventTheAntInTheBed@@UAEPAXI@Z 004615c0 f i IslandEvents.obj
 0001:000605f0       ??1CEventTheAntInTheBed@@UAE@XZ 004615f0 f i IslandEvents.obj
 0001:00060610       ??0CEventTheLoversFemale@@QAE@XZ 00461610 f i IslandEvents.obj
 0001:00060630       ?GetTitle@CEventTheLoversFemale@@UAE?AW4StringId@@XZ 00461630 f i IslandEvents.obj
 0001:00060640       ?GetDescription@CEventTheLoversFemale@@UAE?AW4StringId@@XZ 00461640 f i IslandEvents.obj
 0001:00060650       ?GetChoiceAText@CEventTheLoversFemale@@UAE?AW4StringId@@XZ 00461650 f i IslandEvents.obj
 0001:00060660       ?GetChoiceBText@CEventTheLoversFemale@@UAE?AW4StringId@@XZ 00461660 f i IslandEvents.obj
 0001:00060670       ?CanFire@CEventTheLoversFemale@@UAE_NXZ 00461670 f i IslandEvents.obj
 0001:000606d0       ?GetResultDescription@CEventTheLoversFemale@@UAE?AW4StringId@@H@Z 004616d0 f i IslandEvents.obj
 0001:000606f0       ?ImpactGame@CEventTheLoversFemale@@UAEXH@Z 004616f0 f i IslandEvents.obj
 0001:000607b0       ??_GCEventTheLoversFemale@@UAEPAXI@Z 004617b0 f i IslandEvents.obj
 0001:000607b0       ??_ECEventTheLoversFemale@@UAEPAXI@Z 004617b0 f i IslandEvents.obj
 0001:000607e0       ??1CEventTheLoversFemale@@UAE@XZ 004617e0 f i IslandEvents.obj
 0001:00060800       ??0CEventTheLoversMale@@QAE@XZ 00461800 f i IslandEvents.obj
 0001:00060820       ?GetTitle@CEventTheLoversMale@@UAE?AW4StringId@@XZ 00461820 f i IslandEvents.obj
 0001:00060830       ?GetDescription@CEventTheLoversMale@@UAE?AW4StringId@@XZ 00461830 f i IslandEvents.obj
 0001:00060840       ?GetChoiceAText@CEventTheLoversMale@@UAE?AW4StringId@@XZ 00461840 f i IslandEvents.obj
 0001:00060850       ?GetChoiceBText@CEventTheLoversMale@@UAE?AW4StringId@@XZ 00461850 f i IslandEvents.obj
 0001:00060860       ?CanFire@CEventTheLoversMale@@UAE_NXZ 00461860 f i IslandEvents.obj
 0001:000608c0       ?GetResultDescription@CEventTheLoversMale@@UAE?AW4StringId@@H@Z 004618c0 f i IslandEvents.obj
 0001:000608e0       ?ImpactGame@CEventTheLoversMale@@UAEXH@Z 004618e0 f i IslandEvents.obj
 0001:000609a0       ??_ECEventTheLoversMale@@UAEPAXI@Z 004619a0 f i IslandEvents.obj
 0001:000609a0       ??_GCEventTheLoversMale@@UAEPAXI@Z 004619a0 f i IslandEvents.obj
 0001:000609d0       ??1CEventTheLoversMale@@UAE@XZ 004619d0 f i IslandEvents.obj
 0001:000609f0       ??0CEventTheMedicalEmergency@@QAE@XZ 004619f0 f i IslandEvents.obj
 0001:00060a10       ?GetTitle@CEventTheMedicalEmergency@@UAE?AW4StringId@@XZ 00461a10 f i IslandEvents.obj
 0001:00060a20       ?GetDescription@CEventTheMedicalEmergency@@UAE?AW4StringId@@XZ 00461a20 f i IslandEvents.obj
 0001:00060a30       ?GetChoiceAText@CEventTheMedicalEmergency@@UAE?AW4StringId@@XZ 00461a30 f i IslandEvents.obj
 0001:00060a40       ?GetChoiceBText@CEventTheMedicalEmergency@@UAE?AW4StringId@@XZ 00461a40 f i IslandEvents.obj
 0001:00060a50       ?CanFire@CEventTheMedicalEmergency@@UAE_NXZ 00461a50 f i IslandEvents.obj
 0001:00060ac0       ?GetResultDescription@CEventTheMedicalEmergency@@UAE?AW4StringId@@H@Z 00461ac0 f i IslandEvents.obj
 0001:00060b10       ?ImpactGame@CEventTheMedicalEmergency@@UAEXH@Z 00461b10 f i IslandEvents.obj
 0001:00060bb0       ??_GCEventTheMedicalEmergency@@UAEPAXI@Z 00461bb0 f i IslandEvents.obj
 0001:00060bb0       ??_ECEventTheMedicalEmergency@@UAEPAXI@Z 00461bb0 f i IslandEvents.obj
 0001:00060be0       ??1CEventTheMedicalEmergency@@UAE@XZ 00461be0 f i IslandEvents.obj
 0001:00060c00       ??0CEventTheQuartzPhial@@QAE@XZ 00461c00 f i IslandEvents.obj
 0001:00060c20       ?GetTitle@CEventTheQuartzPhial@@UAE?AW4StringId@@XZ 00461c20 f i IslandEvents.obj
 0001:00060c30       ?GetDescription@CEventTheQuartzPhial@@UAE?AW4StringId@@XZ 00461c30 f i IslandEvents.obj
 0001:00060c40       ?GetChoiceAText@CEventTheQuartzPhial@@UAE?AW4StringId@@XZ 00461c40 f i IslandEvents.obj
 0001:00060c50       ?GetChoiceBText@CEventTheQuartzPhial@@UAE?AW4StringId@@XZ 00461c50 f i IslandEvents.obj
 0001:00060c60       ?CanFire@CEventTheQuartzPhial@@UAE_NXZ 00461c60 f i IslandEvents.obj
 0001:00060ca0       ?GetVillagerPose@CEventTheQuartzPhial@@UAE?AW4EBodyPosition@@XZ 00461ca0 f i IslandEvents.obj
 0001:00060cb0       ?GetResultDescription@CEventTheQuartzPhial@@UAE?AW4StringId@@H@Z 00461cb0 f i IslandEvents.obj
 0001:00060d40       ?ImpactGame@CEventTheQuartzPhial@@UAEXH@Z 00461d40 f i IslandEvents.obj
 0001:00060ec0       ??_GCEventTheQuartzPhial@@UAEPAXI@Z 00461ec0 f i IslandEvents.obj
 0001:00060ec0       ??_ECEventTheQuartzPhial@@UAEPAXI@Z 00461ec0 f i IslandEvents.obj
 0001:00060ef0       ??1CEventTheQuartzPhial@@UAE@XZ 00461ef0 f i IslandEvents.obj
 0001:00060f10       ??0CEventTheObsidianPhial@@QAE@XZ 00461f10 f i IslandEvents.obj
 0001:00060f30       ?GetTitle@CEventTheObsidianPhial@@UAE?AW4StringId@@XZ 00461f30 f i IslandEvents.obj
 0001:00060f40       ?GetDescription@CEventTheObsidianPhial@@UAE?AW4StringId@@XZ 00461f40 f i IslandEvents.obj
 0001:00060f50       ?GetChoiceAText@CEventTheObsidianPhial@@UAE?AW4StringId@@XZ 00461f50 f i IslandEvents.obj
 0001:00060f60       ?GetChoiceBText@CEventTheObsidianPhial@@UAE?AW4StringId@@XZ 00461f60 f i IslandEvents.obj
 0001:00060f70       ?GetResultDescription@CEventTheObsidianPhial@@UAE?AW4StringId@@H@Z 00461f70 f i IslandEvents.obj
 0001:00060fe0       ?ImpactGame@CEventTheObsidianPhial@@UAEXH@Z 00461fe0 f i IslandEvents.obj
 0001:000610a0       ??_GCEventTheObsidianPhial@@UAEPAXI@Z 004620a0 f i IslandEvents.obj
 0001:000610a0       ??_ECEventTheObsidianPhial@@UAEPAXI@Z 004620a0 f i IslandEvents.obj
 0001:000610d0       ??1CEventTheObsidianPhial@@UAE@XZ 004620d0 f i IslandEvents.obj
 0001:000610f0       ??0CEventTheAmberPhial@@QAE@XZ 004620f0 f i IslandEvents.obj
 0001:00061110       ?GetTitle@CEventTheAmberPhial@@UAE?AW4StringId@@XZ 00462110 f i IslandEvents.obj
 0001:00061120       ?GetDescription@CEventTheAmberPhial@@UAE?AW4StringId@@XZ 00462120 f i IslandEvents.obj
 0001:00061130       ?GetChoiceAText@CEventTheAmberPhial@@UAE?AW4StringId@@XZ 00462130 f i IslandEvents.obj
 0001:00061140       ?GetChoiceBText@CEventTheAmberPhial@@UAE?AW4StringId@@XZ 00462140 f i IslandEvents.obj
 0001:00061150       ?CanFire@CEventTheObsidianPhial@@UAE_NXZ 00462150 f i IslandEvents.obj
 0001:00061150       ?CanFire@CEventTheAmberPhial@@UAE_NXZ 00462150 f i IslandEvents.obj
 0001:00061190       ?GetResultDescription@CEventTheAmberPhial@@UAE?AW4StringId@@H@Z 00462190 f i IslandEvents.obj
 0001:00061200       ?ImpactGame@CEventTheAmberPhial@@UAEXH@Z 00462200 f i IslandEvents.obj
 0001:00061330       ??_GCEventTheAmberPhial@@UAEPAXI@Z 00462330 f i IslandEvents.obj
 0001:00061330       ??_ECEventTheAmberPhial@@UAEPAXI@Z 00462330 f i IslandEvents.obj
 0001:00061360       ??1CEventTheAmberPhial@@UAE@XZ 00462360 f i IslandEvents.obj
 0001:00061380       ??0CEventTheMangoAndThePapaya@@QAE@XZ 00462380 f i IslandEvents.obj
 0001:000613a0       ?GetTitle@CEventTheMangoAndThePapaya@@UAE?AW4StringId@@XZ 004623a0 f i IslandEvents.obj
 0001:000613b0       ?GetDescription@CEventTheMangoAndThePapaya@@UAE?AW4StringId@@XZ 004623b0 f i IslandEvents.obj
 0001:000613c0       ?GetChoiceAText@CEventTheMangoAndThePapaya@@UAE?AW4StringId@@XZ 004623c0 f i IslandEvents.obj
 0001:000613d0       ?GetChoiceBText@CEventTheMangoAndThePapaya@@UAE?AW4StringId@@XZ 004623d0 f i IslandEvents.obj
 0001:000613e0       ?CanFire@CEventTheMangoAndThePapaya@@UAE_NXZ 004623e0 f i IslandEvents.obj
 0001:00061430       ?GetVillagerPose@CEventAncientTabletScience1@@UAE?AW4EBodyPosition@@XZ 00462430 f i IslandEvents.obj
 0001:00061430       ?GetVillagerPose@CEventBitterBrownBeansScience2@@UAE?AW4EBodyPosition@@XZ 00462430 f i IslandEvents.obj
 0001:00061430       ?GetVillagerPose@CEventAncientTabletScience2@@UAE?AW4EBodyPosition@@XZ 00462430 f i IslandEvents.obj
 0001:00061430       ?GetVillagerPose@CEventTheLowTide@@UAE?AW4EBodyPosition@@XZ 00462430 f i IslandEvents.obj
 0001:00061430       ?GetVillagerPose@CEventBitterBrownBeansScience1@@UAE?AW4EBodyPosition@@XZ 00462430 f i IslandEvents.obj
 0001:00061430       ?GetVillagerPose@CEventTheObsidianPhial@@UAE?AW4EBodyPosition@@XZ 00462430 f i IslandEvents.obj
 0001:00061430       ?GetVillagerPose@CEventTheMangoAndThePapaya@@UAE?AW4EBodyPosition@@XZ 00462430 f i IslandEvents.obj
 0001:00061430       ?GetVillagerPose@CEventAntsAndGranary@@UAE?AW4EBodyPosition@@XZ 00462430 f i IslandEvents.obj
 0001:00061430       ?GetVillagerPose@CEventTheCrateOfMangosPapayasAndBananas@@UAE?AW4EBodyPosition@@XZ 00462430 f i IslandEvents.obj
 0001:00061430       ?GetVillagerPose@CEventTheAmberPhial@@UAE?AW4EBodyPosition@@XZ 00462430 f i IslandEvents.obj
 0001:00061430       ?GetVillagerPose@CEventXtalOfReflections@@UAE?AW4EBodyPosition@@XZ 00462430 f i IslandEvents.obj
 0001:00061430       ?GetVillagerPose@CEventTheOmenInTheClouds@@UAE?AW4EBodyPosition@@XZ 00462430 f i IslandEvents.obj
 0001:00061430       ?GetVillagerPose@CEventDaredevil@@UAE?AW4EBodyPosition@@XZ 00462430 f i IslandEvents.obj
 0001:00061440       ?GetResultDescription@CEventTheMangoAndThePapaya@@UAE?AW4StringId@@H@Z 00462440 f i IslandEvents.obj
 0001:00061470       ?CalcAward@CEventTheMangoAndThePapaya@@UAEXH@Z 00462470 f i IslandEvents.obj
 0001:000614b0       ?ImpactGame@CEventTheMangoAndThePapaya@@UAEXH@Z 004624b0 f i IslandEvents.obj
 0001:00061580       ??_GCEventTheMangoAndThePapaya@@UAEPAXI@Z 00462580 f i IslandEvents.obj
 0001:00061580       ??_ECEventTheMangoAndThePapaya@@UAEPAXI@Z 00462580 f i IslandEvents.obj
 0001:000615b0       ??1CEventTheMangoAndThePapaya@@UAE@XZ 004625b0 f i IslandEvents.obj
 0001:000615d0       ??0CEventTheCrateOfMangosPapayasAndBananas@@QAE@XZ 004625d0 f i IslandEvents.obj
 0001:000615f0       ?GetTitle@CEventTheCrateOfMangosPapayasAndBananas@@UAE?AW4StringId@@XZ 004625f0 f i IslandEvents.obj
 0001:00061600       ?GetDescription@CEventTheCrateOfMangosPapayasAndBananas@@UAE?AW4StringId@@XZ 00462600 f i IslandEvents.obj
 0001:00061610       ?GetChoiceAText@CEventTheCrateOfMangosPapayasAndBananas@@UAE?AW4StringId@@XZ 00462610 f i IslandEvents.obj
 0001:00061620       ?GetChoiceBText@CEventTheCrateOfMangosPapayasAndBananas@@UAE?AW4StringId@@XZ 00462620 f i IslandEvents.obj
 0001:00061630       ?CanFire@CEventTheCrateOfMangosPapayasAndBananas@@UAE_NXZ 00462630 f i IslandEvents.obj
 0001:00061670       ?GetResultDescription@CEventTheCrateOfMangosPapayasAndBananas@@UAE?AW4StringId@@H@Z 00462670 f i IslandEvents.obj
 0001:000616c0       ?ImpactGame@CEventTheCrateOfMangosPapayasAndBananas@@UAEXH@Z 004626c0 f i IslandEvents.obj
 0001:000618c0       ??_GCEventTheCrateOfMangosPapayasAndBananas@@UAEPAXI@Z 004628c0 f i IslandEvents.obj
 0001:000618c0       ??_ECEventTheCrateOfMangosPapayasAndBananas@@UAEPAXI@Z 004628c0 f i IslandEvents.obj
 0001:000618f0       ??1CEventTheCrateOfMangosPapayasAndBananas@@UAE@XZ 004628f0 f i IslandEvents.obj
 0001:00061910       ??0CEventTheBee@@QAE@XZ    00462910 f i IslandEvents.obj
 0001:00061930       ?GetTitle@CEventTheBee@@UAE?AW4StringId@@XZ 00462930 f i IslandEvents.obj
 0001:00061940       ?GetDescription@CEventTheBee@@UAE?AW4StringId@@XZ 00462940 f i IslandEvents.obj
 0001:00061950       ?GetChoiceAText@CEventTheBee@@UAE?AW4StringId@@XZ 00462950 f i IslandEvents.obj
 0001:00061960       ?GetChoiceBText@CEventTheBee@@UAE?AW4StringId@@XZ 00462960 f i IslandEvents.obj
 0001:00061970       ?CanFire@CEventTheBee@@UAE_NXZ 00462970 f i IslandEvents.obj
 0001:00061970       ?CanFire@CEventTheNoisyBird@@UAE_NXZ 00462970 f i IslandEvents.obj
 0001:000619b0       ?GetResultDescription@CEventTheBee@@UAE?AW4StringId@@H@Z 004629b0 f i IslandEvents.obj
 0001:000619d0       ?ImpactGame@CEventTheBee@@UAEXH@Z 004629d0 f i IslandEvents.obj
 0001:00061aa0       ??_GCEventTheBee@@UAEPAXI@Z 00462aa0 f i IslandEvents.obj
 0001:00061aa0       ??_ECEventTheBee@@UAEPAXI@Z 00462aa0 f i IslandEvents.obj
 0001:00061ad0       ??1CEventTheBee@@UAE@XZ    00462ad0 f i IslandEvents.obj
 0001:00061af0       ??0CEventTheNoisyBird@@QAE@XZ 00462af0 f i IslandEvents.obj
 0001:00061b10       ?GetTitle@CEventTheNoisyBird@@UAE?AW4StringId@@XZ 00462b10 f i IslandEvents.obj
 0001:00061b20       ?GetDescription@CEventTheNoisyBird@@UAE?AW4StringId@@XZ 00462b20 f i IslandEvents.obj
 0001:00061b30       ?GetChoiceAText@CEventTheNoisyBird@@UAE?AW4StringId@@XZ 00462b30 f i IslandEvents.obj
 0001:00061b40       ?GetChoiceBText@CEventTheNoisyBird@@UAE?AW4StringId@@XZ 00462b40 f i IslandEvents.obj
 0001:00061b50       ?GetResultDescription@CEventTheNoisyBird@@UAE?AW4StringId@@H@Z 00462b50 f i IslandEvents.obj
 0001:00061b70       ?ImpactGame@CEventTheNoisyBird@@UAEXH@Z 00462b70 f i IslandEvents.obj
 0001:00061c00       ??_GCEventTheNoisyBird@@UAEPAXI@Z 00462c00 f i IslandEvents.obj
 0001:00061c00       ??_ECEventTheNoisyBird@@UAEPAXI@Z 00462c00 f i IslandEvents.obj
 0001:00061c30       ??1CEventTheNoisyBird@@UAE@XZ 00462c30 f i IslandEvents.obj
 0001:00061c50       ??0CEventTheHoleInTheHut@@QAE@XZ 00462c50 f i IslandEvents.obj
 0001:00061c70       ?GetTitle@CEventTheHoleInTheHut@@UAE?AW4StringId@@XZ 00462c70 f i IslandEvents.obj
 0001:00061c80       ?GetDescription@CEventTheHoleInTheHut@@UAE?AW4StringId@@XZ 00462c80 f i IslandEvents.obj
 0001:00061c90       ?GetChoiceAText@CEventTheHoleInTheHut@@UAE?AW4StringId@@XZ 00462c90 f i IslandEvents.obj
 0001:00061ca0       ?GetChoiceBText@CEventTheHoleInTheHut@@UAE?AW4StringId@@XZ 00462ca0 f i IslandEvents.obj
 0001:00061cb0       ?CanFire@CEventTheHoleInTheHut@@UAE_NXZ 00462cb0 f i IslandEvents.obj
 0001:00061d00       ?GetResultDescription@CEventTheHoleInTheHut@@UAE?AW4StringId@@H@Z 00462d00 f i IslandEvents.obj
 0001:00061d20       ?ImpactGame@CEventTheHoleInTheHut@@UAEXH@Z 00462d20 f i IslandEvents.obj
 0001:00061e00       ??_ECEventTheHoleInTheHut@@UAEPAXI@Z 00462e00 f i IslandEvents.obj
 0001:00061e00       ??_GCEventTheHoleInTheHut@@UAEPAXI@Z 00462e00 f i IslandEvents.obj
 0001:00061e30       ??1CEventTheHoleInTheHut@@UAE@XZ 00462e30 f i IslandEvents.obj
 0001:00061e50       ??0CEventTheRoyalJelly@@QAE@XZ 00462e50 f i IslandEvents.obj
 0001:00061e70       ?GetTitle@CEventTheRoyalJelly@@UAE?AW4StringId@@XZ 00462e70 f i IslandEvents.obj
 0001:00061e80       ?GetDescription@CEventTheRoyalJelly@@UAE?AW4StringId@@XZ 00462e80 f i IslandEvents.obj
 0001:00061e90       ?GetChoiceAText@CEventTheRoyalJelly@@UAE?AW4StringId@@XZ 00462e90 f i IslandEvents.obj
 0001:00061ea0       ?GetChoiceBText@CEventTheRoyalJelly@@UAE?AW4StringId@@XZ 00462ea0 f i IslandEvents.obj
 0001:00061eb0       ?GetResultDescription@CEventTheRoyalJelly@@UAE?AW4StringId@@H@Z 00462eb0 f i IslandEvents.obj
 0001:00061ed0       ?ImpactGame@CEventTheRoyalJelly@@UAEXH@Z 00462ed0 f i IslandEvents.obj
 0001:00061fa0       ??_GCEventTheRoyalJelly@@UAEPAXI@Z 00462fa0 f i IslandEvents.obj
 0001:00061fa0       ??_ECEventTheRoyalJelly@@UAEPAXI@Z 00462fa0 f i IslandEvents.obj
 0001:00061fd0       ??1CEventTheRoyalJelly@@UAE@XZ 00462fd0 f i IslandEvents.obj
 0001:00061ff0       ??0CEventTheShootingStar@@QAE@XZ 00462ff0 f i IslandEvents.obj
 0001:00062010       ?GetTitle@CEventTheShootingStar@@UAE?AW4StringId@@XZ 00463010 f i IslandEvents.obj
 0001:00062020       ?GetDescription@CEventTheShootingStar@@UAE?AW4StringId@@XZ 00463020 f i IslandEvents.obj
 0001:00062030       ?GetChoiceAText@CEventTheShootingStar@@UAE?AW4StringId@@XZ 00463030 f i IslandEvents.obj
 0001:00062040       ?GetChoiceBText@CEventTheShootingStar@@UAE?AW4StringId@@XZ 00463040 f i IslandEvents.obj
 0001:00062050       ?CanFire@CEventTheAntHill@@UAE_NXZ 00463050 f i IslandEvents.obj
 0001:00062050       ?CanFire@CEventAntsAndGranary@@UAE_NXZ 00463050 f i IslandEvents.obj
 0001:00062050       ?CanFire@CEventTheShootingStar@@UAE_NXZ 00463050 f i IslandEvents.obj
 0001:00062050       ?CanFire@CEventThePlayfulOtters@@UAE_NXZ 00463050 f i IslandEvents.obj
 0001:00062090       ?GetResultDescription@CEventTheShootingStar@@UAE?AW4StringId@@H@Z 00463090 f i IslandEvents.obj
 0001:000620b0       ?ImpactGame@CEventTheShootingStar@@UAEXH@Z 004630b0 f i IslandEvents.obj
 0001:00062160       ??_ECEventTheShootingStar@@UAEPAXI@Z 00463160 f i IslandEvents.obj
 0001:00062160       ??_GCEventTheShootingStar@@UAEPAXI@Z 00463160 f i IslandEvents.obj
 0001:00062190       ??1CEventTheShootingStar@@UAE@XZ 00463190 f i IslandEvents.obj
 0001:000621b0       ??0CEventTheReturnOfBiggles@@QAE@XZ 004631b0 f i IslandEvents.obj
 0001:000621d0       ?GetTitle@CEventTheReturnOfBiggles@@UAE?AW4StringId@@XZ 004631d0 f i IslandEvents.obj
 0001:000621e0       ?GetDescription@CEventTheReturnOfBiggles@@UAE?AW4StringId@@XZ 004631e0 f i IslandEvents.obj
 0001:000621f0       ?GetChoiceAText@CEventTheReturnOfBiggles@@UAE?AW4StringId@@XZ 004631f0 f i IslandEvents.obj
 0001:00062200       ?GetChoiceBText@CEventTheReturnOfBiggles@@UAE?AW4StringId@@XZ 00463200 f i IslandEvents.obj
 0001:00062210       ?CanFire@CEventTheReturnOfBiggles@@UAE_NXZ 00463210 f i IslandEvents.obj
 0001:00062250       ?GetResultDescription@CEventTheReturnOfBiggles@@UAE?AW4StringId@@H@Z 00463250 f i IslandEvents.obj
 0001:00062270       ?CalcAward@CEventTheReturnOfBiggles@@UAEXH@Z 00463270 f i IslandEvents.obj
 0001:00062290       ?ImpactGame@CEventTheReturnOfBiggles@@UAEXH@Z 00463290 f i IslandEvents.obj
 0001:00062350       ??_ECEventTheReturnOfBiggles@@UAEPAXI@Z 00463350 f i IslandEvents.obj
 0001:00062350       ??_GCEventTheReturnOfBiggles@@UAEPAXI@Z 00463350 f i IslandEvents.obj
 0001:00062380       ??1CEventTheReturnOfBiggles@@UAE@XZ 00463380 f i IslandEvents.obj
 0001:000623a0       ?ReadyToShow@CIslandEventDialog@@QAE_NXZ 004633a0 f i IslandEvents.obj
 0001:000623c0       ??0CRosterOfDeadDialog@@QAE@XZ 004633c0 f   RosterOfDeadDialog.obj
 0001:000631c0       ??1CRosterOfDeadDialog@@UAE@XZ 004641c0 f   RosterOfDeadDialog.obj
 0001:000631e0       ?DrawNoFadeScene@CRosterOfDeadDialog@@MAEXXZ 004641e0 f   RosterOfDeadDialog.obj
 0001:00063340       ?GetResult@CRosterOfDeadDialog@@UAEHXZ 00464340 f   RosterOfDeadDialog.obj
 0001:00063360       ?HandleMessage@CRosterOfDeadDialog@@UAE_NHJ@Z 00464360 f   RosterOfDeadDialog.obj
 0001:00063420       ?HandleMouse@CRosterOfDeadDialog@@UAE_NHUldwPoint@@@Z 00464420 f   RosterOfDeadDialog.obj
 0001:00063660       ?UpdateList@CRosterOfDeadDialog@@AAEXXZ 00464660 f   RosterOfDeadDialog.obj
 0001:00063940       ??_GCRosterOfDeadDialog@@UAEPAXI@Z 00464940 f i RosterOfDeadDialog.obj
 0001:00063940       ??_ECRosterOfDeadDialog@@UAEPAXI@Z 00464940 f i RosterOfDeadDialog.obj
 0001:00063970       ??0theChangePlayerDlg@@QAE@H@Z 00464970 f   theChangePlayerDlg.obj
 0001:00064320       ??1theChangePlayerDlg@@UAE@XZ 00465320 f   theChangePlayerDlg.obj
 0001:000643d0       ?PlayerHasChanged@theChangePlayerDlg@@QAE_NXZ 004653d0 f   theChangePlayerDlg.obj
 0001:00064400       ?GetResult@theChangePlayerDlg@@UAEHXZ 00465400 f   theChangePlayerDlg.obj
 0001:00064420       ?HandleKey@theChangePlayerDlg@@UAE_NHHH@Z 00465420 f   theChangePlayerDlg.obj
 0001:00064460       ?HandleMessage@theChangePlayerDlg@@UAE_NHJ@Z 00465460 f   theChangePlayerDlg.obj
 0001:00064bf0       ?DrawNoFadeScene@theChangePlayerDlg@@MAEXXZ 00465bf0 f   theChangePlayerDlg.obj
 0001:00064cb0       ?UpdateFocus@theChangePlayerDlg@@IAEXXZ 00465cb0 f   theChangePlayerDlg.obj
 0001:00064d60       ?ChangeFocus@theChangePlayerDlg@@IAEX_N@Z 00465d60 f   theChangePlayerDlg.obj
 0001:00064dd0       ??_EtheChangePlayerDlg@@UAEPAXI@Z 00465dd0 f i theChangePlayerDlg.obj
 0001:00064dd0       ??_GtheChangePlayerDlg@@UAEPAXI@Z 00465dd0 f i theChangePlayerDlg.obj
 0001:00064e00       ?GetSound@CSound@@QAEPAVldwSoundFx@@W4ESound@@@Z 00465e00 f i theChangePlayerDlg.obj
 0001:00064e20       ??0theCreateNickNameDlg@@QAE@H@Z 00465e20 f   theCreateNickNameDlg.obj
 0001:00065270       ??1theCreateNickNameDlg@@UAE@XZ 00466270 f   theCreateNickNameDlg.obj
 0001:00065290       ?GetResult@theCreateNickNameDlg@@UAEHXZ 00466290 f   theCreateNickNameDlg.obj
 0001:000652b0       ?HandleKey@theCreateNickNameDlg@@UAE_NHHH@Z 004662b0 f   theCreateNickNameDlg.obj
 0001:00065300       ?HandleMessage@theCreateNickNameDlg@@UAE_NHJ@Z 00466300 f   theCreateNickNameDlg.obj
 0001:000653e0       ?DrawNoFadeScene@theCreateNickNameDlg@@MAEXXZ 004663e0 f   theCreateNickNameDlg.obj
 0001:000653f0       ??_EtheCreateNickNameDlg@@UAEPAXI@Z 004663f0 f i theCreateNickNameDlg.obj
 0001:000653f0       ??_GtheCreateNickNameDlg@@UAEPAXI@Z 004663f0 f i theCreateNickNameDlg.obj
 0001:00065420       ??0theFernsaceDialog@@QAE@H@Z 00466420 f   theFernsaceDialog.obj
 0001:000658c0       ??1theFernsaceDialog@@UAE@XZ 004668c0 f   theFernsaceDialog.obj
 0001:00065990       ?GetResult@theFernsaceDialog@@UAEHXZ 00466990 f   theFernsaceDialog.obj
 0001:000659b0       ?PrepareString@theFernsaceDialog@@IAEXPAD0@Z 004669b0 f   theFernsaceDialog.obj
 0001:00065df0       ?ComposeDisplay@theFernsaceDialog@@IAE_NH@Z 00466df0 f   theFernsaceDialog.obj
 0001:00065ef0       ?ComposeResult@theFernsaceDialog@@IAEXXZ 00466ef0 f   theFernsaceDialog.obj
 0001:00065f00       ?DrawNoFadeScene@theFernsaceDialog@@MAEXXZ 00466f00 f   theFernsaceDialog.obj
 0001:00065fa0       ?HandleMessage@theFernsaceDialog@@UAE_NHJ@Z 00466fa0 f   theFernsaceDialog.obj
 0001:00066020       ??_GtheFernsaceDialog@@UAEPAXI@Z 00467020 f i theFernsaceDialog.obj
 0001:00066020       ??_EtheFernsaceDialog@@UAEPAXI@Z 00467020 f i theFernsaceDialog.obj
 0001:00066050       ??0theMessageBoxDlg@@QAE@W4StringId@@HW4EMessageBoxType@@@Z 00467050 f   theMessageBoxDlg.obj
 0001:000660d0       ??0theMessageBoxDlg@@QAE@W4StringId@@H_N@Z 004670d0 f   theMessageBoxDlg.obj
 0001:00066160       ??0theMessageBoxDlg@@QAE@PBDH_N@Z 00467160 f   theMessageBoxDlg.obj
 0001:000661e0       ?Init@theMessageBoxDlg@@IAEXPBDHW4EMessageBoxType@@@Z 004671e0 f   theMessageBoxDlg.obj
 0001:00066600       ??1theMessageBoxDlg@@UAE@XZ 00467600 f   theMessageBoxDlg.obj
 0001:00066620       ?GetResult@theMessageBoxDlg@@UAEHXZ 00467620 f   theMessageBoxDlg.obj
 0001:00066640       ?HandleKey@theMessageBoxDlg@@UAE_NHHH@Z 00467640 f   theMessageBoxDlg.obj
 0001:00066690       ?HandleMessage@theMessageBoxDlg@@UAE_NHJ@Z 00467690 f   theMessageBoxDlg.obj
 0001:000666d0       ?DrawNoFadeScene@theMessageBoxDlg@@MAEXXZ 004676d0 f   theMessageBoxDlg.obj
 0001:000666e0       ??_GtheMessageBoxDlg@@UAEPAXI@Z 004676e0 f i theMessageBoxDlg.obj
 0001:000666e0       ??_EtheMessageBoxDlg@@UAEPAXI@Z 004676e0 f i theMessageBoxDlg.obj
 0001:00066710       ??0theOptionsDialog@@QAE@PADW4DialogColorEnum@@@Z 00467710 f   theOptionsDialog.obj
 0001:00066d80       ??1theOptionsDialog@@UAE@XZ 00467d80 f   theOptionsDialog.obj
 0001:00066da0       ?GetResult@theOptionsDialog@@UAEHXZ 00467da0 f   theOptionsDialog.obj
 0001:00066dc0       ?HandleMessage@theOptionsDialog@@UAE_NHJ@Z 00467dc0 f   theOptionsDialog.obj
 0001:00066f50       ?DrawNoFadeScene@theOptionsDialog@@MAEXXZ 00467f50 f   theOptionsDialog.obj
 0001:00067cd0       ?HandleMouse@theOptionsDialog@@UAE_NHUldwPoint@@@Z 00468cd0 f   theOptionsDialog.obj
 0001:000687c0       ??_EtheOptionsDialog@@UAEPAXI@Z 004697c0 f i theOptionsDialog.obj
 0001:000687c0       ??_GtheOptionsDialog@@UAEPAXI@Z 004697c0 f i theOptionsDialog.obj
 0001:000687f0       ?SetVolume@CSound@@QAEXM@Z 004697f0 f i theOptionsDialog.obj
 0001:00068810       ??0theTipDialog@@QAE@W4StringId@@W4ArrowDirection@@HH_N@Z 00469810 f   theTipDialog.obj
 0001:00068910       ??0theTipDialog@@QAE@PBD@Z 00469910 f   theTipDialog.obj
 0001:000689d0       ?Init@theTipDialog@@IAEXPBDW4ArrowDirection@@HH_N@Z 004699d0 f   theTipDialog.obj
 0001:00068f80       ??1theTipDialog@@UAE@XZ    00469f80 f   theTipDialog.obj
 0001:00068ff0       ?GetResult@theTipDialog@@UAEHXZ 00469ff0 f   theTipDialog.obj
 0001:00069010       ?HandleMessage@theTipDialog@@UAE_NHJ@Z 0046a010 f   theTipDialog.obj
 0001:00069050       ?HandleMouse@theTipDialog@@UAE_NHUldwPoint@@@Z 0046a050 f   theTipDialog.obj
 0001:00069060       ?DrawNoFadeScene@theTipDialog@@MAEXXZ 0046a060 f   theTipDialog.obj
 0001:00069540       ??_EtheTipDialog@@UAEPAXI@Z 0046a540 f i theTipDialog.obj
 0001:00069540       ??_GtheTipDialog@@UAEPAXI@Z 0046a540 f i theTipDialog.obj
 0001:00069570       ??0theTombStoneDialog@@QAE@W4TSDialogColorEnum@@PBUSGrave@CGraveyard@@@Z 0046a570 f   theTombStoneDialog.obj
 0001:00069f70       ??1theTombStoneDialog@@UAE@XZ 0046af70 f   theTombStoneDialog.obj
 0001:00069f90       ?GetResult@theTombStoneDialog@@UAEHXZ 0046af90 f   theTombStoneDialog.obj
 0001:00069fb0       ?HandleMessage@theTombStoneDialog@@UAE_NHJ@Z 0046afb0 f   theTombStoneDialog.obj
 0001:0006a000       ?DrawNoFadeScene@theTombStoneDialog@@MAEXXZ 0046b000 f   theTombStoneDialog.obj
 0001:0006a010       ??_GtheTombStoneDialog@@UAEPAXI@Z 0046b010 f i theTombStoneDialog.obj
 0001:0006a010       ??_EtheTombStoneDialog@@UAEPAXI@Z 0046b010 f i theTombStoneDialog.obj
 0001:0006a040       ??0CFog@@QAE@XZ            0046b040 f   Fog.obj
 0001:0006a080       ??1CFog@@QAE@XZ            0046b080 f   Fog.obj
 0001:0006a090       ?Reset@CFog@@QAEXXZ        0046b090 f   Fog.obj
 0001:0006a1b0       ?Stop@CFog@@QAEXXZ         0046b1b0 f   Fog.obj
 0001:0006a1d0       ?LoadAssets@CFog@@QAEXXZ   0046b1d0 f   Fog.obj
 0001:0006a200       ?ReleaseAssets@CFog@@QAEXXZ 0046b200 f   Fog.obj
 0001:0006a210       ?Update@CFog@@QAEXXZ       0046b210 f   Fog.obj
 0001:0006a540       ?Draw@CFog@@QAEXXZ         0046b540 f   Fog.obj
 0001:0006a710       ?CurrentIntensity@CWeather@@QBE?BMXZ 0046b710 f i Fog.obj
 0001:0006a730       ??0CLightning@@QAE@XZ      0046b730 f   Lightning.obj
 0001:0006a750       ??1CLightning@@QAE@XZ      0046b750 f   Lightning.obj
 0001:0006a760       ?Reset@CLightning@@QAEX_N@Z 0046b760 f   Lightning.obj
 0001:0006a7b0       ?Update@CLightning@@QAEXXZ 0046b7b0 f   Lightning.obj
 0001:0006a8c0       ?Draw@CLightning@@QAEXXZ   0046b8c0 f   Lightning.obj
 0001:0006a900       ??0CRain@@QAE@XZ           0046b900 f   Rain.obj
 0001:0006a940       ??1CRain@@QAE@XZ           0046b940 f   Rain.obj
 0001:0006a950       ?Reset@CRain@@QAEX_N@Z     0046b950 f   Rain.obj
 0001:0006aa30       ?Stop@CRain@@QAEXXZ        0046ba30 f   Rain.obj
 0001:0006aa50       ?Update@CRain@@QAEXXZ      0046ba50 f   Rain.obj
 0001:0006ac10       ?Draw@CRain@@QAEXXZ        0046bc10 f   Rain.obj
 0001:0006adf0       ??0CSunBeam@@QAE@XZ        0046bdf0 f   SunBeam.obj
 0001:0006ae30       ??1CSunBeam@@QAE@XZ        0046be30 f   SunBeam.obj
 0001:0006ae40       ?Reset@CSunBeam@@QAEXXZ    0046be40 f   SunBeam.obj
 0001:0006aee0       ?LoadAssets@CSunBeam@@QAEXXZ 0046bee0 f   SunBeam.obj
 0001:0006af10       ?ReleaseAssets@CSunBeam@@QAEXXZ 0046bf10 f   SunBeam.obj
 0001:0006af20       ?Update@CSunBeam@@QAEXXZ   0046bf20 f   SunBeam.obj
 0001:0006b130       ?Draw@CSunBeam@@QAEXXZ     0046c130 f   SunBeam.obj
 0001:0006b1f0       ??0CWeather@@QAE@XZ        0046c1f0 f   Weather.obj
 0001:0006b210       ??1CWeather@@QAE@XZ        0046c210 f   Weather.obj
 0001:0006b220       ?Reset@CWeather@@QAEXXZ    0046c220 f   Weather.obj
 0001:0006b2e0       ?Update@CWeather@@QAEXXZ   0046c2e0 f   Weather.obj
 0001:0006b680       ?Draw@CWeather@@QAEXXZ     0046c680 f   Weather.obj
 0001:0006b720       ?SetCurrent@CWeather@@QAEXW4EWeather@@H@Z 0046c720 f   Weather.obj
 0001:0006b910       ?SetNext@CWeather@@QAEXW4EWeather@@@Z 0046c910 f   Weather.obj
 0001:0006b940       ?CurrentTypeString@CWeather@@QBEPBDXZ 0046c940 f   Weather.obj
 0001:0006b960       ?SetWetness@CWeather@@QAEXH@Z 0046c960 f   Weather.obj
 0001:0006b990       ?SetTargetIntensity@CWeather@@AAEXMH@Z 0046c990 f   Weather.obj
 0001:0006ba20       ?Random@CWeather@@QBE?BW4EWeather@@W42@@Z 0046ca20 f   Weather.obj
 0001:0006ba80       ??0CContentMap@@QAE@XZ     0046ca80 f   ContentMap.obj
 0001:0006bab0       ?Load@CContentMap@@QAEXXZ  0046cab0 f   ContentMap.obj
 0001:0006bb10       ?Save@CContentMap@@IAE?B_NXZ 0046cb10 f   ContentMap.obj
 0001:0006bb80       ?Draw@CContentMap@@IBEX_N0000M@Z 0046cb80 f   ContentMap.obj
 0001:0006be80       ?FindObject@CContentMap@@QBE?BUldwPoint@@W4EObject@1@@Z 0046ce80 f   ContentMap.obj
 0001:0006c000       ?FindLegalTerrain@CContentMap@@QBE?BUldwPoint@@U2@W4EDirection@@_N@Z 0046d000 f   ContentMap.obj
 0001:0006c110       ?Read@CContentMap@@ABEXHHAAUSContent@1@@Z 0046d110 f   ContentMap.obj
 0001:0006c1b0       ?Write@CContentMap@@AAEXHHUSContent@1@@Z 0046d1b0 f   ContentMap.obj
 0001:0006c210       ?ConvertPosToRowColumn@CContentMap@@ABEXUldwPoint@@AAH1@Z 0046d210 f   ContentMap.obj
 0001:0006c290       ?ConvertRowColumnToPos@CContentMap@@ABEXHHAAUldwPoint@@@Z 0046d290 f   ContentMap.obj
 0001:0006c2c0       ?SetContent@CContentMap@@IAEXUldwRect@@_NW4EMaterial@1@W4EObject@1@W4EHotSpot@1@W4ERedirector@1@@Z 0046d2c0 f   ContentMap.obj
 0001:0006c320       ?SetContent@CContentMap@@IAEXUldwRect@@ABUSContent@1@@Z 0046d320 f   ContentMap.obj
 0001:0006c3f0       ?SetContent@CContentMap@@IAEXUldwRect@@ABUSContent@1@_N2222@Z 0046d3f0 f   ContentMap.obj
 0001:0006c530       ?GetContent@CContentMap@@IBEXUldwPoint@@AAUSContent@1@@Z 0046d530 f   ContentMap.obj
 0001:0006c570       ?IsBlocking@CContentMap@@QBE?B_NUldwPoint@@@Z 0046d570 f   ContentMap.obj
 0001:0006c5a0       ?GetMaterial@CContentMap@@QBE?BW4EMaterial@1@UldwPoint@@@Z 0046d5a0 f   ContentMap.obj
 0001:0006c5d0       ?GetObject@CContentMap@@QBE?BW4EObject@1@UldwPoint@@@Z 0046d5d0 f   ContentMap.obj
 0001:0006c600       ?GetHotSpot@CContentMap@@QBE?BW4EHotSpot@1@UldwPoint@@@Z 0046d600 f   ContentMap.obj
 0001:0006c630       ?GetRedirector@CContentMap@@QBE?BW4ERedirector@1@UldwPoint@@@Z 0046d630 f   ContentMap.obj
 0001:0006c660       ?SetObjectBlocking@CContentMap@@QAEXW4EObject@1@_N@Z 0046d660 f   ContentMap.obj
 0001:0006c690       ?SetObjectMaterial@CContentMap@@QAEXW4EObject@1@W4EMaterial@1@@Z 0046d690 f   ContentMap.obj
 0001:0006c6c0       ?SetObjectHotSpot@CContentMap@@QAEXW4EObject@1@W4EHotSpot@1@@Z 0046d6c0 f   ContentMap.obj
 0001:0006c6f0       ?SetObjectRedirector@CContentMap@@QAEXW4EObject@1@W4ERedirector@1@@Z 0046d6f0 f   ContentMap.obj
 0001:0006c720       ?SetObjectContent@CContentMap@@QAEXW4EObject@1@ABUSContent@1@_N222@Z 0046d720 f   ContentMap.obj
 0001:0006c810       ?IsValidSpawnPos@CContentMap@@QBE?B_NUldwPoint@@@Z 0046d810 f   ContentMap.obj
 0001:0006c850       ?ReadObject@CContentMap@@IBE?BW4EObject@1@HH@Z 0046d850 f i ContentMap.obj
 0001:0006c880       ?ReadHotSpot@CContentMap@@IBE?BW4EHotSpot@1@HH@Z 0046d880 f i ContentMap.obj
 0001:0006c8b0       ?ReadRedirector@CContentMap@@IBE?BW4ERedirector@1@HH@Z 0046d8b0 f i ContentMap.obj
 0001:0006c8e0       ?ReadMaterial@CContentMap@@IBE?BW4EMaterial@1@HH@Z 0046d8e0 f i ContentMap.obj
 0001:0006c910       ?ReadBlocking@CContentMap@@IBE?B_NHH@Z 0046d910 f i ContentMap.obj
 0001:0006c940       ??0CEnvironment@@QAE@XZ    0046d940 f   Environment.obj
 0001:0006c9d0       ?Reset@CEnvironment@@QAEXXZ 0046d9d0 f   Environment.obj
 0001:0006cc90       ?LoadAssets@CEnvironment@@QAEXXZ 0046dc90 f   Environment.obj
 0001:0006cd50       ?ReleaseAssets@CEnvironment@@QAEXXZ 0046dd50 f   Environment.obj
 0001:0006cd60       ?Refresh@CEnvironment@@QAEXXZ 0046dd60 f   Environment.obj
 0001:0006cdb0       ?Update@CEnvironment@@QAEXXZ 0046ddb0 f   Environment.obj
 0001:0006cfc0       ?Draw@CEnvironment@@QAEXXZ 0046dfc0 f   Environment.obj
 0001:0006d0b0       ?Draw@CEnvironment@@QBEXH@Z 0046e0b0 f   Environment.obj
 0001:0006d390       ?TechAdvanced@CEnvironment@@UAEXW4ETech@@H@Z 0046e390 f   Environment.obj
 0001:0006d3e0       ??0ITechObserver@@QAE@XZ   0046e3e0 f i Environment.obj
 0001:0006d400       ??0CHotSpot@@QAE@XZ        0046e400 f   HotSpot.obj
 0001:0006d6d0       ?Dispatch@CHotSpot@@QBE?B_NAAVCVillager@@W4EHotSpot@CContentMap@@@Z 0046e6d0 f   HotSpot.obj
 0001:0006d700       ?SetHandler@CHotSpot@@QAEXW4EHotSpot@CContentMap@@P6A?B_NAAVCVillager@@@ZW4EDirection@@@Z 0046e700 f   HotSpot.obj
 0001:0006d730       ?Kindling@CHotSpot@@CA?B_NAAVCVillager@@@Z 0046e730 f   HotSpot.obj
 0001:0006d750       ?Clifftree@CHotSpot@@CA?B_NAAVCVillager@@@Z 0046e750 f   HotSpot.obj
 0001:0006d760       ?Firewood@CHotSpot@@CA?B_NAAVCVillager@@@Z 0046e760 f   HotSpot.obj
 0001:0006d7c0       ?Spring@CHotSpot@@CA?B_NAAVCVillager@@@Z 0046e7c0 f   HotSpot.obj
 0001:0006d830       ?HospitalLab@CHotSpot@@CA?B_NAAVCVillager@@@Z 0046e830 f   HotSpot.obj
 0001:0006d8c0       ?FirePlace@CHotSpot@@CA?B_NAAVCVillager@@@Z 0046e8c0 f   HotSpot.obj
 0001:0006dad0       ?BathHotspot@CHotSpot@@CA?B_NAAVCVillager@@@Z 0046ead0 f   HotSpot.obj
 0001:0006dbf0       ?Ampitheatre@CHotSpot@@CA?B_NAAVCVillager@@@Z 0046ebf0 f   HotSpot.obj
 0001:0006dcf0       ?Foodbin@CHotSpot@@CA?B_NAAVCVillager@@@Z 0046ecf0 f   HotSpot.obj
 0001:0006dde0       ?BrokenLift@CHotSpot@@CA?B_NAAVCVillager@@@Z 0046ede0 f   HotSpot.obj
 0001:0006de70       ?BurnedTorch@CHotSpot@@CA?B_NAAVCVillager@@@Z 0046ee70 f   HotSpot.obj
 0001:0006ded0       ?PathTop@CHotSpot@@CA?B_NAAVCVillager@@@Z 0046eed0 f   HotSpot.obj
 0001:0006df80       ?LiftPlatform@CHotSpot@@CA?B_NAAVCVillager@@@Z 0046ef80 f   HotSpot.obj
 0001:0006dfe0       ?AlchemyTableHandler@CHotSpot@@CA?B_NAAVCVillager@@@Z 0046efe0 f   HotSpot.obj
 0001:0006e110       ?AlchemyPotHotSpot@CHotSpot@@CA?B_NAAVCVillager@@@Z 0046f110 f   HotSpot.obj
 0001:0006e280       ?Herb1@CHotSpot@@CA?B_NAAVCVillager@@@Z 0046f280 f   HotSpot.obj
 0001:0006e300       ?Herb2@CHotSpot@@CA?B_NAAVCVillager@@@Z 0046f300 f   HotSpot.obj
 0001:0006e380       ?Herb3@CHotSpot@@CA?B_NAAVCVillager@@@Z 0046f380 f   HotSpot.obj
 0001:0006e400       ?Herb4@CHotSpot@@CA?B_NAAVCVillager@@@Z 0046f400 f   HotSpot.obj
 0001:0006e480       ?Herb5@CHotSpot@@CA?B_NAAVCVillager@@@Z 0046f480 f   HotSpot.obj
 0001:0006e500       ?Herb6@CHotSpot@@CA?B_NAAVCVillager@@@Z 0046f500 f   HotSpot.obj
 0001:0006e580       ?Herb7@CHotSpot@@CA?B_NAAVCVillager@@@Z 0046f580 f   HotSpot.obj
 0001:0006e600       ?BrokenStatue@CHotSpot@@CA?B_NAAVCVillager@@@Z 0046f600 f   HotSpot.obj
 0001:0006e6c0       ?StatuePath@CHotSpot@@CA?B_NAAVCVillager@@@Z 0046f6c0 f   HotSpot.obj
 0001:0006e830       ?BeehiveHotspot@CHotSpot@@CA?B_NAAVCVillager@@@Z 0046f830 f   HotSpot.obj
 0001:0006e940       ?ResearchHotspot@CHotSpot@@CA?B_NAAVCVillager@@@Z 0046f940 f   HotSpot.obj
 0001:0006e990       ?FruitTree@CHotSpot@@CA?B_NAAVCVillager@@@Z 0046f990 f   HotSpot.obj
 0001:0006ead0       ?SunDiskHotSpot@CHotSpot@@CA?B_NAAVCVillager@@@Z 0046fad0 f   HotSpot.obj
 0001:0006eb70       ?House1@CHotSpot@@CA?B_NAAVCVillager@@@Z 0046fb70 f   HotSpot.obj
 0001:0006ec10       ?House2@CHotSpot@@CA?B_NAAVCVillager@@@Z 0046fc10 f   HotSpot.obj
 0001:0006ecd0       ?House3@CHotSpot@@CA?B_NAAVCVillager@@@Z 0046fcd0 f   HotSpot.obj
 0001:0006ed90       ?Hospital@CHotSpot@@CA?B_NAAVCVillager@@@Z 0046fd90 f   HotSpot.obj
 0001:0006eda0       ?ClothingHut@CHotSpot@@CA?B_NAAVCVillager@@@Z 0046fda0 f   HotSpot.obj
 0001:0006ef00       ?RuinsHotSpot@CHotSpot@@CA?B_NAAVCVillager@@@Z 0046ff00 f   HotSpot.obj
 0001:0006f010       ?KeyJump@CHotSpot@@CA?B_NAAVCVillager@@@Z 00470010 f   HotSpot.obj
 0001:0006f050       ?DivingPlatform@CHotSpot@@CA?B_NAAVCVillager@@@Z 00470050 f   HotSpot.obj
 0001:0006f080       ?ChalkBoardHandler@CHotSpot@@CA?B_NAAVCVillager@@@Z 00470080 f   HotSpot.obj
 0001:0006f170       ?RosterOfTheDeadHandler@CHotSpot@@CA?B_NAAVCVillager@@@Z 00470170 f   HotSpot.obj
 0001:0006f1d0       ?Bias@CHotSpot@@QAE?BW4EDirection@@W4EHotSpot@CContentMap@@@Z 004701d0 f   HotSpot.obj
 0001:0006f1f0       ?ContainsFirewood@CFirePit@@QBE?B_NXZ 004701f0 f i HotSpot.obj
 0001:0006f210       ?WasScaffoldingConstructed@CPrincessStatue@@QBE?B_NXZ 00470210 f i HotSpot.obj
 0001:0006f230       ??0CRedirect@@QAE@XZ       00470230 f   Redirect.obj
 0001:0006f280       ?Dispatch@CRedirect@@QBE?B_NAAVCVillager@@W4ERedirector@CContentMap@@@Z 00470280 f   Redirect.obj
 0001:0006f2b0       ?SetHandler@CRedirect@@QAEXW4ERedirector@CContentMap@@P6AXAAVCVillager@@@Z@Z 004702b0 f   Redirect.obj
 0001:0006f2d0       ?DivingRock@CRedirect@@CAXAAVCVillager@@@Z 004702d0 f   Redirect.obj
 0001:0006f340       ??0CWaypoint@@QAE@XZ       00470340 f   Waypoint.obj
 0001:0006f3b0       ?Load@CWaypoint@@QAEXXZ    004703b0 f   Waypoint.obj
 0001:0006f410       ?Save@CWaypoint@@IAE?B_NXZ 00470410 f   Waypoint.obj
 0001:0006f480       ?GetNearby@CWaypoint@@QBE?BW4EWaypoint@@UldwPoint@@@Z 00470480 f   Waypoint.obj
 0001:0006f4f0       ?GetNearest@CWaypoint@@QBE?BW4EWaypoint@@UldwPoint@@@Z 004704f0 f   Waypoint.obj
 0001:0006f5a0       ??0CWorldMap@@QAE@XZ       004705a0 f   WorldMap.obj
 0001:0006f610       ??1CWorldMap@@QAE@XZ       00470610 f   WorldMap.obj
 0001:0006f620       ?LoadAssets@CWorldMap@@QAEXXZ 00470620 f   WorldMap.obj
 0001:0006f740       ?ReleaseAssets@CWorldMap@@QAEXXZ 00470740 f   WorldMap.obj
 0001:0006f7f0       ?Draw@CWorldMap@@QBEXUldwPoint@@UldwRect@@@Z 004707f0 f   WorldMap.obj
 0001:0006f8b0       ?IsOnMap@CWorldMap@@QBE?B_NUldwPoint@@@Z 004708b0 f   WorldMap.obj
 0001:0006f8f0       ?RandomPoint@CWorldMap@@QBE?BUldwPoint@@XZ 004708f0 f   WorldMap.obj
 0001:0006f980       ??0CWorldPath@@QAE@XZ      00470980 f   WorldPath.obj
 0001:0006f9d0       ?FindPath@CWorldPath@@QAE_NUldwPoint@@0_N@Z 004709d0 f   WorldPath.obj
 0001:0006fa00       ?NextPoint@CWorldPath@@QAE?AUldwPoint@@XZ 00470a00 f   WorldPath.obj
 0001:0006fac0       ?Completed@CWorldPath@@QAE_NXZ 00470ac0 f   WorldPath.obj
 0001:0006faf0       ?CreatePath@CWorldPath@@QAE_NAAV1@UldwPoint@@1_N@Z 00470af0 f   WorldPath.obj
 0001:0006fc10       ?CreatePathGradient@CWorldPath@@AAE_NAAUPathGradient@1@UldwPoint@@1_N@Z 00470c10 f   WorldPath.obj
 0001:00070200       ?OnPathGradientTarget@CWorldPath@@AAE_NAAUPathGradient@1@UldwPoint@@@Z 00471200 f   WorldPath.obj
 0001:00070240       ?GetNextPointFromPathGradient@CWorldPath@@AAE?AUldwPoint@@AAUPathGradient@1@U2@_N@Z 00471240 f   WorldPath.obj
 0001:000704c0       ?PathIsBlocked@CWorldPath@@AAE_NHH_N@Z 004714c0 f   WorldPath.obj
 0001:00070510       ??0CWorldView@@QAE@XZ      00471510 f   WorldView.obj
 0001:00070540       ?Reset@CWorldView@@QAEXXZ  00471540 f   WorldView.obj
 0001:00070590       ?KeepInView@CWorldView@@QAEXUldwPoint@@@Z 00471590 f   WorldView.obj
 0001:00070650       ?Scroll@CWorldView@@QAEXUldwPoint@@@Z 00471650 f   WorldView.obj
 0001:00070680       ?ScrollTo@CWorldView@@QAEXUldwPoint@@@Z 00471680 f   WorldView.obj
 0001:000706b0       ?ScrollAmount@CWorldView@@QAEXUldwPoint@@@Z 004716b0 f   WorldView.obj
 0001:000706e0       ?StopScrolling@CWorldView@@QAEXXZ 004716e0 f   WorldView.obj
 0001:00070710       ?Update@CWorldView@@QAEXXZ 00471710 f   WorldView.obj
 0001:000707e0       ?CenterAtWorldPos@CWorldView@@QAEXHH@Z 004717e0 f   WorldView.obj
 0001:00070830       ?RandomPoint@CWorldView@@QBE?BUldwPoint@@XZ 00471830 f   WorldView.obj
 0001:00070870       ?Constrain@CWorldView@@AAEXXZ 00471870 f   WorldView.obj
 0001:00070900       ??0CEnvironmentalSound@@QAE@XZ 00471900 f   EnvironmentalSound.obj
 0001:00070940       ??1CEnvironmentalSound@@QAE@XZ 00471940 f   EnvironmentalSound.obj
 0001:00070960       ?Reset@CEnvironmentalSound@@QAEXXZ 00471960 f   EnvironmentalSound.obj
 0001:000709a0       ?AddSound@CEnvironmentalSound@@QAE?BHW4ESound@@HW4ESoundType@@UldwPoint@@MM@Z 004719a0 f   EnvironmentalSound.obj
 0001:00070b60       ?RemoveSound@CEnvironmentalSound@@QAEXW4ESound@@@Z 00471b60 f   EnvironmentalSound.obj
 0001:00070bc0       ?Remove@CEnvironmentalSound@@UAEXH@Z 00471bc0 f   EnvironmentalSound.obj
 0001:00070c00       ?Update@CEnvironmentalSound@@QAEXXZ 00471c00 f   EnvironmentalSound.obj
 0001:00070e50       ?Draw@CEnvironmentalSound@@QAEXXZ 00471e50 f   EnvironmentalSound.obj
 0001:00070f00       ?PauseVariantSounds@CEnvironmentalSound@@QAEXXZ 00471f00 f   EnvironmentalSound.obj
 0001:00070f20       ?ResumeVariantSounds@CEnvironmentalSound@@QAEXXZ 00471f20 f   EnvironmentalSound.obj
 0001:00070f40       ?StopSounds@CEnvironmentalSound@@QAEXH@Z 00471f40 f   EnvironmentalSound.obj
 0001:00070fb0       ?SetPos@CEnvironmentalSound@@UAEXHUldwPoint@@@Z 00471fb0 f   EnvironmentalSound.obj
 0001:00070fe0       ??0IVillagerAttachment@@QAE@XZ 00471fe0 f i EnvironmentalSound.obj
 0001:00071000       ??0SSound@CEnvironmentalSound@@QAE@XZ 00472000 f i EnvironmentalSound.obj
 0001:00071020       ?Update@IVillagerAttachment@@UAEXAAVCVillager@@HI@Z 00472020 f i EnvironmentalSound.obj
 0001:00071020       ?Attach@IVillagerAttachment@@UAEXAAVCVillager@@HAAH@Z 00472020 f i EnvironmentalSound.obj
 0001:00071020       ?SetPos@IVillagerAttachment@@UAEXHUldwPoint@@@Z 00472020 f i EnvironmentalSound.obj
 0001:00071030       ?WorldPosAtCenter@CWorldView@@QBE?BUldwPoint@@XZ 00472030 f i EnvironmentalSound.obj
 0001:00071060       ?RandomChance@@YA?B_NM@Z   00472060 f i EnvironmentalSound.obj
 0001:000710a0       ??0CSound@@QAE@XZ          004720a0 f   Sound.obj
 0001:000710f0       ??1CSound@@QAE@XZ          004720f0 f   Sound.obj
 0001:00071100       ?LoadAssets@CSound@@QAEXXZ 00472100 f   Sound.obj
 0001:00071230       ?ReleaseAssets@CSound@@QAEXXZ 00472230 f   Sound.obj
 0001:000712c0       ?Play@CSound@@QAEXW4ESound@@@Z 004722c0 f   Sound.obj
 0001:000712e0       ?Play@CSound@@QAEXW4ESound@@M@Z 004722e0 f   Sound.obj
 0001:00071300       ?Play@CSound@@QAEXW4ESound@@_N@Z 00472300 f   Sound.obj
 0001:00071330       ?Play@CSound@@QAEXW4ESound@@_NM@Z 00472330 f   Sound.obj
 0001:00071450       ?Stop@CSound@@QAEXW4ESound@@@Z 00472450 f   Sound.obj
 0001:000714c0       ?Pause@CSound@@QAEXXZ      004724c0 f   Sound.obj
 0001:00071510       ?Resume@CSound@@QAEXXZ     00472510 f   Sound.obj
 0001:00071560       ?SetVolume@CSound@@QAEXW4ESound@@M@Z 00472560 f   Sound.obj
 0001:000715b0       ?Release@CSound@@QAEXW4ESound@@@Z 004725b0 f   Sound.obj
 0001:00071610       ?GetESoundName@CSound@@QAEPBDW4ESound@@@Z 00472610 f   Sound.obj
 0001:00071650       ?IsPlaying@CSound@@QBE?B_NW4ESound@@@Z 00472650 f   Sound.obj
 0001:00071680       ??_GldwSoundFx@@QAEPAXI@Z  00472680 f i Sound.obj
 0001:000716b0       ??0CSoundTrack@@QAE@XZ     004726b0 f   SoundTrack.obj
 0001:00071710       ??1CSoundTrack@@QAE@XZ     00472710 f   SoundTrack.obj
 0001:00071720       ?LoadAssets@CSoundTrack@@QAEXXZ 00472720 f   SoundTrack.obj
 0001:000717c0       ?ReleaseAssets@CSoundTrack@@QAEXXZ 004727c0 f   SoundTrack.obj
 0001:00071840       ?Start@CSoundTrack@@QAEX_N@Z 00472840 f   SoundTrack.obj
 0001:00071a70       ?Stop@CSoundTrack@@QAEXXZ  00472a70 f   SoundTrack.obj
 0001:00071aa0       ?Update@CSoundTrack@@QAEXW4ESoundTrack@@@Z 00472aa0 f   SoundTrack.obj
 0001:00071b90       ?IsPlaying@CSoundTrack@@QBE?B_NW4ESoundTrack@@@Z 00472b90 f   SoundTrack.obj
 0001:00071bb0       ??_GldwSoundTrack@@QAEPAXI@Z 00472bb0 f i SoundTrack.obj
 0001:00071be0       ??0ldwarialbold@@QAE@XZ    00472be0 f   ldwarialbold.obj
 0001:00071c40       ??1ldwBurweed27@@UAE@XZ    00472c40 f i ldwBurweed27.obj
 0001:00071c40       ??1ldwarialbold@@UAE@XZ    00472c40 f i ldwarialbold.obj
 0001:00071c60       ??0ldwBurweed27@@QAE@XZ    00472c60 f   ldwBurweed27.obj
 0001:00071cc0       ??_Gldwarialbold@@UAEPAXI@Z 00472cc0 f i ldwarialbold.obj
 0001:00071cc0       ??_EldwBurweed27@@UAEPAXI@Z 00472cc0 f i ldwBurweed27.obj
 0001:00071cc0       ??_GldwBurweed27@@UAEPAXI@Z 00472cc0 f i ldwBurweed27.obj
 0001:00071cc0       ??_Eldwarialbold@@UAEPAXI@Z 00472cc0 f i ldwarialbold.obj
 0001:00071cf0       ??0CScore@@QAE@KPBDKKKKKKKKKKKKKK@Z 00472cf0 f   highscore.obj
 0001:00071db0       ??1CScore@@QAE@XZ          00472db0 f   highscore.obj
 0001:00071dc0       ??0CHighScore@@QAE@XZ      00472dc0 f   highscore.obj
 0001:00071e40       ??1CHighScore@@QAE@XZ      00472e40 f   highscore.obj
 0001:00071e80       ?Submit@CHighScore@@QAE_NPAVCScore@@KKKPBD@Z 00472e80 f   highscore.obj
 0001:00071eb0       ?GetFirst@CHighScore@@QAEPAVCScore@@XZ 00472eb0 f   highscore.obj
 0001:00071ed0       ?GetLastMessage@CHighScore@@QAEPBDXZ 00472ed0 f   highscore.obj
 0001:00071ef0       ??0CHighScoreImpl@@QAE@XZ  00472ef0 f i highscore.obj
 0001:00071f40       ??_GCHighScoreImpl@@QAEPAXI@Z 00472f40 f i highscore.obj
 0001:00071f70       ??1CHighScoreImpl@@QAE@XZ  00472f70 f i highscore.obj
 0001:00071ff0       ??_GCScore@@QAEPAXI@Z      00472ff0 f i highscore.obj
 0001:00072020       ?Submit@CHighScoreImpl@@QAE_NPAVCScore@@KKKPBD@Z 00473020 f i highscore.obj
 0001:00072160       ?GetLastMessage@CHighScoreImpl@@QAEPBDXZ 00473160 f i highscore.obj
 0001:00072180       ?BuildDigest@CHighScoreImpl@@QAE_NPADPBDK@Z 00473180 f i highscore.obj
 0001:000724b0       ?ReadFile@CHighScoreImpl@@QAEKXZ 004734b0 f i highscore.obj
 0001:000725f0       ?Parse@CHighScoreImpl@@QAEXPBD@Z 004735f0 f i highscore.obj
 0001:00072b50       ?SetMessage@CHighScoreImpl@@QAEXPBD@Z 00473b50 f i highscore.obj
 0001:00072b70       ??0CHttpClient@@QAE@XZ     00473b70 f   httpclient.obj
 0001:00072bd0       ??1CHttpClient@@QAE@XZ     00473bd0 f   httpclient.obj
 0001:00072c40       ?SetProxy@CHttpClient@@QAEXPBD@Z 00473c40 f   httpclient.obj
 0001:00072cd0       ?SetAuthentication@CHttpClient@@QAEXPBD0@Z 00473cd0 f   httpclient.obj
 0001:00072dc0       ?OpenSession@CHttpClient@@QAEHPBD@Z 00473dc0 f   httpclient.obj
 0001:00072e50       ?CloseSession@CHttpClient@@QAEXXZ 00473e50 f   httpclient.obj
 0001:00072ec0       ?SendRequest@CHttpClient@@QAEHPBD0@Z 00473ec0 f   httpclient.obj
 0001:000730a0       ?ReadData@CHttpClient@@QAEKPADK@Z 004740a0 f   httpclient.obj
 0001:00073110       ?ParseUrl@CHttpClient@@AAEXPBDPAD1@Z 00474110 f   httpclient.obj
 0001:00073200       __tcstok                   00474200 f i httpclient.obj
 0001:00073220       ??0CBird@@QAE@XZ           00474220 f   Bird.obj
 0001:00073260       ??1CBird@@QAE@XZ           00474260 f   Bird.obj
 0001:00073270       ?LoadAssets@CBird@@QAEXXZ  00474270 f   Bird.obj
 0001:000732c0       ?ReleaseAssets@CBird@@QAEXXZ 004742c0 f   Bird.obj
 0001:000732d0       ?Reset@CBird@@QAEXXZ       004742d0 f   Bird.obj
 0001:000734f0       ?AddSpawnArea@CBird@@QAEXUldwRect@@@Z 004744f0 f   Bird.obj
 0001:00073540       ?CreateFlyby@CBird@@QAE?B_NUldwPoint@@@Z 00474540 f   Bird.obj
 0001:00073620       ?Create@CBird@@QAE?B_NUldwPoint@@_N@Z 00474620 f   Bird.obj
 0001:00073720       ?Update@CBird@@QAEXXZ      00474720 f   Bird.obj
 0001:000739a0       ?Draw@CBird@@QBEXXZ        004749a0 f   Bird.obj
 0001:00073a30       ?Draw@CBird@@QBEXH@Z       00474a30 f   Bird.obj
 0001:00073be0       ?ScareNearbyBirds@CBird@@QAE?BHUldwPoint@@H@Z 00474be0 f   Bird.obj
 0001:00073d10       ?AcquireTarget@SInst@CBird@@QAEXXZ 00474d10 f   Bird.obj
 0001:00073d90       ??0SRainDrop@CRain@@QAE@XZ 00474d90 f i Rain.obj
 0001:00073d90       ??0SInst@CBird@@QAE@XZ     00474d90 f i Bird.obj
 0001:00073dc0       ??KldwPoint@@QBE?AU0@ABH@Z 00474dc0 f i Bird.obj
 0001:00073e00       ?Get@theHummingbirdClass@@SAPAV1@XZ 00474e00 f   HummingbirdClass.obj
 0001:00073e80       ?Destroy@theHummingbirdClass@@SAXXZ 00474e80 f   HummingbirdClass.obj
 0001:00073ec0       ??1theHummingbirdClass@@QAE@XZ 00474ec0 f   HummingbirdClass.obj
 0001:00073ee0       ??0theHummingbirdClass@@IAE@XZ 00474ee0 f   HummingbirdClass.obj
 0001:00073f70       ?InitHummingbirds@theHummingbirdClass@@QAEXXZ 00474f70 f   HummingbirdClass.obj
 0001:00074060       ?SpawnHummingbirds@theHummingbirdClass@@QAEXXZ 00475060 f   HummingbirdClass.obj
 0001:000741c0       ?GetFeedingSpot@theHummingbirdClass@@IAEHH@Z 004751c0 f   HummingbirdClass.obj
 0001:00074240       ?GetFeedingFarSpot@theHummingbirdClass@@IAEHH@Z 00475240 f   HummingbirdClass.obj
 0001:000742c0       ?StartFeeding@theHummingbirdClass@@IAEXPAUHummingbirdType@@@Z 004752c0 f   HummingbirdClass.obj
 0001:00074370       ?InitFeedingTarget@theHummingbirdClass@@IAEXPAUHummingbirdType@@@Z 00475370 f   HummingbirdClass.obj
 0001:00074420       ?StartFeedingFar@theHummingbirdClass@@IAEXPAUHummingbirdType@@@Z 00475420 f   HummingbirdClass.obj
 0001:000744c0       ?InitFarFeedingTarget@theHummingbirdClass@@IAEXPAUHummingbirdType@@@Z 004754c0 f   HummingbirdClass.obj
 0001:000745a0       ?ExitLeftOrRight@theHummingbirdClass@@IAEXPAUHummingbirdType@@H@Z 004755a0 f   HummingbirdClass.obj
 0001:00074660       ?StartSpying@theHummingbirdClass@@IAEXPAUHummingbirdType@@H@Z 00475660 f   HummingbirdClass.obj
 0001:00074750       ?StartChasing@theHummingbirdClass@@IAEXPAUHummingbirdType@@@Z 00475750 f   HummingbirdClass.obj
 0001:00074780       ?StartFollowingGC@theHummingbirdClass@@IAEXPAUHummingbirdType@@@Z 00475780 f   HummingbirdClass.obj
 0001:000747d0       ?MouseClick@theHummingbirdClass@@QAEXUldwPoint@@@Z 004757d0 f   HummingbirdClass.obj
 0001:00074880       ?UpdateHummingbirds@theHummingbirdClass@@QAEXUldwPoint@@@Z 00475880 f   HummingbirdClass.obj
 0001:000753a0       ?DrawHummingbirds@theHummingbirdClass@@QAEXXZ 004763a0 f   HummingbirdClass.obj
 0001:000755d0       ?AcquireTarget@theHummingbirdClass@@QAEXHHH@Z 004765d0 f   HummingbirdClass.obj
 0001:00075810       ?AcquireTarget@theHummingbirdClass@@QAEXH@Z 00476810 f   HummingbirdClass.obj
 0001:000759b0       ?NormVel@theHummingbirdClass@@QAEXH@Z 004769b0 f   HummingbirdClass.obj
 0001:00075a60       ??_GtheHummingbirdClass@@QAEPAXI@Z 00476a60 f i HummingbirdClass.obj
 0001:00075a90       ??0HummingbirdType@@QAE@XZ 00476a90 f i HummingbirdClass.obj
 0001:00075a90       ??0ButterflyType@@QAE@XZ   00476a90 f i theButterflyClass.obj
 0001:00075ad0       ??0CShark@@QAE@XZ          00476ad0 f   Shark.obj
 0001:00075b00       ?Reset@CShark@@QAEXXZ      00476b00 f   Shark.obj
 0001:00075b40       ?LoadAssets@CShark@@QAEXXZ 00476b40 f   Shark.obj
 0001:00075b70       ?ReleaseAssets@CShark@@QAEXXZ 00476b70 f   Shark.obj
 0001:00075b80       ?Create@CShark@@QAE?B_NUldwPoint@@@Z 00476b80 f   Shark.obj
 0001:00075c10       ?Update@CShark@@QAEXXZ     00476c10 f   Shark.obj
 0001:00075fc0       ?Draw@CShark@@QBEXXZ       00476fc0 f   Shark.obj
 0001:00076030       ?Draw@CShark@@QBEXH@Z      00477030 f   Shark.obj
 0001:000761e0       ?GetNumberOfSharksNearby@CShark@@QBE?BHUldwPoint@@H@Z 004771e0 f   Shark.obj
 0001:00076290       ?GetNumberOfSharks@CShark@@QBE?BHXZ 00477290 f   Shark.obj
 0001:000762f0       ??0SInst@CShark@@QAE@XZ    004772f0 f i Shark.obj
 0001:00076320       ?cos@@YAMM@Z               00477320 f i Shark.obj
 0001:00076340       _cosf                      00477340 f i Shark.obj
 0001:00076360       ?sin@@YAMM@Z               00477360 f i Shark.obj
 0001:00076380       _sinf                      00477380 f i Shark.obj
 0001:000763a0       ??XldwPoint@@QAEAAU0@ABM@Z 004773a0 f i Shark.obj
 0001:000763e0       ?Get@theButterflyClass@@SAPAV1@XZ 004773e0 f   theButterflyClass.obj
 0001:00076460       ?Destroy@theButterflyClass@@SAXXZ 00477460 f   theButterflyClass.obj
 0001:000764a0       ??1theButterflyClass@@QAE@XZ 004774a0 f   theButterflyClass.obj
 0001:000764b0       ??0theButterflyClass@@IAE@XZ 004774b0 f   theButterflyClass.obj
 0001:00076540       ?InitButterflies@theButterflyClass@@QAEXXZ 00477540 f   theButterflyClass.obj
 0001:00076630       ?SpawnButterflies@theButterflyClass@@QAEX_N@Z 00477630 f   theButterflyClass.obj
 0001:00076830       ?ChangeButterflyStates@theButterflyClass@@QAEXW4ButterflyStateType@@_N@Z 00477830 f   theButterflyClass.obj
 0001:000768d0       ?UpdateButterflies@theButterflyClass@@QAEXUldwPoint@@@Z 004778d0 f   theButterflyClass.obj
 0001:00077060       ?UpdateMiniButterflies@theButterflyClass@@QAEXXZ 00478060 f   theButterflyClass.obj
 0001:000774d0       ?DrawButterflies@theButterflyClass@@QAEX_N@Z 004784d0 f   theButterflyClass.obj
 0001:00077870       ?AcquireTarget@theButterflyClass@@QAEXHHH@Z 00478870 f   theButterflyClass.obj
 0001:00077a00       ?AcquireTarget@theButterflyClass@@QAEXH@Z 00478a00 f   theButterflyClass.obj
 0001:00077bb0       ?NormVel@theButterflyClass@@QAEXH@Z 00478bb0 f   theButterflyClass.obj
 0001:00077c60       ??_GtheButterflyClass@@QAEPAXI@Z 00478c60 f i theButterflyClass.obj
 0001:00077c90       ??0CBFGProtection@@QAE@XZ  00478c90 f   BFGProtection.obj
 0001:00077ca0       ?IsProtectionValid@CBFGProtection@@QAE_NXZ 00478ca0 f   BFGProtection.obj
 0001:00077d40       ??0CDistributor@@QAE@XZ    00478d40 f   Distributor.obj
 0001:00077d70       ?LoadAssets@CDistributor@@QAEXXZ 00478d70 f   Distributor.obj
 0001:00077e60       ?ReleaseAssets@CDistributor@@QAEXXZ 00478e60 f   Distributor.obj
 0001:00077ee0       ?DrawMenuLogo@CDistributor@@QAEXHH@Z 00478ee0 f   Distributor.obj
 0001:00077f30       ?DrawLoadingLogo@CDistributor@@QAEXHH@Z 00478f30 f   Distributor.obj
 0001:00077f90       ?HasMenuLogo@CDistributor@@QAE_NXZ 00478f90 f   Distributor.obj
 0001:00077fb0       ??0CExpiration@@QAE@XZ     00478fb0 f   Expiration.obj
 0001:00077fc0       ?HasGameExpired@CExpiration@@QAE_NXZ 00478fc0 f   Expiration.obj
 0001:00078080       _WinMain@16                00479080 f   main.obj
 0001:000781b0       ??0CFoodStore@@QAE@XZ      004791b0 f   FoodStore.obj
 0001:000781d0       ?Reset@CFoodStore@@QAEXXZ  004791d0 f   FoodStore.obj
 0001:000781f0       ?LoadState@CFoodStore@@QAE?B_NABUSSaveState@1@@Z 004791f0 f   FoodStore.obj
 0001:00078220       ?SaveState@CFoodStore@@QBE?B_NAAUSSaveState@1@@Z 00479220 f   FoodStore.obj
 0001:00078240       ?Adjust@CFoodStore@@QAEXH@Z 00479240 f   FoodStore.obj
 0001:000782e0       ?IncrementFoodGathered@CGameStats@@QAEXI@Z 004792e0 f i FoodStore.obj
 0001:00078300       ??0CGameStats@@QAE@XZ      00479300 f   GameStats.obj
 0001:00078320       ?Reset@CGameStats@@QAEXXZ  00479320 f   GameStats.obj
 0001:00078370       ?LoadState@CGameStats@@QAE?B_NAAUSSaveState@1@@Z 00479370 f   GameStats.obj
 0001:00078390       ?SaveState@CGameStats@@QAE?B_NAAUSSaveState@1@@Z 00479390 f   GameStats.obj
 0001:000783b0       ?Refresh@CGameStats@@QAE?B_NXZ 004793b0 f   GameStats.obj
 0001:000786a0       ??_GCHighScore@@QAEPAXI@Z  004796a0 f i GameStats.obj
 0001:000786d0       ??0CGameTime@@QAE@XZ       004796d0 f   GameTime.obj
 0001:00078710       ?Reset@CGameTime@@QAEXXZ   00479710 f   GameTime.obj
 0001:00078760       ?LoadState@CGameTime@@QAE?B_NABUSSaveState@1@@Z 00479760 f   GameTime.obj
 0001:000787a0       ?SaveState@CGameTime@@QBE?B_NAAUSSaveState@1@@Z 004797a0 f   GameTime.obj
 0001:000787e0       ?RegisterTimer@CGameTime@@QAEXPAVCGameTimer@@@Z 004797e0 f   GameTime.obj
 0001:00078810       ?SetSpeed@CGameTime@@QAEXH@Z 00479810 f   GameTime.obj
 0001:00078980       ?SpeedMultiplier@CGameTime@@QBE?BMXZ 00479980 f   GameTime.obj
 0001:000789a0       ?Seconds@CGameTime@@QBE?BIXZ 004799a0 f   GameTime.obj
 0001:00078a00       ?GetSecondsSincePause@CGameTime@@QAE?BIXZ 00479a00 f   GameTime.obj
 0001:00078a40       ?IsPaused@CGameTime@@QBE?B_NXZ 00479a40 f   GameTime.obj
 0001:00078a80       ??0CGameTimer@@QAE@XZ      00479a80 f   GameTimer.obj
 0001:00078ab0       ?Reset@CGameTimer@@QAEXI@Z 00479ab0 f   GameTimer.obj
 0001:00078ad0       ?Adjust@CGameTimer@@IAEXHM@Z 00479ad0 f   GameTimer.obj
 0001:00078b10       ?Set@CGameTimer@@QAEXI@Z   00479b10 f   GameTimer.obj
 0001:00078b60       ?Get@CGameTimer@@QBE?BIXZ  00479b60 f   GameTimer.obj
 0001:00078b70       ?SecondsRemaining@CGameTimer@@QBE?BIXZ 00479b70 f   GameTimer.obj
 0001:00078be0       ?Increment@CGameTimer@@QAEXI@Z 00479be0 f   GameTimer.obj
 0001:00078c20       ?Pause@CGameTimer@@QAEXXZ  00479c20 f   GameTimer.obj
 0001:00078c50       ?IsActive@CGameTimer@@QBE?B_NXZ 00479c50 f   GameTimer.obj
 0001:00078c70       ?HasExpired@CGameTimer@@QBE?B_NXZ 00479c70 f   GameTimer.obj
 0001:00078cb0       ??0CPotion@@QAE@XZ         00479cb0 f   Potion.obj
 0001:00078cf0       ?Attach@CPotion@@UAEXAAVCVillager@@HAAH@Z 00479cf0 f   Potion.obj
 0001:00079720       ?Remove@CPotion@@UAEXAAVCVillager@@H@Z 0047a720 f   Potion.obj
 0001:00079770       ?Update@CPotion@@UAEXAAVCVillager@@HI@Z 0047a770 f   Potion.obj
 0001:00079790       ?DifficultyLevel@CPotion@@QBE?BHW4EPotion@@@Z 0047a790 f   Potion.obj
 0001:000797b0       ?SetJumpHeight@CVillagerState@@QAEXH@Z 0047a7b0 f i Potion.obj
 0001:000797d0       ??0CTech@@QAE@XZ           0047a7d0 f   Tech.obj
 0001:000797f0       ?Reset@CTech@@QAEXXZ       0047a7f0 f   Tech.obj
 0001:00079840       ?LoadState@CTech@@QAE?B_NABUSSaveState@1@@Z 0047a840 f   Tech.obj
 0001:00079910       ?SaveState@CTech@@QBE?B_NAAUSSaveState@1@@Z 0047a910 f   Tech.obj
 0001:00079950       ?RegisterObserver@CTech@@QAEXPAVITechObserver@@@Z 0047a950 f   Tech.obj
 0001:00079980       ?Level@CTech@@QBE?BHW4ETech@@@Z 0047a980 f   Tech.obj
 0001:000799a0       ?Advance@CTech@@QAEXW4ETech@@@Z 0047a9a0 f   Tech.obj
 0001:00079a20       ?UpgradePrice@CTech@@QBE?BHW4ETech@@@Z 0047aa20 f   Tech.obj
 0001:00079a60       ??0CTechPoints@@QAE@XZ     0047aa60 f   TechPoints.obj
 0001:00079a80       ?Reset@CTechPoints@@QAEXXZ 0047aa80 f   TechPoints.obj
 0001:00079aa0       ?LoadState@CTechPoints@@QAE?B_NABUSSaveState@1@@Z 0047aaa0 f   TechPoints.obj
 0001:00079ad0       ?SaveState@CTechPoints@@QBE?B_NAAUSSaveState@1@@Z 0047aad0 f   TechPoints.obj
 0001:00079af0       ?Adjust@CTechPoints@@QAEXH@Z 0047aaf0 f   TechPoints.obj
 0001:00079b80       ?IncrementPoints@CGameStats@@QAEXI@Z 0047ab80 f i TechPoints.obj
 0001:00079ba0       ?GetId@ldwControl@@QAEHXZ  0047aba0 f i ldwScene.obj
 0001:00079ba0       ?GetSize@?$CSimpleArray@GV?$CSimpleArrayEqualHelper@G@ATL@@@ATL@@QBEHXZ 0047aba0 f i FlashPlayer.obj
 0001:00079ba0       ?LastTimeChecked@CVillagerState@@QBE?BKXZ 0047aba0 f i VillagerManager.obj
 0001:00079ba0       ?GetHeight@ldwGameWindowImpl@@QAEHXZ 0047aba0 f i ldwGameWindow.obj
 0001:00079ba0       ?GetModuleInstance@CAtlBaseModule@ATL@@QAEPAUHINSTANCE__@@XZ 0047aba0 f i FlashPlayer.obj
 0001:00079ba0       ?GetTargetVillager@CIslandEvent@@UAEPAVCVillager@@XZ 0047aba0 f i IslandEvents.obj
 0001:00079ba0       ?Gender@CVillagerBio@@QBE?BW4EGender@@XZ 0047aba0 f i Behavior.obj
 0001:00079ba0       ?GetPointsEarned@CGameStats@@QBE?BIXZ 0047aba0 f i TechPoints.obj
 0001:00079bc0       ??0theGame@@QAE@XZ         0047abc0 f   theGame.obj
 0001:00079c30       ??1theGame@@UAE@XZ         0047ac30 f   theGame.obj
 0001:00079c50       ?Init@theGame@@UAE_NXZ     0047ac50 f   theGame.obj
 0001:00079e00       ?Shutdown@theGame@@UAEXXZ  0047ae00 f   theGame.obj
 0001:0007a140       ?GameUpdate@theGame@@UAEXXZ 0047b140 f   theGame.obj
 0001:0007a780       ?GameDraw@theGame@@UAEXXZ  0047b780 f   theGame.obj
 0001:0007ab20       ?HandleMessage@theGame@@UAE_NHJ@Z 0047bb20 f   theGame.obj
 0001:0007ab70       ?ArmadilloCheckIfRegistered@theGame@@QAE_NXZ 0047bb70 f   theGame.obj
 0001:0007ac20       ??_EtheGame@@UAEPAXI@Z     0047bc20 f i theGame.obj
 0001:0007ac20       ??_GtheGame@@UAEPAXI@Z     0047bc20 f i theGame.obj
 0001:0007ac50       ?Create@theGameState@@SAPAV1@XZ 0047bc50 f   theGameState.obj
 0001:0007ac60       ?Get@theGameState@@SAPAV1@XZ 0047bc60 f   theGameState.obj
 0001:0007ace0       ?Destroy@theGameState@@SAXXZ 0047bce0 f   theGameState.obj
 0001:0007ad30       ??1theGameState@@UAE@XZ    0047bd30 f   theGameState.obj
 0001:0007ad50       ?GetGameTitle@theGameState@@UAEPBDXZ 0047bd50 f   theGameState.obj
 0001:0007ad60       ?GetGameName@theGameState@@UAEPBDXZ 0047bd60 f   theGameState.obj
 0001:0007ad70       ?GetGameWindowWidth@theGameState@@UAEHXZ 0047bd70 f   theGameState.obj
 0001:0007ad80       ?GetGameWindowHeight@theGameState@@UAEHXZ 0047bd80 f   theGameState.obj
 0001:0007ad90       ?GetBitsPerPixel@theGameState@@UAEHXZ 0047bd90 f   theGameState.obj
 0001:0007ada0       ?StartWindowed@theGameState@@UAE_NXZ 0047bda0 f   theGameState.obj
 0001:0007adc0       ?Load@theGameState@@UAE_NH@Z 0047bdc0 f   theGameState.obj
 0001:0007b100       ?LoadCurrentGame@theGameState@@QAE_NXZ 0047c100 f   theGameState.obj
 0001:0007b2c0       ?Load@theGameState@@QAEXXZ 0047c2c0 f   theGameState.obj
 0001:0007b580       ?Save@theGameState@@UAE_NH@Z 0047c580 f   theGameState.obj
 0001:0007b6e0       ?SaveCurrentGame@theGameState@@QAE_NXZ 0047c6e0 f   theGameState.obj
 0001:0007b750       ?AutoSaveGame@theGameState@@QAEXXZ 0047c750 f   theGameState.obj
 0001:0007b790       ?RemoveGameFile@theGameState@@QAEXH@Z 0047c790 f   theGameState.obj
 0001:0007b7b0       ??0theGameState@@IAE@XZ    0047c7b0 f   theGameState.obj
 0001:0007b880       ?Init@theGameState@@QAEXXZ 0047c880 f   theGameState.obj
 0001:0007bda0       ?RestartCurrentGame@theGameState@@QAEXXZ 0047cda0 f   theGameState.obj
 0001:0007be00       ?InitOptions@theGameState@@IAEXXZ 0047ce00 f   theGameState.obj
 0001:0007be80       ?InitGameInfo@theGameState@@QAEXXZ 0047ce80 f   theGameState.obj
 0001:0007bfb0       ?CountSpiritualityRating@theGameState@@QAEHXZ 0047cfb0 f   theGameState.obj
 0001:0007bfc0       ?GetStatRealGameHoursThisGame@theGameState@@QAEJXZ 0047cfc0 f   theGameState.obj
 0001:0007c000       ?PlayerNeedsCorrection@theGameState@@QAEHXZ 0047d000 f   theGameState.obj
 0001:0007c010       ??_GtheGameState@@UAEPAXI@Z 0047d010 f i theGameState.obj
 0001:0007c010       ??_EtheGameState@@UAEPAXI@Z 0047d010 f i theGameState.obj
 0001:0007c040       ??0theGameData@@QAE@XZ     0047d040 f i theGameState.obj
 0001:0007c080       ??0SSaveState@CCollectableItem@@QAE@XZ 0047d080 f i theGameState.obj
 0001:0007c0b0       ??0SSaveState@CVillager@@QAE@XZ 0047d0b0 f i theGameState.obj
 0001:0007c110       ??0SSpawnArea@CCollectableItem@@QAE@XZ 0047d110 f i theGameState.obj
 0001:0007c110       ??0SSpawnArea@CBird@@QAE@XZ 0047d110 f i Bird.obj
 0001:0007c130       ?GetCurrentGameScene@theGameState@@UAEHXZ 0047d130 f i theGameState.obj
 0001:0007c150       ?SetPos@CWorldView@@QAEXHH@Z 0047d150 f i theGameState.obj
 0001:0007c180       ?Get@theRealtimeManager@@SAPAV1@XZ 0047d180 f   theRealtimeManager.obj
 0001:0007c200       ?Destroy@theRealtimeManager@@SAXXZ 0047d200 f   theRealtimeManager.obj
 0001:0007c240       ??0theRealtimeManager@@QAE@XZ 0047d240 f   theRealtimeManager.obj
 0001:0007c280       ??1theRealtimeManager@@QAE@XZ 0047d280 f   theRealtimeManager.obj
 0001:0007c290       ?UpdateAll@theRealtimeManager@@QAEXXZ 0047d290 f   theRealtimeManager.obj
 0001:0007c440       ??_GtheRealtimeManager@@QAEPAXI@Z 0047d440 f i theRealtimeManager.obj
 0001:0007c470       ?SetMaxPopulation@CGameStats@@QAEXH@Z 0047d470 f i theRealtimeManager.obj
 0001:0007c490       ?MaxPopulation@CGameStats@@QBE?BHXZ 0047d490 f i theRealtimeManager.obj
 0001:0007c4b0       ??0CDecal@@QAE@XZ          0047d4b0 f   Decal.obj
 0001:0007c4f0       ?Reset@CDecal@@QAEXXZ      0047d4f0 f   Decal.obj
 0001:0007c530       ?LoadAssets@CDecal@@QAEXXZ 0047d530 f   Decal.obj
 0001:0007c5f0       ?ReleaseAssets@CDecal@@QAEXXZ 0047d5f0 f   Decal.obj
 0001:0007c600       ?AddDecal@CDecal@@QAEXPAVldwImageGrid@@HH@Z 0047d600 f   Decal.obj
 0001:0007c670       ?AddDecal@CDecal@@QAEXPAVldwImageGrid@@HHH@Z 0047d670 f   Decal.obj
 0001:0007c700       ?DrawDecals@CDecal@@QAEXXZ 0047d700 f   Decal.obj
 0001:0007c7d0       ?DrawArrow@CDecal@@QAEXXZ  0047d7d0 f   Decal.obj
 0001:0007c830       ?DrawMiniDecals@CDecal@@QAEXHHM@Z 0047d830 f   Decal.obj
 0001:0007c930       ?InitDecals@CDecal@@QAEXXZ 0047d930 f   Decal.obj
 0001:0007c990       ?RefreshDecals@CDecal@@QAEXXZ 0047d990 f   Decal.obj
 0001:0007cc40       ?ShowArrow@CDecal@@QAEXPAVldwImage@@HH@Z 0047dc40 f   Decal.obj
 0001:0007cc80       ?HideArrow@CDecal@@QAEXXZ  0047dc80 f   Decal.obj
 0001:0007cca0       ??0CFloatingAnim@@QAE@XZ   0047dca0 f   FloatingAnim.obj
 0001:0007cce0       ??1CFloatingAnim@@QAE@XZ   0047dce0 f   FloatingAnim.obj
 0001:0007cd00       ?LoadAssets@CFloatingAnim@@QAEXXZ 0047dd00 f   FloatingAnim.obj
 0001:0007cd50       ?ReleaseAssets@CFloatingAnim@@QAEXXZ 0047dd50 f   FloatingAnim.obj
 0001:0007cd60       ?Reset@CFloatingAnim@@QAEXXZ 0047dd60 f   FloatingAnim.obj
 0001:0007cdb0       ?AddAnim@CFloatingAnim@@QAE?BHW4EFloatingAnim@@UldwPoint@@@Z 0047ddb0 f   FloatingAnim.obj
 0001:0007cde0       ?AddAnim@CFloatingAnim@@QAE?BHW4EFloatingAnim@@UldwPoint@@_N@Z 0047dde0 f   FloatingAnim.obj
 0001:0007ce10       ?AddAnim@CFloatingAnim@@QAE?BHW4EFloatingAnim@@UldwPoint@@H_NW4EFloatingAnimEffect@@W4EScenePriority@@2@Z 0047de10 f   FloatingAnim.obj
 0001:0007cfb0       ?ScareFish@CFloatingAnim@@QAEXUldwPoint@@@Z 0047dfb0 f   FloatingAnim.obj
 0001:0007d0a0       ?RemoveType@CFloatingAnim@@QAEXW4EFloatingAnim@@@Z 0047e0a0 f   FloatingAnim.obj
 0001:0007d0f0       ?Remove@CFloatingAnim@@UAEXH@Z 0047e0f0 f   FloatingAnim.obj
 0001:0007d120       ?UpdateOffset@SInst@CFloatingAnim@@QAEXXZ 0047e120 f   FloatingAnim.obj
 0001:0007d1b0       ?Draw@CFloatingAnim@@QBEXXZ 0047e1b0 f   FloatingAnim.obj
 0001:0007d290       ?DrawOverlays@CFloatingAnim@@QBEXXZ 0047e290 f   FloatingAnim.obj
 0001:0007d2f0       ?Draw@CFloatingAnim@@QBEXH@Z 0047e2f0 f   FloatingAnim.obj
 0001:0007d460       ?Update@CFloatingAnim@@QAEXXZ 0047e460 f   FloatingAnim.obj
 0001:0007d5c0       ?GetNumberOfType@CFloatingAnim@@QBE?BHW4EFloatingAnim@@@Z 0047e5c0 f   FloatingAnim.obj
 0001:0007d620       ?SetPos@CFloatingAnim@@UAEXHUldwPoint@@@Z 0047e620 f   FloatingAnim.obj
 0001:0007d660       ??0SInst@CFloatingAnim@@QAE@XZ 0047e660 f i FloatingAnim.obj
 0001:0007d690       ??0CSmoke@@QAE@XZ          0047e690 f   Smoke.obj
 0001:0007d6d0       ?Reset@CSmoke@@QAEXXZ      0047e6d0 f   Smoke.obj
 0001:0007d710       ?Add@CSmoke@@QAE?BHUldwPoint@@HW4EFloatingAnim@@H@Z 0047e710 f   Smoke.obj
 0001:0007d7c0       ?Remove@CSmoke@@UAEXH@Z    0047e7c0 f   Smoke.obj
 0001:0007d7f0       ?Update@CSmoke@@QAEXXZ     0047e7f0 f   Smoke.obj
 0001:0007d980       ?SetPos@CSmoke@@UAEXHUldwPoint@@@Z 0047e980 f   Smoke.obj
 0001:0007d9b0       ?SetIntensity@CSmoke@@QAEXHH@Z 0047e9b0 f   Smoke.obj
 0001:0007d9e0       ??0DecalsType@@QAE@XZ      0047e9e0 f i Decal.obj
 0001:0007d9e0       ??0SEmitter@CSmoke@@QAE@XZ 0047e9e0 f i Smoke.obj
 0001:0007da00       ??0CBehaviorEditor@@QAE@XZ 0047ea00 f   BehaviorEditor.obj
 0001:0007da50       ?Reset@CBehaviorEditor@@UAEXXZ 0047ea50 f   BehaviorEditor.obj
 0001:0007db20       ?GenerateBehaviorCode@CBehaviorEditor@@AAEXPBD@Z 0047eb20 f   BehaviorEditor.obj
 0001:0007dc70       ?GenerateCodeAtControlPoint@CBehaviorEditor@@AAEXPAU_iobuf@@H@Z 0047ec70 f   BehaviorEditor.obj
 0001:0007def0       ?GenerateOffsetPoint@CBehaviorEditor@@AAEPBDABUSControlPoint@1@@Z 0047eef0 f   BehaviorEditor.obj
 0001:0007df80       ?AddLine@CBehaviorEditor@@AAAXPAU_iobuf@@PBDZZ 0047ef80 f   BehaviorEditor.obj
 0001:0007e060       ?AddControlPointPlans@CBehaviorEditor@@AAEXPAU_iobuf@@ABUSControlPoint@1@@Z 0047f060 f   BehaviorEditor.obj
 0001:0007e440       ?AddControlPoint@CBehaviorEditor@@AAE?BHH@Z 0047f440 f   BehaviorEditor.obj
 0001:0007e540       ?AddControlPoint@CBehaviorEditor@@AAE?BHHW4EWaypoint@@@Z 0047f540 f   BehaviorEditor.obj
 0001:0007e5a0       ?AddControlPoint@CBehaviorEditor@@AAE?BHHW4EObject@CContentMap@@@Z 0047f5a0 f   BehaviorEditor.obj
 0001:0007e600       ?AddControlPoint@CBehaviorEditor@@AAE?BHHUldwPoint@@@Z 0047f600 f   BehaviorEditor.obj
 0001:0007e6d0       ?InsertControlPoint@CBehaviorEditor@@AAE?BHHHUldwPoint@@@Z 0047f6d0 f   BehaviorEditor.obj
 0001:0007e750       ?DeleteControlPoint@CBehaviorEditor@@AAEXH@Z 0047f750 f   BehaviorEditor.obj
 0001:0007e870       ?AddLink@CBehaviorEditor@@AAEXAAUSControlPoint@1@H@Z 0047f870 f   BehaviorEditor.obj
 0001:0007e8c0       ?DeleteLink@CBehaviorEditor@@AAEXAAUSControlPoint@1@H@Z 0047f8c0 f   BehaviorEditor.obj
 0001:0007e960       ?GetControlPoint@CBehaviorEditor@@ABE?BUldwPoint@@H@Z 0047f960 f   BehaviorEditor.obj
 0001:0007ea60       ?GetNearbyControlPoint@CBehaviorEditor@@ABE?BHUldwPoint@@@Z 0047fa60 f   BehaviorEditor.obj
 0001:0007eae0       ?SetControlPoint@CBehaviorEditor@@AAEXHUldwPoint@@@Z 0047fae0 f   BehaviorEditor.obj
 0001:0007eba0       ?SelectControlPointAtWaypoint@CBehaviorEditor@@AAE?B_NW4EWaypoint@@@Z 0047fba0 f   BehaviorEditor.obj
 0001:0007ec20       ?AddPlanToControlPoint@CBehaviorEditor@@AAEXH@Z 0047fc20 f   BehaviorEditor.obj
 0001:0007ece0       ?RemovePlanFromControlPoint@CBehaviorEditor@@AAEXHH@Z 0047fce0 f   BehaviorEditor.obj
 0001:0007ed90       ?MovePlanUp@CBehaviorEditor@@AAEXHAAH@Z 0047fd90 f   BehaviorEditor.obj
 0001:0007ee30       ?MovePlanDown@CBehaviorEditor@@AAEXHAAH@Z 0047fe30 f   BehaviorEditor.obj
 0001:0007eee0       ?UpdatePlanSelections@CBehaviorEditor@@AAEXXZ 0047fee0 f   BehaviorEditor.obj
 0001:0007ef80       ?ToggleSelectionsForPlan@CBehaviorEditor@@AAEXW4EPlan@1@@Z 0047ff80 f   BehaviorEditor.obj
 0001:0007f060       ?Draw@CBehaviorEditor@@UAEXXZ 00480060 f   BehaviorEditor.obj
 0001:0007f9d0       ?DrawControlPoint@CBehaviorEditor@@ABEXH@Z 004809d0 f   BehaviorEditor.obj
 0001:0007fc40       ?HandleKeyCharacter@CBehaviorEditor@@UAE?B_ND@Z 00480c40 f   BehaviorEditor.obj
 0001:000802a0       ?HandleKeyDown@CBehaviorEditor@@UAE?B_NH@Z 004812a0 f   BehaviorEditor.obj
 0001:00080430       ?HandleKeyUp@CBehaviorEditor@@UAE?B_NH@Z 00481430 f   BehaviorEditor.obj
 0001:00080470       ?HandleMouseDown@CBehaviorEditor@@UAE?B_NUldwPoint@@@Z 00481470 f   BehaviorEditor.obj
 0001:000806e0       ?HandleMouseUp@CBehaviorEditor@@UAE?B_NUldwPoint@@@Z 004816e0 f   BehaviorEditor.obj
 0001:00080700       ?HandleMouseMove@CBehaviorEditor@@UAE?B_NUldwPoint@@@Z 00481700 f   BehaviorEditor.obj
 0001:000807c0       ?FindNearestLine@CBehaviorEditor@@QAEXHUldwPoint@@AAH11@Z 004817c0 f   BehaviorEditor.obj
 0001:00080980       ?GetPlanName@CBehaviorEditor@@ABEPBDW4EPlan@1@@Z 00481980 f   BehaviorEditor.obj
 0001:000809a0       ?GetSkillName@CBehaviorEditor@@ABEPBDW4ESkill@@@Z 004819a0 f   BehaviorEditor.obj
 0001:000809c0       ?GetSkillEnumName@CBehaviorEditor@@ABEPBDW4ESkill@@@Z 004819c0 f   BehaviorEditor.obj
 0001:000809e0       ?GetBodyPositionName@CBehaviorEditor@@ABEPBDW4EBodyPosition@@@Z 004819e0 f   BehaviorEditor.obj
 0001:00080a00       ?GetBodyPositionEnumName@CBehaviorEditor@@ABEPBDW4EBodyPosition@@@Z 00481a00 f   BehaviorEditor.obj
 0001:00080a20       ?GetCarryingName@CBehaviorEditor@@ABEPBDW4ECarrying@@@Z 00481a20 f   BehaviorEditor.obj
 0001:00080a40       ?GetCarryingEnumName@CBehaviorEditor@@ABEPBDW4ECarrying@@@Z 00481a40 f   BehaviorEditor.obj
 0001:00080a60       ?GetDirectionName@CBehaviorEditor@@ABEPBDW4EDirection@@@Z 00481a60 f   BehaviorEditor.obj
 0001:00080a80       ?GetDirectionEnumName@CBehaviorEditor@@ABEPBDW4EDirection@@@Z 00481a80 f   BehaviorEditor.obj
 0001:00080aa0       ?GetHeadDirectionName@CBehaviorEditor@@ABEPBDW4EHeadDirection@@@Z 00481aa0 f   BehaviorEditor.obj
 0001:00080ac0       ?GetHeadDirectionEnumName@CBehaviorEditor@@ABEPBDW4EHeadDirection@@@Z 00481ac0 f   BehaviorEditor.obj
 0001:00080ae0       ?GetSoundName@CBehaviorEditor@@ABEPBDW4ESound@@@Z 00481ae0 f   BehaviorEditor.obj
 0001:00080b00       ?GetSoundEnumName@CBehaviorEditor@@ABEPBDW4ESound@@@Z 00481b00 f   BehaviorEditor.obj
 0001:00080b20       ??0IEditor@@QAE@XZ         00481b20 f i BehaviorEditor.obj
 0001:00080b40       ??0SControlPoint@CBehaviorEditor@@QAE@XZ 00481b40 f i BehaviorEditor.obj
 0001:00080b70       ??0CContentMapEditor@@QAE@XZ 00481b70 f   ContentMapEditor.obj
 0001:00080bb0       ?Reset@CContentMapEditor@@UAEXXZ 00481bb0 f   ContentMapEditor.obj
 0001:00080c40       ?Draw@CContentMapEditor@@UAEXXZ 00481c40 f   ContentMapEditor.obj
 0001:000811c0       ?HandleKeyCharacter@CContentMapEditor@@UAE?B_ND@Z 004821c0 f   ContentMapEditor.obj
 0001:00081390       ?HandleKeyDown@CContentMapEditor@@UAE?B_NH@Z 00482390 f   ContentMapEditor.obj
 0001:000814f0       ?HandleKeyUp@CContentMapEditor@@UAE?B_NH@Z 004824f0 f   ContentMapEditor.obj
 0001:00081520       ?HandleMouseDown@CContentMapEditor@@UAE?B_NUldwPoint@@@Z 00482520 f   ContentMapEditor.obj
 0001:00081580       ?HandleMouseUp@CContentMapEditor@@UAE?B_NUldwPoint@@@Z 00482580 f   ContentMapEditor.obj
 0001:00081860       ?HandleMouseMove@CContentMapEditor@@UAE?B_NUldwPoint@@@Z 00482860 f   ContentMapEditor.obj
 0001:00081ab0       ?GetModeName@CContentMapEditor@@ABEPBDW4EMode@1@@Z 00482ab0 f   ContentMapEditor.obj
 0001:00081ad0       ?GetMaterialName@CContentMapEditor@@QBEPBDW4EMaterial@CContentMap@@@Z 00482ad0 f   ContentMapEditor.obj
 0001:00081af0       ?GetObjectName@CContentMapEditor@@QBEPBDW4EObject@CContentMap@@@Z 00482af0 f   ContentMapEditor.obj
 0001:00081b10       ?GetObjectEnumName@CContentMapEditor@@QBEPBDW4EObject@CContentMap@@@Z 00482b10 f   ContentMapEditor.obj
 0001:00081b30       ?GetHotSpotName@CContentMapEditor@@QBEPBDW4EHotSpot@CContentMap@@@Z 00482b30 f   ContentMapEditor.obj
 0001:00081b50       ?GetRedirectorName@CContentMapEditor@@QBEPBDW4ERedirector@CContentMap@@@Z 00482b50 f   ContentMapEditor.obj
 0001:00081b70       ??0CDebugger@@QAE@XZ       00482b70 f   Debugger.obj
 0001:00081ba0       ?Reset@CDebugger@@QAEXXZ   00482ba0 f   Debugger.obj
 0001:00081bd0       ?Register@CDebugger@@QAE?B_NPAVIDebugger@@@Z 00482bd0 f   Debugger.obj
 0001:00081c10       ?AddLine@CDebugger@@QAAXPBDZZ 00482c10 f   Debugger.obj
 0001:00081c80       ?Draw@CDebugger@@QAEXXZ    00482c80 f   Debugger.obj
 0001:00081d90       ?HandleKeyCharacter@CDebugger@@QAE?B_ND@Z 00482d90 f   Debugger.obj
 0001:00081da0       ?HandleKeyDown@CDebugger@@QAE?B_NH@Z 00482da0 f   Debugger.obj
 0001:00081e70       ?HandleKeyUp@CDebugger@@QAE?B_NH@Z 00482e70 f   Debugger.obj
 0001:00081e80       ??0CEditor@@QAE@XZ         00482e80 f   Editor.obj
 0001:00081ea0       ?Reset@CEditor@@QAEXXZ     00482ea0 f   Editor.obj
 0001:00081ee0       ?Draw@CEditor@@QAEXXZ      00482ee0 f   Editor.obj
 0001:00082010       ?HandleKeyCharacter@CEditor@@QAE?B_ND@Z 00483010 f   Editor.obj
 0001:00082040       ?HandleKeyDown@CEditor@@QAE?B_NH@Z 00483040 f   Editor.obj
 0001:00082100       ?HandleKeyUp@CEditor@@QAE?B_NH@Z 00483100 f   Editor.obj
 0001:00082130       ?HandleMouseDown@CEditor@@QAE?B_NUldwPoint@@@Z 00483130 f   Editor.obj
 0001:00082170       ?HandleMouseUp@CEditor@@QAE?B_NUldwPoint@@@Z 00483170 f   Editor.obj
 0001:000821b0       ?HandleMouseMove@CEditor@@QAE?B_NUldwPoint@@@Z 004831b0 f   Editor.obj
 0001:000821f0       ??0CWaypointEditor@@QAE@XZ 004831f0 f   WaypointEditor.obj
 0001:00082220       ?Reset@CWaypointEditor@@UAEXXZ 00483220 f   WaypointEditor.obj
 0001:00082240       ?LoadAssets@CWaypointEditor@@QAEXXZ 00483240 f   WaypointEditor.obj
 0001:00082260       ?ReleaseAssets@CWaypointEditor@@QAEXXZ 00483260 f   WaypointEditor.obj
 0001:00082270       ?Draw@CWaypointEditor@@UAEXXZ 00483270 f   WaypointEditor.obj
 0001:00082360       ?DrawWaypoints@CWaypointEditor@@QAEXXZ 00483360 f   WaypointEditor.obj
 0001:000824a0       ?HandleKeyCharacter@CWaypointEditor@@UAE?B_ND@Z 004834a0 f   WaypointEditor.obj
 0001:00082540       ?HandleKeyDown@CWaypointEditor@@UAE?B_NH@Z 00483540 f   WaypointEditor.obj
 0001:00082570       ?HandleKeyUp@CWaypointEditor@@UAE?B_NH@Z 00483570 f   WaypointEditor.obj
 0001:00082580       ?HandleMouseDown@CWaypointEditor@@UAE?B_NUldwPoint@@@Z 00483580 f   WaypointEditor.obj
 0001:000825e0       ?HandleMouseUp@CWaypointEditor@@UAE?B_NUldwPoint@@@Z 004835e0 f   WaypointEditor.obj
 0001:00082600       ?HandleMouseMove@CWaypointEditor@@UAE?B_NUldwPoint@@@Z 00483600 f   WaypointEditor.obj
 0001:00082680       ?GetWaypointName@CWaypointEditor@@QBEPBDW4EWaypoint@@@Z 00483680 f   WaypointEditor.obj
 0001:000826a0       ?GetWaypointEnumName@CWaypointEditor@@QBEPBDW4EWaypoint@@@Z 004836a0 f   WaypointEditor.obj
 0001:000826c0       ?Set@CWaypoint@@IAEXW4EWaypoint@@UldwPoint@@@Z 004836c0 f i WaypointEditor.obj
 0001:000826e0       ??0CCollectable@@QAE@XZ    004836e0 f   Collectable.obj
 0001:00083000       ?RegisterObserver@CCollectable@@QAEXW4ECarrying@@PAVICollectable@@@Z 00484000 f   Collectable.obj
 0001:00083050       ?ProcessNearbyCollectables@CCollectable@@QBE?B_NAAVCVillager@@@Z 00484050 f   Collectable.obj
 0001:00083160       ?Carry@CCollectable@@QBE?B_NAAVCVillager@@W4ECarrying@@@Z 00484160 f   Collectable.obj
 0001:00083200       ?Drop@CCollectable@@QBEXAAVCVillager@@W4ECarrying@@@Z 00484200 f   Collectable.obj
 0001:00083270       ??0CWindow@ATL@@QAE@PAUHWND__@@@Z 00484270 f i FlashPlayer.obj
 0001:00083270       ??0SConstructionData@@QAE@W4EConstruction@@@Z 00484270 f i VillagerAI.obj
 0001:00083270       ??0CAtlException@ATL@@QAE@J@Z 00484270 f i FlashPlayer.obj
 0001:00083270       ??0SHarvestFruitData@@QAE@H@Z 00484270 f i VillagerAI.obj
 0001:00083270       ??0SGatherHerbsData@@QAE@W4ECarrying@@@Z 00484270 f i HotSpot.obj
 0001:00083270       ??0SPickUpData@@QAE@W4ECarrying@@@Z 00484270 f i Collectable.obj
 0001:00083270       ??0SStringData@@QAE@W4StringId@@@Z 00484270 f i Behavior.obj
 0001:00083270       ??0_U_MENUorID@ATL@@QAE@I@Z 00484270 f i FlashPlayer.obj
 0001:00083270       ??0_U_RECT@ATL@@QAE@PAUtagRECT@@@Z 00484270 f i FlashPlayer.obj
 0001:00083290       ??0CCollectableItem@@QAE@XZ 00484290 f   CollectableItem.obj
 0001:000832f0       ?Reset@CCollectableItem@@QAEXXZ 004842f0 f   CollectableItem.obj
 0001:00083470       ?LoadAssets@CCollectableItem@@QAEXXZ 00484470 f   CollectableItem.obj
 0001:000834a0       ?ReleaseAssets@CCollectableItem@@QAEXXZ 004844a0 f   CollectableItem.obj
 0001:000834b0       ?LoadState@CCollectableItem@@QAE?B_NABUSSaveState@1@@Z 004844b0 f   CollectableItem.obj
 0001:00083590       ?SaveState@CCollectableItem@@QBE?B_NAAUSSaveState@1@@Z 00484590 f   CollectableItem.obj
 0001:00083640       ?AddSpawnArea@CCollectableItem@@QAEXUldwRect@@W4ECarrying@@@Z 00484640 f   CollectableItem.obj
 0001:000836b0       ?Add@CCollectableItem@@QAEXW4ECarrying@@UldwPoint@@@Z 004846b0 f   CollectableItem.obj
 0001:000839e0       ?AddRare@CCollectableItem@@QAEXXZ 004849e0 f   CollectableItem.obj
 0001:00083c10       ?Remove@CCollectableItem@@QAEXH@Z 00484c10 f   CollectableItem.obj
 0001:00083c30       ?AddTutorialItem@CCollectableItem@@QAEXXZ 00484c30 f   CollectableItem.obj
 0001:00083c90       ?Update@CCollectableItem@@QAEXXZ 00484c90 f   CollectableItem.obj
 0001:00083e80       ?Draw@CCollectableItem@@QAEXXZ 00484e80 f   CollectableItem.obj
 0001:00083ed0       ?Draw@CCollectableItem@@QAEXH@Z 00484ed0 f   CollectableItem.obj
 0001:00083f40       ?Carry@CCollectableItem@@UAE?B_NAAVCVillager@@W4ECarrying@@@Z 00484f40 f   CollectableItem.obj
 0001:00084000       ?Drop@CCollectableItem@@UAEXAAVCVillager@@W4ECarrying@@@Z 00485000 f   CollectableItem.obj
 0001:000842a0       ?GetNearbyCollectable@CCollectableItem@@UAE?BW4ECarrying@@AAVCVillager@@UldwPoint@@@Z 004852a0 f   CollectableItem.obj
 0001:00084370       ?IsCommonCollectable@CCollectableItem@@QBE?B_NW4ECarrying@@@Z 00485370 f   CollectableItem.obj
 0001:000843c0       ?IsUncommonCollectable@CCollectableItem@@QBE?B_NW4ECarrying@@@Z 004853c0 f   CollectableItem.obj
 0001:00084410       ?IsRareCollectable@CCollectableItem@@QBE?B_NW4ECarrying@@@Z 00485410 f   CollectableItem.obj
 0001:00084460       ?IsCollectionComplete@CCollectableItem@@QBE?B_NW4ECarrying@@@Z 00485460 f   CollectableItem.obj
 0001:00084490       ?CollectionCount@CCollectableItem@@QBE?BHW4ECarrying@@_N11@Z 00485490 f   CollectableItem.obj
 0001:00084590       ?Count@CCollectableItem@@QBE?BHW4ECarrying@@@Z 00485590 f   CollectableItem.obj
 0001:000845b0       ?WasItemSpawned@CCollectableItem@@QBE?B_NW4ECarrying@@@Z 004855b0 f   CollectableItem.obj
 0001:00084610       ?IsItemBeingCarried@CCollectableItem@@QBE?B_NW4ECarrying@@@Z 00485610 f   CollectableItem.obj
 0001:00084630       ?WasTabletCollected@CCollectableItem@@QBE?B_NW4ECarrying@@@Z 00485630 f   CollectableItem.obj
 0001:00084660       ??0ICollectable@@QAE@XZ    00485660 f i CollectableItem.obj
 0001:00084680       ??0SCollectable@CCollectableItem@@QAE@XZ 00485680 f i CollectableItem.obj
 0001:000846a0       ?IncrementItemsFound@CGameStats@@QAEXH@Z 004856a0 f i CollectableItem.obj
 0001:000846c0       ??0CDealerSay@@QAE@XZ      004856c0 f   DealerSay.obj
 0001:000846e0       ?Reset@CDealerSay@@QAEXXZ  004856e0 f   DealerSay.obj
 0001:00084700       ?Update@CDealerSay@@QAEXXZ 00485700 f   DealerSay.obj
 0001:00084750       ?Say@CDealerSay@@QAEXW4StringId@@H@Z 00485750 f   DealerSay.obj
 0001:000847d0       ?Say@CDealerSay@@QAEXW4StringId@@PBD@Z 004857d0 f   DealerSay.obj
 0001:00084820       ?Say@CDealerSay@@QAEXW4StringId@@W4EGender@@@Z 00485820 f   DealerSay.obj
 0001:000848c0       ?Say@CDealerSay@@QAEXW4StringId@@PBDW4EGender@@1@Z 004858c0 f   DealerSay.obj
 0001:00084920       ?Say@CDealerSay@@QAEXPBD@Z 00485920 f   DealerSay.obj
 0001:00084960       ?Message@CDealerSay@@QBEPBDXZ 00485960 f   DealerSay.obj
 0001:00084970       ??0CSceneManager@@QAE@XZ   00485970 f   SceneManager.obj
 0001:000849b0       ?BeginScene@CSceneManager@@QAEXUldwPoint@@M@Z 004859b0 f   SceneManager.obj
 0001:00084a10       ?EndScene@CSceneManager@@QAEXXZ 00485a10 f   SceneManager.obj
 0001:00084c10       ?AddElement@CSceneManager@@QAEXW4ESceneElement@@HW4EScenePriority@@H@Z 00485c10 f   SceneManager.obj
 0001:00084c80       ?Draw@CSceneManager@@QBEXPAVldwImage@@UldwPoint@@M@Z 00485c80 f   SceneManager.obj
 0001:00084ce0       ?Draw@CSceneManager@@QBEXPAVldwImageGrid@@UldwPoint@@HM@Z 00485ce0 f   SceneManager.obj
 0001:00084d50       ?DrawScaled@CSceneManager@@QBEXPAVldwImage@@UldwPoint@@M_N@Z 00485d50 f   SceneManager.obj
 0001:00084dc0       ?DrawScaled@CSceneManager@@QBEXPAVldwImageGrid@@UldwPoint@@HHM@Z 00485dc0 f   SceneManager.obj
 0001:00084e30       ?Get@theDealerSay@@SAPAV1@XZ 00485e30 f   theDealerSay.obj
 0001:00084eb0       ?Destroy@theDealerSay@@SAXXZ 00485eb0 f   theDealerSay.obj
 0001:00084ef0       ??0theDealerSay@@IAE@XZ    00485ef0 f   theDealerSay.obj
 0001:00084f70       ??1theDealerSay@@IAE@XZ    00485f70 f   theDealerSay.obj
 0001:00084fb0       ?Say@theDealerSay@@QAEXW4StringId@@@Z 00485fb0 f   theDealerSay.obj
 0001:00084fd0       ?Draw@theDealerSay@@QAE_NXZ 00485fd0 f   theDealerSay.obj
 0001:00084ff0       ??_GtheDealerSay@@IAEPAXI@Z 00485ff0 f i theDealerSay.obj
 0001:00085020       ??0theDealerSayImpl@@QAE@XZ 00486020 f i theDealerSay.obj
 0001:00085170       ??_GtheDealerSayImpl@@QAEPAXI@Z 00486170 f i theDealerSay.obj
 0001:000851a0       ??1theDealerSayImpl@@QAE@XZ 004861a0 f i theDealerSay.obj
 0001:000851e0       ?Say@theDealerSayImpl@@QAEXW4StringId@@@Z 004861e0 f i theDealerSay.obj
 0001:00085220       ?Draw@theDealerSayImpl@@QAE_NXZ 00486220 f i theDealerSay.obj
 0001:00085300       ?Get@theGraphicsManager@@SAPAV1@XZ 00486300 f   theGraphicsManager.obj
 0001:00085380       ?Destroy@theGraphicsManager@@SAXXZ 00486380 f   theGraphicsManager.obj
 0001:000853c0       ??0theGraphicsManager@@IAE@XZ 004863c0 f   theGraphicsManager.obj
 0001:00085440       ??1theGraphicsManager@@IAE@XZ 00486440 f   theGraphicsManager.obj
 0001:00085480       ?GetImage@theGraphicsManager@@QAEPAVldwImage@@W4EImage@@@Z 00486480 f   theGraphicsManager.obj
 0001:000854a0       ?ReleaseImage@theGraphicsManager@@QAEXW4EImage@@_N@Z 004864a0 f   theGraphicsManager.obj
 0001:000854c0       ?GetImageStrip@theGraphicsManager@@QAEPAVldwImageStrip@@W4EImage@@@Z 004864c0 f   theGraphicsManager.obj
 0001:000854e0       ?GetImageGrid@theGraphicsManager@@QAEPAVldwImageGrid@@W4EImage@@@Z 004864e0 f   theGraphicsManager.obj
 0001:00085500       ?GetImageType@theGraphicsManager@@QAE?AW4EImageType@@W4EImage@@@Z 00486500 f   theGraphicsManager.obj
 0001:00085520       ?GetCellCount@theGraphicsManager@@QAEHW4EImage@@@Z 00486520 f   theGraphicsManager.obj
 0001:00085590       ?Draw@theGraphicsManager@@QAEXW4EImage@@HHMH@Z 00486590 f   theGraphicsManager.obj
 0001:00085700       ?DrawCell@theGraphicsManager@@QAEXW4EImage@@HHHMH@Z 00486700 f   theGraphicsManager.obj
 0001:00085860       ??_GtheGraphicsManager@@IAEPAXI@Z 00486860 f i theGraphicsManager.obj
 0001:00085890       ??_GtheGraphicsManagerImpl@@QAEPAXI@Z 00486890 f i theGraphicsManager.obj
 0001:000858c0       ??1theGraphicsManagerImpl@@QAE@XZ 004868c0 f i theGraphicsManager.obj
 0001:000859c0       ?GetImage@theGraphicsManagerImpl@@QAEPAVldwImage@@H@Z 004869c0 f i theGraphicsManager.obj
 0001:00085ab0       ?GetImageEntry@theGraphicsManagerImpl@@QAEPAUImageDescriptor@@H@Z 00486ab0 f i theGraphicsManager.obj
 0001:00085b30       ?GetImageStrip@theGraphicsManagerImpl@@QAEPAVldwImageStrip@@H@Z 00486b30 f i theGraphicsManager.obj
 0001:00085c00       ?GetImageGrid@theGraphicsManagerImpl@@QAEPAVldwImageGrid@@H@Z 00486c00 f i theGraphicsManager.obj
 0001:00085d60       ?ReleaseImage@theGraphicsManagerImpl@@QAEXH_N@Z 00486d60 f i theGraphicsManager.obj
 0001:00085e80       ?GetImageType@theGraphicsManagerImpl@@QAE?AW4EImageType@@H@Z 00486e80 f i theGraphicsManager.obj
 0001:00085ed0       ?Get@thePrizeMsgAssembler@@SAPAV1@XZ 00486ed0 f   thePrizeMsgAssembler.obj
 0001:00085f50       ?Destroy@thePrizeMsgAssembler@@SAXXZ 00486f50 f   thePrizeMsgAssembler.obj
 0001:00085f90       ??0thePrizeMsgAssembler@@QAE@XZ 00486f90 f   thePrizeMsgAssembler.obj
 0001:00085fc0       ??1thePrizeMsgAssembler@@QAE@XZ 00486fc0 f   thePrizeMsgAssembler.obj
 0001:00085fd0       ?CompileTechPrize@thePrizeMsgAssembler@@QAEPADPADHH@Z 00486fd0 f   thePrizeMsgAssembler.obj
 0001:00086030       ?CompileFoodPrize@thePrizeMsgAssembler@@QAEPADPADHH@Z 00487030 f   thePrizeMsgAssembler.obj
 0001:00086090       ?CompileMiscPrize@thePrizeMsgAssembler@@QAEPADPADHH0@Z 00487090 f   thePrizeMsgAssembler.obj
 0001:000860e0       ?CompilePrizeMsg@thePrizeMsgAssembler@@AAEXPADH0H@Z 004870e0 f   thePrizeMsgAssembler.obj
 0001:00086390       ?PrepareStringImpl@thePrizeMsgAssembler@@QAEPADPAD00H@Z 00487390 f   thePrizeMsgAssembler.obj
 0001:000866a0       ?PrepareString@thePrizeMsgAssembler@@QAEPADPAD00H@Z 004876a0 f   thePrizeMsgAssembler.obj
 0001:000866d0       ??_GthePrizeMsgAssembler@@QAEPAXI@Z 004876d0 f i thePrizeMsgAssembler.obj
 0001:00086700       ?Get@theSlicedVariableMeter@@SAPAV1@XZ 00487700 f   theSlicedVariableMeter.obj
 0001:00086780       ?Destroy@theSlicedVariableMeter@@SAXXZ 00487780 f   theSlicedVariableMeter.obj
 0001:000867c0       ??0theSlicedVariableMeter@@QAE@XZ 004877c0 f   theSlicedVariableMeter.obj
 0001:00086840       ?DrawPercentMeter@theSlicedVariableMeter@@QAEXW4SlMeterColorEnum@@H@Z 00487840 f   theSlicedVariableMeter.obj
 0001:00086ac0       ??1theSlicedVariableMeter@@QAE@XZ 00487ac0 f   theSlicedVariableMeter.obj
 0001:00086ad0       ??_GtheSlicedVariableMeter@@QAEPAXI@Z 00487ad0 f i theSlicedVariableMeter.obj
 0001:00086b00       ?Get@theStringManager@@SAPAV1@XZ 00487b00 f   theStringManager.obj
 0001:00086b80       ?Destroy@theStringManager@@SAXXZ 00487b80 f   theStringManager.obj
 0001:00086bc0       ??0theStringManager@@IAE@XZ 00487bc0 f   theStringManager.obj
 0001:00086c40       ??1theStringManager@@IAE@XZ 00487c40 f   theStringManager.obj
 0001:00086cb0       ?LoadFonts@theStringManager@@QAEXXZ 00487cb0 f   theStringManager.obj
 0001:00086d20       ?GetString@theStringManager@@QAEPADW4StringId@@@Z 00487d20 f   theStringManager.obj
 0001:00086d40       ?GetStringFromNameGenderTemplate@theStringManager@@QAEXPADHW4StringId@@PBD_NH23@Z 00487d40 f   theStringManager.obj
 0001:000870f0       ??_GtheStringManager@@IAEPAXI@Z 004880f0 f i theStringManager.obj
 0001:00087120       ??0theStringManagerImpl@@QAE@XZ 00488120 f i theStringManager.obj
 0001:000874d0       ?GetStringItem@theStringManagerImpl@@QAEPAUStringItem@@H@Z 004884d0 f i theStringManager.obj
 0001:00087520       ??_GtheStringManagerImpl@@QAEPAXI@Z 00488520 f i theStringManager.obj
 0001:00087550       ??1theStringManagerImpl@@QAE@XZ 00488550 f i theStringManager.obj
 0001:00087580       ?GetString@theStringManagerImpl@@QAEPADH@Z 00488580 f i theStringManager.obj
 0001:000875f0       ?Get@theVariableMeter@@SAPAV1@XZ 004885f0 f   theVariableMeter.obj
 0001:00087670       ?Destroy@theVariableMeter@@SAXXZ 00488670 f   theVariableMeter.obj
 0001:000876b0       ??0theVariableMeter@@QAE@XZ 004886b0 f   theVariableMeter.obj
 0001:00087700       ?DrawPercentMeter@theVariableMeter@@QAEXW4MeterColorEnum@@HHH@Z 00488700 f   theVariableMeter.obj
 0001:000878e0       ??1theVariableMeter@@QAE@XZ 004888e0 f   theVariableMeter.obj
 0001:000878f0       ??_GtheVariableMeter@@QAEPAXI@Z 004888f0 f i theVariableMeter.obj
 0001:00087920       ??0CAlchemyLab@@QAE@XZ     00488920 f   AlchemyLab.obj
 0001:000879a0       ?Reset@CAlchemyLab@@UAEXXZ 004889a0 f   AlchemyLab.obj
 0001:00087c10       ?LoadAssets@CAlchemyLab@@UAEXXZ 00488c10 f   AlchemyLab.obj
 0001:00087c60       ?ReleaseAssets@CAlchemyLab@@UAEXXZ 00488c60 f   AlchemyLab.obj
 0001:00087c70       ?LoadState@CAlchemyLab@@UAE?BHPBE@Z 00488c70 f   AlchemyLab.obj
 0001:00087d60       ?SaveState@CAlchemyLab@@UBE?BHPBEH@Z 00488d60 f   AlchemyLab.obj
 0001:00087de0       ?Complete@CAlchemyLab@@UAEXXZ 00488de0 f   AlchemyLab.obj
 0001:00087e20       ?Draw@CAlchemyLab@@UBEXXZ  00488e20 f   AlchemyLab.obj
 0001:00087e40       ?Draw@CAlchemyLab@@UBEXH@Z 00488e40 f   AlchemyLab.obj
 0001:00087eb0       ?Carry@CAlchemyLab@@UAE?B_NAAVCVillager@@W4ECarrying@@@Z 00488eb0 f   AlchemyLab.obj
 0001:00087f20       ?Drop@CAlchemyLab@@UAEXAAVCVillager@@W4ECarrying@@@Z 00488f20 f   AlchemyLab.obj
 0001:00088070       ?GetNearbyCollectable@CAlchemyLab@@UAE?BW4ECarrying@@AAVCVillager@@UldwPoint@@@Z 00489070 f   AlchemyLab.obj
 0001:000881b0       ?IsRepaired@CAlchemyLab@@QBE?B_NXZ 004891b0 f   AlchemyLab.obj
 0001:000881d0       ??0IPuzzle@@QAE@XZ         004891d0 f i AlchemyLab.obj
 0001:000881f0       ??0SAttachment@CVillager@@QAE@XZ 004891f0 f i Villager.obj
 0001:000881f0       ??0SFruit@COrchard@@QAE@XZ 004891f0 f i Orchard.obj
 0001:000881f0       ??0SPiece@CAlchemyLab@@QAE@XZ 004891f0 f i AlchemyLab.obj
 0001:00088210       ?Advance@IPuzzle@@UAEXAAVCVillager@@H@Z 00489210 f i AlchemyLab.obj
 0001:00088210       ?Remove@IVillagerAttachment@@UAEXAAVCVillager@@H@Z 00489210 f i EnvironmentalSound.obj
 0001:00088220       ??0CAlchemyPot@@QAE@XZ     00489220 f   AlchemyPot.obj
 0001:00088280       ?Reset@CAlchemyPot@@UAEXXZ 00489280 f   AlchemyPot.obj
 0001:00088790       ?LoadAssets@CAlchemyPot@@UAEXXZ 00489790 f   AlchemyPot.obj
 0001:000887a0       ?ReleaseAssets@CAlchemyPot@@UAEXXZ 004897a0 f   AlchemyPot.obj
 0001:000887b0       ?LoadState@CAlchemyPot@@UAE?BHPBE@Z 004897b0 f   AlchemyPot.obj
 0001:00088830       ?SaveState@CAlchemyPot@@UBE?BHPBEH@Z 00489830 f   AlchemyPot.obj
 0001:000888a0       ?ResetPotion@CAlchemyPot@@QAEXXZ 004898a0 f   AlchemyPot.obj
 0001:00088940       ?Refresh@CAlchemyPot@@UAEXXZ 00489940 f   AlchemyPot.obj
 0001:00088970       ?Complete@CAlchemyPot@@UAEXXZ 00489970 f   AlchemyPot.obj
 0001:00088ca0       ?Advance@CAlchemyPot@@UAEXAAVCVillager@@H@Z 00489ca0 f   AlchemyPot.obj
 0001:00088ce0       ?Carry@CAlchemyPot@@UAE?B_NAAVCVillager@@W4ECarrying@@@Z 00489ce0 f   AlchemyPot.obj
 0001:00088cf0       ?Drop@CAlchemyPot@@UAEXAAVCVillager@@W4ECarrying@@@Z 00489cf0 f   AlchemyPot.obj
 0001:00088d70       ?GetNearbyCollectable@CAlchemyPot@@UAE?BW4ECarrying@@AAVCVillager@@UldwPoint@@@Z 00489d70 f   AlchemyPot.obj
 0001:00088d80       ?AddPotionEffect@CAlchemyPot@@QAEXXZ 00489d80 f   AlchemyPot.obj
 0001:00088ee0       ?AddRecipe@CAlchemyPot@@QAE?BHW4ECarrying@@00W4EPotion@@@Z 00489ee0 f   AlchemyPot.obj
 0001:00088fd0       ?MixPotion@CAlchemyPot@@QAE?BW4EPotion@@W4ECarrying@@00@Z 00489fd0 f   AlchemyPot.obj
 0001:000890b0       ?HashIngredients@CAlchemyPot@@QBE?BHW4ECarrying@@00@Z 0048a0b0 f   AlchemyPot.obj
 0001:00089170       ?FindRecipe@CAlchemyPot@@QBE?BHW4ECarrying@@00@Z 0048a170 f   AlchemyPot.obj
 0001:000891e0       ?IsPotionReady@CAlchemyPot@@QBE?B_NXZ 0048a1e0 f   AlchemyPot.obj
 0001:00089200       ?Attach@CVillager@@QAE?B_NAAVIVillagerAttachment@@HH@Z 0048a200 f i AlchemyPot.obj
 0001:00089240       ??0CAlchemyTable@@QAE@XZ   0048a240 f   AlchemyTable.obj
 0001:00089290       ?Reset@CAlchemyTable@@UAEXXZ 0048a290 f   AlchemyTable.obj
 0001:000892f0       ?ResetAll@CAlchemyTable@@QAEXXZ 0048a2f0 f   AlchemyTable.obj
 0001:000893b0       ?LoadAssets@CAlchemyTable@@UAEXXZ 0048a3b0 f   AlchemyTable.obj
 0001:000893d0       ?ReleaseAssets@CAlchemyTable@@UAEXXZ 0048a3d0 f   AlchemyTable.obj
 0001:000893e0       ?LoadState@CAlchemyTable@@UAE?BHPBE@Z 0048a3e0 f   AlchemyTable.obj
 0001:00089410       ?SaveState@CAlchemyTable@@UBE?BHPBEH@Z 0048a410 f   AlchemyTable.obj
 0001:00089440       ?Draw@CAlchemyTable@@UBEXXZ 0048a440 f   AlchemyTable.obj
 0001:00089460       ?Draw@CAlchemyTable@@UBEXH@Z 0048a460 f   AlchemyTable.obj
 0001:00089550       ?Update@CAlchemyTable@@UAEXXZ 0048a550 f   AlchemyTable.obj
 0001:000895f0       ?Complete@CAlchemyTable@@UAEXXZ 0048a5f0 f   AlchemyTable.obj
 0001:00089620       ?StartResetTimer@CAlchemyTable@@QAEXXZ 0048a620 f   AlchemyTable.obj
 0001:00089650       ?Carry@CAlchemyTable@@UAE?B_NAAVCVillager@@W4ECarrying@@@Z 0048a650 f   AlchemyTable.obj
 0001:000896f0       ?Drop@CAlchemyTable@@UAEXAAVCVillager@@W4ECarrying@@@Z 0048a6f0 f   AlchemyTable.obj
 0001:00089790       ?GetNearbyCollectable@CAlchemyTable@@UAE?BW4ECarrying@@AAVCVillager@@UldwPoint@@@Z 0048a790 f   AlchemyTable.obj
 0001:000897a0       ?ContainsEnoughIngredients@CAlchemyTable@@QBE?B_NXZ 0048a7a0 f   AlchemyTable.obj
 0001:000897c0       ?IngredientsRequired@CAlchemyTable@@QBE?BHXZ 0048a7c0 f   AlchemyTable.obj
 0001:000897e0       ?IsAlchemistPresent@CAlchemyTable@@QBE?B_NXZ 0048a7e0 f   AlchemyTable.obj
 0001:00089800       ?Alchemist@CAlchemyTable@@QBEAAVCVillager@@XZ 0048a800 f   AlchemyTable.obj
 0001:00089820       ?SecondsUntilReset@CAlchemyTable@@QBE?BHXZ 0048a820 f   AlchemyTable.obj
 0001:00089850       ??0CAromatherapy@@QAE@XZ   0048a850 f   Aromatherapy.obj
 0001:00089890       ?Reset@CAromatherapy@@UAEXXZ 0048a890 f   Aromatherapy.obj
 0001:000898d0       ?LoadState@CAromatherapy@@UAE?BHPBE@Z 0048a8d0 f   Aromatherapy.obj
 0001:00089920       ?SaveState@CAromatherapy@@UBE?BHPBEH@Z 0048a920 f   Aromatherapy.obj
 0001:00089980       ?Refresh@CAromatherapy@@UAEXXZ 0048a980 f   Aromatherapy.obj
 0001:000899f0       ?Draw@CAromatherapy@@UBEXXZ 0048a9f0 f   Aromatherapy.obj
 0001:00089a10       ?Draw@CAromatherapy@@UBEXH@Z 0048aa10 f   Aromatherapy.obj
 0001:00089a90       ?Advance@CAromatherapy@@UAEXAAVCVillager@@H@Z 0048aa90 f   Aromatherapy.obj
 0001:00089b00       ?Complete@CAromatherapy@@UAEXXZ 0048ab00 f   Aromatherapy.obj
 0001:00089b40       ?Carry@CAromatherapy@@UAE?B_NAAVCVillager@@W4ECarrying@@@Z 0048ab40 f   Aromatherapy.obj
 0001:00089c20       ?Drop@CAromatherapy@@UAEXAAVCVillager@@W4ECarrying@@@Z 0048ac20 f   Aromatherapy.obj
 0001:00089c90       ?GetNearbyCollectable@CAromatherapy@@UAE?BW4ECarrying@@AAVCVillager@@UldwPoint@@@Z 0048ac90 f   Aromatherapy.obj
 0001:00089ca0       ?GetEmptyBurners@CAromatherapy@@QBE?BHPAH@Z 0048aca0 f   Aromatherapy.obj
 0001:00089d00       ?GetUnlitBurners@CAromatherapy@@QBE?BHPAH@Z 0048ad00 f   Aromatherapy.obj
 0001:00089d60       ?BurnerPos@CAromatherapy@@QBE?BUldwPoint@@H@Z 0048ad60 f   Aromatherapy.obj
 0001:00089e50       ?AllBurnersContainHerbs@CAromatherapy@@QBE?B_NXZ 0048ae50 f   Aromatherapy.obj
 0001:00089e90       ??0CBath@@QAE@XZ           0048ae90 f   Bath.obj
 0001:00089ec0       ?Reset@CBath@@UAEXXZ       0048aec0 f   Bath.obj
 0001:00089ee0       ?LoadState@CBath@@UAE?BHPBE@Z 0048aee0 f   Bath.obj
 0001:00089f00       ?SaveState@CBath@@UBE?BHPBEH@Z 0048af00 f   Bath.obj
 0001:00089f30       ?Refresh@CBath@@UAEXXZ     0048af30 f   Bath.obj
 0001:00089f60       ?Advance@CBath@@UAEXAAVCVillager@@H@Z 0048af60 f   Bath.obj
 0001:00089fa0       ?Complete@CBath@@UAEXXZ    0048afa0 f   Bath.obj
 0001:0008a000       ?IsRepaired@CBath@@QBE?B_NXZ 0048b000 f   Bath.obj
 0001:0008a020       ??0CBeeHive@@QAE@XZ        0048b020 f   BeeHive.obj
 0001:0008a0a0       ?Reset@CBeeHive@@UAEXXZ    0048b0a0 f   BeeHive.obj
 0001:0008a0f0       ?LoadAssets@CBeeHive@@UAEXXZ 0048b0f0 f   BeeHive.obj
 0001:0008a110       ?ReleaseAssets@CBeeHive@@UAEXXZ 0048b110 f   BeeHive.obj
 0001:0008a120       ?Complete@CBeeHive@@UAEXXZ 0048b120 f   BeeHive.obj
 0001:0008a170       ?LoadState@CBeeHive@@UAE?BHPBE@Z 0048b170 f   BeeHive.obj
 0001:0008a1e0       ?SaveState@CBeeHive@@UBE?BHPBEH@Z 0048b1e0 f   BeeHive.obj
 0001:0008a240       ?Refresh@CBeeHive@@UAEXXZ  0048b240 f   BeeHive.obj
 0001:0008a330       ?Draw@CBeeHive@@UBEXXZ     0048b330 f   BeeHive.obj
 0001:0008a350       ?Draw@CBeeHive@@UBEXH@Z    0048b350 f   BeeHive.obj
 0001:0008a3b0       ?Update@CBeeHive@@UAEXXZ   0048b3b0 f   BeeHive.obj
 0001:0008a460       ?Carry@CBeeHive@@UAE?B_NAAVCVillager@@W4ECarrying@@@Z 0048b460 f   BeeHive.obj
 0001:0008a620       ?Drop@CBeeHive@@UAEXAAVCVillager@@W4ECarrying@@@Z 0048b620 f   BeeHive.obj
 0001:0008a8b0       ?LightStick@CBeeHive@@QAEXXZ 0048b8b0 f   BeeHive.obj
 0001:0008a990       ?ExtinguishStick@CBeeHive@@QAEXXZ 0048b990 f   BeeHive.obj
 0001:0008a9e0       ?SwarmVillager@CBeeHive@@QAEXAAVCVillager@@@Z 0048b9e0 f   BeeHive.obj
 0001:0008aa80       ?GetNearbyCollectable@CBeeHive@@UAE?BW4ECarrying@@AAVCVillager@@UldwPoint@@@Z 0048ba80 f   BeeHive.obj
 0001:0008aa90       ?IsSmokingStickPresent@CBeeHive@@QBE?B_NXZ 0048ba90 f   BeeHive.obj
 0001:0008aab0       ?IsSwarming@CBeeHive@@QBE?B_NXZ 0048bab0 f   BeeHive.obj
 0001:0008aad0       ?HasHoneyToHarvest@CBeeHive@@QBE?B_NXZ 0048bad0 f   BeeHive.obj
 0001:0008aaf0       ?GetHoneyAvailable@CBeeHive@@QAE?BHXZ 0048baf0 f   BeeHive.obj
 0001:0008ab10       ?SetHoneyAvailable@CBeeHive@@QAEXH@Z 0048bb10 f   BeeHive.obj
 0001:0008ab40       ??0CChalkBoard@@QAE@XZ     0048bb40 f   ChalkBoard.obj
 0001:0008ab70       ?Reset@CChalkBoard@@UAEXXZ 0048bb70 f   ChalkBoard.obj
 0001:0008aba0       ?LoadState@CChalkBoard@@UAE?BHPBE@Z 0048bba0 f   ChalkBoard.obj
 0001:0008abe0       ?SaveState@CChalkBoard@@UBE?BHPBEH@Z 0048bbe0 f   ChalkBoard.obj
 0001:0008ac20       ?Draw@CChalkBoard@@UBEXXZ  0048bc20 f   ChalkBoard.obj
 0001:0008ac70       ?Draw@CChalkBoard@@UBEXH@Z 0048bc70 f   ChalkBoard.obj
 0001:0008ad00       ?Update@CChalkBoard@@UAEXXZ 0048bd00 f   ChalkBoard.obj
 0001:0008ad60       ?Advance@CChalkBoard@@UAEXAAVCVillager@@H@Z 0048bd60 f   ChalkBoard.obj
 0001:0008ad90       ?ContainsPlans@CChalkBoard@@QBE?B_NXZ 0048bd90 f   ChalkBoard.obj
 0001:0008adc0       ?ContainsBathPlans@CChalkBoard@@QBE?B_NXZ 0048bdc0 f   ChalkBoard.obj
 0001:0008ade0       ?ContainsStatuePlans@CChalkBoard@@QBE?B_NXZ 0048bde0 f   ChalkBoard.obj
 0001:0008ae00       ??0CChief@@QAE@XZ          0048be00 f   Chief.obj
 0001:0008ae30       ?Reset@CChief@@UAEXXZ      0048be30 f   Chief.obj
 0001:0008ae40       ?LoadAssets@CChief@@UAEXXZ 0048be40 f   Chief.obj
 0001:0008ae50       ?ReleaseAssets@CChief@@UAEXXZ 0048be50 f   Chief.obj
 0001:0008ae60       ?LoadState@CChief@@UAE?BHPBE@Z 0048be60 f   Chief.obj
 0001:0008ae80       ?SaveState@CChief@@UBE?BHPBEH@Z 0048be80 f   Chief.obj
 0001:0008aeb0       ?Refresh@CChief@@UAEXXZ    0048beb0 f   Chief.obj
 0001:0008aec0       ?Draw@CChief@@UBEXXZ       0048bec0 f   Chief.obj
 0001:0008aed0       ?Complete@CChief@@UAEXXZ   0048bed0 f   Chief.obj
 0001:0008af10       ?Advance@CChief@@UAEXAAVCVillager@@H@Z 0048bf10 f   Chief.obj
 0001:0008af90       ??0CConstruction@@QAE@XZ   0048bf90 f   Construction.obj
 0001:0008afe0       ?Reset@CConstruction@@UAEXXZ 0048bfe0 f   Construction.obj
 0001:0008b080       ?LoadAssets@CConstruction@@UAEXXZ 0048c080 f   Construction.obj
 0001:0008b0e0       ?ReleaseAssets@CConstruction@@UAEXXZ 0048c0e0 f   Construction.obj
 0001:0008b0f0       ?LoadState@CConstruction@@UAE?BHPBE@Z 0048c0f0 f   Construction.obj
 0001:0008b1b0       ?SaveState@CConstruction@@UBE?BHPBEH@Z 0048c1b0 f   Construction.obj
 0001:0008b220       ?Refresh@CConstruction@@UAEXXZ 0048c220 f   Construction.obj
 0001:0008b290       ?Draw@CConstruction@@UBEXXZ 0048c290 f   Construction.obj
 0001:0008b440       ?Draw@CConstruction@@UBEXH@Z 0048c440 f   Construction.obj
 0001:0008b530       ?Update@CConstruction@@UAEXXZ 0048c530 f   Construction.obj
 0001:0008b740       ?Advance@CConstruction@@UAEXAAVCVillager@@H@Z 0048c740 f   Construction.obj
 0001:0008baa0       ?SiteObject@CConstruction@@QBE?BW4EObject@CContentMap@@W4EConstruction@@@Z 0048caa0 f   Construction.obj
 0001:0008bac0       ?Object@CConstruction@@QBE?BW4EObject@CContentMap@@W4EConstruction@@@Z 0048cac0 f   Construction.obj
 0001:0008bae0       ?GetPuzzle@CConstruction@@QBE?BW4EPuzzle@@W4EConstruction@@@Z 0048cae0 f   Construction.obj
 0001:0008bb00       ?IsComplete@CConstruction@@QBE?B_NW4EConstruction@@@Z 0048cb00 f   Construction.obj
 0001:0008bb30       ?PercentComplete@CConstruction@@QBE?BHW4EConstruction@@@Z 0048cb30 f   Construction.obj
 0001:0008bbb0       ?StateOfDisrepair@CConstruction@@QBE?BW4EDisrepair@@W4EConstruction@@@Z 0048cbb0 f   Construction.obj
 0001:0008bc20       ?SetDisrepair@CConstruction@@QAEXW4EConstruction@@W4EDisrepair@@@Z 0048cc20 f   Construction.obj
 0001:0008bc60       ?IsBool@@YA?B_N_N@Z        0048cc60 f i Construction.obj
 0001:0008bc90       ??0CDoorKey@@QAE@XZ        0048cc90 f   DoorKey.obj
 0001:0008bd40       ?Reset@CDoorKey@@UAEXXZ    0048cd40 f   DoorKey.obj
 0001:0008be00       ?LoadAssets@CDoorKey@@UAEXXZ 0048ce00 f   DoorKey.obj
 0001:0008bed0       ?ReleaseAssets@CDoorKey@@UAEXXZ 0048ced0 f   DoorKey.obj
 0001:0008bf60       ?LoadState@CDoorKey@@UAE?BHPBE@Z 0048cf60 f   DoorKey.obj
 0001:0008bfd0       ?SaveState@CDoorKey@@UBE?BHPBEH@Z 0048cfd0 f   DoorKey.obj
 0001:0008c040       ?Refresh@CDoorKey@@UAEXXZ  0048d040 f   DoorKey.obj
 0001:0008c120       ?Draw@CDoorKey@@UBEXXZ     0048d120 f   DoorKey.obj
 0001:0008c1b0       ?Draw@CDoorKey@@UBEXH@Z    0048d1b0 f   DoorKey.obj
 0001:0008c490       ?Update@CDoorKey@@UAEXXZ   0048d490 f   DoorKey.obj
 0001:0008c560       ?Complete@CDoorKey@@UAEXXZ 0048d560 f   DoorKey.obj
 0001:0008c580       ?Carry@CDoorKey@@UAE?B_NAAVCVillager@@W4ECarrying@@@Z 0048d580 f   DoorKey.obj
 0001:0008c7e0       ?Drop@CDoorKey@@UAEXAAVCVillager@@W4ECarrying@@@Z 0048d7e0 f   DoorKey.obj
 0001:0008c950       ?TechAdvanced@CDoorKey@@UAEXW4ETech@@H@Z 0048d950 f   DoorKey.obj
 0001:0008c960       ?GetNearbyCollectable@CDoorKey@@UAE?BW4ECarrying@@AAVCVillager@@UldwPoint@@@Z 0048d960 f   DoorKey.obj
 0001:0008ca90       ?KeysCollected@CDoorKey@@QBE?BHXZ 0048da90 f   DoorKey.obj
 0001:0008caf0       ?IsNearClam@CDoorKey@@QBE?B_NUldwPoint@@@Z 0048daf0 f   DoorKey.obj
 0001:0008cb50       ?IsNearPearl@CDoorKey@@QBE?B_NUldwPoint@@@Z 0048db50 f   DoorKey.obj
 0001:0008cbc0       ?IsNearRoughPearl@CDoorKey@@ABE?B_NUldwPoint@@@Z 0048dbc0 f   DoorKey.obj
 0001:0008cc30       ?IsNearBrokenPearl@CDoorKey@@ABE?B_NUldwPoint@@@Z 0048dc30 f   DoorKey.obj
 0001:0008cca0       ?HotDiamondInFirePit@CDoorKey@@QBE?B_NXZ 0048dca0 f   DoorKey.obj
 0001:0008cd30       ??0CFirePit@@QAE@XZ        0048dd30 f   FirePit.obj
 0001:0008cd90       ?Reset@CFirePit@@UAEXXZ    0048dd90 f   FirePit.obj
 0001:0008cdb0       ?ResetFire@CFirePit@@QAEXXZ 0048ddb0 f   FirePit.obj
 0001:0008ce00       ?LoadAssets@CFirePit@@UAEXXZ 0048de00 f   FirePit.obj
 0001:0008ce40       ?ReleaseAssets@CFirePit@@UAEXXZ 0048de40 f   FirePit.obj
 0001:0008ce50       ?LoadState@CFirePit@@UAE?BHPBE@Z 0048de50 f   FirePit.obj
 0001:0008cef0       ?SaveState@CFirePit@@UBE?BHPBEH@Z 0048def0 f   FirePit.obj
 0001:0008cf70       ?Refresh@CFirePit@@UAEXXZ  0048df70 f   FirePit.obj
 0001:0008d020       ?Draw@CFirePit@@UBEXXZ     0048e020 f   FirePit.obj
 0001:0008d050       ?Draw@CFirePit@@UBEXH@Z    0048e050 f   FirePit.obj
 0001:0008d100       ?Update@CFirePit@@UAEXXZ   0048e100 f   FirePit.obj
 0001:0008d200       ?Advance@CFirePit@@UAEXAAVCVillager@@H@Z 0048e200 f   FirePit.obj
 0001:0008d240       ?Complete@CFirePit@@UAEXXZ 0048e240 f   FirePit.obj
 0001:0008d2a0       ?Carry@CFirePit@@UAE?B_NAAVCVillager@@W4ECarrying@@@Z 0048e2a0 f   FirePit.obj
 0001:0008d2b0       ?Drop@CFirePit@@UAEXAAVCVillager@@W4ECarrying@@@Z 0048e2b0 f   FirePit.obj
 0001:0008d640       ?LightFire@CFirePit@@QAEXXZ 0048e640 f   FirePit.obj
 0001:0008d7b0       ?ExtinguishFire@CFirePit@@QAEXXZ 0048e7b0 f   FirePit.obj
 0001:0008d810       ?Poof@CFirePit@@QAEXXZ     0048e810 f   FirePit.obj
 0001:0008d850       ?GetNearbyCollectable@CFirePit@@UAE?BW4ECarrying@@AAVCVillager@@UldwPoint@@@Z 0048e850 f   FirePit.obj
 0001:0008d860       ?IsLit@CFirePit@@QBE?B_NXZ 0048e860 f   FirePit.obj
 0001:0008d880       ?SecondsRemainingOnFire@CFirePit@@QBE?BHXZ 0048e880 f   FirePit.obj
 0001:0008d8a0       ?TotalBurnTime@CFirePit@@QBE?BHXZ 0048e8a0 f   FirePit.obj
 0001:0008d8c0       ?IsCooling@CFirePit@@QBE?B_NXZ 0048e8c0 f   FirePit.obj
 0001:0008d900       ?HasCooled@CFirePit@@QBE?B_NXZ 0048e900 f   FirePit.obj
 0001:0008d920       ??0COrchard@@QAE@XZ        0048e920 f   Orchard.obj
 0001:0008d9c0       ?Reset@COrchard@@UAEXXZ    0048e9c0 f   Orchard.obj
 0001:0008da60       ?LoadAssets@COrchard@@UAEXXZ 0048ea60 f   Orchard.obj
 0001:0008db10       ?ReleaseAssets@COrchard@@UAEXXZ 0048eb10 f   Orchard.obj
 0001:0008db20       ?LoadState@COrchard@@UAE?BHPBE@Z 0048eb20 f   Orchard.obj
 0001:0008dc00       ?SaveState@COrchard@@UBE?BHPBEH@Z 0048ec00 f   Orchard.obj
 0001:0008dcc0       ?Refresh@COrchard@@UAEXXZ  0048ecc0 f   Orchard.obj
 0001:0008dd30       ?Draw@COrchard@@UBEXXZ     0048ed30 f   Orchard.obj
 0001:0008de00       ?Draw@COrchard@@UBEXH@Z    0048ee00 f   Orchard.obj
 0001:0008e520       ?Update@COrchard@@UAEXXZ   0048f520 f   Orchard.obj
 0001:0008e790       ?Advance@COrchard@@UAEXAAVCVillager@@H@Z 0048f790 f   Orchard.obj
 0001:0008e9e0       ?Complete@COrchard@@UAEXXZ 0048f9e0 f   Orchard.obj
 0001:0008ea00       ?DropFruit@COrchard@@QAEXUldwPoint@@H@Z 0048fa00 f   Orchard.obj
 0001:0008ea50       ?Carry@COrchard@@UAE?B_NAAVCVillager@@W4ECarrying@@@Z 0048fa50 f   Orchard.obj
 0001:0008ec50       ?Drop@COrchard@@UAEXAAVCVillager@@W4ECarrying@@@Z 0048fc50 f   Orchard.obj
 0001:0008eca0       ?DealWithFruitEmergency@COrchard@@QAEXAAVCVillager@@W4ECarrying@@@Z 0048fca0 f   Orchard.obj
 0001:0008ee00       ?GetNearbyCollectable@COrchard@@UAE?BW4ECarrying@@AAVCVillager@@UldwPoint@@@Z 0048fe00 f   Orchard.obj
 0001:0008eec0       ?TreeObject@COrchard@@QBE?BW4EObject@CContentMap@@H@Z 0048fec0 f   Orchard.obj
 0001:0008eee0       ?IsTreeMature@COrchard@@QBE?B_NH@Z 0048fee0 f   Orchard.obj
 0001:0008ef20       ?SecondsUntilMature@COrchard@@QBE?BHH@Z 0048ff20 f   Orchard.obj
 0001:0008ef60       ?TreeExists@COrchard@@QBE?B_NH@Z 0048ff60 f   Orchard.obj
 0001:0008ef80       ?FruitOnTree@COrchard@@QBE?BHH@Z 0048ff80 f   Orchard.obj
 0001:0008efa0       ?ResetFruitOnTree@COrchard@@QAEXH@Z 0048ffa0 f   Orchard.obj
 0001:0008efc0       ?AdjustFruitOnTree@COrchard@@QAEXHH@Z 0048ffc0 f   Orchard.obj
 0001:0008f030       ?GetFruitOnTree@COrchard@@QAE?BHH@Z 00490030 f   Orchard.obj
 0001:0008f050       ?EnoughFruitToHarvest@COrchard@@QAE?B_NH@Z 00490050 f   Orchard.obj
 0001:0008f070       ?GetTreePos@COrchard@@QBE?BUldwPoint@@H@Z 00490070 f   Orchard.obj
 0001:0008f0a0       ?NearestTree@COrchard@@QBE?BHUldwPoint@@@Z 004900a0 f   Orchard.obj
 0001:0008f140       ??0SPlantTreeData@@QAE@UldwPoint@@@Z 00490140 f i Orchard.obj
 0001:0008f170       ??0CPrincessStatue@@QAE@XZ 00490170 f   PrincessStatue.obj
 0001:0008f1c0       ?Reset@CPrincessStatue@@UAEXXZ 004901c0 f   PrincessStatue.obj
 0001:0008f210       ?LoadAssets@CPrincessStatue@@UAEXXZ 00490210 f   PrincessStatue.obj
 0001:0008f270       ?ReleaseAssets@CPrincessStatue@@UAEXXZ 00490270 f   PrincessStatue.obj
 0001:0008f280       ?LoadState@CPrincessStatue@@UAE?BHPBE@Z 00490280 f   PrincessStatue.obj
 0001:0008f310       ?SaveState@CPrincessStatue@@UBE?BHPBEH@Z 00490310 f   PrincessStatue.obj
 0001:0008f370       ?Refresh@CPrincessStatue@@UAEXXZ 00490370 f   PrincessStatue.obj
 0001:0008f380       ?Draw@CPrincessStatue@@UBEXXZ 00490380 f   PrincessStatue.obj
 0001:0008f400       ?Draw@CPrincessStatue@@UBEXH@Z 00490400 f   PrincessStatue.obj
 0001:0008f4c0       ?Update@CPrincessStatue@@UAEXXZ 004904c0 f   PrincessStatue.obj
 0001:0008f670       ?Advance@CPrincessStatue@@UAEXAAVCVillager@@H@Z 00490670 f   PrincessStatue.obj
 0001:0008f7c0       ?Complete@CPrincessStatue@@UAEXXZ 004907c0 f   PrincessStatue.obj
 0001:0008f890       ?AddPusher@CPrincessStatue@@QAE?BUldwPoint@@HH@Z 00490890 f   PrincessStatue.obj
 0001:0008fa40       ?IsNearToStatue@CPrincessStatue@@QBE?B_NUldwPoint@@@Z 00490a40 f   PrincessStatue.obj
 0001:0008faa0       ?IsRoomForAnotherPusher@CPrincessStatue@@QBE?B_NXZ 00490aa0 f   PrincessStatue.obj
 0001:0008fac0       ?IsStatueInTransportingPhase@CPrincessStatue@@QBE?B_NXZ 00490ac0 f   PrincessStatue.obj
 0001:0008fae0       ?IsPusherAtOffset@CPrincessStatue@@QBE?B_NH@Z 00490ae0 f   PrincessStatue.obj
 0001:0008fb30       ?EstimatedRepairTime@CPrincessStatue@@QBE?BHXZ 00490b30 f   PrincessStatue.obj
 0001:0008fb70       ??0CPuzzle@@QAE@XZ         00490b70 f   Puzzle.obj
 0001:0008fc20       ?Reset@CPuzzle@@QAEXXZ     00490c20 f   Puzzle.obj
 0001:0008fc80       ?Reset@CPuzzle@@QAEXW4EPuzzle@@@Z 00490c80 f   Puzzle.obj
 0001:0008fcc0       ?LoadAssets@CPuzzle@@QAEXXZ 00490cc0 f   Puzzle.obj
 0001:0008fd10       ?ReleaseAssets@CPuzzle@@QAEXXZ 00490d10 f   Puzzle.obj
 0001:0008fd60       ?GetPuzzleStateSize@CPuzzle@@QBE?BHXZ 00490d60 f   Puzzle.obj
 0001:0008fd80       ?LoadState@CPuzzle@@QAE?B_NPBE@Z 00490d80 f   Puzzle.obj
 0001:0008fe50       ?SaveState@CPuzzle@@QBE?B_NPBEH@Z 00490e50 f   Puzzle.obj
 0001:0008ff20       ?Refresh@CPuzzle@@QBEXXZ   00490f20 f   Puzzle.obj
 0001:0008ff70       ?Draw@CPuzzle@@QBEXXZ      00490f70 f   Puzzle.obj
 0001:0008ffc0       ?Draw@CPuzzle@@QBEXH@Z     00490fc0 f   Puzzle.obj
 0001:00090000       ?Update@CPuzzle@@QAEXXZ    00491000 f   Puzzle.obj
 0001:00090050       ?Advance@CPuzzle@@QAEXW4EPuzzle@@AAVCVillager@@H@Z 00491050 f   Puzzle.obj
 0001:00090080       ?IncrementProgress@CPuzzle@@QAEXW4EPuzzle@@@Z 00491080 f   Puzzle.obj
 0001:00090100       ?DecrementProgress@CPuzzle@@QAEXW4EPuzzle@@@Z 00491100 f   Puzzle.obj
 0001:00090130       ?IsComplete@CPuzzle@@QBE?B_NW4EPuzzle@@@Z 00491130 f   Puzzle.obj
 0001:00090160       ?PercentComplete@CPuzzle@@QBE?BHW4EPuzzle@@@Z 00491160 f   Puzzle.obj
 0001:000901b0       ?PuzzlesComplete@CPuzzle@@QBE?BHXZ 004911b0 f   Puzzle.obj
 0001:00090200       ?EssentialPuzzlesComplete@CPuzzle@@QBE?BHXZ 00491200 f   Puzzle.obj
 0001:00090250       ?CompletionTime@CPuzzle@@QBE?BHW4EPuzzle@@@Z 00491250 f   Puzzle.obj
 0001:00090270       ?PointsRemaining@CPuzzle@@QBE?BHW4EPuzzle@@@Z 00491270 f   Puzzle.obj
 0001:00090290       ?SetPointsRemaining@CPuzzle@@QAEXW4EPuzzle@@H@Z 00491290 f   Puzzle.obj
 0001:000902c0       ??0CRainLift@@QAE@XZ       004912c0 f   RainLift.obj
 0001:00090300       ?Reset@CRainLift@@UAEXXZ   00491300 f   RainLift.obj
 0001:00090330       ?LoadAssets@CRainLift@@UAEXXZ 00491330 f   RainLift.obj
 0001:00090370       ?ReleaseAssets@CRainLift@@UAEXXZ 00491370 f   RainLift.obj
 0001:00090380       ?LoadState@CRainLift@@UAE?BHPBE@Z 00491380 f   RainLift.obj
 0001:00090400       ?SaveState@CRainLift@@UBE?BHPBEH@Z 00491400 f   RainLift.obj
 0001:00090450       ?Refresh@CRainLift@@UAEXXZ 00491450 f   RainLift.obj
 0001:00090490       ?Draw@CRainLift@@UBEXXZ    00491490 f   RainLift.obj
 0001:000904e0       ?Draw@CRainLift@@UBEXH@Z   004914e0 f   RainLift.obj
 0001:00090560       ?Update@CRainLift@@UAEXXZ  00491560 f   RainLift.obj
 0001:000907f0       ?Advance@CRainLift@@UAEXAAVCVillager@@H@Z 004917f0 f   RainLift.obj
 0001:00090850       ?Complete@CRainLift@@UAEXXZ 00491850 f   RainLift.obj
 0001:000908a0       ?IsRepaired@CRainLift@@QBE?B_NXZ 004918a0 f   RainLift.obj
 0001:000908c0       ?SetScenePriority@CVillager@@QAEXW4EScenePriority@@@Z 004918c0 f i RainLift.obj
 0001:000908e0       ??0CRosterOfTheDead@@QAE@XZ 004918e0 f   RosterOfTheDead.obj
 0001:00090930       ?Reset@CRosterOfTheDead@@UAEXXZ 00491930 f   RosterOfTheDead.obj
 0001:00090940       ?LoadAssets@CRosterOfTheDead@@UAEXXZ 00491940 f   RosterOfTheDead.obj
 0001:00090980       ?ReleaseAssets@CRosterOfTheDead@@UAEXXZ 00491980 f   RosterOfTheDead.obj
 0001:00090990       ?LoadState@CRosterOfTheDead@@UAE?BHPBE@Z 00491990 f   RosterOfTheDead.obj
 0001:000909b0       ?SaveState@CRosterOfTheDead@@UBE?BHPBEH@Z 004919b0 f   RosterOfTheDead.obj
 0001:000909e0       ?Draw@CRosterOfTheDead@@UBEXXZ 004919e0 f   RosterOfTheDead.obj
 0001:00090a10       ?Draw@CRosterOfTheDead@@UBEXH@Z 00491a10 f   RosterOfTheDead.obj
 0001:00090bb0       ?Carry@CRosterOfTheDead@@UAE?B_NAAVCVillager@@W4ECarrying@@@Z 00491bb0 f   RosterOfTheDead.obj
 0001:00090bc0       ?Drop@CRosterOfTheDead@@UAEXAAVCVillager@@W4ECarrying@@@Z 00491bc0 f   RosterOfTheDead.obj
 0001:00090c20       ?GetNearbyCollectable@CRosterOfTheDead@@UAE?BW4ECarrying@@AAVCVillager@@UldwPoint@@@Z 00491c20 f   RosterOfTheDead.obj
 0001:00090c30       ?IsUncovered@CRosterOfTheDead@@QBE?B_NXZ 00491c30 f   RosterOfTheDead.obj
 0001:00090c50       ?Complete@CRosterOfTheDead@@UAEXXZ 00491c50 f   RosterOfTheDead.obj
 0001:00090c70       ??0CRuins@@QAE@XZ          00491c70 f   Ruins.obj
 0001:00090cc0       ?Reset@CRuins@@UAEXXZ      00491cc0 f   Ruins.obj
 0001:00090cd0       ?LoadAssets@CRuins@@UAEXXZ 00491cd0 f   Ruins.obj
 0001:00090d60       ?ReleaseAssets@CRuins@@UAEXXZ 00491d60 f   Ruins.obj
 0001:00090db0       ?LoadState@CRuins@@UAE?BHPBE@Z 00491db0 f   Ruins.obj
 0001:00090dd0       ?SaveState@CRuins@@UBE?BHPBEH@Z 00491dd0 f   Ruins.obj
 0001:00090e00       ?Refresh@CRuins@@UAEXXZ    00491e00 f   Ruins.obj
 0001:00090e10       ?Draw@CRuins@@UBEXXZ       00491e10 f   Ruins.obj
 0001:00090ea0       ?Draw@CRuins@@UBEXH@Z      00491ea0 f   Ruins.obj
 0001:000910d0       ?Carry@CRuins@@UAE?B_NAAVCVillager@@W4ECarrying@@@Z 004920d0 f   Ruins.obj
 0001:000910e0       ?Drop@CRuins@@UAEXAAVCVillager@@W4ECarrying@@@Z 004920e0 f   Ruins.obj
 0001:00091140       ?GetNearbyCollectable@CRuins@@UAE?BW4ECarrying@@AAVCVillager@@UldwPoint@@@Z 00492140 f   Ruins.obj
 0001:00091150       ?AreUncovered@CRuins@@QBE?B_NXZ 00492150 f   Ruins.obj
 0001:00091170       ?Complete@CRuins@@UAEXXZ   00492170 f   Ruins.obj
 0001:000911b0       ??0CSharkCharmer@@QAE@XZ   004921b0 f   SharkCharmer.obj
 0001:000911f0       ?Reset@CSharkCharmer@@UAEXXZ 004921f0 f   SharkCharmer.obj
 0001:00091210       ?LoadState@CSharkCharmer@@UAE?BHPBE@Z 00492210 f   SharkCharmer.obj
 0001:00091250       ?SaveState@CSharkCharmer@@UBE?BHPBEH@Z 00492250 f   SharkCharmer.obj
 0001:00091280       ?Carry@CSharkCharmer@@UAE?B_NAAVCVillager@@W4ECarrying@@@Z 00492280 f   SharkCharmer.obj
 0001:00091290       ?Drop@CSharkCharmer@@UAEXAAVCVillager@@W4ECarrying@@@Z 00492290 f   SharkCharmer.obj
 0001:00091410       ?GetNearbyCollectable@CSharkCharmer@@UAE?BW4ECarrying@@AAVCVillager@@UldwPoint@@@Z 00492410 f   SharkCharmer.obj
 0001:00091420       ?HasBanishedSharksForever@CSharkCharmer@@QBE?B_NXZ 00492420 f   SharkCharmer.obj
 0001:00091440       ?Complete@CSharkCharmer@@UAEXXZ 00492440 f   SharkCharmer.obj
 0001:00091460       ??0CSunDisk@@QAE@XZ        00492460 f   SunDisk.obj
 0001:000914a0       ?Reset@CSunDisk@@UAEXXZ    004924a0 f   SunDisk.obj
 0001:00091500       ?LoadAssets@CSunDisk@@UAEXXZ 00492500 f   SunDisk.obj
 0001:00091550       ?ReleaseAssets@CSunDisk@@UAEXXZ 00492550 f   SunDisk.obj
 0001:00091560       ?LoadState@CSunDisk@@UAE?BHPBE@Z 00492560 f   SunDisk.obj
 0001:000915b0       ?SaveState@CSunDisk@@UBE?BHPBEH@Z 004925b0 f   SunDisk.obj
 0001:00091600       ?Draw@CSunDisk@@UBEXXZ     00492600 f   SunDisk.obj
 0001:00091680       ?Draw@CSunDisk@@UBEXH@Z    00492680 f   SunDisk.obj
 0001:00091810       ?Update@CSunDisk@@UAEXXZ   00492810 f   SunDisk.obj
 0001:00091a00       ?Rotate@CSunDisk@@QAEXXZ   00492a00 f   SunDisk.obj
 0001:00091a70       ?ShowGhosts@CSunDisk@@QAEXXZ 00492a70 f   SunDisk.obj
 0001:00091a90       ?AreGhostsVisible@CSunDisk@@QBE?B_NXZ 00492a90 f   SunDisk.obj
 0001:00091ab0       ?Complete@CSunDisk@@UAEXXZ 00492ab0 f   SunDisk.obj
 0001:00091af0       ??0CWeatherDance@@QAE@XZ   00492af0 f   WeatherDance.obj
 0001:00091b30       ?Reset@CWeatherDance@@UAEXXZ 00492b30 f   WeatherDance.obj
 0001:00091b70       ?LoadState@CWeatherDance@@UAE?BHPBE@Z 00492b70 f   WeatherDance.obj
 0001:00091b90       ?SaveState@CWeatherDance@@UBE?BHPBEH@Z 00492b90 f   WeatherDance.obj
 0001:00091bc0       ?Update@CWeatherDance@@UAEXXZ 00492bc0 f   WeatherDance.obj
 0001:00091d30       ?Advance@CWeatherDance@@UAEXAAVCVillager@@H@Z 00492d30 f   WeatherDance.obj
 0001:00091dd0       ?AddSparkles@CWeatherDance@@QBEXH@Z 00492dd0 f   WeatherDance.obj
 0001:00091e40       ?IsChiefDancing@CWeatherDance@@QBE?B_NXZ 00492e40 f   WeatherDance.obj
 0001:00091e90       ?Complete@CWeatherDance@@UAEXXZ 00492e90 f   WeatherDance.obj
 0001:00091ed0       ??0CMoviePlayer@@QAE@XZ    00492ed0 f   MoviePlayer.obj
 0001:00091f50       ??1CMoviePlayer@@QAE@XZ    00492f50 f   MoviePlayer.obj
 0001:00091fa0       ?Play@CMoviePlayer@@QAE?B_NPBDHH@Z 00492fa0 f   MoviePlayer.obj
 0001:00092010       ?Draw@CMoviePlayer@@QBEXUldwPoint@@@Z 00493010 f   MoviePlayer.obj
 0001:00092070       ?Pause@CMoviePlayer@@QBEXXZ 00493070 f   MoviePlayer.obj
 0001:00092090       ?Stop@CMoviePlayer@@QAEXXZ 00493090 f   MoviePlayer.obj
 0001:000920c0       ?IsPlaying@CMoviePlayer@@QBE?B_NXZ 004930c0 f   MoviePlayer.obj
 0001:000920e0       ?_AtlGetThreadACPThunk@ATL@@YGIXZ 004930e0 f i FlashPlayer.obj
 0001:00092150       ?InterlockedExchangePointer@@YGPAXPAPAXPAX@Z 00493150 f i FlashPlayer.obj
 0001:00092170       ?_AtlGetThreadACPFake@ATL@@YGIXZ 00493170 f i FlashPlayer.obj
 0001:000921f0       ?_AtlGetThreadACPReal@ATL@@YGIXZ 004931f0 f i FlashPlayer.obj
 0001:00092200       ??_Estringdispid@CComTypeInfoHolder@ATL@@QAEPAXI@Z 00493200 f i FlashPlayer.obj
 0001:00092270       ??1stringdispid@CComTypeInfoHolder@ATL@@QAE@XZ 00493270 f i FlashPlayer.obj
 0001:00092290       ??1CComBSTR@ATL@@QAE@XZ    00493290 f i FlashPlayer.obj
 0001:000922b0       ??0CFlashPlayer@@QAE@XZ    004932b0 f   FlashPlayer.obj
 0001:00092300       ??1CFlashPlayer@@UAE@XZ    00493300 f   FlashPlayer.obj
 0001:00092360       ?Shutdown@CFlashPlayer@@UAEXXZ 00493360 f   FlashPlayer.obj
 0001:00092400       ?Load@CFlashPlayer@@UAE?B_NPBDHH@Z 00493400 f   FlashPlayer.obj
 0001:00092ea0       ?GetFrameBuffer@CFlashPlayer@@UAE?B_NPAPAE@Z 00493ea0 f   FlashPlayer.obj
 0001:00092f40       ?Play@CFlashPlayer@@UBEXXZ 00493f40 f   FlashPlayer.obj
 0001:00092f70       ?Pause@CFlashPlayer@@UBEXXZ 00493f70 f   FlashPlayer.obj
 0001:00092fa0       ?Stop@CFlashPlayer@@UBEXXZ 00493fa0 f   FlashPlayer.obj
 0001:00093020       ?GotoFrame@CFlashPlayer@@UBEXH@Z 00494020 f   FlashPlayer.obj
 0001:00093050       ?IsPlaying@CFlashPlayer@@UBE?B_NXZ 00494050 f   FlashPlayer.obj
 0001:00093360       ??_GCFlashPlayer@@UAEPAXI@Z 00494360 f i FlashPlayer.obj
 0001:00093360       ??_ECFlashPlayer@@UAEPAXI@Z 00494360 f i FlashPlayer.obj
 0001:00093390       ??0IFlashPlayer@@QAE@XZ    00494390 f i FlashPlayer.obj
 0001:000933b0       ??_GIFlashPlayer@@UAEPAXI@Z 004943b0 f i FlashPlayer.obj
 0001:000933b0       ??_EIFlashPlayer@@UAEPAXI@Z 004943b0 f i FlashPlayer.obj
 0001:000933e0       ??1IFlashPlayer@@UAE@XZ    004943e0 f i FlashPlayer.obj
 0001:00093400       _AtlAxAttachControl@12     00494400 f i FlashPlayer.obj
 0001:000934e0       _AtlAxWinInit@0            004944e0 f i FlashPlayer.obj
 0001:000936b0       ?SetWindowLongPtrA@@YAJPAUHWND__@@HJ@Z 004946b0 f i FlashPlayer.obj
 0001:000936d0       ?GetWindowLongPtrA@@YAJPAUHWND__@@H@Z 004946d0 f i FlashPlayer.obj
 0001:000936f0       ?_AtlGetConversionACP@ATL@@YGIXZ 004946f0 f i FlashPlayer.obj
 0001:00093700       ?AtlA2WHelper@@YGPAGPAGPBDHI@Z 00494700 f i FlashPlayer.obj
 0001:00093750       ?ParseInitData@_DialogSplitHelper@ATL@@SAJPAUIStream@@PAPAG@Z 00494750 f i FlashPlayer.obj
 0001:000939a0       ??0CComBSTR@ATL@@QAE@H@Z   004949a0 f i FlashPlayer.obj
 0001:000939f0       ?AtlThrow@ATL@@YGXJ@Z      004949f0 f i FlashPlayer.obj
 0001:00093a20       ?Length@CComBSTR@ATL@@QBEIXZ 00494a20 f i FlashPlayer.obj
 0001:00093a50       _AtlAxCreateControlLic@20  00494a50 f i FlashPlayer.obj
 0001:00093a80       _AtlAxCreateControlLicEx@32 00494a80 f i FlashPlayer.obj
 0001:00093bc0       ??0CComBSTR@ATL@@QAE@PBG@Z 00494bc0 f i FlashPlayer.obj
 0001:00093c10       ?GetWndClassName@?$CAxWindowT@VCWindow@ATL@@@ATL@@SAPBDXZ 00494c10 f i FlashPlayer.obj
 0001:00093c20       ?GetWndClassName@?$CAxWindow2T@VCWindow@ATL@@@ATL@@SAPBDXZ 00494c20 f i FlashPlayer.obj
 0001:00093c30       ?CreateInstance@?$CComCreator@V?$CComPolyObject@VCAxHostWindow@ATL@@@ATL@@@ATL@@SGJPAXABU_GUID@@PAPAX@Z 00494c30 f i FlashPlayer.obj
 0001:00093d90       ?KeyChar@CGapiApplication@@MAEXH@Z 00494d90 f i ldwGapiApplication.obj
 0001:00093d90       ?ImpactGame@CIslandEvent@@UAEXH@Z 00494d90 f i IslandEvents.obj
 0001:00093d90       ?CalcAward@CIslandEvent@@UAEXH@Z 00494d90 f i IslandEvents.obj
 0001:00093d90       ?SetVoid@CComObjectRootBase@ATL@@QAEXPAX@Z 00494d90 f i FlashPlayer.obj
 0001:00093d90       ?OnFinalMessage@?$CWindowImplBaseT@VCWindow@ATL@@V?$CWinTraits@$0FGAAAAAA@$0A@@2@@ATL@@UAEXPAUHWND__@@@Z 00494d90 f i FlashPlayer.obj
 0001:00093d90       ?Activate@ldwScene@@MAEX_N@Z 00494d90 f i ldwDialog.obj
 0001:00093d90       ?Attach@IVillagerAttachment@@UAEXH@Z 00494d90 f i EnvironmentalSound.obj
 0001:00093d90       ?Draw@IPuzzle@@UBEXH@Z     00494d90 f i AlchemyLab.obj
 0001:00093d90       ?SetFrameRate@ldwGameWindowImpl@@QAEXH@Z 00494d90 f i ldwGameWindow.obj
 0001:00093d90       ?Remove@IVillagerAttachment@@UAEXH@Z 00494d90 f i EnvironmentalSound.obj
 0001:00093da0       ??0?$CComPolyObject@VCAxHostWindow@ATL@@@ATL@@QAE@PAX@Z 00494da0 f i FlashPlayer.obj
 0001:00093e30       ?FinalConstruct@?$CComPolyObject@VCAxHostWindow@ATL@@@ATL@@QAEJXZ 00494e30 f i FlashPlayer.obj
 0001:00093e70       ?GetVillagerPose@CIslandEvent@@UAE?AW4EBodyPosition@@XZ 00494e70 f i IslandEvents.obj
 0001:00093e70       ?GetExtraKerning@ldwFont@@MAEHXZ 00494e70 f i ldwFont.obj
 0001:00093e70       ?ExitInstance@CGapiApplication@@MAEJXZ 00494e70 f i ldwGameWindow.obj
 0001:00093e70       ?InitInstance@CGapiApplication@@MAEJXZ 00494e70 f i ldwGameWindow.obj
 0001:00093e70       ?_AtlFinalConstruct@CComObjectRootBase@ATL@@QAEJXZ 00494e70 f i FlashPlayer.obj
 0001:00093e70       ?GetTargetVillager2@CIslandEvent@@UAEPAVCVillager@@XZ 00494e70 f i IslandEvents.obj
 0001:00093e70       ?OnMinimize@CGapiApplication@@MAEJXZ 00494e70 f i ldwGapiApplication.obj
 0001:00093e70       ?GetResult@CIslandEventDialog@@UAEHXZ 00494e70 f i IslandEvents.obj
 0001:00093e70       ?FinalConstruct@CComObjectRootBase@ATL@@QAEJXZ 00494e70 f i FlashPlayer.obj
 0001:00093e70       ?OnRestore@CGapiApplication@@MAEJXZ 00494e70 f i ldwGapiApplication.obj
 0001:00093e80       ?InternalAddRef@?$CComObjectRootEx@VCComSingleThreadModel@ATL@@@ATL@@QAEKXZ 00494e80 f i FlashPlayer.obj
 0001:00093ea0       ?InternalRelease@?$CComObjectRootEx@VCComSingleThreadModel@ATL@@@ATL@@QAEKXZ 00494ea0 f i FlashPlayer.obj
 0001:00093ec0       ?Increment@CComSingleThreadModel@ATL@@SGKPAJ@Z 00494ec0 f i FlashPlayer.obj
 0001:00093ee0       ?Decrement@CComSingleThreadModel@ATL@@SGKPAJ@Z 00494ee0 f i FlashPlayer.obj
 0001:00093f00       ?AddRef@?$CComPolyObject@VCAxHostWindow@ATL@@@ATL@@UAGKXZ 00494f00 f i FlashPlayer.obj
 0001:00093f20       ?Release@?$CComPolyObject@VCAxHostWindow@ATL@@@ATL@@UAGKXZ 00494f20 f i FlashPlayer.obj
 0001:00093f70       ?QueryInterface@?$CComPolyObject@VCAxHostWindow@ATL@@@ATL@@UAGJABU_GUID@@PAPAX@Z 00494f70 f i FlashPlayer.obj
 0001:00093fe0       ?InlineIsEqualUnknown@ATL@@YGHABU_GUID@@@Z 00494fe0 f i FlashPlayer.obj
 0001:00094030       ?_InternalQueryInterface@CAxHostWindow@ATL@@QAEJABU_GUID@@PAPAX@Z 00495030 f i FlashPlayer.obj
 0001:00094060       ?InternalQueryInterface@CComObjectRootBase@ATL@@SGJPAXPBU_ATL_INTMAP_ENTRY@2@ABU_GUID@@PAPAX@Z 00495060 f i FlashPlayer.obj
 0001:00094090       ?_GetEntries@CAxHostWindow@ATL@@SGPBU_ATL_INTMAP_ENTRY@2@XZ 00495090 f i FlashPlayer.obj
 0001:000940a0       ?AtlInternalQueryInterface@ATL@@YGJPAXPBU_ATL_INTMAP_ENTRY@1@ABU_GUID@@PAPAX@Z 004950a0 f i FlashPlayer.obj
 0001:000941c0       _InlineIsEqualGUID         004951c0 f i FlashPlayer.obj
 0001:00094220       ??_E?$CComPolyObject@VCAxHostWindow@ATL@@@ATL@@UAEPAXI@Z 00495220 f i FlashPlayer.obj
 0001:00094220       ??_G?$CComPolyObject@VCAxHostWindow@ATL@@@ATL@@UAEPAXI@Z 00495220 f i FlashPlayer.obj
 0001:00094250       ??1?$CComPolyObject@VCAxHostWindow@ATL@@@ATL@@UAE@XZ 00495250 f i FlashPlayer.obj
 0001:000942c0       ??1?$CComContainedObject@VCAxHostWindow@ATL@@@ATL@@UAE@XZ 004952c0 f i FlashPlayer.obj
 0001:000942e0       ??1CAxHostWindow@ATL@@UAE@XZ 004952e0 f i FlashPlayer.obj
 0001:000943d0       ??1?$CWindowImpl@VCAxHostWindow@ATL@@VCWindow@2@V?$CWinTraits@$0FGAAAAAA@$0A@@2@@ATL@@UAE@XZ 004953d0 f i FlashPlayer.obj
 0001:000943d0       ??1?$CWindowImpl@VCAxUIWindow@ATL@@VCWindow@2@V?$CWinTraits@$0FGAAAAAA@$0A@@2@@ATL@@UAE@XZ 004953d0 f i FlashPlayer.obj
 0001:000943d0       ??1?$CWindowImpl@VCAxFrameWindow@ATL@@VCWindow@2@V?$CWinTraits@$0FGAAAAAA@$0A@@2@@ATL@@UAE@XZ 004953d0 f i FlashPlayer.obj
 0001:000943f0       ??1?$CWindowImplBaseT@VCWindow@ATL@@V?$CWinTraits@$0FGAAAAAA@$0A@@2@@ATL@@UAE@XZ 004953f0 f i FlashPlayer.obj
 0001:00094410       ??1?$CWindowImplRoot@VCWindow@ATL@@@ATL@@UAE@XZ 00495410 f i FlashPlayer.obj
 0001:00094430       ??1?$IObjectWithSiteImpl@VCAxHostWindow@ATL@@@ATL@@UAE@XZ 00495430 f i FlashPlayer.obj
 0001:00094450       ??1?$CComPtrBase@UIOleInPlaceActiveObject@@@ATL@@QAE@XZ 00495450 f i FlashPlayer.obj
 0001:00094450       ??1?$CComPtrBase@UIAdviseSink@@@ATL@@QAE@XZ 00495450 f i FlashPlayer.obj
 0001:00094450       ??1?$CComPtrBase@UIAxWinHostWindow@@@ATL@@QAE@XZ 00495450 f i FlashPlayer.obj
 0001:00094450       ??1?$CComPtrBase@UIClassFactory2@@@ATL@@QAE@XZ 00495450 f i FlashPlayer.obj
 0001:00094450       ??1?$CComPtrBase@UIConnectionPointContainer@@@ATL@@QAE@XZ 00495450 f i FlashPlayer.obj
 0001:00094450       ??1?$CComPtrBase@UITypeInfo2@@@ATL@@QAE@XZ 00495450 f i FlashPlayer.obj
 0001:00094450       ??1?$CComPtrBase@UIOleInPlaceFrame@@@ATL@@QAE@XZ 00495450 f i FlashPlayer.obj
 0001:00094450       ??1?$CComPtrBase@UIConnectionPoint@@@ATL@@QAE@XZ 00495450 f i FlashPlayer.obj
 0001:00094450       ??1?$CComPtrBase@UIOleInPlaceObjectWindowless@@@ATL@@QAE@XZ 00495450 f i FlashPlayer.obj
 0001:00094450       ??1?$CComPtrBase@UIUnknown@@@ATL@@QAE@XZ 00495450 f i FlashPlayer.obj
 0001:00094450       ??1?$CComPtrBase@UITypeInfo@@@ATL@@QAE@XZ 00495450 f i FlashPlayer.obj
 0001:00094450       ??1?$CComPtrBase@UIAxWinHostWindowLic@@@ATL@@QAE@XZ 00495450 f i FlashPlayer.obj
 0001:00094450       ??1?$CComPtrBase@UIPersistStreamInit@@@ATL@@QAE@XZ 00495450 f i FlashPlayer.obj
 0001:00094450       ??1?$CComPtrBase@UIViewObjectEx@@@ATL@@QAE@XZ 00495450 f i FlashPlayer.obj
 0001:00094450       ??1?$CComPtrBase@UIDocHostUIHandlerDispatch@@@ATL@@QAE@XZ 00495450 f i FlashPlayer.obj
 0001:00094450       ??1?$CComPtrBase@UIObjectWithSite@@@ATL@@QAE@XZ 00495450 f i FlashPlayer.obj
 0001:00094450       ??1?$CComPtrBase@UIOleControl@@@ATL@@QAE@XZ 00495450 f i FlashPlayer.obj
 0001:00094450       ??1?$CComPtrBase@UIOleObject@@@ATL@@QAE@XZ 00495450 f i FlashPlayer.obj
 0001:00094450       ??1?$CComPtrBase@UIPersistStream@@@ATL@@QAE@XZ 00495450 f i FlashPlayer.obj
 0001:00094450       ??1?$CComPtrBase@UIOleInPlaceUIWindow@@@ATL@@QAE@XZ 00495450 f i FlashPlayer.obj
 0001:00094450       ??1?$CComPtrBase@UIWebBrowser2@@@ATL@@QAE@XZ 00495450 f i FlashPlayer.obj
 0001:00094450       ??1?$CComPtrBase@UIOleClientSite@@@ATL@@QAE@XZ 00495450 f i FlashPlayer.obj
 0001:00094450       ??1?$CComPtrBase@UIDispatch@@@ATL@@QAE@XZ 00495450 f i FlashPlayer.obj
 0001:00094450       ??1?$CComPtrBase@UIStream@@@ATL@@QAE@XZ 00495450 f i FlashPlayer.obj
 0001:00094450       ??1?$CComPtrBase@UIServiceProvider@@@ATL@@QAE@XZ 00495450 f i FlashPlayer.obj
 0001:00094450       ??1?$CComPtrBase@UIFontDisp@@@ATL@@QAE@XZ 00495450 f i FlashPlayer.obj
 0001:00094480       ??1CWndProcThunk@ATL@@QAE@XZ 00495480 f i FlashPlayer.obj
 0001:000944a0       ??1CDynamicStdCallThunk@ATL@@QAE@XZ 004954a0 f i FlashPlayer.obj
 0001:000944d0       ?FinalRelease@?$CComPolyObject@VCAxHostWindow@ATL@@@ATL@@QAEXXZ 004954d0 f i FlashPlayer.obj
 0001:00094500       ?FinalRelease@CAxHostWindow@ATL@@QAEXXZ 00495500 f i FlashPlayer.obj
 0001:00094520       ?ReleaseAll@CAxHostWindow@ATL@@QAEXXZ 00495520 f i FlashPlayer.obj
 0001:000947d0       ?AtlUnadvise@ATL@@YGJPAUIUnknown@@ABU_GUID@@K@Z 004957d0 f i FlashPlayer.obj
 0001:00094890       ?Release@?$CComPtrBase@UIOleObject@@@ATL@@QAEXXZ 00495890 f i FlashPlayer.obj
 0001:00094890       ?Release@?$CComPtrBase@UIServiceProvider@@@ATL@@QAEXXZ 00495890 f i FlashPlayer.obj
 0001:00094890       ?Release@?$CComPtrBase@UIOleInPlaceUIWindow@@@ATL@@QAEXXZ 00495890 f i FlashPlayer.obj
 0001:00094890       ?Release@?$CComPtrBase@UIOleInPlaceFrame@@@ATL@@QAEXXZ 00495890 f i FlashPlayer.obj
 0001:00094890       ?Release@?$CComPtrBase@UIOleInPlaceObjectWindowless@@@ATL@@QAEXXZ 00495890 f i FlashPlayer.obj
 0001:00094890       ?Release@?$CComPtrBase@UIOleInPlaceActiveObject@@@ATL@@QAEXXZ 00495890 f i FlashPlayer.obj
 0001:00094890       ?Release@?$CComPtrBase@UIUnknown@@@ATL@@QAEXXZ 00495890 f i FlashPlayer.obj
 0001:00094890       ?Release@?$CComPtrBase@UIViewObjectEx@@@ATL@@QAEXXZ 00495890 f i FlashPlayer.obj
 0001:000948c0       ??0?$CComContainedObject@VCAxHostWindow@ATL@@@ATL@@QAE@PAX@Z 004958c0 f i FlashPlayer.obj
 0001:00094950       ??0CAxHostWindow@ATL@@QAE@XZ 00495950 f i FlashPlayer.obj
 0001:00094c10       ?OnFinalMessage@CAxHostWindow@ATL@@UAEXPAUHWND__@@@Z 00495c10 f i FlashPlayer.obj
 0001:00094c40       ?ProcessWindowMessage@CAxHostWindow@ATL@@UAEHPAUHWND__@@IIJAAJK@Z 00495c40 f i FlashPlayer.obj
 0001:00095530       ?OnForwardMsg@CAxHostWindow@ATL@@QAEJIIJAAH@Z 00496530 f i FlashPlayer.obj
 0001:000955e0       ?OnGetUnknown@CAxHostWindow@ATL@@QAEJIIJAAH@Z 004965e0 f i FlashPlayer.obj
 0001:00095610       ?OnGetControl@CAxHostWindow@ATL@@QAEJIIJAAH@Z 00496610 f i FlashPlayer.obj
 0001:00095650       ?OnEraseBackground@CAxHostWindow@ATL@@QAEJIIJAAH@Z 00496650 f i FlashPlayer.obj
 0001:00095680       ?OnMouseActivate@CAxHostWindow@ATL@@QAEJIIJAAH@Z 00496680 f i FlashPlayer.obj
 0001:000957a0       ?OnSetFocus@CAxHostWindow@ATL@@QAEJIIJAAH@Z 004967a0 f i FlashPlayer.obj
 0001:00095900       ?IsChild@CWindow@ATL@@QBEHPAUHWND__@@@Z 00496900 f i FlashPlayer.obj
 0001:00095920       ?OnKillFocus@CAxHostWindow@ATL@@QAEJIIJAAH@Z 00496920 f i FlashPlayer.obj
 0001:00095950       ?OnSize@CAxHostWindow@ATL@@QAEJIIJAAH@Z 00496950 f i FlashPlayer.obj
 0001:00095aa0       ?OnDestroy@CAxHostWindow@ATL@@QAEJIIJAAH@Z 00496aa0 f i FlashPlayer.obj
 0001:00095af0       ?OnWindowMessage@CAxHostWindow@ATL@@QAEJIIJAAH@Z 00496af0 f i FlashPlayer.obj
 0001:00095b90       ?OnWindowlessMouseMessage@CAxHostWindow@ATL@@QAEJIIJAAH@Z 00496b90 f i FlashPlayer.obj
 0001:00095c20       ?OnPaint@CAxHostWindow@ATL@@QAEJIIJAAH@Z 00496c20 f i FlashPlayer.obj
 0001:00095f00       ?GetClientRect@CWindow@ATL@@QBEHPAUtagRECT@@@Z 00496f00 f i FlashPlayer.obj
 0001:00095f20       ?CreateControl@CAxHostWindow@ATL@@UAGJPBGPAUHWND__@@PAUIStream@@@Z 00496f20 f i FlashPlayer.obj
 0001:00095fa0       ?CreateControlEx@CAxHostWindow@ATL@@UAGJPBGPAUHWND__@@PAUIStream@@PAPAUIUnknown@@ABU_GUID@@PAU5@@Z 00496fa0 f i FlashPlayer.obj
 0001:00095fd0       ?AttachControl@CAxHostWindow@ATL@@UAGJPAUIUnknown@@PAUHWND__@@@Z 00496fd0 f i FlashPlayer.obj
 0001:000960b0       ?RedrawWindow@CWindow@ATL@@QAEHPBUtagRECT@@PAUHRGN__@@I@Z 004970b0 f i FlashPlayer.obj
 0001:000960e0       ?QueryControl@CAxHostWindow@ATL@@UAGJABU_GUID@@PAPAX@Z 004970e0 f i FlashPlayer.obj
 0001:00096150       ?SetExternalDispatch@CAxHostWindow@ATL@@UAGJPAUIDispatch@@@Z 00497150 f i FlashPlayer.obj
 0001:00096170       ?AtlComPtrAssign@ATL@@YGPAUIUnknown@@PAPAU2@PAU2@@Z 00497170 f i FlashPlayer.obj
 0001:000961c0       ?SetExternalUIHandler@CAxHostWindow@ATL@@UAGJPAUIDocHostUIHandlerDispatch@@@Z 004971c0 f i FlashPlayer.obj
 0001:000961e0       ?CreateControlLic@CAxHostWindow@ATL@@UAGJPBGPAUHWND__@@PAUIStream@@PAG@Z 004971e0 f i FlashPlayer.obj
 0001:00096260       ?CreateControlLicEx@CAxHostWindow@ATL@@UAGJPBGPAUHWND__@@PAUIStream@@PAPAUIUnknown@@ABU_GUID@@PAU5@PAG@Z 00497260 f i FlashPlayer.obj
 0001:000967c0       ?GetStyle@CWindow@ATL@@QBEKXZ 004977c0 f i FlashPlayer.obj
 0001:000967e0       ?SetWindowLongA@CWindow@ATL@@QAEJHJ@Z 004977e0 f i FlashPlayer.obj
 0001:00096810       ?SetWindowPos@CWindow@ATL@@QAEHPAUHWND__@@HHHHI@Z 00497810 f i FlashPlayer.obj
 0001:00096850       ?IsParentDialog@CWindow@ATL@@QAEHXZ 00497850 f i FlashPlayer.obj
 0001:000968a0       ?GetParent@CWindow@ATL@@QBE?AV12@XZ 004978a0 f i FlashPlayer.obj
 0001:000968d0       ?ocslen@@YAHPBG@Z          004978d0 f i FlashPlayer.obj
 0001:000968e0       ??0CComVariant@ATL@@QAE@XZ 004978e0 f i FlashPlayer.obj
 0001:00096900       ??1CComVariant@ATL@@QAE@XZ 00497900 f i FlashPlayer.obj
 0001:00096920       ??0CComVariant@ATL@@QAE@PBG@Z 00497920 f i FlashPlayer.obj
 0001:00096950       ??4CComVariant@ATL@@QAEAAV01@PBG@Z 00497950 f i FlashPlayer.obj
 0001:000969b0       ?Clear@CComVariant@ATL@@QAEJXZ 004979b0 f i FlashPlayer.obj
 0001:000969d0       ?AtlW2AHelper@@YGPADPADPBGHI@Z 004979d0 f i FlashPlayer.obj
 0001:00096a20       ?FindOneOf@CAtlModule@ATL@@SAPBDPBD0@Z 00497a20 f i FlashPlayer.obj
 0001:00096a90       ?ShowContextMenu@CAxHostWindow@ATL@@UAGJKPAUtagPOINT@@PAUIUnknown@@PAUIDispatch@@@Z 00497a90 f i FlashPlayer.obj
 0001:00096b00       ?GetHostInfo@CAxHostWindow@ATL@@UAGJPAU_DOCHOSTUIINFO@@@Z 00497b00 f i FlashPlayer.obj
 0001:00096b70       ?ShowUI@CAxHostWindow@ATL@@UAGJKPAUIOleInPlaceActiveObject@@PAUIOleCommandTarget@@PAUIOleInPlaceFrame@@PAUIOleInPlaceUIWindow@@@Z 00497b70 f i FlashPlayer.obj
 0001:00096be0       ?HideUI@CAxHostWindow@ATL@@UAGJXZ 00497be0 f i FlashPlayer.obj
 0001:00096c30       ?UpdateUI@CAxHostWindow@ATL@@UAGJXZ 00497c30 f i FlashPlayer.obj
 0001:00096c80       ?EnableModeless@CAxHostWindow@ATL@@UAGJH@Z 00497c80 f i FlashPlayer.obj
 0001:00096cd0       ?OnDocWindowActivate@CAxHostWindow@ATL@@UAGJH@Z 00497cd0 f i FlashPlayer.obj
 0001:00096d20       ?OnFrameWindowActivate@CAxHostWindow@ATL@@UAGJH@Z 00497d20 f i FlashPlayer.obj
 0001:00096d70       ?ResizeBorder@CAxHostWindow@ATL@@UAGJPBUtagRECT@@PAUIOleInPlaceUIWindow@@H@Z 00497d70 f i FlashPlayer.obj
 0001:00096de0       ?TranslateAcceleratorA@CAxHostWindow@ATL@@UAGJPAUtagMSG@@PBU_GUID@@K@Z 00497de0 f i FlashPlayer.obj
 0001:00096ea0       ??0CComBSTR@ATL@@QAE@ABU_GUID@@@Z 00497ea0 f i FlashPlayer.obj
 0001:00096f00       ?GetOptionKeyPath@CAxHostWindow@ATL@@UAGJPAPAGK@Z 00497f00 f i FlashPlayer.obj
 0001:00096fe0       ?ocscpy@@YAPAGPAGPBG@Z     00497fe0 f i FlashPlayer.obj
 0001:00097010       ?ByteLength@CComBSTR@ATL@@QBEIXZ 00498010 f i FlashPlayer.obj
 0001:00097040       ?GetDropTarget@CAxHostWindow@ATL@@UAGJPAUIDropTarget@@PAPAU3@@Z 00498040 f i FlashPlayer.obj
 0001:00097130       ?GetExternal@CAxHostWindow@ATL@@UAGJPAPAUIDispatch@@@Z 00498130 f i FlashPlayer.obj
 0001:000971d0       ?TranslateUrl@CAxHostWindow@ATL@@UAGJKPAGPAPAG@Z 004981d0 f i FlashPlayer.obj
 0001:00097320       ?FilterDataObject@CAxHostWindow@ATL@@UAGJPAUIDataObject@@PAPAU3@@Z 00498320 f i FlashPlayer.obj
 0001:00097410       ?Invoke@CAxHostWindow@ATL@@UAGJJABU_GUID@@KGPAUtagDISPPARAMS@@PAUtagVARIANT@@PAUtagEXCEPINFO@@PAI@Z 00498410 f i FlashPlayer.obj
 0001:000974d0       ?FireAmbientPropertyChange@CAxHostWindow@ATL@@QAEJJ@Z 004984d0 f i FlashPlayer.obj
 0001:00097570       ?put_AllowWindowlessActivation@CAxHostWindow@ATL@@UAGJF@Z 00498570 f i FlashPlayer.obj
 0001:000975a0       ?get_AllowWindowlessActivation@CAxHostWindow@ATL@@UAGJPAF@Z 004985a0 f i FlashPlayer.obj
 0001:000975d0       ?put_BackColor@CAxHostWindow@ATL@@UAGJK@Z 004985d0 f i FlashPlayer.obj
 0001:00097610       ?get_BackColor@CAxHostWindow@ATL@@UAGJPAK@Z 00498610 f i FlashPlayer.obj
 0001:00097640       ?put_ForeColor@CAxHostWindow@ATL@@UAGJK@Z 00498640 f i FlashPlayer.obj
 0001:00097670       ?get_ForeColor@CAxHostWindow@ATL@@UAGJPAK@Z 00498670 f i FlashPlayer.obj
 0001:000976a0       ?put_LocaleID@CAxHostWindow@ATL@@UAGJK@Z 004986a0 f i FlashPlayer.obj
 0001:000976d0       ?get_LocaleID@CAxHostWindow@ATL@@UAGJPAK@Z 004986d0 f i FlashPlayer.obj
 0001:00097700       ?put_UserMode@CAxHostWindow@ATL@@UAGJF@Z 00498700 f i FlashPlayer.obj
 0001:00097740       ?get_UserMode@CAxHostWindow@ATL@@UAGJPAF@Z 00498740 f i FlashPlayer.obj
 0001:00097770       ?put_DisplayAsDefault@CAxHostWindow@ATL@@UAGJF@Z 00498770 f i FlashPlayer.obj
 0001:000977b0       ?get_DisplayAsDefault@CAxHostWindow@ATL@@UAGJPAF@Z 004987b0 f i FlashPlayer.obj
 0001:000977e0       ?put_Font@CAxHostWindow@ATL@@UAGJPAUIFontDisp@@@Z 004987e0 f i FlashPlayer.obj
 0001:00097810       ?get_Font@CAxHostWindow@ATL@@UAGJPAPAUIFontDisp@@@Z 00498810 f i FlashPlayer.obj
 0001:00097a20       ?AtlHresultFromLastError@ATL@@YAJXZ 00498a20 f i FlashPlayer.obj
 0001:00097a60       ?put_MessageReflect@CAxHostWindow@ATL@@UAGJF@Z 00498a60 f i FlashPlayer.obj
 0001:00097aa0       ?get_MessageReflect@CAxHostWindow@ATL@@UAGJPAF@Z 00498aa0 f i FlashPlayer.obj
 0001:00097ad0       ?get_ShowGrabHandles@CAxHostWindow@ATL@@UAGJPAF@Z 00498ad0 f i FlashPlayer.obj
 0001:00097af0       ?get_ShowHatching@CAxHostWindow@ATL@@UAGJPAF@Z 00498af0 f i FlashPlayer.obj
 0001:00097b10       ?put_DocHostFlags@CAxHostWindow@ATL@@UAGJK@Z 00498b10 f i FlashPlayer.obj
 0001:00097b40       ?get_DocHostFlags@CAxHostWindow@ATL@@UAGJPAK@Z 00498b40 f i FlashPlayer.obj
 0001:00097b70       ?put_DocHostDoubleClickFlags@CAxHostWindow@ATL@@UAGJK@Z 00498b70 f i FlashPlayer.obj
 0001:00097b90       ?get_DocHostDoubleClickFlags@CAxHostWindow@ATL@@UAGJPAK@Z 00498b90 f i FlashPlayer.obj
 0001:00097bc0       ?put_AllowContextMenu@CAxHostWindow@ATL@@UAGJF@Z 00498bc0 f i FlashPlayer.obj
 0001:00097bf0       ?get_AllowContextMenu@CAxHostWindow@ATL@@UAGJPAF@Z 00498bf0 f i FlashPlayer.obj
 0001:00097c20       ?put_AllowShowUI@CAxHostWindow@ATL@@UAGJF@Z 00498c20 f i FlashPlayer.obj
 0001:00097c50       ?get_AllowShowUI@CAxHostWindow@ATL@@UAGJPAF@Z 00498c50 f i FlashPlayer.obj
 0001:00097c80       ?put_OptionKeyPath@CAxHostWindow@ATL@@UAGJPAG@Z 00498c80 f i FlashPlayer.obj
 0001:00097ca0       ??4CComBSTR@ATL@@QAEAAV01@PBG@Z 00498ca0 f i FlashPlayer.obj
 0001:00097d00       ?get_OptionKeyPath@CAxHostWindow@ATL@@UAGJPAPAG@Z 00498d00 f i FlashPlayer.obj
 0001:00097d30       ?SetAmbientDispatch@CAxHostWindow@ATL@@UAGJPAUIDispatch@@@Z 00498d30 f i FlashPlayer.obj
 0001:00097d50       ?SetSite@CAxHostWindow@ATL@@UAGJPAUIUnknown@@@Z 00498d50 f i FlashPlayer.obj
 0001:00097dd0       ?TransformCoords@CAxHostWindow@ATL@@UAGJPAU_POINTL@@PAUtagPOINTF@@K@Z 00498dd0 f i FlashPlayer.obj
 0001:00097dd0       ?GetMoniker@CAxHostWindow@ATL@@UAGJKKPAPAUIMoniker@@@Z 00498dd0 f i FlashPlayer.obj
 0001:00097de0       ?GetContainer@CAxHostWindow@ATL@@UAGJPAPAUIOleContainer@@@Z 00498de0 f i FlashPlayer.obj
 0001:00097e70       ?ShowObject@CAxHostWindow@ATL@@UAGJXZ 00498e70 f i FlashPlayer.obj
 0001:00097f00       ?GetDC@CWindow@ATL@@QAEPAUHDC__@@XZ 00498f00 f i FlashPlayer.obj
 0001:00097f20       ?ReleaseDC@CWindow@ATL@@QAEHPAUHDC__@@@Z 00498f20 f i FlashPlayer.obj
 0001:00097f40       ?ShowPropertyFrame@CAxHostWindow@ATL@@UAGJXZ 00498f40 f i FlashPlayer.obj
 0001:00097f40       ?DiscardUndoState@CAxHostWindow@ATL@@UAGJXZ 00498f40 f i FlashPlayer.obj
 0001:00097f40       ?RequestNewObjectLayout@CAxHostWindow@ATL@@UAGJXZ 00498f40 f i FlashPlayer.obj
 0001:00097f40       ?DeactivateAndUndo@CAxHostWindow@ATL@@UAGJXZ 00498f40 f i FlashPlayer.obj
 0001:00097f40       ?SaveObject@CAxHostWindow@ATL@@UAGJXZ 00498f40 f i FlashPlayer.obj
 0001:00097f50       ?GetWindow@CAxHostWindow@ATL@@UAGJPAPAUHWND__@@@Z 00498f50 f i FlashPlayer.obj
 0001:00097f70       ?OnShowWindow@CAxHostWindow@ATL@@UAGJH@Z 00498f70 f i FlashPlayer.obj
 0001:00097f70       ?OnPosRectChange@CAxHostWindow@ATL@@UAGJPBUtagRECT@@@Z 00498f70 f i FlashPlayer.obj
 0001:00097f70       ?ContextSensitiveHelp@CAxHostWindow@ATL@@UAGJH@Z 00498f70 f i FlashPlayer.obj
 0001:00097f80       ?OnInPlaceActivate@CAxHostWindow@ATL@@UAGJXZ 00498f80 f i FlashPlayer.obj
 0001:00097ff0       ?OnUIActivate@CAxHostWindow@ATL@@UAGJXZ 00498ff0 f i FlashPlayer.obj
 0001:00098010       ?GetWindowContext@CAxHostWindow@ATL@@UAGJPAPAUIOleInPlaceFrame@@PAPAUIOleInPlaceUIWindow@@PAUtagRECT@@2PAUtagOIFI@@@Z 00499010 f i FlashPlayer.obj
 0001:000981a0       ?OnUIDeactivate@CAxHostWindow@ATL@@UAGJH@Z 004991a0 f i FlashPlayer.obj
 0001:000981c0       ?OnInPlaceDeactivate@CAxHostWindow@ATL@@UAGJXZ 004991c0 f i FlashPlayer.obj
 0001:000981f0       ?OnInPlaceActivateEx@CAxHostWindow@ATL@@UAGJPAHK@Z 004991f0 f i FlashPlayer.obj
 0001:000982f0       ?OnInPlaceDeactivateEx@CAxHostWindow@ATL@@UAGJH@Z 004992f0 f i FlashPlayer.obj
 0001:00098320       ?CanInPlaceActivate@CAxHostWindow@ATL@@UAGJXZ 00499320 f i FlashPlayer.obj
 0001:00098320       ?OnControlInfoChanged@CAxHostWindow@ATL@@UAGJXZ 00499320 f i FlashPlayer.obj
 0001:00098320       ?RequestUIActivate@CAxHostWindow@ATL@@UAGJXZ 00499320 f i FlashPlayer.obj
 0001:00098320       ?Release@CRegObject@ATL@@UAGKXZ 00499320 f i FlashPlayer.obj
 0001:00098330       ?CanWindowlessActivate@CAxHostWindow@ATL@@UAGJXZ 00499330 f i FlashPlayer.obj
 0001:00098350       ?GetCapture@CAxHostWindow@ATL@@UAGJXZ 00499350 f i FlashPlayer.obj
 0001:00098370       ?SetCapture@CAxHostWindow@ATL@@UAGJH@Z 00499370 f i FlashPlayer.obj
 0001:000983b0       ?SetCapture@CWindow@ATL@@QAEPAUHWND__@@XZ 004993b0 f i FlashPlayer.obj
 0001:000983d0       ?GetFocus@CAxHostWindow@ATL@@UAGJXZ 004993d0 f i FlashPlayer.obj
 0001:000983f0       ?SetFocus@CAxHostWindow@ATL@@UAGJH@Z 004993f0 f i FlashPlayer.obj
 0001:00098420       ?GetDC@CAxHostWindow@ATL@@UAGJPBUtagRECT@@KPAPAUHDC__@@@Z 00499420 f i FlashPlayer.obj
 0001:00098550       ?ReleaseDC@CAxHostWindow@ATL@@UAGJPAUHDC__@@@Z 00499550 f i FlashPlayer.obj
 0001:000985d0       ?InvalidateRect@CAxHostWindow@ATL@@UAGJPBUtagRECT@@H@Z 004995d0 f i FlashPlayer.obj
 0001:000985f0       ?InvalidateRect@CWindow@ATL@@QAEHPBUtagRECT@@H@Z 004995f0 f i FlashPlayer.obj
 0001:00098620       ?InvalidateRgn@CAxHostWindow@ATL@@UAGJPAUHRGN__@@H@Z 00499620 f i FlashPlayer.obj
 0001:00098640       ?InvalidateRgn@CWindow@ATL@@QAEXPAUHRGN__@@H@Z 00499640 f i FlashPlayer.obj
 0001:00098670       ?ScrollRect@CAxHostWindow@ATL@@UAGJHHPBUtagRECT@@0@Z 00499670 f i FlashPlayer.obj
 0001:00098680       ?OnDefWindowMessage@CAxHostWindow@ATL@@UAGJIIJPAJ@Z 00499680 f i FlashPlayer.obj
 0001:000986b0       ?LockInPlaceActive@CAxHostWindow@ATL@@UAGJH@Z 004996b0 f i FlashPlayer.obj
 0001:000986b0       ?GetBorder@CAxFrameWindow@ATL@@UAGJPAUtagRECT@@@Z 004996b0 f i FlashPlayer.obj
 0001:000986b0       ?SetBorderSpace@CAxFrameWindow@ATL@@UAGJPBUtagRECT@@@Z 004996b0 f i FlashPlayer.obj
 0001:000986b0       ?EnableModeless@CAxFrameWindow@ATL@@UAGJH@Z 004996b0 f i FlashPlayer.obj
 0001:000986b0       ?SetBorderSpace@CAxUIWindow@ATL@@UAGJPBUtagRECT@@@Z 004996b0 f i FlashPlayer.obj
 0001:000986b0       ?ContextSensitiveHelp@CAxUIWindow@ATL@@UAGJH@Z 004996b0 f i FlashPlayer.obj
 0001:000986b0       ?ContextSensitiveHelp@CAxFrameWindow@ATL@@UAGJH@Z 004996b0 f i FlashPlayer.obj
 0001:000986b0       ?AdjustRect@CAxHostWindow@ATL@@UAGJPAUtagRECT@@@Z 004996b0 f i FlashPlayer.obj
 0001:000986b0       ?RemoveMenus@CAxFrameWindow@ATL@@UAGJPAUHMENU__@@@Z 004996b0 f i FlashPlayer.obj
 0001:000986b0       ?SetStatusText@CAxFrameWindow@ATL@@UAGJPBG@Z 004996b0 f i FlashPlayer.obj
 0001:000986b0       ?GetBorder@CAxUIWindow@ATL@@UAGJPAUtagRECT@@@Z 004996b0 f i FlashPlayer.obj
 0001:000986c0       ?GetExtendedControl@CAxHostWindow@ATL@@UAGJPAPAUIDispatch@@@Z 004996c0 f i FlashPlayer.obj
 0001:000986f0       ?OnFocus@CAxHostWindow@ATL@@UAGJH@Z 004996f0 f i FlashPlayer.obj
 0001:00098720       ?OnDataChange@CAxHostWindow@ATL@@UAGXPAUtagFORMATETC@@PAUtagSTGMEDIUM@@@Z 00499720 f i FlashPlayer.obj
 0001:00098720       ?OnViewChange@CAxHostWindow@ATL@@UAGXKJ@Z 00499720 f i FlashPlayer.obj
 0001:00098730       ?OnRename@CAxHostWindow@ATL@@UAGXPAUIMoniker@@@Z 00499730 f i FlashPlayer.obj
 0001:00098740       ?OnClose@CAxHostWindow@ATL@@UAGXXZ 00499740 f i FlashPlayer.obj
 0001:00098740       ?OnSave@CAxHostWindow@ATL@@UAGXXZ 00499740 f i FlashPlayer.obj
 0001:00098750       ?ParseDisplayName@CAxHostWindow@ATL@@UAGJPAUIBindCtx@@PAGPAKPAPAUIMoniker@@@Z 00499750 f i FlashPlayer.obj
 0001:00098760       ?EnumObjects@CAxHostWindow@ATL@@UAGJKPAPAUIEnumUnknown@@@Z 00499760 f i FlashPlayer.obj
 0001:000988a0       ?LockContainer@CAxHostWindow@ATL@@UAGJH@Z 004998a0 f i FlashPlayer.obj
 0001:000988d0       ?ActivateAx@CAxHostWindow@ATL@@QAEJPAUIUnknown@@_NPAUIStream@@@Z 004998d0 f i FlashPlayer.obj
 0001:00098f00       ?SubclassWindow@CAxHostWindow@ATL@@QAEXPAUHWND__@@@Z 00499f00 f i FlashPlayer.obj
 0001:00098f40       ?ReleaseWindow@CAxHostWindow@ATL@@QAEXXZ 00499f40 f i FlashPlayer.obj
 0001:00098f90       ?ReflectNotifications@CAxHostWindow@ATL@@QAEJIIJAAH@Z 00499f90 f i FlashPlayer.obj
 0001:00099220       ?GetDlgItem@CWindow@ATL@@QBE?AV12@H@Z 0049a220 f i FlashPlayer.obj
 0001:00099250       ?QueryService@CAxHostWindow@ATL@@UAGJABU_GUID@@0PAPAX@Z 0049a250 f i FlashPlayer.obj
 0001:000992d0       ??0?$IObjectWithSiteImpl@VCAxHostWindow@ATL@@@ATL@@QAE@XZ 0049a2d0 f i FlashPlayer.obj
 0001:00099300       ??0?$IDispatchImpl@UIAxWinAmbientDispatchEx@@$1?_GUID_b2d0778b_ac99_4c58_a5c8_e7724e5316b5@@3U__s_GUID@@B$1?m_libid@CAtlModule@ATL@@2U_GUID@@A$0PPPP@$0PPPP@VCComTypeInfoHolder@ATL@@@ATL@@QAE@XZ 0049a300 f i FlashPlayer.obj
 0001:00099300       ??0IOleInPlaceSiteWindowless@@QAE@XZ 0049a300 f i FlashPlayer.obj
 0001:00099320       ??1?$CComQIPtr@UIOleClientSite@@$1?_GUID_00000118_0000_0000_c000_000000000046@@3U__s_GUID@@B@ATL@@QAE@XZ 0049a320 f i FlashPlayer.obj
 0001:00099320       ??1?$CComQIPtr@UIOleInPlaceActiveObject@@$1?_GUID_00000117_0000_0000_c000_000000000046@@3U__s_GUID@@B@ATL@@QAE@XZ 0049a320 f i FlashPlayer.obj
 0001:00099320       ??1?$CComQIPtr@UIOleControl@@$1?_GUID_b196b288_bab4_101a_b69c_00aa00341d07@@3U__s_GUID@@B@ATL@@QAE@XZ 0049a320 f i FlashPlayer.obj
 0001:00099320       ??1?$CComQIPtr@UIAdviseSink@@$1?_GUID_0000010f_0000_0000_c000_000000000046@@3U__s_GUID@@B@ATL@@QAE@XZ 0049a320 f i FlashPlayer.obj
 0001:00099320       ??1?$CComQIPtr@UIPersistStreamInit@@$1?_GUID_7fd52380_4e07_101b_ae2d_08002b2ec713@@3U__s_GUID@@B@ATL@@QAE@XZ 0049a320 f i FlashPlayer.obj
 0001:00099320       ??1?$CComQIPtr@UIPersistStream@@$1?_GUID_00000109_0000_0000_c000_000000000046@@3U__s_GUID@@B@ATL@@QAE@XZ 0049a320 f i FlashPlayer.obj
 0001:00099340       ??1?$CComPtr@UIOleInPlaceObjectWindowless@@@ATL@@QAE@XZ 0049a340 f i FlashPlayer.obj
 0001:00099340       ??1?$CComPtr@UIDispatch@@@ATL@@QAE@XZ 0049a340 f i FlashPlayer.obj
 0001:00099340       ??1?$CComPtr@UIOleObject@@@ATL@@QAE@XZ 0049a340 f i FlashPlayer.obj
 0001:00099340       ??1?$CComPtr@UITypeInfo@@@ATL@@QAE@XZ 0049a340 f i FlashPlayer.obj
 0001:00099340       ??1?$CComPtr@UIPersistStream@@@ATL@@QAE@XZ 0049a340 f i FlashPlayer.obj
 0001:00099340       ??1?$CComPtr@UIDocHostUIHandlerDispatch@@@ATL@@QAE@XZ 0049a340 f i FlashPlayer.obj
 0001:00099340       ??1?$CComPtr@UIOleInPlaceActiveObject@@@ATL@@QAE@XZ 0049a340 f i FlashPlayer.obj
 0001:00099340       ??1?$CComPtr@UITypeInfo2@@@ATL@@QAE@XZ 0049a340 f i FlashPlayer.obj
 0001:00099340       ??1?$CComPtr@UIStream@@@ATL@@QAE@XZ 0049a340 f i FlashPlayer.obj
 0001:00099340       ??1?$CComPtr@UIServiceProvider@@@ATL@@QAE@XZ 0049a340 f i FlashPlayer.obj
 0001:00099340       ??1?$CComPtr@UIWebBrowser2@@@ATL@@QAE@XZ 0049a340 f i FlashPlayer.obj
 0001:00099340       ??1?$CComPtr@UIOleInPlaceFrame@@@ATL@@QAE@XZ 0049a340 f i FlashPlayer.obj
 0001:00099340       ??1?$CComPtr@UIViewObjectEx@@@ATL@@QAE@XZ 0049a340 f i FlashPlayer.obj
 0001:00099340       ??1?$CComPtr@UIUnknown@@@ATL@@QAE@XZ 0049a340 f i FlashPlayer.obj
 0001:00099340       ??1?$CComPtr@UIConnectionPoint@@@ATL@@QAE@XZ 0049a340 f i FlashPlayer.obj
 0001:00099340       ??1?$CComPtr@UIPersistStreamInit@@@ATL@@QAE@XZ 0049a340 f i FlashPlayer.obj
 0001:00099340       ??1?$CComPtr@UIOleClientSite@@@ATL@@QAE@XZ 0049a340 f i FlashPlayer.obj
 0001:00099340       ??1?$CComPtr@UIConnectionPointContainer@@@ATL@@QAE@XZ 0049a340 f i FlashPlayer.obj
 0001:00099340       ??1?$CComPtr@UIObjectWithSite@@@ATL@@QAE@XZ 0049a340 f i FlashPlayer.obj
 0001:00099340       ??1?$CComPtr@UIFontDisp@@@ATL@@QAE@XZ 0049a340 f i FlashPlayer.obj
 0001:00099340       ??1?$CComPtr@UIClassFactory2@@@ATL@@QAE@XZ 0049a340 f i FlashPlayer.obj
 0001:00099340       ??1?$CComPtr@UIAdviseSink@@@ATL@@QAE@XZ 0049a340 f i FlashPlayer.obj
 0001:00099340       ??1?$CComPtr@UIOleInPlaceUIWindow@@@ATL@@QAE@XZ 0049a340 f i FlashPlayer.obj
 0001:00099340       ??1?$CComPtr@UIAxWinHostWindow@@@ATL@@QAE@XZ 0049a340 f i FlashPlayer.obj
 0001:00099340       ??1?$CComPtr@UIOleControl@@@ATL@@QAE@XZ 0049a340 f i FlashPlayer.obj
 0001:00099340       ??1?$CComPtr@UIAxWinHostWindowLic@@@ATL@@QAE@XZ 0049a340 f i FlashPlayer.obj
 0001:00099360       ?AtlHiMetricToPixel@ATL@@YGXPBUtagSIZE@@PAU2@@Z 0049a360 f i FlashPlayer.obj
 0001:000993e0       ?AtlPixelToHiMetric@ATL@@YGXPBUtagSIZE@@PAU2@@Z 0049a3e0 f i FlashPlayer.obj
 0001:00099460       ?AtlAdvise@ATL@@YGJPAUIUnknown@@0ABU_GUID@@PAK@Z 0049a460 f i FlashPlayer.obj
 0001:00099520       ??0?$CComPtr@UIUnknown@@@ATL@@QAE@PAUIUnknown@@@Z 0049a520 f i FlashPlayer.obj
 0001:00099540       ??0?$CWindowImplBaseT@VCWindow@ATL@@V?$CWinTraits@$0FGAAAAAA@$0A@@2@@ATL@@QAE@XZ 0049a540 f i FlashPlayer.obj
 0001:00099570       ?GetWindowProc@?$CWindowImplBaseT@VCWindow@ATL@@V?$CWinTraits@$0FGAAAAAA@$0A@@2@@ATL@@UAEP6GJPAUHWND__@@IIJ@ZXZ 0049a570 f i FlashPlayer.obj
 0001:00099580       ?DestroyWindow@?$CWindowImplBaseT@VCWindow@ATL@@V?$CWinTraits@$0FGAAAAAA@$0A@@2@@ATL@@QAEHXZ 0049a580 f i FlashPlayer.obj
 0001:000995a0       ?DefWindowProcA@?$CWindowImplBaseT@VCWindow@ATL@@V?$CWinTraits@$0FGAAAAAA@$0A@@2@@ATL@@QAEJXZ 0049a5a0 f i FlashPlayer.obj
 0001:000995f0       ?DefWindowProcA@?$CWindowImplBaseT@VCWindow@ATL@@V?$CWinTraits@$0FGAAAAAA@$0A@@2@@ATL@@QAEJIIJ@Z 0049a5f0 f i FlashPlayer.obj
 0001:00099620       ?SetSite@?$IObjectWithSiteImpl@VCAxHostWindow@ATL@@@ATL@@UAGJPAUIUnknown@@@Z 0049a620 f i FlashPlayer.obj
 0001:00099660       ?GetSite@?$IObjectWithSiteImpl@VCAxHostWindow@ATL@@@ATL@@UAGJABU_GUID@@PAPAX@Z 0049a660 f i FlashPlayer.obj
 0001:000996e0       ?GetTypeInfoCount@?$IDispatchImpl@UIAxWinAmbientDispatchEx@@$1?_GUID_b2d0778b_ac99_4c58_a5c8_e7724e5316b5@@3U__s_GUID@@B$1?m_libid@CAtlModule@ATL@@2U_GUID@@A$0PPPP@$0PPPP@VCComTypeInfoHolder@ATL@@@ATL@@UAGJPAI@Z 0049a6e0 f i FlashPlayer.obj
 0001:00099700       ?GetTypeInfo@?$IDispatchImpl@UIAxWinAmbientDispatchEx@@$1?_GUID_b2d0778b_ac99_4c58_a5c8_e7724e5316b5@@3U__s_GUID@@B$1?m_libid@CAtlModule@ATL@@2U_GUID@@A$0PPPP@$0PPPP@VCComTypeInfoHolder@ATL@@@ATL@@UAGJIKPAPAUITypeInfo@@@Z 0049a700 f i FlashPlayer.obj
 0001:00099720       ?GetTypeInfo@CComTypeInfoHolder@ATL@@QAEJIKPAPAUITypeInfo@@@Z 0049a720 f i FlashPlayer.obj
 0001:00099740       ?GetTI@CComTypeInfoHolder@ATL@@QAEJKPAPAUITypeInfo@@@Z 0049a740 f i FlashPlayer.obj
 0001:000997b0       ?GetTI@CComTypeInfoHolder@ATL@@QAEJK@Z 0049a7b0 f i FlashPlayer.obj
 0001:00099be0       ?_AtlVerifyStackAvailable@_ATL_SAFE_ALLOCA_IMPL@ATL@@YA_NK@Z 0049abe0 f i FlashPlayer.obj
 0001:00099c80       ?Cleanup@CComTypeInfoHolder@ATL@@SGXK@Z 0049ac80 f i FlashPlayer.obj
 0001:00099d00       ?LoadNameCache@CComTypeInfoHolder@ATL@@QAEJPAUITypeInfo@@@Z 0049ad00 f i FlashPlayer.obj
 0001:00099f30       ?Attach@CComBSTR@ATL@@QAEXPAG@Z 0049af30 f i FlashPlayer.obj
 0001:00099f60       ??0stringdispid@CComTypeInfoHolder@ATL@@QAE@XZ 0049af60 f i FlashPlayer.obj
 0001:00099f90       ?AddTermFunc@CAtlModule@ATL@@QAEJP6GXK@ZK@Z 0049af90 f i FlashPlayer.obj
 0001:00099fd0       ?Allocate@?$CAtlSafeAllocBufferManager@VCCRTAllocator@ATL@@@_ATL_SAFE_ALLOCA_IMPL@ATL@@QAEPAXK@Z 0049afd0 f i FlashPlayer.obj
 0001:0009a020       ?Allocate@CCRTAllocator@ATL@@SAPAXI@Z 0049b020 f i FlashPlayer.obj
 0001:0009a040       ??1?$CAtlSafeAllocBufferManager@VCCRTAllocator@ATL@@@_ATL_SAFE_ALLOCA_IMPL@ATL@@QAE@XZ 0049b040 f i FlashPlayer.obj
 0001:0009a080       ?Free@CCRTAllocator@ATL@@SAXPAX@Z 0049b080 f i FlashPlayer.obj
 0001:0009a0a0       ?AtlModuleAddTermFunc@ATL@@YGJPAU_ATL_MODULE70@1@P6GXK@ZK@Z 0049b0a0 f i FlashPlayer.obj
 0001:0009a1b0       ??0?$CComPtr@UITypeInfo@@@ATL@@QAE@ABV01@@Z 0049b1b0 f i FlashPlayer.obj
 0001:0009a1d0       ?GetIDsOfNames@?$IDispatchImpl@UIAxWinAmbientDispatchEx@@$1?_GUID_b2d0778b_ac99_4c58_a5c8_e7724e5316b5@@3U__s_GUID@@B$1?m_libid@CAtlModule@ATL@@2U_GUID@@A$0PPPP@$0PPPP@VCComTypeInfoHolder@ATL@@@ATL@@UAGJABU_GUID@@PAPAGIKPAJ@Z 0049b1d0 f i FlashPlayer.obj
 0001:0009a200       ?GetIDsOfNames@CComTypeInfoHolder@ATL@@QAEJABU_GUID@@PAPAGIKPAJ@Z 0049b200 f i FlashPlayer.obj
 0001:0009a310       ?EnsureTI@CComTypeInfoHolder@ATL@@QAEJK@Z 0049b310 f i FlashPlayer.obj
 0001:0009a350       ?Invoke@?$IDispatchImpl@UIAxWinAmbientDispatchEx@@$1?_GUID_b2d0778b_ac99_4c58_a5c8_e7724e5316b5@@3U__s_GUID@@B$1?m_libid@CAtlModule@ATL@@2U_GUID@@A$0PPPP@$0PPPP@VCComTypeInfoHolder@ATL@@@ATL@@UAGJJABU_GUID@@KGPAUtagDISPPARAMS@@PAUtagVARIANT@@PAUtagEXCEPINFO@@PAI@Z 0049b350 f i FlashPlayer.obj
 0001:0009a390       ?Invoke@CComTypeInfoHolder@ATL@@QAEJPAUIDispatch@@JABU_GUID@@KGPAUtagDISPPARAMS@@PAUtagVARIANT@@PAUtagEXCEPINFO@@PAI@Z 0049b390 f i FlashPlayer.obj
 0001:0009a3f0       ??0?$CComPtr@UIServiceProvider@@@ATL@@QAE@XZ 0049b3f0 f i FlashPlayer.obj
 0001:0009a3f0       ??0?$CComPtr@UIConnectionPoint@@@ATL@@QAE@XZ 0049b3f0 f i FlashPlayer.obj
 0001:0009a3f0       ??0?$CComPtr@UIObjectWithSite@@@ATL@@QAE@XZ 0049b3f0 f i FlashPlayer.obj
 0001:0009a3f0       ??0?$CComPtr@UIWebBrowser2@@@ATL@@QAE@XZ 0049b3f0 f i FlashPlayer.obj
 0001:0009a3f0       ??0?$CComPtr@UIOleInPlaceUIWindow@@@ATL@@QAE@XZ 0049b3f0 f i FlashPlayer.obj
 0001:0009a3f0       ??0?$CComPtr@UIUnknown@@@ATL@@QAE@XZ 0049b3f0 f i FlashPlayer.obj
 0001:0009a3f0       ??0?$CComPtr@UIFontDisp@@@ATL@@QAE@XZ 0049b3f0 f i FlashPlayer.obj
 0001:0009a3f0       ??0?$CComPtr@UIOleClientSite@@@ATL@@QAE@XZ 0049b3f0 f i FlashPlayer.obj
 0001:0009a3f0       ??0?$CComPtr@UIDocHostUIHandlerDispatch@@@ATL@@QAE@XZ 0049b3f0 f i FlashPlayer.obj
 0001:0009a3f0       ??0?$CComPtr@UIAxWinHostWindow@@@ATL@@QAE@XZ 0049b3f0 f i FlashPlayer.obj
 0001:0009a3f0       ??0?$CComPtr@UIPersistStream@@@ATL@@QAE@XZ 0049b3f0 f i FlashPlayer.obj
 0001:0009a3f0       ??0?$CComPtr@UITypeInfo@@@ATL@@QAE@XZ 0049b3f0 f i FlashPlayer.obj
 0001:0009a3f0       ??0?$CComPtr@UIOleInPlaceObjectWindowless@@@ATL@@QAE@XZ 0049b3f0 f i FlashPlayer.obj
 0001:0009a3f0       ??0?$CComPtr@UITypeInfo2@@@ATL@@QAE@XZ 0049b3f0 f i FlashPlayer.obj
 0001:0009a3f0       ??0?$CComPtr@UIOleInPlaceActiveObject@@@ATL@@QAE@XZ 0049b3f0 f i FlashPlayer.obj
 0001:0009a3f0       ??0?$CComPtr@UIAdviseSink@@@ATL@@QAE@XZ 0049b3f0 f i FlashPlayer.obj
 0001:0009a3f0       ??0?$CComPtr@UIAxWinHostWindowLic@@@ATL@@QAE@XZ 0049b3f0 f i FlashPlayer.obj
 0001:0009a3f0       ??0?$CComPtr@UIOleControl@@@ATL@@QAE@XZ 0049b3f0 f i FlashPlayer.obj
 0001:0009a3f0       ??0?$CComPtr@UIOleInPlaceFrame@@@ATL@@QAE@XZ 0049b3f0 f i FlashPlayer.obj
 0001:0009a3f0       ??0?$CComPtr@UIViewObjectEx@@@ATL@@QAE@XZ 0049b3f0 f i FlashPlayer.obj
 0001:0009a3f0       ??0?$CComPtr@UIStream@@@ATL@@QAE@XZ 0049b3f0 f i FlashPlayer.obj
 0001:0009a3f0       ??0?$CComObjectRootEx@VCComSingleThreadModel@ATL@@@ATL@@QAE@XZ 0049b3f0 f i FlashPlayer.obj
 0001:0009a3f0       ??0?$CComPtr@UIOleObject@@@ATL@@QAE@XZ 0049b3f0 f i FlashPlayer.obj
 0001:0009a3f0       ??0?$CComPtr@UIDispatch@@@ATL@@QAE@XZ 0049b3f0 f i FlashPlayer.obj
 0001:0009a3f0       ??0?$CComPtr@UIPersistStreamInit@@@ATL@@QAE@XZ 0049b3f0 f i FlashPlayer.obj
 0001:0009a3f0       ??0?$CComPtr@UIClassFactory2@@@ATL@@QAE@XZ 0049b3f0 f i FlashPlayer.obj
 0001:0009a3f0       ??0?$CComPtr@UIConnectionPointContainer@@@ATL@@QAE@XZ 0049b3f0 f i FlashPlayer.obj
 0001:0009a410       ??7?$CComPtrBase@UIOleInPlaceFrame@@@ATL@@QBE_NXZ 0049b410 f i FlashPlayer.obj
 0001:0009a410       ??7?$CComPtrBase@UIOleInPlaceUIWindow@@@ATL@@QBE_NXZ 0049b410 f i FlashPlayer.obj
 0001:0009a430       ?CopyTo@?$CComPtrBase@UIDispatch@@@ATL@@QAEJPAPAUIDispatch@@@Z 0049b430 f i FlashPlayer.obj
 0001:0009a430       ?CopyTo@?$CComPtrBase@UIOleInPlaceFrame@@@ATL@@QAEJPAPAUIOleInPlaceFrame@@@Z 0049b430 f i FlashPlayer.obj
 0001:0009a430       ?CopyTo@?$CComPtrBase@UIFontDisp@@@ATL@@QAEJPAPAUIFontDisp@@@Z 0049b430 f i FlashPlayer.obj
 0001:0009a430       ?CopyTo@?$CComPtrBase@UIOleInPlaceUIWindow@@@ATL@@QAEJPAPAUIOleInPlaceUIWindow@@@Z 0049b430 f i FlashPlayer.obj
 0001:0009a470       ??8?$CComPtrBase@UIViewObjectEx@@@ATL@@QBE_NPAUIViewObjectEx@@@Z 0049b470 f i FlashPlayer.obj
 0001:0009a470       ??8?$CComPtrBase@UIUnknown@@@ATL@@QBE_NPAUIUnknown@@@Z 0049b470 f i FlashPlayer.obj
 0001:0009a470       ??8?$CComPtrBase@UIFontDisp@@@ATL@@QBE_NPAUIFontDisp@@@Z 0049b470 f i FlashPlayer.obj
 0001:0009a490       ??4?$CComPtr@UIUnknown@@@ATL@@QAEPAUIUnknown@@PAU2@@Z 0049b490 f i FlashPlayer.obj
 0001:0009a490       ??4?$CComPtr@UIDispatch@@@ATL@@QAEPAUIDispatch@@PAU2@@Z 0049b490 f i FlashPlayer.obj
 0001:0009a490       ??4?$CComPtr@UIOleInPlaceActiveObject@@@ATL@@QAEPAUIOleInPlaceActiveObject@@PAU2@@Z 0049b490 f i FlashPlayer.obj
 0001:0009a490       ??4?$CComPtr@UIFontDisp@@@ATL@@QAEPAUIFontDisp@@PAU2@@Z 0049b490 f i FlashPlayer.obj
 0001:0009a490       ??4?$CComPtr@UIDocHostUIHandlerDispatch@@@ATL@@QAEPAUIDocHostUIHandlerDispatch@@PAU2@@Z 0049b490 f i FlashPlayer.obj
 0001:0009a4b0       ??ICComBSTR@ATL@@QAEPAPAGXZ 0049b4b0 f i FlashPlayer.obj
 0001:0009a4b0       ?GetCodeAddress@_stdcallthunk@ATL@@QAEPAXXZ 0049b4b0 f i FlashPlayer.obj
 0001:0009a4b0       ??I?$CComPtrBase@UIFontDisp@@@ATL@@QAEPAPAUIFontDisp@@XZ 0049b4b0 f i FlashPlayer.obj
 0001:0009a4b0       ??I?$CComPtrBase@UIOleInPlaceUIWindow@@@ATL@@QAEPAPAUIOleInPlaceUIWindow@@XZ 0049b4b0 f i FlashPlayer.obj
 0001:0009a4b0       ??I?$CComPtrBase@UIOleInPlaceFrame@@@ATL@@QAEPAPAUIOleInPlaceFrame@@XZ 0049b4b0 f i FlashPlayer.obj
 0001:0009a4b0       ??I?$CComPtrBase@UITypeInfo@@@ATL@@QAEPAPAUITypeInfo@@XZ 0049b4b0 f i FlashPlayer.obj
 0001:0009a4b0       ??I?$CComPtrBase@UIOleClientSite@@@ATL@@QAEPAPAUIOleClientSite@@XZ 0049b4b0 f i FlashPlayer.obj
 0001:0009a4b0       ??I?$CComPtrBase@UITypeInfo2@@@ATL@@QAEPAPAUITypeInfo2@@XZ 0049b4b0 f i FlashPlayer.obj
 0001:0009a4b0       ??I?$CComPtrBase@UIAxWinHostWindowLic@@@ATL@@QAEPAPAUIAxWinHostWindowLic@@XZ 0049b4b0 f i FlashPlayer.obj
 0001:0009a4b0       ??I?$CComPtrBase@UIOleObject@@@ATL@@QAEPAPAUIOleObject@@XZ 0049b4b0 f i FlashPlayer.obj
 0001:0009a4b0       ??0IUnknown@@QAE@XZ        0049b4b0 f i FlashPlayer.obj
 0001:0009a4b0       ??0theGraphicsManagerImpl@@QAE@XZ 0049b4b0 f i theGraphicsManager.obj
 0001:0009a4b0       ??I?$CComPtrBase@UIViewObjectEx@@@ATL@@QAEPAPAUIViewObjectEx@@XZ 0049b4b0 f i FlashPlayer.obj
 0001:0009a4b0       ??I?$CComPtrBase@UIStream@@@ATL@@QAEPAPAUIStream@@XZ 0049b4b0 f i FlashPlayer.obj
 0001:0009a4b0       ??I?$CComPtrBase@UIClassFactory2@@@ATL@@QAEPAPAUIClassFactory2@@XZ 0049b4b0 f i FlashPlayer.obj
 0001:0009a4b0       ??I?$CComPtrBase@UIServiceProvider@@@ATL@@QAEPAPAUIServiceProvider@@XZ 0049b4b0 f i FlashPlayer.obj
 0001:0009a4b0       ??I?$CComPtrBase@UIAxWinHostWindow@@@ATL@@QAEPAPAUIAxWinHostWindow@@XZ 0049b4b0 f i FlashPlayer.obj
 0001:0009a4b0       ??I?$CComPtrBase@UIUnknown@@@ATL@@QAEPAPAUIUnknown@@XZ 0049b4b0 f i FlashPlayer.obj
 0001:0009a4b0       ??I?$CComPtrBase@UIPersistStreamInit@@@ATL@@QAEPAPAUIPersistStreamInit@@XZ 0049b4b0 f i FlashPlayer.obj
 0001:0009a4b0       ??0CMessageMap@ATL@@QAE@XZ 0049b4b0 f i FlashPlayer.obj
 0001:0009a4b0       ??I?$CComPtrBase@UIConnectionPointContainer@@@ATL@@QAEPAPAUIConnectionPointContainer@@XZ 0049b4b0 f i FlashPlayer.obj
 0001:0009a4b0       ??I?$CComPtrBase@UIWebBrowser2@@@ATL@@QAEPAPAUIWebBrowser2@@XZ 0049b4b0 f i FlashPlayer.obj
 0001:0009a4b0       ??I?$CComPtrBase@UIConnectionPoint@@@ATL@@QAEPAPAUIConnectionPoint@@XZ 0049b4b0 f i FlashPlayer.obj
 0001:0009a4b0       ??I?$CComPtrBase@UIObjectWithSite@@@ATL@@QAEPAPAUIObjectWithSite@@XZ 0049b4b0 f i FlashPlayer.obj
 0001:0009a4b0       ??I?$CComPtrBase@UIOleInPlaceObjectWindowless@@@ATL@@QAEPAPAUIOleInPlaceObjectWindowless@@XZ 0049b4b0 f i FlashPlayer.obj
 0001:0009a4c0       ??0?$CComQIPtr@UIOleInPlaceActiveObject@@$1?_GUID_00000117_0000_0000_c000_000000000046@@3U__s_GUID@@B@ATL@@QAE@PAUIUnknown@@@Z 0049b4c0 f i FlashPlayer.obj
 0001:0009a500       ??0?$CComQIPtr@UIOleControl@@$1?_GUID_b196b288_bab4_101a_b69c_00aa00341d07@@3U__s_GUID@@B@ATL@@QAE@PAUIUnknown@@@Z 0049b500 f i FlashPlayer.obj
 0001:0009a540       ??0?$CComObject@V?$CComEnum@UIEnumUnknown@@$1?_GUID_00000100_0000_0000_c000_000000000046@@3U__s_GUID@@BPAUIUnknown@@V?$_CopyInterface@UIUnknown@@@ATL@@VCComMultiThreadModel@6@@ATL@@@ATL@@QAE@PAX@Z 0049b540 f i FlashPlayer.obj
 0001:0009a580       ?AddRef@?$CComObject@V?$CComEnum@UIEnumUnknown@@$1?_GUID_00000100_0000_0000_c000_000000000046@@3U__s_GUID@@BPAUIUnknown@@V?$_CopyInterface@UIUnknown@@@ATL@@VCComMultiThreadModel@6@@ATL@@@ATL@@UAGKXZ 0049b580 f i FlashPlayer.obj
 0001:0009a5a0       ?Release@?$CComObject@V?$CComEnum@UIEnumUnknown@@$1?_GUID_00000100_0000_0000_c000_000000000046@@3U__s_GUID@@BPAUIUnknown@@V?$_CopyInterface@UIUnknown@@@ATL@@VCComMultiThreadModel@6@@ATL@@@ATL@@UAGKXZ 0049b5a0 f i FlashPlayer.obj
 0001:0009a5f0       ?QueryInterface@?$CComObject@V?$CComEnum@UIEnumUnknown@@$1?_GUID_00000100_0000_0000_c000_000000000046@@3U__s_GUID@@BPAUIUnknown@@V?$_CopyInterface@UIUnknown@@@ATL@@VCComMultiThreadModel@6@@ATL@@@ATL@@UAGJABU_GUID@@PAPAX@Z 0049b5f0 f i FlashPlayer.obj
 0001:0009a610       ?Reset@?$CComEnumImpl@UIEnumUnknown@@$1?_GUID_00000100_0000_0000_c000_000000000046@@3U__s_GUID@@BPAUIUnknown@@V?$_CopyInterface@UIUnknown@@@ATL@@@ATL@@UAGJXZ 0049b610 f i FlashPlayer.obj
 0001:0009a630       ??0?$CComQIPtr@UIOleClientSite@@$1?_GUID_00000118_0000_0000_c000_000000000046@@3U__s_GUID@@B@ATL@@QAE@PAUIUnknown@@@Z 0049b630 f i FlashPlayer.obj
 0001:0009a670       ??0?$CComQIPtr@UIPersistStreamInit@@$1?_GUID_7fd52380_4e07_101b_ae2d_08002b2ec713@@3U__s_GUID@@B@ATL@@QAE@PAUIUnknown@@@Z 0049b670 f i FlashPlayer.obj
 0001:0009a6b0       ??0?$CComQIPtr@UIPersistStream@@$1?_GUID_00000109_0000_0000_c000_000000000046@@3U__s_GUID@@B@ATL@@QAE@PAUIUnknown@@@Z 0049b6b0 f i FlashPlayer.obj
 0001:0009a6f0       ??0?$CComQIPtr@UIAdviseSink@@$1?_GUID_0000010f_0000_0000_c000_000000000046@@3U__s_GUID@@B@ATL@@QAE@PAUIUnknown@@@Z 0049b6f0 f i FlashPlayer.obj
 0001:0009a730       ??_E?$CComObject@V?$CComEnum@UIEnumUnknown@@$1?_GUID_00000100_0000_0000_c000_000000000046@@3U__s_GUID@@BPAUIUnknown@@V?$_CopyInterface@UIUnknown@@@ATL@@VCComMultiThreadModel@6@@ATL@@@ATL@@UAEPAXI@Z 0049b730 f i FlashPlayer.obj
 0001:0009a730       ??_G?$CComObject@V?$CComEnum@UIEnumUnknown@@$1?_GUID_00000100_0000_0000_c000_000000000046@@3U__s_GUID@@BPAUIUnknown@@V?$_CopyInterface@UIUnknown@@@ATL@@VCComMultiThreadModel@6@@ATL@@@ATL@@UAEPAXI@Z 0049b730 f i FlashPlayer.obj
 0001:0009a760       ??1?$CComObject@V?$CComEnum@UIEnumUnknown@@$1?_GUID_00000100_0000_0000_c000_000000000046@@3U__s_GUID@@BPAUIUnknown@@V?$_CopyInterface@UIUnknown@@@ATL@@VCComMultiThreadModel@6@@ATL@@@ATL@@UAE@XZ 0049b760 f i FlashPlayer.obj
 0001:0009a7b0       ??0?$CComEnum@UIEnumUnknown@@$1?_GUID_00000100_0000_0000_c000_000000000046@@3U__s_GUID@@BPAUIUnknown@@V?$_CopyInterface@UIUnknown@@@ATL@@VCComMultiThreadModel@6@@ATL@@QAE@XZ 0049b7b0 f i FlashPlayer.obj
 0001:0009a800       ??0?$CComObjectRootEx@VCComMultiThreadModel@ATL@@@ATL@@QAE@XZ 0049b800 f i FlashPlayer.obj
 0001:0009a830       ??0CComAutoCriticalSection@ATL@@QAE@XZ 0049b830 f i FlashPlayer.obj
 0001:0009a870       ??0CComCriticalSection@ATL@@QAE@XZ 0049b870 f i FlashPlayer.obj
 0001:0009a890       ?Init@CComCriticalSection@ATL@@QAEJXZ 0049b890 f i FlashPlayer.obj
 0001:0009a930       ??1?$CComEnum@UIEnumUnknown@@$1?_GUID_00000100_0000_0000_c000_000000000046@@3U__s_GUID@@BPAUIUnknown@@V?$_CopyInterface@UIUnknown@@@ATL@@VCComMultiThreadModel@6@@ATL@@UAE@XZ 0049b930 f i FlashPlayer.obj
 0001:0009a970       ??1?$CComObjectRootEx@VCComMultiThreadModel@ATL@@@ATL@@QAE@XZ 0049b970 f i FlashPlayer.obj
 0001:0009a990       ??1CComAutoCriticalSection@ATL@@QAE@XZ 0049b990 f i FlashPlayer.obj
 0001:0009a9b0       ?Term@CComCriticalSection@ATL@@QAEJXZ 0049b9b0 f i FlashPlayer.obj
 0001:0009a9d0       ??0?$CComPtrBase@UIUnknown@@@ATL@@IAE@PAUIUnknown@@@Z 0049b9d0 f i FlashPlayer.obj
 0001:0009a9d0       ??0?$CComPtrBase@UITypeInfo@@@ATL@@IAE@PAUITypeInfo@@@Z 0049b9d0 f i FlashPlayer.obj
 0001:0009aa00       ??0?$CWindowImplRoot@VCWindow@ATL@@@ATL@@QAE@XZ 0049ba00 f i FlashPlayer.obj
 0001:0009aa50       ?InternalAddRef@?$CComObjectRootEx@VCComMultiThreadModel@ATL@@@ATL@@QAEKXZ 0049ba50 f i FlashPlayer.obj
 0001:0009aa70       ?Increment@CComMultiThreadModel@ATL@@SGKPAJ@Z 0049ba70 f i FlashPlayer.obj
 0001:0009aa90       ?InternalRelease@?$CComObjectRootEx@VCComMultiThreadModel@ATL@@@ATL@@QAEKXZ 0049ba90 f i FlashPlayer.obj
 0001:0009aab0       ?Decrement@CComMultiThreadModel@ATL@@SGKPAJ@Z 0049bab0 f i FlashPlayer.obj
 0001:0009aad0       ??0?$CAtlSafeAllocBufferManager@VCCRTAllocator@ATL@@@_ATL_SAFE_ALLOCA_IMPL@ATL@@QAE@XZ 0049bad0 f i FlashPlayer.obj
 0001:0009aad0       ??0?$CComPtrBase@UIPersistStreamInit@@@ATL@@IAE@XZ 0049bad0 f i FlashPlayer.obj
 0001:0009aad0       ??0?$CComPtrBase@UIDocHostUIHandlerDispatch@@@ATL@@IAE@XZ 0049bad0 f i FlashPlayer.obj
 0001:0009aad0       ??0?$CComPtrBase@UIWebBrowser2@@@ATL@@IAE@XZ 0049bad0 f i FlashPlayer.obj
 0001:0009aad0       ??0?$CComPtrBase@UIOleInPlaceActiveObject@@@ATL@@IAE@XZ 0049bad0 f i FlashPlayer.obj
 0001:0009aad0       ??0?$CComPtrBase@UIObjectWithSite@@@ATL@@IAE@XZ 0049bad0 f i FlashPlayer.obj
 0001:0009aad0       ??0CDynamicStdCallThunk@ATL@@QAE@XZ 0049bad0 f i FlashPlayer.obj
 0001:0009aad0       ??0?$CComPtrBase@UIOleControl@@@ATL@@IAE@XZ 0049bad0 f i FlashPlayer.obj
 0001:0009aad0       ??0?$CComPtrBase@UIConnectionPointContainer@@@ATL@@IAE@XZ 0049bad0 f i FlashPlayer.obj
 0001:0009aad0       ??0?$CComPtrBase@UIViewObjectEx@@@ATL@@IAE@XZ 0049bad0 f i FlashPlayer.obj
 0001:0009aad0       ??0?$CComPtrBase@UITypeInfo2@@@ATL@@IAE@XZ 0049bad0 f i FlashPlayer.obj
 0001:0009aad0       ??0?$CComPtrBase@UIDispatch@@@ATL@@IAE@XZ 0049bad0 f i FlashPlayer.obj
 0001:0009aad0       ??0?$CTempBuffer@D$0BAA@VCCRTAllocator@ATL@@@ATL@@QAE@XZ 0049bad0 f i FlashPlayer.obj
 0001:0009aad0       ??0?$CComPtrBase@UIAxWinHostWindowLic@@@ATL@@IAE@XZ 0049bad0 f i FlashPlayer.obj
 0001:0009aad0       ??0?$CComPtrBase@UITypeInfo@@@ATL@@IAE@XZ 0049bad0 f i FlashPlayer.obj
 0001:0009aad0       ??0CComBSTR@ATL@@QAE@XZ    0049bad0 f i FlashPlayer.obj
 0001:0009aad0       ??0?$CComPtrBase@UIConnectionPoint@@@ATL@@IAE@XZ 0049bad0 f i FlashPlayer.obj
 0001:0009aad0       ??0?$CComPtrBase@UIAxWinHostWindow@@@ATL@@IAE@XZ 0049bad0 f i FlashPlayer.obj
 0001:0009aad0       ??0?$CComPtrBase@UIStream@@@ATL@@IAE@XZ 0049bad0 f i FlashPlayer.obj
 0001:0009aad0       ??0?$CComPtrBase@UIAdviseSink@@@ATL@@IAE@XZ 0049bad0 f i FlashPlayer.obj
 0001:0009aad0       ??0?$CComPtrBase@UIOleObject@@@ATL@@IAE@XZ 0049bad0 f i FlashPlayer.obj
 0001:0009aad0       ??0?$CComPtrBase@UIClassFactory2@@@ATL@@IAE@XZ 0049bad0 f i FlashPlayer.obj
 0001:0009aad0       ??0?$CComPtrBase@UIUnknown@@@ATL@@IAE@XZ 0049bad0 f i FlashPlayer.obj
 0001:0009aad0       ??0?$CComPtrBase@UIOleClientSite@@@ATL@@IAE@XZ 0049bad0 f i FlashPlayer.obj
 0001:0009aad0       ??0?$CComPtrBase@UIPersistStream@@@ATL@@IAE@XZ 0049bad0 f i FlashPlayer.obj
 0001:0009aad0       ??0?$CComPtrBase@UIServiceProvider@@@ATL@@IAE@XZ 0049bad0 f i FlashPlayer.obj
 0001:0009aad0       ??0?$CComPtrBase@UIOleInPlaceUIWindow@@@ATL@@IAE@XZ 0049bad0 f i FlashPlayer.obj
 0001:0009aad0       ??0?$CTempBuffer@E$0BAA@VCCRTAllocator@ATL@@@ATL@@QAE@XZ 0049bad0 f i FlashPlayer.obj
 0001:0009aad0       ??0CRegKey@ATL@@QAE@XZ     0049bad0 f i FlashPlayer.obj
 0001:0009aad0       ??0?$CComPtrBase@UIOleInPlaceFrame@@@ATL@@IAE@XZ 0049bad0 f i FlashPlayer.obj
 0001:0009aad0       ??0CComObjectRootBase@ATL@@QAE@XZ 0049bad0 f i FlashPlayer.obj
 0001:0009aad0       ??0?$CTempBuffer@D$0EAA@VCCRTAllocator@ATL@@@ATL@@QAE@XZ 0049bad0 f i FlashPlayer.obj
 0001:0009aad0       ??0?$CComPtrBase@UIOleInPlaceObjectWindowless@@@ATL@@IAE@XZ 0049bad0 f i FlashPlayer.obj
 0001:0009aad0       ??0?$CComPtrBase@UIFontDisp@@@ATL@@IAE@XZ 0049bad0 f i FlashPlayer.obj
 0001:0009aaf0       ?_InternalQueryInterface@?$CComEnum@UIEnumUnknown@@$1?_GUID_00000100_0000_0000_c000_000000000046@@3U__s_GUID@@BPAUIUnknown@@V?$_CopyInterface@UIUnknown@@@ATL@@VCComMultiThreadModel@6@@ATL@@QAEJABU_GUID@@PAPAX@Z 0049baf0 f i FlashPlayer.obj
 0001:0009ab20       ??0?$CComEnumImpl@UIEnumUnknown@@$1?_GUID_00000100_0000_0000_c000_000000000046@@3U__s_GUID@@BPAUIUnknown@@V?$_CopyInterface@UIUnknown@@@ATL@@@ATL@@QAE@XZ 0049bb20 f i FlashPlayer.obj
 0001:0009ab70       ?GetData@CAtlSafeAllocBufferNode@?$CAtlSafeAllocBufferManager@VCCRTAllocator@ATL@@@_ATL_SAFE_ALLOCA_IMPL@ATL@@QAEPAXXZ 0049bb70 f i FlashPlayer.obj
 0001:0009ab90       ?AddRef@?$CComContainedObject@VCAxHostWindow@ATL@@@ATL@@UAGKXZ 0049bb90 f i FlashPlayer.obj
 0001:0009abb0       ?OuterAddRef@CComObjectRootBase@ATL@@QAEKXZ 0049bbb0 f i FlashPlayer.obj
 0001:0009abd0       ?Release@?$CComContainedObject@VCAxHostWindow@ATL@@@ATL@@UAGKXZ 0049bbd0 f i FlashPlayer.obj
 0001:0009abf0       ?OuterRelease@CComObjectRootBase@ATL@@QAEKXZ 0049bbf0 f i FlashPlayer.obj
 0001:0009ac10       ?QueryInterface@?$CComContainedObject@VCAxHostWindow@ATL@@@ATL@@UAGJABU_GUID@@PAPAX@Z 0049bc10 f i FlashPlayer.obj
 0001:0009ac30       ?OuterQueryInterface@CComObjectRootBase@ATL@@QAEJABU_GUID@@PAPAX@Z 0049bc30 f i FlashPlayer.obj
 0001:0009ac60       ?GetControllingUnknown@?$CComContainedObject@VCAxHostWindow@ATL@@@ATL@@UAEPAUIUnknown@@XZ 0049bc60 f i FlashPlayer.obj
 0001:0009ac80       ??0CWndProcThunk@ATL@@QAE@XZ 0049bc80 f i FlashPlayer.obj
 0001:0009aca0       ?_GetEntries@?$CComEnum@UIEnumUnknown@@$1?_GUID_00000100_0000_0000_c000_000000000046@@3U__s_GUID@@BPAUIUnknown@@V?$_CopyInterface@UIUnknown@@@ATL@@VCComMultiThreadModel@6@@ATL@@SGPBU_ATL_INTMAP_ENTRY@2@XZ 0049bca0 f i FlashPlayer.obj
 0001:0009acb0       ??_E?$CComContainedObject@VCAxHostWindow@ATL@@@ATL@@UAEPAXI@Z 0049bcb0 f i FlashPlayer.obj
 0001:0009acb0       ??_G?$CComContainedObject@VCAxHostWindow@ATL@@@ATL@@UAEPAXI@Z 0049bcb0 f i FlashPlayer.obj
 0001:0009ace0       ??0?$CComCritSecLock@VCComCriticalSection@ATL@@@ATL@@QAE@AAVCComCriticalSection@1@_N@Z 0049bce0 f i FlashPlayer.obj
 0001:0009ad30       ??1?$CComCritSecLock@VCComCriticalSection@ATL@@@ATL@@QAE@XZ 0049bd30 f i FlashPlayer.obj
 0001:0009ad50       ?Lock@?$CComCritSecLock@VCComCriticalSection@ATL@@@ATL@@QAEJXZ 0049bd50 f i FlashPlayer.obj
 0001:0009ad80       ?Lock@CComCriticalSection@ATL@@QAEJXZ 0049bd80 f i FlashPlayer.obj
 0001:0009ada0       ??$QueryInterface@UITypeInfo2@@@IUnknown@@QAGJPAPAUITypeInfo2@@@Z 0049bda0 f i FlashPlayer.obj
 0001:0009adc0       ??$?4UITypeInfo2@@@?$CComPtr@UITypeInfo@@@ATL@@QAEPAUITypeInfo@@ABV?$CComPtr@UITypeInfo2@@@1@@Z 0049bdc0 f i FlashPlayer.obj
 0001:0009adf0       ?AtlComQIPtrAssign@ATL@@YGPAUIUnknown@@PAPAU2@PAU2@ABU_GUID@@@Z 0049bdf0 f i FlashPlayer.obj
 0001:0009ae50       ?WindowProc@?$CWindowImplBaseT@VCWindow@ATL@@V?$CWinTraits@$0FGAAAAAA@$0A@@2@@ATL@@SGJPAUHWND__@@IIJ@Z 0049be50 f i FlashPlayer.obj
 0001:0009afb0       ??0_ATL_MSG@ATL@@QAE@PAUHWND__@@IIJH@Z 0049bfb0 f i FlashPlayer.obj
 0001:0009b020       ?SubclassWindow@?$CWindowImplBaseT@VCWindow@ATL@@V?$CWinTraits@$0FGAAAAAA@$0A@@2@@ATL@@QAEHPAUHWND__@@@Z 0049c020 f i FlashPlayer.obj
 0001:0009b090       ?Init@CWndProcThunk@ATL@@QAEXP6GJPAUHWND__@@IIJ@ZPAX@Z 0049c090 f i FlashPlayer.obj
 0001:0009b0b0       ?GetWNDPROC@CWndProcThunk@ATL@@QAEP6GJPAUHWND__@@IIJ@ZXZ 0049c0b0 f i FlashPlayer.obj
 0001:0009b0d0       ?Init@CDynamicStdCallThunk@ATL@@QAEXKPAX@Z 0049c0d0 f i FlashPlayer.obj
 0001:0009b110       ?Init@_stdcallthunk@ATL@@QAEXKPAX@Z 0049c110 f i FlashPlayer.obj
 0001:0009b160       ?GetCodeAddress@CDynamicStdCallThunk@ATL@@QAEPAXXZ 0049c160 f i FlashPlayer.obj
 0001:0009b180       ?UnsubclassWindow@?$CWindowImplBaseT@VCWindow@ATL@@V?$CWinTraits@$0FGAAAAAA@$0A@@2@@ATL@@QAEPAUHWND__@@H@Z 0049c180 f i FlashPlayer.obj
 0001:0009b210       ?CreateInstance@?$CComObject@VCAxFrameWindow@ATL@@@ATL@@SGJPAPAV12@@Z 0049c210 f i FlashPlayer.obj
 0001:0009b350       ?CreateInstance@?$CComObject@VCAxUIWindow@ATL@@@ATL@@SGJPAPAV12@@Z 0049c350 f i FlashPlayer.obj
 0001:0009b490       ??$QueryInterface@UIDispatch@@@?$CComPtrBase@UIOleObject@@@ATL@@QBEJPAPAUIDispatch@@@Z 0049c490 f i FlashPlayer.obj
 0001:0009b4c0       ??1?$CComEnumImpl@UIEnumUnknown@@$1?_GUID_00000100_0000_0000_c000_000000000046@@3U__s_GUID@@BPAUIUnknown@@V?$_CopyInterface@UIUnknown@@@ATL@@@ATL@@UAE@XZ 0049c4c0 f i FlashPlayer.obj
 0001:0009b560       ?Next@?$CComEnumImpl@UIEnumUnknown@@$1?_GUID_00000100_0000_0000_c000_000000000046@@3U__s_GUID@@BPAUIUnknown@@V?$_CopyInterface@UIUnknown@@@ATL@@@ATL@@UAGJKPAPAUIUnknown@@PAK@Z 0049c560 f i FlashPlayer.obj
 0001:0009b6b0       ?Skip@?$CComEnumImpl@UIEnumUnknown@@$1?_GUID_00000100_0000_0000_c000_000000000046@@3U__s_GUID@@BPAUIUnknown@@V?$_CopyInterface@UIUnknown@@@ATL@@@ATL@@UAGJK@Z 0049c6b0 f i FlashPlayer.obj
 0001:0009b720       ?Clone@?$CComEnumImpl@UIEnumUnknown@@$1?_GUID_00000100_0000_0000_c000_000000000046@@3U__s_GUID@@BPAUIUnknown@@V?$_CopyInterface@UIUnknown@@@ATL@@@ATL@@UAGJPAPAUIEnumUnknown@@@Z 0049c720 f i FlashPlayer.obj
 0001:0009b870       ?Init@?$CComEnumImpl@UIEnumUnknown@@$1?_GUID_00000100_0000_0000_c000_000000000046@@3U__s_GUID@@BPAUIUnknown@@V?$_CopyInterface@UIUnknown@@@ATL@@@ATL@@QAEJPAPAUIUnknown@@0PAU3@W4CComEnumFlags@2@@Z 0049c870 f i FlashPlayer.obj
 0001:0009ba30       ??$QueryInterface@UIAxWinHostWindow@@@IUnknown@@QAGJPAPAUIAxWinHostWindow@@@Z 0049ca30 f i FlashPlayer.obj
 0001:0009ba50       ??0?$CComObject@VCAxFrameWindow@ATL@@@ATL@@QAE@PAX@Z 0049ca50 f i FlashPlayer.obj
 0001:0009ba90       ??0CAxFrameWindow@ATL@@QAE@XZ 0049ca90 f i FlashPlayer.obj
 0001:0009bb00       ?ProcessWindowMessage@CAxUIWindow@ATL@@UAEHPAUHWND__@@IIJAAJK@Z 0049cb00 f i FlashPlayer.obj
 0001:0009bb00       ?ProcessWindowMessage@CAxFrameWindow@ATL@@UAEHPAUHWND__@@IIJAAJK@Z 0049cb00 f i FlashPlayer.obj
 0001:0009bb10       ?GetWindow@CAxFrameWindow@ATL@@UAGJPAPAUHWND__@@@Z 0049cb10 f i FlashPlayer.obj
 0001:0009bb70       ?SetActiveObject@CAxUIWindow@ATL@@UAGJPAUIOleInPlaceActiveObject@@PBG@Z 0049cb70 f i FlashPlayer.obj
 0001:0009bb70       ?SetActiveObject@CAxFrameWindow@ATL@@UAGJPAUIOleInPlaceActiveObject@@PBG@Z 0049cb70 f i FlashPlayer.obj
 0001:0009bb90       ?InsertMenus@CAxFrameWindow@ATL@@UAGJPAUHMENU__@@PAUtagOleMenuGroupWidths@@@Z 0049cb90 f i FlashPlayer.obj
 0001:0009bba0       ?SetMenu@CAxFrameWindow@ATL@@UAGJPAUHMENU__@@PAXPAUHWND__@@@Z 0049cba0 f i FlashPlayer.obj
 0001:0009bbb0       ?TranslateAcceleratorA@CAxFrameWindow@ATL@@UAGJPAUtagMSG@@G@Z 0049cbb0 f i FlashPlayer.obj
 0001:0009bbb0       ?TranslateAcceleratorA@CAxHostWindow@ATL@@UAGJPAUtagMSG@@K@Z 0049cbb0 f i FlashPlayer.obj
 0001:0009bbc0       ??0IOleInPlaceFrame@@QAE@XZ 0049cbc0 f i FlashPlayer.obj
 0001:0009bbc0       ??0IAxWinAmbientDispatchEx@@QAE@XZ 0049cbc0 f i FlashPlayer.obj
 0001:0009bbc0       ??0IOleInPlaceSiteEx@@QAE@XZ 0049cbc0 f i FlashPlayer.obj
 0001:0009bbe0       ??0IAxWinAmbientDispatch@@QAE@XZ 0049cbe0 f i FlashPlayer.obj
 0001:0009bbe0       ??0IOleInPlaceUIWindow@@QAE@XZ 0049cbe0 f i FlashPlayer.obj
 0001:0009bbe0       ??0IAxWinHostWindowLic@@QAE@XZ 0049cbe0 f i FlashPlayer.obj
 0001:0009bbe0       ??0IOleInPlaceSite@@QAE@XZ 0049cbe0 f i FlashPlayer.obj
 0001:0009bbe0       ??0IOleContainer@@QAE@XZ   0049cbe0 f i FlashPlayer.obj
 0001:0009bc00       ?Create@?$CWindowImpl@VCAxFrameWindow@ATL@@VCWindow@2@V?$CWinTraits@$0FGAAAAAA@$0A@@2@@ATL@@QAEPAUHWND__@@PAU3@V_U_RECT@2@PBDKKV_U_MENUorID@2@PAX@Z 0049cc00 f i FlashPlayer.obj
 0001:0009bca0       ?Register@_ATL_WNDCLASSINFOA@ATL@@QAEGPAP6GJPAUHWND__@@IIJ@Z@Z 0049cca0 f i FlashPlayer.obj
 0001:0009bcd0       ?AtlWinModuleRegisterWndClassInfoA@ATL@@YGGPAU_ATL_WIN_MODULE70@1@PAU_ATL_BASE_MODULE70@1@PAU_ATL_WNDCLASSINFOA@1@PAP6GJPAUHWND__@@IIJ@Z@Z 0049ccd0 f i FlashPlayer.obj
 0001:0009bd00       ?AddRef@?$CComObject@VCAxFrameWindow@ATL@@@ATL@@UAGKXZ 0049cd00 f i FlashPlayer.obj
 0001:0009bd00       ?AddRef@?$CComObject@VCAxUIWindow@ATL@@@ATL@@UAGKXZ 0049cd00 f i FlashPlayer.obj
 0001:0009bd20       ?Release@?$CComObject@VCAxFrameWindow@ATL@@@ATL@@UAGKXZ 0049cd20 f i FlashPlayer.obj
 0001:0009bd20       ?Release@?$CComObject@VCAxUIWindow@ATL@@@ATL@@UAGKXZ 0049cd20 f i FlashPlayer.obj
 0001:0009bd80       ?QueryInterface@?$CComObject@VCAxFrameWindow@ATL@@@ATL@@UAGJABU_GUID@@PAPAX@Z 0049cd80 f i FlashPlayer.obj
 0001:0009bda0       ?_InternalQueryInterface@CAxFrameWindow@ATL@@QAEJABU_GUID@@PAPAX@Z 0049cda0 f i FlashPlayer.obj
 0001:0009bdd0       ?_GetEntries@CAxFrameWindow@ATL@@SGPBU_ATL_INTMAP_ENTRY@2@XZ 0049cdd0 f i FlashPlayer.obj
 0001:0009bde0       ??_E?$CComObject@VCAxFrameWindow@ATL@@@ATL@@UAEPAXI@Z 0049cde0 f i FlashPlayer.obj
 0001:0009bde0       ??_G?$CComObject@VCAxFrameWindow@ATL@@@ATL@@UAEPAXI@Z 0049cde0 f i FlashPlayer.obj
 0001:0009be10       ??1?$CComObject@VCAxFrameWindow@ATL@@@ATL@@UAE@XZ 0049ce10 f i FlashPlayer.obj
 0001:0009be60       ??1CAxFrameWindow@ATL@@UAE@XZ 0049ce60 f i FlashPlayer.obj
 0001:0009be60       ??1CAxUIWindow@ATL@@UAE@XZ 0049ce60 f i FlashPlayer.obj
 0001:0009bed0       ?GetWndClassInfo@?$CWindowImpl@VCAxFrameWindow@ATL@@VCWindow@2@V?$CWinTraits@$0FGAAAAAA@$0A@@2@@ATL@@SAAAU_ATL_WNDCLASSINFOA@2@XZ 0049ced0 f i FlashPlayer.obj
 0001:0009bee0       ?GetWndStyle@?$CWindowImplBaseT@VCWindow@ATL@@V?$CWinTraits@$0FGAAAAAA@$0A@@2@@ATL@@SAKK@Z 0049cee0 f i FlashPlayer.obj
 0001:0009bf00       ?GetWndExStyle@?$CWindowImplBaseT@VCWindow@ATL@@V?$CWinTraits@$0FGAAAAAA@$0A@@2@@ATL@@SAKK@Z 0049cf00 f i FlashPlayer.obj
 0001:0009bf20       ?GetWndStyle@?$CWinTraits@$0FGAAAAAA@$0A@@ATL@@SAKK@Z 0049cf20 f i FlashPlayer.obj
 0001:0009bf40       ?GetWndExStyle@?$CWinTraits@$0FGAAAAAA@$0A@@ATL@@SAKK@Z 0049cf40 f i FlashPlayer.obj
 0001:0009bf50       ?StartWindowProc@?$CWindowImplBaseT@VCWindow@ATL@@V?$CWinTraits@$0FGAAAAAA@$0A@@2@@ATL@@SGJPAUHWND__@@IIJ@Z 0049cf50 f i FlashPlayer.obj
 0001:0009bfd0       ?ExtractCreateWndData@CAtlWinModule@ATL@@QAEPAXXZ 0049cfd0 f i FlashPlayer.obj
 0001:0009bff0       ?AtlWinModuleExtractCreateWndData@ATL@@YGPAXPAU_ATL_WIN_MODULE70@1@@Z 0049cff0 f i FlashPlayer.obj
 0001:0009c0c0       ?Create@?$CWindowImplBaseT@VCWindow@ATL@@V?$CWinTraits@$0FGAAAAAA@$0A@@2@@ATL@@QAEPAUHWND__@@PAU3@V_U_RECT@2@PBDKKV_U_MENUorID@2@GPAX@Z 0049d0c0 f i FlashPlayer.obj
 0001:0009c170       ?AddCreateWndData@CAtlWinModule@ATL@@QAEXPAU_AtlCreateWndData@2@PAX@Z 0049d170 f i FlashPlayer.obj
 0001:0009c190       ?AtlWinModuleAddCreateWndData@ATL@@YGXPAU_ATL_WIN_MODULE70@1@PAU_AtlCreateWndData@1@PAX@Z 0049d190 f i FlashPlayer.obj
 0001:0009c220       ?_AtlRaiseException@ATL@@YAXKK@Z 0049d220 f i FlashPlayer.obj
 0001:0009c240       ??$AtlModuleRegisterWndClassInfoT@VAtlModuleRegisterWndClassInfoParamA@ATL@@@ATL@@YAGPAU_ATL_BASE_MODULE70@0@PAU_ATL_WIN_MODULE70@0@PAU_ATL_WNDCLASSINFOA@0@PAP6GJPAUHWND__@@IIJ@ZVAtlModuleRegisterWndClassInfoParamA@0@@Z 0049d240 f i FlashPlayer.obj
 0001:0009c4a0       ?GetClassInfoExA@AtlModuleRegisterWndClassInfoParamA@ATL@@SAHPAUHINSTANCE__@@PBDPAUtagWNDCLASSEXA@@@Z 0049d4a0 f i FlashPlayer.obj
 0001:0009c4c0       ?FormatWindowClassName@AtlModuleRegisterWndClassInfoParamA@ATL@@SAXPADPAX@Z 0049d4c0 f i FlashPlayer.obj
 0001:0009c4e0       ?LoadCursorA@AtlModuleRegisterWndClassInfoParamA@ATL@@SAPAUHICON__@@PAUHINSTANCE__@@PBD@Z 0049d4e0 f i FlashPlayer.obj
 0001:0009c500       ?RegisterClassExA@AtlModuleRegisterWndClassInfoParamA@ATL@@SAGPAU_ATL_WIN_MODULE70@2@PBUtagWNDCLASSEXA@@@Z 0049d500 f i FlashPlayer.obj
 0001:0009c520       ?AtlWinModuleRegisterClassExA@ATL@@YGGPAU_ATL_WIN_MODULE70@1@PBUtagWNDCLASSEXA@@@Z 0049d520 f i FlashPlayer.obj
 0001:0009c570       ?Add@?$CSimpleArray@GV?$CSimpleArrayEqualHelper@G@ATL@@@ATL@@QAEHABG@Z 0049d570 f i FlashPlayer.obj
 0001:0009c610       ?InternalSetAtIndex@?$CSimpleArray@GV?$CSimpleArrayEqualHelper@G@ATL@@@ATL@@QAEXHABG@Z 0049d610 f i FlashPlayer.obj
 0001:0009c690       ??0Wrapper@?$CSimpleArray@GV?$CSimpleArrayEqualHelper@G@ATL@@@ATL@@QAE@ABG@Z 0049d690 f i FlashPlayer.obj
 0001:0009c6b0       ??$?2G@Wrapper@?$CSimpleArray@GV?$CSimpleArrayEqualHelper@G@ATL@@@ATL@@SAPAXIPAG@Z 0049d6b0 f i FlashPlayer.obj
 0001:0009c6b0       ??$?2PAD@?$Wrapper@PAD@?$CSimpleMap@PADPAGVCExpansionVectorEqualHelper@ATL@@@ATL@@SAPAXIPAPAD@Z 0049d6b0 f i FlashPlayer.obj
 0001:0009c6b0       ??$?2PAG@?$Wrapper@PAG@?$CSimpleMap@PADPAGVCExpansionVectorEqualHelper@ATL@@@ATL@@SAPAXIPAPAG@Z 0049d6b0 f i FlashPlayer.obj
 0001:0009c6c0       ??0?$CComObject@VCAxUIWindow@ATL@@@ATL@@QAE@PAX@Z 0049d6c0 f i FlashPlayer.obj
 0001:0009c700       ??0CAxUIWindow@ATL@@QAE@XZ 0049d700 f i FlashPlayer.obj
 0001:0009c770       ?GetWindow@CAxUIWindow@ATL@@UAGJPAPAUHWND__@@@Z 0049d770 f i FlashPlayer.obj
 0001:0009c7d0       ?RequestBorderSpace@CAxUIWindow@ATL@@UAGJPBUtagRECT@@@Z 0049d7d0 f i FlashPlayer.obj
 0001:0009c7d0       ?RequestBorderSpace@CAxFrameWindow@ATL@@UAGJPBUtagRECT@@@Z 0049d7d0 f i FlashPlayer.obj
 0001:0009c7e0       ??0?$CWindowImpl@VCAxHostWindow@ATL@@VCWindow@2@V?$CWinTraits@$0FGAAAAAA@$0A@@2@@ATL@@QAE@XZ 0049d7e0 f i FlashPlayer.obj
 0001:0009c7e0       ??0?$CWindowImpl@VCAxFrameWindow@ATL@@VCWindow@2@V?$CWinTraits@$0FGAAAAAA@$0A@@2@@ATL@@QAE@XZ 0049d7e0 f i FlashPlayer.obj
 0001:0009c7e0       ??0?$CWindowImpl@VCAxUIWindow@ATL@@VCWindow@2@V?$CWinTraits@$0FGAAAAAA@$0A@@2@@ATL@@QAE@XZ 0049d7e0 f i FlashPlayer.obj
 0001:0009c800       ?Create@?$CWindowImpl@VCAxUIWindow@ATL@@VCWindow@2@V?$CWinTraits@$0FGAAAAAA@$0A@@2@@ATL@@QAEPAUHWND__@@PAU3@V_U_RECT@2@PBDKKV_U_MENUorID@2@PAX@Z 0049d800 f i FlashPlayer.obj
 0001:0009c8a0       ?QueryInterface@?$CComObject@VCAxUIWindow@ATL@@@ATL@@UAGJABU_GUID@@PAPAX@Z 0049d8a0 f i FlashPlayer.obj
 0001:0009c8c0       ?_InternalQueryInterface@CAxUIWindow@ATL@@QAEJABU_GUID@@PAPAX@Z 0049d8c0 f i FlashPlayer.obj
 0001:0009c8f0       ?_GetEntries@CAxUIWindow@ATL@@SGPBU_ATL_INTMAP_ENTRY@2@XZ 0049d8f0 f i FlashPlayer.obj
 0001:0009c900       ??_E?$CComObject@VCAxUIWindow@ATL@@@ATL@@UAEPAXI@Z 0049d900 f i FlashPlayer.obj
 0001:0009c900       ??_G?$CComObject@VCAxUIWindow@ATL@@@ATL@@UAEPAXI@Z 0049d900 f i FlashPlayer.obj
 0001:0009c930       ??1?$CComObject@VCAxUIWindow@ATL@@@ATL@@UAE@XZ 0049d930 f i FlashPlayer.obj
 0001:0009c980       ?FinalRelease@CAxUIWindow@ATL@@QAEXXZ 0049d980 f i FlashPlayer.obj
 0001:0009c980       ?FinalRelease@CAxFrameWindow@ATL@@QAEXXZ 0049d980 f i FlashPlayer.obj
 0001:0009c9b0       ?GetWndClassInfo@?$CWindowImpl@VCAxUIWindow@ATL@@VCWindow@2@V?$CWinTraits@$0FGAAAAAA@$0A@@2@@ATL@@SAAAU_ATL_WNDCLASSINFOA@2@XZ 0049d9b0 f i FlashPlayer.obj
 0001:0009c9c0       ?GetWndClassName@CWindow@ATL@@SAPBDXZ 0049d9c0 f i FlashPlayer.obj
 0001:0009c9c0       ?GetWndCaption@?$CWindowImpl@VCAxFrameWindow@ATL@@VCWindow@2@V?$CWinTraits@$0FGAAAAAA@$0A@@2@@ATL@@SAPBDXZ 0049d9c0 f i FlashPlayer.obj
 0001:0009c9c0       ?GetWndCaption@?$CWindowImpl@VCAxUIWindow@ATL@@VCWindow@2@V?$CWinTraits@$0FGAAAAAA@$0A@@2@@ATL@@SAPBDXZ 0049d9c0 f i FlashPlayer.obj
 0001:0009c9d0       ?copy@?$_CopyInterface@UIUnknown@@@ATL@@SAJPAPAUIUnknown@@0@Z 0049d9d0 f i FlashPlayer.obj
 0001:0009ca00       ?destroy@?$_CopyInterface@UIUnknown@@@ATL@@SAXPAPAUIUnknown@@@Z 0049da00 f i FlashPlayer.obj
 0001:0009ca20       ?Unlock@?$CComCritSecLock@VCComCriticalSection@ATL@@@ATL@@QAEXXZ 0049da20 f i FlashPlayer.obj
 0001:0009ca40       ?Unlock@CComCriticalSection@ATL@@QAEJXZ 0049da40 f i FlashPlayer.obj
 0001:0009ca60       ?CreateInstance@?$CComObject@V?$CComEnum@UIEnumUnknown@@$1?_GUID_00000100_0000_0000_c000_000000000046@@3U__s_GUID@@BPAUIUnknown@@V?$_CopyInterface@UIUnknown@@@ATL@@VCComMultiThreadModel@6@@ATL@@@ATL@@SGJPAPAV12@@Z 0049da60 f i FlashPlayer.obj
 0001:0009cba0       ?QueryInterface@?$CComContainedObject@VCAxHostWindow@ATL@@@ATL@@W3AGJABU_GUID@@PAPAX@Z 0049dba0 f i FlashPlayer.obj
 0001:0009cbb0       ?AddRef@?$CComContainedObject@VCAxHostWindow@ATL@@@ATL@@W3AGKXZ 0049dbb0 f i FlashPlayer.obj
 0001:0009cbc0       ?Release@?$CComContainedObject@VCAxHostWindow@ATL@@@ATL@@W3AGKXZ 0049dbc0 f i FlashPlayer.obj
 0001:0009cbd0       ?QueryInterface@?$CComContainedObject@VCAxHostWindow@ATL@@@ATL@@W7AGJABU_GUID@@PAPAX@Z 0049dbd0 f i FlashPlayer.obj
 0001:0009cbe0       ?AddRef@?$CComContainedObject@VCAxHostWindow@ATL@@@ATL@@W7AGKXZ 0049dbe0 f i FlashPlayer.obj
 0001:0009cbf0       ?Release@?$CComContainedObject@VCAxHostWindow@ATL@@@ATL@@W7AGKXZ 0049dbf0 f i FlashPlayer.obj
 0001:0009cc00       ?QueryInterface@?$CComContainedObject@VCAxHostWindow@ATL@@@ATL@@WM@AGJABU_GUID@@PAPAX@Z 0049dc00 f i FlashPlayer.obj
 0001:0009cc10       ?AddRef@?$CComContainedObject@VCAxHostWindow@ATL@@@ATL@@WM@AGKXZ 0049dc10 f i FlashPlayer.obj
 0001:0009cc20       ?Release@?$CComContainedObject@VCAxHostWindow@ATL@@@ATL@@WM@AGKXZ 0049dc20 f i FlashPlayer.obj
 0001:0009cc30       ?QueryInterface@?$CComContainedObject@VCAxHostWindow@ATL@@@ATL@@WBA@AGJABU_GUID@@PAPAX@Z 0049dc30 f i FlashPlayer.obj
 0001:0009cc40       ?AddRef@?$CComContainedObject@VCAxHostWindow@ATL@@@ATL@@WBA@AGKXZ 0049dc40 f i FlashPlayer.obj
 0001:0009cc50       ?Release@?$CComContainedObject@VCAxHostWindow@ATL@@@ATL@@WBA@AGKXZ 0049dc50 f i FlashPlayer.obj
 0001:0009cc60       ?QueryInterface@?$CComContainedObject@VCAxHostWindow@ATL@@@ATL@@WBE@AGJABU_GUID@@PAPAX@Z 0049dc60 f i FlashPlayer.obj
 0001:0009cc70       ?AddRef@?$CComContainedObject@VCAxHostWindow@ATL@@@ATL@@WBE@AGKXZ 0049dc70 f i FlashPlayer.obj
 0001:0009cc80       ?Release@?$CComContainedObject@VCAxHostWindow@ATL@@@ATL@@WBE@AGKXZ 0049dc80 f i FlashPlayer.obj
 0001:0009cc90       ??_E?$CComContainedObject@VCAxHostWindow@ATL@@@ATL@@WDI@AEPAXI@Z 0049dc90 f i FlashPlayer.obj
 0001:0009cca0       ?QueryInterface@?$CComContainedObject@VCAxHostWindow@ATL@@@ATL@@WBM@AGJABU_GUID@@PAPAX@Z 0049dca0 f i FlashPlayer.obj
 0001:0009ccb0       ?AddRef@?$CComContainedObject@VCAxHostWindow@ATL@@@ATL@@WBM@AGKXZ 0049dcb0 f i FlashPlayer.obj
 0001:0009ccc0       ?Release@?$CComContainedObject@VCAxHostWindow@ATL@@@ATL@@WBM@AGKXZ 0049dcc0 f i FlashPlayer.obj
 0001:0009ccd0       ?QueryInterface@?$CComContainedObject@VCAxHostWindow@ATL@@@ATL@@WCA@AGJABU_GUID@@PAPAX@Z 0049dcd0 f i FlashPlayer.obj
 0001:0009cce0       ?AddRef@?$CComContainedObject@VCAxHostWindow@ATL@@@ATL@@WCA@AGKXZ 0049dce0 f i FlashPlayer.obj
 0001:0009ccf0       ?Release@?$CComContainedObject@VCAxHostWindow@ATL@@@ATL@@WCA@AGKXZ 0049dcf0 f i FlashPlayer.obj
 0001:0009cd00       ?QueryInterface@?$CComContainedObject@VCAxHostWindow@ATL@@@ATL@@WCE@AGJABU_GUID@@PAPAX@Z 0049dd00 f i FlashPlayer.obj
 0001:0009cd10       ?AddRef@?$CComContainedObject@VCAxHostWindow@ATL@@@ATL@@WCE@AGKXZ 0049dd10 f i FlashPlayer.obj
 0001:0009cd20       ?Release@?$CComContainedObject@VCAxHostWindow@ATL@@@ATL@@WCE@AGKXZ 0049dd20 f i FlashPlayer.obj
 0001:0009cd30       ?QueryInterface@?$CComContainedObject@VCAxHostWindow@ATL@@@ATL@@WCI@AGJABU_GUID@@PAPAX@Z 0049dd30 f i FlashPlayer.obj
 0001:0009cd40       ?AddRef@?$CComContainedObject@VCAxHostWindow@ATL@@@ATL@@WCI@AGKXZ 0049dd40 f i FlashPlayer.obj
 0001:0009cd50       ?Release@?$CComContainedObject@VCAxHostWindow@ATL@@@ATL@@WCI@AGKXZ 0049dd50 f i FlashPlayer.obj
 0001:0009cd60       ??0CAtlWinModule@ATL@@QAE@XZ 0049dd60 f i FlashPlayer.obj
 0001:0009cda0       ??0_ATL_WIN_MODULE70@ATL@@QAE@XZ 0049dda0 f i FlashPlayer.obj
 0001:0009cdd0       ?AtlWinModuleInit@ATL@@YGJPAU_ATL_WIN_MODULE70@1@@Z 0049ddd0 f i FlashPlayer.obj
 0001:0009ce20       ??0?$CSimpleArray@GV?$CSimpleArrayEqualHelper@G@ATL@@@ATL@@QAE@XZ 0049de20 f i FlashPlayer.obj
 0001:0009ce20       ??0?$CSimpleMap@PADPAGVCExpansionVectorEqualHelper@ATL@@@ATL@@QAE@XZ 0049de20 f i FlashPlayer.obj
 0001:0009ce50       ??0CComModule@ATL@@QAE@XZ  0049de50 f i FlashPlayer.obj
 0001:0009ce80       ?Lock@CAtlModule@ATL@@UAEJXZ 0049de80 f i FlashPlayer.obj
 0001:0009cea0       ?Unlock@CAtlModule@ATL@@UAEJXZ 0049dea0 f i FlashPlayer.obj
 0001:0009cec0       ?GetGITPtr@CAtlModule@ATL@@UAEJPAPAUIGlobalInterfaceTable@@@Z 0049dec0 f i FlashPlayer.obj
 0001:0009cf30       ?UpdateRegistryFromResourceD@CComModule@ATL@@UAGJIHPAU_ATL_REGMAP_ENTRY@2@@Z 0049df30 f i FlashPlayer.obj
 0001:0009cf30       ?UpdateRegistryFromResourceD@CComModule@ATL@@UAGJPBDHPAU_ATL_REGMAP_ENTRY@2@@Z 0049df30 f i FlashPlayer.obj
 0001:0009cf40       ?UpdateRegistryFromResourceS@CComModule@ATL@@UAGJPBDHPAU_ATL_REGMAP_ENTRY@2@@Z 0049df40 f i FlashPlayer.obj
 0001:0009cf60       ?UpdateRegistryFromResourceS@CComModule@ATL@@UAGJIHPAU_ATL_REGMAP_ENTRY@2@@Z 0049df60 f i FlashPlayer.obj
 0001:0009cf80       ??_GCComModule@ATL@@UAEPAXI@Z 0049df80 f i FlashPlayer.obj
 0001:0009cf80       ??_ECComModule@ATL@@UAEPAXI@Z 0049df80 f i FlashPlayer.obj
 0001:0009cfb0       ??1CComModule@ATL@@UAE@XZ  0049dfb0 f i FlashPlayer.obj
 0001:0009cfd0       ??1?$CAtlModuleT@VCComModule@ATL@@@ATL@@UAE@XZ 0049dfd0 f i FlashPlayer.obj
 0001:0009cff0       ??1CAtlModule@ATL@@UAE@XZ  0049dff0 f i FlashPlayer.obj
 0001:0009d010       ?Term@CAtlModule@ATL@@QAEXXZ 0049e010 f i FlashPlayer.obj
 0001:0009d090       ?UpdateRegistryFromResourceS@CAtlModule@ATL@@QAGJPBDHPAU_ATL_REGMAP_ENTRY@2@@Z 0049e090 f i FlashPlayer.obj
 0001:0009d590       ?EscapeSingleQuote@CAtlModule@ATL@@SAXPAGPBG@Z 0049e590 f i FlashPlayer.obj
 0001:0009d5f0       ??1CRegObject@ATL@@UAE@XZ  0049e5f0 f i FlashPlayer.obj
 0001:0009d660       ??1CExpansionVector@ATL@@QAE@XZ 0049e660 f i FlashPlayer.obj
 0001:0009d6b0       ?ClearReplacements@CExpansionVector@ATL@@QAEJXZ 0049e6b0 f i FlashPlayer.obj
 0001:0009d730       ?Scroll@CAxHostWindow@ATL@@UAGJUtagSIZE@@@Z 0049e730 f i FlashPlayer.obj
 0001:0009d730       ?QueryInterface@CRegObject@ATL@@UAGJABU_GUID@@PAPAX@Z 0049e730 f i FlashPlayer.obj
 0001:0009d740       ?AddRef@CRegObject@ATL@@UAGKXZ 0049e740 f i FlashPlayer.obj
 0001:0009d750       ??_ECRegObject@ATL@@UAEPAXI@Z 0049e750 f i FlashPlayer.obj
 0001:0009d750       ??_GCRegObject@ATL@@UAEPAXI@Z 0049e750 f i FlashPlayer.obj
 0001:0009d780       ?AddReplacement@CRegObject@ATL@@UAGJPBG0@Z 0049e780 f i FlashPlayer.obj
 0001:0009d8e0       ?Add@CExpansionVector@ATL@@QAEHPBDPBG@Z 0049e8e0 f i FlashPlayer.obj
 0001:0009da60       ?ResourceRegisterSz@CRegObject@ATL@@QAGJPBG00@Z 0049ea60 f i FlashPlayer.obj
 0001:0009dc40       ?RegisterFromResource@CRegObject@ATL@@IAEJPBGPBD1H@Z 0049ec40 f i FlashPlayer.obj
 0001:0009df10       ?ResourceUnregisterSz@CRegObject@ATL@@QAGJPBG00@Z 0049ef10 f i FlashPlayer.obj
 0001:0009e0f0       ?ClearReplacements@CRegObject@ATL@@UAGJXZ 0049f0f0 f i FlashPlayer.obj
 0001:0009e130       ??0CRegParser@ATL@@QAE@PAVCRegObject@1@@Z 0049f130 f i FlashPlayer.obj
 0001:0009e160       ?RegisterBuffer@CRegParser@ATL@@QAEJPADH@Z 0049f160 f i FlashPlayer.obj
 0001:0009e320       ?GenerateError@CRegParser@ATL@@IAEJI@Z 0049f320 f i FlashPlayer.obj
 0001:0009e340       ?HKeyFromString@CRegParser@ATL@@KAPAUHKEY__@@PAD@Z 0049f340 f i FlashPlayer.obj
 0001:0009e390       ?SkipWhiteSpace@CRegParser@ATL@@IAEXXZ 0049f390 f i FlashPlayer.obj
 0001:0009e3d0       ?IsSpace@CRegParser@ATL@@IAEHD@Z 0049f3d0 f i FlashPlayer.obj
 0001:0009e430       ?NextToken@CRegParser@ATL@@IAEJPAD@Z 0049f430 f i FlashPlayer.obj
 0001:0009e620       ?EndOfVar@CRegParser@ATL@@IAEHXZ 0049f620 f i FlashPlayer.obj
 0001:0009e670       ?PreProcessBuffer@CRegParser@ATL@@QAEJPADPAPAD@Z 0049f670 f i FlashPlayer.obj
 0001:0009e8a0       ??0CParseBuffer@CRegParser@ATL@@QAE@H@Z 0049f8a0 f i FlashPlayer.obj
 0001:0009e900       ??1CParseBuffer@CRegParser@ATL@@QAE@XZ 0049f900 f i FlashPlayer.obj
 0001:0009e920       ?AddChar@CParseBuffer@CRegParser@ATL@@QAEHPBD@Z 0049f920 f i FlashPlayer.obj
 0001:0009e950       ?Append@CParseBuffer@CRegParser@ATL@@QAEHPBDH@Z 0049f950 f i FlashPlayer.obj
 0001:0009ea00       ?AddString@CParseBuffer@CRegParser@ATL@@QAEHPBG@Z 0049fa00 f i FlashPlayer.obj
 0001:0009eb10       ?Detach@CParseBuffer@CRegParser@ATL@@QAEPADXZ 0049fb10 f i FlashPlayer.obj
 0001:0009eb50       ?StrFromMap@CRegObject@ATL@@QAEPBGPAD@Z 0049fb50 f i FlashPlayer.obj
 0001:0009eb90       ?StrChrA@CRegParser@ATL@@KAPADPADD@Z 0049fb90 f i FlashPlayer.obj
 0001:0009ebe0       ?RegisterSubkeys@CRegParser@ATL@@IAEJPADPAUHKEY__@@HH@Z 0049fbe0 f i FlashPlayer.obj
 0001:0009f400       ?AtlHresultFromWin32@ATL@@YAJK@Z 004a0400 f i FlashPlayer.obj
 0001:0009f440       ??1CRegKey@ATL@@QAE@XZ     004a0440 f i FlashPlayer.obj
 0001:0009f460       ?Detach@?$CComPtrBase@UITypeInfo@@@ATL@@QAEPAUITypeInfo@@XZ 004a0460 f i FlashPlayer.obj
 0001:0009f460       ?Detach@CComBSTR@ATL@@QAEPAGXZ 004a0460 f i FlashPlayer.obj
 0001:0009f460       ?Detach@CRegKey@ATL@@QAEPAUHKEY__@@XZ 004a0460 f i FlashPlayer.obj
 0001:0009f460       ?Detach@?$CComPtrBase@UIUnknown@@@ATL@@QAEPAUIUnknown@@XZ 004a0460 f i FlashPlayer.obj
 0001:0009f490       ?DeleteSubKey@CRegKey@ATL@@QAEJPBD@Z 004a0490 f i FlashPlayer.obj
 0001:0009f4b0       ?DeleteValue@CRegKey@ATL@@QAEJPBD@Z 004a04b0 f i FlashPlayer.obj
 0001:0009f4d0       ?Close@CRegKey@ATL@@QAEJXZ 004a04d0 f i FlashPlayer.obj
 0001:0009f510       ?Create@CRegKey@ATL@@QAEJPAUHKEY__@@PBDPADKKPAU_SECURITY_ATTRIBUTES@@PAK@Z 004a0510 f i FlashPlayer.obj
 0001:0009f580       ?Open@CRegKey@ATL@@QAEJPAUHKEY__@@PBDK@Z 004a0580 f i FlashPlayer.obj
 0001:0009f5d0       ?RecurseDeleteKey@CRegKey@ATL@@QAEJPBD@Z 004a05d0 f i FlashPlayer.obj
 0001:0009f6c0       ?AddValue@CRegParser@ATL@@IAEJAAVCRegKey@2@PBDPAD@Z 004a06c0 f i FlashPlayer.obj
 0001:0009fd00       ?SetDWORDValue@CRegKey@ATL@@QAEJPBDK@Z 004a0d00 f i FlashPlayer.obj
 0001:0009fd30       ?SetStringValue@CRegKey@ATL@@QAEJPBD0K@Z 004a0d30 f i FlashPlayer.obj
 0001:0009fd70       ?SetMultiStringValue@CRegKey@ATL@@QAEJPBD0@Z 004a0d70 f i FlashPlayer.obj
 0001:0009fdd0       ?VTFromRegType@CRegParser@ATL@@KAHPBDAAG@Z 004a0dd0 f i FlashPlayer.obj
 0001:0009fe90       ?ChToByte@CRegParser@ATL@@KAED@Z 004a0e90 f i FlashPlayer.obj
 0001:0009ff30       ?CanForceRemoveKey@CRegParser@ATL@@IAEHPBD@Z 004a0f30 f i FlashPlayer.obj
 0001:0009ff80       ?HasSubKeys@CRegParser@ATL@@IAEHPAUHKEY__@@@Z 004a0f80 f i FlashPlayer.obj
 0001:0009ffd0       ?SkipAssignment@CRegParser@ATL@@IAEJPAD@Z 004a0fd0 f i FlashPlayer.obj
 0001:000a0060       ??0CRegObject@ATL@@QAE@XZ  004a1060 f i FlashPlayer.obj
 0001:000a00d0       ??0IOleClientSite@@QAE@XZ  004a10d0 f i FlashPlayer.obj
 0001:000a00d0       ??0IEnumUnknown@@QAE@XZ    004a10d0 f i FlashPlayer.obj
 0001:000a00d0       ??0IRegistrarBase@@QAE@XZ  004a10d0 f i FlashPlayer.obj
 0001:000a00d0       ??0IOleControlSite@@QAE@XZ 004a10d0 f i FlashPlayer.obj
 0001:000a00d0       ??0IDocHostUIHandler@@QAE@XZ 004a10d0 f i FlashPlayer.obj
 0001:000a00d0       ??0IObjectWithSite@@QAE@XZ 004a10d0 f i FlashPlayer.obj
 0001:000a00d0       ??0IParseDisplayName@@QAE@XZ 004a10d0 f i FlashPlayer.obj
 0001:000a00d0       ??0IAxWinHostWindow@@QAE@XZ 004a10d0 f i FlashPlayer.obj
 0001:000a00d0       ??0IServiceProvider@@QAE@XZ 004a10d0 f i FlashPlayer.obj
 0001:000a00d0       ??0IAdviseSink@@QAE@XZ     004a10d0 f i FlashPlayer.obj
 0001:000a00d0       ??0IDispatch@@QAE@XZ       004a10d0 f i FlashPlayer.obj
 0001:000a00d0       ??0IOleWindow@@QAE@XZ      004a10d0 f i FlashPlayer.obj
 0001:000a00f0       ??0CExpansionVector@ATL@@QAE@XZ 004a10f0 f i FlashPlayer.obj
 0001:000a0110       ?UpdateRegistryFromResourceS@CAtlModule@ATL@@QAGJIHPAU_ATL_REGMAP_ENTRY@2@@Z 004a1110 f i FlashPlayer.obj
 0001:000a0520       ?ResourceRegister@CRegObject@ATL@@QAGJPBGI0@Z 004a1520 f i FlashPlayer.obj
 0001:000a0640       ?ResourceUnregister@CRegObject@ATL@@QAGJPBGI0@Z 004a1640 f i FlashPlayer.obj
 0001:000a0760       ?AtlCallTermFunc@ATL@@YGXPAU_ATL_MODULE70@1@@Z 004a1760 f i FlashPlayer.obj
 0001:000a07d0       ??0?$CAtlModuleT@VCComModule@ATL@@@ATL@@QAE@XZ 004a17d0 f i FlashPlayer.obj
 0001:000a07f0       ??0CAtlModule@ATL@@QAE@XZ  004a17f0 f i FlashPlayer.obj
 0001:000a0850       ??0_ATL_MODULE70@ATL@@QAE@XZ 004a1850 f i FlashPlayer.obj
 0001:000a0870       ?AddCommonRGSReplacements@?$CAtlModuleT@VCComModule@ATL@@@ATL@@UAEJPAUIRegistrarBase@@@Z 004a1870 f i FlashPlayer.obj
 0001:000a08a0       ??1?$CSimpleMap@PADPAGVCExpansionVectorEqualHelper@ATL@@@ATL@@QAE@XZ 004a18a0 f i FlashPlayer.obj
 0001:000a08c0       ?Add@?$CSimpleMap@PADPAGVCExpansionVectorEqualHelper@ATL@@@ATL@@QAEHABQADABQAG@Z 004a18c0 f i FlashPlayer.obj
 0001:000a0960       ?RemoveAll@?$CSimpleMap@PADPAGVCExpansionVectorEqualHelper@ATL@@@ATL@@QAEXXZ 004a1960 f i FlashPlayer.obj
 0001:000a09e0       ?Lookup@?$CSimpleMap@PADPAGVCExpansionVectorEqualHelper@ATL@@@ATL@@QBEPAGABQAD@Z 004a19e0 f i FlashPlayer.obj
 0001:000a0a20       ?GetKeyAt@?$CSimpleMap@PADPAGVCExpansionVectorEqualHelper@ATL@@@ATL@@QBEAAPADH@Z 004a1a20 f i FlashPlayer.obj
 0001:000a0a60       ?GetValueAt@?$CSimpleMap@PADPAGVCExpansionVectorEqualHelper@ATL@@@ATL@@QBEAAPAGH@Z 004a1a60 f i FlashPlayer.obj
 0001:000a0aa0       ??1?$CTempBuffer@E$0BAA@VCCRTAllocator@ATL@@@ATL@@QAE@XZ 004a1aa0 f i FlashPlayer.obj
 0001:000a0aa0       ??1?$CTempBuffer@D$0EAA@VCCRTAllocator@ATL@@@ATL@@QAE@XZ 004a1aa0 f i FlashPlayer.obj
 0001:000a0aa0       ??1?$CTempBuffer@D$0BAA@VCCRTAllocator@ATL@@@ATL@@QAE@XZ 004a1aa0 f i FlashPlayer.obj
 0001:000a0ac0       ?Allocate@?$CTempBuffer@D$0EAA@VCCRTAllocator@ATL@@@ATL@@QAEPADI@Z 004a1ac0 f i FlashPlayer.obj
 0001:000a0ae0       ??B?$CComPtrBase@UIUnknown@@@ATL@@QBEPAUIUnknown@@XZ 004a1ae0 f i FlashPlayer.obj
 0001:000a0ae0       ??BCRegKey@ATL@@QBEPAUHKEY__@@XZ 004a1ae0 f i FlashPlayer.obj
 0001:000a0ae0       ??B?$CComPtrBase@UIOleObject@@@ATL@@QBEPAUIOleObject@@XZ 004a1ae0 f i FlashPlayer.obj
 0001:000a0ae0       ??B?$CComPtrBase@UIStream@@@ATL@@QBEPAUIStream@@XZ 004a1ae0 f i FlashPlayer.obj
 0001:000a0ae0       ??C?$CComPtrBase@UIOleInPlaceActiveObject@@@ATL@@QBEPAV?$_NoAddRefReleaseOnCComPtr@UIOleInPlaceActiveObject@@@1@XZ 004a1ae0 f i FlashPlayer.obj
 0001:000a0ae0       ??C?$CComPtrBase@UIUnknown@@@ATL@@QBEPAV?$_NoAddRefReleaseOnCComPtr@UIUnknown@@@1@XZ 004a1ae0 f i FlashPlayer.obj
 0001:000a0ae0       ??C?$CComPtrBase@UIObjectWithSite@@@ATL@@QBEPAV?$_NoAddRefReleaseOnCComPtr@UIObjectWithSite@@@1@XZ 004a1ae0 f i FlashPlayer.obj
 0001:000a0ae0       ?Points@CTechPoints@@QBE?BHXZ 004a1ae0 f i VillagerAI.obj
 0001:000a0ae0       ??C?$CComPtrBase@UIConnectionPoint@@@ATL@@QBEPAV?$_NoAddRefReleaseOnCComPtr@UIConnectionPoint@@@1@XZ 004a1ae0 f i FlashPlayer.obj
 0001:000a0ae0       ??B?$CComPtrBase@UIDocHostUIHandlerDispatch@@@ATL@@QBEPAUIDocHostUIHandlerDispatch@@XZ 004a1ae0 f i FlashPlayer.obj
 0001:000a0ae0       ?Current@CWeather@@QBE?BW4EWeather@@XZ 004a1ae0 f i Villager.obj
 0001:000a0ae0       ??C?$CComPtrBase@UIViewObjectEx@@@ATL@@QBEPAV?$_NoAddRefReleaseOnCComPtr@UIViewObjectEx@@@1@XZ 004a1ae0 f i FlashPlayer.obj
 0001:000a0ae0       ?CurrentAction@CVillagerPlans@@QBE?BW4EAction@@XZ 004a1ae0 f i VillagerAI.obj
 0001:000a0ae0       ??B?$CComPtrBase@UIPersistStreamInit@@@ATL@@QBEPAUIPersistStreamInit@@XZ 004a1ae0 f i FlashPlayer.obj
 0001:000a0ae0       ??C?$CComPtrBase@UIPersistStream@@@ATL@@QBEPAV?$_NoAddRefReleaseOnCComPtr@UIPersistStream@@@1@XZ 004a1ae0 f i FlashPlayer.obj
 0001:000a0ae0       ??C?$CComPtrBase@UIServiceProvider@@@ATL@@QBEPAV?$_NoAddRefReleaseOnCComPtr@UIServiceProvider@@@1@XZ 004a1ae0 f i FlashPlayer.obj
 0001:000a0ae0       ?GetWidth@ldwGameWindowImpl@@QAEHXZ 004a1ae0 f i ldwGameWindow.obj
 0001:000a0ae0       ??C?$CComPtrBase@UIDispatch@@@ATL@@QBEPAV?$_NoAddRefReleaseOnCComPtr@UIDispatch@@@1@XZ 004a1ae0 f i FlashPlayer.obj
 0001:000a0ae0       ??C?$CComPtrBase@UIOleObject@@@ATL@@QBEPAV?$_NoAddRefReleaseOnCComPtr@UIOleObject@@@1@XZ 004a1ae0 f i FlashPlayer.obj
 0001:000a0ae0       ??C?$CComPtrBase@UIAxWinHostWindowLic@@@ATL@@QBEPAV?$_NoAddRefReleaseOnCComPtr@UIAxWinHostWindowLic@@@1@XZ 004a1ae0 f i FlashPlayer.obj
 0001:000a0ae0       ??B?$CComPtrBase@UIObjectWithSite@@@ATL@@QBEPAUIObjectWithSite@@XZ 004a1ae0 f i FlashPlayer.obj
 0001:000a0ae0       ??B?$CComPtrBase@UIViewObjectEx@@@ATL@@QBEPAUIViewObjectEx@@XZ 004a1ae0 f i FlashPlayer.obj
 0001:000a0ae0       ??B?$CComPtrBase@UIPersistStream@@@ATL@@QBEPAUIPersistStream@@XZ 004a1ae0 f i FlashPlayer.obj
 0001:000a0ae0       ??BCComBSTR@ATL@@QBEPAGXZ  004a1ae0 f i FlashPlayer.obj
 0001:000a0ae0       ??B?$CComPtrBase@UIOleClientSite@@@ATL@@QBEPAUIOleClientSite@@XZ 004a1ae0 f i FlashPlayer.obj
 0001:000a0ae0       ??B?$CComPtrBase@UIDispatch@@@ATL@@QBEPAUIDispatch@@XZ 004a1ae0 f i FlashPlayer.obj
 0001:000a0ae0       ?Level@CFoodStore@@QBE?BHXZ 004a1ae0 f i Behavior.obj
 0001:000a0ae0       ??B?$CComPtrBase@UIServiceProvider@@@ATL@@QBEPAUIServiceProvider@@XZ 004a1ae0 f i FlashPlayer.obj
 0001:000a0ae0       ?SecondsAccumulated@CVillagerState@@QAE?BKXZ 004a1ae0 f i VillagerManager.obj
 0001:000a0ae0       ??B?$CComPtrBase@UIOleInPlaceActiveObject@@@ATL@@QBEPAUIOleInPlaceActiveObject@@XZ 004a1ae0 f i FlashPlayer.obj
 0001:000a0ae0       ??C?$CComPtrBase@UIOleControl@@@ATL@@QBEPAV?$_NoAddRefReleaseOnCComPtr@UIOleControl@@@1@XZ 004a1ae0 f i FlashPlayer.obj
 0001:000a0ae0       ??C?$CComPtrBase@UIAxWinHostWindow@@@ATL@@QBEPAV?$_NoAddRefReleaseOnCComPtr@UIAxWinHostWindow@@@1@XZ 004a1ae0 f i FlashPlayer.obj
 0001:000a0ae0       ??B?$CComPtrBase@UIOleControl@@@ATL@@QBEPAUIOleControl@@XZ 004a1ae0 f i FlashPlayer.obj
 0001:000a0ae0       ??B?$CTempBuffer@D$0EAA@VCCRTAllocator@ATL@@@ATL@@QBEPADXZ 004a1ae0 f i FlashPlayer.obj
 0001:000a0ae0       ??B?$CComPtrBase@UIAdviseSink@@@ATL@@QBEPAUIAdviseSink@@XZ 004a1ae0 f i FlashPlayer.obj
 0001:000a0ae0       ??B?$CComPtrBase@UIWebBrowser2@@@ATL@@QBEPAUIWebBrowser2@@XZ 004a1ae0 f i FlashPlayer.obj
 0001:000a0ae0       ?GameStartTime@CGameStats@@QBE?BIXZ 004a1ae0 f i theLoadingScene.obj
 0001:000a0ae0       ??B?$CComPtrBase@UITypeInfo2@@@ATL@@QBEPAUITypeInfo2@@XZ 004a1ae0 f i FlashPlayer.obj
 0001:000a0ae0       ??B?$CTempBuffer@E$0BAA@VCCRTAllocator@ATL@@@ATL@@QBEPAEXZ 004a1ae0 f i FlashPlayer.obj
 0001:000a0ae0       ??C?$CComPtrBase@UIDocHostUIHandlerDispatch@@@ATL@@QBEPAV?$_NoAddRefReleaseOnCComPtr@UIDocHostUIHandlerDispatch@@@1@XZ 004a1ae0 f i FlashPlayer.obj
 0001:000a0ae0       ??B?$CComPtrBase@UIOleInPlaceObjectWindowless@@@ATL@@QBEPAUIOleInPlaceObjectWindowless@@XZ 004a1ae0 f i FlashPlayer.obj
 0001:000a0ae0       ??B?$CTempBuffer@D$0BAA@VCCRTAllocator@ATL@@@ATL@@QBEPADXZ 004a1ae0 f i FlashPlayer.obj
 0001:000a0ae0       ??C?$CComPtrBase@UIWebBrowser2@@@ATL@@QBEPAV?$_NoAddRefReleaseOnCComPtr@UIWebBrowser2@@@1@XZ 004a1ae0 f i FlashPlayer.obj
 0001:000a0ae0       ??C?$CComPtrBase@UITypeInfo@@@ATL@@QBEPAV?$_NoAddRefReleaseOnCComPtr@UITypeInfo@@@1@XZ 004a1ae0 f i FlashPlayer.obj
 0001:000a0ae0       ?Age@CVillagerBio@@QBE?BHXZ 004a1ae0 f i Behavior.obj
 0001:000a0ae0       ??C?$CComPtrBase@UIOleInPlaceObjectWindowless@@@ATL@@QBEPAV?$_NoAddRefReleaseOnCComPtr@UIOleInPlaceObjectWindowless@@@1@XZ 004a1ae0 f i FlashPlayer.obj
 0001:000a0ae0       ??C?$CComPtrBase@UIClassFactory2@@@ATL@@QBEPAV?$_NoAddRefReleaseOnCComPtr@UIClassFactory2@@@1@XZ 004a1ae0 f i FlashPlayer.obj
 0001:000a0ae0       ??BCWindow@ATL@@QBEPAUHWND__@@XZ 004a1ae0 f i FlashPlayer.obj
 0001:000a0ae0       ??C?$CComPtrBase@UIConnectionPointContainer@@@ATL@@QBEPAV?$_NoAddRefReleaseOnCComPtr@UIConnectionPointContainer@@@1@XZ 004a1ae0 f i FlashPlayer.obj
 0001:000a0ae0       ??C?$CComPtrBase@UIPersistStreamInit@@@ATL@@QBEPAV?$_NoAddRefReleaseOnCComPtr@UIPersistStreamInit@@@1@XZ 004a1ae0 f i FlashPlayer.obj
 0001:000a0af0       ?Allocate@?$CTempBuffer@D$0BAA@VCCRTAllocator@ATL@@@ATL@@QAEPADI@Z 004a1af0 f i FlashPlayer.obj
 0001:000a0af0       ?Allocate@?$CTempBuffer@E$0BAA@VCCRTAllocator@ATL@@@ATL@@QAEPAEI@Z 004a1af0 f i FlashPlayer.obj
 0001:000a0b10       ?GetAppId@?$CAtlModuleT@VCComModule@ATL@@@ATL@@SAPBGXZ 004a1b10 f i FlashPlayer.obj
 0001:000a0b20       ?FindKey@?$CSimpleMap@PADPAGVCExpansionVectorEqualHelper@ATL@@@ATL@@QBEHABQAD@Z 004a1b20 f i FlashPlayer.obj
 0001:000a0b80       ?IsEqualKey@CExpansionVectorEqualHelper@ATL@@SA_NQAD0@Z 004a1b80 f i FlashPlayer.obj
 0001:000a0ba0       ?InternalSetAtIndex@?$CSimpleMap@PADPAGVCExpansionVectorEqualHelper@ATL@@@ATL@@QAEXHABQADABQAG@Z 004a1ba0 f i FlashPlayer.obj
 0001:000a0c70       ?AllocateBytes@?$CTempBuffer@D$0EAA@VCCRTAllocator@ATL@@@ATL@@QAEPADI@Z 004a1c70 f i FlashPlayer.obj
 0001:000a0cb0       ?AllocateBytes@?$CTempBuffer@D$0BAA@VCCRTAllocator@ATL@@@ATL@@QAEPADI@Z 004a1cb0 f i FlashPlayer.obj
 0001:000a0cb0       ?AllocateBytes@?$CTempBuffer@E$0BAA@VCCRTAllocator@ATL@@@ATL@@QAEPAEI@Z 004a1cb0 f i FlashPlayer.obj
 0001:000a0cf0       ?FreeHeap@?$CTempBuffer@D$0BAA@VCCRTAllocator@ATL@@@ATL@@AAEXXZ 004a1cf0 f i FlashPlayer.obj
 0001:000a0cf0       ?FreeHeap@?$CTempBuffer@D$0EAA@VCCRTAllocator@ATL@@@ATL@@AAEXXZ 004a1cf0 f i FlashPlayer.obj
 0001:000a0cf0       ?FreeHeap@?$CTempBuffer@E$0BAA@VCCRTAllocator@ATL@@@ATL@@AAEXXZ 004a1cf0 f i FlashPlayer.obj
 0001:000a0d10       ?AllocateHeap@?$CTempBuffer@D$0EAA@VCCRTAllocator@ATL@@@ATL@@AAEXI@Z 004a1d10 f i FlashPlayer.obj
 0001:000a0d10       ?AllocateHeap@?$CTempBuffer@E$0BAA@VCCRTAllocator@ATL@@@ATL@@AAEXI@Z 004a1d10 f i FlashPlayer.obj
 0001:000a0d10       ?AllocateHeap@?$CTempBuffer@D$0BAA@VCCRTAllocator@ATL@@@ATL@@AAEXI@Z 004a1d10 f i FlashPlayer.obj
 0001:000a0d50       ??0?$Wrapper@PAG@?$CSimpleMap@PADPAGVCExpansionVectorEqualHelper@ATL@@@ATL@@QAE@ABQAG@Z 004a1d50 f i FlashPlayer.obj
 0001:000a0d50       ??0?$Wrapper@PAD@?$CSimpleMap@PADPAGVCExpansionVectorEqualHelper@ATL@@@ATL@@QAE@ABQAD@Z 004a1d50 f i FlashPlayer.obj
 0001:000a0d70       ??$?3PAD@?$Wrapper@PAD@?$CSimpleMap@PADPAGVCExpansionVectorEqualHelper@ATL@@@ATL@@SAXPAXPAPAD@Z 004a1d70 f i FlashPlayer.obj
 0001:000a0d70       ?init@?$_CopyInterface@UIUnknown@@@ATL@@SAXPAPAUIUnknown@@@Z 004a1d70 f i FlashPlayer.obj
 0001:000a0d70       ?InitLibId@?$CAtlModuleT@VCComModule@ATL@@@ATL@@SAXXZ 004a1d70 f i FlashPlayer.obj
 0001:000a0d70       ??$?3PAG@?$Wrapper@PAG@?$CSimpleMap@PADPAGVCExpansionVectorEqualHelper@ATL@@@ATL@@SAXPAXPAPAG@Z 004a1d70 f i FlashPlayer.obj
 0001:000a0d70       ??$?3G@Wrapper@?$CSimpleArray@GV?$CSimpleArrayEqualHelper@G@ATL@@@ATL@@SAXPAXPAG@Z 004a1d70 f i FlashPlayer.obj
 0001:000a0d80       ??1CAtlWinModule@ATL@@QAE@XZ 004a1d80 f i FlashPlayer.obj
 0001:000a0dd0       ?Term@CAtlWinModule@ATL@@QAEXXZ 004a1dd0 f i FlashPlayer.obj
 0001:000a0df0       ??1_ATL_WIN_MODULE70@ATL@@QAE@XZ 004a1df0 f i FlashPlayer.obj
 0001:000a0e10       ?AtlWinModuleTerm@ATL@@YGJPAU_ATL_WIN_MODULE70@1@PAUHINSTANCE__@@@Z 004a1e10 f i FlashPlayer.obj
 0001:000a0eb0       ??1?$CSimpleArray@GV?$CSimpleArrayEqualHelper@G@ATL@@@ATL@@QAE@XZ 004a1eb0 f i FlashPlayer.obj
 0001:000a0ed0       ?RemoveAll@?$CSimpleArray@GV?$CSimpleArrayEqualHelper@G@ATL@@@ATL@@QAEXXZ 004a1ed0 f i FlashPlayer.obj
 0001:000a0f30       ??A?$CSimpleArray@GV?$CSimpleArrayEqualHelper@G@ATL@@@ATL@@QAEAAGH@Z 004a1f30 f i FlashPlayer.obj
 0001:000a0f70       ??0CAchievement@@QAE@XZ    004a1f70 f   Achievement.obj
 0001:000a0f90       ?Reset@CAchievement@@QAEXXZ 004a1f90 f   Achievement.obj
 0001:000a0fd0       ?LoadState@CAchievement@@QAE?B_NAAUSSaveState@1@@Z 004a1fd0 f   Achievement.obj
 0001:000a1020       ?SaveState@CAchievement@@QAE?B_NAAUSSaveState@1@@Z 004a2020 f   Achievement.obj
 0001:000a1070       ?SetComplete@CAchievement@@QAEXW4EAchievement@@@Z 004a2070 f   Achievement.obj
 0001:000a10e0       ?IsComplete@CAchievement@@QBE?B_NW4EAchievement@@@Z 004a20e0 f   Achievement.obj
 0001:000a1100       ?AchievementsComplete@CAchievement@@QBE?BHXZ 004a2100 f   Achievement.obj
 0001:000a1150       ?CompletionTime@CAchievement@@QBE?BHW4EAchievement@@@Z 004a2150 f   Achievement.obj
 0001:000a1170       ??0CTutorialTip@@QAE@XZ    004a2170 f   TutorialTip.obj
 0001:000a1190       ?Reset@CTutorialTip@@QAEXXZ 004a2190 f   TutorialTip.obj
 0001:000a1460       ?LoadState@CTutorialTip@@QAE?B_NABUSSaveState@1@@Z 004a2460 f   TutorialTip.obj
 0001:000a1540       ?SaveState@CTutorialTip@@QBE?B_NAAUSSaveState@1@@Z 004a2540 f   TutorialTip.obj
 0001:000a15a0       ?ConfigureTip@CTutorialTip@@QAEXW4StringId@@IW4ArrowDirection@@HH_NHH@Z 004a25a0 f   TutorialTip.obj
 0001:000a1630       ?HandleSpecialCase@CTutorialTip@@QAE_NW4StringId@@@Z 004a2630 f   TutorialTip.obj
 0001:000a1940       ?Update@CTutorialTip@@QAE?BW4StringId@@W4EGameScene@@PAVldwScene@@@Z 004a2940 f   TutorialTip.obj
 0001:000a1a50       ?Queue@CTutorialTip@@QAEXW4StringId@@W4EGameScene@@_N@Z 004a2a50 f   TutorialTip.obj
 0001:000a1b20       ?Display@CTutorialTip@@QAEHW4StringId@@PAVldwScene@@@Z 004a2b20 f   TutorialTip.obj
 0001:000a1dc0       ?DisableTips@CTutorialTip@@QAEX_N@Z 004a2dc0 f   TutorialTip.obj
 0001:000a1e30       ?RepeatLastTip@CTutorialTip@@QAEXXZ 004a2e30 f   TutorialTip.obj
 0001:000a1e80       ?QueueNextInstruction@CTutorialTip@@QAEXXZ 004a2e80 f   TutorialTip.obj
 0001:000a1ef0       ?SetDisplayed@CTutorialTip@@QAEXW4StringId@@@Z 004a2ef0 f   TutorialTip.obj
 0001:000a1f20       ?IsDisplayed@CTutorialTip@@QBE?B_NXZ 004a2f20 f   TutorialTip.obj
 0001:000a1f40       ?WasDisplayed@CTutorialTip@@QBE?B_NW4StringId@@@Z 004a2f40 f   TutorialTip.obj
 0001:000a1f70       ?IsInstruction@CTutorialTip@@QBE?B_NW4StringId@@@Z 004a2f70 f   TutorialTip.obj
 0001:000a1fb0       ?IsNonInstructionQueuedFor@CTutorialTip@@QBE?B_NW4EGameScene@@@Z 004a2fb0 f   TutorialTip.obj
 0001:000a2010       ?LastTip@CTutorialTip@@QBE?BW4StringId@@XZ 004a3010 f   TutorialTip.obj
 0001:000a2030       ?Enter@CIntroPage1@@UAEXXZ 004a3030 f   Pages.obj
 0001:000a2100       ?FadeImage@CIntroPage1@@UAE?B_NXZ 004a3100 f   Pages.obj
 0001:000a2170       ?FadeOut@CIntroPage1@@UAE?B_NXZ 004a3170 f   Pages.obj
 0001:000a2230       ?Exit@CIntroPage1@@UAEXXZ  004a3230 f   Pages.obj
 0001:000a2260       ?Enter@CIntroPage2@@UAEXXZ 004a3260 f   Pages.obj
 0001:000a2320       ?Exit@CIntroPage2@@UAEXXZ  004a3320 f   Pages.obj
 0001:000a2350       ?FadeImage@CIntroPage2@@UAE?B_NXZ 004a3350 f   Pages.obj
 0001:000a23a0       ?FadeOut@CIntroPage2@@UAE?B_NXZ 004a33a0 f   Pages.obj
 0001:000a2460       ?Enter@CIntroPage3@@UAEXXZ 004a3460 f   Pages.obj
 0001:000a2500       ?FadeImage@CIntroPage3@@UAE?B_NXZ 004a3500 f   Pages.obj
 0001:000a2560       ?FadeOut@CIntroPage3@@UAE?B_NXZ 004a3560 f   Pages.obj
 0001:000a25c0       ?Enter@CIntroPage4@@UAEXXZ 004a35c0 f   Pages.obj
 0001:000a2620       ?FadeImage@CIntroPage4@@UAE?B_NXZ 004a3620 f   Pages.obj
 0001:000a2670       ?FadeOut@CIntroPage4@@UAE?B_NXZ 004a3670 f   Pages.obj
 0001:000a26d0       ?Enter@CIntroPage5@@UAEXXZ 004a36d0 f   Pages.obj
 0001:000a2760       ?Exit@CIntroPage5@@UAEXXZ  004a3760 f   Pages.obj
 0001:000a2790       ?FadeImage@CIntroPage5@@UAE?B_NXZ 004a3790 f   Pages.obj
 0001:000a2840       ?FadeImageSkipped@CIntroPage5@@UAEXXZ 004a3840 f   Pages.obj
 0001:000a2880       ?Update@CIntroPage5@@UAEXXZ 004a3880 f   Pages.obj
 0001:000a28b0       ?FadeOut@CIntroPage5@@UAE?B_NXZ 004a38b0 f   Pages.obj
 0001:000a2900       ?Enter@CMidGamePage1@@UAEXXZ 004a3900 f   Pages.obj
 0001:000a29d0       ?FadeImage@CMidGamePage1@@UAE?B_NXZ 004a39d0 f   Pages.obj
 0001:000a2a50       ?Update@CMidGamePage1@@UAEXXZ 004a3a50 f   Pages.obj
 0001:000a2ac0       ?FadeOut@CMidGamePage1@@UAE?B_NXZ 004a3ac0 f   Pages.obj
 0001:000a2b30       ?Enter@CMidGamePage2@@UAEXXZ 004a3b30 f   Pages.obj
 0001:000a2c30       ?FadeImage@CMidGamePage2@@UAE?B_NXZ 004a3c30 f   Pages.obj
 0001:000a2ca0       ?FadeOut@CMidGamePage2@@UAE?B_NXZ 004a3ca0 f   Pages.obj
 0001:000a2d00       ?Enter@CMidGamePage3@@UAEXXZ 004a3d00 f   Pages.obj
 0001:000a2ec0       ?FadeImage@CMidGamePage3@@UAE?B_NXZ 004a3ec0 f   Pages.obj
 0001:000a2f50       ?Update@CMidGamePage3@@UAEXXZ 004a3f50 f   Pages.obj
 0001:000a2fc0       ?FadeOut@CMidGamePage3@@UAE?B_NXZ 004a3fc0 f   Pages.obj
 0001:000a3040       ?Enter@CEndGamePage1@@UAEXXZ 004a4040 f   Pages.obj
 0001:000a3120       ?FadeImage@CEndGamePage1@@UAE?B_NXZ 004a4120 f   Pages.obj
 0001:000a31a0       ?Update@CEndGamePage1@@UAEXXZ 004a41a0 f   Pages.obj
 0001:000a3210       ?FadeOut@CEndGamePage1@@UAE?B_NXZ 004a4210 f   Pages.obj
 0001:000a3270       ?Enter@CEndGamePage2@@UAEXXZ 004a4270 f   Pages.obj
 0001:000a3350       ?FadeImage@CEndGamePage2@@UAE?B_NXZ 004a4350 f   Pages.obj
 0001:000a33c0       ?FadeOut@CEndGamePage2@@UAE?B_NXZ 004a43c0 f   Pages.obj
 0001:000a3410       ?Enter@CEndGamePage3@@UAEXXZ 004a4410 f   Pages.obj
 0001:000a3480       ?FadeImage@CEndGamePage3@@UAE?B_NXZ 004a4480 f   Pages.obj
 0001:000a34e0       ?FadeOut@CEndGamePage3@@UAE?B_NXZ 004a44e0 f   Pages.obj
 0001:000a3530       ?Enter@CEndGamePage4@@UAEXXZ 004a4530 f   Pages.obj
 0001:000a3600       ?FadeImage@CEndGamePage4@@UAE?B_NXZ 004a4600 f   Pages.obj
 0001:000a3670       ?FadeOut@CEndGamePage4@@UAE?B_NXZ 004a4670 f   Pages.obj
 0001:000a36c0       ?Alpha@CStory@@QBE?BMH@Z   004a46c0 f i Pages.obj
 0001:000a36e0       ?Scale@CStory@@QBE?BMH@Z   004a46e0 f i Pages.obj
 0001:000a3700       ?XPos@CStory@@QBE?BHH@Z    004a4700 f i Pages.obj
 0001:000a3730       ?SetTextSpeed@CStory@@QAEXM@Z 004a4730 f i Pages.obj
 0001:000a3750       ?IsTextDisplayed@CStory@@QBE?B_NXZ 004a4750 f i Pages.obj
 0001:000a3770       ?IsSkipPressed@CStory@@QAE?B_NXZ 004a4770 f i Pages.obj
 0001:000a3790       ??0CIntroPage1@@QAE@XZ     004a4790 f i Pages.obj
 0001:000a37b0       ??0IPage@@QAE@XZ           004a47b0 f i Pages.obj
 0001:000a37d0       ??0CIntroPage2@@QAE@XZ     004a47d0 f i Pages.obj
 0001:000a37f0       ??0CIntroPage3@@QAE@XZ     004a47f0 f i Pages.obj
 0001:000a3810       ??0CIntroPage4@@QAE@XZ     004a4810 f i Pages.obj
 0001:000a3830       ??0CIntroPage5@@QAE@XZ     004a4830 f i Pages.obj
 0001:000a3850       ??0CMidGamePage1@@QAE@XZ   004a4850 f i Pages.obj
 0001:000a3870       ??0CMidGamePage2@@QAE@XZ   004a4870 f i Pages.obj
 0001:000a3890       ??0CMidGamePage3@@QAE@XZ   004a4890 f i Pages.obj
 0001:000a38b0       ??0CEndGamePage1@@QAE@XZ   004a48b0 f i Pages.obj
 0001:000a38d0       ??0CEndGamePage2@@QAE@XZ   004a48d0 f i Pages.obj
 0001:000a38f0       ??0CEndGamePage3@@QAE@XZ   004a48f0 f i Pages.obj
 0001:000a3910       ??0CEndGamePage4@@QAE@XZ   004a4910 f i Pages.obj
 0001:000a3930       ??0CStory@@QAE@XZ          004a4930 f   Story.obj
 0001:000a3a40       ?AddPage@CStory@@AAEXW4EStory@1@PAVIPage@@@Z 004a4a40 f   Story.obj
 0001:000a3a90       ?Enter@CStory@@QAEXXZ      004a4a90 f   Story.obj
 0001:000a3b20       ?Exit@CStory@@QAEXXZ       004a4b20 f   Story.obj
 0001:000a3c00       ?Draw@CStory@@QAEXXZ       004a4c00 f   Story.obj
 0001:000a3f60       ?Update@CStory@@QAEXXZ     004a4f60 f   Story.obj
 0001:000a45b0       ?HandleMouseDown@CStory@@QAEXXZ 004a55b0 f   Story.obj
 0001:000a4790       ?GotoPage@CStory@@AAEXH@Z  004a5790 f   Story.obj
 0001:000a4900       ?AddTutorialTipButtons@CStory@@QAEXXZ 004a5900 f   Story.obj
 0001:000a4920       ?AddText@CStory@@QAEXW4StringId@@@Z 004a5920 f   Story.obj
 0001:000a4960       ?AddImage@CStory@@QAE?BHW4EImage@@HHH@Z 004a5960 f   Story.obj
 0001:000a4a70       ?ReleaseImages@CStory@@QAEXXZ 004a5a70 f   Story.obj
 0001:000a4ad0       ?SetStory@CStory@@QAEXW4EStory@1@@Z 004a5ad0 f   Story.obj
 0001:000a4af0       ?SetTextPos@CStory@@QAEXHH@Z 004a5af0 f   Story.obj
 0001:000a4b20       ?SetAlpha@CStory@@QAEXHM@Z 004a5b20 f   Story.obj
 0001:000a4b40       ?SetTargetAlpha@CStory@@QAEXHMH@Z 004a5b40 f   Story.obj
 0001:000a4ba0       ?SetScale@CStory@@QAEXHM@Z 004a5ba0 f   Story.obj
 0001:000a4bc0       ?SetTargetScale@CStory@@QAEXHMH@Z 004a5bc0 f   Story.obj
 0001:000a4c20       ?SetPos@CStory@@QAEXHHH@Z  004a5c20 f   Story.obj
 0001:000a4c60       ?SetTargetPos@CStory@@QAEXHHHH@Z 004a5c60 f   Story.obj
 0001:000a4cd0       ?PlayNarrative@CStory@@QAEXW4ESound@@@Z 004a5cd0 f   Story.obj
 0001:000a4d00       ?Volume@CSoundTrack@@QAE?BMXZ 004a5d00 f i Story.obj
 0001:000a4d12       _FSOUND_Sample_Load@20     004a5d12 f   fmodvc:fmod.dll
 0001:000a4d18       _FSOUND_Init@12            004a5d18 f   fmodvc:fmod.dll
 0001:000a4d1e       _FSOUND_Sample_Free@4      004a5d1e f   fmodvc:fmod.dll
 0001:000a4d24       _FSOUND_Close@0            004a5d24 f   fmodvc:fmod.dll
 0001:000a4d2a       _FSOUND_SetVolume@8        004a5d2a f   fmodvc:fmod.dll
 0001:000a4d30       _FSOUND_PlaySound@8        004a5d30 f   fmodvc:fmod.dll
 0001:000a4d36       _FSOUND_Sample_SetMode@8   004a5d36 f   fmodvc:fmod.dll
 0001:000a4d3c       _FSOUND_StopSound@4        004a5d3c f   fmodvc:fmod.dll
 0001:000a4d42       _FSOUND_SetSFXMasterVolume@4 004a5d42 f   fmodvc:fmod.dll
 0001:000a4d48       _FSOUND_IsPlaying@4        004a5d48 f   fmodvc:fmod.dll
 0001:000a4d4e       _FMUSIC_LoadSong@4         004a5d4e f   fmodvc:fmod.dll
 0001:000a4d54       _FSOUND_Stream_Open@16     004a5d54 f   fmodvc:fmod.dll
 0001:000a4d5a       _FMUSIC_SetMasterVolume@8  004a5d5a f   fmodvc:fmod.dll
 0001:000a4d60       _FMUSIC_FreeSong@4         004a5d60 f   fmodvc:fmod.dll
 0001:000a4d66       _FSOUND_Stream_Close@4     004a5d66 f   fmodvc:fmod.dll
 0001:000a4d6c       _FMUSIC_PlaySong@4         004a5d6c f   fmodvc:fmod.dll
 0001:000a4d72       _FMUSIC_SetLooping@8       004a5d72 f   fmodvc:fmod.dll
 0001:000a4d78       _FSOUND_Stream_Play@8      004a5d78 f   fmodvc:fmod.dll
 0001:000a4d7e       _FSOUND_Stream_SetMode@8   004a5d7e f   fmodvc:fmod.dll
 0001:000a4d84       _FMUSIC_StopAllSongs@0     004a5d84 f   fmodvc:fmod.dll
 0001:000a4d8a       _FMUSIC_StopSong@4         004a5d8a f   fmodvc:fmod.dll
 0001:000a4d90       _FSOUND_Stream_Stop@4      004a5d90 f   fmodvc:fmod.dll
 0001:000a4d96       _FMUSIC_IsPlaying@4        004a5d96 f   fmodvc:fmod.dll
 0001:000a4d9c       _FMUSIC_GetTime@4          004a5d9c f   fmodvc:fmod.dll
 0001:000a4da2       _FSOUND_Stream_GetTime@4   004a5da2 f   fmodvc:fmod.dll
 0001:000a4db0       ?DecodePNGRGBA@gdalphaimage@@YAJPAVCGapiSurfaceHelper@@KAAVCGapiRGBASurface@@PAEK@Z 004a5db0 f   gapidraw:GapiRGBASurface.obj
 0001:000a5500       ??1_PNGReader@gdalphaimage@@QAE@XZ 004a6500 f i gapidraw:GapiRGBASurface.obj
 0001:000a5500       ??1_PNGReader@gdimage@@QAE@XZ 004a6500 f i gapidraw:GapiSurface.obj
 0001:000a5540       ??0CGapiRGBASurface@@QAE@PAVCGapiDraw@@@Z 004a6540 f   gapidraw:GapiRGBASurface.obj
 0001:000a5570       ??_ECGapiRGBASurface@@UAEPAXI@Z 004a6570 f i gapidraw:GapiRGBASurface.obj
 0001:000a5570       ??_GCGapiRGBASurface@@UAEPAXI@Z 004a6570 f i gapidraw:GapiRGBASurface.obj
 0001:000a55c0       ?CreateSurface@CGapiRGBASurface@@QAEJKKK@Z 004a65c0 f   gapidraw:GapiRGBASurface.obj
 0001:000a59c0       ?CreateSurface@CGapiRGBASurface@@QAEJKPAEK@Z 004a69c0 f   gapidraw:GapiRGBASurface.obj
 0001:000a5a60       ?CreateSurface@CGapiRGBASurface@@QAEJKPBD@Z 004a6a60 f   gapidraw:GapiRGBASurface.obj
 0001:000a5c50       ?GetWidth@CGapiRGBASurface@@QAEKXZ 004a6c50 f   gapidraw:GapiRGBASurface.obj
 0001:000a5c60       ?GetHeight@CGapiRGBASurface@@QAEKXZ 004a6c60 f   gapidraw:GapiRGBASurface.obj
 0001:000a5c60       ?GetWidth@CGapiSurface@@QAEKXZ 004a6c60 f   gapidraw:GapiSurface.obj
 0001:000a5c70       ?GetBuffer@CGapiRGBASurface@@QAEJPAU_GDBUFFERDESC@@@Z 004a6c70 f   gapidraw:GapiRGBASurface.obj
 0001:000a5d80       ?ReleaseBuffer@CGapiRGBASurface@@QAEJXZ 004a6d80 f   gapidraw:GapiRGBASurface.obj
 0001:000a5db0       ??1_MemFile@gdio@@QAE@XZ   004a6db0 f i gapidraw:GapiRGBASurface.obj
 0001:000a5de0       ?AlignMemorySurface@CGapiSurfaceHelper@@QAEXAAU_GDSURFACE@gdinternal@@@Z 004a6de0 f i gapidraw:GapiRGBASurface.obj
 0001:000a6040       ??0CGapiSurface@@QAE@PAVCGapiDraw@@@Z 004a7040 f   gapidraw:GapiSurface.obj
 0001:000a6080       ??_GCGapiSurface@@UAEPAXI@Z 004a7080 f i gapidraw:GapiSurface.obj
 0001:000a6080       ??_ECGapiSurface@@UAEPAXI@Z 004a7080 f i gapidraw:GapiSurface.obj
 0001:000a60b0       ??1CGapiSurface@@UAE@XZ    004a70b0 f   gapidraw:GapiSurface.obj
 0001:000a60c0       ?FreeResources@CGapiSurface@@IAEJXZ 004a70c0 f   gapidraw:GapiSurface.obj
 0001:000a6220       ?CreateSurface@CGapiSurface@@QAEJKKK@Z 004a7220 f   gapidraw:GapiSurface.obj
 0001:000a6be0       ?CreateSurface@CGapiSurface@@QAEJKPAEK@Z 004a7be0 f   gapidraw:GapiSurface.obj
 0001:000a6eb0       ?CreateSurface@CGapiSurface@@QAEJKPBD@Z 004a7eb0 f   gapidraw:GapiSurface.obj
 0001:000a7080       ?GetHeight@CGapiSurface@@QAEKXZ 004a8080 f   gapidraw:GapiSurface.obj
 0001:000a7090       ?SetColorKey@CGapiSurface@@QAEJK@Z 004a8090 f   gapidraw:GapiSurface.obj
 0001:000a7130       ?GetColorKey@CGapiSurface@@QAEJPAK@Z 004a8130 f   gapidraw:GapiSurface.obj
 0001:000a7150       ?GetDC@CGapiSurface@@QAEJPAPAUHDC__@@@Z 004a8150 f   gapidraw:GapiSurface.obj
 0001:000a7490       ?ReleaseDC@CGapiSurface@@QAEJPAUHDC__@@@Z 004a8490 f   gapidraw:GapiSurface.obj
 0001:000a7690       ?LockVideoSurface@CGapiSurface@@QAEJXZ 004a8690 f   gapidraw:GapiSurface.obj
 0001:000a7800       ?UnlockVideoSurface@CGapiSurface@@QAEJXZ 004a8800 f   gapidraw:GapiSurface.obj
 0001:000a7910       ?GetBuffer@CGapiSurface@@QAEJPAU_GDBUFFERDESC@@@Z 004a8910 f   gapidraw:GapiSurface.obj
 0001:000a7b00       ?ReleaseBuffer@CGapiSurface@@QAEJXZ 004a8b00 f   gapidraw:GapiSurface.obj
 0001:000a7c20       ?SaveSurface@CGapiSurface@@QAEJPBDK@Z 004a8c20 f   gapidraw:GapiSurface.obj
 0001:000a7e00       ?ColorrefToNative@CGapiSurface@@QAEJKPAK@Z 004a8e00 f   gapidraw:GapiSurface.obj
 0001:000a7eb0       ?GetPixel@CGapiSurface@@QAEJJJPAK@Z 004a8eb0 f   gapidraw:GapiSurface.obj
 0001:000a8120       ?SetPixel@CGapiSurface@@QAEJJJK@Z 004a9120 f   gapidraw:GapiSurface.obj
 0001:000a83e0       ?IsEmpty@CRect@@QBEHXZ     004a93e0 f i gapidraw:GapiSurface.obj
 0001:000a8400       ?PtInRect@CRect@@QBEHUtagPOINT@@@Z 004a9400 f i gapidraw:GapiSurface.obj
 0001:000a8430       ?SetRect@CRect@@QAEXJJJJ@Z 004a9430 f i gapidraw:GapiSurface.obj
 0001:000a8450       ?DrawLine@CGapiSurface@@QAEJJJJJKKPAU_GDLINEFX@@@Z 004a9450 f   gapidraw:GapiSurface.obj
 0001:000a8980       ??0CRect@@QAE@ABUtagRECT@@@Z 004a9980 f i gapidraw:GapiSurface.obj
 0001:000a89b0       ?BltFast@CGapiSurface@@QAEJJJPAV1@PAUtagRECT@@KPAU_GDBLTFASTFX@@@Z 004a99b0 f   gapidraw:GapiSurface.obj
 0001:000a9640       ??0CRect@@QAE@JJJJ@Z       004aa640 f i gapidraw:GapiSurface.obj
 0001:000a9660       ?Intersect@CRect@@QAEXPAUtagRECT@@@Z 004aa660 f i gapidraw:GapiSurface.obj
 0001:000a96d0       ?AlphaBlt@CGapiSurface@@QAEJPAUtagRECT@@PAVCGapiRGBASurface@@0KPAU_GDALPHABLTFX@@@Z 004aa6d0 f   gapidraw:GapiSurface.obj
 0001:000aa1a0       ?AlignVideoSurface@CGapiSurfaceHelper@@QAEXAAU_GDSURFACE@gdinternal@@JJ@Z 004ab1a0 f i gapidraw:GapiSurface.obj
 0001:000aa450       ?AlphaBltFast@CGapiSurface@@QAEJJJPAVCGapiRGBASurface@@PAUtagRECT@@KPAU_GDALPHABLTFASTFX@@@Z 004ab450 f   gapidraw:GapiSurface.obj
 0001:000aaa70       ?FillRect@CGapiSurface@@QAEJPAUtagRECT@@KKPAU_GDFILLRECTFX@@@Z 004aba70 f   gapidraw:GapiSurface.obj
 0001:000ab170       ?MemSetW@gdutil@@YAXPAGGK@Z 004ac170 f i gapidraw:GapiSurface.obj
 0001:000ab2b0       ?Blt@CGapiSurface@@QAEJPAUtagRECT@@PAV1@0KPAU_GDBLTFX@@@Z 004ac2b0 f   gapidraw:GapiSurface.obj
 0001:000ac610       ?Normalize@CRect@@QAEXXZ   004ad610 f i gapidraw:GapiSurface.obj
 0001:000ac630       ?DrawHLine@?$CGapiSurfaceAdapter@VCGapiDisplay555@@@@QAEJPAGKKJKKPAU_GDLINEFX@@@Z 004ad630 f i gapidraw:GapiSurface.obj
 0001:000ac630       ?DrawVLine@?$CGapiSurfaceAdapter@VCGapiDisplay555@@@@QAEJPAGKKJKKPAU_GDLINEFX@@@Z 004ad630 f i gapidraw:GapiSurface.obj
 0001:000ac870       ?DrawLine@gdblit@@YAJPAVCGapiSurfaceHelper@@PAGKKKKJJKKPAU_GDLINEFX@@@Z 004ad870 f i gapidraw:GapiSurface.obj
 0001:000acc10       ?FillRect@gdblit@@YAJPAVCGapiSurfaceHelper@@PAGJJJKPAU_GDFILLRECTFX@@K@Z 004adc10 f i gapidraw:GapiSurface.obj
 0001:000ace60       ?Blt@?$CGapiSurfaceAdapter@VCGapiDisplay555@@@@QAEJPAG0JJJJJJJJJKPAU_GDBLTFX@@K@Z 004ade60 f i gapidraw:GapiSurface.obj
 0001:000ad930       ?BltRot@?$CGapiSurfaceAdapter@VCGapiDisplay555@@@@QAEJPAG0JJJJJJJJKPAU_GDBLTFX@@KKAAVCPoint@@@Z 004ae930 f i gapidraw:GapiSurface.obj
 0001:000ae780       ?AlignRect@gdhw@@YAXPAVCGapiSurfaceHelper@@PAUtagRECT@@KK@Z 004af780 f i gapidraw:GapiSurface.obj
 0001:000ae850       ?Lock@gdhw@@YAJPAVCGapiSurfaceHelper@@AAU_GDSURFACE@gdinternal@@@Z 004af850 f i gapidraw:GapiSurface.obj
 0001:000aeae0       ?Unlock@gdhw@@YAJAAU_GDSURFACE@gdinternal@@@Z 004afae0 f i gapidraw:GapiSurface.obj
 0001:000aeb20       ?BltFast@?$CGapiSurfaceAdapter@VCGapiDisplay555@@@@QAEJPAG0JJJJKPAU_GDBLTFASTFX@@K@Z 004afb20 f i gapidraw:GapiSurface.obj
 0001:000b01e0       ?LockTemporary@CBufferLock@gdhw@@QAEJXZ 004b11e0 f i gapidraw:GapiSurface.obj
 0001:000b02c0       ??1CBufferLock@gdhw@@QAE@XZ 004b12c0 f i gapidraw:GapiSurface.obj
 0001:000b0370       ?DecodeBMP@gdbmp@@YAJPAVCGapiSurfaceHelper@@KAAVCGapiSurface@@PAEKK@Z 004b1370 f i gapidraw:GapiSurface.obj
 0001:000b18d0       ?BltFastFx@?$CGapiSurfaceAdapter@VCGapiDisplay555@@@@QAEJPAG0JJJJKPAU_GDBLTFASTFX@@K@Z 004b28d0 f i gapidraw:GapiSurface.obj
 0001:000b26c0       ?EncodeBMP@gdimage@@YAJPAVCGapiSurfaceHelper@@PAU_GDSURFACE@gdinternal@@PBD@Z 004b36c0 f i gapidraw:GapiSurface.obj
 0001:000b29c0       ?AlphaBlt16@?$CGapiSurfaceAdapter@VCGapiDisplay555@@@@QAEJPAG0JJJJJJJJJKPAU_GDALPHABLTFX@@@Z 004b39c0 f i gapidraw:GapiSurface.obj
 0001:000b2e50       ?EncodePNG@gdimage@@YAJPAVCGapiSurfaceHelper@@PAU_GDSURFACE@gdinternal@@PBD@Z 004b3e50 f i gapidraw:GapiSurface.obj
 0001:000b31c0       ?user_write_data@gdimage@@YAXPAUpng_struct_def@@PAEI@Z 004b41c0 f i gapidraw:GapiSurface.obj
 0001:000b3200       ?user_flush_data@gdimage@@YAXPAUpng_struct_def@@@Z 004b4200 f i gapidraw:GapiSurface.obj
 0001:000b3230       ?AlphaBltFast16@?$CGapiSurfaceAdapter@VCGapiDisplay555@@@@QAEJPAG0JJJJKPAU_GDALPHABLTFASTFX@@@Z 004b4230 f i gapidraw:GapiSurface.obj
 0001:000b39d0       ?DecodePNG@gdimage@@YAJPAVCGapiSurfaceHelper@@KAAVCGapiSurface@@PAEK@Z 004b49d0 f i gapidraw:GapiSurface.obj
 0001:000b42a0       ?UnlockPermanent@CBufferLock@gdhw@@QAEJXZ 004b52a0 f i gapidraw:GapiSurface.obj
 0001:000b4300       ??1CSimpleMemFile@gdalphaimage@@QAE@XZ 004b5300 f i gapidraw:GapiRGBASurface.obj
 0001:000b4300       ??1CSimpleMemFile@gdimage@@QAE@XZ 004b5300 f i gapidraw:GapiSurface.obj
 0001:000b4310       ?user_read_data@gdimage@@YAXPAUpng_struct_def@@PAEI@Z 004b5310 f i gapidraw:GapiSurface.obj
 0001:000b4310       ?user_read_data@gdalphaimage@@YAXPAUpng_struct_def@@PAEI@Z 004b5310 f i gapidraw:GapiRGBASurface.obj
 0001:000b4380       ?AlphaBltFast32@?$CGapiSurfaceAdapter@VCGapiDisplay555@@@@QAEJPAGPAKJJJJKPAU_GDALPHABLTFASTFX@@@Z 004b5380 f i gapidraw:GapiSurface.obj
 0001:000b46e0       ?CreateSurface@gdimage@@YAJPAVCGapiSurfaceHelper@@KAAVCGapiSurface@@PAEK@Z 004b56e0 f i gapidraw:GapiSurface.obj
 0001:000b4940       ?DrawVLine@?$CGapiSurfaceAdapter@VCGapiDisplay565@@@@QAEJPAGKKJKKPAU_GDLINEFX@@@Z 004b5940 f i gapidraw:GapiSurface.obj
 0001:000b4940       ?DrawHLine@?$CGapiSurfaceAdapter@VCGapiDisplay565@@@@QAEJPAGKKJKKPAU_GDLINEFX@@@Z 004b5940 f i gapidraw:GapiSurface.obj
 0001:000b4b70       ?Blt@?$CGapiSurfaceAdapter@VCGapiDisplay565@@@@QAEJPAG0JJJJJJJJJKPAU_GDBLTFX@@K@Z 004b5b70 f i gapidraw:GapiSurface.obj
 0001:000b55e0       ?BltRot@?$CGapiSurfaceAdapter@VCGapiDisplay565@@@@QAEJPAG0JJJJJJJJKPAU_GDBLTFX@@KKAAVCPoint@@@Z 004b65e0 f i gapidraw:GapiSurface.obj
 0001:000b6410       ?BltFast@?$CGapiSurfaceAdapter@VCGapiDisplay565@@@@QAEJPAG0JJJJKPAU_GDBLTFASTFX@@K@Z 004b7410 f i gapidraw:GapiSurface.obj
 0001:000b7a60       ?BltFastFx@?$CGapiSurfaceAdapter@VCGapiDisplay565@@@@QAEJPAG0JJJJKPAU_GDBLTFASTFX@@K@Z 004b8a60 f i gapidraw:GapiSurface.obj
 0001:000b8850       ?AlphaBlt16@?$CGapiSurfaceAdapter@VCGapiDisplay565@@@@QAEJPAG0JJJJJJJJJKPAU_GDALPHABLTFX@@@Z 004b9850 f i gapidraw:GapiSurface.obj
 0001:000b8ce0       ?AlphaBlt32@?$CGapiSurfaceAdapter@VCGapiDisplay565@@@@QAEJPAGPAKJJJJJJJJJKPAU_GDALPHABLTFX@@@Z 004b9ce0 f i gapidraw:GapiSurface.obj
 0001:000b9120       ?AlphaBltFast16@?$CGapiSurfaceAdapter@VCGapiDisplay565@@@@QAEJPAG0JJJJKPAU_GDALPHABLTFASTFX@@@Z 004ba120 f i gapidraw:GapiSurface.obj
 0001:000b98b0       ?AlphaBltFast32@?$CGapiSurfaceAdapter@VCGapiDisplay565@@@@QAEJPAGPAKJJJJKPAU_GDALPHABLTFASTFX@@@Z 004ba8b0 f i gapidraw:GapiSurface.obj
 0001:000b9c10       ?DrawLineAA@rasterop@@YAJAAV?$PixelAlphaBlend@VCGapiDisplay555@@@operators@@AAVAlphaOpacityFast@3@KKPAGKKKKJJ@Z 004bac10 f i gapidraw:GapiSurface.obj
 0001:000ba0d0       ?DrawLineAA@rasterop@@YAJAAV?$PixelAlphaBlend@VCGapiDisplay555@@@operators@@AAVAlphaOpacityNormal@3@KKPAGKKKKJJ@Z 004bb0d0 f i gapidraw:GapiSurface.obj
 0001:000ba5a0       ?DrawLineAA@rasterop@@YAJAAV?$PixelAlphaBlend@VCGapiDisplay555@@@operators@@AAVAlphaOpacityNone@3@KKPAGKKKKJJ@Z 004bb5a0 f i gapidraw:GapiSurface.obj
 0001:000baa60       ?DrawLine@rasterop@@YAJAAV?$PixelAlphaBlendFast@VCGapiDisplay555@@@operators@@KKPAGKKKKJJ@Z 004bba60 f i gapidraw:GapiSurface.obj
 0001:000babf0       ?DrawLine@rasterop@@YAJAAV?$PixelAlphaBlend@VCGapiDisplay555@@@operators@@KKPAGKKKKJJ@Z 004bbbf0 f i gapidraw:GapiSurface.obj
 0001:000baea0       ?DrawLine@rasterop@@YAJAAVPixelCopy@operators@@KKPAGKKKKJJ@Z 004bbea0 f i gapidraw:GapiSurface.obj
 0001:000bafe0       ?FillRect@rasterop@@YAJAAVCGapiDisplay555@@AAV?$PixelAlphaBlendFast@VCGapiDisplay555@@@operators@@AAV?$PixelAlphaBlendFast32@VCGapiDisplay555@@@4@KKPAGJJJ@Z 004bbfe0 f i gapidraw:GapiSurface.obj
 0001:000bb3a0       ?FillRect@rasterop@@YAJAAVCGapiDisplay555@@AAV?$PixelAlphaBlend@VCGapiDisplay555@@@operators@@AAV?$PixelAlphaBlend32@VCGapiDisplay555@@@4@KKPAGJJJ@Z 004bc3a0 f i gapidraw:GapiSurface.obj
 0001:000bc220       ?FillRect@rasterop@@YAJAAVCGapiDisplay555@@AAVPixelCopy@operators@@AAVPixelCopy32@4@KKPAGJJJ@Z 004bd220 f i gapidraw:GapiSurface.obj
 0001:000bc220       ?FillRect@rasterop@@YAJAAVCGapiDisplay565@@AAVPixelCopy@operators@@AAVPixelCopy32@4@KKPAGJJJ@Z 004bd220 f i gapidraw:GapiSurface.obj
 0001:000bc3e0       ?Blt@rasterop@@YAJAAVSourcePixel@operators@@AAVPredicateCopy@3@AAV?$PixelAlphaBlendFast@VCGapiDisplay555@@@3@KKKPAG3JJJJJJJJJ@Z 004bd3e0 f i gapidraw:GapiSurface.obj
 0001:000bc4c0       ?Blt@rasterop@@YAJAAVSourcePixel@operators@@AAVPredicateCopy@3@AAV?$PixelAlphaBlend@VCGapiDisplay555@@@3@KKKPAG3JJJJJJJJJ@Z 004bd4c0 f i gapidraw:GapiSurface.obj
 0001:000bc5f0       ?Blt@rasterop@@YAJAAVSourcePixel@operators@@AAVPredicateCopy@3@AAVPixelCopy@3@KKKPAG3JJJJJJJJJ@Z 004bd5f0 f i gapidraw:GapiSurface.obj
 0001:000bc6b0       ?BltRot@rasterop@@YAJAAVSourceColorfill@operators@@AAVPredicateDoNothing@3@AAV?$PixelAlphaBlend@VCGapiDisplay555@@@3@KKKJJPAG3JJJJJJJJJJ@Z 004bd6b0 f i gapidraw:GapiSurface.obj
 0001:000bc830       ?BltRot@rasterop@@YAJAAVSourceColorfill@operators@@AAVPredicateDoNothing@3@AAVPixelCopy@3@KKKJJPAG3JJJJJJJJJJ@Z 004bd830 f i gapidraw:GapiSurface.obj
 0001:000bc950       ?BltRot@rasterop@@YAJAAVSourcePixel@operators@@AAVPredicateCopy@3@AAV?$PixelAlphaBlendFast@VCGapiDisplay555@@@3@KKKJJPAG3JJJJJJJJJJ@Z 004bd950 f i gapidraw:GapiSurface.obj
 0001:000bcaa0       ?BltRot@rasterop@@YAJAAVSourcePixel@operators@@AAVPredicateCopy@3@AAV?$PixelAlphaBlend@VCGapiDisplay555@@@3@KKKJJPAG3JJJJJJJJJJ@Z 004bdaa0 f i gapidraw:GapiSurface.obj
 0001:000bcc40       ?BltRot@rasterop@@YAJAAVSourcePixel@operators@@AAVPredicateCopy@3@AAVPixelCopy@3@KKKJJPAG3JJJJJJJJJJ@Z 004bdc40 f i gapidraw:GapiSurface.obj
 0001:000bcd80       ?BltFastDU@rasterop@@YAJAAVSourceColorfill@operators@@AAVPredicateMask@3@AAVPredicateMask32a@3@AAVPredicateMask32b@3@AAVPredicateMask32bCheckOnly@3@AAV?$PixelAlphaBlendFast@VCGapiDisplay555@@@3@AAV?$PixelAlphaBlendFast32@VCGapiDisplay555@@@3@KKKPAG7JJJJ@Z 004bdd80 f i gapidraw:GapiSurface.obj
 0001:000bcef0       ?BltFastDU@rasterop@@YAJAAVSourceColorfill@operators@@AAVPredicateMask@3@AAVPredicateMask32a@3@AAVPredicateMask32b@3@AAVPredicateMask32bCheckOnly@3@AAV?$PixelAlphaBlend@VCGapiDisplay555@@@3@AAV?$PixelAlphaBlend32@VCGapiDisplay555@@@3@KKKPAG7JJJJ@Z 004bdef0 f i gapidraw:GapiSurface.obj
 0001:000bd150       ?BltFastDU@rasterop@@YAJAAVSourceColorfill@operators@@AAVPredicateMask@3@AAVPredicateMask32a@3@AAVPredicateMask32b@3@AAVPredicateMask32bCheckOnly@3@AAVPixelCopy@3@AAVPixelCopy32@3@KKKPAG7JJJJ@Z 004be150 f i gapidraw:GapiSurface.obj
 0001:000bd240       ?BltFastDU@rasterop@@YAJAAVSourcePixel@operators@@AAVPredicateMask@3@AAVPredicateMask32a@3@AAVPredicateMask32b@3@AAVPredicateMask32bCheckOnly@3@AAV?$PixelAlphaBlendFast@VCGapiDisplay555@@@3@AAV?$PixelAlphaBlendFast32@VCGapiDisplay555@@@3@KKKPAG7JJJJ@Z 004be240 f i gapidraw:GapiSurface.obj
 0001:000bd380       ?BltFastDU@rasterop@@YAJAAVSourcePixel@operators@@AAVPredicateMask@3@AAVPredicateMask32a@3@AAVPredicateMask32b@3@AAVPredicateMask32bCheckOnly@3@AAV?$PixelAlphaBlend@VCGapiDisplay555@@@3@AAV?$PixelAlphaBlend32@VCGapiDisplay555@@@3@KKKPAG7JJJJ@Z 004be380 f i gapidraw:GapiSurface.obj
 0001:000bd5e0       ?BltFastDU@rasterop@@YAJAAVSourcePixel@operators@@AAVPredicateMask@3@AAVPredicateMask32a@3@AAVPredicateMask32b@3@AAVPredicateMask32bCheckOnly@3@AAVPixelCopy@3@AAVPixelCopy32@3@KKKPAG7JJJJ@Z 004be5e0 f i gapidraw:GapiSurface.obj
 0001:000bd6d0       ?BltFastDU@rasterop@@YAJAAVSourcePixel@operators@@AAVPredicateCopy@3@AAVPredicateCopy32a@3@AAVPredicateCopy32b@3@AAVPredicateDoNothing32@3@AAV?$PixelAlphaBlendFast@VCGapiDisplay555@@@3@AAV?$PixelAlphaBlendFast32@VCGapiDisplay555@@@3@KKKPAG7JJJJ@Z 004be6d0 f i gapidraw:GapiSurface.obj
 0001:000bd7f0       ?BltFastDU@rasterop@@YAJAAVSourcePixel@operators@@AAVPredicateCopy@3@AAVPredicateCopy32a@3@AAVPredicateCopy32b@3@AAVPredicateDoNothing32@3@AAV?$PixelAlphaBlend@VCGapiDisplay555@@@3@AAV?$PixelAlphaBlend32@VCGapiDisplay555@@@3@KKKPAG7JJJJ@Z 004be7f0 f i gapidraw:GapiSurface.obj
 0001:000bd9e0       ?BltFastDU@rasterop@@YAJAAVSourcePixel@operators@@AAVPredicateCopy@3@AAVPredicateCopy32a@3@AAVPredicateCopy32b@3@AAVPredicateDoNothing32@3@AAVPixelCopy@3@AAVPixelCopy32@3@KKKPAG7JJJJ@Z 004be9e0 f i gapidraw:GapiSurface.obj
 0001:000bdaa0       ?BltFastSU@rasterop@@YAJAAVSourceColorfill@operators@@AAVPredicateMask@3@AAV?$PixelAlphaBlendFast@VCGapiDisplay555@@@3@KKKPAG3JJJJ@Z 004beaa0 f i gapidraw:GapiSurface.obj
 0001:000bdb40       ?BltFastSU@rasterop@@YAJAAVSourceColorfill@operators@@AAVPredicateMask@3@AAV?$PixelAlphaBlend@VCGapiDisplay555@@@3@KKKPAG3JJJJ@Z 004beb40 f i gapidraw:GapiSurface.obj
 0001:000bdc50       ?BltFastSU@rasterop@@YAJAAVSourceColorfill@operators@@AAVPredicateMask@3@AAVPixelCopy@3@KKKPAG3JJJJ@Z 004bec50 f i gapidraw:GapiSurface.obj
 0001:000bdcd0       ?BltFastSU@rasterop@@YAJAAVSourcePixel@operators@@AAVPredicateMask@3@AAV?$PixelAlphaBlendFast@VCGapiDisplay555@@@3@KKKPAG3JJJJ@Z 004becd0 f i gapidraw:GapiSurface.obj
 0001:000bdd70       ?BltFastSU@rasterop@@YAJAAVSourcePixel@operators@@AAVPredicateMask@3@AAV?$PixelAlphaBlend@VCGapiDisplay555@@@3@KKKPAG3JJJJ@Z 004bed70 f i gapidraw:GapiSurface.obj
 0001:000bde70       ?BltFastSU@rasterop@@YAJAAVSourcePixel@operators@@AAVPredicateMask@3@AAVPixelCopy@3@KKKPAG3JJJJ@Z 004bee70 f i gapidraw:GapiSurface.obj
 0001:000bdef0       ?BltFastSU@rasterop@@YAJAAVSourcePixel@operators@@AAVPredicateCopy@3@AAV?$PixelAlphaBlendFast@VCGapiDisplay555@@@3@KKKPAG3JJJJ@Z 004beef0 f i gapidraw:GapiSurface.obj
 0001:000bdf80       ?BltFastSU@rasterop@@YAJAAVSourcePixel@operators@@AAVPredicateCopy@3@AAV?$PixelAlphaBlend@VCGapiDisplay555@@@3@KKKPAG3JJJJ@Z 004bef80 f i gapidraw:GapiSurface.obj
 0001:000be070       ?BltFastSU@rasterop@@YAJAAVSourcePixel@operators@@AAVPredicateCopy@3@AAVPixelCopy@3@KKKPAG3JJJJ@Z 004bf070 f i gapidraw:GapiSurface.obj
 0001:000be0e0       ?AlphaBlt32@rasterop@@YAJAAVCGapiDisplay555@@AAVAlphaOpacityFast@operators@@KPAGPAKJJJJJJJJJ@Z 004bf0e0 f i gapidraw:GapiSurface.obj
 0001:000be230       ?AlphaBlt32@rasterop@@YAJAAVCGapiDisplay555@@AAVAlphaOpacityNormal@operators@@KPAGPAKJJJJJJJJJ@Z 004bf230 f i gapidraw:GapiSurface.obj
 0001:000be380       ?AlphaBlt32@rasterop@@YAJAAVCGapiDisplay555@@AAVAlphaOpacityNone@operators@@KPAGPAKJJJJJJJJJ@Z 004bf380 f i gapidraw:GapiSurface.obj
 0001:000be4d0       ?AlphaBltFast16SUDU@rasterop@@YAJAAVCGapiDisplay555@@AAVAlphaOpacityNormal@operators@@KPAG2JJJJ@Z 004bf4d0 f i gapidraw:GapiSurface.obj
 0001:000be960       ?AlphaBltFast16SUDU@rasterop@@YAJAAVCGapiDisplay555@@AAVAlphaOpacityNone@operators@@KPAG2JJJJ@Z 004bf960 f i gapidraw:GapiSurface.obj
 0001:000bedc0       ?AlphaBltFast16DU@rasterop@@YAJAAVCGapiDisplay555@@AAVAlphaOpacityFast@operators@@KPAG2JJJJ@Z 004bfdc0 f i gapidraw:GapiSurface.obj
 0001:000bf120       ?AlphaBltFast16DU@rasterop@@YAJAAVCGapiDisplay555@@AAVAlphaOpacityNormal@operators@@KPAG2JJJJ@Z 004c0120 f i gapidraw:GapiSurface.obj
 0001:000bf450       ?AlphaBltFast16DU@rasterop@@YAJAAVCGapiDisplay555@@AAVAlphaOpacityNone@operators@@KPAG2JJJJ@Z 004c0450 f i gapidraw:GapiSurface.obj
 0001:000bf760       ?AlphaBltFast16SU@rasterop@@YAJAAVCGapiDisplay555@@AAVAlphaOpacityNormal@operators@@KPAG2JJJJ@Z 004c0760 f i gapidraw:GapiSurface.obj
 0001:000bf890       ?AlphaBltFast16SU@rasterop@@YAJAAVCGapiDisplay555@@AAVAlphaOpacityNone@operators@@KPAG2JJJJ@Z 004c0890 f i gapidraw:GapiSurface.obj
 0001:000bf9b0       ?DrawLineAA@rasterop@@YAJAAV?$PixelAlphaBlend@VCGapiDisplay565@@@operators@@AAVAlphaOpacityFast@3@KKPAGKKKKJJ@Z 004c09b0 f i gapidraw:GapiSurface.obj
 0001:000bfe00       ?DrawLineAA@rasterop@@YAJAAV?$PixelAlphaBlend@VCGapiDisplay565@@@operators@@AAVAlphaOpacityNormal@3@KKPAGKKKKJJ@Z 004c0e00 f i gapidraw:GapiSurface.obj
 0001:000c0260       ?DrawLineAA@rasterop@@YAJAAV?$PixelAlphaBlend@VCGapiDisplay565@@@operators@@AAVAlphaOpacityNone@3@KKPAGKKKKJJ@Z 004c1260 f i gapidraw:GapiSurface.obj
 0001:000c06b0       ?DrawLine@rasterop@@YAJAAV?$PixelAlphaBlendFast@VCGapiDisplay565@@@operators@@KKPAGKKKKJJ@Z 004c16b0 f i gapidraw:GapiSurface.obj
 0001:000c0840       ?DrawLine@rasterop@@YAJAAV?$PixelAlphaBlend@VCGapiDisplay565@@@operators@@KKPAGKKKKJJ@Z 004c1840 f i gapidraw:GapiSurface.obj
 0001:000c0ac0       ?FillRect@rasterop@@YAJAAVCGapiDisplay565@@AAV?$PixelAlphaBlendFast@VCGapiDisplay565@@@operators@@AAV?$PixelAlphaBlendFast32@VCGapiDisplay565@@@4@KKPAGJJJ@Z 004c1ac0 f i gapidraw:GapiSurface.obj
 0001:000c0e80       ?FillRect@rasterop@@YAJAAVCGapiDisplay565@@AAV?$PixelAlphaBlend@VCGapiDisplay565@@@operators@@AAV?$PixelAlphaBlend32@VCGapiDisplay565@@@4@KKPAGJJJ@Z 004c1e80 f i gapidraw:GapiSurface.obj
 0001:000c1d00       ?Blt@rasterop@@YAJAAVSourcePixel@operators@@AAVPredicateCopy@3@AAV?$PixelAlphaBlendFast@VCGapiDisplay565@@@3@KKKPAG3JJJJJJJJJ@Z 004c2d00 f i gapidraw:GapiSurface.obj
 0001:000c1de0       ?Blt@rasterop@@YAJAAVSourcePixel@operators@@AAVPredicateCopy@3@AAV?$PixelAlphaBlend@VCGapiDisplay565@@@3@KKKPAG3JJJJJJJJJ@Z 004c2de0 f i gapidraw:GapiSurface.obj
 0001:000c1f10       ?BltRot@rasterop@@YAJAAVSourceColorfill@operators@@AAVPredicateDoNothing@3@AAV?$PixelAlphaBlend@VCGapiDisplay565@@@3@KKKJJPAG3JJJJJJJJJJ@Z 004c2f10 f i gapidraw:GapiSurface.obj
 0001:000c2090       ?BltRot@rasterop@@YAJAAVSourcePixel@operators@@AAVPredicateCopy@3@AAV?$PixelAlphaBlendFast@VCGapiDisplay565@@@3@KKKJJPAG3JJJJJJJJJJ@Z 004c3090 f i gapidraw:GapiSurface.obj
 0001:000c21e0       ?BltRot@rasterop@@YAJAAVSourcePixel@operators@@AAVPredicateCopy@3@AAV?$PixelAlphaBlend@VCGapiDisplay565@@@3@KKKJJPAG3JJJJJJJJJJ@Z 004c31e0 f i gapidraw:GapiSurface.obj
 0001:000c2380       ?BltFastSUDU@rasterop@@YAJAAVCGapiDisplay555@@AAVSourcePixel@operators@@AAVPredicateCopy@4@AAVPredicateCopy32a@4@AAVPredicateCopy32b@4@AAVPredicateDoNothing32@4@AAVPixelCopy@4@AAVPixelCopy32@4@KKKPAG8JJJJ@Z 004c3380 f i gapidraw:GapiSurface.obj
 0001:000c2380       ?BltFastSUDU@rasterop@@YAJAAVCGapiDisplay565@@AAVSourcePixel@operators@@AAVPredicateCopy@4@AAVPredicateCopy32a@4@AAVPredicateCopy32b@4@AAVPredicateDoNothing32@4@AAVPixelCopy@4@AAVPixelCopy32@4@KKKPAG8JJJJ@Z 004c3380 f i gapidraw:GapiSurface.obj
 0001:000c2490       ?BltFastDU@rasterop@@YAJAAVSourceColorfill@operators@@AAVPredicateMask@3@AAVPredicateMask32a@3@AAVPredicateMask32b@3@AAVPredicateMask32bCheckOnly@3@AAV?$PixelAlphaBlendFast@VCGapiDisplay565@@@3@AAV?$PixelAlphaBlendFast32@VCGapiDisplay565@@@3@KKKPAG7JJJJ@Z 004c3490 f i gapidraw:GapiSurface.obj
 0001:000c2600       ?BltFastDU@rasterop@@YAJAAVSourceColorfill@operators@@AAVPredicateMask@3@AAVPredicateMask32a@3@AAVPredicateMask32b@3@AAVPredicateMask32bCheckOnly@3@AAV?$PixelAlphaBlend@VCGapiDisplay565@@@3@AAV?$PixelAlphaBlend32@VCGapiDisplay565@@@3@KKKPAG7JJJJ@Z 004c3600 f i gapidraw:GapiSurface.obj
 0001:000c2870       ?BltFastDU@rasterop@@YAJAAVSourcePixel@operators@@AAVPredicateMask@3@AAVPredicateMask32a@3@AAVPredicateMask32b@3@AAVPredicateMask32bCheckOnly@3@AAV?$PixelAlphaBlendFast@VCGapiDisplay565@@@3@AAV?$PixelAlphaBlendFast32@VCGapiDisplay565@@@3@KKKPAG7JJJJ@Z 004c3870 f i gapidraw:GapiSurface.obj
 0001:000c29b0       ?BltFastDU@rasterop@@YAJAAVSourcePixel@operators@@AAVPredicateMask@3@AAVPredicateMask32a@3@AAVPredicateMask32b@3@AAVPredicateMask32bCheckOnly@3@AAV?$PixelAlphaBlend@VCGapiDisplay565@@@3@AAV?$PixelAlphaBlend32@VCGapiDisplay565@@@3@KKKPAG7JJJJ@Z 004c39b0 f i gapidraw:GapiSurface.obj
 0001:000c2c10       ?BltFastDU@rasterop@@YAJAAVSourcePixel@operators@@AAVPredicateCopy@3@AAVPredicateCopy32a@3@AAVPredicateCopy32b@3@AAVPredicateDoNothing32@3@AAV?$PixelAlphaBlendFast@VCGapiDisplay565@@@3@AAV?$PixelAlphaBlendFast32@VCGapiDisplay565@@@3@KKKPAG7JJJJ@Z 004c3c10 f i gapidraw:GapiSurface.obj
 0001:000c2d30       ?BltFastDU@rasterop@@YAJAAVSourcePixel@operators@@AAVPredicateCopy@3@AAVPredicateCopy32a@3@AAVPredicateCopy32b@3@AAVPredicateDoNothing32@3@AAV?$PixelAlphaBlend@VCGapiDisplay565@@@3@AAV?$PixelAlphaBlend32@VCGapiDisplay565@@@3@KKKPAG7JJJJ@Z 004c3d30 f i gapidraw:GapiSurface.obj
 0001:000c2f20       ?BltFastSU@rasterop@@YAJAAVSourceColorfill@operators@@AAVPredicateMask@3@AAV?$PixelAlphaBlendFast@VCGapiDisplay565@@@3@KKKPAG3JJJJ@Z 004c3f20 f i gapidraw:GapiSurface.obj
 0001:000c2fc0       ?BltFastSU@rasterop@@YAJAAVSourceColorfill@operators@@AAVPredicateMask@3@AAV?$PixelAlphaBlend@VCGapiDisplay565@@@3@KKKPAG3JJJJ@Z 004c3fc0 f i gapidraw:GapiSurface.obj
 0001:000c30c0       ?BltFastSU@rasterop@@YAJAAVSourcePixel@operators@@AAVPredicateMask@3@AAV?$PixelAlphaBlendFast@VCGapiDisplay565@@@3@KKKPAG3JJJJ@Z 004c40c0 f i gapidraw:GapiSurface.obj
 0001:000c3160       ?BltFastSU@rasterop@@YAJAAVSourcePixel@operators@@AAVPredicateMask@3@AAV?$PixelAlphaBlend@VCGapiDisplay565@@@3@KKKPAG3JJJJ@Z 004c4160 f i gapidraw:GapiSurface.obj
 0001:000c3260       ?BltFastSU@rasterop@@YAJAAVSourcePixel@operators@@AAVPredicateCopy@3@AAV?$PixelAlphaBlendFast@VCGapiDisplay565@@@3@KKKPAG3JJJJ@Z 004c4260 f i gapidraw:GapiSurface.obj
 0001:000c32f0       ?BltFastSU@rasterop@@YAJAAVSourcePixel@operators@@AAVPredicateCopy@3@AAV?$PixelAlphaBlend@VCGapiDisplay565@@@3@KKKPAG3JJJJ@Z 004c42f0 f i gapidraw:GapiSurface.obj
 0001:000c33e0       ?AlphaBltFast16SUDU@rasterop@@YAJAAVCGapiDisplay565@@AAVAlphaOpacityNormal@operators@@KPAG2JJJJ@Z 004c43e0 f i gapidraw:GapiSurface.obj
 0001:000c3870       ?AlphaBltFast16SUDU@rasterop@@YAJAAVCGapiDisplay565@@AAVAlphaOpacityNone@operators@@KPAG2JJJJ@Z 004c4870 f i gapidraw:GapiSurface.obj
 0001:000c3cc0       ?AlphaBltFast16DU@rasterop@@YAJAAVCGapiDisplay565@@AAVAlphaOpacityFast@operators@@KPAG2JJJJ@Z 004c4cc0 f i gapidraw:GapiSurface.obj
 0001:000c4010       ?AlphaBltFast16DU@rasterop@@YAJAAVCGapiDisplay565@@AAVAlphaOpacityNormal@operators@@KPAG2JJJJ@Z 004c5010 f i gapidraw:GapiSurface.obj
 0001:000c4330       ?AlphaBltFast16DU@rasterop@@YAJAAVCGapiDisplay565@@AAVAlphaOpacityNone@operators@@KPAG2JJJJ@Z 004c5330 f i gapidraw:GapiSurface.obj
 0001:000c4630       ?AlphaBltFast16SU@rasterop@@YAJAAVCGapiDisplay565@@AAVAlphaOpacityNormal@operators@@KPAG2JJJJ@Z 004c5630 f i gapidraw:GapiSurface.obj
 0001:000c4760       ?AlphaBltFast16SU@rasterop@@YAJAAVCGapiDisplay565@@AAVAlphaOpacityNone@operators@@KPAG2JJJJ@Z 004c5760 f i gapidraw:GapiSurface.obj
 0001:000c4880       ??0CGapiTimer@@QAE@PAVCGapiDraw@@@Z 004c5880 f   gapidraw:GapiTimer.obj
 0001:000c48b0       ??_ECGapiTimer@@UAEPAXI@Z  004c58b0 f i gapidraw:GapiTimer.obj
 0001:000c48b0       ??_GCGapiTimer@@UAEPAXI@Z  004c58b0 f i gapidraw:GapiTimer.obj
 0001:000c4900       ?StartTimer@CGapiTimer@@QAEJK@Z 004c5900 f   gapidraw:GapiTimer.obj
 0001:000c4a40       ?UpdateTimer@CGapiTimer@@QAEJXZ 004c5a40 f   gapidraw:GapiTimer.obj
 0001:000c4c10       ??0CGapiInput@@QAE@PAVCGapiDraw@@@Z 004c5c10 f   gapidraw:GapiInputWin32.obj
 0001:000c4c30       ??_GCGapiInput@@UAEPAXI@Z  004c5c30 f i gapidraw:GapiInputWin32.obj
 0001:000c4c30       ??_ECGapiInput@@UAEPAXI@Z  004c5c30 f i gapidraw:GapiInputWin32.obj
 0001:000c4cb0       ?GetKeyList@CGapiInput@@QAEJPAU_GDKEYLIST@@@Z 004c5cb0 f   gapidraw:GapiInputWin32.obj
 0001:000c4d40       ?OpenInput@CGapiInput@@QAEJXZ 004c5d40 f   gapidraw:GapiInputWin32.obj
 0001:000c4e50       ?CloseInput@CGapiInput@@QAEJXZ 004c5e50 f   gapidraw:GapiInputWin32.obj
 0001:000c4ec0       ?DeviceToLogical@gdinput@@YAKPAVCGapiSurfaceHelper@@K@Z 004c5ec0 f   gapidraw:GapiInputWin32.obj
 0001:000c5050       ?instance@?1??GetInstance@CGapiLib@@SAPAV1@XZ@$AV1@A 004c6050 f i gapidraw:GapiInputWin32.obj
 0001:000c5080       ??_GCGapiLib@@UAEPAXI@Z    004c6080 f i gapidraw:GapiInputWin32.obj
 0001:000c5080       ??_ECGapiLib@@UAEPAXI@Z    004c6080 f i gapidraw:GapiInputWin32.obj
 0001:000c50c0       ??0CGapiDraw@@QAE@XZ       004c60c0 f   gapidraw:GapiDraw.obj
 0001:000c5330       ??_ECGapiDraw@@UAEPAXI@Z   004c6330 f i gapidraw:GapiDraw.obj
 0001:000c5330       ??_GCGapiDraw@@UAEPAXI@Z   004c6330 f i gapidraw:GapiDraw.obj
 0001:000c5360       ?FreeResources@CGapiDraw@@AAEXXZ 004c6360 f   gapidraw:GapiDraw.obj
 0001:000c53e0       ?IsInitialized@CGapiDraw@@QAEHXZ 004c63e0 f   gapidraw:GapiDraw.obj
 0001:000c53f0       ??0?$CGapiSurfaceAdapter@VCGapiDisplay555@@@@QAE@XZ 004c63f0 f i gapidraw:GapiDraw.obj
 0001:000c54c0       ??_E?$CGapiSurfaceAdapter@VCGapiDisplay555@@@@UAEPAXI@Z 004c64c0 f i gapidraw:GapiDraw.obj
 0001:000c54c0       ??_G?$CGapiSurfaceAdapter@VCGapiDisplay555@@@@UAEPAXI@Z 004c64c0 f i gapidraw:GapiDraw.obj
 0001:000c54e0       ??1?$CGapiSurfaceAdapter@VCGapiDisplay555@@@@UAE@XZ 004c64e0 f i gapidraw:GapiDraw.obj
 0001:000c55b0       ??_E?$PixelAlphaBlend@VCGapiDisplay555@@@operators@@UAEPAXI@Z 004c65b0 f i gapidraw:GapiDraw.obj
 0001:000c55b0       ??_G?$PixelAlphaBlend@VCGapiDisplay555@@@operators@@UAEPAXI@Z 004c65b0 f i gapidraw:GapiDraw.obj
 0001:000c55d0       ??1?$PixelAlphaBlend@VCGapiDisplay555@@@operators@@UAE@XZ 004c65d0 f i gapidraw:GapiDraw.obj
 0001:000c55e0       ??_G?$PixelAlphaBlend32@VCGapiDisplay555@@@operators@@UAEPAXI@Z 004c65e0 f i gapidraw:GapiDraw.obj
 0001:000c55e0       ??_E?$PixelAlphaBlend32@VCGapiDisplay555@@@operators@@UAEPAXI@Z 004c65e0 f i gapidraw:GapiDraw.obj
 0001:000c5600       ??1?$PixelAlphaBlend32@VCGapiDisplay555@@@operators@@UAE@XZ 004c6600 f i gapidraw:GapiDraw.obj
 0001:000c5610       ??_E?$PixelAlphaBlendFast@VCGapiDisplay555@@@operators@@UAEPAXI@Z 004c6610 f i gapidraw:GapiDraw.obj
 0001:000c5610       ??_G?$PixelAlphaBlendFast@VCGapiDisplay555@@@operators@@UAEPAXI@Z 004c6610 f i gapidraw:GapiDraw.obj
 0001:000c5630       ??1?$PixelAlphaBlendFast@VCGapiDisplay555@@@operators@@UAE@XZ 004c6630 f i gapidraw:GapiDraw.obj
 0001:000c5640       ??_E?$PixelAlphaBlendFast32@VCGapiDisplay555@@@operators@@UAEPAXI@Z 004c6640 f i gapidraw:GapiDraw.obj
 0001:000c5640       ??_G?$PixelAlphaBlendFast32@VCGapiDisplay555@@@operators@@UAEPAXI@Z 004c6640 f i gapidraw:GapiDraw.obj
 0001:000c5660       ??1?$PixelAlphaBlendFast32@VCGapiDisplay555@@@operators@@UAE@XZ 004c6660 f i gapidraw:GapiDraw.obj
 0001:000c5670       ??0?$CGapiSurfaceAdapter@VCGapiDisplay565@@@@QAE@XZ 004c6670 f i gapidraw:GapiDraw.obj
 0001:000c5740       ??_E?$CGapiSurfaceAdapter@VCGapiDisplay565@@@@UAEPAXI@Z 004c6740 f i gapidraw:GapiDraw.obj
 0001:000c5740       ??_G?$CGapiSurfaceAdapter@VCGapiDisplay565@@@@UAEPAXI@Z 004c6740 f i gapidraw:GapiDraw.obj
 0001:000c5760       ??1?$CGapiSurfaceAdapter@VCGapiDisplay565@@@@UAE@XZ 004c6760 f i gapidraw:GapiDraw.obj
 0001:000c5830       ??_E?$PixelAlphaBlend@VCGapiDisplay565@@@operators@@UAEPAXI@Z 004c6830 f i gapidraw:GapiDraw.obj
 0001:000c5830       ??_G?$PixelAlphaBlend@VCGapiDisplay565@@@operators@@UAEPAXI@Z 004c6830 f i gapidraw:GapiDraw.obj
 0001:000c5850       ??1?$PixelAlphaBlend@VCGapiDisplay565@@@operators@@UAE@XZ 004c6850 f i gapidraw:GapiDraw.obj
 0001:000c5860       ??_G?$PixelAlphaBlend32@VCGapiDisplay565@@@operators@@UAEPAXI@Z 004c6860 f i gapidraw:GapiDraw.obj
 0001:000c5860       ??_E?$PixelAlphaBlend32@VCGapiDisplay565@@@operators@@UAEPAXI@Z 004c6860 f i gapidraw:GapiDraw.obj
 0001:000c5880       ??1?$PixelAlphaBlend32@VCGapiDisplay565@@@operators@@UAE@XZ 004c6880 f i gapidraw:GapiDraw.obj
 0001:000c5890       ??_E?$PixelAlphaBlendFast@VCGapiDisplay565@@@operators@@UAEPAXI@Z 004c6890 f i gapidraw:GapiDraw.obj
 0001:000c5890       ??_G?$PixelAlphaBlendFast@VCGapiDisplay565@@@operators@@UAEPAXI@Z 004c6890 f i gapidraw:GapiDraw.obj
 0001:000c58b0       ??1?$PixelAlphaBlendFast@VCGapiDisplay565@@@operators@@UAE@XZ 004c68b0 f i gapidraw:GapiDraw.obj
 0001:000c58c0       ??_E?$PixelAlphaBlendFast32@VCGapiDisplay565@@@operators@@UAEPAXI@Z 004c68c0 f i gapidraw:GapiDraw.obj
 0001:000c58c0       ??_G?$PixelAlphaBlendFast32@VCGapiDisplay565@@@operators@@UAEPAXI@Z 004c68c0 f i gapidraw:GapiDraw.obj
 0001:000c58e0       ??1?$PixelAlphaBlendFast32@VCGapiDisplay565@@@operators@@UAE@XZ 004c68e0 f i gapidraw:GapiDraw.obj
 0001:000c58f0       ?CreateFontA@CGapiSurfaceHelper@@QAEXXZ 004c68f0 f i gapidraw:GapiDraw.obj
 0001:000c78c0       ??_ECGapiSurfaceHelper@@UAEPAXI@Z 004c88c0 f i gapidraw:GapiDraw.obj
 0001:000c78c0       ??_GCGapiSurfaceHelper@@UAEPAXI@Z 004c88c0 f i gapidraw:GapiDraw.obj
 0001:000c78e0       ??_ESourcePixel@operators@@UAEPAXI@Z 004c88e0 f i gapidraw:GapiDraw.obj
 0001:000c78e0       ??_GSourcePixel@operators@@UAEPAXI@Z 004c88e0 f i gapidraw:GapiDraw.obj
 0001:000c7900       ??_ESourceColorfill@operators@@UAEPAXI@Z 004c8900 f i gapidraw:GapiDraw.obj
 0001:000c7900       ??_GSourceColorfill@operators@@UAEPAXI@Z 004c8900 f i gapidraw:GapiDraw.obj
 0001:000c7920       ??_EPredicateMask@operators@@UAEPAXI@Z 004c8920 f i gapidraw:GapiDraw.obj
 0001:000c7920       ??_GPredicateMask@operators@@UAEPAXI@Z 004c8920 f i gapidraw:GapiDraw.obj
 0001:000c7940       ??_EPredicateMask32a@operators@@UAEPAXI@Z 004c8940 f i gapidraw:GapiDraw.obj
 0001:000c7940       ??_GPredicateMask32a@operators@@UAEPAXI@Z 004c8940 f i gapidraw:GapiDraw.obj
 0001:000c7960       ??_GPredicateMask32b@operators@@UAEPAXI@Z 004c8960 f i gapidraw:GapiDraw.obj
 0001:000c7960       ??_EPredicateMask32b@operators@@UAEPAXI@Z 004c8960 f i gapidraw:GapiDraw.obj
 0001:000c7980       ??_EPredicateMask32bCheckOnly@operators@@UAEPAXI@Z 004c8980 f i gapidraw:GapiDraw.obj
 0001:000c7980       ??_GPredicateMask32bCheckOnly@operators@@UAEPAXI@Z 004c8980 f i gapidraw:GapiDraw.obj
 0001:000c79a0       ??_GPredicateCopy@operators@@UAEPAXI@Z 004c89a0 f i gapidraw:GapiDraw.obj
 0001:000c79a0       ??_EPredicateCopy@operators@@UAEPAXI@Z 004c89a0 f i gapidraw:GapiDraw.obj
 0001:000c79c0       ??_GPredicateCopy32a@operators@@UAEPAXI@Z 004c89c0 f i gapidraw:GapiDraw.obj
 0001:000c79c0       ??_EPredicateCopy32a@operators@@UAEPAXI@Z 004c89c0 f i gapidraw:GapiDraw.obj
 0001:000c79e0       ??_GPredicateCopy32b@operators@@UAEPAXI@Z 004c89e0 f i gapidraw:GapiDraw.obj
 0001:000c79e0       ??_EPredicateCopy32b@operators@@UAEPAXI@Z 004c89e0 f i gapidraw:GapiDraw.obj
 0001:000c7a00       ??_EPredicateDoNothing@operators@@UAEPAXI@Z 004c8a00 f i gapidraw:GapiDraw.obj
 0001:000c7a00       ??_GPredicateDoNothing@operators@@UAEPAXI@Z 004c8a00 f i gapidraw:GapiDraw.obj
 0001:000c7a20       ??_EPredicateDoNothing32@operators@@UAEPAXI@Z 004c8a20 f i gapidraw:GapiDraw.obj
 0001:000c7a20       ??_GPredicateDoNothing32@operators@@UAEPAXI@Z 004c8a20 f i gapidraw:GapiDraw.obj
 0001:000c7a40       ??_GPixelCopy@operators@@UAEPAXI@Z 004c8a40 f i gapidraw:GapiDraw.obj
 0001:000c7a40       ??_EPixelCopy@operators@@UAEPAXI@Z 004c8a40 f i gapidraw:GapiDraw.obj
 0001:000c7a60       ??_GPixelCopy32@operators@@UAEPAXI@Z 004c8a60 f i gapidraw:GapiDraw.obj
 0001:000c7a60       ??_EPixelCopy32@operators@@UAEPAXI@Z 004c8a60 f i gapidraw:GapiDraw.obj
 0001:000c7a80       ??_GAlphaOpacityNone@operators@@UAEPAXI@Z 004c8a80 f i gapidraw:GapiDraw.obj
 0001:000c7a80       ??_EAlphaOpacityNone@operators@@UAEPAXI@Z 004c8a80 f i gapidraw:GapiDraw.obj
 0001:000c7aa0       ??_GAlphaOpacityFast@operators@@UAEPAXI@Z 004c8aa0 f i gapidraw:GapiDraw.obj
 0001:000c7aa0       ??_EAlphaOpacityFast@operators@@UAEPAXI@Z 004c8aa0 f i gapidraw:GapiDraw.obj
 0001:000c7ac0       ??_GAlphaOpacityNormal@operators@@UAEPAXI@Z 004c8ac0 f i gapidraw:GapiDraw.obj
 0001:000c7ac0       ??_EAlphaOpacityNormal@operators@@UAEPAXI@Z 004c8ac0 f i gapidraw:GapiDraw.obj
 0001:000c7ae0       ??_GCoordNormal@operators@@UAEPAXI@Z 004c8ae0 f i gapidraw:GapiDraw.obj
 0001:000c7ae0       ??_ECoordNormal@operators@@UAEPAXI@Z 004c8ae0 f i gapidraw:GapiDraw.obj
 0001:000c7b00       ??_GCoordFixedPoint@operators@@UAEPAXI@Z 004c8b00 f i gapidraw:GapiDraw.obj
 0001:000c7b00       ??_ECoordFixedPoint@operators@@UAEPAXI@Z 004c8b00 f i gapidraw:GapiDraw.obj
 0001:000c7b20       ??_GCoordVerify@operators@@UAEPAXI@Z 004c8b20 f i gapidraw:GapiDraw.obj
 0001:000c7b20       ??_ECoordVerify@operators@@UAEPAXI@Z 004c8b20 f i gapidraw:GapiDraw.obj
 0001:000c7b40       ??_GCoordAcceptInvalid@operators@@UAEPAXI@Z 004c8b40 f i gapidraw:GapiDraw.obj
 0001:000c7b40       ??_ECoordAcceptInvalid@operators@@UAEPAXI@Z 004c8b40 f i gapidraw:GapiDraw.obj
 0001:000c7b60       ??_ECGapiDisplay555@@UAEPAXI@Z 004c8b60 f i gapidraw:GapiDraw.obj
 0001:000c7b60       ??_GCGapiDisplay555@@UAEPAXI@Z 004c8b60 f i gapidraw:GapiDraw.obj
 0001:000c7b80       ??_GCGapiDisplay565@@UAEPAXI@Z 004c8b80 f i gapidraw:GapiDraw.obj
 0001:000c7b80       ??_ECGapiDisplay565@@UAEPAXI@Z 004c8b80 f i gapidraw:GapiDraw.obj
 0001:000c7ba0       ??0CGapiDisplay@@QAE@PAVCGapiDraw@@@Z 004c8ba0 f   gapidraw:GapiDisplayDDraw.obj
 0001:000c7c60       ??_GCGapiDisplay@@UAEPAXI@Z 004c8c60 f i gapidraw:GapiDisplayDDraw.obj
 0001:000c7c60       ??_ECGapiDisplay@@UAEPAXI@Z 004c8c60 f i gapidraw:GapiDisplayDDraw.obj
 0001:000c7c80       ??1CGapiDisplay@@UAE@XZ    004c8c80 f   gapidraw:GapiDisplayDDraw.obj
 0001:000c7d60       ?CloseDisplay@CGapiDisplay@@QAEJXZ 004c8d60 f   gapidraw:GapiDisplayDDraw.obj
 0001:000c7de0       ?OpenDisplay@CGapiDisplay@@QAEJKPAUHWND__@@KKKKKK@Z 004c8de0 f   gapidraw:GapiDisplayDDraw.obj
 0001:000c87b0       ?PrepareSurfaceBitFormat@CColorConverter@gddisplay@@IAEXKPAK0@Z 004c97b0 f i gapidraw:GapiDisplayDDraw.obj
 0001:000c8800       ?GetBackBuffer@CGapiDisplay@@QAEPAVCGapiSurface@@XZ 004c9800 f   gapidraw:GapiDisplayDDraw.obj
 0001:000c8840       ?Flip@CGapiDisplay@@QAEJXZ 004c9840 f   gapidraw:GapiDisplayDDraw.obj
 0001:000c8ca0       ?SuspendDisplay@CGapiDisplay@@QAEJXZ 004c9ca0 f   gapidraw:GapiDisplayDDraw.obj
 0001:000c8d00       ?ResumeDisplay@CGapiDisplay@@QAEJXZ 004c9d00 f   gapidraw:GapiDisplayDDraw.obj
 0001:000c8d60       ?SetDisplayMode@CGapiDisplay@@QAEJK@Z 004c9d60 f   gapidraw:GapiDisplayDDraw.obj
 0001:000c90b0       ?GetHWStatus@CGapiDisplay@@QAEJPAK@Z 004ca0b0 f   gapidraw:GapiDisplayDDraw.obj
 0001:000c9110       ?SurfacesAreLost@CGapiDisplay@@QAEJXZ 004ca110 f   gapidraw:GapiDisplayDDraw.obj
 0001:000c9140       ?RestoreAllVideoSurfaces@CGapiDisplay@@QAEJXZ 004ca140 f   gapidraw:GapiDisplayDDraw.obj
 0001:000c91a0       ?DeviceToLogical@CGapiDisplay@@QAEJPAUtagPOINT@@@Z 004ca1a0 f   gapidraw:GapiDisplayDDraw.obj
 0001:000c9370       _png_error                 004ca370 f   gapidraw:pngerror.obj
 0001:000c9480       _png_warning               004ca480 f   gapidraw:pngerror.obj
 0001:000c9540       _png_chunk_error           004ca540 f   gapidraw:pngerror.obj
 0001:000c9600       _png_chunk_warning         004ca600 f   gapidraw:pngerror.obj
 0001:000c96d0       _png_set_error_fn          004ca6d0 f   gapidraw:pngerror.obj
 0001:000c96f0       _png_sig_cmp               004ca6f0 f   gapidraw:png.obj
 0001:000c9770       _png_zalloc                004ca770 f   gapidraw:png.obj
 0001:000c97f0       _png_zfree                 004ca7f0 f   gapidraw:png.obj
 0001:000c9810       _png_reset_crc             004ca810 f   gapidraw:png.obj
 0001:000c9830       _png_calculate_crc         004ca830 f   gapidraw:png.obj
 0001:000c9880       _png_create_info_struct    004ca880 f   gapidraw:png.obj
 0001:000c98c0       _png_free_data             004ca8c0 f   gapidraw:png.obj
 0001:000c9c80       _png_info_destroy          004cac80 f   gapidraw:png.obj
 0001:000c9ce0       _png_get_io_ptr            004cace0 f   gapidraw:png.obj
 0001:000c9cf0       _png_handle_as_unknown     004cacf0 f   gapidraw:png.obj
 0001:000c9d40       _png_init_mmx_flags        004cad40 f   gapidraw:png.obj
 0001:000c9d70       _png_create_read_struct    004cad70 f   gapidraw:pngread.obj
 0001:000c9da0       _png_create_read_struct_2  004cada0 f   gapidraw:pngread.obj
 0001:000c9fc0       _png_read_info             004cafc0 f   gapidraw:pngread.obj
 0001:000ca380       _png_read_update_info      004cb380 f   gapidraw:pngread.obj
 0001:000ca3d0       _png_read_row              004cb3d0 f   gapidraw:pngread.obj
 0001:000ca860       _png_destroy_read_struct   004cb860 f   gapidraw:pngread.obj
 0001:000ca920       _png_read_destroy          004cb920 f   gapidraw:pngread.obj
 0001:000cab90       _png_set_packing           004cbb90 f   gapidraw:pngtrans.obj
 0001:000cabb0       _png_set_interlace_handling 004cbbb0 f   gapidraw:pngtrans.obj
 0001:000cabe0       _png_set_filler            004cbbe0 f   gapidraw:pngtrans.obj
 0001:000cac40       _png_do_invert             004cbc40 f   gapidraw:pngtrans.obj
 0001:000cacd0       _png_do_swap               004cbcd0 f   gapidraw:pngtrans.obj
 0001:000cad00       _png_do_packswap           004cbd00 f   gapidraw:pngtrans.obj
 0001:000cad50       _png_do_strip_filler       004cbd50 f   gapidraw:pngtrans.obj
 0001:000caf60       _png_do_bgr                004cbf60 f   gapidraw:pngtrans.obj
 0001:000cb030       _png_set_strip_16          004cc030 f   gapidraw:pngrtran.obj
 0001:000cb040       _png_set_gray_1_2_4_to_8   004cc040 f   gapidraw:pngrtran.obj
 0001:000cb040       _png_set_expand            004cc040 f   gapidraw:pngrtran.obj
 0001:000cb040       _png_set_tRNS_to_alpha     004cc040 f   gapidraw:pngrtran.obj
 0001:000cb050       _png_set_gray_to_rgb       004cc050 f   gapidraw:pngrtran.obj
 0001:000cb060       _png_init_read_transformations 004cc060 f   gapidraw:pngrtran.obj
 0001:000cbaf0       _png_read_transform_info   004ccaf0 f   gapidraw:pngrtran.obj
 0001:000cbc80       _png_do_read_transformations 004ccc80 f   gapidraw:pngrtran.obj
 0001:000cc120       _png_do_unpack             004cd120 f   gapidraw:pngrtran.obj
 0001:000cc250       _png_do_unshift            004cd250 f   gapidraw:pngrtran.obj
 0001:000cc430       _png_do_read_swap_alpha    004cd430 f   gapidraw:pngrtran.obj
 0001:000cc530       _png_do_read_invert_alpha  004cd530 f   gapidraw:pngrtran.obj
 0001:000cc600       _png_do_read_filler        004cd600 f   gapidraw:pngrtran.obj
 0001:000cc870       _png_do_gray_to_rgb        004cd870 f   gapidraw:pngrtran.obj
 0001:000cc9b0       _png_do_rgb_to_gray        004cd9b0 f   gapidraw:pngrtran.obj
 0001:000cd100       _png_do_background         004ce100 f   gapidraw:pngrtran.obj
 0001:000ce100       _png_do_gamma              004cf100 f   gapidraw:pngrtran.obj
 0001:000ce4f0       _png_do_expand_palette     004cf4f0 f   gapidraw:pngrtran.obj
 0001:000ce720       _png_do_expand             004cf720 f   gapidraw:pngrtran.obj
 0001:000ceab0       _png_do_dither             004cfab0 f   gapidraw:pngrtran.obj
 0001:000cebd0       _png_build_gamma_table     004cfbd0 f   gapidraw:pngrtran.obj
 0001:000cf230       _png_do_read_intrapixel    004d0230 f   gapidraw:pngrtran.obj
 0001:000cf300       _png_get_valid             004d0300 f   gapidraw:pngget.obj
 0001:000cf320       _png_get_IHDR              004d0320 f   gapidraw:pngget.obj
 0001:000cf480       _png_read_data             004d0480 f   gapidraw:pngrio.obj
 0001:000cf4b0       _png_default_read_data     004d04b0 f   gapidraw:pngrio.obj
 0001:000cf4f0       _png_set_read_fn           004d04f0 f   gapidraw:pngrio.obj
 0001:000cf550       ??0CDisplay@@QAE@XZ        004d0550 f   gapidraw:ddutil.obj
 0001:000cf570       ??1CDisplay@@QAE@XZ        004d0570 f   gapidraw:ddutil.obj
 0001:000cf580       ?DestroyObjects@CDisplay@@UAEJXZ 004d0580 f   gapidraw:ddutil.obj
 0001:000cf5e0       ?CreateFullScreenDisplay@CDisplay@@QAEJPAUHWND__@@KKKK@Z 004d05e0 f   gapidraw:ddutil.obj
 0001:000cf780       ?CreateWindowedDisplay@CDisplay@@QAEJPAUHWND__@@KKKK@Z 004d0780 f   gapidraw:ddutil.obj
 0001:000cfa50       ?Create16bitVideoSurface@CDisplay@@QAEJPAPAVCSurface@@KKK@Z 004d0a50 f   gapidraw:ddutil.obj
 0001:000cfb70       ?PresentWindow@CDisplay@@QAEJXZ 004d0b70 f   gapidraw:ddutil.obj
 0001:000cfbd0       ?PresentFullscreen@CDisplay@@QAEJH@Z 004d0bd0 f   gapidraw:ddutil.obj
 0001:000cfc40       ?UpdateBounds@CDisplay@@QAEJXZ 004d0c40 f   gapidraw:ddutil.obj
 0001:000cfcc0       ??0CSurface@@QAE@XZ        004d0cc0 f   gapidraw:ddutil.obj
 0001:000cfce0       ?Create@CSurface@@QAEJPAUIDirectDrawSurface7@@H@Z 004d0ce0 f   gapidraw:ddutil.obj
 0001:000cfd20       ?Lock@CSurface@@QAEJPAUtagRECT@@PAU_DDSURFACEDESC2@@KPAX@Z 004d0d20 f   gapidraw:ddutil.obj
 0001:000cfd80       ?Unlock@CSurface@@QAEJPAUtagRECT@@@Z 004d0d80 f   gapidraw:ddutil.obj
 0001:000cfdd0       ?FreeFont@gdfont@@YAXPAU_GDBITMAPFONT@gdinternal@@@Z 004d0dd0 f   gapidraw:GapiBitmapFont.obj
 0001:000cfe50       ?InitializeFont@gdfont@@YAJPAU_GDBITMAPFONT@gdinternal@@@Z 004d0e50 f   gapidraw:GapiBitmapFont.obj
 0001:000cff60       ??0CGapiBitmapFont@@QAE@PAVCGapiDraw@@@Z 004d0f60 f   gapidraw:GapiBitmapFont.obj
 0001:000cff90       ??_GCGapiBitmapFont@@UAEPAXI@Z 004d0f90 f i gapidraw:GapiBitmapFont.obj
 0001:000cff90       ??_ECGapiBitmapFont@@UAEPAXI@Z 004d0f90 f i gapidraw:GapiBitmapFont.obj
 0001:000cffb0       ??1CGapiBitmapFont@@UAE@XZ 004d0fb0 f   gapidraw:GapiBitmapFont.obj
 0001:000cffd0       ?CreateFontA@CGapiBitmapFont@@QAEJPBDKKPAU_GDFONTFX@@@Z 004d0fd0 f   gapidraw:GapiBitmapFont.obj
 0001:000d0780       _png_write_info_before_PLTE 004d1780 f   gapidraw:pngwrite.obj
 0001:000d0960       _png_write_info            004d1960 f   gapidraw:pngwrite.obj
 0001:000d0c40       _png_write_end             004d1c40 f   gapidraw:pngwrite.obj
 0001:000d0da0       _png_create_write_struct   004d1da0 f   gapidraw:pngwrite.obj
 0001:000d0dd0       _png_create_write_struct_2 004d1dd0 f   gapidraw:pngwrite.obj
 0001:000d0f60       _png_write_row             004d1f60 f   gapidraw:pngwrite.obj
 0001:000d11c0       _png_write_flush           004d21c0 f   gapidraw:pngwrite.obj
 0001:000d12a0       _png_destroy_write_struct  004d22a0 f   gapidraw:pngwrite.obj
 0001:000d1340       _png_write_destroy         004d2340 f   gapidraw:pngwrite.obj
 0001:000d1460       _png_set_filter_heuristics 004d2460 f   gapidraw:pngwrite.obj
 0001:000d1690       _png_set_bKGD              004d2690 f   gapidraw:pngset.obj
 0001:000d16d0       _png_set_cHRM              004d26d0 f   gapidraw:pngset.obj
 0001:000d1990       _png_set_cHRM_fixed        004d2990 f   gapidraw:pngset.obj
 0001:000d1be0       _png_set_gAMA              004d2be0 f   gapidraw:pngset.obj
 0001:000d1c60       _png_set_gAMA_fixed        004d2c60 f   gapidraw:pngset.obj
 0001:000d1ce0       _png_set_hIST              004d2ce0 f   gapidraw:pngset.obj
 0001:000d1d80       _png_set_IHDR              004d2d80 f   gapidraw:pngset.obj
 0001:000d1f90       _png_set_oFFs              004d2f90 f   gapidraw:pngset.obj
 0001:000d1fc0       _png_set_pCAL              004d2fc0 f   gapidraw:pngset.obj
 0001:000d2110       _png_set_sCAL              004d3110 f   gapidraw:pngset.obj
 0001:000d2160       _png_set_pHYs              004d3160 f   gapidraw:pngset.obj
 0001:000d2190       _png_set_PLTE              004d3190 f   gapidraw:pngset.obj
 0001:000d2240       _png_set_sBIT              004d3240 f   gapidraw:pngset.obj
 0001:000d2270       _png_set_sRGB_gAMA_and_cHRM 004d3270 f   gapidraw:pngset.obj
 0001:000d2340       _png_set_iCCP              004d3340 f   gapidraw:pngset.obj
 0001:000d2430       _png_set_text              004d3430 f   gapidraw:pngset.obj
 0001:000d2610       _png_set_tIME              004d3610 f   gapidraw:pngset.obj
 0001:000d2650       _png_set_tRNS              004d3650 f   gapidraw:pngset.obj
 0001:000d2700       _png_set_sPLT              004d3700 f   gapidraw:pngset.obj
 0001:000d2860       _png_set_unknown_chunks    004d3860 f   gapidraw:pngset.obj
 0001:000d29b0       _png_write_data            004d39b0 f   gapidraw:pngwio.obj
 0001:000d29e0       _png_default_write_data    004d39e0 f   gapidraw:pngwio.obj
 0001:000d2a20       _png_flush                 004d3a20 f   gapidraw:pngwio.obj
 0001:000d2a40       _png_default_flush         004d3a40 f   gapidraw:pngwio.obj
 0001:000d2a60       _png_set_write_fn          004d3a60 f   gapidraw:pngwio.obj
 0001:000d2ad0       ?LoadGAPI@CGapiLib@@QAEJXZ 004d3ad0 f   gapidraw:GapiLib.obj
 0001:000d2b40       ?GXOpenInput@@YAHXZ        004d3b40 f i gapidraw:GapiLib.obj
 0001:000d2b40       ?GXSetViewport@@YAHKKKK@Z  004d3b40 f i gapidraw:GapiLib.obj
 0001:000d2b40       ?GXCloseDisplay@@YAHXZ     004d3b40 f i gapidraw:GapiLib.obj
 0001:000d2b40       ?GXSuspend@@YAHXZ          004d3b40 f i gapidraw:GapiLib.obj
 0001:000d2b40       ?GXResume@@YAHXZ           004d3b40 f i gapidraw:GapiLib.obj
 0001:000d2b40       ?GXIsDisplayDRAMBuffer@@YAHXZ 004d3b40 f i gapidraw:GapiLib.obj
 0001:000d2b40       ?GXOpenDisplay@@YAHPAUHWND__@@K@Z 004d3b40 f i gapidraw:GapiLib.obj
 0001:000d2b40       ?GXCloseInput@@YAHXZ       004d3b40 f i gapidraw:GapiLib.obj
 0001:000d2b40       ?GXEndDraw@@YAHXZ          004d3b40 f i gapidraw:GapiLib.obj
 0001:000d2b50       ?GXBeginDraw@@YAPAXXZ      004d3b50 f i gapidraw:GapiLib.obj
 0001:000d2b60       ?GXGetDisplayProperties@@YA?AUGXDisplayProperties@@XZ 004d3b60 f i gapidraw:GapiLib.obj
 0001:000d2b90       ?GXGetDefaultKeys@@YA?AUGXKeyList@@H@Z 004d3b90 f i gapidraw:GapiLib.obj
 0001:000d2c20       ?gddisplaycommon_RenderSystemFont@@YAJPAVCGapiSurfaceHelper@@K@Z 004d3c20 f   gapidraw:GapiDisplayCommon.obj
 0001:000d2da0       ?DrawSystemFont@?$CGapiSurfaceAdapter@VCGapiDisplay555@@@@QAEJPAVCGapiSurfaceHelper@@PAGJJPBDAAKKK@Z 004d3da0 f i gapidraw:GapiDisplayCommon.obj
 0001:000d3060       ?DrawSystemFont@?$CGapiSurfaceAdapter@VCGapiDisplay565@@@@QAEJPAVCGapiSurfaceHelper@@PAGJJPBDAAKKK@Z 004d4060 f i gapidraw:GapiDisplayCommon.obj
 0001:000d3320       ?RenderSystemFont@gdimage@@YAJPAVCGapiSurfaceHelper@@H@Z 004d4320 f i gapidraw:GapiDisplayCommon.obj
 0001:000d3770       _png_create_struct_2       004d4770 f   gapidraw:pngmem.obj
 0001:000d37f0       _png_destroy_struct        004d47f0 f   gapidraw:pngmem.obj
 0001:000d3800       _png_destroy_struct_2      004d4800 f   gapidraw:pngmem.obj
 0001:000d3850       _png_malloc                004d4850 f   gapidraw:pngmem.obj
 0001:000d38d0       _png_free                  004d48d0 f   gapidraw:pngmem.obj
 0001:000d3900       _png_memcpy_check          004d4900 f   gapidraw:pngmem.obj
 0001:000d3930       _png_memset_check          004d4930 f   gapidraw:pngmem.obj
 0001:000d3970       _png_set_mem_fn            004d4970 f   gapidraw:pngmem.obj
 0001:000d39a0       _crc32                     004d49a0 f   gapidraw:crc32.obj
 0001:000d3ae0       _inflateReset              004d4ae0 f   gapidraw:inflate.obj
 0001:000d3b30       _inflateEnd                004d4b30 f   gapidraw:inflate.obj
 0001:000d3b80       _inflateInit2_             004d4b80 f   gapidraw:inflate.obj
 0001:000d3cf0       _inflateInit_              004d4cf0 f   gapidraw:inflate.obj
 0001:000d3d10       _inflate                   004d4d10 f   gapidraw:inflate.obj
 0001:000d4140       _png_get_uint_32           004d5140 f   gapidraw:pngrutil.obj
 0001:000d4170       _png_crc_read              004d5170 f   gapidraw:pngrutil.obj
 0001:000d41a0       _png_crc_finish            004d51a0 f   gapidraw:pngrutil.obj
 0001:000d42f0       _png_crc_error             004d52f0 f   gapidraw:pngrutil.obj
 0001:000d4390       _png_decompress_chunk      004d5390 f   gapidraw:pngrutil.obj
 0001:000d46d0       _png_handle_IHDR           004d56d0 f   gapidraw:pngrutil.obj
 0001:000d4960       _png_handle_PLTE           004d5960 f   gapidraw:pngrutil.obj
 0001:000d4dd0       _png_handle_IEND           004d5dd0 f   gapidraw:pngrutil.obj
 0001:000d4f40       _png_handle_gAMA           004d5f40 f   gapidraw:pngrutil.obj
 0001:000d53a0       _png_handle_sBIT           004d63a0 f   gapidraw:pngrutil.obj
 0001:000d5810       _png_handle_cHRM           004d6810 f   gapidraw:pngrutil.obj
 0001:000d62b0       _png_handle_sRGB           004d72b0 f   gapidraw:pngrutil.obj
 0001:000d67c0       _png_handle_iCCP           004d77c0 f   gapidraw:pngrutil.obj
 0001:000d6cb0       _png_handle_sPLT           004d7cb0 f   gapidraw:pngrutil.obj
 0001:000d7020       _png_handle_tRNS           004d8020 f   gapidraw:pngrutil.obj
 0001:000d7590       _png_handle_bKGD           004d8590 f   gapidraw:pngrutil.obj
 0001:000d7a70       _png_handle_hIST           004d8a70 f   gapidraw:pngrutil.obj
 0001:000d7ee0       _png_handle_pHYs           004d8ee0 f   gapidraw:pngrutil.obj
 0001:000d82a0       _png_handle_oFFs           004d92a0 f   gapidraw:pngrutil.obj
 0001:000d8660       _png_handle_pCAL           004d9660 f   gapidraw:pngrutil.obj
 0001:000d8ba0       _png_handle_sCAL           004d9ba0 f   gapidraw:pngrutil.obj
 0001:000d9060       _png_handle_tIME           004da060 f   gapidraw:pngrutil.obj
 0001:000d9420       _png_handle_tEXt           004da420 f   gapidraw:pngrutil.obj
 0001:000d95c0       _png_handle_zTXt           004da5c0 f   gapidraw:pngrutil.obj
 0001:000d97b0       _png_handle_unknown        004da7b0 f   gapidraw:pngrutil.obj
 0001:000d9a70       _png_combine_row           004daa70 f   gapidraw:pngrutil.obj
 0001:000d9d90       _png_do_read_interlace     004dad90 f   gapidraw:pngrutil.obj
 0001:000da1c0       _png_read_filter_row       004db1c0 f   gapidraw:pngrutil.obj
 0001:000da3a0       _png_read_finish_row       004db3a0 f   gapidraw:pngrutil.obj
 0001:000da750       _png_read_start_row        004db750 f   gapidraw:pngrutil.obj
 0001:000da9c0       _DirectDrawCreateEx@16     004db9c0 f   gapidraw:DDRAW.dll
 0001:000da9d0       _png_save_uint_32          004db9d0 f   gapidraw:pngwutil.obj
 0001:000daa00       _png_write_chunk           004dba00 f   gapidraw:pngwutil.obj
 0001:000daab0       _png_write_chunk_data      004dbab0 f   gapidraw:pngwutil.obj
 0001:000daae0       _png_write_sig             004dbae0 f   gapidraw:pngwutil.obj
 0001:000dab50       _png_write_IHDR            004dbb50 f   gapidraw:pngwutil.obj
 0001:000daf80       _png_write_PLTE            004dbf80 f   gapidraw:pngwutil.obj
 0001:000db0c0       _png_write_IDAT            004dc0c0 f   gapidraw:pngwutil.obj
 0001:000db180       _png_write_IEND            004dc180 f   gapidraw:pngwutil.obj
 0001:000db210       _png_write_gAMA            004dc210 f   gapidraw:pngwutil.obj
 0001:000db2f0       _png_write_sRGB            004dc2f0 f   gapidraw:pngwutil.obj
 0001:000db3c0       _png_write_iCCP            004dc3c0 f   gapidraw:pngwutil.obj
 0001:000db8e0       _png_write_sPLT            004dc8e0 f   gapidraw:pngwutil.obj
 0001:000dbb10       _png_write_sBIT            004dcb10 f   gapidraw:pngwutil.obj
 0001:000dbc90       _png_write_cHRM            004dcc90 f   gapidraw:pngwutil.obj
 0001:000dc110       _png_write_tRNS            004dd110 f   gapidraw:pngwutil.obj
 0001:000dc3e0       _png_write_bKGD            004dd3e0 f   gapidraw:pngwutil.obj
 0001:000dc6b0       _png_write_hIST            004dd6b0 f   gapidraw:pngwutil.obj
 0001:000dc7b0       _png_check_keyword         004dd7b0 f   gapidraw:pngwutil.obj
 0001:000dc960       _png_write_tEXt            004dd960 f   gapidraw:pngwutil.obj
 0001:000dcaa0       _png_write_zTXt            004ddaa0 f   gapidraw:pngwutil.obj
 0001:000dcd40       _png_write_oFFs            004ddd40 f   gapidraw:pngwutil.obj
 0001:000dce50       _png_write_pCAL            004dde50 f   gapidraw:pngwutil.obj
 0001:000dd0d0       _png_write_sCAL            004de0d0 f   gapidraw:pngwutil.obj
 0001:000dd260       _png_write_pHYs            004de260 f   gapidraw:pngwutil.obj
 0001:000dd370       _png_write_tIME            004de370 f   gapidraw:pngwutil.obj
 0001:000dd4b0       _png_write_start_row       004de4b0 f   gapidraw:pngwutil.obj
 0001:000dd650       _png_write_finish_row      004de650 f   gapidraw:pngwutil.obj
 0001:000dd970       _png_do_write_interlace    004de970 f   gapidraw:pngwutil.obj
 0001:000ddc00       _png_write_find_filter     004dec00 f   gapidraw:pngwutil.obj
 0001:000de7c0       _png_write_filtered_row    004df7c0 f   gapidraw:pngwutil.obj
 0001:000de940       _png_do_write_transformations 004df940 f   gapidraw:pngwtran.obj
 0001:000deaa0       _png_do_pack               004dfaa0 f   gapidraw:pngwtran.obj
 0001:000debb0       _png_do_shift              004dfbb0 f   gapidraw:pngwtran.obj
 0001:000dee40       _png_do_write_swap_alpha   004dfe40 f   gapidraw:pngwtran.obj
 0001:000def50       _png_do_write_invert_alpha 004dff50 f   gapidraw:pngwtran.obj
 0001:000df060       _png_do_write_intrapixel   004e0060 f   gapidraw:pngwtran.obj
 0001:000df130       _deflateInit2_             004e0130 f   gapidraw:deflate.obj
 0001:000df430       _deflateReset              004e0430 f   gapidraw:deflate.obj
 0001:000df540       _deflate                   004e0540 f   gapidraw:deflate.obj
 0001:000df9b0       _deflateEnd                004e09b0 f   gapidraw:deflate.obj
 0001:000e09b0       _inflate_blocks_reset      004e19b0 f   gapidraw:infblock.obj
 0001:000e0a30       _inflate_blocks_new        004e1a30 f   gapidraw:infblock.obj
 0001:000e0af0       _inflate_blocks            004e1af0 f   gapidraw:infblock.obj
 0001:000e1800       _inflate_blocks_free       004e2800 f   gapidraw:infblock.obj
 0001:000e1890       _adler32                   004e2890 f   gapidraw:adler32.obj
 0001:000e19c0       _zcalloc                   004e29c0 f   gapidraw:zutil.obj
 0001:000e19e0       _zcfree                    004e29e0 f   gapidraw:zutil.obj
 0001:000e19f0       __tr_init                  004e29f0 f   gapidraw:trees.obj
 0001:000e1ab0       __tr_stored_block          004e2ab0 f   gapidraw:trees.obj
 0001:000e1c10       __tr_align                 004e2c10 f   gapidraw:trees.obj
 0001:000e1f70       __tr_flush_block           004e2f70 f   gapidraw:trees.obj
 0001:000e3570       _inflate_codes_new         004e4570 f   gapidraw:infcodes.obj
 0001:000e35b0       _inflate_codes             004e45b0 f   gapidraw:infcodes.obj
 0001:000e3d60       _inflate_codes_free        004e4d60 f   gapidraw:infcodes.obj
 0001:000e3d80       _inflate_trees_bits        004e4d80 f   gapidraw:inftrees.obj
 0001:000e42f0       _inflate_trees_dynamic     004e52f0 f   gapidraw:inftrees.obj
 0001:000e4480       _inflate_trees_fixed       004e5480 f   gapidraw:inftrees.obj
 0001:000e44b0       _inflate_flush             004e54b0 f   gapidraw:infutil.obj
 0001:000e45f0       _inflate_fast              004e55f0 f   gapidraw:inffast.obj
 0001:000e49c0       ??3@YAXPAX@Z               004e59c0 f   LIBC:delete.obj
 0001:000e49c5       ??2@YAPAXI@Z               004e59c5 f   LIBC:new.obj
 0001:000e49d3       ?_JumpToContinuation@@YGXPAXPAUEHRegistrationNode@@@Z 004e59d3 f   LIBC:trnsctrl.obj
 0001:000e4a03       ?_CallMemberFunction2@@YGXPAX00H@Z 004e5a03 f   LIBC:trnsctrl.obj
 0001:000e4a03       ?_CallMemberFunction0@@YGXPAX0@Z 004e5a03 f   LIBC:trnsctrl.obj
 0001:000e4a03       ?_CallMemberFunction1@@YGXPAX00@Z 004e5a03 f   LIBC:trnsctrl.obj
 0001:000e4a0a       ?_UnwindNestedFrames@@YGXPAUEHRegistrationNode@@PAUEHExceptionRecord@@@Z 004e5a0a f   LIBC:trnsctrl.obj
 0001:000e4a5c       ___CxxFrameHandler         004e5a5c f   LIBC:trnsctrl.obj
 0001:000e4a92       ___CxxLongjmpUnwind@4      004e5a92 f   LIBC:trnsctrl.obj
 0001:000e4ae7       ?_CallSETranslator@@YAHPAUEHExceptionRecord@@PAUEHRegistrationNode@@PAX2PBU_s_FuncInfo@@H1@Z 004e5ae7 f   LIBC:trnsctrl.obj
 0001:000e4c5e       ?_GetRangeOfTrysToCheck@@YAPBU_s_TryBlockMapEntry@@PBU_s_FuncInfo@@HHPAI1@Z 004e5c5e f   LIBC:trnsctrl.obj
 0001:000e4cd8       ?_CreateFrameInfo@@YAPAUFrameInfo@@PAU1@PAX@Z 004e5cd8 f   LIBC:trnsctrl.obj
 0001:000e4cf1       ?IsExceptionObjectToBeDestroyed@@YAHPAX@Z 004e5cf1 f   LIBC:trnsctrl.obj
 0001:000e4d0c       ?_FindAndUnlinkFrame@@YAXPAUFrameInfo@@@Z 004e5d0c f   LIBC:trnsctrl.obj
 0001:000e4d45       ?_CallCatchBlock2@@YAPAXPAUEHRegistrationNode@@PBU_s_FuncInfo@@PAXHK@Z 004e5d45 f   LIBC:trnsctrl.obj
 0001:000e4da0       __global_unwind2           004e5da0 f   LIBC:exsup.obj
 0001:000e4de2       __local_unwind2            004e5de2 f   LIBC:exsup.obj
 0001:000e4e3a       __NLG_Return2              004e5e3a     LIBC:exsup.obj
 0001:000e4e4a       __abnormal_termination     004e5e4a f   LIBC:exsup.obj
 0001:000e4e6d       __NLG_Notify1              004e5e6d f   LIBC:exsup.obj
 0001:000e4e76       __NLG_Notify               004e5e76 f   LIBC:exsup.obj
 0001:000e4e89       __NLG_Dispatch             004e5e89     LIBC:exsup.obj
 0001:000e4e90       _strcpy                    004e5e90 f   LIBC:strcat.obj
 0001:000e4ea0       _strcat                    004e5ea0 f   LIBC:strcat.obj
 0001:000e4f90       _strlen                    004e5f90 f   LIBC:strlen.obj
 0001:000e501b       __purecall                 004e601b f   LIBC:purevirt.obj
 0001:000e502f       __fpclear                  004e602f f   LIBC:fpinit.obj
 0001:000e5030       __cfltcvt_init             004e6030 f   LIBC:fpinit.obj
 0001:000e5068       __fpmath                   004e6068 f   LIBC:fpinit.obj
 0001:000e5086       _time                      004e6086 f   LIBC:time.obj
 0001:000e50bf       _sprintf                   004e60bf f   LIBC:sprintf.obj
 0001:000e5117       ___crtExitProcess          004e6117 f   LIBC:crt0dat.obj
 0001:000e5147       __cinit                    004e6147 f   LIBC:crt0dat.obj
 0001:000e5272       _exit                      004e6272 f   LIBC:crt0dat.obj
 0001:000e5283       __exit                     004e6283 f   LIBC:crt0dat.obj
 0001:000e5294       __cexit                    004e6294 f   LIBC:crt0dat.obj
 0001:000e52a3       __c_exit                   004e62a3 f   LIBC:crt0dat.obj
 0001:000e52d0       _strchr                    004e62d0 f   LIBC:strchr.obj
 0001:000e52d6       ___from_strstr_to_strchr   004e62d6     LIBC:strchr.obj
 0001:000e5390       _strncat                   004e6390 f   LIBC:strncat.obj
 0001:000e54c5       _srand                     004e64c5 f   LIBC:rand.obj
 0001:000e54cf       _rand                      004e64cf f   LIBC:rand.obj
 0001:000e54f2       _fclose                    004e64f2 f   LIBC:fclose.obj
 0001:000e5548       __fsopen                   004e6548 f   LIBC:fopen.obj
 0001:000e5572       _fopen                     004e6572 f   LIBC:fopen.obj
 0001:000e5585       _difftime                  004e6585 f   LIBC:difftime.obj
 0001:000e5598       __ftol2                    004e6598 f   LIBC:ftol2.obj
 0001:000e560d       _fwrite                    004e660d f   LIBC:fwrite.obj
 0001:000e5714       _fread                     004e6714 f   LIBC:fread.obj
 0001:000e57fd       _remove                    004e67fd f   LIBC:unlink.obj
 0001:000e5830       _memset                    004e6830 f   LIBC:memset.obj
 0001:000e5890       _memcpy                    004e6890 f   LIBC:memcpy.obj
 0001:000e5bcd       _tolower                   004e6bcd f   LIBC:tolower.obj
 0001:000e5cb0       _strcmp                    004e6cb0 f   LIBC:strcmp.obj
 0001:000e5d38       _fprintf                   004e6d38 f   LIBC:fprintf.obj
 0001:000e5d6a       _vfprintf                  004e6d6a f   LIBC:vfprintf.obj
 0001:000e5d9b       _asctime                   004e6d9b f   LIBC:asctime.obj
 0001:000e5e85       _localtime                 004e6e85 f   LIBC:localtim.obj
 0001:000e6005       __flush                    004e7005 f   LIBC:fflush.obj
 0001:000e6062       _fflush                    004e7062 f   LIBC:fflush.obj
 0001:000e610a       __flushall                 004e710a f   LIBC:fflush.obj
 0001:000e6120       _strncpy                   004e7120 f   LIBC:strncpy.obj
 0001:000e6244       _atol                      004e7244 f   LIBC:atox.obj
 0001:000e629c       _atoi                      004e729c f   LIBC:atox.obj
 0001:000e62a1       _calloc                    004e72a1 f   LIBC:calloc.obj
 0001:000e6332       _free                      004e7332 f   LIBC:free.obj
 0001:000e636a       __heap_alloc               004e736a f   LIBC:malloc.obj
 0001:000e63b0       __nh_malloc                004e73b0 f   LIBC:malloc.obj
 0001:000e63dc       _malloc                    004e73dc f   LIBC:malloc.obj
 0001:000e63f0       __allshr                   004e73f0 f   LIBC:llshr.obj
 0001:000e6411       __mbsstr                   004e7411 f   LIBC:mbsstr.obj
 0001:000e64a0       __mbsnbcpy                 004e74a0 f   LIBC:mbsnbcpy.obj
 0001:000e6521       _abs                       004e7521 f   LIBC:abs.obj
 0001:000e6530       __CIsqrt                   004e7530 f   LIBC:sqrt.obj
 0001:000e6544       _sqrt                      004e7544     LIBC:sqrt.obj
 0001:000e65f0       __alloca_probe             004e75f0     LIBC:chkstk.obj
 0001:000e65f0       __chkstk                   004e75f0 f   LIBC:chkstk.obj
 0001:000e6630       __CIcos                    004e7630 f   LIBC:cos.obj
 0001:000e6644       _cos                       004e7644     LIBC:cos.obj
 0001:000e66e0       __CIsin                    004e76e0 f   LIBC:sin.obj
 0001:000e66f4       _sin                       004e76f4     LIBC:sin.obj
 0001:000e678e       __onexit                   004e778e f   LIBC:onexit.obj
 0001:000e6810       _atexit                    004e7810 f   LIBC:onexit.obj
 0001:000e6822       ___onexitinit              004e7822 f   LIBC:onexit.obj
 0001:000e6850       _strstr                    004e7850 f   LIBC:strstr.obj
 0001:000e68d6       _strtok                    004e78d6 f   LIBC:strtok.obj
 0001:000e698d       __mbstok                   004e798d f   LIBC:mbstok.obj
 0001:000e6a30       _atan2                     004e7a30 f   LIBC:87ctriga.obj
 0001:000e6a3a       __CIatan2                  004e7a3a f   LIBC:87ctriga.obj
 0001:000e6a44       _vsprintf                  004e7a44 f   LIBC:vsprintf.obj
 0001:000e6a9b       __snprintf                 004e7a9b f   LIBC:snprintf.obj
 0001:000e6af2       _ftell                     004e7af2 f   LIBC:ftell.obj
 0001:000e6c4b       _fseek                     004e7c4b f   LIBC:fseek.obj
 0001:000e6cd9       ??_V@YAXPAX@Z              004e7cd9 f   LIBC:delete2.obj
 0001:000e6cde       ?__ArrayUnwind@@YGXPAXIHP6EX0@Z@Z 004e7cde f   LIBC:ehvecdtr.obj
 0001:000e6d3c       ??_M@YGXPAXIHP6EX0@Z@Z     004e7d3c f   LIBC:ehvecdtr.obj
 0001:000e6d9c       _swprintf                  004e7d9c f   LIBC:swprintf.obj
 0001:000e6e0b       ??1type_info@@UAE@XZ       004e7e0b f   LIBC:typinfo.obj
 0001:000e6e20       ??_Gtype_info@@UAEPAXI@Z   004e7e20 f i LIBC:typinfo.obj
 0001:000e6e20       ??_Etype_info@@UAEPAXI@Z   004e7e20 f i LIBC:typinfo.obj
 0001:000e6e3c       __CxxThrowException@8      004e7e3c f   LIBC:throw.obj
 0001:000e6e76       __resetstkoflw             004e7e76 f   LIBC:resetstk.obj
 0001:000e6f64       __except_handler3          004e7f64 f   LIBC:exsup3.obj
 0001:000e704a       __seh_longjmp_unwind@4     004e804a f   LIBC:exsup3.obj
 0001:000e7065       ??_L@YGXPAXIHP6EX0@Z1@Z    004e8065 f   LIBC:ehvecctr.obj
 0001:000e70c7       ??_U@YAPAXI@Z              004e80c7 f   LIBC:new2.obj
 0001:000e70d0       _memcmp                    004e80d0 f   LIBC:memcmp.obj
 0001:000e7188       _realloc                   004e8188 f   LIBC:realloc.obj
 0001:000e72f0       __amsg_exit                004e82f0 f   LIBC:wincrt0.obj
 0001:000e7315       _WinMainCRTStartup         004e8315 f   LIBC:wincrt0.obj
 0001:000e74f4       __setjmp3                  004e84f4 f   LIBC:setjmp3.obj
 0001:000e7570       __ftol                     004e8570 f   LIBC:ftol.obj
 0001:000e75a0       __alldiv                   004e85a0 f   LIBC:lldiv.obj
 0001:000e7650       __allmul                   004e8650 f   LIBC:llmul.obj
 0001:000e7684       _longjmp                   004e8684 f   LIBC:longjmp.obj
 0001:000e76fd       ___initstdio               004e86fd f   LIBC:_file.obj
 0001:000e77a3       ___endstdio                004e87a3 f   LIBC:_file.obj
 0001:000e77b7       _abort                     004e87b7 f   LIBC:abort.obj
 0001:000e77d0       _pow                       004e87d0 f   LIBC:pow.obj
 0001:000e7810       __CIpow                    004e8810 f   LIBC:pow.obj
 0001:000e784b       __CIpow_default            004e884b f   LIBC:pow.obj
 0001:000e7864       __pow_default              004e8864     LIBC:pow.obj
 0001:000e7a60       _strncmp                   004e8a60 f   LIBC:strncmp.obj
 0001:000e7a99       _gmtime                    004e8a99 f   LIBC:gmtime.obj
 0001:000e7b8e       _strtod                    004e8b8e f   LIBC:strtod.obj
 0001:000e7c8e       ___FrameUnwindToState      004e8c8e f   LIBC:frame.obj
 0001:000e7d4b       ___DestructExceptionObject 004e8d4b f   LIBC:frame.obj
 0001:000e83ea       ___InternalCxxFrameHandler 004e93ea f   LIBC:frame.obj
 0001:000e848c       ?terminate@@YAXXZ          004e948c f   LIBC:hooks.obj
 0001:000e84b9       ?_inconsistency@@YAXXZ     004e94b9 f   LIBC:hooks.obj
 0001:000e84f0       __CallSettingFrame@12      004e94f0 f   LIBC:lowhelpr.obj
 0001:000e8517       __NLG_Return               004e9517     LIBC:lowhelpr.obj
 0001:000e853c       __forcdecpt                004e953c f   LIBC:cvt.obj
 0001:000e8594       __cropzeros                004e9594 f   LIBC:cvt.obj
 0001:000e85df       __positive                 004e95df f   LIBC:cvt.obj
 0001:000e85f9       __fassign                  004e95f9 f   LIBC:cvt.obj
 0001:000e8654       __cftoe                    004e9654 f   LIBC:cvt.obj
 0001:000e8745       __cftof                    004e9745 f   LIBC:cvt.obj
 0001:000e8822       __cftog                    004e9822 f   LIBC:cvt.obj
 0001:000e88cc       __cfltcvt                  004e98cc f   LIBC:cvt.obj
 0001:000e891d       __setdefaultprecision      004e991d f   LIBC:fp8.obj
 0001:000e892f       __ms_p5_test_fdiv          004e992f f   LIBC:testfdiv.obj
 0001:000e896f       __ms_p5_mp_test_fdiv       004e996f f   LIBC:testfdiv.obj
 0001:000e89a0       __aulldiv                  004e99a0 f   LIBC:ulldiv.obj
 0001:000e8a08       __flsbuf                   004e9a08 f   LIBC:_flsbuf.obj
 0001:000e8bac       __output                   004e9bac f   LIBC:output.obj
 0001:000e9368       __RTC_Initialize           004ea368 f   LIBC:initsect.obj
 0001:000e93ac       __RTC_Terminate            004ea3ac f   LIBC:initsect.obj
 0001:000e93f0       __close                    004ea3f0 f   LIBC:close.obj
 0001:000e94a3       __freebuf                  004ea4a3 f   LIBC:_freebuf.obj
 0001:000e94ce       __openfile                 004ea4ce f   LIBC:_open.obj
 0001:000e9636       __getstream                004ea636 f   LIBC:stream.obj
 0001:000e96a8       __write                    004ea6a8 f   LIBC:write.obj
 0001:000e9876       __filbuf                   004ea876 f   LIBC:_filbuf.obj
 0001:000e9954       __read                     004ea954 f   LIBC:read.obj
 0001:000e9b44       __dosmaperr                004eab44 f   LIBC:dosmap.obj
 0001:000e9ba3       ___crtLCMapStringA         004eaba3 f   LIBC:a_map.obj
 0001:000e9f79       __isctype                  004eaf79 f   LIBC:isctype.obj
 0001:000e9ff7       __stbuf                    004eaff7 f   LIBC:_sftbuf.obj
 0001:000ea07f       __ftbuf                    004eb07f f   LIBC:_sftbuf.obj
 0001:000ea0bb       __tzset                    004eb0bb f   LIBC:tzset.obj
 0001:000ea4c6       __isindst                  004eb4c6 f   LIBC:tzset.obj
 0001:000ea653       ___tzset                   004eb653 f   LIBC:tzset.obj
 0001:000ea668       __commit                   004eb668 f   LIBC:commit.obj
 0001:000ea6bf       __ismbcspace               004eb6bf f   LIBC:ismbspc.obj
 0001:000ea74f       __callnewh                 004eb74f f   LIBC:handler.obj
 0001:000ea76a       ___heap_select             004eb76a f   LIBC:heapinit.obj
 0001:000ea784       __heap_init                004eb784 f   LIBC:heapinit.obj
 0001:000ea7d5       ___sbh_heap_init           004eb7d5 f   LIBC:sbheap.obj
 0001:000ea81d       ___sbh_find_block          004eb81d f   LIBC:sbheap.obj
 0001:000ea848       ___sbh_free_block          004eb848 f   LIBC:sbheap.obj
 0001:000eab60       ___sbh_alloc_new_region    004ebb60 f   LIBC:sbheap.obj
 0001:000eac17       ___sbh_alloc_new_group     004ebc17 f   LIBC:sbheap.obj
 0001:000ead1d       ___sbh_resize_block        004ebd1d f   LIBC:sbheap.obj
 0001:000eaffc       ___sbh_alloc_block         004ebffc f   LIBC:sbheap.obj
 0001:000eb4eb       __setmbcp                  004ec4eb f   LIBC:mbctype.obj
 0001:000eb6d5       ___initmbctable            004ec6d5 f   LIBC:mbctype.obj
 0001:000eb700       __trandisp1                004ec700 f   LIBC:87disp.obj
 0001:000eb767       __trandisp2                004ec767 f   LIBC:87disp.obj
 0001:000eb7f3       __rttospopde               004ec7f3     LIBC:87disp.obj
 0001:000eb7f8       __rttospop                 004ec7f8     LIBC:87disp.obj
 0001:000eb7fa       __rtnospop                 004ec7fa     LIBC:87disp.obj
 0001:000eb7fc       __rttosnpop                004ec7fc     LIBC:87disp.obj
 0001:000eb7fd       __rtnospopde               004ec7fd     LIBC:87disp.obj
 0001:000eb804       __rtzeropop                004ec804     LIBC:87disp.obj
 0001:000eb806       __rtzeronpop               004ec806     LIBC:87disp.obj
 0001:000eb80b       __rtonepop                 004ec80b     LIBC:87disp.obj
 0001:000eb80d       __rtonenpop                004ec80d     LIBC:87disp.obj
 0001:000eb812       __tosnan1                  004ec812     LIBC:87disp.obj
 0001:000eb83d       __nosnan2                  004ec83d     LIBC:87disp.obj
 0001:000eb83f       __tosnan2                  004ec83f     LIBC:87disp.obj
 0001:000eb867       __nan2                     004ec867     LIBC:87disp.obj
 0001:000eb8a6       __rtindfpop                004ec8a6     LIBC:87disp.obj
 0001:000eb8a8       __rtindfnpop               004ec8a8     LIBC:87disp.obj
 0001:000eb8b9       __rttosnpopde              004ec8b9     LIBC:87disp.obj
 0001:000eb8c3       __rtchsifneg               004ec8c3     LIBC:87disp.obj
 0001:000eb8d0       __startTwoArgErrorHandling 004ec8d0 f   LIBC:genexcep.obj
 0001:000eb8e7       __startOneArgErrorHandling 004ec8e7 f   LIBC:genexcep.obj
 0001:000eb930       __twoToTOS                 004ec930 f   LIBC:common.obj
 0001:000eb945       __load_CW                  004ec945 f   LIBC:common.obj
 0001:000eb95c       __convertTOStoQNaN         004ec95c f   LIBC:common.obj
 0001:000eb975       __fload_withFB             004ec975 f   LIBC:common.obj
 0001:000eb9b8       __checkTOS_withFB          004ec9b8 f   LIBC:common.obj
 0001:000eb9ce       __fast_exit                004ec9ce f   LIBC:common.obj
 0001:000eb9db       __math_exit                004ec9db f   LIBC:common.obj
 0001:000eba05       __check_overflow_exit      004eca05 f   LIBC:common.obj
 0001:000eba19       __check_range_exit         004eca19 f   LIBC:common.obj
 0001:000ebabc       __msize                    004ecabc f   LIBC:msize.obj
 0001:000ebb25       @__security_check_cookie@4 004ecb25 f   LIBC:secchk.obj
 0001:000ebb33       __mbspbrk                  004ecb33 f   LIBC:mbspbrk.obj
 0001:000ebbac       __mbsspnp                  004ecbac f   LIBC:mbsspnp.obj
 0001:000ebc5c       __fFATN2                   004ecc5c     LIBC:87triga.obj
 0001:000ebcac       __rtpiby2                  004eccac     LIBC:87triga.obj
 0001:000ebcf0       __cintrindisp2             004eccf0 f   LIBC:87cdisp.obj
 0001:000ebd2e       __cintrindisp1             004ecd2e f   LIBC:87cdisp.obj
 0001:000ebd64       __ctrandisp2               004ecd64 f   LIBC:87cdisp.obj
 0001:000ebeea       __ctrandisp1               004eceea f   LIBC:87cdisp.obj
 0001:000ebf16       __fload                    004ecf16 f   LIBC:87cdisp.obj
 0001:000ebf52       __ioinit                   004ecf52 f   LIBC:ioinit.obj
 0001:000ec0fd       __lseek                    004ed0fd f   LIBC:lseek.obj
 0001:000ec18c       __SEH_prolog               004ed18c f   LIBC:sehprolg.obj
 0001:000ec1c7       __SEH_epilog               004ed1c7 f   LIBC:sehprolg.obj
 0001:000ec25f       __woutput                  004ed25f f   LIBC:woutput.obj
 0001:000eca4b       ?__CxxUnhandledExceptionFilter@@YGJPAU_EXCEPTION_POINTERS@@@Z 004eda4b f   LIBC:unhandld.obj
 0001:000eca99       ?__CxxSetUnhandledExceptionFilter@@YAHXZ 004eda99 f   LIBC:unhandld.obj
 0001:000ecaac       ?__CxxRestoreUnhandledExceptionFilter@@YAXXZ 004edaac f   LIBC:unhandld.obj
 0001:000ecab9       __ValidateEH3RN            004edab9 f   LIBC:eh3valid.obj
 0001:000ecce2       __NMSG_WRITE               004edce2 f   LIBC:crt0msg.obj
 0001:000ece5a       __FF_MSGBANNER             004ede5a f   LIBC:crt0msg.obj
 0001:000ece93       __XcptFilter               004ede93 f   LIBC:winxfltr.obj
 0001:000ed004       __wincmdln                 004ee004 f   LIBC:wincmdln.obj
 0001:000ed061       __setenvp                  004ee061 f   LIBC:stdenvp.obj
 0001:000ed294       __setargv                  004ee294 f   LIBC:stdargv.obj
 0001:000ed336       ___crtGetEnvironmentStringsA 004ee336 f   LIBC:a_env.obj
 0001:000ed458       __rt_probe_read4@4         004ee458 f   LIBC:sehsupp.obj
 0001:000ed49a       __fcloseall                004ee49a f   LIBC:closeall.obj
 0001:000ed52b       _raise                     004ee52b f   LIBC:winsig.obj
 0001:000ed689       ___sse2_available_init     004ee689 f   LIBC:cpu_disp.obj
 0001:000ed760       __CIpow_pentium4           004ee760 f   LIBC:pow_pentium4.obj
 0001:000ed779       __pow_pentium4             004ee779     LIBC:pow_pentium4.obj
 0001:000ee2c1       __fFEXP                    004ef2c1     LIBC:87tran.obj
 0001:000ee328       __rtinfpopse               004ef328     LIBC:87tran.obj
 0001:000ee32a       __rtinfnpopse              004ef32a     LIBC:87tran.obj
 0001:000ee33a       __fFLN                     004ef33a     LIBC:87tran.obj
 0001:000ee3ef       __rtinfpop                 004ef3ef     LIBC:87tran.obj
 0001:000ee3f1       __rtinfnpop                004ef3f1     LIBC:87tran.obj
 0001:000ee40e       __ffexpm1                  004ef40e     LIBC:87tran.obj
 0001:000ee4b7       __d_inttype                004ef4b7 f   LIBC:powhlp.obj
 0001:000ee525       __powhlp                   004ef525 f   LIBC:powhlp.obj
 0001:000ee688       __fltin                    004ef688 f   LIBC:cfin.obj
 0001:000ee727       ?_ValidateRead@@YAHPBXI@Z  004ef727 f   LIBC:validate.obj
 0001:000ee743       ?_ValidateWrite@@YAHPAXI@Z 004ef743 f   LIBC:validate.obj
 0001:000ee75f       ?_ValidateExecute@@YAHP6GHXZ@Z 004ef75f f   LIBC:validate.obj
 0001:000ee780       _memmove                   004ef780 f   LIBC:memmove.obj
 0001:000eeabd       __ZeroTail                 004efabd f   LIBC:intrncvt.obj
 0001:000eeaef       __IncMan                   004efaef f   LIBC:intrncvt.obj
 0001:000eeb3c       __RoundMan                 004efb3c f   LIBC:intrncvt.obj
 0001:000eebae       __CopyMan                  004efbae f   LIBC:intrncvt.obj
 0001:000eebc9       __IsZeroMan                004efbc9 f   LIBC:intrncvt.obj
 0001:000eebe2       __ShrMan                   004efbe2 f   LIBC:intrncvt.obj
 0001:000eec5d       __ld12cvt                  004efc5d f   LIBC:intrncvt.obj
 0001:000eedb5       __ld12tod                  004efdb5 f   LIBC:intrncvt.obj
 0001:000eedcb       __ld12tof                  004efdcb f   LIBC:intrncvt.obj
 0001:000eede1       __atodbl                   004efde1 f   LIBC:intrncvt.obj
 0001:000eee26       __atoflt                   004efe26 f   LIBC:intrncvt.obj
 0001:000eee6b       __fptostr                  004efe6b f   LIBC:_fptostr.obj
 0001:000eeee2       ___dtold                   004efee2 f   LIBC:cfout.obj
 0001:000eef9c       __fltout                   004eff9c f   LIBC:cfout.obj
 0001:000ef014       __fptrap                   004f0014 f   LIBC:crt0fp.obj
 0001:000ef13d       __control87                004f013d f   LIBC:ieee87.obj
 0001:000ef16f       __controlfp                004f016f f   LIBC:ieee87.obj
 0001:000ef185       __getbuf                   004f0185 f   LIBC:_getbuf.obj
 0001:000ef1c9       __isatty                   004f01c9 f   LIBC:isatty.obj
 0001:000ef1f0       _wctomb                    004f01f0 f   LIBC:wctomb.obj
 0001:000ef260       __aulldvrm                 004f0260 f   LIBC:ulldvrm.obj
 0001:000ef2f5       __alloc_osfhnd             004f02f5 f   LIBC:osfinfo.obj
 0001:000ef392       __set_osfhnd               004f0392 f   LIBC:osfinfo.obj
 0001:000ef409       __free_osfhnd              004f0409 f   LIBC:osfinfo.obj
 0001:000ef483       __get_osfhandle            004f0483 f   LIBC:osfinfo.obj
 0001:000ef4bf       __sopen                    004f04bf f   LIBC:open.obj
 0001:000ef78f       __lseeki64                 004f078f f   LIBC:lseeki64.obj
 0001:000ef82e       ___ansicp                  004f082e f   LIBC:convrtcp.obj
 0001:000ef875       ___convertcp               004f0875 f   LIBC:convrtcp.obj
 0001:000efa4f       ___crtGetStringTypeA       004f0a4f f   LIBC:a_str.obj
 0001:000efc09       _getenv                    004f0c09 f   LIBC:getenv.obj
 0001:000efc8a       __87except                 004f0c8a f   LIBC:87except.obj
 0001:000efd86       ___security_init_cookie    004f0d86 f   LIBC:seccinit.obj
 0001:000efdec       ___security_error_handler  004f0dec f   LIBC:secfail.obj
 0001:000eff40       _strpbrk                   004f0f40 f   LIBC:strpbrk.obj
 0001:000eff80       _strspn                    004f0f80 f   LIBC:strspn.obj
 0001:000effc6       _fputwc                    004f0fc6 f   LIBC:fputwc.obj
 0001:000f009c       _mbtowc                    004f109c f   LIBC:mbtowc.obj
 0001:000f0164       ___crtMessageBoxA          004f1164 f   LIBC:crtmbox.obj
 0001:000f0290       __ismbblead                004f1290 f   LIBC:ismbbyte.obj
 0001:000f02a1       ___libm_error_support      004f12a1 f   LIBC:libm_error.obj
 0001:000f0520       _fdiv_main_routine         004f1520 f   LIBC:adj_fdiv.obj
 0001:000f0637       __adj_fdiv_r               004f1637 f   LIBC:adj_fdiv.obj
 0001:000f0ad6       __fdivp_sti_st             004f1ad6 f   LIBC:adj_fdiv.obj
 0001:000f0ae9       __fdivrp_sti_st            004f1ae9 f   LIBC:adj_fdiv.obj
 0001:000f0afc       __adj_fdiv_m32             004f1afc f   LIBC:adj_fdiv.obj
 0001:000f0b48       __adj_fdiv_m64             004f1b48 f   LIBC:adj_fdiv.obj
 0001:000f0b94       __adj_fdiv_m16i            004f1b94 f   LIBC:adj_fdiv.obj
 0001:000f0bc8       __adj_fdiv_m32i            004f1bc8 f   LIBC:adj_fdiv.obj
 0001:000f0bfc       __adj_fdivr_m32            004f1bfc f   LIBC:adj_fdiv.obj
 0001:000f0c48       __adj_fdivr_m64            004f1c48 f   LIBC:adj_fdiv.obj
 0001:000f0c94       __adj_fdivr_m16i           004f1c94 f   LIBC:adj_fdiv.obj
 0001:000f0cc8       __adj_fdivr_m32i           004f1cc8 f   LIBC:adj_fdiv.obj
 0001:000f0cfc       __safe_fdiv                004f1cfc f   LIBC:adj_fdiv.obj
 0001:000f0d11       __safe_fdivr               004f1d11 f   LIBC:adj_fdiv.obj
 0001:000f0d26       __fprem_common             004f1d26 f   LIBC:adj_fdiv.obj
 0001:000f0f2c       __adj_fprem                004f1f2c f   LIBC:adj_fdiv.obj
 0001:000f0fde       __fprem1_common            004f1fde f   LIBC:adj_fdiv.obj
 0001:000f11e4       __adj_fprem1               004f21e4 f   LIBC:adj_fdiv.obj
 0001:000f1299       __safe_fprem               004f2299 f   LIBC:adj_fdiv.obj
 0001:000f129f       __safe_fprem1              004f229f f   LIBC:adj_fdiv.obj
 0001:000f12a5       __adj_fpatan               004f22a5 f   LIBC:adj_fdiv.obj
 0001:000f12a8       __adj_fptan                004f22a8 f   LIBC:adj_fdiv.obj
 0001:000f12ab       __frnd                     004f22ab f   LIBC:frnd.obj
 0001:000f12bc       __fpclass                  004f22bc f   LIBC:ieeemisc.obj
 0001:000f1358       __set_exp                  004f2358 f   LIBC:util.obj
 0001:000f1382       __sptype                   004f2382 f   LIBC:util.obj
 0001:000f13dd       __decomp                   004f23dd f   LIBC:util.obj
 0001:000f1499       ___strgtold12              004f2499 f   LIBC:strgtold.obj
 0001:000f1931       ___addl                    004f2931 f   LIBC:mantold.obj
 0001:000f1952       ___add_12                  004f2952 f   LIBC:mantold.obj
 0001:000f19b0       ___shl_12                  004f29b0 f   LIBC:mantold.obj
 0001:000f19de       ___shr_12                  004f29de f   LIBC:mantold.obj
 0001:000f1a0b       ___mtold12                 004f2a0b f   LIBC:mantold.obj
 0001:000f1af3       _$I10_OUTPUT               004f2af3 f   LIBC:x10fout.obj
 0001:000f1d8f       __chsize                   004f2d8f f   LIBC:chsize.obj
 0001:000f1ef5       __mbsnbicoll               004f2ef5 f   LIBC:mbsnbico.obj
 0001:000f1f34       ___wtomb_environ           004f2f34 f   LIBC:wtombenv.obj
 0001:000f1fc4       __raise_exc                004f2fc4 f   LIBC:fpexcept.obj
 0001:000f2269       __handle_exc               004f3269 f   LIBC:fpexcept.obj
 0001:000f248d       __set_errno                004f348d f   LIBC:fpexcept.obj
 0001:000f24b3       __matherr                  004f34b3 f   LIBC:matherr.obj
 0001:000f24b6       __statfp                   004f34b6 f   LIBC:fpctrl.obj
 0001:000f24c1       __clrfp                    004f34c1 f   LIBC:fpctrl.obj
 0001:000f24cd       __ctrlfp                   004f34cd f   LIBC:fpctrl.obj
 0001:000f24f1       __set_statfp               004f34f1 f   LIBC:fpctrl.obj
 0001:000f2547       __flswbuf                  004f3547 f   LIBC:_flswbuf.obj
 0001:000f266c       ___ld12mul                 004f366c f   LIBC:tenpow.obj
 0001:000f28a2       ___multtenpow12            004f38a2 f   LIBC:tenpow.obj
 0001:000f2930       __setmode                  004f3930 f   LIBC:setmode.obj
 0001:000f29ce       ___crtCompareStringA       004f39ce f   LIBC:a_cmp.obj
 0001:000f2e06       ___crtsetenv               004f3e06 f   LIBC:setenv.obj
 0001:000f2fdc       _strdup                    004f3fdc f   LIBC:strdup.obj
 0001:000f2fdc       __strdup                   004f3fdc f   LIBC:strdup.obj
 0001:000f3007       __mbschr                   004f4007 f   LIBC:mbschr.obj
 0001:000f306e       ?RemoveAll@?$CSimpleArray@PAUHINSTANCE__@@V?$CSimpleArrayEqualHelper@PAUHINSTANCE__@@@ATL@@@ATL@@QAEXXZ 004f406e f i atls:atlbase.obj
 0001:000f308b       ??0_ATL_BASE_MODULE70@ATL@@QAE@XZ 004f408b f i atls:atlbase.obj
 0001:000f30a5       ??1CAtlBaseModule@ATL@@QAE@XZ 004f40a5 f   atls:atlbase.obj
 0001:000f30bb       ??0CAtlBaseModule@ATL@@QAE@XZ 004f40bb f   atls:atlbase.obj
 0001:000f316a       _RtlUnwind@16              004f416a f   kernel32:KERNEL32.dll
 0001:000f3170       _stricmp                   004f4170 f   LIBC:stricmp.obj
 0001:000f3170       __stricmp                  004f4170 f   LIBC:stricmp.obj
 0001:000f31c0       ___ascii_stricmp           004f41c0 f   LIBC:_stricmp.obj
 0002:00000000       __imp__RegCreateKeyExA@36  0050a000     advapi32:ADVAPI32.dll
 0002:00000004       __imp__RegCloseKey@4       0050a004     advapi32:ADVAPI32.dll
 0002:00000008       __imp__RegQueryInfoKeyA@48 0050a008     advapi32:ADVAPI32.dll
 0002:0000000c       __imp__RegSetValueExA@24   0050a00c     advapi32:ADVAPI32.dll
 0002:00000010       __imp__RegEnumKeyExA@32    0050a010     advapi32:ADVAPI32.dll
 0002:00000014       __imp__RegQueryValueExA@24 0050a014     advapi32:ADVAPI32.dll
 0002:00000018       __imp__RegOpenKeyA@12      0050a018     advapi32:ADVAPI32.dll
 0002:0000001c       __imp__RegDeleteKeyA@8     0050a01c     advapi32:ADVAPI32.dll
 0002:00000020       __imp__RegDeleteValueA@8   0050a020     advapi32:ADVAPI32.dll
 0002:00000024       __imp__RegOpenKeyExA@20    0050a024     advapi32:ADVAPI32.dll
 0002:00000028       \177ADVAPI32_NULL_THUNK_DATA 0050a028     advapi32:ADVAPI32.dll
 0002:0000002c       __imp__DirectDrawCreateEx@16 0050a02c     gapidraw:DDRAW.dll
 0002:00000030       \177DDRAW_NULL_THUNK_DATA  0050a030     gapidraw:DDRAW.dll
 0002:00000034       __imp__GdiFlush@0          0050a034     gdi32:GDI32.dll
 0002:00000038       __imp__GetStockObject@4    0050a038     gdi32:GDI32.dll
 0002:0000003c       __imp__GetObjectA@12       0050a03c     gdi32:GDI32.dll
 0002:00000040       __imp__GetDeviceCaps@8     0050a040     gdi32:GDI32.dll
 0002:00000044       __imp__CreateSolidBrush@4  0050a044     gdi32:GDI32.dll
 0002:00000048       __imp__CreateCompatibleBitmap@12 0050a048     gdi32:GDI32.dll
 0002:0000004c       __imp__BitBlt@36           0050a04c     gdi32:GDI32.dll
 0002:00000050       __imp__CreateCompatibleDC@4 0050a050     gdi32:GDI32.dll
 0002:00000054       __imp__CreateDIBSection@24 0050a054     gdi32:GDI32.dll
 0002:00000058       __imp__SelectObject@8      0050a058     gdi32:GDI32.dll
 0002:0000005c       __imp__DeleteDC@4          0050a05c     gdi32:GDI32.dll
 0002:00000060       __imp__DeleteObject@4      0050a060     gdi32:GDI32.dll
 0002:00000064       \177GDI32_NULL_THUNK_DATA  0050a064     gdi32:GDI32.dll
 0002:00000068       __imp__GetModuleFileNameA@12 0050a068     kernel32:KERNEL32.dll
 0002:0000006c       __imp__GetPrivateProfileIntA@16 0050a06c     kernel32:KERNEL32.dll
 0002:00000070       __imp__GetPrivateProfileStringA@24 0050a070     kernel32:KERNEL32.dll
 0002:00000074       __imp__CreateDirectoryA@8  0050a074     kernel32:KERNEL32.dll
 0002:00000078       __imp__SetThreadPriority@8 0050a078     kernel32:KERNEL32.dll
 0002:0000007c       __imp__GetCurrentThread@0  0050a07c     kernel32:KERNEL32.dll
 0002:00000080       __imp__SetFilePointer@16   0050a080     kernel32:KERNEL32.dll
 0002:00000084       __imp__CreateFileA@28      0050a084     kernel32:KERNEL32.dll
 0002:00000088       __imp__CloseHandle@4       0050a088     kernel32:KERNEL32.dll
 0002:0000008c       __imp__ReadFile@20         0050a08c     kernel32:KERNEL32.dll
 0002:00000090       __imp__SystemTimeToFileTime@8 0050a090     kernel32:KERNEL32.dll
 0002:00000094       __imp__GetCurrentDirectoryA@8 0050a094     kernel32:KERNEL32.dll
 0002:00000098       __imp__LocalFileTimeToFileTime@8 0050a098     kernel32:KERNEL32.dll
 0002:0000009c       __imp__GetFileAttributesA@4 0050a09c     kernel32:KERNEL32.dll
 0002:000000a0       __imp__SetFileTime@16      0050a0a0     kernel32:KERNEL32.dll
 0002:000000a4       __imp__WriteFile@20        0050a0a4     kernel32:KERNEL32.dll
 0002:000000a8       __imp__GetVersionExA@4     0050a0a8     kernel32:KERNEL32.dll
 0002:000000ac       __imp__GetLastError@0      0050a0ac     kernel32:KERNEL32.dll
 0002:000000b0       __imp__CreateMutexA@12     0050a0b0     kernel32:KERNEL32.dll
 0002:000000b4       __imp__GetEnvironmentVariableA@12 0050a0b4     kernel32:KERNEL32.dll
 0002:000000b8       __imp__InterlockedExchange@8 0050a0b8     kernel32:KERNEL32.dll
 0002:000000bc       __imp__GetACP@0            0050a0bc     kernel32:KERNEL32.dll
 0002:000000c0       __imp__GetLocaleInfoA@16   0050a0c0     kernel32:KERNEL32.dll
 0002:000000c4       __imp__GetThreadLocale@0   0050a0c4     kernel32:KERNEL32.dll
 0002:000000c8       __imp__FreeLibrary@4       0050a0c8     kernel32:KERNEL32.dll
 0002:000000cc       __imp__GetProcAddress@8    0050a0cc     kernel32:KERNEL32.dll
 0002:000000d0       __imp__LoadLibraryA@4      0050a0d0     kernel32:KERNEL32.dll
 0002:000000d4       __imp__lstrlenA@4          0050a0d4     kernel32:KERNEL32.dll
 0002:000000d8       __imp__GlobalUnlock@4      0050a0d8     kernel32:KERNEL32.dll
 0002:000000dc       __imp__GlobalLock@4        0050a0dc     kernel32:KERNEL32.dll
 0002:000000e0       __imp__GlobalAlloc@8       0050a0e0     kernel32:KERNEL32.dll
 0002:000000e4       __imp__MultiByteToWideChar@24 0050a0e4     kernel32:KERNEL32.dll
 0002:000000e8       __imp__HeapFree@12         0050a0e8     kernel32:KERNEL32.dll
 0002:000000ec       __imp__GetProcessHeap@0    0050a0ec     kernel32:KERNEL32.dll
 0002:000000f0       __imp__lstrcmpA@8          0050a0f0     kernel32:KERNEL32.dll
 0002:000000f4       __imp__lstrlenW@4          0050a0f4     kernel32:KERNEL32.dll
 0002:000000f8       __imp__WideCharToMultiByte@32 0050a0f8     kernel32:KERNEL32.dll
 0002:000000fc       __imp__MulDiv@12           0050a0fc     kernel32:KERNEL32.dll
 0002:00000100       __imp__InitializeCriticalSection@4 0050a100     kernel32:KERNEL32.dll
 0002:00000104       __imp__Sleep@4             0050a104     kernel32:KERNEL32.dll
 0002:00000108       __imp__InterlockedIncrement@4 0050a108     kernel32:KERNEL32.dll
 0002:0000010c       __imp__InterlockedDecrement@4 0050a10c     kernel32:KERNEL32.dll
 0002:00000110       __imp__EnterCriticalSection@4 0050a110     kernel32:KERNEL32.dll
 0002:00000114       __imp__HeapAlloc@12        0050a114     kernel32:KERNEL32.dll
 0002:00000118       __imp__FlushInstructionCache@12 0050a118     kernel32:KERNEL32.dll
 0002:0000011c       __imp__GetCurrentProcess@0 0050a11c     kernel32:KERNEL32.dll
 0002:00000120       __imp__GetCurrentThreadId@0 0050a120     kernel32:KERNEL32.dll
 0002:00000124       __imp__RaiseException@16   0050a124     kernel32:KERNEL32.dll
 0002:00000128       __imp__LeaveCriticalSection@4 0050a128     kernel32:KERNEL32.dll
 0002:0000012c       __imp__GetModuleHandleA@4  0050a12c     kernel32:KERNEL32.dll
 0002:00000130       __imp__SizeofResource@8    0050a130     kernel32:KERNEL32.dll
 0002:00000134       __imp__LoadResource@8      0050a134     kernel32:KERNEL32.dll
 0002:00000138       __imp__FindResourceA@12    0050a138     kernel32:KERNEL32.dll
 0002:0000013c       __imp__LoadLibraryExA@12   0050a13c     kernel32:KERNEL32.dll
 0002:00000140       __imp__lstrcmpiA@8         0050a140     kernel32:KERNEL32.dll
 0002:00000144       __imp__lstrcpynA@12        0050a144     kernel32:KERNEL32.dll
 0002:00000148       __imp__IsDBCSLeadByte@4    0050a148     kernel32:KERNEL32.dll
 0002:0000014c       __imp__UnmapViewOfFile@4   0050a14c     kernel32:KERNEL32.dll
 0002:00000150       __imp__GetFileSize@8       0050a150     kernel32:KERNEL32.dll
 0002:00000154       __imp__MapViewOfFile@20    0050a154     kernel32:KERNEL32.dll
 0002:00000158       __imp__CreateFileMappingA@24 0050a158     kernel32:KERNEL32.dll
 0002:0000015c       __imp__GetFullPathNameA@16 0050a15c     kernel32:KERNEL32.dll
 0002:00000160       __imp__GlobalFree@4        0050a160     kernel32:KERNEL32.dll
 0002:00000164       __imp__QueryPerformanceCounter@4 0050a164     kernel32:KERNEL32.dll
 0002:00000168       __imp__QueryPerformanceFrequency@4 0050a168     kernel32:KERNEL32.dll
 0002:0000016c       __imp__GetTickCount@0      0050a16c     kernel32:KERNEL32.dll
 0002:00000170       __imp__LCMapStringW@24     0050a170     kernel32:KERNEL32.dll
 0002:00000174       __imp__GetTimeZoneInformation@4 0050a174     kernel32:KERNEL32.dll
 0002:00000178       __imp__FlushFileBuffers@4  0050a178     kernel32:KERNEL32.dll
 0002:0000017c       __imp__HeapDestroy@4       0050a17c     kernel32:KERNEL32.dll
 0002:00000180       __imp__HeapCreate@12       0050a180     kernel32:KERNEL32.dll
 0002:00000184       __imp__VirtualFree@12      0050a184     kernel32:KERNEL32.dll
 0002:00000188       __imp__IsBadWritePtr@8     0050a188     kernel32:KERNEL32.dll
 0002:0000018c       __imp__GetOEMCP@0          0050a18c     kernel32:KERNEL32.dll
 0002:00000190       __imp__GetCPInfo@8         0050a190     kernel32:KERNEL32.dll
 0002:00000194       __imp__HeapSize@12         0050a194     kernel32:KERNEL32.dll
 0002:00000198       __imp__SetHandleCount@4    0050a198     kernel32:KERNEL32.dll
 0002:0000019c       __imp__GetStdHandle@4      0050a19c     kernel32:KERNEL32.dll
 0002:000001a0       __imp__RtlUnwind@16        0050a1a0     kernel32:KERNEL32.dll
 0002:000001a4       __imp__GetFileType@4       0050a1a4     kernel32:KERNEL32.dll
 0002:000001a8       __imp__GetSystemTimeAsFileTime@4 0050a1a8     kernel32:KERNEL32.dll
 0002:000001ac       __imp__ExitProcess@4       0050a1ac     kernel32:KERNEL32.dll
 0002:000001b0       __imp__TerminateProcess@8  0050a1b0     kernel32:KERNEL32.dll
 0002:000001b4       __imp__DeleteFileA@4       0050a1b4     kernel32:KERNEL32.dll
 0002:000001b8       __imp__VirtualProtect@16   0050a1b8     kernel32:KERNEL32.dll
 0002:000001bc       __imp__VirtualAlloc@16     0050a1bc     kernel32:KERNEL32.dll
 0002:000001c0       __imp__GetSystemInfo@4     0050a1c0     kernel32:KERNEL32.dll
 0002:000001c4       __imp__VirtualQuery@12     0050a1c4     kernel32:KERNEL32.dll
 0002:000001c8       __imp__HeapReAlloc@16      0050a1c8     kernel32:KERNEL32.dll
 0002:000001cc       __imp__GetStartupInfoA@4   0050a1cc     kernel32:KERNEL32.dll
 0002:000001d0       __imp__GetCommandLineA@0   0050a1d0     kernel32:KERNEL32.dll
 0002:000001d4       __imp__LCMapStringA@24     0050a1d4     kernel32:KERNEL32.dll
 0002:000001d8       __imp__SetUnhandledExceptionFilter@4 0050a1d8     kernel32:KERNEL32.dll
 0002:000001dc       __imp__UnhandledExceptionFilter@4 0050a1dc     kernel32:KERNEL32.dll
 0002:000001e0       __imp__FreeEnvironmentStringsA@4 0050a1e0     kernel32:KERNEL32.dll
 0002:000001e4       __imp__GetEnvironmentStrings@0 0050a1e4     kernel32:KERNEL32.dll
 0002:000001e8       __imp__FreeEnvironmentStringsW@4 0050a1e8     kernel32:KERNEL32.dll
 0002:000001ec       __imp__GetEnvironmentStringsW@0 0050a1ec     kernel32:KERNEL32.dll
 0002:000001f0       __imp__IsBadReadPtr@8      0050a1f0     kernel32:KERNEL32.dll
 0002:000001f4       __imp__IsBadCodePtr@4      0050a1f4     kernel32:KERNEL32.dll
 0002:000001f8       __imp__SetStdHandle@8      0050a1f8     kernel32:KERNEL32.dll
 0002:000001fc       __imp__GetStringTypeA@20   0050a1fc     kernel32:KERNEL32.dll
 0002:00000200       __imp__GetStringTypeW@16   0050a200     kernel32:KERNEL32.dll
 0002:00000204       __imp__GetCurrentProcessId@0 0050a204     kernel32:KERNEL32.dll
 0002:00000208       __imp__SetEndOfFile@4      0050a208     kernel32:KERNEL32.dll
 0002:0000020c       __imp__CompareStringA@24   0050a20c     kernel32:KERNEL32.dll
 0002:00000210       __imp__CompareStringW@24   0050a210     kernel32:KERNEL32.dll
 0002:00000214       __imp__DeleteCriticalSection@4 0050a214     kernel32:KERNEL32.dll
 0002:00000218       __imp__SetEnvironmentVariableA@8 0050a218     kernel32:KERNEL32.dll
 0002:0000021c       \177KERNEL32_NULL_THUNK_DATA 0050a21c     kernel32:KERNEL32.dll
 0002:00000220       __imp__SysFreeString@4     0050a220     oleaut32:OLEAUT32.dll
 0002:00000224       __imp__SysAllocStringLen@8 0050a224     oleaut32:OLEAUT32.dll
 0002:00000228       __imp__SysStringLen@4      0050a228     oleaut32:OLEAUT32.dll
 0002:0000022c       __imp__SysAllocString@4    0050a22c     oleaut32:OLEAUT32.dll
 0002:00000230       __imp__VariantInit@4       0050a230     oleaut32:OLEAUT32.dll
 0002:00000234       __imp__VariantClear@4      0050a234     oleaut32:OLEAUT32.dll
 0002:00000238       __imp__SysStringByteLen@4  0050a238     oleaut32:OLEAUT32.dll
 0002:0000023c       __imp__OleCreateFontIndirect@12 0050a23c     oleaut32:OLEAUT32.dll
 0002:00000240       __imp__LoadRegTypeLib@20   0050a240     oleaut32:OLEAUT32.dll
 0002:00000244       __imp__LoadTypeLib@8       0050a244     oleaut32:OLEAUT32.dll
 0002:00000248       __imp__VarUI4FromStr@16    0050a248     oleaut32:OLEAUT32.dll
 0002:0000024c       __imp__OleLoadPicture@20   0050a24c     oleaut32:OLEAUT32.dll
 0002:00000250       \177OLEAUT32_NULL_THUNK_DATA 0050a250     oleaut32:OLEAUT32.dll
 0002:00000254       __imp__ShellExecuteA@24    0050a254     shell32:SHELL32.dll
 0002:00000258       __imp__SHGetSpecialFolderPathA@16 0050a258     shell32:SHELL32.dll
 0002:0000025c       \177SHELL32_NULL_THUNK_DATA 0050a25c     shell32:SHELL32.dll
 0002:00000260       __imp__SetRect@20          0050a260     user32:USER32.dll
 0002:00000264       __imp__ClientToScreen@8    0050a264     user32:USER32.dll
 0002:00000268       __imp__GetSystemMetrics@4  0050a268     user32:USER32.dll
 0002:0000026c       __imp__SystemParametersInfoA@16 0050a26c     user32:USER32.dll
 0002:00000270       __imp__AdjustWindowRectEx@16 0050a270     user32:USER32.dll
 0002:00000274       __imp__GetMenu@4           0050a274     user32:USER32.dll
 0002:00000278       __imp__SendMessageA@16     0050a278     user32:USER32.dll
 0002:0000027c       __imp__InvalidateRgn@12    0050a27c     user32:USER32.dll
 0002:00000280       __imp__InvalidateRect@12   0050a280     user32:USER32.dll
 0002:00000284       __imp__SetCapture@4        0050a284     user32:USER32.dll
 0002:00000288       __imp__ReleaseCapture@0    0050a288     user32:USER32.dll
 0002:0000028c       __imp__CreateAcceleratorTableA@8 0050a28c     user32:USER32.dll
 0002:00000290       __imp__ReleaseDC@8         0050a290     user32:USER32.dll
 0002:00000294       __imp__GetDesktopWindow@0  0050a294     user32:USER32.dll
 0002:00000298       __imp__CharNextA@4         0050a298     user32:USER32.dll
 0002:0000029c       __imp__GetParent@4         0050a29c     user32:USER32.dll
 0002:000002a0       __imp__GetClassNameA@12    0050a2a0     user32:USER32.dll
 0002:000002a4       __imp__UnregisterClassA@8  0050a2a4     user32:USER32.dll
 0002:000002a8       __imp__RedrawWindow@16     0050a2a8     user32:USER32.dll
 0002:000002ac       __imp__IsWindow@4          0050a2ac     user32:USER32.dll
 0002:000002b0       __imp__BeginPaint@8        0050a2b0     user32:USER32.dll
 0002:000002b4       __imp__FillRect@12         0050a2b4     user32:USER32.dll
 0002:000002b8       __imp__EndPaint@8          0050a2b8     user32:USER32.dll
 0002:000002bc       __imp__IsChild@8           0050a2bc     user32:USER32.dll
 0002:000002c0       __imp__GetFocus@0          0050a2c0     user32:USER32.dll
 0002:000002c4       __imp__GetWindow@8         0050a2c4     user32:USER32.dll
 0002:000002c8       __imp__GetSysColor@4       0050a2c8     user32:USER32.dll
 0002:000002cc       __imp__DestroyAcceleratorTable@4 0050a2cc     user32:USER32.dll
 0002:000002d0       __imp__GetWindowTextLengthA@4 0050a2d0     user32:USER32.dll
 0002:000002d4       __imp__GetWindowTextA@12   0050a2d4     user32:USER32.dll
 0002:000002d8       __imp__SetWindowTextA@8    0050a2d8     user32:USER32.dll
 0002:000002dc       __imp__RegisterWindowMessageA@4 0050a2dc     user32:USER32.dll
 0002:000002e0       __imp__GetClassInfoExA@12  0050a2e0     user32:USER32.dll
 0002:000002e4       __imp__LoadCursorA@8       0050a2e4     user32:USER32.dll
 0002:000002e8       __imp__RegisterClassExA@4  0050a2e8     user32:USER32.dll
 0002:000002ec       __imp__GetClientRect@8     0050a2ec     user32:USER32.dll
 0002:000002f0       __imp__GetDC@4             0050a2f0     user32:USER32.dll
 0002:000002f4       __imp__CallWindowProcA@20  0050a2f4     user32:USER32.dll
 0002:000002f8       __imp__SetWindowPos@28     0050a2f8     user32:USER32.dll
 0002:000002fc       __imp__GetDlgItem@8        0050a2fc     user32:USER32.dll
 0002:00000300       __imp__SetForegroundWindow@4 0050a300     user32:USER32.dll
 0002:00000304       __imp__IsIconic@4          0050a304     user32:USER32.dll
 0002:00000308       __imp__wsprintfA           0050a308     user32:USER32.dll
 0002:0000030c       __imp__GetWindowLongA@8    0050a30c     user32:USER32.dll
 0002:00000310       __imp__SetWindowLongA@12   0050a310     user32:USER32.dll
 0002:00000314       __imp__MsgWaitForMultipleObjects@20 0050a314     user32:USER32.dll
 0002:00000318       __imp__GetCursorPos@4      0050a318     user32:USER32.dll
 0002:0000031c       __imp__ScreenToClient@8    0050a31c     user32:USER32.dll
 0002:00000320       __imp__PostQuitMessage@4   0050a320     user32:USER32.dll
 0002:00000324       __imp__SetCursor@4         0050a324     user32:USER32.dll
 0002:00000328       __imp__PostMessageA@16     0050a328     user32:USER32.dll
 0002:0000032c       __imp__DefWindowProcA@16   0050a32c     user32:USER32.dll
 0002:00000330       __imp__DestroyWindow@4     0050a330     user32:USER32.dll
 0002:00000334       __imp__LoadIconA@8         0050a334     user32:USER32.dll
 0002:00000338       __imp__RegisterClassA@4    0050a338     user32:USER32.dll
 0002:0000033c       __imp__CreateWindowExA@48  0050a33c     user32:USER32.dll
 0002:00000340       __imp__GetWindowRect@8     0050a340     user32:USER32.dll
 0002:00000344       __imp__MoveWindow@24       0050a344     user32:USER32.dll
 0002:00000348       __imp__SetFocus@4          0050a348     user32:USER32.dll
 0002:0000034c       __imp__ShowWindow@8        0050a34c     user32:USER32.dll
 0002:00000350       __imp__UpdateWindow@4      0050a350     user32:USER32.dll
 0002:00000354       __imp__PeekMessageA@20     0050a354     user32:USER32.dll
 0002:00000358       __imp__TranslateMessage@4  0050a358     user32:USER32.dll
 0002:0000035c       __imp__DispatchMessageA@4  0050a35c     user32:USER32.dll
 0002:00000360       __imp__GetKeyState@4       0050a360     user32:USER32.dll
 0002:00000364       __imp__MessageBoxA@16      0050a364     user32:USER32.dll
 0002:00000368       \177USER32_NULL_THUNK_DATA 0050a368     user32:USER32.dll
 0002:0000036c       __imp__InternetCloseHandle@4 0050a36c     wininet:WININET.dll
 0002:00000370       __imp__HttpSendRequestA@20 0050a370     wininet:WININET.dll
 0002:00000374       __imp__HttpOpenRequestA@32 0050a374     wininet:WININET.dll
 0002:00000378       __imp__InternetConnectA@32 0050a378     wininet:WININET.dll
 0002:0000037c       __imp__InternetReadFile@16 0050a37c     wininet:WININET.dll
 0002:00000380       __imp__InternetOpenA@20    0050a380     wininet:WININET.dll
 0002:00000384       \177WININET_NULL_THUNK_DATA 0050a384     wininet:WININET.dll
 0002:00000388       __imp__timeEndPeriod@4     0050a388     gapidraw:WINMM.dll
 0002:0000038c       __imp__timeBeginPeriod@4   0050a38c     gapidraw:WINMM.dll
 0002:00000390       __imp__timeGetTime@0       0050a390     gapidraw:WINMM.dll
 0002:00000394       \177WINMM_NULL_THUNK_DATA  0050a394     gapidraw:WINMM.dll
 0002:00000398       __imp__FSOUND_PlaySound@8  0050a398     fmodvc:fmod.dll
 0002:0000039c       __imp__FSOUND_SetVolume@8  0050a39c     fmodvc:fmod.dll
 0002:000003a0       __imp__FSOUND_StopSound@4  0050a3a0     fmodvc:fmod.dll
 0002:000003a4       __imp__FSOUND_SetSFXMasterVolume@4 0050a3a4     fmodvc:fmod.dll
 0002:000003a8       __imp__FSOUND_IsPlaying@4  0050a3a8     fmodvc:fmod.dll
 0002:000003ac       __imp__FMUSIC_LoadSong@4   0050a3ac     fmodvc:fmod.dll
 0002:000003b0       __imp__FSOUND_Stream_Open@16 0050a3b0     fmodvc:fmod.dll
 0002:000003b4       __imp__FMUSIC_SetMasterVolume@8 0050a3b4     fmodvc:fmod.dll
 0002:000003b8       __imp__FMUSIC_FreeSong@4   0050a3b8     fmodvc:fmod.dll
 0002:000003bc       __imp__FSOUND_Close@0      0050a3bc     fmodvc:fmod.dll
 0002:000003c0       __imp__FSOUND_Sample_Free@4 0050a3c0     fmodvc:fmod.dll
 0002:000003c4       __imp__FSOUND_Init@12      0050a3c4     fmodvc:fmod.dll
 0002:000003c8       __imp__FSOUND_Sample_SetMode@8 0050a3c8     fmodvc:fmod.dll
 0002:000003cc       __imp__FSOUND_Stream_GetTime@4 0050a3cc     fmodvc:fmod.dll
 0002:000003d0       __imp__FMUSIC_GetTime@4    0050a3d0     fmodvc:fmod.dll
 0002:000003d4       __imp__FMUSIC_IsPlaying@4  0050a3d4     fmodvc:fmod.dll
 0002:000003d8       __imp__FSOUND_Stream_Stop@4 0050a3d8     fmodvc:fmod.dll
 0002:000003dc       __imp__FMUSIC_StopSong@4   0050a3dc     fmodvc:fmod.dll
 0002:000003e0       __imp__FMUSIC_StopAllSongs@0 0050a3e0     fmodvc:fmod.dll
 0002:000003e4       __imp__FSOUND_Stream_SetMode@8 0050a3e4     fmodvc:fmod.dll
 0002:000003e8       __imp__FSOUND_Stream_Play@8 0050a3e8     fmodvc:fmod.dll
 0002:000003ec       __imp__FMUSIC_SetLooping@8 0050a3ec     fmodvc:fmod.dll
 0002:000003f0       __imp__FMUSIC_PlaySong@4   0050a3f0     fmodvc:fmod.dll
 0002:000003f4       __imp__FSOUND_Stream_Close@4 0050a3f4     fmodvc:fmod.dll
 0002:000003f8       __imp__FSOUND_Sample_Load@20 0050a3f8     fmodvc:fmod.dll
 0002:000003fc       \177fmod_NULL_THUNK_DATA   0050a3fc     fmodvc:fmod.dll
 0002:00000400       __imp__OleUninitialize@0   0050a400     ole32:ole32.dll
 0002:00000404       __imp__CreateStreamOnHGlobal@12 0050a404     ole32:ole32.dll
 0002:00000408       __imp__OleInitialize@4     0050a408     ole32:ole32.dll
 0002:0000040c       __imp__CoGetClassObject@20 0050a40c     ole32:ole32.dll
 0002:00000410       __imp__CLSIDFromProgID@8   0050a410     ole32:ole32.dll
 0002:00000414       __imp__CLSIDFromString@8   0050a414     ole32:ole32.dll
 0002:00000418       __imp__StringFromGUID2@12  0050a418     ole32:ole32.dll
 0002:0000041c       __imp__CoTaskMemAlloc@4    0050a41c     ole32:ole32.dll
 0002:00000420       __imp__OleLockRunning@12   0050a420     ole32:ole32.dll
 0002:00000424       __imp__CoTaskMemFree@4     0050a424     ole32:ole32.dll
 0002:00000428       __imp__CoTaskMemRealloc@8  0050a428     ole32:ole32.dll
 0002:0000042c       __imp__CoCreateInstance@20 0050a42c     ole32:ole32.dll
 0002:00000430       \177ole32_NULL_THUNK_DATA  0050a430     ole32:ole32.dll
 0002:00000440       ??_7ldwButton@@6B@         0050a440     ldwButton.obj
 0002:0000046c       ??_7ldwButtonImpl@@6B@     0050a46c     ldwButton.obj
 0002:0000047c       ??_7ldwEventHandler@@6B@   0050a47c     ldwButton.obj
 0002:0000048c       ??_7ldwDialog@@6B@         0050a48c     ldwDialog.obj
 0002:000004bc       ??_7ldwFont@@6B@           0050a4bc     ldwFont.obj
 0002:000004f4       ??_7ldwGame@@6B@           0050a4f4     ldwGame.obj
 0002:000005c8       ??_7ldwGameState@@6B@      0050a5c8     ldwGameState.obj
 0002:00000608       __real@0000000000000000    0050a608     ldwGameState.obj
 0002:00000614       ??_C@_08KEGJFKPE@UseVsync?$AA@ 0050a614     ldwGameWindow.obj
 0002:00000620       ??_C@_07LKOONPMF@ldw?4ini?$AA@ 0050a620     ldwGameWindow.obj
 0002:00000628       ??_7ldwGapiApp@@6B@        0050a628     ldwGameWindow.obj
 0002:00000674       __real@40000000            0050a674     ldwGameWindow.obj
 0002:00000678       __real@3f000000            0050a678     ldwGameWindow.obj
 0002:0000067c       __real@437f0000            0050a67c     ldwGameWindow.obj
 0002:00000680       __real@42c80000            0050a680     ldwGameWindow.obj
 0002:00000684       __real@3f400000            0050a684     ldwGameWindow.obj
 0002:00000688       ??_C@_00CNPNBAHC@?$AA@     0050a688     ldwGameWindow.obj
 0002:0000068c       ??_C@_04EEOGCCFB@?4png?$AA@ 0050a68c     ldwGameWindow.obj
 0002:00000818       ??_7CGapiApplication@@6B@  0050a818     ldwGapiApplication.obj
 0002:00000864       ??_7ldwHintControl@@6B@    0050a864     ldwHintControl.obj
 0002:00000884       ??_7ldwHintControlImpl@@6B@ 0050a884     ldwHintControl.obj
 0002:00000894       ??_7ldwControl@@6B@        0050a894     ldwHintControl.obj
 0002:000008c0       ??_7ldwImage@@6B@          0050a8c0     ldwImage.obj
 0002:000008c4       ??_7ldwImageStrip@@6B@     0050a8c4     ldwImage.obj
 0002:000008c8       ??_7ldwImageGrid@@6B@      0050a8c8     ldwImage.obj
 0002:0000099c       ??_C@_02BKFDOEMK@wt?$AA@   0050a99c     ldwLog.obj
 0002:000009a0       ??_C@_02CPIDLAI@at?$AA@    0050a9a0     ldwLog.obj
 0002:000009a4       ??_C@_0L@BPFILHAC@ldwLog?4txt?$AA@ 0050a9a4     ldwLog.obj
 0002:000009b0       ??_C@_04PFAOODAA@?$CFs?3?5?$AA@ 0050a9b0     ldwLog.obj
 0002:000009b8       ??_7ldwRadioButton@@6B@    0050a9b8     ldwRadioButton.obj
 0002:000009d8       ??_7ldwRadioButtonImpl@@6B@ 0050a9d8     ldwRadioButton.obj
 0002:000009e8       ??_7ldwScene@@6B@          0050a9e8     ldwScene.obj
 0002:00000a10       ??_C@_0BN@EFBNMPLE@ldwSoundFx?5Missing?5File?5?9?$DO?$CFs?$AA@ 0050aa10     ldwSound.obj
 0002:00000a30       ??_C@_03NKNKOHHD@ogg?$AA@  0050aa30     ldwSound.obj
 0002:00000a34       ??_C@_03BICDMHKB@wav?$AA@  0050aa34     ldwSound.obj
 0002:00000a38       ??_C@_03LHGNACFN@mp3?$AA@  0050aa38     ldwSound.obj
 0002:00000a3c       ??_7ldwSoundTrackImpl@@6B@ 0050aa3c     ldwSound.obj
 0002:00000a4c       __real@43800000            0050aa4c     ldwSound.obj
 0002:00000a50       ??_7ldwTextControl@@6B@    0050aa50     ldwTextControl.obj
 0002:00000a70       ??_7ldwTextControlImpl@@6B@ 0050aa70     ldwTextControl.obj
 0002:00000a80       ??_C@_02DPKJAMEF@?$CFd?$AA@ 0050aa80     ldwTextControl.obj
 0002:00000a84       ??_7ldwTiledBackground@@6B@ 0050aa84     ldwTiledBackground.obj
 0002:00000a98       ??_7ldwBackground@@6B@     0050aa98     ldwTiledBackground.obj
 0002:00000aa8       ??_7ldwTiledDialog@@6B@    0050aaa8     ldwTiledDialog.obj
 0002:00000adc       __real@00000000            0050aadc     ldwTiledDialog.obj
 0002:00000ae0       __real@3f800000            0050aae0     ldwTiledDialog.obj
 0002:00000ae4       __real@3f333333            0050aae4     ldwTiledDialog.obj
 0002:00001dd0       ?inflate_copyright@@3QBDB  0050bdd0     unzip.obj
 0002:00002b10       __real@4008000000000000    0050cb10     Villager.obj
 0002:00002b18       __real@3fc00000            0050cb18     Villager.obj
 0002:00002b1c       __real@442f0000            0050cb1c     Villager.obj
 0002:00002b20       __real@425c0000            0050cb20     Villager.obj
 0002:00002b24       __real@41a00000            0050cb24     Villager.obj
 0002:000036b4       ??_7CVillagerManager@@6B@  0050d6b4     VillagerManager.obj
 0002:000036b8       ??_7IDebugger@@6B@         0050d6b8     VillagerManager.obj
 0002:000036bc       __real@42a00000            0050d6bc     VillagerManager.obj
 0002:000036c0       __real@41600000            0050d6c0     VillagerManager.obj
 0002:00003724       ??_7CCollectionScene@@6B@  0050d724     CollectionScene.obj
 0002:00003768       ??_7CProgressScene@@6B@    0050d768     ProgressScene.obj
 0002:00003794       ??_7CStoryScene@@6B@       0050d794     StoryScene.obj
 0002:000037e8       ??_7CTechScene@@6B@        0050d7e8     TechScene.obj
 0002:00003810       __real@3ca3d70a            0050d810     TechScene.obj
 0002:00003818       ??_7theHelpScene@@6B@      0050d818     theHelpScene.obj
 0002:00003844       ??_7theLoadingScene@@6B@   0050d844     theLoadingScene.obj
 0002:00003a80       ??_7theMainScene@@6BIDebugger@@@ 0050da80     theMainScene.obj
 0002:00003a84       ??_7theMainScene@@6BldwScene@@@ 0050da84     theMainScene.obj
 0002:00003b60       ??_7theMenuScene@@6B@      0050db60     theMenuScene.obj
 0002:00003b88       __real@3d4ccccd            0050db88     theMenuScene.obj
 0002:00003bb4       ??_7theOverviewScene@@6B@  0050dbb4     theOverviewScene.obj
 0002:00003bdc       __real@3d23d70a            0050dbdc     theOverviewScene.obj
 0002:00003be0       __real@45000000            0050dbe0     theOverviewScene.obj
 0002:00003be4       __real@43d40000            0050dbe4     theOverviewScene.obj
 0002:00003c94       ??_7theSplashScene@@6B@    0050dc94     theSplashScene.obj
 0002:00003cf8       ??_7theVillagerScene@@6B@  0050dcf8     theVillagerScene.obj
 0002:00003d38       ??_7CIslandEventDialog@@6B@ 0050dd38     IslandEvents.obj
 0002:00003d70       ??_7CEventTsunami@@6B@     0050dd70     IslandEvents.obj
 0002:00003db0       ??_7CIslandEvent@@6B@      0050ddb0     IslandEvents.obj
 0002:00003df0       ??_7CEventPlagueOfAnts@@6B@ 0050ddf0     IslandEvents.obj
 0002:00003e30       ??_7CEventScienceFair@@6B@ 0050de30     IslandEvents.obj
 0002:00003e70       ??_7CEventAllergySeason@@6B@ 0050de70     IslandEvents.obj
 0002:00003eb0       ??_7CEventIsolaDay@@6B@    0050deb0     IslandEvents.obj
 0002:00003ef0       ??_7CEventBlessingsDay@@6B@ 0050def0     IslandEvents.obj
 0002:00003f30       ??_7CEventCanoeFromOtherSide@@6B@ 0050df30     IslandEvents.obj
 0002:00003f70       ??_7CEventMysteriousFogFoodBonus@@6B@ 0050df70     IslandEvents.obj
 0002:00003fb0       ??_7CEventMysteriousFogFoodPenalty@@6B@ 0050dfb0     IslandEvents.obj
 0002:00003ff0       ??_7CEventMysteriousFogTechBonus@@6B@ 0050dff0     IslandEvents.obj
 0002:00004030       ??_7CEventMysteriousFogTechPenalty@@6B@ 0050e030     IslandEvents.obj
 0002:00004070       ??_7CEventDayOfHonor@@6B@  0050e070     IslandEvents.obj
 0002:000040b0       ??_7CEventMiraculousBloom@@6B@ 0050e0b0     IslandEvents.obj
 0002:000040f0       ??_7CEventTheReflectionInTheWater@@6B@ 0050e0f0     IslandEvents.obj
 0002:00004130       ??_7CEventTheChiefsAddress@@6B@ 0050e130     IslandEvents.obj
 0002:00004170       ??_7CEventTheRainySeason@@6B@ 0050e170     IslandEvents.obj
 0002:000041b0       ??_7CEventTheColdSnap@@6B@ 0050e1b0     IslandEvents.obj
 0002:000041f0       ??_7CEventTheSaltyAir@@6B@ 0050e1f0     IslandEvents.obj
 0002:00004230       ??_7CEventTheOppressiveHumidity@@6B@ 0050e230     IslandEvents.obj
 0002:00004270       ??_7CEventFoggyHeaded@@6B@ 0050e270     IslandEvents.obj
 0002:000042b0       ??_7CEventTheStingingJellyfish@@6B@ 0050e2b0     IslandEvents.obj
 0002:000042f0       ??_7CEventTheMushroomCelebration@@6B@ 0050e2f0     IslandEvents.obj
 0002:00004330       ??_7CEventTheYellowGeckos@@6B@ 0050e330     IslandEvents.obj
 0002:00004370       ??_7CEventAnotherBarrelOBabies@@6B@ 0050e370     IslandEvents.obj
 0002:000043b0       ??_7CEventDaredevil@@6B@   0050e3b0     IslandEvents.obj
 0002:000043f0       ??_7CIslandEventChoiceAB@@6B@ 0050e3f0     IslandEvents.obj
 0002:00004430       ??_7CEventGhostlyNatureDream@@6B@ 0050e430     IslandEvents.obj
 0002:00004470       ??_7CEventGhostlyMagicDream@@6B@ 0050e470     IslandEvents.obj
 0002:000044b0       ??_7CEventXtalOfReflections@@6B@ 0050e4b0     IslandEvents.obj
 0002:000044f0       ??_7CEventBitterBrownBeansScience1@@6B@ 0050e4f0     IslandEvents.obj
 0002:00004530       ??_7CEventBitterBrownBeansScience2@@6B@ 0050e530     IslandEvents.obj
 0002:00004570       ??_7CEventAncientTabletScience1@@6B@ 0050e570     IslandEvents.obj
 0002:000045b0       ??_7CEventAncientTabletScience2@@6B@ 0050e5b0     IslandEvents.obj
 0002:000045f0       ??_7CEventTheLowTide@@6B@  0050e5f0     IslandEvents.obj
 0002:00004630       ??_7CEventAntsAndGranary@@6B@ 0050e630     IslandEvents.obj
 0002:00004670       __real@3ea8f5c3            0050e670     IslandEvents.obj
 0002:00004678       ??_7CEventTheGreenPearl@@6B@ 0050e678     IslandEvents.obj
 0002:000046b8       ??_7CEventTheBluePearl@@6B@ 0050e6b8     IslandEvents.obj
 0002:000046f8       ??_7CEventTheLazyApprentice@@6B@ 0050e6f8     IslandEvents.obj
 0002:00004738       ??_7CEventTheOmenInTheClouds@@6B@ 0050e738     IslandEvents.obj
 0002:00004778       ??_7CEventThePlayfulOtters@@6B@ 0050e778     IslandEvents.obj
 0002:000047b8       ??_7CEventTheAntHill@@6B@  0050e7b8     IslandEvents.obj
 0002:000047f8       ??_7CEventTheRedStarfish@@6B@ 0050e7f8     IslandEvents.obj
 0002:00004838       ??_7CEventTheBlueStarfish@@6B@ 0050e838     IslandEvents.obj
 0002:00004878       ??_7CEventTheAntInTheBed@@6B@ 0050e878     IslandEvents.obj
 0002:000048b8       ??_C@_0CL@JOBODING@Ant?5in?5Bed?5Event?3?5?$CFs?5got?5sick?5he@ 0050e8b8     IslandEvents.obj
 0002:000048e8       ??_7CEventTheLoversFemale@@6B@ 0050e8e8     IslandEvents.obj
 0002:00004928       ??_7CEventTheLoversMale@@6B@ 0050e928     IslandEvents.obj
 0002:00004968       ??_7CEventTheMedicalEmergency@@6B@ 0050e968     IslandEvents.obj
 0002:000049a8       ??_7CEventTheQuartzPhial@@6B@ 0050e9a8     IslandEvents.obj
 0002:000049e8       ??_7CEventTheObsidianPhial@@6B@ 0050e9e8     IslandEvents.obj
 0002:00004a28       ??_7CEventTheAmberPhial@@6B@ 0050ea28     IslandEvents.obj
 0002:00004a68       ??_7CEventTheMangoAndThePapaya@@6B@ 0050ea68     IslandEvents.obj
 0002:00004aa8       ??_7CEventTheCrateOfMangosPapayasAndBananas@@6B@ 0050eaa8     IslandEvents.obj
 0002:00004ae8       ??_C@_0EC@MBFHEEMA@TheCrateOfMangosPapayasAndBanana@ 0050eae8     IslandEvents.obj
 0002:00004b30       ??_7CEventTheBee@@6B@      0050eb30     IslandEvents.obj
 0002:00004b70       ??_7CEventTheNoisyBird@@6B@ 0050eb70     IslandEvents.obj
 0002:00004bb0       ??_7CEventTheHoleInTheHut@@6B@ 0050ebb0     IslandEvents.obj
 0002:00004bf0       ??_7CEventTheRoyalJelly@@6B@ 0050ebf0     IslandEvents.obj
 0002:00004c30       ??_7CEventTheShootingStar@@6B@ 0050ec30     IslandEvents.obj
 0002:00004c70       ??_7CEventTheReturnOfBiggles@@6B@ 0050ec70     IslandEvents.obj
 0002:00004cb0       ??_C@_01OGPIMHDM@?$DP?$AA@ 0050ecb0     IslandEvents.obj
 0002:00004cc4       ??_7CRosterOfDeadDialog@@6B@ 0050ecc4     RosterOfDeadDialog.obj
 0002:00004d18       ??_7theChangePlayerDlg@@6B@ 0050ed18     theChangePlayerDlg.obj
 0002:00004d50       ??_7theCreateNickNameDlg@@6B@ 0050ed50     theCreateNickNameDlg.obj
 0002:00004d88       ??_7theFernsaceDialog@@6B@ 0050ed88     theFernsaceDialog.obj
 0002:00004dc0       ??_7theMessageBoxDlg@@6B@  0050edc0     theMessageBoxDlg.obj
 0002:00004e3c       __real@436c0000            0050ee3c     theOptionsDialog.obj
 0002:00004e40       ??_7theOptionsDialog@@6B@  0050ee40     theOptionsDialog.obj
 0002:00004e74       __real@3b8ad8f3            0050ee74     theOptionsDialog.obj
 0002:00004e80       __real@c076800000000000    0050ee80     theTipDialog.obj
 0002:00004e88       ??_7theTipDialog@@6B@      0050ee88     theTipDialog.obj
 0002:00004ec0       __real@4066800000000000    0050eec0     theTipDialog.obj
 0002:00004ec8       __real@400921f9f01b866e    0050eec8     theTipDialog.obj
 0002:00004ef8       ??_7theTombStoneDialog@@6B@ 0050eef8     theTombStoneDialog.obj
 0002:00004f30       __real@3e4ccccd            0050ef30     Fog.obj
 0002:00004f34       __real@3ba3d70a            0050ef34     Fog.obj
 0002:00004f38       __real@3d99999a            0050ef38     Fog.obj
 0002:00004f3c       __real@3e800000            0050ef3c     Fog.obj
 0002:00004f40       __real@43000000            0050ef40     Rain.obj
 0002:00004f44       __real@42700000            0050ef44     Rain.obj
 0002:00004f48       __real@44000000            0050ef48     Rain.obj
 0002:00004f50       __real@c2f00000            0050ef50     SunBeam.obj
 0002:00004f7c       __real@447a0000            0050ef7c     Weather.obj
 0002:00004fa4       __real@3f19999a            0050efa4     ContentMap.obj
 0002:00004fa8       __real@3e400000            0050efa8     ContentMap.obj
 0002:00004fac       __real@3ec00000            0050efac     ContentMap.obj
 0002:00004fb4       ??_7CEnvironment@@6B@      0050efb4     Environment.obj
 0002:00004fb8       ??_7ITechObserver@@6B@     0050efb8     Environment.obj
 0002:00005004       ??_7CEnvironmentalSound@@6B@ 0050f004     EnvironmentalSound.obj
 0002:0000501c       ??_7IVillagerAttachment@@6B@ 0050f01c     EnvironmentalSound.obj
 0002:00005034       __real@3dcccccd            0050f034     EnvironmentalSound.obj
 0002:00005038       __real@43480000            0050f038     EnvironmentalSound.obj
 0002:000062dc       ??_7ldwarialbold@@6B@      005102dc     ldwarialbold.obj
 0002:000062f4       ??_7ldwBurweed27@@6B@      005102f4     ldwBurweed27.obj
 0002:000062fc       ??_C@_07IPNMCAN@success?$AA@ 005102fc     highscore.obj
 0002:00006304       ??_C@_0CJ@IOAANKOE@http?3?1?1www?4ldwsoftware?4com?1score@ 00510304     highscore.obj
 0002:00006330       ??_C@_0P@NHEHBKG@GameWebBrowser?$AA@ 00510330     highscore.obj
 0002:00006340       ??_C@_0BCI@IHGIBODL@game?$DN?$CFd?$CGname?$DN?$CFs?$CGscore_id?$DN?$CFu?$CGscor@ 00510340     highscore.obj
 0002:00006468       ??_C@_02MLAGHBOD@?0?6?$AA@ 00510468     highscore.obj
 0002:0000646c       ??_C@_0L@KLCLFNIA@highscores?$AA@ 0051046c     highscore.obj
 0002:000064d8       __real@40a00000            005104d8     Bird.obj
 0002:000064f0       __real@c0e00000            005104f0     Shark.obj
 0002:000064f4       __real@c0a00000            005104f4     Shark.obj
 0002:000064f8       __real@c0400000            005104f8     Shark.obj
 0002:000064fc       __real@bf800000            005104fc     Shark.obj
 0002:00006500       __real@40400000            00510500     Shark.obj
 0002:00006504       __real@41000000            00510504     Shark.obj
 0002:00006508       __real@40e00000            00510508     Shark.obj
 0002:000065fc       __real@40c00000            005105fc     GameTime.obj
 0002:00006704       ??_7CPotion@@6B@           00510704     Potion.obj
 0002:000067c8       ??_7theGame@@6B@           005107c8     theGame.obj
 0002:00006898       ??_7theGameState@@6B@      00510898     theGameState.obj
 0002:000068e4       ??_7CFloatingAnim@@6B@     005108e4     FloatingAnim.obj
 0002:000068fc       ??_7CSmoke@@6B@            005108fc     Smoke.obj
 0002:00007f40       ??_7CBehaviorEditor@@6B@   00511f40     BehaviorEditor.obj
 0002:00007f60       ??_7IEditor@@6B@           00511f60     BehaviorEditor.obj
 0002:000089d4       ??_7CContentMapEditor@@6B@ 005129d4     ContentMapEditor.obj
 0002:00008b38       ??_7CWaypointEditor@@6B@   00512b38     WaypointEditor.obj
 0002:00008b5c       ??_7CCollectableItem@@6B@  00512b5c     CollectableItem.obj
 0002:00008b68       ??_7ICollectable@@6B@      00512b68     CollectableItem.obj
 0002:00023c98       ??_C@_0DN@HMLOEIEJ@String?5Table?5?$CIsm?4xml?$CJ?5malformed?5@ 0052dc98     theStringManager.obj
 0002:00023cd8       ??_C@_07LDBMOIP@?$DM?1Text?$DO?$AA@ 0052dcd8     theStringManager.obj
 0002:00023ce0       ??_C@_0CI@JCCIOACC@String?5Table?5?$CIsm?4xml?$CJ?5malformed?5@ 0052dce0     theStringManager.obj
 0002:00023d08       ??_C@_07EPIMFEMC@id?$DN?$CC?$CFs?$CC?$AA@ 0052dd08     theStringManager.obj
 0002:00023d10       ??_C@_06FCEEJDHN@sm?4xml?$AA@ 0052dd10     theStringManager.obj
 0002:00023d18       ??_C@_02JDPG@rb?$AA@       0052dd18     theStringManager.obj
 0002:00023d1c       ??_C@_0BG@DGEPLHPK@Unknown?5String?5Id?$CB?$CB?$CB?$CB?$AA@ 0052dd1c     theStringManager.obj
 0002:00023d64       ??_7CAlchemyLab@@6BICollectable@@@ 0052dd64     AlchemyLab.obj
 0002:00023d70       ??_7CAlchemyLab@@6BIPuzzle@@@ 0052dd70     AlchemyLab.obj
 0002:00023d9c       ??_7IPuzzle@@6B@           0052dd9c     AlchemyLab.obj
 0002:00023e0c       ??_7CAlchemyPot@@6BICollectable@@@ 0052de0c     AlchemyPot.obj
 0002:00023e18       ??_7CAlchemyPot@@6BIPuzzle@@@ 0052de18     AlchemyPot.obj
 0002:00023e64       ??_7CAlchemyTable@@6BICollectable@@@ 0052de64     AlchemyTable.obj
 0002:00023e70       ??_7CAlchemyTable@@6BIPuzzle@@@ 0052de70     AlchemyTable.obj
 0002:00023ebc       ??_7CAromatherapy@@6BICollectable@@@ 0052debc     Aromatherapy.obj
 0002:00023ec8       ??_7CAromatherapy@@6BIPuzzle@@@ 0052dec8     Aromatherapy.obj
 0002:00023f14       ??_7CBath@@6B@             0052df14     Bath.obj
 0002:00023f68       ??_7CBeeHive@@6BICollectable@@@ 0052df68     BeeHive.obj
 0002:00023f74       ??_7CBeeHive@@6BIPuzzle@@@ 0052df74     BeeHive.obj
 0002:00023fa0       ??_7CChalkBoard@@6B@       0052dfa0     ChalkBoard.obj
 0002:00023fcc       __real@3c23d70a            0052dfcc     ChalkBoard.obj
 0002:00023fec       ??_7CChief@@6B@            0052dfec     Chief.obj
 0002:00024080       ??_7CConstruction@@6B@     0052e080     Construction.obj
 0002:00024110       ??_7CDoorKey@@6BITechObserver@@@ 0052e110     DoorKey.obj
 0002:00024114       ??_7CDoorKey@@6BICollectable@@@ 0052e114     DoorKey.obj
 0002:00024120       ??_7CDoorKey@@6BIPuzzle@@@ 0052e120     DoorKey.obj
 0002:0002416c       ??_7CFirePit@@6BICollectable@@@ 0052e16c     FirePit.obj
 0002:00024178       ??_7CFirePit@@6BIPuzzle@@@ 0052e178     FirePit.obj
 0002:000241a8       ??_7COrchard@@6BICollectable@@@ 0052e1a8     Orchard.obj
 0002:000241b4       ??_7COrchard@@6BIPuzzle@@@ 0052e1b4     Orchard.obj
 0002:0002421c       ??_7CPrincessStatue@@6B@   0052e21c     PrincessStatue.obj
 0002:00024248       __real@40800000            0052e248     PrincessStatue.obj
 0002:0002424c       __real@4952f000            0052e24c     PrincessStatue.obj
 0002:00024258       ?scm_iPointsRequired@CPuzzle@@0QBHB 0052e258     Puzzle.obj
 0002:000242dc       ??_7CRainLift@@6B@         0052e2dc     RainLift.obj
 0002:00024308       ??_7CRosterOfTheDead@@6BICollectable@@@ 0052e308     RosterOfTheDead.obj
 0002:00024314       ??_7CRosterOfTheDead@@6BIPuzzle@@@ 0052e314     RosterOfTheDead.obj
 0002:00024374       ??_7CRuins@@6BICollectable@@@ 0052e374     Ruins.obj
 0002:00024380       ??_7CRuins@@6BIPuzzle@@@   0052e380     Ruins.obj
 0002:000243ac       ??_7CSharkCharmer@@6BICollectable@@@ 0052e3ac     SharkCharmer.obj
 0002:000243b8       ??_7CSharkCharmer@@6BIPuzzle@@@ 0052e3b8     SharkCharmer.obj
 0002:00024408       ??_7CSunDisk@@6B@          0052e408     SunDisk.obj
 0002:00024438       __real@4069000000000000    0052e438     SunDisk.obj
 0002:00024440       __real@3a83126f            0052e440     SunDisk.obj
 0002:0002446c       ??_7CWeatherDance@@6B@     0052e46c     WeatherDance.obj
 0002:000245e8       ?rgszNeverDelete@CRegParser@ATL@@1QBQBDB 0052e5e8     FlashPlayer.obj
 0002:00024618       _CLSID_StdGlobalInterfaceTable 0052e618     FlashPlayer.obj
 0002:00024628       ??_7CFlashPlayer@@6B@      0052e628     FlashPlayer.obj
 0002:0002464c       ??_7IFlashPlayer@@6B@      0052e64c     FlashPlayer.obj
 0002:00024670       __GUID_d27cdb6c_ae6d_11cf_96b8_444553540000 0052e670     FlashPlayer.obj
 0002:00024680       __GUID_00000000_0000_0000_c000_000000000046 0052e680     FlashPlayer.obj
 0002:00024690       ??_C@_0BB@ICJMLDDL@WM_ATLGETCONTROL?$AA@ 0052e690     FlashPlayer.obj
 0002:000246a4       ??_C@_0O@POPOELFC@WM_ATLGETHOST?$AA@ 0052e6a4     FlashPlayer.obj
 0002:000246b4       __GUID_b6ea2050_048a_11d1_82b9_00c04fb9942e 0052e6b4     FlashPlayer.obj
 0002:000246c4       __GUID_3935bda8_4ed9_495c_8650_e01fc1e38a4b 0052e6c4     FlashPlayer.obj
 0002:000246d4       ??_C@_0L@EFNCNKLF@AtlAxWin71?$AA@ 0052e6d4     FlashPlayer.obj
 0002:000246e0       ??_C@_0O@HHPDHHJB@AtlAxWinLic71?$AA@ 0052e6e0     FlashPlayer.obj
 0002:000246f0       ??_7?$CComPolyObject@VCAxHostWindow@ATL@@@ATL@@6B@ 0052e6f0     FlashPlayer.obj
 0002:00024700       __GUID_0000010f_0000_0000_c000_000000000046 0052e700     FlashPlayer.obj
 0002:00024710       __GUID_bd3f23c0_d43e_11cf_893b_00aa00bdce1a 0052e710     FlashPlayer.obj
 0002:00024720       __GUID_b6ea2051_048a_11d1_82b9_00c04fb9942e 0052e720     FlashPlayer.obj
 0002:00024730       __GUID_b2d0778b_ac99_4c58_a5c8_e7724e5316b5 0052e730     FlashPlayer.obj
 0002:00024740       __GUID_6d5140c1_7436_11ce_8034_00aa006009fa 0052e740     FlashPlayer.obj
 0002:00024750       __GUID_fc4801a3_2ba9_11cf_a229_00aa003d7352 0052e750     FlashPlayer.obj
 0002:00024760       __GUID_0000011b_0000_0000_c000_000000000046 0052e760     FlashPlayer.obj
 0002:00024770       __GUID_b196b289_bab4_101a_b69c_00aa00341d07 0052e770     FlashPlayer.obj
 0002:00024780       __GUID_00000114_0000_0000_c000_000000000046 0052e780     FlashPlayer.obj
 0002:00024790       __GUID_00000119_0000_0000_c000_000000000046 0052e790     FlashPlayer.obj
 0002:000247a0       __GUID_9c2cad80_3424_11cf_b670_00aa004cd6d8 0052e7a0     FlashPlayer.obj
 0002:000247b0       __GUID_922eada0_3424_11cf_b670_00aa004cd6d8 0052e7b0     FlashPlayer.obj
 0002:000247c0       __GUID_00000118_0000_0000_c000_000000000046 0052e7c0     FlashPlayer.obj
 0002:000247d0       __GUID_00020400_0000_0000_c000_000000000046 0052e7d0     FlashPlayer.obj
 0002:000247e0       ?_entries@?1??_GetEntries@CAxHostWindow@ATL@@SGPBU_ATL_INTMAP_ENTRY@3@XZ@4QBU43@B 0052e7e0     FlashPlayer.obj
 0002:000248ac       __GUID_b196b284_bab4_101a_b69c_00aa00341d07 0052e8ac     FlashPlayer.obj
 0002:000248c0       ??_7?$CComContainedObject@VCAxHostWindow@ATL@@@ATL@@6B?$IDispatchImpl@UIAxWinAmbientDispatchEx@@$1?_GUID_b2d0778b_ac99_4c58_a5c8_e7724e5316b5@@3U__s_GUID@@B$1?m_libid@CAtlModule@ATL@@2U_GUID@@A$0PPPP@$0PPPP@VCComTypeInfoHolder@ATL@@@1@@ 0052e8c0     FlashPlayer.obj
 0002:00024950       ??_7?$CComContainedObject@VCAxHostWindow@ATL@@@ATL@@6BIDocHostUIHandler@@@ 0052e950     FlashPlayer.obj
 0002:00024998       ??_7?$CComContainedObject@VCAxHostWindow@ATL@@@ATL@@6BIAdviseSink@@@ 0052e998     FlashPlayer.obj
 0002:000249b8       ??_7?$CComContainedObject@VCAxHostWindow@ATL@@@ATL@@6BIServiceProvider@@@ 0052e9b8     FlashPlayer.obj
 0002:000249c8       ??_7?$CComContainedObject@VCAxHostWindow@ATL@@@ATL@@6B?$IObjectWithSiteImpl@VCAxHostWindow@ATL@@@1@@ 0052e9c8     FlashPlayer.obj
 0002:000249e0       ??_7?$CComContainedObject@VCAxHostWindow@ATL@@@ATL@@6BIOleContainer@@@ 0052e9e0     FlashPlayer.obj
 0002:000249f8       ??_7?$CComContainedObject@VCAxHostWindow@ATL@@@ATL@@6BIOleControlSite@@@ 0052e9f8     FlashPlayer.obj
 0002:00024a20       ??_7?$CComContainedObject@VCAxHostWindow@ATL@@@ATL@@6BIOleInPlaceSiteWindowless@@@ 0052ea20     FlashPlayer.obj
 0002:00024a98       ??_7?$CComContainedObject@VCAxHostWindow@ATL@@@ATL@@6BIOleClientSite@@@ 0052ea98     FlashPlayer.obj
 0002:00024abc       ??_7?$CComContainedObject@VCAxHostWindow@ATL@@@ATL@@6BIAxWinHostWindowLic@@@ 0052eabc     FlashPlayer.obj
 0002:00024ae8       ??_7?$CComContainedObject@VCAxHostWindow@ATL@@@ATL@@6B?$CWindowImpl@VCAxHostWindow@ATL@@VCWindow@2@V?$CWinTraits@$0FGAAAAAA@$0A@@2@@1@@ 0052eae8     FlashPlayer.obj
 0002:00024afc       __GUID_d30c1661_cdaf_11d0_8a3e_00c04fc9e26e 0052eafc     FlashPlayer.obj
 0002:00024b0c       __GUID_7fd52380_4e07_101b_ae2d_08002b2ec713 0052eb0c     FlashPlayer.obj
 0002:00024b1c       ??_C@_06FGFHJIJL@?$CD32770?$AA@ 0052eb1c     FlashPlayer.obj
 0002:00024b24       __GUID_b196b28f_bab4_101a_b69c_00aa00341d07 0052eb24     FlashPlayer.obj
 0002:00024b34       __GUID_8856f961_340a_11d0_a96b_00c04fd705a2 0052eb34     FlashPlayer.obj
 0002:00024b44       __GUID_25336920_03f9_11cf_8fd0_00aa00686f13 0052eb44     FlashPlayer.obj
 0002:00024b54       __GUID_00000122_0000_0000_c000_000000000046 0052eb54     FlashPlayer.obj
 0002:00024b64       __GUID_0000010e_0000_0000_c000_000000000046 0052eb64     FlashPlayer.obj
 0002:00024b74       __GUID_bef6e003_a874_101a_8bba_00aa00300cab 0052eb74     FlashPlayer.obj
 0002:00024b84       __GUID_00000113_0000_0000_c000_000000000046 0052eb84     FlashPlayer.obj
 0002:00024b94       __GUID_00000115_0000_0000_c000_000000000046 0052eb94     FlashPlayer.obj
 0002:00024ba4       __GUID_00000116_0000_0000_c000_000000000046 0052eba4     FlashPlayer.obj
 0002:00024bb4       __GUID_1c2056cc_5ef4_101b_8bc8_00aa003e3b29 0052ebb4     FlashPlayer.obj
 0002:00024bc4       __GUID_00000100_0000_0000_c000_000000000046 0052ebc4     FlashPlayer.obj
 0002:00024bd4       ??_C@_1M@IJFAIKMG@?$AAA?$AAX?$AAW?$AAI?$AAN?$AA?$AA@ 0052ebd4     FlashPlayer.obj
 0002:00024be0       __GUID_0000010d_0000_0000_c000_000000000046 0052ebe0     FlashPlayer.obj
 0002:00024bf0       __GUID_00000127_0000_0000_c000_000000000046 0052ebf0     FlashPlayer.obj
 0002:00024c00       __GUID_3af24292_0c96_11ce_a0cf_00aa00600ab8 0052ec00     FlashPlayer.obj
 0002:00024c10       __GUID_00000112_0000_0000_c000_000000000046 0052ec10     FlashPlayer.obj
 0002:00024c2c       __GUID_00000117_0000_0000_c000_000000000046 0052ec2c     FlashPlayer.obj
 0002:00024c3c       __GUID_b196b288_bab4_101a_b69c_00aa00341d07 0052ec3c     FlashPlayer.obj
 0002:00024c4c       ??_7?$CComObject@V?$CComEnum@UIEnumUnknown@@$1?_GUID_00000100_0000_0000_c000_000000000046@@3U__s_GUID@@BPAUIUnknown@@V?$_CopyInterface@UIUnknown@@@ATL@@VCComMultiThreadModel@6@@ATL@@@ATL@@6B@ 0052ec4c     FlashPlayer.obj
 0002:00024c6c       __GUID_00000109_0000_0000_c000_000000000046 0052ec6c     FlashPlayer.obj
 0002:00024c8c       ?_entries@?1??_GetEntries@?$CComEnum@UIEnumUnknown@@$1?_GUID_00000100_0000_0000_c000_000000000046@@3U__s_GUID@@BPAUIUnknown@@V?$_CopyInterface@UIUnknown@@@ATL@@VCComMultiThreadModel@6@@ATL@@SGPBU_ATL_INTMAP_ENTRY@3@XZ@4QBU43@B 0052ec8c     FlashPlayer.obj
 0002:00024ca4       __GUID_00020412_0000_0000_c000_000000000046 0052eca4     FlashPlayer.obj
 0002:00024cb4       __GUID_00020401_0000_0000_c000_000000000046 0052ecb4     FlashPlayer.obj
 0002:00024cc4       ??_7?$CComObject@VCAxFrameWindow@ATL@@@ATL@@6BIOleInPlaceFrame@@@ 0052ecc4     FlashPlayer.obj
 0002:00024d00       ??_7?$CComObject@VCAxFrameWindow@ATL@@@ATL@@6B?$CWindowImpl@VCAxFrameWindow@ATL@@VCWindow@2@V?$CWinTraits@$0FGAAAAAA@$0A@@2@@1@@ 0052ed00     FlashPlayer.obj
 0002:00024d10       ??_C@_0BD@LIOMMJMF@AXWIN?5Frame?5Window?$AA@ 0052ed10     FlashPlayer.obj
 0002:00024d24       ?_entries@?1??_GetEntries@CAxFrameWindow@ATL@@SGPBU_ATL_INTMAP_ENTRY@3@XZ@4QBU43@B 0052ed24     FlashPlayer.obj
 0002:00024d54       ??_C@_09OOFFBKGI@ATL?3?$CF8?48X?$AA@ 0052ed54     FlashPlayer.obj
 0002:00024d60       ??_7?$CComObject@VCAxUIWindow@ATL@@@ATL@@6BIOleInPlaceUIWindow@@@ 0052ed60     FlashPlayer.obj
 0002:00024d84       ??_7?$CComObject@VCAxUIWindow@ATL@@@ATL@@6B?$CWindowImpl@VCAxUIWindow@ATL@@VCWindow@2@V?$CWinTraits@$0FGAAAAAA@$0A@@2@@1@@ 0052ed84     FlashPlayer.obj
 0002:00024d94       ??_C@_0BA@FJBCDDKK@AXWIN?5UI?5Window?$AA@ 0052ed94     FlashPlayer.obj
 0002:00024da4       ?_entries@?1??_GetEntries@CAxUIWindow@ATL@@SGPBU_ATL_INTMAP_ENTRY@3@XZ@4QBU43@B 0052eda4     FlashPlayer.obj
 0002:00024dc8       ??_7CComModule@ATL@@6B@    0052edc8     FlashPlayer.obj
 0002:00024df0       __GUID_00000146_0000_0000_c000_000000000046 0052edf0     FlashPlayer.obj
 0002:00024e00       ??_C@_1BC@KAILKFFG@?$AAR?$AAE?$AAG?$AAI?$AAS?$AAT?$AAR?$AAY?$AA?$AA@ 0052ee00     FlashPlayer.obj
 0002:00024e14       ??_C@_1BG@JBACFMF@?$AAM?$AAo?$AAd?$AAu?$AAl?$AAe?$AA_?$AAR?$AAa?$AAw?$AA?$AA@ 0052ee14     FlashPlayer.obj
 0002:00024e2c       ??_C@_1O@MNLDABAF@?$AAM?$AAo?$AAd?$AAu?$AAl?$AAe?$AA?$AA@ 0052ee2c     FlashPlayer.obj
 0002:00024e3c       ??_7CRegObject@ATL@@6B@    0052ee3c     FlashPlayer.obj
 0002:00024e54       ??_C@_0BE@NLNNHLLF@HKEY_CURRENT_CONFIG?$AA@ 0052ee54     FlashPlayer.obj
 0002:00024e68       ??_C@_0O@MJDLIIGK@HKEY_DYN_DATA?$AA@ 0052ee68     FlashPlayer.obj
 0002:00024e78       ??_C@_0BG@IDBEHNDO@HKEY_PERFORMANCE_DATA?$AA@ 0052ee78     FlashPlayer.obj
 0002:00024e90       ??_C@_0L@OEMMANAM@HKEY_USERS?$AA@ 0052ee90     FlashPlayer.obj
 0002:00024e9c       ??_C@_0BD@GIIFIKDM@HKEY_LOCAL_MACHINE?$AA@ 0052ee9c     FlashPlayer.obj
 0002:00024eb0       ??_C@_0BC@GMMMKLBI@HKEY_CURRENT_USER?$AA@ 0052eeb0     FlashPlayer.obj
 0002:00024ec4       ??_C@_0BC@JBJOLKMF@HKEY_CLASSES_ROOT?$AA@ 0052eec4     FlashPlayer.obj
 0002:00024ed8       ??_C@_04LEMDOLAJ@HKCC?$AA@ 0052eed8     FlashPlayer.obj
 0002:00024ee0       ??_C@_04POMNGLEL@HKDD?$AA@ 0052eee0     FlashPlayer.obj
 0002:00024ee8       ??_C@_04OFOCGAOH@HKPD?$AA@ 0052eee8     FlashPlayer.obj
 0002:00024ef0       ??_C@_03DLBIJLAB@HKU?$AA@  0052eef0     FlashPlayer.obj
 0002:00024ef4       ??_C@_04CBBMIBLK@HKLM?$AA@ 0052eef4     FlashPlayer.obj
 0002:00024efc       ??_C@_04KIFLFONO@HKCU?$AA@ 0052eefc     FlashPlayer.obj
 0002:00024f04       ??_C@_04OHBKMIBJ@HKCR?$AA@ 0052ef04     FlashPlayer.obj
 0002:00024f10       ?map@?2??HKeyFromString@CRegParser@ATL@@KAPAUHKEY__@@PAD@Z@4QBUkeymap@23@B 0052ef10     FlashPlayer.obj
 0002:00024f80       ??_C@_1M@PPPPCDEP@?$AAA?$AAP?$AAP?$AAI?$AAD?$AA?$AA@ 0052ef80     FlashPlayer.obj
 0002:00024f8c       ??_C@_11LOCGONAA@?$AA?$AA@ 0052ef8c     FlashPlayer.obj
 0002:00024fb4       ??_7CIntroPage1@@6B@       0052efb4     Pages.obj
 0002:00024fcc       ??_7IPage@@6B@             0052efcc     Pages.obj
 0002:00024fe4       ??_7CIntroPage2@@6B@       0052efe4     Pages.obj
 0002:00024ffc       ??_7CIntroPage3@@6B@       0052effc     Pages.obj
 0002:00025014       ??_7CIntroPage4@@6B@       0052f014     Pages.obj
 0002:0002502c       ??_7CIntroPage5@@6B@       0052f02c     Pages.obj
 0002:00025044       ??_7CMidGamePage1@@6B@     0052f044     Pages.obj
 0002:0002505c       ??_7CMidGamePage2@@6B@     0052f05c     Pages.obj
 0002:00025074       ??_7CMidGamePage3@@6B@     0052f074     Pages.obj
 0002:0002508c       ??_7CEndGamePage1@@6B@     0052f08c     Pages.obj
 0002:000250a4       ??_7CEndGamePage2@@6B@     0052f0a4     Pages.obj
 0002:000250bc       ??_7CEndGamePage3@@6B@     0052f0bc     Pages.obj
 0002:000250d4       ??_7CEndGamePage4@@6B@     0052f0d4     Pages.obj
 0002:00025100       ??_7CGapiRGBASurface@@6B@  0052f100     gapidraw:GapiRGBASurface.obj
 0002:00025104       ??_7CGapiSurface@@6B@      0052f104     gapidraw:GapiSurface.obj
 0002:00025108       __real@8@400e8000000000000000 0052f108     gapidraw:GapiSurface.obj
 0002:00025110       __real@4@400f8000000000000000 0052f110     gapidraw:GapiSurface.obj
 0002:00025114       __real@4@3fff8000000000000000 0052f114     gapidraw:GapiSurface.obj
 0002:00025118       __real@4@3ffe8000000000000000 0052f118     gapidraw:GapiSurface.obj
 0002:0002511c       __real@4@3ff8a3d70a3d70a3d800 0052f11c     gapidraw:GapiSurface.obj
 0002:00025120       __real@8@3ff2b702d34afc0c8800 0052f120     gapidraw:GapiSurface.obj
 0002:00025128       __real@4@4015c800000000000000 0052f128     gapidraw:GapiSurface.obj
 0002:00025130       __real@8@00000000000000000000 0052f130     gapidraw:GapiSurface.obj
 0002:00025138       __real@8@40078000000000000000 0052f138     gapidraw:GapiSurface.obj
 0002:00025140       __real@8@3ff98efa351294e9c800 0052f140     gapidraw:GapiSurface.obj
 0002:00025148       ??_7CGapiTimer@@6B@        0052f148     gapidraw:GapiTimer.obj
 0002:00025150       __real@8@4008fa00000000000000 0052f150     gapidraw:GapiTimer.obj
 0002:00025158       ??_7CGapiInput@@6B@        0052f158     gapidraw:GapiInputWin32.obj
 0002:0002515c       ??_7CGapiLib@@6B@          0052f15c     gapidraw:GapiInputWin32.obj
 0002:00025160       ??_7CGapiSurfaceHelper@@6B@ 0052f160     gapidraw:GapiDraw.obj
 0002:00025164       ??_7CGapiDraw@@6B@         0052f164     gapidraw:GapiDraw.obj
 0002:00025168       ??_7?$CGapiSurfaceAdapter@VCGapiDisplay555@@@@6B@ 0052f168     gapidraw:GapiDraw.obj
 0002:0002516c       ??_7CoordAcceptInvalid@operators@@6B@ 0052f16c     gapidraw:GapiDraw.obj
 0002:00025170       ??_7CoordVerify@operators@@6B@ 0052f170     gapidraw:GapiDraw.obj
 0002:00025174       ??_7CoordFixedPoint@operators@@6B@ 0052f174     gapidraw:GapiDraw.obj
 0002:00025178       ??_7CoordNormal@operators@@6B@ 0052f178     gapidraw:GapiDraw.obj
 0002:0002517c       ??_7AlphaOpacityNormal@operators@@6B@ 0052f17c     gapidraw:GapiDraw.obj
 0002:00025180       ??_7AlphaOpacityFast@operators@@6B@ 0052f180     gapidraw:GapiDraw.obj
 0002:00025184       ??_7AlphaOpacityNone@operators@@6B@ 0052f184     gapidraw:GapiDraw.obj
 0002:00025188       ??_7?$PixelAlphaBlendFast32@VCGapiDisplay555@@@operators@@6B@ 0052f188     gapidraw:GapiDraw.obj
 0002:0002518c       ??_7?$PixelAlphaBlendFast@VCGapiDisplay555@@@operators@@6B@ 0052f18c     gapidraw:GapiDraw.obj
 0002:00025190       ??_7?$PixelAlphaBlend32@VCGapiDisplay555@@@operators@@6B@ 0052f190     gapidraw:GapiDraw.obj
 0002:00025194       ??_7?$PixelAlphaBlend@VCGapiDisplay555@@@operators@@6B@ 0052f194     gapidraw:GapiDraw.obj
 0002:00025198       ??_7PixelCopy32@operators@@6B@ 0052f198     gapidraw:GapiDraw.obj
 0002:0002519c       ??_7PixelCopy@operators@@6B@ 0052f19c     gapidraw:GapiDraw.obj
 0002:000251a0       ??_7PredicateDoNothing32@operators@@6B@ 0052f1a0     gapidraw:GapiDraw.obj
 0002:000251a4       ??_7PredicateDoNothing@operators@@6B@ 0052f1a4     gapidraw:GapiDraw.obj
 0002:000251a8       ??_7PredicateCopy32b@operators@@6B@ 0052f1a8     gapidraw:GapiDraw.obj
 0002:000251ac       ??_7PredicateCopy32a@operators@@6B@ 0052f1ac     gapidraw:GapiDraw.obj
 0002:000251b0       ??_7PredicateCopy@operators@@6B@ 0052f1b0     gapidraw:GapiDraw.obj
 0002:000251b4       ??_7PredicateMask32bCheckOnly@operators@@6B@ 0052f1b4     gapidraw:GapiDraw.obj
 0002:000251b8       ??_7PredicateMask32b@operators@@6B@ 0052f1b8     gapidraw:GapiDraw.obj
 0002:000251bc       ??_7PredicateMask32a@operators@@6B@ 0052f1bc     gapidraw:GapiDraw.obj
 0002:000251c0       ??_7PredicateMask@operators@@6B@ 0052f1c0     gapidraw:GapiDraw.obj
 0002:000251c4       ??_7SourceColorfill@operators@@6B@ 0052f1c4     gapidraw:GapiDraw.obj
 0002:000251c8       ??_7SourcePixel@operators@@6B@ 0052f1c8     gapidraw:GapiDraw.obj
 0002:000251cc       ??_7CGapiDisplay555@@6B@   0052f1cc     gapidraw:GapiDraw.obj
 0002:000251d0       ??_7?$CGapiSurfaceAdapter@VCGapiDisplay565@@@@6B@ 0052f1d0     gapidraw:GapiDraw.obj
 0002:000251d4       ??_7?$PixelAlphaBlendFast32@VCGapiDisplay565@@@operators@@6B@ 0052f1d4     gapidraw:GapiDraw.obj
 0002:000251d8       ??_7?$PixelAlphaBlendFast@VCGapiDisplay565@@@operators@@6B@ 0052f1d8     gapidraw:GapiDraw.obj
 0002:000251dc       ??_7?$PixelAlphaBlend32@VCGapiDisplay565@@@operators@@6B@ 0052f1dc     gapidraw:GapiDraw.obj
 0002:000251e0       ??_7?$PixelAlphaBlend@VCGapiDisplay565@@@operators@@6B@ 0052f1e0     gapidraw:GapiDraw.obj
 0002:000251e4       ??_7CGapiDisplay565@@6B@   0052f1e4     gapidraw:GapiDraw.obj
 0002:000251e8       ??_7CGapiDisplay@@6B@      0052f1e8     gapidraw:GapiDisplayDDraw.obj
 0002:000251fc       _png_libpng_ver            0052f1fc     gapidraw:png.obj
 0002:00025210       _png_sig                   0052f210     gapidraw:png.obj
 0002:00025218       _png_IHDR                  0052f218     gapidraw:png.obj
 0002:00025220       _png_IDAT                  0052f220     gapidraw:png.obj
 0002:00025228       _png_IEND                  0052f228     gapidraw:png.obj
 0002:00025230       _png_PLTE                  0052f230     gapidraw:png.obj
 0002:00025238       _png_bKGD                  0052f238     gapidraw:png.obj
 0002:00025240       _png_cHRM                  0052f240     gapidraw:png.obj
 0002:00025248       _png_gAMA                  0052f248     gapidraw:png.obj
 0002:00025250       _png_hIST                  0052f250     gapidraw:png.obj
 0002:00025258       _png_iCCP                  0052f258     gapidraw:png.obj
 0002:00025260       _png_iTXt                  0052f260     gapidraw:png.obj
 0002:00025268       _png_oFFs                  0052f268     gapidraw:png.obj
 0002:00025270       _png_pCAL                  0052f270     gapidraw:png.obj
 0002:00025278       _png_sCAL                  0052f278     gapidraw:png.obj
 0002:00025280       _png_pHYs                  0052f280     gapidraw:png.obj
 0002:00025288       _png_sBIT                  0052f288     gapidraw:png.obj
 0002:00025290       _png_sPLT                  0052f290     gapidraw:png.obj
 0002:00025298       _png_sRGB                  0052f298     gapidraw:png.obj
 0002:000252a0       _png_tEXt                  0052f2a0     gapidraw:png.obj
 0002:000252a8       _png_tIME                  0052f2a8     gapidraw:png.obj
 0002:000252b0       _png_tRNS                  0052f2b0     gapidraw:png.obj
 0002:000252b8       _png_zTXt                  0052f2b8     gapidraw:png.obj
 0002:000252c0       _png_pass_start            0052f2c0     gapidraw:png.obj
 0002:000252dc       _png_pass_inc              0052f2dc     gapidraw:png.obj
 0002:000252f8       _png_pass_ystart           0052f2f8     gapidraw:png.obj
 0002:00025314       _png_pass_yinc             0052f314     gapidraw:png.obj
 0002:00025330       _png_pass_mask             0052f330     gapidraw:png.obj
 0002:0002534c       _png_pass_dsp_mask         0052f34c     gapidraw:png.obj
 0002:00025398       __real@8@3ffaccccccccccccd000 0052f398     gapidraw:pngrtran.obj
 0002:000253a0       __real@8@3fff8000000000000000 0052f3a0     gapidraw:pngrtran.obj
 0002:000253a8       __real@8@3ffe8000000000000000 0052f3a8     gapidraw:pngrtran.obj
 0002:000253b0       __real@8@400fc350000000000000 0052f3b0     gapidraw:pngrtran.obj
 0002:000253b8       __real@8@4006ff00000000000000 0052f3b8     gapidraw:pngrtran.obj
 0002:000253c0       __real@8@3ff78080808080808000 0052f3c0     gapidraw:pngrtran.obj
 0002:000253c8       __real@8@400effff000000000000 0052f3c8     gapidraw:pngrtran.obj
 0002:000253d0       __real@8@3fef8000800080008000 0052f3d0     gapidraw:pngrtran.obj
 0002:000253d8       __real@8@3ff78000000000000000 0052f3d8     gapidraw:pngrtran.obj
 0002:000253e0       __real@8@3feb8637bd05af6c6800 0052f3e0     gapidraw:pngrtran.obj
 0002:000253e8       ??_7CDisplay@@6B@          0052f3e8     gapidraw:ddutil.obj
 0002:000253ec       ??_7CGapiBitmapFont@@6B@   0052f3ec     gapidraw:GapiBitmapFont.obj
 0002:000253f0       __real@8@40028000000000000000 0052f3f0     gapidraw:pngwrite.obj
 0002:000253f8       __real@8@400da7c5a8f5c28f6000 0052f3f8     gapidraw:pngset.obj
 0002:00025400       __real@8@3feea7c5ac471b478800 0052f400     gapidraw:pngset.obj
 0002:00025408       __real@8@401dfffffffe00000000 0052f408     gapidraw:pngset.obj
 0002:00025814       __real@4@3feea7c5ac471b478800 0052f814     gapidraw:pngrutil.obj
 0002:00025818       _IID_IDirectDraw7          0052f818     gapidraw:dxguid.obj
 0002:00025828       __real@8@3ffeccccccccccccd000 0052f828     gapidraw:pngwutil.obj
 0002:00025830       _deflate_copyright         0052f830     gapidraw:deflate.obj
 0002:00025f70       __dist_code                0052ff70     gapidraw:trees.obj
 0002:00026170       __length_code              00530170     gapidraw:trees.obj
 0002:0002635c       _inflate_copyright         0053035c     gapidraw:inftrees.obj
 0002:00026574       _IID_IViewObject           00530574     uuid:oleidl_i.obj
 0002:00026584       _IID_IOleObject            00530584     uuid:oleidl_i.obj
 0002:00026594       _IID_IClassFactory         00530594     uuid:unknwn_i.obj
 0002:000265a4       _GUID_NULL                 005305a4     uuid:cguid_i.obj
 0002:000265b4       _IID_IPicture              005305b4     uuid:ocidl_i.obj
 0002:000265c4       ??_C@_0P@MIGLKIOC@CorExitProcess?$AA@ 005305c4     LIBC:crt0dat.obj
 0002:000265d4       ??_C@_0M@MBOPBNBK@mscoree?4dll?$AA@ 005305d4     LIBC:crt0dat.obj
 0002:00026600       ??_7type_info@@6B@         00530600     LIBC:typinfo.obj
 0002:000266b4       ??_C@_05KLBDPFGC@e?$CL000?$AA@ 005306b4     LIBC:cvt.obj
 0002:000266c0       __real@3ff0000000000000    005306c0     LIBC:testfdiv.obj
 0002:000266c8       __real@4150017ec0000000    005306c8     LIBC:testfdiv.obj
 0002:000266d0       __real@4147ffff80000000    005306d0     LIBC:testfdiv.obj
 0002:000266d8       ??_C@_0BK@NHEOCAHP@IsProcessorFeaturePresent?$AA@ 005306d8     LIBC:testfdiv.obj
 0002:000266f4       ??_C@_08CPNIBGIE@KERNEL32?$AA@ 005306f4     LIBC:testfdiv.obj
 0002:00026700       ___lookuptable             00530700     LIBC:output.obj
 0002:0002675c       ??_C@_1O@CEDCILHN@?$AA?$CI?$AAn?$AAu?$AAl?$AAl?$AA?$CJ?$AA?$AA@ 0053075c     LIBC:output.obj
 0002:0002676c       ??_C@_06OJHGLDPL@?$CInull?$CJ?$AA@ 0053076c     LIBC:output.obj
 0002:00026794       ??_C@_13NOLLCAOD@?$AA?$AA?$AA?$AA@ 00530794     LIBC:a_map.obj
 0002:000267c0       ___newctype                005307c0     LIBC:ctype.obj
 0002:00026ac0       __wctype                   00530ac0     LIBC:ctype.obj
 0002:00026cc4       ___dnames                  00530cc4     LIBC:timeset.obj
 0002:00026cdc       ___mnames                  00530cdc     LIBC:timeset.obj
 0002:00026d04       ??_C@_02CLFPBFFP@TZ?$AA@   00530d04     LIBC:tzset.obj
 0002:00026d18       __DEFAULT_CW_in_mem        00530d18     LIBC:common.obj
 0002:00026d1a       __pi_by_2_to_61            00530d1a     LIBC:common.obj
 0002:00026da0       ??_C@_0P@GGKDKEEG@runtime?5error?5?$AA@ 00530da0     LIBC:crt0msg.obj
 0002:00026db0       ??_C@_02PCIJFNDE@?$AN?6?$AA@ 00530db0     LIBC:crt0msg.obj
 0002:00026db4       ??_C@_0O@MJNIPGOH@TLOSS?5error?$AN?6?$AA@ 00530db4     LIBC:crt0msg.obj
 0002:00026dc4       ??_C@_0N@BONNPDHF@SING?5error?$AN?6?$AA@ 00530dc4     LIBC:crt0msg.obj
 0002:00026dd4       ??_C@_0P@MBDAJNE@DOMAIN?5error?$AN?6?$AA@ 00530dd4     LIBC:crt0msg.obj
 0002:00026de8       ??_C@_0KC@BDDGGBEJ@R6029?$AN?6?9?5This?5application?5cannot@ 00530de8     LIBC:crt0msg.obj
 0002:00026e8c       ??_C@_0CF@KJDAIALP@R6028?$AN?6?9?5unable?5to?5initialize?5he@ 00530e8c     LIBC:crt0msg.obj
 0002:00026eb4       ??_C@_0DF@GAKBPDFP@R6027?$AN?6?9?5not?5enough?5space?5for?5lo@ 00530eb4     LIBC:crt0msg.obj
 0002:00026eec       ??_C@_0DF@IBLNNAIG@R6026?$AN?6?9?5not?5enough?5space?5for?5st@ 00530eec     LIBC:crt0msg.obj
 0002:00026f24       ??_C@_0CG@IOHKGFNJ@R6025?$AN?6?9?5pure?5virtual?5function?5c@ 00530f24     LIBC:crt0msg.obj
 0002:00026f4c       ??_C@_0DF@JIJJFJDC@R6024?$AN?6?9?5not?5enough?5space?5for?5_o@ 00530f4c     LIBC:crt0msg.obj
 0002:00026f84       ??_C@_0CJ@EGEJHFME@R6019?$AN?6?9?5unable?5to?5open?5console?5@ 00530f84     LIBC:crt0msg.obj
 0002:00026fb0       ??_C@_0CB@GNHNIELH@R6018?$AN?6?9?5unexpected?5heap?5error?$AN?6@ 00530fb0     LIBC:crt0msg.obj
 0002:00026fd4       ??_C@_0CN@FOLDKNG@R6017?$AN?6?9?5unexpected?5multithread?5@ 00530fd4     LIBC:crt0msg.obj
 0002:00027004       ??_C@_0CM@FAHFJNHO@R6016?$AN?6?9?5not?5enough?5space?5for?5th@ 00531004     LIBC:crt0msg.obj
 0002:00027030       ??_C@_0JG@LBKMGKLD@?$AN?6This?5application?5has?5requested@ 00531030     LIBC:crt0msg.obj
 0002:000270c8       ??_C@_0CM@FLCNIPKK@R6009?$AN?6?9?5not?5enough?5space?5for?5en@ 005310c8     LIBC:crt0msg.obj
 0002:000270f4       ??_C@_0CK@KMMJOAPP@R6008?$AN?6?9?5not?5enough?5space?5for?5ar@ 005310f4     LIBC:crt0msg.obj
 0002:00027120       ??_C@_0CF@HOHMHDEK@R6002?$AN?6?9?5floating?5point?5not?5load@ 00531120     LIBC:crt0msg.obj
 0002:00027148       ??_C@_0CF@GOGNBNAK@Microsoft?5Visual?5C?$CL?$CL?5Runtime?5Lib@ 00531148     LIBC:crt0msg.obj
 0002:00027170       ??_C@_02PHMGELLB@?6?6?$AA@ 00531170     LIBC:crt0msg.obj
 0002:00027174       ??_C@_0BK@OFGJDLJJ@Runtime?5Error?$CB?6?6Program?3?5?$AA@ 00531174     LIBC:crt0msg.obj
 0002:00027190       ??_C@_03KHICJKCI@?4?4?4?$AA@ 00531190     LIBC:crt0msg.obj
 0002:00027194       ??_C@_0BH@DNAGHKFM@?$DMprogram?5name?5unknown?$DO?$AA@ 00531194     LIBC:crt0msg.obj
 0002:000271cc       ??_C@_0N@FFJGBINN@AuthenticAMD?$AA@ 005311cc     LIBC:cpu_disp.obj
 0002:0002ab10       __real@4000000000000000    00534b10     LIBC:powhlp.obj
 0002:0002ab34       ??_C@_09KLGCKDOD@Program?3?5?$AA@ 00534b34     LIBC:secfail.obj
 0002:0002ab40       ??_C@_0KA@JEHFIFGP@A?5buffer?5overrun?5has?5been?5detect@ 00534b40     LIBC:secfail.obj
 0002:0002abe0       ??_C@_0BJ@MDEKIEOJ@Buffer?5overrun?5detected?$CB?$AA@ 00534be0     LIBC:secfail.obj
 0002:0002ac00       ??_C@_0LB@BPLHHLFD@A?5security?5error?5of?5unknown?5caus@ 00534c00     LIBC:secfail.obj
 0002:0002acb4       ??_C@_0CD@GMKACBEK@Unknown?5security?5failure?5detecte@ 00534cb4     LIBC:secfail.obj
 0002:0002ace4       ??_C@_0BI@DFKBFLJE@GetProcessWindowStation?$AA@ 00534ce4     LIBC:crtmbox.obj
 0002:0002acfc       ??_C@_0BK@CIDNPOGP@GetUserObjectInformationA?$AA@ 00534cfc     LIBC:crtmbox.obj
 0002:0002ad18       ??_C@_0BD@HHGDFDBJ@GetLastActivePopup?$AA@ 00534d18     LIBC:crtmbox.obj
 0002:0002ad2c       ??_C@_0BA@HNOPNCHB@GetActiveWindow?$AA@ 00534d2c     LIBC:crtmbox.obj
 0002:0002ad3c       ??_C@_0M@CHKKJDAI@MessageBoxA?$AA@ 00534d3c     LIBC:crtmbox.obj
 0002:0002ad48       ??_C@_0L@GMPLCCII@user32?4dll?$AA@ 00534d48     LIBC:crtmbox.obj
 0002:0002adc0       ??_C@_04MLLJIGOK@atan?$AA@ 00534dc0     LIBC:libm_error.obj
 0002:0002adc8       ??_C@_04GFPJNGEK@ceil?$AA@ 00534dc8     LIBC:libm_error.obj
 0002:0002add0       ??_C@_05PBJFFIGL@floor?$AA@ 00534dd0     LIBC:libm_error.obj
 0002:0002add8       ??_C@_04EHEDPDJG@modf?$AA@ 00534dd8     LIBC:libm_error.obj
 0002:0002ade0       ??_C@_04HPAFEEIN@exp2?$AA@ 00534de0     LIBC:libm_error.obj
 0002:0002ade8       ??_C@_05EOHGHCHD@exp10?$AA@ 00534de8     LIBC:libm_error.obj
 0002:0002adf0       ??_C@_04KGLCPMCP@log2?$AA@ 00534df0     LIBC:libm_error.obj
 0002:0002adf8       ??_C@_03JGHBODFD@pow?$AA@  00534df8     LIBC:libm_error.obj
 0002:0002adfc       ??_C@_03MGHMBJCF@log?$AA@  00534dfc     LIBC:libm_error.obj
 0002:0002ae00       ??_C@_05HGHHAHAP@log10?$AA@ 00534e00     LIBC:libm_error.obj
 0002:0002ae08       ??_C@_03KHJOGHMM@exp?$AA@  00534e08     LIBC:libm_error.obj
 0002:0002ae0c       ??_C@_06IMKFLFPG@1?$CDQNAN?$AA@ 00534e0c     LIBC:x10fout.obj
 0002:0002ae14       ??_C@_05DNEBIAHO@1?$CDINF?$AA@ 00534e14     LIBC:x10fout.obj
 0002:0002ae1c       ??_C@_05PHHOCPM@1?$CDIND?$AA@ 00534e1c     LIBC:x10fout.obj
 0002:0002ae24       ??_C@_06PGGFOGJG@1?$CDSNAN?$AA@ 00534e24     LIBC:x10fout.obj
 0002:0002ae2c       ??_C@_0L@KDOEJCKC@_nextafter?$AA@ 00534e2c     LIBC:fpexcept.obj
 0002:0002ae38       ??_C@_05JGDBENOH@_logb?$AA@ 00534e38     LIBC:fpexcept.obj
 0002:0002ae40       ??_C@_03ONILCKOB@_yn?$AA@  00534e40     LIBC:fpexcept.obj
 0002:0002ae44       ??_C@_03NAKIGLHK@_y1?$AA@  00534e44     LIBC:fpexcept.obj
 0002:0002ae48       ??_C@_03MJLDFKDL@_y0?$AA@  00534e48     LIBC:fpexcept.obj
 0002:0002ae4c       ??_C@_05GKKHEGJL@frexp?$AA@ 00534e4c     LIBC:fpexcept.obj
 0002:0002ae54       ??_C@_04KEPJIHGP@fmod?$AA@ 00534e54     LIBC:fpexcept.obj
 0002:0002ae5c       ??_C@_06MEIMCGCF@_hypot?$AA@ 00534e5c     LIBC:fpexcept.obj
 0002:0002ae64       ??_C@_05KBKMEMPO@_cabs?$AA@ 00534e64     LIBC:fpexcept.obj
 0002:0002ae6c       ??_C@_05CEJMAHNP@ldexp?$AA@ 00534e6c     LIBC:fpexcept.obj
 0002:0002ae74       ??_C@_04ODHECPBC@fabs?$AA@ 00534e74     LIBC:fpexcept.obj
 0002:0002ae7c       ??_C@_03IIINPABG@tan?$AA@  00534e7c     LIBC:fpexcept.obj
 0002:0002ae80       ??_C@_03LALBNOCG@cos?$AA@  00534e80     LIBC:fpexcept.obj
 0002:0002ae84       ??_C@_03BLEJJJBH@sin?$AA@  00534e84     LIBC:fpexcept.obj
 0002:0002ae88       ??_C@_04EIAKFFMI@sqrt?$AA@ 00534e88     LIBC:fpexcept.obj
 0002:0002ae90       ??_C@_05KNGEOGJB@atan2?$AA@ 00534e90     LIBC:fpexcept.obj
 0002:0002ae98       ??_C@_04PDIFKINK@acos?$AA@ 00534e98     LIBC:fpexcept.obj
 0002:0002aea0       ??_C@_04FIHNOPOL@asin?$AA@ 00534ea0     LIBC:fpexcept.obj
 0002:0002aea8       ??_C@_04FJHINJAO@tanh?$AA@ 00534ea8     LIBC:fpexcept.obj
 0002:0002aeb0       ??_C@_04HPJJNFIM@cosh?$AA@ 00534eb0     LIBC:fpexcept.obj
 0002:0002aeb8       ??_C@_04COOMCNPB@sinh?$AA@ 00534eb8     LIBC:fpexcept.obj
 0002:0002aed8       _GUID_ATLVer30             00534ed8     atls:atlbase.obj
 0002:0002aee8       _GUID_ATLVer70             00534ee8     atls:atlbase.obj
 0002:0002aef8       ??_R1A@?0A@A@type_info@@8  00534ef8     LIBC:typinfo.obj
 0002:0002af10       ??_R2type_info@@8          00534f10     LIBC:typinfo.obj
 0002:0002af18       ??_R3type_info@@8          00534f18     LIBC:typinfo.obj
 0002:0002af28       ??_R4type_info@@6B@        00534f28     LIBC:typinfo.obj
 0002:0002af3c       ___rtc_iaa                 00534f3c     LIBC:initsect.obj
 0002:0002af40       ___rtc_izz                 00534f40     LIBC:initsect.obj
 0002:0002af44       ___rtc_taa                 00534f44     LIBC:initsect.obj
 0002:0002af48       ___rtc_tzz                 00534f48     LIBC:initsect.obj
 0002:0002d050       __CT??_R0?AVCAtlException@ATL@@@84 00537050     FlashPlayer.obj
 0002:0002d06c       __CTA1?AVCAtlException@ATL@@ 0053706c     FlashPlayer.obj
 0002:0002d074       __TI1?AVCAtlException@ATL@@ 00537074     FlashPlayer.obj
 0002:0002df88       __IMPORT_DESCRIPTOR_fmod   00537f88     fmodvc:fmod.dll
 0002:0002df9c       __IMPORT_DESCRIPTOR_WINMM  00537f9c     gapidraw:WINMM.dll
 0002:0002dfb0       __IMPORT_DESCRIPTOR_DDRAW  00537fb0     gapidraw:DDRAW.dll
 0002:0002dfc4       __IMPORT_DESCRIPTOR_KERNEL32 00537fc4     kernel32:KERNEL32.dll
 0002:0002dfd8       __IMPORT_DESCRIPTOR_USER32 00537fd8     user32:USER32.dll
 0002:0002dfec       __IMPORT_DESCRIPTOR_GDI32  00537fec     gdi32:GDI32.dll
 0002:0002e000       __IMPORT_DESCRIPTOR_ADVAPI32 00538000     advapi32:ADVAPI32.dll
 0002:0002e014       __IMPORT_DESCRIPTOR_SHELL32 00538014     shell32:SHELL32.dll
 0002:0002e028       __IMPORT_DESCRIPTOR_ole32  00538028     ole32:ole32.dll
 0002:0002e03c       __IMPORT_DESCRIPTOR_OLEAUT32 0053803c     oleaut32:OLEAUT32.dll
 0002:0002e050       __IMPORT_DESCRIPTOR_WININET 00538050     wininet:WININET.dll
 0002:0002e064       __NULL_IMPORT_DESCRIPTOR   00538064     fmodvc:fmod.dll
 0003:00000000       ___xc_a                    0053a000     LIBC:crt0init.obj
 0003:000022e0       ___xc_z                    0053c2e0     LIBC:crt0init.obj
 0003:000022e4       ___xi_a                    0053c2e4     LIBC:crt0init.obj
 0003:000022fc       ___xi_z                    0053c2fc     LIBC:crt0init.obj
 0003:00002300       ___xp_a                    0053c300     LIBC:crt0init.obj
 0003:00002308       ___xp_z                    0053c308     LIBC:crt0init.obj
 0003:0000230c       ___xt_a                    0053c30c     LIBC:crt0init.obj
 0003:00002314       ___xt_z                    0053c314     LIBC:crt0init.obj
 0003:0000235c       ?m_eDetailHeadDirection@CVillager@@0W4EDirection@@A 0053c35c     Villager.obj
 0003:00002380       ?sm_sCollectable@CCollectionScene@@0PAUSCollectable@1@A 0053c380     CollectionScene.obj
 0003:000025e0       ?sm_sTech@CTechScene@@0PAUSTech@1@A 0053c5e0     TechScene.obj
 0003:00003004       ?m_sSoundTrackFile@CSoundTrack@@0PAPADA 0053d004     SoundTrack.obj
 0003:00005040       ?sm_iDifficultyLevel@CPotion@@0PAHA 0053f040     Potion.obj
 0003:000050e8       ?sm_sTechPrice@CTech@@0PAUSTechPrice@1@A 0053f0e8     Tech.obj
 0003:00005158       ?m_sAnim@CFloatingAnim@@0PAUSAnim@1@A 0053f158     FloatingAnim.obj
 0003:00005ce0       ?ImageList@@3PAUImageDescriptor@@A 0053fce0     theGraphicsManager.obj
 0003:0000ca88       ?sm_pPuzzle@CPuzzle@@0PAPAVIPuzzle@@A 00546a88     Puzzle.obj
 0003:0000cb10       ?rcDefault@CWindow@ATL@@2UtagRECT@@A 00546b10     FlashPlayer.obj
 0003:0000cb20       ?g_pfnGetThreadACP@ATL@@3P6GIXZA 00546b20     FlashPlayer.obj
 0003:0000cb24       ??_R0?AVCAtlException@ATL@@@8 00546b24     FlashPlayer.obj
 0003:0000cb44       ?_tih@?$IDispatchImpl@UIAxWinAmbientDispatchEx@@$1?_GUID_b2d0778b_ac99_4c58_a5c8_e7724e5316b5@@3U__s_GUID@@B$1?m_libid@CAtlModule@ATL@@2U_GUID@@A$0PPPP@$0PPPP@VCComTypeInfoHolder@ATL@@@ATL@@1VCComTypeInfoHolder@2@A 00546b44     FlashPlayer.obj
 0003:0000cb60       ?wc@?1??GetWndClassInfo@?$CWindowImpl@VCAxFrameWindow@ATL@@VCWindow@2@V?$CWinTraits@$0FGAAAAAA@$0A@@2@@ATL@@SAAAU_ATL_WNDCLASSINFOA@3@XZ@4U43@A 00546b60     FlashPlayer.obj
 0003:0000cbc8       ?wc@?1??GetWndClassInfo@?$CWindowImpl@VCAxUIWindow@ATL@@VCWindow@2@V?$CWinTraits@$0FGAAAAAA@$0A@@2@@ATL@@SAAAU_ATL_WNDCLASSINFOA@3@XZ@4U43@A 00546bc8     FlashPlayer.obj
 0003:0000cc3c       ??_C@_0L@BGJF@Read?5Error?$AA@ 00546c3c     gapidraw:GapiRGBASurface.obj
 0003:0000cc48       ??_C@_05CNKG@1?42?43?$AA@  00546c48     gapidraw:GapiRGBASurface.obj
 0003:0000cc50       ??_C@_02NGAF@wb?$AA@       00546c50     gapidraw:GapiSurface.obj
 0003:0000cc54       ??_C@_0M@KPPG@Write?5Error?$AA@ 00546c54     gapidraw:GapiSurface.obj
 0003:0000cc60       ??_C@_0GA@DIIM@Failed?5initializing?5DirectDraw?4?5@ 00546c60     gapidraw:GapiDisplayDDraw.obj
 0003:0000ccc0       ??_C@_0CA@IMNI@Failed?5initializing?5DirectDraw?4?$AA@ 00546cc0     gapidraw:GapiDisplayDDraw.obj
 0003:0000cce0       ??_C@_0CC@JKIJ@Could?5not?5initialize?5main?5window@ 00546ce0     gapidraw:GapiDisplayDDraw.obj
 0003:0000cd04       ??_C@_08GBMG@GapiDraw?$AA@ 00546d04     gapidraw:GapiDisplayDDraw.obj
 0003:0000cd10       ??_C@_0DH@HGNP@This?5display?5card?5does?5not?5suppo@ 00546d10     gapidraw:GapiDisplayDDraw.obj
 0003:0000cd48       ??_C@_0BC@FHOF@libpng?5error?3?5?$CFs?6?$AA@ 00546d48     gapidraw:pngerror.obj
 0003:0000cd5c       ??_C@_0BN@DKH@libpng?5error?3?5?$CFs?0?5offset?$DN?$CFd?6?$AA@ 00546d5c     gapidraw:pngerror.obj
 0003:0000cd7c       ??_C@_0BJ@NKNN@libpng?5error?5no?4?5?$CFs?3?5?$CFs?6?$AA@ 00546d7c     gapidraw:pngerror.obj
 0003:0000cd98       ??_C@_0BE@NAGM@libpng?5warning?3?5?$CFs?6?$AA@ 00546d98     gapidraw:pngerror.obj
 0003:0000cdac       ??_C@_0BL@LHKO@libpng?5warning?5no?4?5?$CFs?3?5?$CFs?6?$AA@ 00546dac     gapidraw:pngerror.obj
 0003:0000cdc8       ??_C@_0BD@OLIJ@Unknown?5zlib?5error?$AA@ 00546dc8     gapidraw:pngread.obj
 0003:0000cddc       ??_C@_0BD@ECPC@zlib?5version?5error?$AA@ 00546ddc     gapidraw:pngread.obj
 0003:0000cdf0       ??_C@_0BC@NMAB@zlib?5memory?5error?$AA@ 00546df0     gapidraw:pngread.obj
 0003:0000ce04       ??_C@_05IOHI@1?41?44?$AA@  00546e04     gapidraw:pngread.obj
 0003:0000ce0c       ??_C@_0DH@ELIJ@Incompatible?5libpng?5version?5in?5a@ 00546e0c     gapidraw:pngread.obj
 0003:0000ce44       ??_C@_0DG@IFOL@Application?5?5is?5?5running?5with?5pn@ 00546e44     gapidraw:pngread.obj
 0003:0000ce7c       ??_C@_0DG@EBPO@Application?5was?5compiled?5with?5pn@ 00546e7c     gapidraw:pngread.obj
 0003:0000ceb4       ??_C@_0BJ@MIGL@Missing?5PLTE?5before?5IDAT?$AA@ 00546eb4     gapidraw:pngread.obj
 0003:0000ced0       ??_C@_0BJ@FENO@Missing?5IHDR?5before?5IDAT?$AA@ 00546ed0     gapidraw:pngread.obj
 0003:0000ceec       ??_C@_0BG@BPPM@Invalid?5chunk?5length?4?$AA@ 00546eec     gapidraw:pngread.obj
 0003:0000cf04       ??_C@_0CH@BGD@PNG?5file?5corrupted?5by?5ASCII?5conv@ 00546f04     gapidraw:pngread.obj
 0003:0000cf2c       ??_C@_0P@NFKI@Not?5a?5PNG?5file?$AA@ 00546f2c     gapidraw:pngread.obj
 0003:0000cf3c       ??_C@_0EH@IFBC@Ignoring?5extra?5png_read_update_i@ 00546f3c     gapidraw:pngread.obj
 0003:0000cf84       ??_C@_0BG@KFHH@Extra?5compressed?5data?$AA@ 00546f84     gapidraw:pngread.obj
 0003:0000cf9c       ??_C@_0BE@OJIF@Decompression?5error?$AA@ 00546f9c     gapidraw:pngread.obj
 0003:0000cfb0       ??_C@_0BG@DOBA@Not?5enough?5image?5data?$AA@ 00546fb0     gapidraw:pngread.obj
 0003:0000cfc8       ??_C@_0CB@JOHD@Invalid?5attempt?5to?5read?5row?5data@ 00546fc8     gapidraw:pngread.obj
 0003:0000d30c       ??_C@_0CC@KNMH@png_do_dither?5returned?5rowbytes?$DN@ 0054730c     gapidraw:pngrtran.obj
 0003:0000d330       ??_C@_0CH@KGHA@png_do_rgb_to_gray?5found?5nongray@ 00547330     gapidraw:pngrtran.obj
 0003:0000d358       ??_C@_0CF@MPLO@NULL?5row?5buffer?5for?5row?5?$CFld?0?5pas@ 00547358     gapidraw:pngrtran.obj
 0003:0000d380       ??_C@_0DC@JCPM@Width?5too?5large?5for?5libpng?5to?5pr@ 00547380     gapidraw:pngget.obj
 0003:0000d3b4       ??_C@_0BF@LOBB@Invalid?5image?5height?$AA@ 005473b4     gapidraw:pngget.obj
 0003:0000d3cc       ??_C@_0BE@BKGJ@Invalid?5image?5width?$AA@ 005473cc     gapidraw:pngget.obj
 0003:0000d3e0       ??_C@_0BD@IGKH@Invalid?5color?5type?$AA@ 005473e0     gapidraw:pngget.obj
 0003:0000d3f4       ??_C@_0BC@OEEB@Invalid?5bit?5depth?$AA@ 005473f4     gapidraw:pngget.obj
 0003:0000d408       ??_C@_0BL@KBLO@Call?5to?5NULL?5read?5function?$AA@ 00547408     gapidraw:pngrio.obj
 0003:0000d424       ??_C@_0DC@OFCG@same?5structure?4?5?5Resetting?5write@ 00547424     gapidraw:pngrio.obj
 0003:0000d458       ??_C@_0EB@EPNC@It?8s?5an?5error?5to?5set?5both?5read_d@ 00547458     gapidraw:pngrio.obj
 0003:0000d49c       ??_C@_0GB@FFKO@?5?$CB?$CC?$CD$?$CF?$CG?8?$CI?$CJ?$CK?$CL?0?9?4?10123456789?3?$DL?$DM?$DN?$DO?$DP@ 0054749c     gapidraw:GapiBitmapFont.obj
 0003:0000d500       ??_C@_0DC@PLKM@MNG?5features?5are?5not?5allowed?5in?5@ 00547500     gapidraw:pngwrite.obj
 0003:0000d534       ??_C@_0CE@PPL@Unable?5to?5write?5international?5te@ 00547534     gapidraw:pngwrite.obj
 0003:0000d558       ??_C@_0CM@EFKO@Valid?5palette?5required?5for?5palet@ 00547558     gapidraw:pngwrite.obj
 0003:0000d584       ??_C@_0BL@FGAG@No?5IDATs?5written?5into?5file?$AA@ 00547584     gapidraw:pngwrite.obj
 0003:0000d5a0       ??_C@_0DG@OOAH@png_write_info?5was?5never?5called?5@ 005475a0     gapidraw:pngwrite.obj
 0003:0000d5d8       ??_C@_0L@OCGE@zlib?5error?$AA@ 005475d8     gapidraw:pngwrite.obj
 0003:0000d5e4       ??_C@_0CA@FLOC@Unknown?5filter?5heuristic?5method?$AA@ 005475e4     gapidraw:pngwrite.obj
 0003:0000d604       ??_C@_0DE@LFLJ@Ignoring?5attempt?5to?5set?5negative@ 00547604     gapidraw:pngset.obj
 0003:0000d638       ??_C@_0DO@FCJI@Ignoring?5attempt?5to?5set?5chromati@ 00547638     gapidraw:pngset.obj
 0003:0000d678       ??_C@_0BA@GNLC@Setting?5gamma?$DN0?$AA@ 00547678     gapidraw:pngset.obj
 0003:0000d688       ??_C@_0BL@CMAA@Limiting?5gamma?5to?521474?483?$AA@ 00547688     gapidraw:pngset.obj
 0003:0000d6a4       ??_C@_0BP@DPOP@Setting?5negative?5gamma?5to?5zero?$AA@ 005476a4     gapidraw:pngset.obj
 0003:0000d6c4       ??_C@_0CJ@CIB@Palette?5size?50?0?5hIST?5allocation?5@ 005476c4     gapidraw:pngset.obj
 0003:0000d6f0       ??_C@_0DP@POIO@Width?5too?5large?5to?5process?5image@ 005476f0     gapidraw:pngset.obj
 0003:0000d730       ??_C@_0BO@CIHE@Invalid?5filter?5method?5in?5IHDR?$AA@ 00547730     gapidraw:pngset.obj
 0003:0000d750       ??_C@_0BO@DEOD@Unknown?5filter?5method?5in?5IHDR?$AA@ 00547750     gapidraw:pngset.obj
 0003:0000d770       ??_C@_0CD@IFNF@Unknown?5compression?5method?5in?5IH@ 00547770     gapidraw:pngset.obj
 0003:0000d794       ??_C@_0CB@IFMD@Unknown?5interlace?5method?5in?5IHDR@ 00547794     gapidraw:pngset.obj
 0003:0000d7b8       ??_C@_0DB@ODDM@Invalid?5color?5type?1bit?5depth?5com@ 005477b8     gapidraw:pngset.obj
 0003:0000d7ec       ??_C@_0BL@OGOG@Invalid?5color?5type?5in?5IHDR?$AA@ 005477ec     gapidraw:pngset.obj
 0003:0000d808       ??_C@_0BK@KFCG@Invalid?5bit?5depth?5in?5IHDR?$AA@ 00547808     gapidraw:pngset.obj
 0003:0000d824       ??_C@_0BL@JLGM@Invalid?5image?5size?5in?5IHDR?$AA@ 00547824     gapidraw:pngset.obj
 0003:0000d840       ??_C@_0CG@JJAH@Image?5width?5or?5height?5is?5zero?5in@ 00547840     gapidraw:pngset.obj
 0003:0000d868       ??_C@_0BJ@ENIB@Unable?5to?5malloc?5palette?$AA@ 00547868     gapidraw:pngset.obj
 0003:0000d884       ??_C@_0BK@GDCC@iTXt?5chunk?5not?5supported?4?$AA@ 00547884     gapidraw:pngset.obj
 0003:0000d8a0       ??_C@_0BM@FDOB@Call?5to?5NULL?5write?5function?$AA@ 005478a0     gapidraw:pngwio.obj
 0003:0000d8bc       ??_C@_0DF@GNBJ@the?5same?5structure?4?5?5Resetting?5r@ 005478bc     gapidraw:pngwio.obj
 0003:0000d8f4       ??_C@_0DI@NEHN@Attempted?5to?5set?5both?5read_data_@ 005478f4     gapidraw:pngwio.obj
 0003:0000d92c       ??_C@_0FM@POGE@?5?$CB?$CC?$CD$?$CF?$CG?8?$CI?$CJ?$CK?$CL?0?9?4?10123456789?3?$DL?$DM?$DN?$DO?$DP@ 0054792c     gapidraw:GapiDisplayCommon.obj
 0003:0000d988       ??_C@_0O@HJOL@Out?5of?5Memory?$AA@ 00547988     gapidraw:pngmem.obj
 0003:0000d998       ??_C@_0P@CCAO@Out?5of?5Memory?$CB?$AA@ 00547998     gapidraw:pngmem.obj
 0003:0000d9a8       ??_C@_0BA@FKCH@need?5dictionary?$AA@ 005479a8     gapidraw:inflate.obj
 0003:0000d9b8       ??_C@_0BF@OBFI@incorrect?5data?5check?$AA@ 005479b8     gapidraw:inflate.obj
 0003:0000d9d0       ??_C@_0BH@NLIB@incorrect?5header?5check?$AA@ 005479d0     gapidraw:inflate.obj
 0003:0000d9e8       ??_C@_0BE@FAJE@invalid?5window?5size?$AA@ 005479e8     gapidraw:inflate.obj
 0003:0000d9fc       ??_C@_0BL@KPEJ@unknown?5compression?5method?$AA@ 005479fc     gapidraw:inflate.obj
 0003:0000da38       ??_C@_09IBKM@CRC?5error?$AA@ 00547a38     gapidraw:pngrutil.obj
 0003:0000da44       ??_C@_0CB@FAAD@Unknown?5zTXt?5compression?5type?5?$CFd@ 00547a44     gapidraw:pngrutil.obj
 0003:0000da68       ??_C@_0CN@GICF@Incomplete?5compressed?5datastream@ 00547a68     gapidraw:pngrutil.obj
 0003:0000da98       ??_C@_0DA@DHKF@Data?5error?5in?5compressed?5datastr@ 00547a98     gapidraw:pngrutil.obj
 0003:0000dac8       ??_C@_0DC@OOKL@Buffer?5error?5in?5compressed?5datas@ 00547ac8     gapidraw:pngrutil.obj
 0003:0000dafc       ??_C@_0BD@EHAN@Invalid?5IHDR?5chunk?$AA@ 00547afc     gapidraw:pngrutil.obj
 0003:0000db10       ??_C@_0BC@HKAL@Out?5of?5place?5IHDR?$AA@ 00547b10     gapidraw:pngrutil.obj
 0003:0000db24       ??_C@_0CM@EPPF@Truncating?5incorrect?5info?5tRNS?5c@ 00547b24     gapidraw:pngrutil.obj
 0003:0000db50       ??_C@_0CH@DPCK@Truncating?5incorrect?5tRNS?5chunk?5@ 00547b50     gapidraw:pngrutil.obj
 0003:0000db78       ??_C@_0BG@FAPJ@Invalid?5palette?5chunk?$AA@ 00547b78     gapidraw:pngrutil.obj
 0003:0000db90       ??_C@_0CF@JNML@Ignoring?5PLTE?5chunk?5in?5grayscale@ 00547b90     gapidraw:pngrutil.obj
 0003:0000dbb8       ??_C@_0BF@LHNN@Duplicate?5PLTE?5chunk?$AA@ 00547bb8     gapidraw:pngrutil.obj
 0003:0000dbd0       ??_C@_0BI@ENAH@Invalid?5PLTE?5after?5IDAT?$AA@ 00547bd0     gapidraw:pngrutil.obj
 0003:0000dbe8       ??_C@_0BJ@LLMG@Missing?5IHDR?5before?5PLTE?$AA@ 00547be8     gapidraw:pngrutil.obj
 0003:0000dc04       ??_C@_0BM@MMMK@Incorrect?5IEND?5chunk?5length?$AA@ 00547c04     gapidraw:pngrutil.obj
 0003:0000dc20       ??_C@_0BB@GHB@No?5image?5in?5file?$AA@ 00547c20     gapidraw:pngrutil.obj
 0003:0000dc34       ??_C@_0BF@POGI@gamma?5?$DN?5?$CI?$CFd?1100000?$CJ?6?$AA@ 00547c34     gapidraw:pngrutil.obj
 0003:0000dc4c       ??_C@_0DI@MPAH@Ignoring?5incorrect?5gAMA?5value?5wh@ 00547c4c     gapidraw:pngrutil.obj
 0003:0000dc84       ??_C@_0CB@LLBB@Ignoring?5gAMA?5chunk?5with?5gamma?$DN0@ 00547c84     gapidraw:pngrutil.obj
 0003:0000dca8       ??_C@_0BF@PEDD@Duplicate?5gAMA?5chunk?$AA@ 00547ca8     gapidraw:pngrutil.obj
 0003:0000dcc0       ??_C@_0BI@PGJN@Out?5of?5place?5gAMA?5chunk?$AA@ 00547cc0     gapidraw:pngrutil.obj
 0003:0000dcd8       ??_C@_0BI@CGIA@Invalid?5gAMA?5after?5IDAT?$AA@ 00547cd8     gapidraw:pngrutil.obj
 0003:0000dcf0       ??_C@_0BM@DAMG@Incorrect?5gAMA?5chunk?5length?$AA@ 00547cf0     gapidraw:pngrutil.obj
 0003:0000dd0c       ??_C@_0BJ@FHOJ@Missing?5IHDR?5before?5gAMA?$AA@ 00547d0c     gapidraw:pngrutil.obj
 0003:0000dd28       ??_C@_0BM@OOJJ@Incorrect?5sBIT?5chunk?5length?$AA@ 00547d28     gapidraw:pngrutil.obj
 0003:0000dd44       ??_C@_0BF@CMOF@Duplicate?5sBIT?5chunk?$AA@ 00547d44     gapidraw:pngrutil.obj
 0003:0000dd5c       ??_C@_0BI@COEL@Out?5of?5place?5sBIT?5chunk?$AA@ 00547d5c     gapidraw:pngrutil.obj
 0003:0000dd74       ??_C@_0BI@KHKI@Invalid?5sBIT?5after?5IDAT?$AA@ 00547d74     gapidraw:pngrutil.obj
 0003:0000dd8c       ??_C@_0BJ@JCKK@Missing?5IHDR?5before?5sBIT?$AA@ 00547d8c     gapidraw:pngrutil.obj
 0003:0000dda8       ??_C@_0BJ@DMKC@Invalid?5cHRM?5white?5point?$AA@ 00547da8     gapidraw:pngrutil.obj
 0003:0000ddc4       ??_C@_0BH@LBIB@Invalid?5cHRM?5red?5point?$AA@ 00547dc4     gapidraw:pngrutil.obj
 0003:0000dddc       ??_C@_0BJ@NPFJ@Invalid?5cHRM?5green?5point?$AA@ 00547ddc     gapidraw:pngrutil.obj
 0003:0000ddf8       ??_C@_0BI@MPFH@Invalid?5cHRM?5blue?5point?$AA@ 00547df8     gapidraw:pngrutil.obj
 0003:0000de10       ??_C@_0BM@HBMJ@gx?$DN?$CFf?0?5gy?$DN?$CFf?0?5bx?$DN?$CFf?0?5by?$DN?$CFf?6?$AA@ 00547e10     gapidraw:pngrutil.obj
 0003:0000de2c       ??_C@_0BM@CJCB@wx?$DN?$CFf?0?5wy?$DN?$CFf?0?5rx?$DN?$CFf?0?5ry?$DN?$CFf?6?$AA@ 00547e2c     gapidraw:pngrutil.obj
 0003:0000de48       ??_C@_0DI@HOBM@Ignoring?5incorrect?5cHRM?5value?5wh@ 00547e48     gapidraw:pngrutil.obj
 0003:0000de80       ??_C@_0BF@OOJM@Duplicate?5cHRM?5chunk?$AA@ 00547e80     gapidraw:pngrutil.obj
 0003:0000de98       ??_C@_0BJ@NMPL@Missing?5PLTE?5before?5cHRM?$AA@ 00547e98     gapidraw:pngrutil.obj
 0003:0000deb4       ??_C@_0BI@HNJF@Invalid?5cHRM?5after?5IDAT?$AA@ 00547eb4     gapidraw:pngrutil.obj
 0003:0000decc       ??_C@_0BM@DODO@Incorrect?5cHRM?5chunk?5length?$AA@ 00547ecc     gapidraw:pngrutil.obj
 0003:0000dee8       ??_C@_0BJ@EAEO@Missing?5IHDR?5before?5cHRM?$AA@ 00547ee8     gapidraw:pngrutil.obj
 0003:0000df04       ??_C@_0BN@MJP@incorrect?5gamma?$DN?$CI?$CFd?1100000?$CJ?6?$AA@ 00547f04     gapidraw:pngrutil.obj
 0003:0000df24       ??_C@_0BE@NIIK@Unknown?5sRGB?5intent?$AA@ 00547f24     gapidraw:pngrutil.obj
 0003:0000df38       ??_C@_0BF@PHND@Duplicate?5sRGB?5chunk?$AA@ 00547f38     gapidraw:pngrutil.obj
 0003:0000df50       ??_C@_0BI@PFHN@Out?5of?5place?5sRGB?5chunk?$AA@ 00547f50     gapidraw:pngrutil.obj
 0003:0000df68       ??_C@_0BI@HMGK@Invalid?5sRGB?5after?5IDAT?$AA@ 00547f68     gapidraw:pngrutil.obj
 0003:0000df80       ??_C@_0BM@KMIB@Incorrect?5sRGB?5chunk?5length?$AA@ 00547f80     gapidraw:pngrutil.obj
 0003:0000df9c       ??_C@_0BJ@CHGJ@Missing?5IHDR?5before?5sRGB?$AA@ 00547f9c     gapidraw:pngrutil.obj
 0003:0000dfb8       ??_C@_0CL@BDL@Profile?5size?5field?5missing?5from?5@ 00547fb8     gapidraw:pngrutil.obj
 0003:0000dfe4       ??_C@_0CC@NAP@Ignoring?5truncated?5iCCP?5profile?4@ 00547fe4     gapidraw:pngrutil.obj
 0003:0000e008       ??_C@_0DA@OPJP@Ignoring?5nonzero?5compression?5typ@ 00548008     gapidraw:pngrutil.obj
 0003:0000e038       ??_C@_0BF@DGKF@Malformed?5iCCP?5chunk?$AA@ 00548038     gapidraw:pngrutil.obj
 0003:0000e050       ??_C@_0BF@BIGA@Duplicate?5iCCP?5chunk?$AA@ 00548050     gapidraw:pngrutil.obj
 0003:0000e068       ??_C@_0BI@BKMO@Out?5of?5place?5iCCP?5chunk?$AA@ 00548068     gapidraw:pngrutil.obj
 0003:0000e080       ??_C@_0BI@CDKA@Invalid?5iCCP?5after?5IDAT?$AA@ 00548080     gapidraw:pngrutil.obj
 0003:0000e098       ??_C@_0BJ@MHPE@Missing?5IHDR?5before?5iCCP?$AA@ 00548098     gapidraw:pngrutil.obj
 0003:0000e0b4       ??_C@_0BK@JMC@sPLT?5chunk?5has?5bad?5length?$AA@ 005480b4     gapidraw:pngrutil.obj
 0003:0000e0d0       ??_C@_0BF@LFGE@malformed?5sPLT?5chunk?$AA@ 005480d0     gapidraw:pngrutil.obj
 0003:0000e0e8       ??_C@_0BI@PGMG@Invalid?5sPLT?5after?5IDAT?$AA@ 005480e8     gapidraw:pngrutil.obj
 0003:0000e100       ??_C@_0BJ@FLON@Missing?5IHDR?5before?5sPLT?$AA@ 00548100     gapidraw:pngrutil.obj
 0003:0000e11c       ??_C@_0CK@NLHG@tRNS?5chunk?5not?5allowed?5with?5alph@ 0054811c     gapidraw:pngrutil.obj
 0003:0000e148       ??_C@_0BH@BEAK@Zero?5length?5tRNS?5chunk?$AA@ 00548148     gapidraw:pngrutil.obj
 0003:0000e160       ??_C@_0BM@BCIB@Incorrect?5tRNS?5chunk?5length?$AA@ 00548160     gapidraw:pngrutil.obj
 0003:0000e17c       ??_C@_0BF@JGAJ@Duplicate?5tRNS?5chunk?$AA@ 0054817c     gapidraw:pngrutil.obj
 0003:0000e194       ??_C@_0BI@FIEL@Invalid?5tRNS?5after?5IDAT?$AA@ 00548194     gapidraw:pngrutil.obj
 0003:0000e1ac       ??_C@_0BJ@OBHL@Missing?5PLTE?5before?5tRNS?$AA@ 005481ac     gapidraw:pngrutil.obj
 0003:0000e1c8       ??_C@_0BJ@HNMO@Missing?5IHDR?5before?5tRNS?$AA@ 005481c8     gapidraw:pngrutil.obj
 0003:0000e1e4       ??_C@_0CB@DAOE@Incorrect?5bKGD?5chunk?5index?5value@ 005481e4     gapidraw:pngrutil.obj
 0003:0000e208       ??_C@_0BM@OIKG@Incorrect?5bKGD?5chunk?5length?$AA@ 00548208     gapidraw:pngrutil.obj
 0003:0000e224       ??_C@_0BF@JHMD@Duplicate?5bKGD?5chunk?$AA@ 00548224     gapidraw:pngrutil.obj
 0003:0000e23c       ??_C@_0BJ@NHBE@Missing?5PLTE?5before?5bKGD?$AA@ 0054823c     gapidraw:pngrutil.obj
 0003:0000e258       ??_C@_0BI@FPHM@Invalid?5bKGD?5after?5IDAT?$AA@ 00548258     gapidraw:pngrutil.obj
 0003:0000e270       ??_C@_0BJ@ELKB@Missing?5IHDR?5before?5bKGD?$AA@ 00548270     gapidraw:pngrutil.obj
 0003:0000e28c       ??_C@_0BF@DJMM@Duplicate?5hIST?5chunk?$AA@ 0054828c     gapidraw:pngrutil.obj
 0003:0000e2a4       ??_C@_0BJ@IKHO@Missing?5PLTE?5before?5hIST?$AA@ 005482a4     gapidraw:pngrutil.obj
 0003:0000e2c0       ??_C@_0BI@CFN@Invalid?5hIST?5after?5IDAT?$AA@ 005482c0     gapidraw:pngrutil.obj
 0003:0000e2d8       ??_C@_0BM@MHPM@Incorrect?5hIST?5chunk?5length?$AA@ 005482d8     gapidraw:pngrutil.obj
 0003:0000e2f4       ??_C@_0BJ@BGML@Missing?5IHDR?5before?5hIST?$AA@ 005482f4     gapidraw:pngrutil.obj
 0003:0000e310       ??_C@_0BF@LDMH@Duplicate?5pHYs?5chunk?$AA@ 00548310     gapidraw:pngrutil.obj
 0003:0000e328       ??_C@_0BI@IHL@Invalid?5pHYs?5after?5IDAT?$AA@ 00548328     gapidraw:pngrutil.obj
 0003:0000e340       ??_C@_0BM@POPF@Incorrect?5pHYs?5chunk?5length?$AA@ 00548340     gapidraw:pngrutil.obj
 0003:0000e35c       ??_C@_0BJ@KEGI@Missing?5IHDR?5before?5pHYs?$AA@ 0054835c     gapidraw:pngrutil.obj
 0003:0000e378       ??_C@_0BF@DKBL@Duplicate?5oFFs?5chunk?$AA@ 00548378     gapidraw:pngrutil.obj
 0003:0000e390       ??_C@_0BI@JCMB@Invalid?5oFFs?5after?5IDAT?$AA@ 00548390     gapidraw:pngrutil.obj
 0003:0000e3a8       ??_C@_0BM@GJPO@Incorrect?5oFFs?5chunk?5length?$AA@ 005483a8     gapidraw:pngrutil.obj
 0003:0000e3c4       ??_C@_0BJ@ODAN@Missing?5IHDR?5before?5oFFs?$AA@ 005483c4     gapidraw:pngrutil.obj
 0003:0000e3e0       ??_C@_0CK@FOJK@Unrecognized?5equation?5type?5for?5p@ 005483e0     gapidraw:pngrutil.obj
 0003:0000e40c       ??_C@_0CK@ECLA@Invalid?5pCAL?5parameters?5for?5equa@ 0054840c     gapidraw:pngrutil.obj
 0003:0000e438       ??_C@_0BC@DJMJ@Invalid?5pCAL?5data?$AA@ 00548438     gapidraw:pngrutil.obj
 0003:0000e44c       ??_C@_0BF@KCGI@Duplicate?5pCAL?5chunk?$AA@ 0054844c     gapidraw:pngrutil.obj
 0003:0000e464       ??_C@_0BI@HKIK@Invalid?5pCAL?5after?5IDAT?$AA@ 00548464     gapidraw:pngrutil.obj
 0003:0000e47c       ??_C@_0BJ@OHNG@Missing?5IHDR?5before?5pCAL?$AA@ 0054847c     gapidraw:pngrutil.obj
 0003:0000e498       ??_C@_0BC@HPBB@Invalid?5sCAL?5data?$AA@ 00548498     gapidraw:pngrutil.obj
 0003:0000e4ac       ??_C@_0CG@LJOP@malformed?5height?5string?5in?5sCAL?5@ 005484ac     gapidraw:pngrutil.obj
 0003:0000e4d4       ??_C@_0CF@DIMJ@malformed?5width?5string?5in?5sCAL?5c@ 005484d4     gapidraw:pngrutil.obj
 0003:0000e4fc       ??_C@_0BF@DCCO@Duplicate?5sCAL?5chunk?$AA@ 005484fc     gapidraw:pngrutil.obj
 0003:0000e514       ??_C@_0BI@DNGK@Invalid?5sCAL?5after?5IDAT?$AA@ 00548514     gapidraw:pngrutil.obj
 0003:0000e52c       ??_C@_0BJ@IICA@Missing?5IHDR?5before?5sCAL?$AA@ 0054852c     gapidraw:pngrutil.obj
 0003:0000e548       ??_C@_0BF@DAEG@Duplicate?5tIME?5chunk?$AA@ 00548548     gapidraw:pngrutil.obj
 0003:0000e560       ??_C@_0BM@OBOI@Incorrect?5tIME?5chunk?5length?$AA@ 00548560     gapidraw:pngrutil.obj
 0003:0000e57c       ??_C@_0BI@DCOI@Out?5of?5place?5tIME?5chunk?$AA@ 0054857c     gapidraw:pngrutil.obj
 0003:0000e594       ??_C@_0BJ@PIJG@Missing?5IHDR?5before?5tEXt?$AA@ 00548594     gapidraw:pngrutil.obj
 0003:0000e5b0       ??_C@_0CH@LDIG@Unknown?5compression?5type?5in?5zTXt@ 005485b0     gapidraw:pngrutil.obj
 0003:0000e5d8       ??_C@_0BH@OOHH@Zero?5length?5zTXt?5chunk?$AA@ 005485d8     gapidraw:pngrutil.obj
 0003:0000e5f0       ??_C@_0BJ@HOJG@Missing?5IHDR?5before?5zTXt?$AA@ 005485f0     gapidraw:pngrutil.obj
 0003:0000e60c       ??_C@_0BH@CPMG@unknown?5critical?5chunk?$AA@ 0054860c     gapidraw:pngrutil.obj
 0003:0000e624       ??_C@_0BD@LAFO@invalid?5chunk?5type?$AA@ 00548624     gapidraw:pngrutil.obj
 0003:0000e638       ??_C@_0CC@GHFK@Ignoring?5bad?5adaptive?5filter?5typ@ 00548638     gapidraw:pngrutil.obj
 0003:0000e65c       ??_C@_0BH@GFFD@Extra?5compression?5data?$AA@ 0054865c     gapidraw:pngrutil.obj
 0003:0000e674       ??_C@_0BE@ONCP@Decompression?5Error?$AA@ 00548674     gapidraw:pngrutil.obj
 0003:0000e688       ??_C@_0CB@OJBF@Invalid?5interlace?5type?5specified@ 00548688     gapidraw:pngwutil.obj
 0003:0000e6ac       ??_C@_0BO@JCBH@Invalid?5filter?5type?5specified?$AA@ 005486ac     gapidraw:pngwutil.obj
 0003:0000e6cc       ??_C@_0CD@OGII@Invalid?5compression?5type?5specifi@ 005486cc     gapidraw:pngwutil.obj
 0003:0000e6f0       ??_C@_0CD@ONMI@Invalid?5image?5color?5type?5specifi@ 005486f0     gapidraw:pngwutil.obj
 0003:0000e714       ??_C@_0CB@IOGH@Invalid?5bit?5depth?5for?5RGBA?5image@ 00548714     gapidraw:pngwutil.obj
 0003:0000e738       ??_C@_0CM@IGJG@Invalid?5bit?5depth?5for?5grayscale?$CL@ 00548738     gapidraw:pngwutil.obj
 0003:0000e764       ??_C@_0CF@LMPA@Invalid?5bit?5depth?5for?5paletted?5i@ 00548764     gapidraw:pngwutil.obj
 0003:0000e78c       ??_C@_0CA@CNP@Invalid?5bit?5depth?5for?5RGB?5image?$AA@ 0054878c     gapidraw:pngwutil.obj
 0003:0000e7ac       ??_C@_0CG@DOMJ@Invalid?5bit?5depth?5for?5grayscale?5@ 005487ac     gapidraw:pngwutil.obj
 0003:0000e7d4       ??_C@_0DI@DBPL@Ignoring?5request?5to?5write?5a?5PLTE@ 005487d4     gapidraw:pngwutil.obj
 0003:0000e80c       ??_C@_0CE@BDI@Invalid?5number?5of?5colors?5in?5pale@ 0054880c     gapidraw:pngwutil.obj
 0003:0000e830       ??_C@_0CI@BGIB@Invalid?5sRGB?5rendering?5intent?5sp@ 00548830     gapidraw:pngwutil.obj
 0003:0000e858       ??_C@_0BM@FCFH@Empty?5keyword?5in?5iCCP?5chunk?$AA@ 00548858     gapidraw:pngwutil.obj
 0003:0000e874       ??_C@_0CH@MHJC@Unknown?5compression?5type?5in?5iCCP@ 00548874     gapidraw:pngwutil.obj
 0003:0000e89c       ??_C@_0BM@ELPH@Unknown?5compression?5type?5?$CFd?$AA@ 0054889c     gapidraw:pngwutil.obj
 0003:0000e8b8       ??_C@_0BM@KOFE@Empty?5keyword?5in?5sPLT?5chunk?$AA@ 005488b8     gapidraw:pngwutil.obj
 0003:0000e8d4       ??_C@_0BN@IIED@Invalid?5sBIT?5depth?5specified?$AA@ 005488d4     gapidraw:pngwutil.obj
 0003:0000e8f4       ??_C@_0BI@MIBN@white_x?$DN?$CFf?0?5white_y?$DN?$CFf?6?$AA@ 005488f4     gapidraw:pngwutil.obj
 0003:0000e90c       ??_C@_0CD@LIOJ@Invalid?5cHRM?5white?5point?5specifi@ 0054890c     gapidraw:pngwutil.obj
 0003:0000e930       ??_C@_0CB@JMFI@Invalid?5cHRM?5red?5point?5specified@ 00548930     gapidraw:pngwutil.obj
 0003:0000e954       ??_C@_0CD@OEBJ@Invalid?5cHRM?5green?5point?5specifi@ 00548954     gapidraw:pngwutil.obj
 0003:0000e978       ??_C@_0CC@BDBB@Invalid?5cHRM?5blue?5point?5specifie@ 00548978     gapidraw:pngwutil.obj
 0003:0000e99c       ??_C@_0CH@EACP@Can?8t?5write?5tRNS?5with?5an?5alpha?5c@ 0054899c     gapidraw:pngwutil.obj
 0003:0000e9c4       ??_C@_0EA@PCBD@Ignoring?5attempt?5to?5write?516?9bit@ 005489c4     gapidraw:pngwutil.obj
 0003:0000ea04       ??_C@_0EA@DCOG@Ignoring?5attempt?5to?5write?5tRNS?5c@ 00548a04     gapidraw:pngwutil.obj
 0003:0000ea44       ??_C@_0CP@LIOC@Invalid?5number?5of?5transparent?5co@ 00548a44     gapidraw:pngwutil.obj
 0003:0000ea74       ??_C@_0EA@LJJN@Ignoring?5attempt?5to?5write?5bKGD?5c@ 00548a74     gapidraw:pngwutil.obj
 0003:0000eab4       ??_C@_0EA@GLI@Ignoring?5attempt?5to?5write?516?9bit@ 00548ab4     gapidraw:pngwutil.obj
 0003:0000eaf4       ??_C@_0CB@HLMH@Invalid?5background?5palette?5index@ 00548af4     gapidraw:pngwutil.obj
 0003:0000eb18       ??_C@_0CO@MCGM@Invalid?5number?5of?5histogram?5entr@ 00548b18     gapidraw:pngwutil.obj
 0003:0000eb48       ??_C@_0BE@LNHL@zero?5length?5keyword?$AA@ 00548b48     gapidraw:pngwutil.obj
 0003:0000eb5c       ??_C@_0CJ@MFCD@keyword?5length?5must?5be?51?5?9?579?5ch@ 00548b5c     gapidraw:pngwutil.obj
 0003:0000eb88       ??_C@_0BE@HPMF@Zero?5length?5keyword?$AA@ 00548b88     gapidraw:pngwutil.obj
 0003:0000eb9c       ??_C@_0CL@OPHM@extra?5interior?5spaces?5removed?5fr@ 00548b9c     gapidraw:pngwutil.obj
 0003:0000ebc8       ??_C@_0CE@GCCB@leading?5spaces?5removed?5from?5keyw@ 00548bc8     gapidraw:pngwutil.obj
 0003:0000ebec       ??_C@_0CF@CMLN@trailing?5spaces?5removed?5from?5key@ 00548bec     gapidraw:pngwutil.obj
 0003:0000ec14       ??_C@_0CB@GNKN@invalid?5keyword?5character?50x?$CF02X@ 00548c14     gapidraw:pngwutil.obj
 0003:0000ec38       ??_C@_0BM@JOBG@Empty?5keyword?5in?5tEXt?5chunk?$AA@ 00548c38     gapidraw:pngwutil.obj
 0003:0000ec54       ??_C@_0BM@CGED@Empty?5keyword?5in?5zTXt?5chunk?$AA@ 00548c54     gapidraw:pngwutil.obj
 0003:0000ec70       ??_C@_0CG@OIOA@Unrecognized?5unit?5type?5for?5oFFs?5@ 00548c70     gapidraw:pngwutil.obj
 0003:0000ec98       ??_C@_07HALG@?$CF12?412e?$AA@ 00548c98     gapidraw:pngwutil.obj
 0003:0000eca0       ??_C@_0CG@GBDM@Unrecognized?5unit?5type?5for?5pHYs?5@ 00548ca0     gapidraw:pngwutil.obj
 0003:0000ecc8       ??_C@_0CG@MMFJ@Invalid?5time?5specified?5for?5tIME?5@ 00548cc8     gapidraw:pngwutil.obj
 0003:0000ecf4       ??_C@_0BK@BNJN@invalid?5bit?5length?5repeat?$AA@ 00548cf4     gapidraw:infblock.obj
 0003:0000ed10       ??_C@_0CE@LAKP@too?5many?5length?5or?5distance?5symb@ 00548d10     gapidraw:infblock.obj
 0003:0000ed34       ??_C@_0BN@DBOJ@invalid?5stored?5block?5lengths?$AA@ 00548d34     gapidraw:infblock.obj
 0003:0000ed54       ??_C@_0BD@IFBC@invalid?5block?5type?$AA@ 00548d54     gapidraw:infblock.obj
 0003:0000ed68       _z_errmsg                  00548d68     gapidraw:zutil.obj
 0003:0000ed90       ??_C@_0BF@HPBB@incompatible?5version?$AA@ 00548d90     gapidraw:zutil.obj
 0003:0000eda8       ??_C@_0N@EHHN@buffer?5error?$AA@ 00548da8     gapidraw:zutil.obj
 0003:0000edb8       ??_C@_0BE@EMHE@insufficient?5memory?$AA@ 00548db8     gapidraw:zutil.obj
 0003:0000edcc       ??_C@_0L@EBEB@data?5error?$AA@ 00548dcc     gapidraw:zutil.obj
 0003:0000edd8       ??_C@_0N@OPOA@stream?5error?$AA@ 00548dd8     gapidraw:zutil.obj
 0003:0000ede8       ??_C@_0L@DFEP@file?5error?$AA@ 00548de8     gapidraw:zutil.obj
 0003:0000edf4       ??_C@_0L@JPFB@stream?5end?$AA@ 00548df4     gapidraw:zutil.obj
 0003:0000ee44       ??_C@_0BG@EGK@invalid?5distance?5code?$AA@ 00548e44     gapidraw:infcodes.obj
 0003:0000ee5c       ??_C@_0BM@CHJP@invalid?5literal?1length?5code?$AA@ 00548e5c     gapidraw:infcodes.obj
 0003:0000ff80       ??_C@_0CE@MFNM@incomplete?5dynamic?5bit?5lengths?5t@ 00549f80     gapidraw:inftrees.obj
 0003:0000ffa4       ??_C@_0CI@BBGL@oversubscribed?5dynamic?5bit?5lengt@ 00549fa4     gapidraw:inftrees.obj
 0003:0000ffcc       ??_C@_0BP@KPP@incomplete?5literal?1length?5tree?$AA@ 00549fcc     gapidraw:inftrees.obj
 0003:0000ffec       ??_C@_0CD@ODII@oversubscribed?5literal?1length?5tr@ 00549fec     gapidraw:inftrees.obj
 0003:00010010       ??_C@_0CB@INA@empty?5distance?5tree?5with?5lengths@ 0054a010     gapidraw:inftrees.obj
 0003:00010034       ??_C@_0BJ@NKOC@incomplete?5distance?5tree?$AA@ 0054a034     gapidraw:inftrees.obj
 0003:00010050       ??_C@_0BN@OAAG@oversubscribed?5distance?5tree?$AA@ 0054a050     gapidraw:inftrees.obj
 0003:00010070       _inflate_mask              0054a070     gapidraw:infutil.obj
 0003:000100b4       __NLG_Destination          0054a0b4     LIBC:exsup.obj
 0003:000100d0       __fltused                  0054a0d0     LIBC:fpinit.obj
 0003:000100d4       __ldused                   0054a0d4     LIBC:fpinit.obj
 0003:000100d8       __FPinit                   0054a0d8     LIBC:fpinit.obj
 0003:000100dc       __FPmtinit                 0054a0dc     LIBC:fpinit.obj
 0003:000100e0       __FPmtterm                 0054a0e0     LIBC:fpinit.obj
 0003:00010130       ??_R0?AVtype_info@@@8      0054a130     LIBC:typinfo.obj
 0003:00010148       ?__pMyUnhandledExceptionFilter@@3PAXA 0054a148     LIBC:throw.obj
 0003:00010150       __aexit_rtn                0054a150     LIBC:wincrt0.obj
 0003:00010154       ___app_type                0054a154     LIBC:wincrt0.obj
 0003:00010160       __iob                      0054a160     LIBC:_file.obj
 0003:000103e0       __half                     0054a3e0     LIBC:pow.obj
 0003:000103f4       ___security_cookie         0054a3f4     LIBC:seccook.obj
 0003:000103f8       ?__pUnexpected@@3P6AXXZA   0054a3f8     LIBC:hooks.obj
 0003:000103fc       ?__pInconsistency@@3P6AXXZA 0054a3fc     LIBC:hooks.obj
 0003:00010400       __cfltcvt_tab              0054a400     LIBC:cmiscdat.obj
 0003:00010420       ___nullstring              0054a420     LIBC:output.obj
 0003:00010424       ___wnullstring             0054a424     LIBC:output.obj
 0003:00010590       ___lc_clike                0054a590     LIBC:nlsdata2.obj
 0003:00010594       __pctype                   0054a594     LIBC:ctype.obj
 0003:00010598       __pwctype                  0054a598     LIBC:ctype.obj
 0003:0001059c       ___mb_cur_max              0054a59c     LIBC:nlsdata1.obj
 0003:000105a0       ___decimal_point           0054a5a0     LIBC:nlsdata1.obj
 0003:000105a4       ___decimal_point_length    0054a5a4     LIBC:nlsdata1.obj
 0003:000105a8       __timezone                 0054a5a8     LIBC:timeset.obj
 0003:000105ac       __daylight                 0054a5ac     LIBC:timeset.obj
 0003:000105b0       __dstbias                  0054a5b0     LIBC:timeset.obj
 0003:00010638       __tzname                   0054a638     LIBC:timeset.obj
 0003:00010658       __amblksiz                 0054a658     LIBC:heapinit.obj
 0003:00010760       __indefinite               0054a760     LIBC:87disp.obj
 0003:0001076a       __piby2                    0054a76a     LIBC:87disp.obj
 0003:0001077c       __cpower                   0054a77c     LIBC:87disp.obj
 0003:00010790       __OP_ATAN2jmptab           0054a790     LIBC:87triga.obj
 0003:000107e0       ___badioinfo               0054a7e0     LIBC:ioinit.obj
 0003:00010880       __XcptActTab               0054a880     LIBC:winxfltr.obj
 0003:000108f8       __First_FPE_Indx           0054a8f8     LIBC:winxfltr.obj
 0003:000108fc       __Num_FPE                  0054a8fc     LIBC:winxfltr.obj
 0003:00010900       __XcptActTabCount          0054a900     LIBC:winxfltr.obj
 0003:00010904       __fpecode                  0054a904     LIBC:winxfltr.obj
 0003:00010910       __infinity                 0054a910     LIBC:87tran.obj
 0003:0001091a       __minfinity                0054a91a     LIBC:87tran.obj
 0003:00010924       __logemax                  0054a924     LIBC:87tran.obj
 0003:00010954       __OP_EXPjmptab             0054a954     LIBC:87tran.obj
 0003:00010974       __lpdays                   0054a974     LIBC:days.obj
 0003:000109a8       __days                     0054a9a8     LIBC:days.obj
 0003:000109dc       __HUGE                     0054a9dc     LIBC:huge.obj
 0003:00010a20       __pmatherr                 0054aa20     LIBC:libm_error.obj
 0003:00010b90       __d_inf                    0054ab90     LIBC:util.obj
 0003:00010b98       __d_ind                    0054ab98     LIBC:util.obj
 0003:00010ba0       __d_max                    0054aba0     LIBC:util.obj
 0003:00010ba8       __d_min                    0054aba8     LIBC:util.obj
 0003:00010bb0       __d_mzero                  0054abb0     LIBC:util.obj
 0003:00010ca0       __matherr_flag             0054aca0     LIBC:matherr.obj
 0003:00010cc0       __pow10pos                 0054acc0     LIBC:constpow.obj
 0003:00010e20       __pow10neg                 0054ae20     LIBC:constpow.obj
 0003:00010fbc       ?mInstance@ldwEventManager@@0PAV1@A 0054afbc     ldwEventManager.obj
 0003:00011030       ?mInstance@ldwGameState@@1PAV1@A 0054b030     ldwGameState.obj
 0003:00011650       ?mInstance@ldwGameWindow@@0PAV1@A 0054b650     ldwGameWindow.obj
 0003:00011670       ?m_pGapiDraw@CGapiApplication@@2PAVCGapiDraw@@A 0054b670     ldwGapiApplication.obj
 0003:00011904       ?mInstance@ldwLog@@0PAV1@A 0054b904     ldwLog.obj
 0003:0001195c       ?mGlobalMute@ldwSoundTrackImpl@@2_NA 0054b95c     ldwSound.obj
 0003:000119f4       ?lasterrorU@@3KA           0054b9f4     unzip.obj
 0003:00011a18       ?AnimManager@@3VCAnimManager@@A 0054ba18     AnimManager.obj
 0003:00012b68       ?Behavior@@3VCBehavior@@A  0054cb68     Behavior.obj
 0003:000136d8       ?Graveyard@@3VCGraveyard@@A 0054d6d8     Graveyard.obj
 0003:0001a6a8       ?VillagerManager@@3VCVillagerManager@@A 005546a8     VillagerManager.obj
 0003:00142540       ?m_pInstance@CCollectionScene@@0PAV1@A 0067c540     CollectionScene.obj
 0003:00142604       ?m_pInstance@CProgressScene@@0PAV1@A 0067c604     ProgressScene.obj
 0003:001426bc       ?m_pInstance@CStoryScene@@0PAV1@A 0067c6bc     StoryScene.obj
 0003:00142760       ?m_pInstance@CTechScene@@0PAV1@A 0067c760     TechScene.obj
 0003:00142944       ?m_pInstance@theMainScene@@0PAV1@A 0067c944     theMainScene.obj
 0003:00142d20       ?mInstance@CIslandEvents@@0PAV1@A 0067cd20     IslandEvents.obj
 0003:00142d24       ?mEventHasFired@CIslandEvents@@0PA_NA 0067cd24     IslandEvents.obj
 0003:00142d60       ?mEventList@CIslandEvents@@0PAPAVCIslandEvent@@A 0067cd60     IslandEvents.obj
 0003:00143420       ?Fog@@3VCFog@@A            0067d420     Fog.obj
 0003:0014483c       ?Lightning@@3VCLightning@@A 0067e83c     Lightning.obj
 0003:00144878       ?Rain@@3VCRain@@A          0067e878     Rain.obj
 0003:001478d8       ?SunBeam@@3VCSunBeam@@A    006818d8     SunBeam.obj
 0003:00147e30       ?Weather@@3VCWeather@@A    00681e30     Weather.obj
 0003:00147ee8       ?ContentMap@@3VCContentMap@@A 00681ee8     ContentMap.obj
 0003:00187fcc       ?Environment@@3VCEnvironment@@A 006c1fcc     Environment.obj
 0003:00188090       ?HotSpot@@3VCHotSpot@@A    006c2090     HotSpot.obj
 0003:001882c8       ?Redirect@@3VCRedirect@@A  006c22c8     Redirect.obj
 0003:00188308       ?Waypoint@@3VCWaypoint@@A  006c2308     Waypoint.obj
 0003:00188358       ?WorldMap@@3VCWorldMap@@A  006c2358     WorldMap.obj
 0003:00188440       ?mPathGradient@CWorldPath@@0UPathGradient@1@A 006c2440     WorldPath.obj
 0003:001a845c       ?scm_sRect@CWorldView@@0UldwRect@@B 006e245c     WorldView.obj
 0003:001a8480       ?WorldView@@3VCWorldView@@A 006e2480     WorldView.obj
 0003:001a84f0       ?EnvironmentalSound@@3VCEnvironmentalSound@@A 006e24f0     EnvironmentalSound.obj
 0003:001a9538       ?Sound@@3VCSound@@A        006e3538     Sound.obj
 0003:001a9cbc       ?SoundTrack@@3VCSoundTrack@@A 006e3cbc     SoundTrack.obj
 0003:001a9d98       ?Bird@@3VCBird@@A          006e3d98     Bird.obj
 0003:001aa014       ?mInstance@theHummingbirdClass@@1PAV1@A 006e4014     HummingbirdClass.obj
 0003:001aa0f8       ?Shark@@3VCShark@@A        006e40f8     Shark.obj
 0003:001aa190       ?mInstance@theButterflyClass@@1PAV1@A 006e4190     theButterflyClass.obj
 0003:001aa230       ?BFGProtection@@3VCBFGProtection@@A 006e4230     BFGProtection.obj
 0003:001aa244       ?Distributor@@3VCDistributor@@A 006e4244     Distributor.obj
 0003:001aa288       ?Expiration@@3VCExpiration@@A 006e4288     Expiration.obj
 0003:001aa290       ?ghInst@@3PAUHINSTANCE__@@A 006e4290     main.obj
 0003:001aa348       ?FoodStore@@3VCFoodStore@@A 006e4348     FoodStore.obj
 0003:001aa3a8       ?GameStats@@3VCGameStats@@A 006e43a8     GameStats.obj
 0003:001aa51c       ?sm_iNumTimers@CGameTime@@0HA 006e451c     GameTime.obj
 0003:001aa578       ?GameTime@@3VCGameTime@@A  006e4578     GameTime.obj
 0003:001aa6d0       ?Potion@@3VCPotion@@A      006e46d0     Potion.obj
 0003:001aa6f8       ?sm_iNumObservers@CTech@@0HA 006e46f8     Tech.obj
 0003:001aa6fc       ?Tech@@3VCTech@@A          006e46fc     Tech.obj
 0003:001aa72c       ?TechPoints@@3VCTechPoints@@A 006e472c     TechPoints.obj
 0003:001aa8b4       ?mInstance@theRealtimeManager@@1PAV1@A 006e48b4     theRealtimeManager.obj
 0003:001aa9b0       ?Decal@@3VCDecal@@A        006e49b0     Decal.obj
 0003:001abf00       ?FloatingAnim@@3VCFloatingAnim@@A 006e5f00     FloatingAnim.obj
 0003:001b4770       ?Smoke@@3VCSmoke@@A        006ee770     Smoke.obj
 0003:001b49d0       ?BehaviorEditor@@3VCBehaviorEditor@@A 006ee9d0     BehaviorEditor.obj
 0003:001b71d8       ?ContentMapEditor@@3VCContentMapEditor@@A 006f11d8     ContentMapEditor.obj
 0003:001b722c       ?Debugger@@3VCDebugger@@A  006f122c     Debugger.obj
 0003:001b72b4       ?Editor@@3VCEditor@@A      006f12b4     Editor.obj
 0003:001b72f8       ?WaypointEditor@@3VCWaypointEditor@@A 006f12f8     WaypointEditor.obj
 0003:001b7360       ?Collectable@@3VCCollectable@@A 006f1360     Collectable.obj
 0003:001b7ab0       ?CollectableItem@@3VCCollectableItem@@A 006f1ab0     CollectableItem.obj
 0003:001b7d00       ?DealerSay@@3VCDealerSay@@A 006f1d00     DealerSay.obj
 0003:001b7ec8       ?SceneManager@@3VCSceneManager@@A 006f1ec8     SceneManager.obj
 0003:001baf08       ?mInstance@theDealerSay@@1PAV1@A 006f4f08     theDealerSay.obj
 0003:001bafa8       ?mInstance@theGraphicsManager@@1PAV1@A 006f4fa8     theGraphicsManager.obj
 0003:001bb060       ?mInstance@thePrizeMsgAssembler@@1PAV1@A 006f5060     thePrizeMsgAssembler.obj
 0003:001bb104       ?mInstance@theSlicedVariableMeter@@1PAV1@A 006f5104     theSlicedVariableMeter.obj
 0003:001bc4e8       ?mInstance@theStringManager@@1PAV1@A 006f64e8     theStringManager.obj
 0003:001bc508       ?mInstance@theVariableMeter@@1PAV1@A 006f6508     theVariableMeter.obj
 0003:001bc628       ?AlchemyLab@@3VCAlchemyLab@@A 006f6628     AlchemyLab.obj
 0003:001bc700       ?AlchemyPot@@3VCAlchemyPot@@A 006f6700     AlchemyPot.obj
 0003:001bd0cc       ?AlchemyTable@@3VCAlchemyTable@@A 006f70cc     AlchemyTable.obj
 0003:001bd1c8       ?Aromatherapy@@3VCAromatherapy@@A 006f71c8     Aromatherapy.obj
 0003:001bd27c       ?Bath@@3VCBath@@A          006f727c     Bath.obj
 0003:001bd2e4       ?BeeHive@@3VCBeeHive@@A    006f72e4     BeeHive.obj
 0003:001bd3d4       ?ChalkBoard@@3VCChalkBoard@@A 006f73d4     ChalkBoard.obj
 0003:001bd46c       ?Chief@@3VCChief@@A        006f746c     Chief.obj
 0003:001bd4b0       ?Construction@@3VCConstruction@@A 006f74b0     Construction.obj
 0003:001bd5e0       ?scm_sPossiblePearlPosition@CDoorKey@@0QBUldwPoint@@B 006f75e0     DoorKey.obj
 0003:001bd6a8       ?DoorKey@@3VCDoorKey@@A    006f76a8     DoorKey.obj
 0003:001bd6f4       ?FirePit@@3VCFirePit@@A    006f76f4     FirePit.obj
 0003:001bd8c0       ?Orchard@@3VCOrchard@@A    006f78c0     Orchard.obj
 0003:001bd9e8       ?scm_sPusherOffset@CPrincessStatue@@0QBUldwPoint@@B 006f79e8     PrincessStatue.obj
 0003:001bda88       ?PrincessStatue@@3VCPrincessStatue@@A 006f7a88     PrincessStatue.obj
 0003:001bdc80       ?Puzzle@@3VCPuzzle@@A      006f7c80     Puzzle.obj
 0003:001bdeb8       ?RainLift@@3VCRainLift@@A  006f7eb8     RainLift.obj
 0003:001bdf80       ?RosterOfTheDead@@3VCRosterOfTheDead@@A 006f7f80     RosterOfTheDead.obj
 0003:001be07c       ?Ruins@@3VCRuins@@A        006f807c     Ruins.obj
 0003:001be100       ?SharkCharmer@@3VCSharkCharmer@@A 006f8100     SharkCharmer.obj
 0003:001be16c       ?SunDisk@@3VCSunDisk@@A    006f816c     SunDisk.obj
 0003:001be218       ?WeatherDance@@3VCWeatherDance@@A 006f8218     WeatherDance.obj
 0003:001be290       ?MoviePlayer@@3VCMoviePlayer@@A 006f8290     MoviePlayer.obj
 0003:001be2ac       ?WM_ATLGETCONTROL@ATL@@3IA 006f82ac     FlashPlayer.obj
 0003:001be2b0       ?WM_ATLGETHOST@ATL@@3IA    006f82b0     FlashPlayer.obj
 0003:001be2b4       ?_pModule@ATL@@3PAVCComModule@1@A 006f82b4     FlashPlayer.obj
 0003:001be2b8       ?m_libid@CAtlModule@ATL@@2U_GUID@@A 006f82b8     FlashPlayer.obj
 0003:001be2c8       ?_pAtlModule@ATL@@3PAVCAtlModule@1@A 006f82c8     FlashPlayer.obj
 0003:001be2cc       ?m_bInitFailed@CAtlBaseModule@ATL@@2_NA 006f82cc     FlashPlayer.obj
 0003:001be2d0       ?_AtlWinModule@ATL@@3VCAtlWinModule@1@A 006f82d0     FlashPlayer.obj
 0003:001be2fc       ?map@?2??VTFromRegType@CRegParser@ATL@@KAHPBDAAG@Z@4QBUtypemap@23@B 006f82fc     FlashPlayer.obj
 0003:001be31c       ?$S4@?2??VTFromRegType@CRegParser@ATL@@KAHPBDAAG@Z@4IA 006f831c     FlashPlayer.obj
 0003:001be320       ?_Module@@3VCComModule@ATL@@A 006f8320     FlashPlayer.obj
 0003:001be3a8       ?Achievement@@3VCAchievement@@A 006f83a8     Achievement.obj
 0003:001be498       ?TutorialTip@@3VCTutorialTip@@A 006f8498     TutorialTip.obj
 0003:001bf0c0       ?IntroPage5@@3VCIntroPage5@@A 006f90c0     Pages.obj
 0003:001bf0d8       ?MidGamePage3@@3VCMidGamePage3@@A 006f90d8     Pages.obj
 0003:001bf11c       ?EndGamePage3@@3VCEndGamePage3@@A 006f911c     Pages.obj
 0003:001bf128       ?IntroPage3@@3VCIntroPage3@@A 006f9128     Pages.obj
 0003:001bf130       ?IntroPage2@@3VCIntroPage2@@A 006f9130     Pages.obj
 0003:001bf140       ?MidGamePage2@@3VCMidGamePage2@@A 006f9140     Pages.obj
 0003:001bf148       ?IntroPage4@@3VCIntroPage4@@A 006f9148     Pages.obj
 0003:001bf150       ?EndGamePage2@@3VCEndGamePage2@@A 006f9150     Pages.obj
 0003:001bf15c       ?IntroPage1@@3VCIntroPage1@@A 006f915c     Pages.obj
 0003:001bf16c       ?EndGamePage1@@3VCEndGamePage1@@A 006f916c     Pages.obj
 0003:001bf180       ?MidGamePage1@@3VCMidGamePage1@@A 006f9180     Pages.obj
 0003:001bf190       ?EndGamePage4@@3VCEndGamePage4@@A 006f9190     Pages.obj
 0003:001bf208       ?Story@@3VCStory@@A        006f9208     Story.obj
 0003:001bf704       ?g_pDisplay@@3PAVCDisplay@@A 006f9704     gapidraw:GapiDisplayDDraw.obj
 0003:001bf708       ?g_pColorConverter@@3PAVCColorConverter@gddisplay@@A 006f9708     gapidraw:GapiDisplayDDraw.obj
 0003:001bf710       ?hWnd@gdgdi@@3PAUHWND__@@A 006f9710     gapidraw:GapiLib.obj
 0003:001bf714       ?bSuspended@gdgdi@@3HA     006f9714     gapidraw:GapiLib.obj
 0003:001bf718       ?hBitmap@gdgdi@@3PAUHBITMAP__@@A 006f9718     gapidraw:GapiLib.obj
 0003:001bf71c       ?pBitmapBits@gdgdi@@3PAEA  006f971c     gapidraw:GapiLib.obj
 0003:001bf720       ?dp@gdgdi@@3UGXDisplayProperties@@A 006f9720     gapidraw:GapiLib.obj
 0003:001bf738       ??_C@_00A@?$AA@            006f9738     gapidraw:zutil.obj
 0003:001bf740       ___pPurecall               006f9740     LIBC:purevirt.obj
 0003:001bf744       ___fastflag                006f9744     LIBC:fpinit.obj
 0003:001bf748       __adjust_fdiv              006f9748     LIBC:fpinit.obj
 0003:001bf74c       _errno                     006f974c     LIBC:crt0dat.obj
 0003:001bf750       __doserrno                 006f9750     LIBC:crt0dat.obj
 0003:001bf754       __umaskval                 006f9754     LIBC:crt0dat.obj
 0003:001bf758       __osplatform               006f9758     LIBC:crt0dat.obj
 0003:001bf75c       __osver                    006f975c     LIBC:crt0dat.obj
 0003:001bf760       __winver                   006f9760     LIBC:crt0dat.obj
 0003:001bf764       __winmajor                 006f9764     LIBC:crt0dat.obj
 0003:001bf768       __winminor                 006f9768     LIBC:crt0dat.obj
 0003:001bf76c       ___argc                    006f976c     LIBC:crt0dat.obj
 0003:001bf770       ___argv                    006f9770     LIBC:crt0dat.obj
 0003:001bf774       ___wargv                   006f9774     LIBC:crt0dat.obj
 0003:001bf778       __environ                  006f9778     LIBC:crt0dat.obj
 0003:001bf77c       ___initenv                 006f977c     LIBC:crt0dat.obj
 0003:001bf780       __wenviron                 006f9780     LIBC:crt0dat.obj
 0003:001bf784       ___winitenv                006f9784     LIBC:crt0dat.obj
 0003:001bf788       __pgmptr                   006f9788     LIBC:crt0dat.obj
 0003:001bf78c       __wpgmptr                  006f978c     LIBC:crt0dat.obj
 0003:001bf790       __exitflag                 006f9790     LIBC:crt0dat.obj
 0003:001bf794       __C_Termination_Done       006f9794     LIBC:crt0dat.obj
 0003:001bf798       __C_Exit_Done              006f9798     LIBC:crt0dat.obj
 0003:001bf7c0       __aenvptr                  006f97c0     LIBC:wincrt0.obj
 0003:001bf7c4       __wenvptr                  006f97c4     LIBC:wincrt0.obj
 0003:001bf7c8       ___error_mode              006f97c8     LIBC:wincrt0.obj
 0003:001bf7cc       __cflush                   006f97cc     LIBC:_file.obj
 0003:001bf7f4       ?_pCurrentException@@3PAUEHExceptionRecord@@A 006f97f4     LIBC:frame.obj
 0003:001bf7f8       ?_pCurrentExContext@@3PAU_CONTEXT@@A 006f97f8     LIBC:frame.obj
 0003:001bf7fc       ?__ProcessingThrow@@3HA    006f97fc     LIBC:frame.obj
 0003:001bf800       ?__pSETranslator@@3P6AXIPAU_EXCEPTION_POINTERS@@@ZA 006f9800     LIBC:hooks.obj
 0003:001bf804       ?__pTerminate@@3P6AXXZA    006f9804     LIBC:hooks.obj
 0003:001bf81c       ___lc_handle               006f981c     LIBC:nlsdata2.obj
 0003:001bf834       ___lc_codepage             006f9834     LIBC:nlsdata2.obj
 0003:001bf838       ___lc_collate_cp           006f9838     LIBC:nlsdata2.obj
 0003:001bf83c       __stdbuf                   006f983c     LIBC:_sftbuf.obj
 0003:001bf900       ?_pnhHeap@@3P6AHI@ZA       006f9900     LIBC:handler.obj
 0003:001bf904       __newmode                  006f9904     LIBC:_newmode.obj
 0003:001bf96c       __adbgmsg                  006f996c     LIBC:crt0msg.obj
 0003:001bf970       __pxcptinfoptrs            006f9970     LIBC:winxfltr.obj
 0003:001bfadc       __commode                  006f9adc     LIBC:ncommode.obj
 0003:001bfafc       __fmode                    006f9afc     LIBC:txtmode.obj
 0003:001bfb04       ?_AtlBaseModule@ATL@@3VCAtlBaseModule@1@A 006f9b04     atls:atlbase.obj
 0003:001bfb40       ?$S1@?1??GetInstance@CGapiLib@@SAPAV2@XZ@4EA 006f9b40     <common>
 0003:001bfb60       ?instance@?1??GetInstance@CGapiLib@@SAPAV2@XZ@4V2@A 006f9b60     <common>
 0003:001bfb9c       ___use_sse2_mathfcns       006f9b9c     <common>
 0003:001bfba0       ___sse2_available          006f9ba0     <common>
 0003:001bfba4       __nhandle                  006f9ba4     <common>
 0003:001bfbc0       ___pioinfo                 006f9bc0     <common>
 0003:001bfcc0       ___mblcid                  006f9cc0     <common>
 0003:001bfcc4       ___ismbcodepage            006f9cc4     <common>
 0003:001bfce0       __mbctype                  006f9ce0     <common>
 0003:001bfde4       ___mbcodepage              006f9de4     <common>
 0003:001bfdf0       ___mbulinfo                006f9df0     <common>
 0003:001bfe00       __mbcasemap                006f9e00     <common>
 0003:001bff00       ___sbh_pHeaderDefer        006f9f00     <common>
 0003:001bff04       ___sbh_cntHeaderList       006f9f04     <common>
 0003:001bff08       ___sbh_pHeaderList         006f9f08     <common>
 0003:001bff0c       ___sbh_threshold           006f9f0c     <common>
 0003:001bff10       ___sbh_pHeaderScan         006f9f10     <common>
 0003:001bff14       ___sbh_sizeHeaderList      006f9f14     <common>
 0003:001bff18       ___sbh_indGroupDefer       006f9f18     <common>
 0003:001bff1c       __crtheap                  006f9f1c     <common>
 0003:001bff20       ___active_heap             006f9f20     <common>
 0003:001bff24       ___piob                    006f9f24     <common>
 0003:001bff40       __bufin                    006f9f40     <common>
 0003:001c0f40       __nstream                  006faf40     <common>
 0003:001c0f44       __acmdln                   006faf44     <common>
 0003:001c0f48       ___env_initialized         006faf48     <common>
 0003:001c0f4c       ___onexitend               006faf4c     <common>
 0003:001c0f50       ___onexitbegin             006faf50     <common>
 0003:001c0f54       ___mbctype_initialized     006faf54     <common>
 0004:00000000       ?hGlobal@@3PAUHWND__@@A    006fb000     main.obj

 entry point at        0001:000e7315

 Static symbols

 0001:0000b730       ?FindZipEntryIndex@@YAHPAUHZIP__@@PBDAAUZIPENTRY@@@Z 0040c730 f   ldwImageImpl.obj
 0001:000346b0       ?IsString@@YA?B_NPBDH@Z    004356b0 f   Graveyard.obj
 0001:000711e0       ?GetSoundItem@@YAPAUSoundItem@@W4ESound@@@Z 004721e0 f   Sound.obj
 0001:0007860c       $L8858                     0047960c f   GameStats.obj
 0001:00092511       $L133943                   00493511 f   FlashPlayer.obj
 0001:00092800       ?AtlAxWindowProc@ATL@@YGJPAUHWND__@@IIJ@Z 00493800 f   FlashPlayer.obj
 0001:00092b10       ?AtlAxWindowProc2@ATL@@YGJPAUHWND__@@IIJ@Z 00493b10 f   FlashPlayer.obj
 0001:000930c0       ?CreateNormalizedObject@ATL@@YAJPBGABU_GUID@@PAPAXAA_NPAG@Z 004940c0 f   FlashPlayer.obj
 0001:00093cd0       $L134050                   00494cd0 f i FlashPlayer.obj
 0001:000987e0       $L134505                   004997e0 f i FlashPlayer.obj
 0001:00099dea       $L134659                   0049adea f i FlashPlayer.obj
 0001:0009a102       $L134686                   0049b102 f i FlashPlayer.obj
 0001:0009b297       $L134885                   0049c297 f i FlashPlayer.obj
 0001:0009b3d7       $L134903                   0049c3d7 f i FlashPlayer.obj
 0001:0009b8cf       $L134951                   0049c8cf f i FlashPlayer.obj
 0001:0009cae7       $L135148                   0049dae7 f i FlashPlayer.obj
 0001:0009d95a       $L135274                   0049e95a f i FlashPlayer.obj
 0001:0009d9a7       $L135276                   0049e9a7 f i FlashPlayer.obj
 0001:0009de3c       $L135313                   0049ee3c f i FlashPlayer.obj
 0001:0009f829       $L135437                   004a0829 f i FlashPlayer.obj
 0001:0009fb72       $L135439                   004a0b72 f i FlashPlayer.obj
 0001:000c9570       _png_format_buffer         004ca570 f   gapidraw:pngerror.obj
 0001:000db520       _png_text_compress         004dc520 f   gapidraw:pngwutil.obj
 0001:000db7e0       _png_write_compressed_data_out 004dc7e0 f   gapidraw:pngwutil.obj
 0001:000dfa60       _deflate_stored            004e0a60 f   gapidraw:deflate.obj
 0001:000dfd00       _fill_window               004e0d00 f   gapidraw:deflate.obj
 0001:000dfea0       _deflate_fast              004e0ea0 f   gapidraw:deflate.obj
 0001:000e02c0       _longest_match             004e12c0 f   gapidraw:deflate.obj
 0001:000e0430       _deflate_slow              004e1430 f   gapidraw:deflate.obj
 0001:000e24d0       _build_tree                004e34d0 f   gapidraw:trees.obj
 0001:000e2960       _pqdownheap                004e3960 f   gapidraw:trees.obj
 0001:000e2a40       _scan_tree                 004e3a40 f   gapidraw:trees.obj
 0001:000e2b30       _send_tree                 004e3b30 f   gapidraw:trees.obj
 0001:000e30b0       _compress_block            004e40b0 f   gapidraw:trees.obj
 0001:000e34f0       _bi_windup                 004e44f0 f   gapidraw:trees.obj
 0001:000e3e30       _huft_build                004e4e30 f   gapidraw:inftrees.obj
 0001:000e4aac       ?CatchGuardHandler@@YA?AW4_EXCEPTION_DISPOSITION@@PAUEHExceptionRecord@@PAUCatchGuardRN@@PAX2@Z 004e5aac f   LIBC:trnsctrl.obj
 0001:000e4bac       ?TranslatorGuardHandler@@YA?AW4_EXCEPTION_DISPOSITION@@PAUEHExceptionRecord@@PAUTranslatorGuardRN@@PAX2@Z 004e5bac f   LIBC:trnsctrl.obj
 0001:000e4da0       $$$00001                   004e5da0 f   LIBC:exsup.obj
 0001:000e4dc0       $$$00003                   004e5dc0 f   LIBC:exsup.obj
 0001:000e4dc0       __unwind_handler           004e5dc0 f   LIBC:exsup.obj
 0001:000e4de2       $$$00005                   004e5de2 f   LIBC:exsup.obj
 0001:000e4e4a       $$$00007                   004e5e4a f   LIBC:exsup.obj
 0001:000e4e8e       $$$00011                   004e5e8e f   LIBC:exsup.obj
 0001:000e51b1       _doexit                    004e61b1 f   LIBC:crt0dat.obj
 0001:000e52c0       _$$$00001                  004e62c0 f   LIBC:strchr.obj
 0001:000e609d       _flsall                    004e709d f   LIBC:fflush.obj
 0001:000e7065       $$$00003                   004e8065 f   LIBC:exsup3.obj
 0001:000e756f       $$$00002                   004e856f f   LIBC:setjmp3.obj
 0001:000e7684       $$$00001                   004e8684 f   LIBC:longjmp.obj
 0001:000e76fd       $$$00003                   004e86fd f   LIBC:longjmp.obj
 0001:000e780f       _$$$00002                  004e880f f   LIBC:pow.obj
 0001:000e7c26       ?TypeMatch@@YAHPBU_s_HandlerType@@PBU_s_CatchableType@@PBU_s_ThrowInfo@@@Z 004e8c26 f   LIBC:frame.obj
 0001:000e7c75       ?FrameUnwindFilter@@YAHPAU_EXCEPTION_POINTERS@@@Z 004e8c75 f   LIBC:frame.obj
 0001:000e7d90       ?AdjustPointer@@YAPAXPAXABUPMD@@@Z 004e8d90 f   LIBC:frame.obj
 0001:000e7daf       ?CallCatchBlock@@YAPAXPAUEHExceptionRecord@@PAUEHRegistrationNode@@PAU_CONTEXT@@PBU_s_FuncInfo@@PAXHK@Z 004e8daf f   LIBC:frame.obj
 0001:000e7f59       ?BuildCatchObject@@YAXPAUEHExceptionRecord@@PAXPBU_s_HandlerType@@PBU_s_CatchableType@@@Z 004e8f59 f   LIBC:frame.obj
 0001:000e80d5       ?CatchIt@@YAXPAUEHExceptionRecord@@PAUEHRegistrationNode@@PAU_CONTEXT@@PAXPBU_s_FuncInfo@@PBU_s_HandlerType@@PBU_s_CatchableType@@PBU_s_TryBlockMapEntry@@H1E@Z 004e90d5 f   LIBC:frame.obj
 0001:000e813c       ?FindHandlerForForeignException@@YAXPAUEHExceptionRecord@@PAUEHRegistrationNode@@PAU_CONTEXT@@PAXPBU_s_FuncInfo@@HH1@Z 004e913c f   LIBC:frame.obj
 0001:000e81f8       ?FindHandler@@YAXPAUEHExceptionRecord@@PAUEHRegistrationNode@@PAU_CONTEXT@@PAXPBU_s_FuncInfo@@EH1@Z 004e91f8 f   LIBC:frame.obj
 0001:000e8637       __shift                    004e9637 f   LIBC:cvt.obj
 0001:000e8b1e       _write_char                004e9b1e f   LIBC:output.obj
 0001:000e8b51       _write_multi_char          004e9b51 f   LIBC:output.obj
 0001:000e8b75       _write_string              004e9b75 f   LIBC:output.obj
 0001:000ea30e       _cvtdate                   004eb30e f   LIBC:tzset.obj
 0001:000eb2f8       _CPtoLCID                  004ec2f8 f   LIBC:mbctype.obj
 0001:000eb327       _setSBCS                   004ec327 f   LIBC:mbctype.obj
 0001:000eb350       _setSBUpLow                004ec350 f   LIBC:mbctype.obj
 0001:000eb7f3       _$$$00003                  004ec7f3 f   LIBC:87disp.obj
 0001:000ebaf4       _report_failure            004ecaf4 f   LIBC:secchk.obj
 0001:000ebc40       _$$$00001                  004ecc40 f   LIBC:87triga.obj
 0001:000ec1d8       _write_char                004ed1d8 f   LIBC:woutput.obj
 0001:000ec1fd       _write_multi_char          004ed1fd f   LIBC:woutput.obj
 0001:000ec222       _write_string              004ed222 f   LIBC:woutput.obj
 0001:000ed128       _parse_cmdline             004ee128 f   LIBC:stdargv.obj
 0001:000ed4f2       _siglookup                 004ee4f2 f   LIBC:winsig.obj
 0001:000ed654       _has_osfxsr_set            004ee654 f   LIBC:cpu_disp.obj
 0001:000ee2b0       _$$$00001                  004ef2b0 f   LIBC:87tran.obj
 0001:000ef01d       __abstract_cw              004f001d f   LIBC:ieee87.obj
 0001:000ef0af       __hw_cw                    004f00af f   LIBC:ieee87.obj
 0001:000f025d       _x_ismbbtype               004f125d f   LIBC:ismbbyte.obj
 0001:000f29b2       _strncnt                   004f39b2 f   LIBC:a_cmp.obj
 0001:000f2d58       _findenv                   004f3d58 f   LIBC:setenv.obj
 0001:000f2da5       _copy_environ              004f3da5 f   LIBC:setenv.obj
 0001:000f3210       $L2205                     004f4210 f   ldwButton.obj
 0001:000f3218       $L2206                     004f4218 f   ldwButton.obj
 0001:000f3223       __ehhandler$??0ldwButton@@QAE@HPBDUldwPoint@@PAVldwScene@@_N@Z 004f4223 f   ldwButton.obj
 0001:000f322d       $L2260                     004f422d f   ldwButton.obj
 0001:000f3235       $L2261                     004f4235 f   ldwButton.obj
 0001:000f3240       __ehhandler$??0ldwButton@@QAE@HPAVldwImageStrip@@UldwPoint@@PAVldwScene@@_N@Z 004f4240 f   ldwButton.obj
 0001:000f324a       $L2279                     004f424a f   ldwButton.obj
 0001:000f3252       __ehhandler$??1ldwButton@@UAE@XZ 004f4252 f   ldwButton.obj
 0001:000f3260       $L2220                     004f4260 f   ldwButton.obj
 0001:000f3268       $L2221                     004f4268 f   ldwButton.obj
 0001:000f3273       __ehhandler$??0ldwButtonImpl@@QAE@HPBDUldwPoint@@PAVldwScene@@PAVldwHintControl@@_N@Z 004f4273 f   ldwButton.obj
 0001:000f3280       $L2247                     004f4280 f   ldwButton.obj
 0001:000f3288       __ehhandler$??1ldwButtonImpl@@UAE@XZ 004f4288 f   ldwButton.obj
 0001:000f32a0       $L2267                     004f42a0 f   ldwButton.obj
 0001:000f32a8       __ehhandler$??0ldwButtonImpl@@QAE@HPAVldwImageStrip@@UldwPoint@@PAVldwScene@@PAVldwHintControl@@_N@Z 004f42a8 f   ldwButton.obj
 0001:000f32c0       $L1361                     004f42c0 f   ldwDialog.obj
 0001:000f32c8       __ehhandler$??1ldwDialog@@UAE@XZ 004f42c8 f   ldwDialog.obj
 0001:000f32e0       $L56441                    004f42e0 f   ldwEventManager.obj
 0001:000f32eb       __ehhandler$?Get@ldwEventManager@@SAPAV1@XZ 004f42eb f   ldwEventManager.obj
 0001:000f32f5       $L56499                    004f42f5 f   ldwEventManager.obj
 0001:000f3300       __ehhandler$??0ldwEventManager@@AAE@XZ 004f4300 f   ldwEventManager.obj
 0001:000f3310       $L56462                    004f4310 f   ldwEventManager.obj
 0001:000f331b       __ehhandler$?Subscribe@ldwEventManagerImpl@@QAEXPAVldwEventHandler@@H_N@Z 004f431b f   ldwEventManager.obj
 0001:000f3330       $L875                      004f4330 f   ldwFont.obj
 0001:000f333b       __ehhandler$??0ldwFont@@QAE@XZ 004f433b f   ldwFont.obj
 0001:000f3350       $L58013                    004f4350 f   ldwFontImpl.obj
 0001:000f335e       __ehhandler$?Load@ldwFontImpl@@QAE_NPBDPAUFontTableEx@ldwFont@@H@Z 004f435e f   ldwFontImpl.obj
 0001:000f3368       $L58031                    004f4368 f   ldwFontImpl.obj
 0001:000f3373       $L58032                    004f4373 f   ldwFontImpl.obj
 0001:000f337e       __ehhandler$?GetImage@ldwFontImpl@@QAEPAVCGapiRGBASurface@@UldwColor@@@Z 004f437e f   ldwFontImpl.obj
 0001:000f3390       $L56274                    004f4390 f   ldwGame.obj
 0001:000f3398       __ehhandler$??0ldwGame@@QAE@XZ 004f4398 f   ldwGame.obj
 0001:000f33a2       $L56285                    004f43a2 f   ldwGame.obj
 0001:000f33aa       __ehhandler$??1ldwGame@@UAE@XZ 004f43aa f   ldwGame.obj
 0001:000f33c0       $L59858                    004f43c0 f   ldwGameWindow.obj
 0001:000f33cb       __ehhandler$?Create@ldwGameWindow@@SAPAV1@HHPBD_NH@Z 004f43cb f   ldwGameWindow.obj
 0001:000f33d5       $L59879                    004f43d5 f   ldwGameWindow.obj
 0001:000f33e0       __ehhandler$??0ldwGameWindow@@AAE@HHPBD_NH@Z 004f43e0 f   ldwGameWindow.obj
 0001:000f33f0       $L59889                    004f43f0 f   ldwGameWindow.obj
 0001:000f33fb       __ehhandler$??0ldwGameWindowImpl@@QAE@HHHPBD_N@Z 004f43fb f   ldwGameWindow.obj
 0001:000f3410       $L59897                    004f4410 f   ldwGameWindow.obj
 0001:000f3418       __ehhandler$??0ldwGapiApp@@QAE@ABU_GDAPPCONFIG@@@Z 004f4418 f   ldwGameWindow.obj
 0001:000f3430       $L60118                    004f4430 f   ldwGameWindow.obj
 0001:000f343b       __ehhandler$?GetSnapShot@ldwGameWindowImpl@@QAEPAVldwImage@@XZ 004f443b f   ldwGameWindow.obj
 0001:000f3450       $L60137                    004f4450 f   ldwGameWindow.obj
 0001:000f345e       __ehhandler$?SaveScreenRect@ldwGameWindowImpl@@QAE_NPBDAAUldwRect@@@Z 004f445e f   ldwGameWindow.obj
 0001:000f3470       $L57750                    004f4470 f   ldwGapiApplication.obj
 0001:000f347b       $L57751                    004f447b f   ldwGapiApplication.obj
 0001:000f3486       $L57752                    004f4486 f   ldwGapiApplication.obj
 0001:000f3491       $L57753                    004f4491 f   ldwGapiApplication.obj
 0001:000f349c       __ehhandler$??0CGapiApplication@@QAE@ABU_GDAPPCONFIG@@@Z 004f449c f   ldwGapiApplication.obj
 0001:000f34b0       $L2138                     004f44b0 f   ldwHintControl.obj
 0001:000f34b8       $L2139                     004f44b8 f   ldwHintControl.obj
 0001:000f34c3       __ehhandler$??0ldwHintControl@@QAE@H@Z 004f44c3 f   ldwHintControl.obj
 0001:000f34cd       $L2182                     004f44cd f   ldwHintControl.obj
 0001:000f34d5       $L2183                     004f44d5 f   ldwHintControl.obj
 0001:000f34e0       __ehhandler$??0ldwHintControl@@QAE@HAAUldwRect@@PAVldwScene@@PBDUldwColor@@PAVldwFont@@PAVldwBackground@@@Z 004f44e0 f   ldwHintControl.obj
 0001:000f34ea       $L2197                     004f44ea f   ldwHintControl.obj
 0001:000f34f2       $L2198                     004f44f2 f   ldwHintControl.obj
 0001:000f34fd       __ehhandler$??0ldwHintControl@@QAE@HAAUldwRect@@PAVldwScene@@PAGUldwColor@@PAVldwFont@@PAVldwBackground@@@Z 004f44fd f   ldwHintControl.obj
 0001:000f3507       $L2211                     004f4507 f   ldwHintControl.obj
 0001:000f350f       __ehhandler$??1ldwHintControl@@UAE@XZ 004f450f f   ldwHintControl.obj
 0001:000f3520       $L2149                     004f4520 f   ldwHintControl.obj
 0001:000f3528       __ehhandler$??0ldwHintControlImpl@@QAE@HUldwRect@@PAVldwScene@@@Z 004f4528 f   ldwHintControl.obj
 0001:000f3540       $L2168                     004f4540 f   ldwHintControl.obj
 0001:000f3548       __ehhandler$??1ldwHintControlImpl@@UAE@XZ 004f4548 f   ldwHintControl.obj
 0001:000f3560       $L1292                     004f4560 f   ldwImage.obj
 0001:000f356b       __ehhandler$??0ldwImage@@QAE@PBD@Z 004f456b f   ldwImage.obj
 0001:000f3575       $L1323                     004f4575 f   ldwImage.obj
 0001:000f357d       __ehhandler$??0ldwImageStrip@@QAE@PBDH@Z 004f457d f   ldwImage.obj
 0001:000f3587       $L1334                     004f4587 f   ldwImage.obj
 0001:000f358f       __ehhandler$??0ldwImageGrid@@QAE@PBDHH@Z 004f458f f   ldwImage.obj
 0001:000f3599       $L1346                     004f4599 f   ldwImage.obj
 0001:000f35a4       $L1347                     004f45a4 f   ldwImage.obj
 0001:000f35b2       __ehhandler$??0ldwImageGrid@@QAE@PBD0HHHH@Z 004f45b2 f   ldwImage.obj
 0001:000f35bc       $L1358                     004f45bc f   ldwImage.obj
 0001:000f35c4       __ehhandler$??1ldwImageGrid@@UAE@XZ 004f45c4 f   ldwImage.obj
 0001:000f35d0       $L57798                    004f45d0 f   ldwImageImpl.obj
 0001:000f35de       $L57799                    004f45de f   ldwImageImpl.obj
 0001:000f35ec       __ehhandler$??0ldwImageImpl@@QAE@PBD@Z 004f45ec f   ldwImageImpl.obj
 0001:000f3600       $L1580                     004f4600 f   ldwLog.obj
 0001:000f360b       __ehhandler$?Create@ldwLog@@SAPAV1@PBD_N@Z 004f460b f   ldwLog.obj
 0001:000f3615       $L1594                     004f4615 f   ldwLog.obj
 0001:000f3620       __ehhandler$?Get@ldwLog@@SAPAV1@XZ 004f4620 f   ldwLog.obj
 0001:000f362a       $L1627                     004f462a f   ldwLog.obj
 0001:000f3635       __ehhandler$??0ldwLog@@AAE@PBD_N@Z 004f4635 f   ldwLog.obj
 0001:000f363f       $L1638                     004f463f f   ldwLog.obj
 0001:000f364a       __ehhandler$??0ldwLog@@AAE@XZ 004f464a f   ldwLog.obj
 0001:000f3660       $L2051                     004f4660 f   ldwRadioButton.obj
 0001:000f3668       $L2052                     004f4668 f   ldwRadioButton.obj
 0001:000f3673       __ehhandler$??0ldwRadioButton@@QAE@HPAVldwImageStrip@@UldwPoint@@PAVldwScene@@PBDUldwColor@@PAVldwFont@@@Z 004f4673 f   ldwRadioButton.obj
 0001:000f367d       $L2102                     004f467d f   ldwRadioButton.obj
 0001:000f3685       __ehhandler$??1ldwRadioButton@@UAE@XZ 004f4685 f   ldwRadioButton.obj
 0001:000f3690       $L2062                     004f4690 f   ldwRadioButton.obj
 0001:000f3698       __ehhandler$??0ldwRadioButtonImpl@@QAE@PAVldwRadioButton@@HPAVldwImageStrip@@UldwPoint@@PAVldwScene@@PBDUldwColor@@PAVldwFont@@PAVldwHintControl@@@Z 004f4698 f   ldwRadioButton.obj
 0001:000f36b0       $L2086                     004f46b0 f   ldwRadioButton.obj
 0001:000f36b8       __ehhandler$??1ldwRadioButtonImpl@@UAE@XZ 004f46b8 f   ldwRadioButton.obj
 0001:000f36d0       $L1433                     004f46d0 f   ldwScene.obj
 0001:000f36d8       $L1434                     004f46d8 f   ldwScene.obj
 0001:000f36e3       __ehhandler$??0ldwScene@@QAE@XZ 004f46e3 f   ldwScene.obj
 0001:000f36ed       $L1450                     004f46ed f   ldwScene.obj
 0001:000f36f5       __ehhandler$??1ldwScene@@UAE@XZ 004f46f5 f   ldwScene.obj
 0001:000f36ff       $L1469                     004f46ff f   ldwScene.obj
 0001:000f370a       __ehhandler$?AddControl@ldwScene@@IAEXPAVldwControl@@@Z 004f470a f   ldwScene.obj
 0001:000f3720       $L2805                     004f4720 f   ldwSound.obj
 0001:000f372b       __ehhandler$??0ldwSoundFx@@QAE@PBD@Z 004f472b f   ldwSound.obj
 0001:000f3735       $L2847                     004f4735 f   ldwSound.obj
 0001:000f3740       __ehhandler$??0ldwSoundTrack@@QAE@PBD@Z 004f4740 f   ldwSound.obj
 0001:000f3750       $L2853                     004f4750 f   ldwSound.obj
 0001:000f3758       __ehhandler$??0ldwSoundTrackImpl@@QAE@PBD@Z 004f4758 f   ldwSound.obj
 0001:000f3770       $L2867                     004f4770 f   ldwSound.obj
 0001:000f3778       __ehhandler$??1ldwSoundTrackImpl@@UAE@XZ 004f4778 f   ldwSound.obj
 0001:000f3790       $L2991                     004f4790 f   ldwTextControl.obj
 0001:000f3798       $L2992                     004f4798 f   ldwTextControl.obj
 0001:000f37a3       __ehhandler$??0ldwTextControl@@QAE@PAVldwScene@@UldwPoint@@PBDHPAVldwFont@@@Z 004f47a3 f   ldwTextControl.obj
 0001:000f37ad       $L3043                     004f47ad f   ldwTextControl.obj
 0001:000f37b5       $L3044                     004f47b5 f   ldwTextControl.obj
 0001:000f37c0       __ehhandler$??0ldwTextControl@@QAE@PAVldwScene@@HUldwPoint@@PBDPAVldwFont@@H_N@Z 004f47c0 f   ldwTextControl.obj
 0001:000f37ca       $L3054                     004f47ca f   ldwTextControl.obj
 0001:000f37d2       $L3055                     004f47d2 f   ldwTextControl.obj
 0001:000f37dd       __ehhandler$??0ldwTextControl@@QAE@PAVldwScene@@UldwPoint@@PBGHPAVldwFont@@@Z 004f47dd f   ldwTextControl.obj
 0001:000f37e7       $L3074                     004f47e7 f   ldwTextControl.obj
 0001:000f37ef       $L3075                     004f47ef f   ldwTextControl.obj
 0001:000f37fa       __ehhandler$??0ldwTextControl@@QAE@PAVldwScene@@HUldwPoint@@PBGPAVldwFont@@H_N@Z 004f47fa f   ldwTextControl.obj
 0001:000f3804       $L3085                     004f4804 f   ldwTextControl.obj
 0001:000f380c       __ehhandler$??1ldwTextControl@@UAE@XZ 004f480c f   ldwTextControl.obj
 0001:000f3820       $L3002                     004f4820 f   ldwTextControl.obj
 0001:000f3820       $L3061                     004f4820 f   ldwTextControl.obj
 0001:000f3820       $L3030                     004f4820 f   ldwTextControl.obj
 0001:000f3828       __ehhandler$??1ldwTextControlImpl@@UAE@XZ 004f4828 f   ldwTextControl.obj
 0001:000f3828       __ehhandler$??0ldwTextControlImpl@@QAE@HUldwPoint@@PAVldwScene@@PBGPAVldwFont@@H_NPAVldwHintControl@@@Z 004f4828 f   ldwTextControl.obj
 0001:000f3828       __ehhandler$??0ldwTextControlImpl@@QAE@HUldwPoint@@PAVldwScene@@PBDPAVldwFont@@H_NPAVldwHintControl@@@Z 004f4828 f   ldwTextControl.obj
 0001:000f3840       $L1562                     004f4840 f   ldwTiledDialog.obj
 0001:000f3848       __ehhandler$??0ldwTiledDialog@@QAE@_N@Z 004f4848 f   ldwTiledDialog.obj
 0001:000f3852       $L1578                     004f4852 f   ldwTiledDialog.obj
 0001:000f385a       __ehhandler$??1ldwTiledDialog@@UAE@XZ 004f485a f   ldwTiledDialog.obj
 0001:000f3864       $L1588                     004f4864 f   ldwTiledDialog.obj
 0001:000f386f       __ehhandler$?SetTiling@ldwTiledDialog@@IAEXPAVldwImageGrid@@HH@Z 004f486f f   ldwTiledDialog.obj
 0001:000f3880       $L58693                    004f4880 f   unzip.obj
 0001:000f388b       __ehhandler$?OpenZipInternal@@YAPAUHZIP__@@PAXIKPBD@Z 004f488b f   unzip.obj
 0001:000f38a0       $L10602                    004f48a0 f   VillagerManager.obj
 0001:000f38ae       $L10603                    004f48ae f   VillagerManager.obj
 0001:000f38bc       __ehhandler$?DrawVillager@CVillagerManager@@QAEXH@Z 004f48bc f   VillagerManager.obj
 0001:000f38d0       $L9858                     004f48d0 f   CollectionScene.obj
 0001:000f38db       $L9859                     004f48db f   CollectionScene.obj
 0001:000f38e6       $L9860                     004f48e6 f   CollectionScene.obj
 0001:000f38f1       $L9861                     004f48f1 f   CollectionScene.obj
 0001:000f38fc       $L9862                     004f48fc f   CollectionScene.obj
 0001:000f3907       $L9863                     004f4907 f   CollectionScene.obj
 0001:000f3912       $L9864                     004f4912 f   CollectionScene.obj
 0001:000f391d       $L9865                     004f491d f   CollectionScene.obj
 0001:000f392b       $L9866                     004f492b f   CollectionScene.obj
 0001:000f3939       $L9867                     004f4939 f   CollectionScene.obj
 0001:000f3947       $L9868                     004f4947 f   CollectionScene.obj
 0001:000f3955       $L9869                     004f4955 f   CollectionScene.obj
 0001:000f3963       $L9870                     004f4963 f   CollectionScene.obj
 0001:000f3971       $L9871                     004f4971 f   CollectionScene.obj
 0001:000f397f       __ehhandler$??0CCollectionScene@@AAE@XZ 004f497f f   CollectionScene.obj
 0001:000f3989       $L9903                     004f4989 f   CollectionScene.obj
 0001:000f3991       __ehhandler$??1CCollectionScene@@EAE@XZ 004f4991 f   CollectionScene.obj
 0001:000f399b       $L9913                     004f499b f   CollectionScene.obj
 0001:000f39a6       __ehhandler$?Get@CCollectionScene@@SAPAV1@XZ 004f49a6 f   CollectionScene.obj
 0001:000f39b0       $L9923                     004f49b0 f   CollectionScene.obj
 0001:000f39bb       __ehhandler$?Ref@CCollectionScene@@SAAAV1@XZ 004f49bb f   CollectionScene.obj
 0001:000f39d0       $L9832                     004f49d0 f   ProgressScene.obj
 0001:000f39db       $L9833                     004f49db f   ProgressScene.obj
 0001:000f39e9       $L9834                     004f49e9 f   ProgressScene.obj
 0001:000f39f7       $L9835                     004f49f7 f   ProgressScene.obj
 0001:000f3a05       $L9836                     004f4a05 f   ProgressScene.obj
 0001:000f3a13       $L9837                     004f4a13 f   ProgressScene.obj
 0001:000f3a21       $L9838                     004f4a21 f   ProgressScene.obj
 0001:000f3a2f       $L9839                     004f4a2f f   ProgressScene.obj
 0001:000f3a3d       $L9840                     004f4a3d f   ProgressScene.obj
 0001:000f3a4b       $L9841                     004f4a4b f   ProgressScene.obj
 0001:000f3a59       $L9842                     004f4a59 f   ProgressScene.obj
 0001:000f3a67       $L9843                     004f4a67 f   ProgressScene.obj
 0001:000f3a75       __ehhandler$??0CProgressScene@@AAE@XZ 004f4a75 f   ProgressScene.obj
 0001:000f3a7f       $L9891                     004f4a7f f   ProgressScene.obj
 0001:000f3a87       __ehhandler$??1CProgressScene@@EAE@XZ 004f4a87 f   ProgressScene.obj
 0001:000f3a91       $L9901                     004f4a91 f   ProgressScene.obj
 0001:000f3a9c       __ehhandler$?Get@CProgressScene@@SAPAV1@XZ 004f4a9c f   ProgressScene.obj
 0001:000f3aa6       $L9911                     004f4aa6 f   ProgressScene.obj
 0001:000f3ab1       __ehhandler$?Ref@CProgressScene@@SAAAV1@XZ 004f4ab1 f   ProgressScene.obj
 0001:000f3abb       $L9935                     004f4abb f   ProgressScene.obj
 0001:000f3ac9       __ehhandler$?RefreshTab@CProgressScene@@AAEXXZ 004f4ac9 f   ProgressScene.obj
 0001:000f3ad3       $L9943                     004f4ad3 f   ProgressScene.obj
 0001:000f3ade       $L9944                     004f4ade f   ProgressScene.obj
 0001:000f3ae9       __ehhandler$?HandleMouse@CProgressScene@@UAE_NHUldwPoint@@@Z 004f4ae9 f   ProgressScene.obj
 0001:000f3b00       $L9415                     004f4b00 f   StoryScene.obj
 0001:000f3b08       $L9416                     004f4b08 f   StoryScene.obj
 0001:000f3b13       $L9417                     004f4b13 f   StoryScene.obj
 0001:000f3b1e       $L9418                     004f4b1e f   StoryScene.obj
 0001:000f3b29       $L9419                     004f4b29 f   StoryScene.obj
 0001:000f3b34       __ehhandler$??0CStoryScene@@AAE@XZ 004f4b34 f   StoryScene.obj
 0001:000f3b3e       $L9443                     004f4b3e f   StoryScene.obj
 0001:000f3b46       __ehhandler$??1CStoryScene@@EAE@XZ 004f4b46 f   StoryScene.obj
 0001:000f3b50       $L9453                     004f4b50 f   StoryScene.obj
 0001:000f3b5b       __ehhandler$?Get@CStoryScene@@SAPAV1@XZ 004f4b5b f   StoryScene.obj
 0001:000f3b65       $L9463                     004f4b65 f   StoryScene.obj
 0001:000f3b70       __ehhandler$?Ref@CStoryScene@@SAAAV1@XZ 004f4b70 f   StoryScene.obj
 0001:000f3b7a       $L9477                     004f4b7a f   StoryScene.obj
 0001:000f3b82       __ehhandler$?HandleMessage@CStoryScene@@UAE_NHJ@Z 004f4b82 f   StoryScene.obj
 0001:000f3b90       $L9766                     004f4b90 f   TechScene.obj
 0001:000f3b9b       $L9767                     004f4b9b f   TechScene.obj
 0001:000f3ba6       $L9768                     004f4ba6 f   TechScene.obj
 0001:000f3bb1       $L9769                     004f4bb1 f   TechScene.obj
 0001:000f3bbc       $L9770                     004f4bbc f   TechScene.obj
 0001:000f3bc7       $L9771                     004f4bc7 f   TechScene.obj
 0001:000f3bd2       $L9772                     004f4bd2 f   TechScene.obj
 0001:000f3be0       $L9773                     004f4be0 f   TechScene.obj
 0001:000f3bee       $L9774                     004f4bee f   TechScene.obj
 0001:000f3bfc       $L9775                     004f4bfc f   TechScene.obj
 0001:000f3c0a       $L9776                     004f4c0a f   TechScene.obj
 0001:000f3c18       __ehhandler$??0CTechScene@@AAE@XZ 004f4c18 f   TechScene.obj
 0001:000f3c22       $L9805                     004f4c22 f   TechScene.obj
 0001:000f3c2a       __ehhandler$??1CTechScene@@EAE@XZ 004f4c2a f   TechScene.obj
 0001:000f3c34       $L9815                     004f4c34 f   TechScene.obj
 0001:000f3c3f       __ehhandler$?Get@CTechScene@@SAPAV1@XZ 004f4c3f f   TechScene.obj
 0001:000f3c49       $L9825                     004f4c49 f   TechScene.obj
 0001:000f3c54       __ehhandler$?Ref@CTechScene@@SAAAV1@XZ 004f4c54 f   TechScene.obj
 0001:000f3c5e       $L9851                     004f4c5e f   TechScene.obj
 0001:000f3c69       __ehhandler$?ShowTechInfo@CTechScene@@AAEXW4ETech@@@Z 004f4c69 f   TechScene.obj
 0001:000f3c73       $L9864                     004f4c73 f   TechScene.obj
 0001:000f3c7b       __ehhandler$?HandleMessage@CTechScene@@UAE_NHJ@Z 004f4c7b f   TechScene.obj
 0001:000f3c90       $L9120                     004f4c90 f   theHelpScene.obj
 0001:000f3c98       $L9121                     004f4c98 f   theHelpScene.obj
 0001:000f3ca3       $L9122                     004f4ca3 f   theHelpScene.obj
 0001:000f3cae       $L9123                     004f4cae f   theHelpScene.obj
 0001:000f3cb9       $L9124                     004f4cb9 f   theHelpScene.obj
 0001:000f3cc4       $L9125                     004f4cc4 f   theHelpScene.obj
 0001:000f3ccf       __ehhandler$??0theHelpScene@@QAE@XZ 004f4ccf f   theHelpScene.obj
 0001:000f3cd9       $L9141                     004f4cd9 f   theHelpScene.obj
 0001:000f3ce1       __ehhandler$??1theHelpScene@@UAE@XZ 004f4ce1 f   theHelpScene.obj
 0001:000f3cf0       $L9165                     004f4cf0 f   theLoadingScene.obj
 0001:000f3cf8       $L9166                     004f4cf8 f   theLoadingScene.obj
 0001:000f3d03       $L9167                     004f4d03 f   theLoadingScene.obj
 0001:000f3d0e       __ehhandler$??0theLoadingScene@@QAE@XZ 004f4d0e f   theLoadingScene.obj
 0001:000f3d18       $L9179                     004f4d18 f   theLoadingScene.obj
 0001:000f3d20       __ehhandler$??1theLoadingScene@@UAE@XZ 004f4d20 f   theLoadingScene.obj
 0001:000f3d30       $L13801                    004f4d30 f   theMainScene.obj
 0001:000f3d3b       $L13802                    004f4d3b f   theMainScene.obj
 0001:000f3d46       $L13803                    004f4d46 f   theMainScene.obj
 0001:000f3d51       $L13804                    004f4d51 f   theMainScene.obj
 0001:000f3d5c       $L13805                    004f4d5c f   theMainScene.obj
 0001:000f3d67       $L13806                    004f4d67 f   theMainScene.obj
 0001:000f3d75       $L13807                    004f4d75 f   theMainScene.obj
 0001:000f3d83       $L13808                    004f4d83 f   theMainScene.obj
 0001:000f3d91       $L13809                    004f4d91 f   theMainScene.obj
 0001:000f3d9f       $L13810                    004f4d9f f   theMainScene.obj
 0001:000f3dad       $L13811                    004f4dad f   theMainScene.obj
 0001:000f3dbb       $L13812                    004f4dbb f   theMainScene.obj
 0001:000f3dc9       $L13813                    004f4dc9 f   theMainScene.obj
 0001:000f3dd7       $L13814                    004f4dd7 f   theMainScene.obj
 0001:000f3de5       $L13815                    004f4de5 f   theMainScene.obj
 0001:000f3df3       $L13816                    004f4df3 f   theMainScene.obj
 0001:000f3e01       $L13817                    004f4e01 f   theMainScene.obj
 0001:000f3e0f       $L13818                    004f4e0f f   theMainScene.obj
 0001:000f3e1d       $L13819                    004f4e1d f   theMainScene.obj
 0001:000f3e2b       $L13820                    004f4e2b f   theMainScene.obj
 0001:000f3e39       $L13821                    004f4e39 f   theMainScene.obj
 0001:000f3e47       __ehhandler$??0theMainScene@@AAE@XZ 004f4e47 f   theMainScene.obj
 0001:000f3e51       $L13841                    004f4e51 f   theMainScene.obj
 0001:000f3e59       __ehhandler$??1theMainScene@@EAE@XZ 004f4e59 f   theMainScene.obj
 0001:000f3e63       $L13852                    004f4e63 f   theMainScene.obj
 0001:000f3e6e       __ehhandler$?Get@theMainScene@@SAPAV1@XZ 004f4e6e f   theMainScene.obj
 0001:000f3e78       $L13862                    004f4e78 f   theMainScene.obj
 0001:000f3e83       __ehhandler$?Ref@theMainScene@@SAAAV1@XZ 004f4e83 f   theMainScene.obj
 0001:000f3e8d       $L13887                    004f4e8d f   theMainScene.obj
 0001:000f3e95       $L13888                    004f4e95 f   theMainScene.obj
 0001:000f3ea0       __ehhandler$?UpdateScene@theMainScene@@MAEXXZ 004f4ea0 f   theMainScene.obj
 0001:000f3eaa       $L13940                    004f4eaa f   theMainScene.obj
 0001:000f3eb5       __ehhandler$?HandleMouseDown@theMainScene@@QAE?B_NUldwPoint@@@Z 004f4eb5 f   theMainScene.obj
 0001:000f3ebf       $L14034                    004f4ebf f   theMainScene.obj
 0001:000f3eca       __ehhandler$?MapClickFeedback@theMainScene@@QAEXUldwPoint@@@Z 004f4eca f   theMainScene.obj
 0001:000f3ee0       $L10353                    004f4ee0 f   theMenuScene.obj
 0001:000f3eeb       $L10354                    004f4eeb f   theMenuScene.obj
 0001:000f3ef9       $L10355                    004f4ef9 f   theMenuScene.obj
 0001:000f3f07       $L10356                    004f4f07 f   theMenuScene.obj
 0001:000f3f15       $L10357                    004f4f15 f   theMenuScene.obj
 0001:000f3f23       $L10358                    004f4f23 f   theMenuScene.obj
 0001:000f3f31       $L10359                    004f4f31 f   theMenuScene.obj
 0001:000f3f3f       $L10360                    004f4f3f f   theMenuScene.obj
 0001:000f3f4d       $L10361                    004f4f4d f   theMenuScene.obj
 0001:000f3f5b       $L10362                    004f4f5b f   theMenuScene.obj
 0001:000f3f69       $L10363                    004f4f69 f   theMenuScene.obj
 0001:000f3f77       $L10364                    004f4f77 f   theMenuScene.obj
 0001:000f3f85       __ehhandler$??0theMenuScene@@QAE@XZ 004f4f85 f   theMenuScene.obj
 0001:000f3f8f       $L10388                    004f4f8f f   theMenuScene.obj
 0001:000f3f97       __ehhandler$??1theMenuScene@@UAE@XZ 004f4f97 f   theMenuScene.obj
 0001:000f3fa1       $L10421                    004f4fa1 f   theMenuScene.obj
 0001:000f3fa9       $L10422                    004f4fa9 f   theMenuScene.obj
 0001:000f3fb4       $L10423                    004f4fb4 f   theMenuScene.obj
 0001:000f3fbf       $L10424                    004f4fbf f   theMenuScene.obj
 0001:000f3fca       __ehhandler$?HandleMessage@theMenuScene@@UAE_NHJ@Z 004f4fca f   theMenuScene.obj
 0001:000f3fe0       $L9981                     004f4fe0 f   theOverviewScene.obj
 0001:000f3feb       $L9982                     004f4feb f   theOverviewScene.obj
 0001:000f3ff6       $L9983                     004f4ff6 f   theOverviewScene.obj
 0001:000f4001       $L9984                     004f5001 f   theOverviewScene.obj
 0001:000f400c       $L9985                     004f500c f   theOverviewScene.obj
 0001:000f4017       $L9986                     004f5017 f   theOverviewScene.obj
 0001:000f4022       $L9987                     004f5022 f   theOverviewScene.obj
 0001:000f402d       $L9988                     004f502d f   theOverviewScene.obj
 0001:000f403b       $L9989                     004f503b f   theOverviewScene.obj
 0001:000f4049       $L9990                     004f5049 f   theOverviewScene.obj
 0001:000f4057       __ehhandler$??0theOverviewScene@@QAE@XZ 004f5057 f   theOverviewScene.obj
 0001:000f4061       $L10006                    004f5061 f   theOverviewScene.obj
 0001:000f4069       __ehhandler$??1theOverviewScene@@UAE@XZ 004f5069 f   theOverviewScene.obj
 0001:000f4080       $L27430                    004f5080 f   theSplashScene.obj
 0001:000f4088       $L27431                    004f5088 f   theSplashScene.obj
 0001:000f4093       $L27432                    004f5093 f   theSplashScene.obj
 0001:000f409e       $L27433                    004f509e f   theSplashScene.obj
 0001:000f40a9       $L27434                    004f50a9 f   theSplashScene.obj
 0001:000f40b4       __ehhandler$??0theSplashScene@@QAE@XZ 004f50b4 f   theSplashScene.obj
 0001:000f40be       $L27449                    004f50be f   theSplashScene.obj
 0001:000f40c6       __ehhandler$??1theSplashScene@@UAE@XZ 004f50c6 f   theSplashScene.obj
 0001:000f40d0       $L10039                    004f50d0 f   theVillagerScene.obj
 0001:000f40db       $L10040                    004f50db f   theVillagerScene.obj
 0001:000f40e6       $L10041                    004f50e6 f   theVillagerScene.obj
 0001:000f40f1       $L10042                    004f50f1 f   theVillagerScene.obj
 0001:000f40fc       $L10043                    004f50fc f   theVillagerScene.obj
 0001:000f4107       $L10044                    004f5107 f   theVillagerScene.obj
 0001:000f4112       $L10045                    004f5112 f   theVillagerScene.obj
 0001:000f411d       $L10046                    004f511d f   theVillagerScene.obj
 0001:000f4128       $L10047                    004f5128 f   theVillagerScene.obj
 0001:000f4136       $L10048                    004f5136 f   theVillagerScene.obj
 0001:000f4144       $L10049                    004f5144 f   theVillagerScene.obj
 0001:000f4152       $L10050                    004f5152 f   theVillagerScene.obj
 0001:000f4160       $L10051                    004f5160 f   theVillagerScene.obj
 0001:000f416e       $L10052                    004f516e f   theVillagerScene.obj
 0001:000f417c       $L10053                    004f517c f   theVillagerScene.obj
 0001:000f418a       $L10054                    004f518a f   theVillagerScene.obj
 0001:000f4198       $L10055                    004f5198 f   theVillagerScene.obj
 0001:000f41a6       $L10056                    004f51a6 f   theVillagerScene.obj
 0001:000f41b4       $L10057                    004f51b4 f   theVillagerScene.obj
 0001:000f41c2       $L10058                    004f51c2 f   theVillagerScene.obj
 0001:000f41d0       $L10059                    004f51d0 f   theVillagerScene.obj
 0001:000f41de       $L10060                    004f51de f   theVillagerScene.obj
 0001:000f41ec       $L10061                    004f51ec f   theVillagerScene.obj
 0001:000f41fa       $L10062                    004f51fa f   theVillagerScene.obj
 0001:000f4208       $L10063                    004f5208 f   theVillagerScene.obj
 0001:000f4216       $L10064                    004f5216 f   theVillagerScene.obj
 0001:000f4224       $L10065                    004f5224 f   theVillagerScene.obj
 0001:000f4232       $L10066                    004f5232 f   theVillagerScene.obj
 0001:000f4240       $L10067                    004f5240 f   theVillagerScene.obj
 0001:000f424e       $L10068                    004f524e f   theVillagerScene.obj
 0001:000f425c       __ehhandler$??0theVillagerScene@@QAE@XZ 004f525c f   theVillagerScene.obj
 0001:000f4266       $L10082                    004f5266 f   theVillagerScene.obj
 0001:000f426e       __ehhandler$??1theVillagerScene@@UAE@XZ 004f526e f   theVillagerScene.obj
 0001:000f4280       $L13459                    004f5280 f   IslandEvents.obj
 0001:000f428b       $L13460                    004f528b f   IslandEvents.obj
 0001:000f4296       $L13461                    004f5296 f   IslandEvents.obj
 0001:000f42a4       $L13462                    004f52a4 f   IslandEvents.obj
 0001:000f42b2       __ehhandler$??0CIslandEventDialog@@QAE@PAVCIslandEvent@@@Z 004f52b2 f   IslandEvents.obj
 0001:000f42bc       $L13497                    004f52bc f   IslandEvents.obj
 0001:000f42c4       __ehhandler$??1CIslandEventDialog@@UAE@XZ 004f52c4 f   IslandEvents.obj
 0001:000f42ce       $L13521                    004f52ce f   IslandEvents.obj
 0001:000f42d9       __ehhandler$?Get@CIslandEvents@@SAPAV1@XZ 004f52d9 f   IslandEvents.obj
 0001:000f42e3       $L13766                    004f52e3 f   IslandEvents.obj
 0001:000f42ee       $L13767                    004f52ee f   IslandEvents.obj
 0001:000f42f9       $L13768                    004f52f9 f   IslandEvents.obj
 0001:000f4304       $L13769                    004f5304 f   IslandEvents.obj
 0001:000f430f       $L13770                    004f530f f   IslandEvents.obj
 0001:000f431a       $L13771                    004f531a f   IslandEvents.obj
 0001:000f4325       $L13772                    004f5325 f   IslandEvents.obj
 0001:000f4330       $L13773                    004f5330 f   IslandEvents.obj
 0001:000f433b       $L13774                    004f533b f   IslandEvents.obj
 0001:000f4346       $L13775                    004f5346 f   IslandEvents.obj
 0001:000f4351       $L13776                    004f5351 f   IslandEvents.obj
 0001:000f435c       $L13777                    004f535c f   IslandEvents.obj
 0001:000f4367       $L13778                    004f5367 f   IslandEvents.obj
 0001:000f4372       $L13779                    004f5372 f   IslandEvents.obj
 0001:000f437d       $L13780                    004f537d f   IslandEvents.obj
 0001:000f438b       $L13781                    004f538b f   IslandEvents.obj
 0001:000f4399       $L13782                    004f5399 f   IslandEvents.obj
 0001:000f43a7       $L13783                    004f53a7 f   IslandEvents.obj
 0001:000f43b5       $L13784                    004f53b5 f   IslandEvents.obj
 0001:000f43c3       $L13785                    004f53c3 f   IslandEvents.obj
 0001:000f43d1       $L13786                    004f53d1 f   IslandEvents.obj
 0001:000f43df       $L13787                    004f53df f   IslandEvents.obj
 0001:000f43ed       $L13788                    004f53ed f   IslandEvents.obj
 0001:000f43fb       $L13789                    004f53fb f   IslandEvents.obj
 0001:000f4409       $L13790                    004f5409 f   IslandEvents.obj
 0001:000f4417       $L13791                    004f5417 f   IslandEvents.obj
 0001:000f4425       $L13792                    004f5425 f   IslandEvents.obj
 0001:000f4433       $L13793                    004f5433 f   IslandEvents.obj
 0001:000f4441       $L13794                    004f5441 f   IslandEvents.obj
 0001:000f444f       $L13795                    004f544f f   IslandEvents.obj
 0001:000f445d       $L13796                    004f545d f   IslandEvents.obj
 0001:000f446b       $L13797                    004f546b f   IslandEvents.obj
 0001:000f4479       $L13798                    004f5479 f   IslandEvents.obj
 0001:000f4487       $L13799                    004f5487 f   IslandEvents.obj
 0001:000f4495       $L13800                    004f5495 f   IslandEvents.obj
 0001:000f44a3       $L13801                    004f54a3 f   IslandEvents.obj
 0001:000f44b1       $L13802                    004f54b1 f   IslandEvents.obj
 0001:000f44bf       $L13803                    004f54bf f   IslandEvents.obj
 0001:000f44cd       $L13804                    004f54cd f   IslandEvents.obj
 0001:000f44db       $L13805                    004f54db f   IslandEvents.obj
 0001:000f44e9       $L13806                    004f54e9 f   IslandEvents.obj
 0001:000f44f7       $L13807                    004f54f7 f   IslandEvents.obj
 0001:000f4505       $L13808                    004f5505 f   IslandEvents.obj
 0001:000f4513       $L13809                    004f5513 f   IslandEvents.obj
 0001:000f4521       $L13810                    004f5521 f   IslandEvents.obj
 0001:000f452f       $L13811                    004f552f f   IslandEvents.obj
 0001:000f453d       $L13812                    004f553d f   IslandEvents.obj
 0001:000f454b       $L13813                    004f554b f   IslandEvents.obj
 0001:000f4559       $L13814                    004f5559 f   IslandEvents.obj
 0001:000f4567       $L13815                    004f5567 f   IslandEvents.obj
 0001:000f4575       $L13816                    004f5575 f   IslandEvents.obj
 0001:000f4583       $L13817                    004f5583 f   IslandEvents.obj
 0001:000f4591       $L13818                    004f5591 f   IslandEvents.obj
 0001:000f459f       $L13819                    004f559f f   IslandEvents.obj
 0001:000f45ad       $L13820                    004f55ad f   IslandEvents.obj
 0001:000f45bb       $L13821                    004f55bb f   IslandEvents.obj
 0001:000f45c9       $L13822                    004f55c9 f   IslandEvents.obj
 0001:000f45d7       $L13823                    004f55d7 f   IslandEvents.obj
 0001:000f45e5       __ehhandler$??0CIslandEvents@@AAE@XZ 004f55e5 f   IslandEvents.obj
 0001:000f45ef       $L14554                    004f55ef f   IslandEvents.obj
 0001:000f45fa       __ehhandler$?FireEvent@CIslandEvents@@QAE_NPAVldwScene@@@Z 004f55fa f   IslandEvents.obj
 0001:000f4604       $L14563                    004f5604 f   IslandEvents.obj
 0001:000f460f       __ehhandler$?ForceEvent@CIslandEvents@@QAE_NPAVldwScene@@W4IslandEventId@@@Z 004f560f f   IslandEvents.obj
 0001:000f4620       $L8461                     004f5620 f   RosterOfDeadDialog.obj
 0001:000f462b       $L8462                     004f562b f   RosterOfDeadDialog.obj
 0001:000f4639       $L8463                     004f5639 f   RosterOfDeadDialog.obj
 0001:000f4647       $L8464                     004f5647 f   RosterOfDeadDialog.obj
 0001:000f4655       $L8465                     004f5655 f   RosterOfDeadDialog.obj
 0001:000f4663       $L8466                     004f5663 f   RosterOfDeadDialog.obj
 0001:000f4671       $L8467                     004f5671 f   RosterOfDeadDialog.obj
 0001:000f467f       $L8468                     004f567f f   RosterOfDeadDialog.obj
 0001:000f468d       $L8469                     004f568d f   RosterOfDeadDialog.obj
 0001:000f469b       $L8470                     004f569b f   RosterOfDeadDialog.obj
 0001:000f46a9       $L8471                     004f56a9 f   RosterOfDeadDialog.obj
 0001:000f46b7       $L8472                     004f56b7 f   RosterOfDeadDialog.obj
 0001:000f46c5       $L8473                     004f56c5 f   RosterOfDeadDialog.obj
 0001:000f46d3       $L8474                     004f56d3 f   RosterOfDeadDialog.obj
 0001:000f46e1       __ehhandler$??0CRosterOfDeadDialog@@QAE@XZ 004f56e1 f   RosterOfDeadDialog.obj
 0001:000f46f0       $L9293                     004f56f0 f   theChangePlayerDlg.obj
 0001:000f46fb       $L9294                     004f56fb f   theChangePlayerDlg.obj
 0001:000f4706       $L9295                     004f5706 f   theChangePlayerDlg.obj
 0001:000f4711       $L9296                     004f5711 f   theChangePlayerDlg.obj
 0001:000f471c       $L9297                     004f571c f   theChangePlayerDlg.obj
 0001:000f472a       $L9298                     004f572a f   theChangePlayerDlg.obj
 0001:000f4738       $L9299                     004f5738 f   theChangePlayerDlg.obj
 0001:000f4746       $L9300                     004f5746 f   theChangePlayerDlg.obj
 0001:000f4754       $L9301                     004f5754 f   theChangePlayerDlg.obj
 0001:000f4762       __ehhandler$??0theChangePlayerDlg@@QAE@H@Z 004f5762 f   theChangePlayerDlg.obj
 0001:000f476c       $L9317                     004f576c f   theChangePlayerDlg.obj
 0001:000f4774       __ehhandler$??1theChangePlayerDlg@@UAE@XZ 004f5774 f   theChangePlayerDlg.obj
 0001:000f477e       $L9329                     004f577e f   theChangePlayerDlg.obj
 0001:000f4786       __ehhandler$?HandleMessage@theChangePlayerDlg@@UAE_NHJ@Z 004f5786 f   theChangePlayerDlg.obj
 0001:000f4790       $L9066                     004f5790 f   theCreateNickNameDlg.obj
 0001:000f479b       $L9067                     004f579b f   theCreateNickNameDlg.obj
 0001:000f47a6       $L9068                     004f57a6 f   theCreateNickNameDlg.obj
 0001:000f47b1       $L9069                     004f57b1 f   theCreateNickNameDlg.obj
 0001:000f47bc       $L9070                     004f57bc f   theCreateNickNameDlg.obj
 0001:000f47c7       __ehhandler$??0theCreateNickNameDlg@@QAE@H@Z 004f57c7 f   theCreateNickNameDlg.obj
 0001:000f47e0       $L9528                     004f57e0 f   theFernsaceDialog.obj
 0001:000f47e8       $L9529                     004f57e8 f   theFernsaceDialog.obj
 0001:000f47f3       $L9530                     004f57f3 f   theFernsaceDialog.obj
 0001:000f47fe       $L9531                     004f57fe f   theFernsaceDialog.obj
 0001:000f4809       __ehhandler$??0theFernsaceDialog@@QAE@H@Z 004f5809 f   theFernsaceDialog.obj
 0001:000f4813       $L9551                     004f5813 f   theFernsaceDialog.obj
 0001:000f481b       __ehhandler$??1theFernsaceDialog@@UAE@XZ 004f581b f   theFernsaceDialog.obj
 0001:000f4830       $L9078                     004f5830 f   theMessageBoxDlg.obj
 0001:000f4838       __ehhandler$??0theMessageBoxDlg@@QAE@W4StringId@@HW4EMessageBoxType@@@Z 004f5838 f   theMessageBoxDlg.obj
 0001:000f4842       $L9089                     004f5842 f   theMessageBoxDlg.obj
 0001:000f484a       __ehhandler$??0theMessageBoxDlg@@QAE@W4StringId@@H_N@Z 004f584a f   theMessageBoxDlg.obj
 0001:000f4854       $L9095                     004f5854 f   theMessageBoxDlg.obj
 0001:000f485c       __ehhandler$??0theMessageBoxDlg@@QAE@PBDH_N@Z 004f585c f   theMessageBoxDlg.obj
 0001:000f4866       $L9122                     004f5866 f   theMessageBoxDlg.obj
 0001:000f4871       $L9123                     004f5871 f   theMessageBoxDlg.obj
 0001:000f487c       $L9124                     004f587c f   theMessageBoxDlg.obj
 0001:000f4887       __ehhandler$?Init@theMessageBoxDlg@@IAEXPBDHW4EMessageBoxType@@@Z 004f5887 f   theMessageBoxDlg.obj
 0001:000f48a0       $L9349                     004f58a0 f   theOptionsDialog.obj
 0001:000f48a8       $L9350                     004f58a8 f   theOptionsDialog.obj
 0001:000f48b3       $L9351                     004f58b3 f   theOptionsDialog.obj
 0001:000f48be       $L9352                     004f58be f   theOptionsDialog.obj
 0001:000f48c9       $L9353                     004f58c9 f   theOptionsDialog.obj
 0001:000f48d4       $L9354                     004f58d4 f   theOptionsDialog.obj
 0001:000f48df       __ehhandler$??0theOptionsDialog@@QAE@PADW4DialogColorEnum@@@Z 004f58df f   theOptionsDialog.obj
 0001:000f48f0       $L9911                     004f58f0 f   theTipDialog.obj
 0001:000f48f8       __ehhandler$??0theTipDialog@@QAE@W4StringId@@W4ArrowDirection@@HH_N@Z 004f58f8 f   theTipDialog.obj
 0001:000f4902       $L9925                     004f5902 f   theTipDialog.obj
 0001:000f490a       __ehhandler$??0theTipDialog@@QAE@PBD@Z 004f590a f   theTipDialog.obj
 0001:000f4914       $L9938                     004f5914 f   theTipDialog.obj
 0001:000f491f       __ehhandler$?Init@theTipDialog@@IAEXPBDW4ArrowDirection@@HH_N@Z 004f591f f   theTipDialog.obj
 0001:000f4929       $L9945                     004f5929 f   theTipDialog.obj
 0001:000f4931       __ehhandler$??1theTipDialog@@UAE@XZ 004f5931 f   theTipDialog.obj
 0001:000f4940       $L9465                     004f5940 f   theTombStoneDialog.obj
 0001:000f494b       $L9466                     004f594b f   theTombStoneDialog.obj
 0001:000f4959       $L9467                     004f5959 f   theTombStoneDialog.obj
 0001:000f4967       $L9468                     004f5967 f   theTombStoneDialog.obj
 0001:000f4975       $L9469                     004f5975 f   theTombStoneDialog.obj
 0001:000f4983       $L9470                     004f5983 f   theTombStoneDialog.obj
 0001:000f4991       $L9471                     004f5991 f   theTombStoneDialog.obj
 0001:000f499f       $L9472                     004f599f f   theTombStoneDialog.obj
 0001:000f49ad       $L9473                     004f59ad f   theTombStoneDialog.obj
 0001:000f49bb       $L9474                     004f59bb f   theTombStoneDialog.obj
 0001:000f49c9       __ehhandler$??0theTombStoneDialog@@QAE@W4TSDialogColorEnum@@PBUSGrave@CGraveyard@@@Z 004f59c9 f   theTombStoneDialog.obj
 0001:000f49e0       $L1574                     004f59e0 f   WorldMap.obj
 0001:000f49eb       __ehhandler$?LoadAssets@CWorldMap@@QAEXXZ 004f59eb f   WorldMap.obj
 0001:000f4a00       $L9177                     004f5a00 f   Sound.obj
 0001:000f4a0b       __ehhandler$?LoadAssets@CSound@@QAEXXZ 004f5a0b f   Sound.obj
 0001:000f4a15       $L9201                     004f5a15 f   Sound.obj
 0001:000f4a20       __ehhandler$?Play@CSound@@QAEXW4ESound@@_NM@Z 004f5a20 f   Sound.obj
 0001:000f4a30       $L8807                     004f5a30 f   SoundTrack.obj
 0001:000f4a3b       __ehhandler$?LoadAssets@CSoundTrack@@QAEXXZ 004f5a3b f   SoundTrack.obj
 0001:000f4a50       $L715                      004f5a50 f   ldwarialbold.obj
 0001:000f4a58       __ehhandler$??0ldwarialbold@@QAE@XZ 004f5a58 f   ldwarialbold.obj
 0001:000f4a70       $L715                      004f5a70 f   ldwBurweed27.obj
 0001:000f4a78       __ehhandler$??0ldwBurweed27@@QAE@XZ 004f5a78 f   ldwBurweed27.obj
 0001:000f4a90       $L22246                    004f5a90 f   highscore.obj
 0001:000f4a9b       __ehhandler$??0CHighScore@@QAE@XZ 004f5a9b f   highscore.obj
 0001:000f4ab0       $L22268                    004f5ab0 f   highscore.obj
 0001:000f4ab8       __ehhandler$??1CHighScoreImpl@@QAE@XZ 004f5ab8 f   highscore.obj
 0001:000f4ad0       $L22291                    004f5ad0 f   highscore.obj
 0001:000f4ade       __ehhandler$?Parse@CHighScoreImpl@@QAEXPBD@Z 004f5ade f   highscore.obj
 0001:000f4af0       $L10275                    004f5af0 f   HummingbirdClass.obj
 0001:000f4afb       __ehhandler$?Get@theHummingbirdClass@@SAPAV1@XZ 004f5afb f   HummingbirdClass.obj
 0001:000f4b10       $L10112                    004f5b10 f   theButterflyClass.obj
 0001:000f4b1b       __ehhandler$?Get@theButterflyClass@@SAPAV1@XZ 004f5b1b f   theButterflyClass.obj
 0001:000f4b30       $L1452                     004f5b30 f   Distributor.obj
 0001:000f4b3b       $L1453                     004f5b3b f   Distributor.obj
 0001:000f4b46       __ehhandler$?LoadAssets@CDistributor@@QAEXXZ 004f5b46 f   Distributor.obj
 0001:000f4b50       $L8859                     004f5b50 f   GameStats.obj
 0001:000f4b5b       $L8860                     004f5b5b f   GameStats.obj
 0001:000f4b66       __ehhandler$?Refresh@CGameStats@@QAE?B_NXZ 004f5b66 f   GameStats.obj
 0001:000f4b70       $L65420                    004f5b70 f   theGame.obj
 0001:000f4b7b       $L65421                    004f5b7b f   theGame.obj
 0001:000f4b86       $L65422                    004f5b86 f   theGame.obj
 0001:000f4b91       __ehhandler$?Init@theGame@@UAE_NXZ 004f5b91 f   theGame.obj
 0001:000f4b9b       $L65489                    004f5b9b f   theGame.obj
 0001:000f4ba6       $L65490                    004f5ba6 f   theGame.obj
 0001:000f4bb1       $L65491                    004f5bb1 f   theGame.obj
 0001:000f4bbc       $L65492                    004f5bbc f   theGame.obj
 0001:000f4bc7       __ehhandler$?GameUpdate@theGame@@UAEXXZ 004f5bc7 f   theGame.obj
 0001:000f4be0       $L9887                     004f5be0 f   theGameState.obj
 0001:000f4beb       __ehhandler$?Get@theGameState@@SAPAV1@XZ 004f5beb f   theGameState.obj
 0001:000f4bf5       $L9933                     004f5bf5 f   theGameState.obj
 0001:000f4bfd       __ehhandler$??0theGameState@@IAE@XZ 004f5bfd f   theGameState.obj
 0001:000f4c10       $L8799                     004f5c10 f   theRealtimeManager.obj
 0001:000f4c1b       __ehhandler$?Get@theRealtimeManager@@SAPAV1@XZ 004f5c1b f   theRealtimeManager.obj
 0001:000f4c30       $L8806                     004f5c30 f   theDealerSay.obj
 0001:000f4c3b       __ehhandler$?Get@theDealerSay@@SAPAV1@XZ 004f5c3b f   theDealerSay.obj
 0001:000f4c45       $L8826                     004f5c45 f   theDealerSay.obj
 0001:000f4c50       __ehhandler$??0theDealerSay@@IAE@XZ 004f5c50 f   theDealerSay.obj
 0001:000f4c60       $L8836                     004f5c60 f   theDealerSay.obj
 0001:000f4c6b       __ehhandler$??0theDealerSayImpl@@QAE@XZ 004f5c6b f   theDealerSay.obj
 0001:000f4c80       $L9402                     004f5c80 f   theGraphicsManager.obj
 0001:000f4c8b       __ehhandler$?Get@theGraphicsManager@@SAPAV1@XZ 004f5c8b f   theGraphicsManager.obj
 0001:000f4c95       $L9422                     004f5c95 f   theGraphicsManager.obj
 0001:000f4ca0       __ehhandler$??0theGraphicsManager@@IAE@XZ 004f5ca0 f   theGraphicsManager.obj
 0001:000f4cb0       $L9453                     004f5cb0 f   theGraphicsManager.obj
 0001:000f4cb0       $L9466                     004f5cb0 f   theGraphicsManager.obj
 0001:000f4cbb       __ehhandler$?GetImage@theGraphicsManagerImpl@@QAEPAVldwImage@@H@Z 004f5cbb f   theGraphicsManager.obj
 0001:000f4cbb       __ehhandler$?GetImageStrip@theGraphicsManagerImpl@@QAEPAVldwImageStrip@@H@Z 004f5cbb f   theGraphicsManager.obj
 0001:000f4cd0       $L9482                     004f5cd0 f   theGraphicsManager.obj
 0001:000f4cdb       $L9483                     004f5cdb f   theGraphicsManager.obj
 0001:000f4ce6       __ehhandler$?GetImageGrid@theGraphicsManagerImpl@@QAEPAVldwImageGrid@@H@Z 004f5ce6 f   theGraphicsManager.obj
 0001:000f4cf0       $L9339                     004f5cf0 f   thePrizeMsgAssembler.obj
 0001:000f4cfb       __ehhandler$?Get@thePrizeMsgAssembler@@SAPAV1@XZ 004f5cfb f   thePrizeMsgAssembler.obj
 0001:000f4d10       $L9045                     004f5d10 f   theSlicedVariableMeter.obj
 0001:000f4d1b       __ehhandler$?Get@theSlicedVariableMeter@@SAPAV1@XZ 004f5d1b f   theSlicedVariableMeter.obj
 0001:000f4d30       $L5331                     004f5d30 f   theStringManager.obj
 0001:000f4d3b       __ehhandler$?Get@theStringManager@@SAPAV1@XZ 004f5d3b f   theStringManager.obj
 0001:000f4d45       $L5351                     004f5d45 f   theStringManager.obj
 0001:000f4d50       __ehhandler$??0theStringManager@@IAE@XZ 004f5d50 f   theStringManager.obj
 0001:000f4d5a       $L5376                     004f5d5a f   theStringManager.obj
 0001:000f4d65       __ehhandler$?LoadFonts@theStringManager@@QAEXXZ 004f5d65 f   theStringManager.obj
 0001:000f4d70       $L1614                     004f5d70 f   theVariableMeter.obj
 0001:000f4d7b       __ehhandler$?Get@theVariableMeter@@SAPAV1@XZ 004f5d7b f   theVariableMeter.obj
 0001:000f4d90       $L8215                     004f5d90 f   AlchemyLab.obj
 0001:000f4d9e       __ehhandler$?Reset@CAlchemyLab@@UAEXXZ 004f5d9e f   AlchemyLab.obj
 0001:000f4da8       $L8237                     004f5da8 f   AlchemyLab.obj
 0001:000f4db6       __ehhandler$?Drop@CAlchemyLab@@UAEXAAVCVillager@@W4ECarrying@@@Z 004f5db6 f   AlchemyLab.obj
 0001:000f4dc0       $L8074                     004f5dc0 f   AlchemyTable.obj
 0001:000f4dce       __ehhandler$?Draw@CAlchemyTable@@UBEXH@Z 004f5dce f   AlchemyTable.obj
 0001:000f4de0       $L7820                     004f5de0 f   Aromatherapy.obj
 0001:000f4dee       __ehhandler$?BurnerPos@CAromatherapy@@QBE?BUldwPoint@@H@Z 004f5dee f   Aromatherapy.obj
 0001:000f4e00       $L8461                     004f5e00 f   DoorKey.obj
 0001:000f4e0b       $L8462                     004f5e0b f   DoorKey.obj
 0001:000f4e16       __ehhandler$?LoadAssets@CDoorKey@@UAEXXZ 004f5e16 f   DoorKey.obj
 0001:000f4e20       $L10070                    004f5e20 f   Orchard.obj
 0001:000f4e2e       $L10071                    004f5e2e f   Orchard.obj
 0001:000f4e3c       $L10072                    004f5e3c f   Orchard.obj
 0001:000f4e4a       $L10073                    004f5e4a f   Orchard.obj
 0001:000f4e58       __ehhandler$?Draw@COrchard@@UBEXH@Z 004f5e58 f   Orchard.obj
 0001:000f4e70       $L7958                     004f5e70 f   RosterOfTheDead.obj
 0001:000f4e7e       __ehhandler$?Draw@CRosterOfTheDead@@UBEXH@Z 004f5e7e f   RosterOfTheDead.obj
 0001:000f4e90       $L8015                     004f5e90 f   Ruins.obj
 0001:000f4e9b       __ehhandler$?LoadAssets@CRuins@@UAEXXZ 004f5e9b f   Ruins.obj
 0001:000f4ea5       $L8034                     004f5ea5 f   Ruins.obj
 0001:000f4eb3       __ehhandler$?Draw@CRuins@@UBEXH@Z 004f5eb3 f   Ruins.obj
 0001:000f4ec0       $L48596                    004f5ec0 f   MoviePlayer.obj
 0001:000f4ecb       __ehhandler$??0CMoviePlayer@@QAE@XZ 004f5ecb f   MoviePlayer.obj
 0001:000f4ee0       $L133930                   004f5ee0 f   FlashPlayer.obj
 0001:000f4ee8       __ehhandler$??1CFlashPlayer@@UAE@XZ 004f5ee8 f   FlashPlayer.obj
 0001:000f4ef2       __ehhandler$?Load@CFlashPlayer@@UAE?B_NPBDHH@Z 004f5ef2 f   FlashPlayer.obj
 0001:000f4efc       $L133967                   004f5efc f   FlashPlayer.obj
 0001:000f4f04       $L133968                   004f5f04 f   FlashPlayer.obj
 0001:000f4f0c       __ehhandler$?AtlAxWindowProc@ATL@@YGJPAUHWND__@@IIJ@Z 004f5f0c f   FlashPlayer.obj
 0001:000f4f16       $L133985                   004f5f16 f   FlashPlayer.obj
 0001:000f4f1e       $L133986                   004f5f1e f   FlashPlayer.obj
 0001:000f4f26       $L133987                   004f5f26 f   FlashPlayer.obj
 0001:000f4f2e       __ehhandler$?AtlAxWindowProc2@ATL@@YGJPAUHWND__@@IIJ@Z 004f5f2e f   FlashPlayer.obj
 0001:000f4f38       $L134337                   004f5f38 f   FlashPlayer.obj
 0001:000f4f40       __ehhandler$?CreateNormalizedObject@ATL@@YAJPBGABU_GUID@@PAPAXAA_NPAG@Z 004f5f40 f   FlashPlayer.obj
 0001:000f4f50       $L133997                   004f5f50 f   FlashPlayer.obj
 0001:000f4f58       __ehhandler$?ParseInitData@_DialogSplitHelper@ATL@@SAJPAUIStream@@PAPAG@Z 004f5f58 f   FlashPlayer.obj
 0001:000f4f70       $L134051                   004f5f70 f   FlashPlayer.obj
 0001:000f4f7b       __ehhandler$?CreateInstance@?$CComCreator@V?$CComPolyObject@VCAxHostWindow@ATL@@@ATL@@@ATL@@SGJPAXABU_GUID@@PAPAX@Z 004f5f7b f   FlashPlayer.obj
 0001:000f4f90       $L134114                   004f5f90 f   FlashPlayer.obj
 0001:000f4f90       $L134079                   004f5f90 f   FlashPlayer.obj
 0001:000f4f9b       __ehhandler$??1?$CComPolyObject@VCAxHostWindow@ATL@@@ATL@@UAE@XZ 004f5f9b f   FlashPlayer.obj
 0001:000f4f9b       __ehhandler$??0?$CComPolyObject@VCAxHostWindow@ATL@@@ATL@@QAE@PAX@Z 004f5f9b f   FlashPlayer.obj
 0001:000f4fb0       $L134126                   004f5fb0 f   FlashPlayer.obj
 0001:000f4fb8       __ehhandler$??1CAxHostWindow@ATL@@UAE@XZ 004f5fb8 f   FlashPlayer.obj
 0001:000f4fd0       $L134262                   004f5fd0 f   FlashPlayer.obj
 0001:000f4fd0       $L134283                   004f5fd0 f   FlashPlayer.obj
 0001:000f4fd0       $L134181                   004f5fd0 f   FlashPlayer.obj
 0001:000f4fd0       $L134254                   004f5fd0 f   FlashPlayer.obj
 0001:000f4fd0       $L134300                   004f5fd0 f   FlashPlayer.obj
 0001:000f4fd8       __ehhandler$?CreateControl@CAxHostWindow@ATL@@UAGJPBGPAUHWND__@@PAUIStream@@@Z 004f5fd8 f   FlashPlayer.obj
 0001:000f4fd8       __ehhandler$?CreateControlLic@CAxHostWindow@ATL@@UAGJPBGPAUHWND__@@PAUIStream@@PAG@Z 004f5fd8 f   FlashPlayer.obj
 0001:000f4fd8       __ehhandler$?OnMouseActivate@CAxHostWindow@ATL@@QAEJIIJAAH@Z 004f5fd8 f   FlashPlayer.obj
 0001:000f4fd8       __ehhandler$?OnSetFocus@CAxHostWindow@ATL@@QAEJIIJAAH@Z 004f5fd8 f   FlashPlayer.obj
 0001:000f4fd8       __ehhandler$?ReleaseAll@CAxHostWindow@ATL@@QAEXXZ 004f5fd8 f   FlashPlayer.obj
 0001:000f4ff0       $L134243                   004f5ff0 f   FlashPlayer.obj
 0001:000f4ff8       __ehhandler$?OnForwardMsg@CAxHostWindow@ATL@@QAEJIIJAAH@Z 004f5ff8 f   FlashPlayer.obj
 0001:000f5010       $L134308                   004f6010 f   FlashPlayer.obj
 0001:000f5018       $L134309                   004f6018 f   FlashPlayer.obj
 0001:000f5020       $L134310                   004f6020 f   FlashPlayer.obj
 0001:000f5028       $L134311                   004f6028 f   FlashPlayer.obj
 0001:000f5030       $L134312                   004f6030 f   FlashPlayer.obj
 0001:000f5038       $L134313                   004f6038 f   FlashPlayer.obj
 0001:000f5040       __ehhandler$?CreateControlLicEx@CAxHostWindow@ATL@@UAGJPBGPAUHWND__@@PAUIStream@@PAPAUIUnknown@@ABU_GUID@@PAU5@PAG@Z 004f6040 f   FlashPlayer.obj
 0001:000f5050       $L134356                   004f6050 f   FlashPlayer.obj
 0001:000f5058       __ehhandler$?TranslateAcceleratorA@CAxHostWindow@ATL@@UAGJPAUtagMSG@@PBU_GUID@@K@Z 004f6058 f   FlashPlayer.obj
 0001:000f5070       $L134370                   004f6070 f   FlashPlayer.obj
 0001:000f5070       $L134391                   004f6070 f   FlashPlayer.obj
 0001:000f5078       __ehhandler$?FilterDataObject@CAxHostWindow@ATL@@UAGJPAUIDataObject@@PAPAU3@@Z 004f6078 f   FlashPlayer.obj
 0001:000f5078       __ehhandler$?GetDropTarget@CAxHostWindow@ATL@@UAGJPAUIDropTarget@@PAPAU3@@Z 004f6078 f   FlashPlayer.obj
 0001:000f5090       $L134381                   004f6090 f   FlashPlayer.obj
 0001:000f5098       $L134382                   004f6098 f   FlashPlayer.obj
 0001:000f50a0       __ehhandler$?TranslateUrl@CAxHostWindow@ATL@@UAGJKPAGPAPAG@Z 004f60a0 f   FlashPlayer.obj
 0001:000f50b0       $L134401                   004f60b0 f   FlashPlayer.obj
 0001:000f50b8       __ehhandler$?FireAmbientPropertyChange@CAxHostWindow@ATL@@QAEJJ@Z 004f60b8 f   FlashPlayer.obj
 0001:000f50d0       __ehhandler$?EnumObjects@CAxHostWindow@ATL@@UAGJKPAPAUIEnumUnknown@@@Z 004f60d0 f   FlashPlayer.obj
 0001:000f50e0       $L134518                   004f60e0 f   FlashPlayer.obj
 0001:000f50e8       $L134519                   004f60e8 f   FlashPlayer.obj
 0001:000f50f0       $L134520                   004f60f0 f   FlashPlayer.obj
 0001:000f50f8       $L134521                   004f60f8 f   FlashPlayer.obj
 0001:000f5100       $L134522                   004f6100 f   FlashPlayer.obj
 0001:000f5108       $L134523                   004f6108 f   FlashPlayer.obj
 0001:000f5110       $L134524                   004f6110 f   FlashPlayer.obj
 0001:000f5118       __ehhandler$?ActivateAx@CAxHostWindow@ATL@@QAEJPAUIUnknown@@_NPAUIStream@@@Z 004f6118 f   FlashPlayer.obj
 0001:000f5130       $L134623                   004f6130 f   FlashPlayer.obj
 0001:000f5138       $L134624                   004f6138 f   FlashPlayer.obj
 0001:000f5143       $L134625                   004f6143 f   FlashPlayer.obj
 0001:000f514e       $L134626                   004f614e f   FlashPlayer.obj
 0001:000f5159       $L134627                   004f6159 f   FlashPlayer.obj
 0001:000f5164       __ehhandler$?GetTI@CComTypeInfoHolder@ATL@@QAEJK@Z 004f6164 f   FlashPlayer.obj
 0001:000f5170       $L134660                   004f6170 f   FlashPlayer.obj
 0001:000f517b       $L134661                   004f617b f   FlashPlayer.obj
 0001:000f5183       __ehhandler$?LoadNameCache@CComTypeInfoHolder@ATL@@QAEJPAUITypeInfo@@@Z 004f6183 f   FlashPlayer.obj
 0001:000f5190       $L134687                   004f6190 f   FlashPlayer.obj
 0001:000f5198       __ehhandler$?AtlModuleAddTermFunc@ATL@@YGJPAU_ATL_MODULE70@1@P6GXK@ZK@Z 004f6198 f   FlashPlayer.obj
 0001:000f51b0       $L134780                   004f61b0 f   FlashPlayer.obj
 0001:000f51b8       __ehhandler$??0?$CComEnum@UIEnumUnknown@@$1?_GUID_00000100_0000_0000_c000_000000000046@@3U__s_GUID@@BPAUIUnknown@@V?$_CopyInterface@UIUnknown@@@ATL@@VCComMultiThreadModel@6@@ATL@@QAE@XZ 004f61b8 f   FlashPlayer.obj
 0001:000f51d0       __ehhandler$?CreateInstance@?$CComObject@VCAxFrameWindow@ATL@@@ATL@@SGJPAPAV12@@Z 004f61d0 f   FlashPlayer.obj
 0001:000f51e0       __ehhandler$?CreateInstance@?$CComObject@VCAxUIWindow@ATL@@@ATL@@SGJPAPAV12@@Z 004f61e0 f   FlashPlayer.obj
 0001:000f51f0       $L134915                   004f61f0 f   FlashPlayer.obj
 0001:000f51fb       __ehhandler$??1?$CComEnumImpl@UIEnumUnknown@@$1?_GUID_00000100_0000_0000_c000_000000000046@@3U__s_GUID@@BPAUIUnknown@@V?$_CopyInterface@UIUnknown@@@ATL@@@ATL@@UAE@XZ 004f61fb f   FlashPlayer.obj
 0001:000f5210       $L134938                   004f6210 f   FlashPlayer.obj
 0001:000f5229       __ehhandler$?Clone@?$CComEnumImpl@UIEnumUnknown@@$1?_GUID_00000100_0000_0000_c000_000000000046@@3U__s_GUID@@BPAUIUnknown@@V?$_CopyInterface@UIUnknown@@@ATL@@@ATL@@UAGJPAPAUIEnumUnknown@@@Z 004f6229 f   FlashPlayer.obj
 0001:000f5240       __ehhandler$?Init@?$CComEnumImpl@UIEnumUnknown@@$1?_GUID_00000100_0000_0000_c000_000000000046@@3U__s_GUID@@BPAUIUnknown@@V?$_CopyInterface@UIUnknown@@@ATL@@@ATL@@QAEJPAPAUIUnknown@@0PAU3@W4CComEnumFlags@2@@Z 004f6240 f   FlashPlayer.obj
 0001:000f5250       $L135083                   004f6250 f   FlashPlayer.obj
 0001:000f5250       $L134964                   004f6250 f   FlashPlayer.obj
 0001:000f525b       __ehhandler$??0CAxUIWindow@ATL@@QAE@XZ 004f625b f   FlashPlayer.obj
 0001:000f525b       __ehhandler$??0CAxFrameWindow@ATL@@QAE@XZ 004f625b f   FlashPlayer.obj
 0001:000f5270       $L135121                   004f6270 f   FlashPlayer.obj
 0001:000f5270       $L135017                   004f6270 f   FlashPlayer.obj
 0001:000f5297       __ehhandler$??1CAxUIWindow@ATL@@UAE@XZ 004f6297 f   FlashPlayer.obj
 0001:000f5297       __ehhandler$??1CAxFrameWindow@ATL@@UAE@XZ 004f6297 f   FlashPlayer.obj
 0001:000f52b0       $L135051                   004f62b0 f   FlashPlayer.obj
 0001:000f52b8       __ehhandler$??$AtlModuleRegisterWndClassInfoT@VAtlModuleRegisterWndClassInfoParamA@ATL@@@ATL@@YAGPAU_ATL_BASE_MODULE70@0@PAU_ATL_WIN_MODULE70@0@PAU_ATL_WNDCLASSINFOA@0@PAP6GJPAUHWND__@@IIJ@ZVAtlModuleRegisterWndClassInfoParamA@0@@Z 004f62b8 f   FlashPlayer.obj
 0001:000f52d0       $L135071                   004f62d0 f   FlashPlayer.obj
 0001:000f52e9       __ehhandler$?InternalSetAtIndex@?$CSimpleArray@GV?$CSimpleArrayEqualHelper@G@ATL@@@ATL@@QAEXHABG@Z 004f62e9 f   FlashPlayer.obj
 0001:000f5300       __ehhandler$?CreateInstance@?$CComObject@V?$CComEnum@UIEnumUnknown@@$1?_GUID_00000100_0000_0000_c000_000000000046@@3U__s_GUID@@BPAUIUnknown@@V?$_CopyInterface@UIUnknown@@@ATL@@VCComMultiThreadModel@6@@ATL@@@ATL@@SGJPAPAV12@@Z 004f6300 f   FlashPlayer.obj
 0001:000f5310       $L135231                   004f6310 f   FlashPlayer.obj
 0001:000f531b       $L135232                   004f631b f   FlashPlayer.obj
 0001:000f5326       __ehhandler$??1CRegObject@ATL@@UAE@XZ 004f6326 f   FlashPlayer.obj
 0001:000f5330       $L135240                   004f6330 f   FlashPlayer.obj
 0001:000f5338       __ehhandler$??1CExpansionVector@ATL@@QAE@XZ 004f6338 f   FlashPlayer.obj
 0001:000f5350       __ehhandler$?Add@CExpansionVector@ATL@@QAEHPBDPBG@Z 004f6350 f   FlashPlayer.obj
 0001:000f5360       $L135314                   004f6360 f   FlashPlayer.obj
 0001:000f5368       $L135315                   004f6368 f   FlashPlayer.obj
 0001:000f5373       __ehhandler$?RegisterFromResource@CRegObject@ATL@@IAEJPBGPBD1H@Z 004f6373 f   FlashPlayer.obj
 0001:000f5380       $L135336                   004f6380 f   FlashPlayer.obj
 0001:000f5380       $L135298                   004f6380 f   FlashPlayer.obj
 0001:000f5388       __ehhandler$?ResourceUnregisterSz@CRegObject@ATL@@QAGJPBG00@Z 004f6388 f   FlashPlayer.obj
 0001:000f5388       __ehhandler$?ResourceRegisterSz@CRegObject@ATL@@QAGJPBG00@Z 004f6388 f   FlashPlayer.obj
 0001:000f53a0       $L135360                   004f63a0 f   FlashPlayer.obj
 0001:000f53a8       __ehhandler$?PreProcessBuffer@CRegParser@ATL@@QAEJPADPAPAD@Z 004f63a8 f   FlashPlayer.obj
 0001:000f53c0       $L135396                   004f63c0 f   FlashPlayer.obj
 0001:000f53c8       $L135397                   004f63c8 f   FlashPlayer.obj
 0001:000f53d3       $L135398                   004f63d3 f   FlashPlayer.obj
 0001:000f53de       __ehhandler$?RegisterSubkeys@CRegParser@ATL@@IAEJPADPAUHKEY__@@HH@Z 004f63de f   FlashPlayer.obj
 0001:000f53f0       $L135440                   004f63f0 f   FlashPlayer.obj
 0001:000f53fb       $L135441                   004f63fb f   FlashPlayer.obj
 0001:000f5406       $L135442                   004f6406 f   FlashPlayer.obj
 0001:000f5411       __ehhandler$?AddValue@CRegParser@ATL@@IAEJAAVCRegKey@2@PBDPAD@Z 004f6411 f   FlashPlayer.obj
 0001:000f5420       $L135465                   004f6420 f   FlashPlayer.obj
 0001:000f542b       __ehhandler$??0CRegObject@ATL@@QAE@XZ 004f642b f   FlashPlayer.obj
 0001:000f5440       $L135511                   004f6440 f   FlashPlayer.obj
 0001:000f5440       $L135377                   004f6440 f   FlashPlayer.obj
 0001:000f5440       $L135497                   004f6440 f   FlashPlayer.obj
 0001:000f5440       $L135261                   004f6440 f   FlashPlayer.obj
 0001:000f5448       __ehhandler$?ResourceRegister@CRegObject@ATL@@QAGJPBGI0@Z 004f6448 f   FlashPlayer.obj
 0001:000f5448       __ehhandler$?ResourceUnregister@CRegObject@ATL@@QAGJPBGI0@Z 004f6448 f   FlashPlayer.obj
 0001:000f5448       __ehhandler$?AddString@CParseBuffer@CRegParser@ATL@@QAEHPBG@Z 004f6448 f   FlashPlayer.obj
 0001:000f5448       __ehhandler$?AddReplacement@CRegObject@ATL@@UAGJPBG0@Z 004f6448 f   FlashPlayer.obj
 0001:000f5460       $L135557                   004f6460 f   FlashPlayer.obj
 0001:000f5479       $L135558                   004f6479 f   FlashPlayer.obj
 0001:000f5493       __ehhandler$?InternalSetAtIndex@?$CSimpleMap@PADPAGVCExpansionVectorEqualHelper@ATL@@@ATL@@QAEXHABQADABQAG@Z 004f6493 f   FlashPlayer.obj
 0001:000f54a0       $L135583                   004f64a0 f   FlashPlayer.obj
 0001:000f54a8       __ehhandler$??1CAtlWinModule@ATL@@QAE@XZ 004f64a8 f   FlashPlayer.obj
 0001:000f54c0       $L9018                     004f64c0 f   TutorialTip.obj
 0001:000f54cb       __ehhandler$?Display@CTutorialTip@@QAEHW4StringId@@PAVldwScene@@@Z 004f64cb f   TutorialTip.obj
 0001:000f57f0       _$E1                       004f67f0 f   ldwButton.obj
 0001:000f5810       _$E3                       004f6810 f   ldwButton.obj
 0001:000f5820       _$E5                       004f6820 f   ldwButton.obj
 0001:000f5850       _$E7                       004f6850 f   ldwButton.obj
 0001:000f5880       _$E9                       004f6880 f   ldwButton.obj
 0001:000f58a0       _$E11                      004f68a0 f   ldwButton.obj
 0001:000f58c0       _$E13                      004f68c0 f   ldwButton.obj
 0001:000f58e0       _$E15                      004f68e0 f   ldwButton.obj
 0001:000f5900       _$E1                       004f6900 f   ldwDialog.obj
 0001:000f5920       _$E3                       004f6920 f   ldwDialog.obj
 0001:000f5930       _$E5                       004f6930 f   ldwDialog.obj
 0001:000f5960       _$E7                       004f6960 f   ldwDialog.obj
 0001:000f5990       _$E9                       004f6990 f   ldwDialog.obj
 0001:000f59b0       _$E11                      004f69b0 f   ldwDialog.obj
 0001:000f59d0       _$E13                      004f69d0 f   ldwDialog.obj
 0001:000f59f0       _$E1                       004f69f0 f   ldwEventManager.obj
 0001:000f5a10       _$E3                       004f6a10 f   ldwEventManager.obj
 0001:000f5a20       _$E5                       004f6a20 f   ldwEventManager.obj
 0001:000f5a50       _$E7                       004f6a50 f   ldwEventManager.obj
 0001:000f5a80       _$E9                       004f6a80 f   ldwEventManager.obj
 0001:000f5aa0       _$E11                      004f6aa0 f   ldwEventManager.obj
 0001:000f5ac0       _$E13                      004f6ac0 f   ldwEventManager.obj
 0001:000f5ae0       _$E1                       004f6ae0 f   ldwFont.obj
 0001:000f5b00       _$E3                       004f6b00 f   ldwFont.obj
 0001:000f5b10       _$E5                       004f6b10 f   ldwFont.obj
 0001:000f5b40       _$E7                       004f6b40 f   ldwFont.obj
 0001:000f5b70       _$E9                       004f6b70 f   ldwFont.obj
 0001:000f5b90       _$E11                      004f6b90 f   ldwFont.obj
 0001:000f5bb0       _$E13                      004f6bb0 f   ldwFont.obj
 0001:000f5bd0       _$E1                       004f6bd0 f   ldwFontImpl.obj
 0001:000f5bf0       _$E3                       004f6bf0 f   ldwFontImpl.obj
 0001:000f5c00       _$E5                       004f6c00 f   ldwFontImpl.obj
 0001:000f5c30       _$E7                       004f6c30 f   ldwFontImpl.obj
 0001:000f5c60       _$E9                       004f6c60 f   ldwFontImpl.obj
 0001:000f5c80       _$E11                      004f6c80 f   ldwFontImpl.obj
 0001:000f5ca0       _$E13                      004f6ca0 f   ldwFontImpl.obj
 0001:000f5cc0       _$E1                       004f6cc0 f   ldwGame.obj
 0001:000f5ce0       _$E3                       004f6ce0 f   ldwGame.obj
 0001:000f5cf0       _$E5                       004f6cf0 f   ldwGame.obj
 0001:000f5d20       _$E7                       004f6d20 f   ldwGame.obj
 0001:000f5d50       _$E9                       004f6d50 f   ldwGame.obj
 0001:000f5d70       _$E11                      004f6d70 f   ldwGame.obj
 0001:000f5d90       _$E13                      004f6d90 f   ldwGame.obj
 0001:000f5db0       _$E1                       004f6db0 f   ldwGameState.obj
 0001:000f5dd0       _$E3                       004f6dd0 f   ldwGameState.obj
 0001:000f5de0       _$E5                       004f6de0 f   ldwGameState.obj
 0001:000f5e10       _$E7                       004f6e10 f   ldwGameState.obj
 0001:000f5e40       _$E9                       004f6e40 f   ldwGameState.obj
 0001:000f5e60       _$E11                      004f6e60 f   ldwGameState.obj
 0001:000f5e80       _$E13                      004f6e80 f   ldwGameState.obj
 0001:000f5ea0       _$E1                       004f6ea0 f   ldwGameWindow.obj
 0001:000f5ec0       _$E3                       004f6ec0 f   ldwGameWindow.obj
 0001:000f5ed0       _$E5                       004f6ed0 f   ldwGameWindow.obj
 0001:000f5f00       _$E7                       004f6f00 f   ldwGameWindow.obj
 0001:000f5f30       _$E9                       004f6f30 f   ldwGameWindow.obj
 0001:000f5f50       _$E11                      004f6f50 f   ldwGameWindow.obj
 0001:000f5f70       _$E13                      004f6f70 f   ldwGameWindow.obj
 0001:000f5f90       _$E1                       004f6f90 f   ldwGapiApplication.obj
 0001:000f5fb0       _$E3                       004f6fb0 f   ldwGapiApplication.obj
 0001:000f5fc0       _$E5                       004f6fc0 f   ldwGapiApplication.obj
 0001:000f5ff0       _$E7                       004f6ff0 f   ldwGapiApplication.obj
 0001:000f6020       _$E9                       004f7020 f   ldwGapiApplication.obj
 0001:000f6040       _$E11                      004f7040 f   ldwGapiApplication.obj
 0001:000f6060       _$E13                      004f7060 f   ldwGapiApplication.obj
 0001:000f6080       _$E1                       004f7080 f   ldwHintControl.obj
 0001:000f60a0       _$E3                       004f70a0 f   ldwHintControl.obj
 0001:000f60b0       _$E5                       004f70b0 f   ldwHintControl.obj
 0001:000f60e0       _$E7                       004f70e0 f   ldwHintControl.obj
 0001:000f6110       _$E9                       004f7110 f   ldwHintControl.obj
 0001:000f6130       _$E11                      004f7130 f   ldwHintControl.obj
 0001:000f6150       _$E13                      004f7150 f   ldwHintControl.obj
 0001:000f6170       _$E15                      004f7170 f   ldwHintControl.obj
 0001:000f6190       _$E17                      004f7190 f   ldwHintControl.obj
 0001:000f61c0       _$E19                      004f71c0 f   ldwHintControl.obj
 0001:000f61d0       _$E1                       004f71d0 f   ldwImage.obj
 0001:000f61f0       _$E3                       004f71f0 f   ldwImage.obj
 0001:000f6200       _$E5                       004f7200 f   ldwImage.obj
 0001:000f6230       _$E7                       004f7230 f   ldwImage.obj
 0001:000f6260       _$E9                       004f7260 f   ldwImage.obj
 0001:000f6280       _$E11                      004f7280 f   ldwImage.obj
 0001:000f62a0       _$E13                      004f72a0 f   ldwImage.obj
 0001:000f62c0       _$E1                       004f72c0 f   ldwImageImpl.obj
 0001:000f62e0       _$E3                       004f72e0 f   ldwImageImpl.obj
 0001:000f62f0       _$E5                       004f72f0 f   ldwImageImpl.obj
 0001:000f6320       _$E7                       004f7320 f   ldwImageImpl.obj
 0001:000f6350       _$E9                       004f7350 f   ldwImageImpl.obj
 0001:000f6370       _$E11                      004f7370 f   ldwImageImpl.obj
 0001:000f6390       _$E13                      004f7390 f   ldwImageImpl.obj
 0001:000f63b0       _$E1                       004f73b0 f   ldwLog.obj
 0001:000f63d0       _$E3                       004f73d0 f   ldwLog.obj
 0001:000f63e0       _$E5                       004f73e0 f   ldwLog.obj
 0001:000f6410       _$E7                       004f7410 f   ldwLog.obj
 0001:000f6440       _$E9                       004f7440 f   ldwLog.obj
 0001:000f6460       _$E11                      004f7460 f   ldwLog.obj
 0001:000f6480       _$E13                      004f7480 f   ldwLog.obj
 0001:000f64a0       _$E1                       004f74a0 f   ldwRadioButton.obj
 0001:000f64c0       _$E3                       004f74c0 f   ldwRadioButton.obj
 0001:000f64d0       _$E5                       004f74d0 f   ldwRadioButton.obj
 0001:000f6500       _$E7                       004f7500 f   ldwRadioButton.obj
 0001:000f6530       _$E9                       004f7530 f   ldwRadioButton.obj
 0001:000f6550       _$E11                      004f7550 f   ldwRadioButton.obj
 0001:000f6570       _$E13                      004f7570 f   ldwRadioButton.obj
 0001:000f6590       _$E1                       004f7590 f   ldwScene.obj
 0001:000f65b0       _$E3                       004f75b0 f   ldwScene.obj
 0001:000f65c0       _$E5                       004f75c0 f   ldwScene.obj
 0001:000f65f0       _$E7                       004f75f0 f   ldwScene.obj
 0001:000f6620       _$E9                       004f7620 f   ldwScene.obj
 0001:000f6640       _$E11                      004f7640 f   ldwScene.obj
 0001:000f6660       _$E13                      004f7660 f   ldwScene.obj
 0001:000f6680       _$E1                       004f7680 f   ldwSound.obj
 0001:000f66a0       _$E3                       004f76a0 f   ldwSound.obj
 0001:000f66b0       _$E5                       004f76b0 f   ldwSound.obj
 0001:000f66e0       _$E7                       004f76e0 f   ldwSound.obj
 0001:000f6710       _$E9                       004f7710 f   ldwSound.obj
 0001:000f6730       _$E11                      004f7730 f   ldwSound.obj
 0001:000f6750       _$E13                      004f7750 f   ldwSound.obj
 0001:000f6770       _$E15                      004f7770 f   ldwSound.obj
 0001:000f6780       _$E1                       004f7780 f   ldwTextControl.obj
 0001:000f67a0       _$E3                       004f77a0 f   ldwTextControl.obj
 0001:000f67b0       _$E5                       004f77b0 f   ldwTextControl.obj
 0001:000f67e0       _$E7                       004f77e0 f   ldwTextControl.obj
 0001:000f6810       _$E9                       004f7810 f   ldwTextControl.obj
 0001:000f6830       _$E11                      004f7830 f   ldwTextControl.obj
 0001:000f6850       _$E13                      004f7850 f   ldwTextControl.obj
 0001:000f6870       _$E1                       004f7870 f   ldwTiledBackground.obj
 0001:000f6890       _$E3                       004f7890 f   ldwTiledBackground.obj
 0001:000f68a0       _$E5                       004f78a0 f   ldwTiledBackground.obj
 0001:000f68d0       _$E7                       004f78d0 f   ldwTiledBackground.obj
 0001:000f6900       _$E9                       004f7900 f   ldwTiledBackground.obj
 0001:000f6920       _$E11                      004f7920 f   ldwTiledBackground.obj
 0001:000f6940       _$E13                      004f7940 f   ldwTiledBackground.obj
 0001:000f6960       _$E1                       004f7960 f   ldwTiledDialog.obj
 0001:000f6980       _$E3                       004f7980 f   ldwTiledDialog.obj
 0001:000f6990       _$E5                       004f7990 f   ldwTiledDialog.obj
 0001:000f69c0       _$E7                       004f79c0 f   ldwTiledDialog.obj
 0001:000f69f0       _$E9                       004f79f0 f   ldwTiledDialog.obj
 0001:000f6a10       _$E11                      004f7a10 f   ldwTiledDialog.obj
 0001:000f6a30       _$E13                      004f7a30 f   ldwTiledDialog.obj
 0001:000f6a50       _$E1                       004f7a50 f   ldwWString.obj
 0001:000f6a70       _$E3                       004f7a70 f   ldwWString.obj
 0001:000f6a80       _$E5                       004f7a80 f   ldwWString.obj
 0001:000f6ab0       _$E7                       004f7ab0 f   ldwWString.obj
 0001:000f6ae0       _$E9                       004f7ae0 f   ldwWString.obj
 0001:000f6b00       _$E11                      004f7b00 f   ldwWString.obj
 0001:000f6b20       _$E13                      004f7b20 f   ldwWString.obj
 0001:000f6b40       _$E1                       004f7b40 f   AnimControl.obj
 0001:000f6b60       _$E3                       004f7b60 f   AnimControl.obj
 0001:000f6b70       _$E5                       004f7b70 f   AnimControl.obj
 0001:000f6ba0       _$E7                       004f7ba0 f   AnimControl.obj
 0001:000f6bd0       _$E9                       004f7bd0 f   AnimControl.obj
 0001:000f6bf0       _$E11                      004f7bf0 f   AnimControl.obj
 0001:000f6c10       _$E13                      004f7c10 f   AnimControl.obj
 0001:000f6c30       _$E1                       004f7c30 f   AnimManager.obj
 0001:000f6c50       _$E3                       004f7c50 f   AnimManager.obj
 0001:000f6c60       _$E5                       004f7c60 f   AnimManager.obj
 0001:000f6c90       _$E7                       004f7c90 f   AnimManager.obj
 0001:000f6cc0       _$E9                       004f7cc0 f   AnimManager.obj
 0001:000f6ce0       _$E11                      004f7ce0 f   AnimManager.obj
 0001:000f6d00       _$E13                      004f7d00 f   AnimManager.obj
 0001:000f6d20       _$E15                      004f7d20 f   AnimManager.obj
 0001:000f6d30       _$E1                       004f7d30 f   Behavior.obj
 0001:000f6d50       _$E3                       004f7d50 f   Behavior.obj
 0001:000f6d60       _$E5                       004f7d60 f   Behavior.obj
 0001:000f6d90       _$E7                       004f7d90 f   Behavior.obj
 0001:000f6dc0       _$E9                       004f7dc0 f   Behavior.obj
 0001:000f6de0       _$E11                      004f7de0 f   Behavior.obj
 0001:000f6e00       _$E13                      004f7e00 f   Behavior.obj
 0001:000f6e20       _$E15                      004f7e20 f   Behavior.obj
 0001:000f6e40       _$E17                      004f7e40 f   Behavior.obj
 0001:000f6e70       _$E19                      004f7e70 f   Behavior.obj
 0001:000f6eb0       _$E21                      004f7eb0 f   Behavior.obj
 0001:000f6ed0       _$E23                      004f7ed0 f   Behavior.obj
 0001:000f6ef0       _$E25                      004f7ef0 f   Behavior.obj
 0001:000f6f10       _$E27                      004f7f10 f   Behavior.obj
 0001:000f6f30       _$E29                      004f7f30 f   Behavior.obj
 0001:000f6f50       _$E31                      004f7f50 f   Behavior.obj
 0001:000f6f70       _$E33                      004f7f70 f   Behavior.obj
 0001:000f6f90       _$E35                      004f7f90 f   Behavior.obj
 0001:000f6fb0       _$E37                      004f7fb0 f   Behavior.obj
 0001:000f6fd0       _$E39                      004f7fd0 f   Behavior.obj
 0001:000f6ff0       _$E41                      004f7ff0 f   Behavior.obj
 0001:000f7010       _$E43                      004f8010 f   Behavior.obj
 0001:000f7030       _$E45                      004f8030 f   Behavior.obj
 0001:000f7050       _$E47                      004f8050 f   Behavior.obj
 0001:000f7070       _$E49                      004f8070 f   Behavior.obj
 0001:000f7090       _$E51                      004f8090 f   Behavior.obj
 0001:000f70b0       _$E53                      004f80b0 f   Behavior.obj
 0001:000f70d0       _$E55                      004f80d0 f   Behavior.obj
 0001:000f7120       _$E57                      004f8120 f   Behavior.obj
 0001:000f7140       _$E59                      004f8140 f   Behavior.obj
 0001:000f7160       _$E61                      004f8160 f   Behavior.obj
 0001:000f7180       _$E63                      004f8180 f   Behavior.obj
 0001:000f7190       _$E1                       004f8190 f   DislikeList.obj
 0001:000f71b0       _$E3                       004f81b0 f   DislikeList.obj
 0001:000f71c0       _$E5                       004f81c0 f   DislikeList.obj
 0001:000f71f0       _$E7                       004f81f0 f   DislikeList.obj
 0001:000f7220       _$E9                       004f8220 f   DislikeList.obj
 0001:000f7240       _$E11                      004f8240 f   DislikeList.obj
 0001:000f7260       _$E13                      004f8260 f   DislikeList.obj
 0001:000f7280       _$E1                       004f8280 f   Graveyard.obj
 0001:000f72a0       _$E3                       004f82a0 f   Graveyard.obj
 0001:000f72b0       _$E5                       004f82b0 f   Graveyard.obj
 0001:000f72e0       _$E7                       004f82e0 f   Graveyard.obj
 0001:000f7310       _$E9                       004f8310 f   Graveyard.obj
 0001:000f7330       _$E11                      004f8330 f   Graveyard.obj
 0001:000f7350       _$E13                      004f8350 f   Graveyard.obj
 0001:000f7370       _$E15                      004f8370 f   Graveyard.obj
 0001:000f7390       _$E17                      004f8390 f   Graveyard.obj
 0001:000f73c0       _$E19                      004f83c0 f   Graveyard.obj
 0001:000f7400       _$E21                      004f8400 f   Graveyard.obj
 0001:000f7420       _$E23                      004f8420 f   Graveyard.obj
 0001:000f7440       _$E25                      004f8440 f   Graveyard.obj
 0001:000f7460       _$E27                      004f8460 f   Graveyard.obj
 0001:000f7480       _$E29                      004f8480 f   Graveyard.obj
 0001:000f74a0       _$E31                      004f84a0 f   Graveyard.obj
 0001:000f74c0       _$E33                      004f84c0 f   Graveyard.obj
 0001:000f74e0       _$E35                      004f84e0 f   Graveyard.obj
 0001:000f7500       _$E37                      004f8500 f   Graveyard.obj
 0001:000f7520       _$E39                      004f8520 f   Graveyard.obj
 0001:000f7540       _$E41                      004f8540 f   Graveyard.obj
 0001:000f7560       _$E43                      004f8560 f   Graveyard.obj
 0001:000f7570       _$E1                       004f8570 f   LikeList.obj
 0001:000f7590       _$E3                       004f8590 f   LikeList.obj
 0001:000f75a0       _$E5                       004f85a0 f   LikeList.obj
 0001:000f75d0       _$E7                       004f85d0 f   LikeList.obj
 0001:000f7600       _$E9                       004f8600 f   LikeList.obj
 0001:000f7620       _$E11                      004f8620 f   LikeList.obj
 0001:000f7640       _$E13                      004f8640 f   LikeList.obj
 0001:000f7660       _$E1                       004f8660 f   Villager.obj
 0001:000f7680       _$E3                       004f8680 f   Villager.obj
 0001:000f7690       _$E5                       004f8690 f   Villager.obj
 0001:000f76c0       _$E7                       004f86c0 f   Villager.obj
 0001:000f76f0       _$E9                       004f86f0 f   Villager.obj
 0001:000f7710       _$E11                      004f8710 f   Villager.obj
 0001:000f7730       _$E13                      004f8730 f   Villager.obj
 0001:000f7750       _$E15                      004f8750 f   Villager.obj
 0001:000f7770       _$E17                      004f8770 f   Villager.obj
 0001:000f77a0       _$E19                      004f87a0 f   Villager.obj
 0001:000f77e0       _$E21                      004f87e0 f   Villager.obj
 0001:000f7800       _$E23                      004f8800 f   Villager.obj
 0001:000f7820       _$E25                      004f8820 f   Villager.obj
 0001:000f7840       _$E27                      004f8840 f   Villager.obj
 0001:000f7860       _$E29                      004f8860 f   Villager.obj
 0001:000f7880       _$E31                      004f8880 f   Villager.obj
 0001:000f78a0       _$E33                      004f88a0 f   Villager.obj
 0001:000f78c0       _$E35                      004f88c0 f   Villager.obj
 0001:000f78e0       _$E37                      004f88e0 f   Villager.obj
 0001:000f7900       _$E39                      004f8900 f   Villager.obj
 0001:000f7920       _$E41                      004f8920 f   Villager.obj
 0001:000f7940       _$E43                      004f8940 f   Villager.obj
 0001:000f7960       _$E1                       004f8960 f   VillagerAI.obj
 0001:000f7980       _$E3                       004f8980 f   VillagerAI.obj
 0001:000f7990       _$E5                       004f8990 f   VillagerAI.obj
 0001:000f79c0       _$E7                       004f89c0 f   VillagerAI.obj
 0001:000f79f0       _$E9                       004f89f0 f   VillagerAI.obj
 0001:000f7a10       _$E11                      004f8a10 f   VillagerAI.obj
 0001:000f7a30       _$E13                      004f8a30 f   VillagerAI.obj
 0001:000f7a50       _$E15                      004f8a50 f   VillagerAI.obj
 0001:000f7a70       _$E17                      004f8a70 f   VillagerAI.obj
 0001:000f7aa0       _$E19                      004f8aa0 f   VillagerAI.obj
 0001:000f7ae0       _$E21                      004f8ae0 f   VillagerAI.obj
 0001:000f7b00       _$E23                      004f8b00 f   VillagerAI.obj
 0001:000f7b20       _$E25                      004f8b20 f   VillagerAI.obj
 0001:000f7b40       _$E27                      004f8b40 f   VillagerAI.obj
 0001:000f7b60       _$E29                      004f8b60 f   VillagerAI.obj
 0001:000f7b80       _$E31                      004f8b80 f   VillagerAI.obj
 0001:000f7ba0       _$E33                      004f8ba0 f   VillagerAI.obj
 0001:000f7bc0       _$E35                      004f8bc0 f   VillagerAI.obj
 0001:000f7be0       _$E37                      004f8be0 f   VillagerAI.obj
 0001:000f7c00       _$E39                      004f8c00 f   VillagerAI.obj
 0001:000f7c20       _$E41                      004f8c20 f   VillagerAI.obj
 0001:000f7c40       _$E43                      004f8c40 f   VillagerAI.obj
 0001:000f7c60       _$E45                      004f8c60 f   VillagerAI.obj
 0001:000f7c80       _$E47                      004f8c80 f   VillagerAI.obj
 0001:000f7ca0       _$E49                      004f8ca0 f   VillagerAI.obj
 0001:000f7cf0       _$E51                      004f8cf0 f   VillagerAI.obj
 0001:000f7d10       _$E53                      004f8d10 f   VillagerAI.obj
 0001:000f7d30       _$E55                      004f8d30 f   VillagerAI.obj
 0001:000f7d50       _$E57                      004f8d50 f   VillagerAI.obj
 0001:000f7d70       _$E59                      004f8d70 f   VillagerAI.obj
 0001:000f7da0       _$E61                      004f8da0 f   VillagerAI.obj
 0001:000f7dc0       _$E63                      004f8dc0 f   VillagerAI.obj
 0001:000f7de0       _$E1                       004f8de0 f   VillagerBio.obj
 0001:000f7e00       _$E3                       004f8e00 f   VillagerBio.obj
 0001:000f7e10       _$E5                       004f8e10 f   VillagerBio.obj
 0001:000f7e40       _$E7                       004f8e40 f   VillagerBio.obj
 0001:000f7e70       _$E9                       004f8e70 f   VillagerBio.obj
 0001:000f7e90       _$E11                      004f8e90 f   VillagerBio.obj
 0001:000f7eb0       _$E13                      004f8eb0 f   VillagerBio.obj
 0001:000f7ed0       _$E15                      004f8ed0 f   VillagerBio.obj
 0001:000f7ef0       _$E17                      004f8ef0 f   VillagerBio.obj
 0001:000f7f20       _$E19                      004f8f20 f   VillagerBio.obj
 0001:000f7f60       _$E21                      004f8f60 f   VillagerBio.obj
 0001:000f7f80       _$E23                      004f8f80 f   VillagerBio.obj
 0001:000f7fa0       _$E25                      004f8fa0 f   VillagerBio.obj
 0001:000f7fc0       _$E27                      004f8fc0 f   VillagerBio.obj
 0001:000f7fe0       _$E29                      004f8fe0 f   VillagerBio.obj
 0001:000f8000       _$E31                      004f9000 f   VillagerBio.obj
 0001:000f8020       _$E33                      004f9020 f   VillagerBio.obj
 0001:000f8040       _$E35                      004f9040 f   VillagerBio.obj
 0001:000f8060       _$E37                      004f9060 f   VillagerBio.obj
 0001:000f8080       _$E39                      004f9080 f   VillagerBio.obj
 0001:000f80a0       _$E41                      004f90a0 f   VillagerBio.obj
 0001:000f80c0       _$E1                       004f90c0 f   VillagerManager.obj
 0001:000f80e0       _$E3                       004f90e0 f   VillagerManager.obj
 0001:000f80f0       _$E5                       004f90f0 f   VillagerManager.obj
 0001:000f8120       _$E7                       004f9120 f   VillagerManager.obj
 0001:000f8150       _$E9                       004f9150 f   VillagerManager.obj
 0001:000f8170       _$E11                      004f9170 f   VillagerManager.obj
 0001:000f8190       _$E13                      004f9190 f   VillagerManager.obj
 0001:000f81b0       _$E15                      004f91b0 f   VillagerManager.obj
 0001:000f81d0       _$E17                      004f91d0 f   VillagerManager.obj
 0001:000f8200       _$E19                      004f9200 f   VillagerManager.obj
 0001:000f8240       _$E21                      004f9240 f   VillagerManager.obj
 0001:000f8260       _$E23                      004f9260 f   VillagerManager.obj
 0001:000f8280       _$E25                      004f9280 f   VillagerManager.obj
 0001:000f82a0       _$E27                      004f92a0 f   VillagerManager.obj
 0001:000f82c0       _$E29                      004f92c0 f   VillagerManager.obj
 0001:000f82e0       _$E31                      004f92e0 f   VillagerManager.obj
 0001:000f8300       _$E33                      004f9300 f   VillagerManager.obj
 0001:000f8320       _$E35                      004f9320 f   VillagerManager.obj
 0001:000f8340       _$E37                      004f9340 f   VillagerManager.obj
 0001:000f8360       _$E39                      004f9360 f   VillagerManager.obj
 0001:000f8380       _$E41                      004f9380 f   VillagerManager.obj
 0001:000f83a0       _$E43                      004f93a0 f   VillagerManager.obj
 0001:000f83c0       _$E45                      004f93c0 f   VillagerManager.obj
 0001:000f83e0       _$E47                      004f93e0 f   VillagerManager.obj
 0001:000f8400       _$E51                      004f9400 f   VillagerManager.obj
 0001:000f8410       _$E1                       004f9410 f   VillagerPlans.obj
 0001:000f8430       _$E3                       004f9430 f   VillagerPlans.obj
 0001:000f8440       _$E5                       004f9440 f   VillagerPlans.obj
 0001:000f8470       _$E7                       004f9470 f   VillagerPlans.obj
 0001:000f84a0       _$E9                       004f94a0 f   VillagerPlans.obj
 0001:000f84c0       _$E11                      004f94c0 f   VillagerPlans.obj
 0001:000f84e0       _$E13                      004f94e0 f   VillagerPlans.obj
 0001:000f8500       _$E15                      004f9500 f   VillagerPlans.obj
 0001:000f8520       _$E17                      004f9520 f   VillagerPlans.obj
 0001:000f8550       _$E19                      004f9550 f   VillagerPlans.obj
 0001:000f8590       _$E21                      004f9590 f   VillagerPlans.obj
 0001:000f85b0       _$E23                      004f95b0 f   VillagerPlans.obj
 0001:000f85d0       _$E25                      004f95d0 f   VillagerPlans.obj
 0001:000f85f0       _$E27                      004f95f0 f   VillagerPlans.obj
 0001:000f8610       _$E29                      004f9610 f   VillagerPlans.obj
 0001:000f8630       _$E31                      004f9630 f   VillagerPlans.obj
 0001:000f8650       _$E33                      004f9650 f   VillagerPlans.obj
 0001:000f8670       _$E35                      004f9670 f   VillagerPlans.obj
 0001:000f8690       _$E37                      004f9690 f   VillagerPlans.obj
 0001:000f86b0       _$E39                      004f96b0 f   VillagerPlans.obj
 0001:000f86d0       _$E41                      004f96d0 f   VillagerPlans.obj
 0001:000f86f0       _$E1                       004f96f0 f   VillagerSkills.obj
 0001:000f8710       _$E3                       004f9710 f   VillagerSkills.obj
 0001:000f8720       _$E5                       004f9720 f   VillagerSkills.obj
 0001:000f8750       _$E7                       004f9750 f   VillagerSkills.obj
 0001:000f8780       _$E9                       004f9780 f   VillagerSkills.obj
 0001:000f87a0       _$E11                      004f97a0 f   VillagerSkills.obj
 0001:000f87c0       _$E13                      004f97c0 f   VillagerSkills.obj
 0001:000f87e0       _$E15                      004f97e0 f   VillagerSkills.obj
 0001:000f8800       _$E17                      004f9800 f   VillagerSkills.obj
 0001:000f8830       _$E19                      004f9830 f   VillagerSkills.obj
 0001:000f8870       _$E21                      004f9870 f   VillagerSkills.obj
 0001:000f8890       _$E23                      004f9890 f   VillagerSkills.obj
 0001:000f88b0       _$E25                      004f98b0 f   VillagerSkills.obj
 0001:000f88d0       _$E27                      004f98d0 f   VillagerSkills.obj
 0001:000f88f0       _$E29                      004f98f0 f   VillagerSkills.obj
 0001:000f8910       _$E1                       004f9910 f   VillagerState.obj
 0001:000f8930       _$E3                       004f9930 f   VillagerState.obj
 0001:000f8940       _$E5                       004f9940 f   VillagerState.obj
 0001:000f8970       _$E7                       004f9970 f   VillagerState.obj
 0001:000f89a0       _$E9                       004f99a0 f   VillagerState.obj
 0001:000f89c0       _$E11                      004f99c0 f   VillagerState.obj
 0001:000f89e0       _$E13                      004f99e0 f   VillagerState.obj
 0001:000f8a00       _$E15                      004f9a00 f   VillagerState.obj
 0001:000f8a20       _$E17                      004f9a20 f   VillagerState.obj
 0001:000f8a50       _$E19                      004f9a50 f   VillagerState.obj
 0001:000f8a90       _$E21                      004f9a90 f   VillagerState.obj
 0001:000f8ab0       _$E23                      004f9ab0 f   VillagerState.obj
 0001:000f8ad0       _$E25                      004f9ad0 f   VillagerState.obj
 0001:000f8af0       _$E27                      004f9af0 f   VillagerState.obj
 0001:000f8b10       _$E29                      004f9b10 f   VillagerState.obj
 0001:000f8b30       _$E31                      004f9b30 f   VillagerState.obj
 0001:000f8b50       _$E33                      004f9b50 f   VillagerState.obj
 0001:000f8b70       _$E35                      004f9b70 f   VillagerState.obj
 0001:000f8b90       _$E37                      004f9b90 f   VillagerState.obj
 0001:000f8bb0       _$E39                      004f9bb0 f   VillagerState.obj
 0001:000f8bd0       _$E41                      004f9bd0 f   VillagerState.obj
 0001:000f8bf0       _$E1                       004f9bf0 f   CollectionScene.obj
 0001:000f8c10       _$E3                       004f9c10 f   CollectionScene.obj
 0001:000f8c20       _$E5                       004f9c20 f   CollectionScene.obj
 0001:000f8c50       _$E7                       004f9c50 f   CollectionScene.obj
 0001:000f8c80       _$E9                       004f9c80 f   CollectionScene.obj
 0001:000f8ca0       _$E11                      004f9ca0 f   CollectionScene.obj
 0001:000f8cc0       _$E13                      004f9cc0 f   CollectionScene.obj
 0001:000f8ce0       _$E15                      004f9ce0 f   CollectionScene.obj
 0001:000f8d00       _$E17                      004f9d00 f   CollectionScene.obj
 0001:000f8d20       _$E19                      004f9d20 f   CollectionScene.obj
 0001:000f8d40       _$E21                      004f9d40 f   CollectionScene.obj
 0001:000f8d60       _$E23                      004f9d60 f   CollectionScene.obj
 0001:000f8d80       _$E25                      004f9d80 f   CollectionScene.obj
 0001:000f8da0       _$E27                      004f9da0 f   CollectionScene.obj
 0001:000f8dc0       _$E29                      004f9dc0 f   CollectionScene.obj
 0001:000f8df0       _$E31                      004f9df0 f   CollectionScene.obj
 0001:000f8e30       _$E33                      004f9e30 f   CollectionScene.obj
 0001:000f8e50       _$E35                      004f9e50 f   CollectionScene.obj
 0001:000f8e70       _$E37                      004f9e70 f   CollectionScene.obj
 0001:000f8e90       _$E39                      004f9e90 f   CollectionScene.obj
 0001:000f8eb0       _$E41                      004f9eb0 f   CollectionScene.obj
 0001:000f8ed0       _$E43                      004f9ed0 f   CollectionScene.obj
 0001:000f8ef0       _$E45                      004f9ef0 f   CollectionScene.obj
 0001:000f8f10       _$E47                      004f9f10 f   CollectionScene.obj
 0001:000f8f30       _$E49                      004f9f30 f   CollectionScene.obj
 0001:000f8f50       _$E51                      004f9f50 f   CollectionScene.obj
 0001:000f8f70       _$E1                       004f9f70 f   ProgressScene.obj
 0001:000f8f90       _$E3                       004f9f90 f   ProgressScene.obj
 0001:000f8fa0       _$E5                       004f9fa0 f   ProgressScene.obj
 0001:000f8fd0       _$E7                       004f9fd0 f   ProgressScene.obj
 0001:000f9000       _$E9                       004fa000 f   ProgressScene.obj
 0001:000f9020       _$E11                      004fa020 f   ProgressScene.obj
 0001:000f9040       _$E13                      004fa040 f   ProgressScene.obj
 0001:000f9060       _$E15                      004fa060 f   ProgressScene.obj
 0001:000f9080       _$E17                      004fa080 f   ProgressScene.obj
 0001:000f90a0       _$E19                      004fa0a0 f   ProgressScene.obj
 0001:000f90c0       _$E21                      004fa0c0 f   ProgressScene.obj
 0001:000f90f0       _$E23                      004fa0f0 f   ProgressScene.obj
 0001:000f9130       _$E25                      004fa130 f   ProgressScene.obj
 0001:000f9150       _$E27                      004fa150 f   ProgressScene.obj
 0001:000f9170       _$E29                      004fa170 f   ProgressScene.obj
 0001:000f9190       _$E31                      004fa190 f   ProgressScene.obj
 0001:000f91b0       _$E33                      004fa1b0 f   ProgressScene.obj
 0001:000f91d0       _$E35                      004fa1d0 f   ProgressScene.obj
 0001:000f91f0       _$E37                      004fa1f0 f   ProgressScene.obj
 0001:000f9210       _$E39                      004fa210 f   ProgressScene.obj
 0001:000f9230       _$E41                      004fa230 f   ProgressScene.obj
 0001:000f9250       _$E43                      004fa250 f   ProgressScene.obj
 0001:000f9270       _$E45                      004fa270 f   ProgressScene.obj
 0001:000f9290       _$E1                       004fa290 f   StoryScene.obj
 0001:000f92b0       _$E3                       004fa2b0 f   StoryScene.obj
 0001:000f92c0       _$E5                       004fa2c0 f   StoryScene.obj
 0001:000f92f0       _$E7                       004fa2f0 f   StoryScene.obj
 0001:000f9320       _$E9                       004fa320 f   StoryScene.obj
 0001:000f9340       _$E11                      004fa340 f   StoryScene.obj
 0001:000f9360       _$E13                      004fa360 f   StoryScene.obj
 0001:000f9380       _$E15                      004fa380 f   StoryScene.obj
 0001:000f93a0       _$E17                      004fa3a0 f   StoryScene.obj
 0001:000f93c0       _$E19                      004fa3c0 f   StoryScene.obj
 0001:000f93f0       _$E21                      004fa3f0 f   StoryScene.obj
 0001:000f9430       _$E23                      004fa430 f   StoryScene.obj
 0001:000f9450       _$E25                      004fa450 f   StoryScene.obj
 0001:000f9470       _$E27                      004fa470 f   StoryScene.obj
 0001:000f9490       _$E29                      004fa490 f   StoryScene.obj
 0001:000f94b0       _$E31                      004fa4b0 f   StoryScene.obj
 0001:000f94d0       _$E33                      004fa4d0 f   StoryScene.obj
 0001:000f94f0       _$E35                      004fa4f0 f   StoryScene.obj
 0001:000f9510       _$E37                      004fa510 f   StoryScene.obj
 0001:000f9530       _$E39                      004fa530 f   StoryScene.obj
 0001:000f9550       _$E41                      004fa550 f   StoryScene.obj
 0001:000f9570       _$E43                      004fa570 f   StoryScene.obj
 0001:000f9590       _$E1                       004fa590 f   TechScene.obj
 0001:000f95b0       _$E3                       004fa5b0 f   TechScene.obj
 0001:000f95c0       _$E5                       004fa5c0 f   TechScene.obj
 0001:000f95f0       _$E7                       004fa5f0 f   TechScene.obj
 0001:000f9620       _$E9                       004fa620 f   TechScene.obj
 0001:000f9640       _$E11                      004fa640 f   TechScene.obj
 0001:000f9660       _$E13                      004fa660 f   TechScene.obj
 0001:000f9680       _$E15                      004fa680 f   TechScene.obj
 0001:000f96a0       _$E17                      004fa6a0 f   TechScene.obj
 0001:000f96c0       _$E19                      004fa6c0 f   TechScene.obj
 0001:000f96e0       _$E21                      004fa6e0 f   TechScene.obj
 0001:000f9700       _$E23                      004fa700 f   TechScene.obj
 0001:000f9720       _$E25                      004fa720 f   TechScene.obj
 0001:000f9740       _$E27                      004fa740 f   TechScene.obj
 0001:000f9760       _$E29                      004fa760 f   TechScene.obj
 0001:000f9790       _$E31                      004fa790 f   TechScene.obj
 0001:000f97d0       _$E33                      004fa7d0 f   TechScene.obj
 0001:000f97f0       _$E35                      004fa7f0 f   TechScene.obj
 0001:000f9810       _$E37                      004fa810 f   TechScene.obj
 0001:000f9830       _$E39                      004fa830 f   TechScene.obj
 0001:000f9850       _$E41                      004fa850 f   TechScene.obj
 0001:000f9870       _$E43                      004fa870 f   TechScene.obj
 0001:000f9890       _$E1                       004fa890 f   theHelpScene.obj
 0001:000f98b0       _$E3                       004fa8b0 f   theHelpScene.obj
 0001:000f98c0       _$E5                       004fa8c0 f   theHelpScene.obj
 0001:000f98f0       _$E7                       004fa8f0 f   theHelpScene.obj
 0001:000f9920       _$E9                       004fa920 f   theHelpScene.obj
 0001:000f9940       _$E11                      004fa940 f   theHelpScene.obj
 0001:000f9960       _$E13                      004fa960 f   theHelpScene.obj
 0001:000f9980       _$E15                      004fa980 f   theHelpScene.obj
 0001:000f99a0       _$E17                      004fa9a0 f   theHelpScene.obj
 0001:000f99d0       _$E19                      004fa9d0 f   theHelpScene.obj
 0001:000f9a10       _$E21                      004faa10 f   theHelpScene.obj
 0001:000f9a30       _$E23                      004faa30 f   theHelpScene.obj
 0001:000f9a50       _$E25                      004faa50 f   theHelpScene.obj
 0001:000f9a70       _$E27                      004faa70 f   theHelpScene.obj
 0001:000f9a90       _$E29                      004faa90 f   theHelpScene.obj
 0001:000f9ab0       _$E31                      004faab0 f   theHelpScene.obj
 0001:000f9ad0       _$E33                      004faad0 f   theHelpScene.obj
 0001:000f9af0       _$E35                      004faaf0 f   theHelpScene.obj
 0001:000f9b10       _$E37                      004fab10 f   theHelpScene.obj
 0001:000f9b30       _$E39                      004fab30 f   theHelpScene.obj
 0001:000f9b50       _$E41                      004fab50 f   theHelpScene.obj
 0001:000f9b70       _$E43                      004fab70 f   theHelpScene.obj
 0001:000f9b90       _$E1                       004fab90 f   theLoadingScene.obj
 0001:000f9bb0       _$E3                       004fabb0 f   theLoadingScene.obj
 0001:000f9bc0       _$E5                       004fabc0 f   theLoadingScene.obj
 0001:000f9bf0       _$E7                       004fabf0 f   theLoadingScene.obj
 0001:000f9c20       _$E9                       004fac20 f   theLoadingScene.obj
 0001:000f9c40       _$E11                      004fac40 f   theLoadingScene.obj
 0001:000f9c60       _$E13                      004fac60 f   theLoadingScene.obj
 0001:000f9c80       _$E15                      004fac80 f   theLoadingScene.obj
 0001:000f9ca0       _$E17                      004faca0 f   theLoadingScene.obj
 0001:000f9cd0       _$E19                      004facd0 f   theLoadingScene.obj
 0001:000f9d10       _$E21                      004fad10 f   theLoadingScene.obj
 0001:000f9d30       _$E23                      004fad30 f   theLoadingScene.obj
 0001:000f9d50       _$E25                      004fad50 f   theLoadingScene.obj
 0001:000f9d70       _$E27                      004fad70 f   theLoadingScene.obj
 0001:000f9d90       _$E29                      004fad90 f   theLoadingScene.obj
 0001:000f9db0       _$E31                      004fadb0 f   theLoadingScene.obj
 0001:000f9dd0       _$E33                      004fadd0 f   theLoadingScene.obj
 0001:000f9df0       _$E35                      004fadf0 f   theLoadingScene.obj
 0001:000f9e10       _$E37                      004fae10 f   theLoadingScene.obj
 0001:000f9e30       _$E39                      004fae30 f   theLoadingScene.obj
 0001:000f9e50       _$E41                      004fae50 f   theLoadingScene.obj
 0001:000f9e70       _$E43                      004fae70 f   theLoadingScene.obj
 0001:000f9e90       _$E1                       004fae90 f   theMainScene.obj
 0001:000f9eb0       _$E3                       004faeb0 f   theMainScene.obj
 0001:000f9ec0       _$E5                       004faec0 f   theMainScene.obj
 0001:000f9ef0       _$E7                       004faef0 f   theMainScene.obj
 0001:000f9f20       _$E9                       004faf20 f   theMainScene.obj
 0001:000f9f40       _$E11                      004faf40 f   theMainScene.obj
 0001:000f9f60       _$E13                      004faf60 f   theMainScene.obj
 0001:000f9f80       _$E15                      004faf80 f   theMainScene.obj
 0001:000f9fa0       _$E17                      004fafa0 f   theMainScene.obj
 0001:000f9fd0       _$E19                      004fafd0 f   theMainScene.obj
 0001:000fa010       _$E21                      004fb010 f   theMainScene.obj
 0001:000fa030       _$E23                      004fb030 f   theMainScene.obj
 0001:000fa050       _$E25                      004fb050 f   theMainScene.obj
 0001:000fa070       _$E27                      004fb070 f   theMainScene.obj
 0001:000fa090       _$E29                      004fb090 f   theMainScene.obj
 0001:000fa0b0       _$E31                      004fb0b0 f   theMainScene.obj
 0001:000fa0d0       _$E33                      004fb0d0 f   theMainScene.obj
 0001:000fa0f0       _$E35                      004fb0f0 f   theMainScene.obj
 0001:000fa110       _$E37                      004fb110 f   theMainScene.obj
 0001:000fa130       _$E39                      004fb130 f   theMainScene.obj
 0001:000fa150       _$E41                      004fb150 f   theMainScene.obj
 0001:000fa170       _$E43                      004fb170 f   theMainScene.obj
 0001:000fa190       _$E45                      004fb190 f   theMainScene.obj
 0001:000fa1b0       _$E47                      004fb1b0 f   theMainScene.obj
 0001:000fa1d0       _$E49                      004fb1d0 f   theMainScene.obj
 0001:000fa1f0       _$E51                      004fb1f0 f   theMainScene.obj
 0001:000fa210       _$E53                      004fb210 f   theMainScene.obj
 0001:000fa230       _$E55                      004fb230 f   theMainScene.obj
 0001:000fa250       _$E57                      004fb250 f   theMainScene.obj
 0001:000fa270       _$E59                      004fb270 f   theMainScene.obj
 0001:000fa290       _$E61                      004fb290 f   theMainScene.obj
 0001:000fa2b0       _$E63                      004fb2b0 f   theMainScene.obj
 0001:000fa2d0       _$E65                      004fb2d0 f   theMainScene.obj
 0001:000fa320       _$E67                      004fb320 f   theMainScene.obj
 0001:000fa340       _$E69                      004fb340 f   theMainScene.obj
 0001:000fa360       _$E71                      004fb360 f   theMainScene.obj
 0001:000fa380       _$E73                      004fb380 f   theMainScene.obj
 0001:000fa3a0       _$E75                      004fb3a0 f   theMainScene.obj
 0001:000fa3d0       _$E1                       004fb3d0 f   theMenuScene.obj
 0001:000fa3f0       _$E3                       004fb3f0 f   theMenuScene.obj
 0001:000fa400       _$E5                       004fb400 f   theMenuScene.obj
 0001:000fa430       _$E7                       004fb430 f   theMenuScene.obj
 0001:000fa460       _$E9                       004fb460 f   theMenuScene.obj
 0001:000fa480       _$E11                      004fb480 f   theMenuScene.obj
 0001:000fa4a0       _$E13                      004fb4a0 f   theMenuScene.obj
 0001:000fa4c0       _$E15                      004fb4c0 f   theMenuScene.obj
 0001:000fa4e0       _$E17                      004fb4e0 f   theMenuScene.obj
 0001:000fa510       _$E19                      004fb510 f   theMenuScene.obj
 0001:000fa550       _$E21                      004fb550 f   theMenuScene.obj
 0001:000fa570       _$E23                      004fb570 f   theMenuScene.obj
 0001:000fa590       _$E25                      004fb590 f   theMenuScene.obj
 0001:000fa5b0       _$E27                      004fb5b0 f   theMenuScene.obj
 0001:000fa5d0       _$E29                      004fb5d0 f   theMenuScene.obj
 0001:000fa5f0       _$E31                      004fb5f0 f   theMenuScene.obj
 0001:000fa610       _$E33                      004fb610 f   theMenuScene.obj
 0001:000fa630       _$E35                      004fb630 f   theMenuScene.obj
 0001:000fa650       _$E37                      004fb650 f   theMenuScene.obj
 0001:000fa670       _$E39                      004fb670 f   theMenuScene.obj
 0001:000fa690       _$E41                      004fb690 f   theMenuScene.obj
 0001:000fa6b0       _$E43                      004fb6b0 f   theMenuScene.obj
 0001:000fa6d0       _$E1                       004fb6d0 f   theOverviewScene.obj
 0001:000fa6f0       _$E3                       004fb6f0 f   theOverviewScene.obj
 0001:000fa700       _$E5                       004fb700 f   theOverviewScene.obj
 0001:000fa730       _$E7                       004fb730 f   theOverviewScene.obj
 0001:000fa760       _$E9                       004fb760 f   theOverviewScene.obj
 0001:000fa780       _$E11                      004fb780 f   theOverviewScene.obj
 0001:000fa7a0       _$E13                      004fb7a0 f   theOverviewScene.obj
 0001:000fa7c0       _$E15                      004fb7c0 f   theOverviewScene.obj
 0001:000fa7e0       _$E17                      004fb7e0 f   theOverviewScene.obj
 0001:000fa800       _$E19                      004fb800 f   theOverviewScene.obj
 0001:000fa820       _$E21                      004fb820 f   theOverviewScene.obj
 0001:000fa840       _$E23                      004fb840 f   theOverviewScene.obj
 0001:000fa860       _$E25                      004fb860 f   theOverviewScene.obj
 0001:000fa880       _$E27                      004fb880 f   theOverviewScene.obj
 0001:000fa8a0       _$E29                      004fb8a0 f   theOverviewScene.obj
 0001:000fa8d0       _$E31                      004fb8d0 f   theOverviewScene.obj
 0001:000fa910       _$E33                      004fb910 f   theOverviewScene.obj
 0001:000fa930       _$E35                      004fb930 f   theOverviewScene.obj
 0001:000fa950       _$E37                      004fb950 f   theOverviewScene.obj
 0001:000fa970       _$E39                      004fb970 f   theOverviewScene.obj
 0001:000fa990       _$E41                      004fb990 f   theOverviewScene.obj
 0001:000fa9b0       _$E43                      004fb9b0 f   theOverviewScene.obj
 0001:000fa9d0       _$E45                      004fb9d0 f   theOverviewScene.obj
 0001:000fa9f0       _$E47                      004fb9f0 f   theOverviewScene.obj
 0001:000faa10       _$E49                      004fba10 f   theOverviewScene.obj
 0001:000faa30       _$E1                       004fba30 f   theSplashScene.obj
 0001:000faa50       _$E3                       004fba50 f   theSplashScene.obj
 0001:000faa60       _$E5                       004fba60 f   theSplashScene.obj
 0001:000faa90       _$E7                       004fba90 f   theSplashScene.obj
 0001:000faac0       _$E9                       004fbac0 f   theSplashScene.obj
 0001:000faae0       _$E11                      004fbae0 f   theSplashScene.obj
 0001:000fab00       _$E13                      004fbb00 f   theSplashScene.obj
 0001:000fab20       _$E15                      004fbb20 f   theSplashScene.obj
 0001:000fab40       _$E17                      004fbb40 f   theSplashScene.obj
 0001:000fab70       _$E19                      004fbb70 f   theSplashScene.obj
 0001:000fabb0       _$E21                      004fbbb0 f   theSplashScene.obj
 0001:000fabd0       _$E23                      004fbbd0 f   theSplashScene.obj
 0001:000fabf0       _$E25                      004fbbf0 f   theSplashScene.obj
 0001:000fac10       _$E27                      004fbc10 f   theSplashScene.obj
 0001:000fac30       _$E29                      004fbc30 f   theSplashScene.obj
 0001:000fac50       _$E31                      004fbc50 f   theSplashScene.obj
 0001:000fac70       _$E33                      004fbc70 f   theSplashScene.obj
 0001:000fac90       _$E35                      004fbc90 f   theSplashScene.obj
 0001:000facb0       _$E37                      004fbcb0 f   theSplashScene.obj
 0001:000facd0       _$E39                      004fbcd0 f   theSplashScene.obj
 0001:000facf0       _$E41                      004fbcf0 f   theSplashScene.obj
 0001:000fad10       _$E43                      004fbd10 f   theSplashScene.obj
 0001:000fad30       _$E1                       004fbd30 f   theVillagerScene.obj
 0001:000fad50       _$E3                       004fbd50 f   theVillagerScene.obj
 0001:000fad60       _$E5                       004fbd60 f   theVillagerScene.obj
 0001:000fad90       _$E7                       004fbd90 f   theVillagerScene.obj
 0001:000fadc0       _$E9                       004fbdc0 f   theVillagerScene.obj
 0001:000fade0       _$E11                      004fbde0 f   theVillagerScene.obj
 0001:000fae00       _$E13                      004fbe00 f   theVillagerScene.obj
 0001:000fae20       _$E15                      004fbe20 f   theVillagerScene.obj
 0001:000fae40       _$E17                      004fbe40 f   theVillagerScene.obj
 0001:000fae70       _$E19                      004fbe70 f   theVillagerScene.obj
 0001:000faeb0       _$E21                      004fbeb0 f   theVillagerScene.obj
 0001:000faed0       _$E23                      004fbed0 f   theVillagerScene.obj
 0001:000faef0       _$E25                      004fbef0 f   theVillagerScene.obj
 0001:000faf10       _$E27                      004fbf10 f   theVillagerScene.obj
 0001:000faf30       _$E29                      004fbf30 f   theVillagerScene.obj
 0001:000faf50       _$E31                      004fbf50 f   theVillagerScene.obj
 0001:000faf70       _$E33                      004fbf70 f   theVillagerScene.obj
 0001:000faf90       _$E35                      004fbf90 f   theVillagerScene.obj
 0001:000fafb0       _$E37                      004fbfb0 f   theVillagerScene.obj
 0001:000fafd0       _$E39                      004fbfd0 f   theVillagerScene.obj
 0001:000faff0       _$E41                      004fbff0 f   theVillagerScene.obj
 0001:000fb010       _$E43                      004fc010 f   theVillagerScene.obj
 0001:000fb030       _$E1                       004fc030 f   IslandEvents.obj
 0001:000fb050       _$E3                       004fc050 f   IslandEvents.obj
 0001:000fb060       _$E5                       004fc060 f   IslandEvents.obj
 0001:000fb090       _$E7                       004fc090 f   IslandEvents.obj
 0001:000fb0c0       _$E9                       004fc0c0 f   IslandEvents.obj
 0001:000fb0e0       _$E11                      004fc0e0 f   IslandEvents.obj
 0001:000fb100       _$E13                      004fc100 f   IslandEvents.obj
 0001:000fb120       _$E15                      004fc120 f   IslandEvents.obj
 0001:000fb140       _$E17                      004fc140 f   IslandEvents.obj
 0001:000fb170       _$E19                      004fc170 f   IslandEvents.obj
 0001:000fb1b0       _$E21                      004fc1b0 f   IslandEvents.obj
 0001:000fb1d0       _$E23                      004fc1d0 f   IslandEvents.obj
 0001:000fb1f0       _$E25                      004fc1f0 f   IslandEvents.obj
 0001:000fb210       _$E27                      004fc210 f   IslandEvents.obj
 0001:000fb230       _$E29                      004fc230 f   IslandEvents.obj
 0001:000fb250       _$E31                      004fc250 f   IslandEvents.obj
 0001:000fb270       _$E33                      004fc270 f   IslandEvents.obj
 0001:000fb290       _$E35                      004fc290 f   IslandEvents.obj
 0001:000fb2b0       _$E37                      004fc2b0 f   IslandEvents.obj
 0001:000fb2d0       _$E39                      004fc2d0 f   IslandEvents.obj
 0001:000fb2f0       _$E41                      004fc2f0 f   IslandEvents.obj
 0001:000fb310       _$E43                      004fc310 f   IslandEvents.obj
 0001:000fb330       _$E45                      004fc330 f   IslandEvents.obj
 0001:000fb350       _$E47                      004fc350 f   IslandEvents.obj
 0001:000fb370       _$E1                       004fc370 f   RosterOfDeadDialog.obj
 0001:000fb390       _$E3                       004fc390 f   RosterOfDeadDialog.obj
 0001:000fb3a0       _$E5                       004fc3a0 f   RosterOfDeadDialog.obj
 0001:000fb3d0       _$E7                       004fc3d0 f   RosterOfDeadDialog.obj
 0001:000fb400       _$E9                       004fc400 f   RosterOfDeadDialog.obj
 0001:000fb420       _$E11                      004fc420 f   RosterOfDeadDialog.obj
 0001:000fb440       _$E13                      004fc440 f   RosterOfDeadDialog.obj
 0001:000fb460       _$E15                      004fc460 f   RosterOfDeadDialog.obj
 0001:000fb480       _$E17                      004fc480 f   RosterOfDeadDialog.obj
 0001:000fb4a0       _$E19                      004fc4a0 f   RosterOfDeadDialog.obj
 0001:000fb4c0       _$E21                      004fc4c0 f   RosterOfDeadDialog.obj
 0001:000fb4e0       _$E23                      004fc4e0 f   RosterOfDeadDialog.obj
 0001:000fb500       _$E25                      004fc500 f   RosterOfDeadDialog.obj
 0001:000fb520       _$E27                      004fc520 f   RosterOfDeadDialog.obj
 0001:000fb550       _$E29                      004fc550 f   RosterOfDeadDialog.obj
 0001:000fb590       _$E31                      004fc590 f   RosterOfDeadDialog.obj
 0001:000fb5b0       _$E33                      004fc5b0 f   RosterOfDeadDialog.obj
 0001:000fb5d0       _$E35                      004fc5d0 f   RosterOfDeadDialog.obj
 0001:000fb5f0       _$E37                      004fc5f0 f   RosterOfDeadDialog.obj
 0001:000fb610       _$E39                      004fc610 f   RosterOfDeadDialog.obj
 0001:000fb630       _$E41                      004fc630 f   RosterOfDeadDialog.obj
 0001:000fb650       _$E43                      004fc650 f   RosterOfDeadDialog.obj
 0001:000fb670       _$E1                       004fc670 f   theChangePlayerDlg.obj
 0001:000fb690       _$E3                       004fc690 f   theChangePlayerDlg.obj
 0001:000fb6a0       _$E5                       004fc6a0 f   theChangePlayerDlg.obj
 0001:000fb6d0       _$E7                       004fc6d0 f   theChangePlayerDlg.obj
 0001:000fb700       _$E9                       004fc700 f   theChangePlayerDlg.obj
 0001:000fb720       _$E11                      004fc720 f   theChangePlayerDlg.obj
 0001:000fb740       _$E13                      004fc740 f   theChangePlayerDlg.obj
 0001:000fb760       _$E15                      004fc760 f   theChangePlayerDlg.obj
 0001:000fb780       _$E17                      004fc780 f   theChangePlayerDlg.obj
 0001:000fb7b0       _$E19                      004fc7b0 f   theChangePlayerDlg.obj
 0001:000fb7f0       _$E21                      004fc7f0 f   theChangePlayerDlg.obj
 0001:000fb810       _$E23                      004fc810 f   theChangePlayerDlg.obj
 0001:000fb830       _$E25                      004fc830 f   theChangePlayerDlg.obj
 0001:000fb850       _$E27                      004fc850 f   theChangePlayerDlg.obj
 0001:000fb870       _$E29                      004fc870 f   theChangePlayerDlg.obj
 0001:000fb890       _$E31                      004fc890 f   theChangePlayerDlg.obj
 0001:000fb8b0       _$E33                      004fc8b0 f   theChangePlayerDlg.obj
 0001:000fb8d0       _$E35                      004fc8d0 f   theChangePlayerDlg.obj
 0001:000fb8f0       _$E37                      004fc8f0 f   theChangePlayerDlg.obj
 0001:000fb910       _$E39                      004fc910 f   theChangePlayerDlg.obj
 0001:000fb930       _$E41                      004fc930 f   theChangePlayerDlg.obj
 0001:000fb950       _$E43                      004fc950 f   theChangePlayerDlg.obj
 0001:000fb970       _$E1                       004fc970 f   theCreateNickNameDlg.obj
 0001:000fb990       _$E3                       004fc990 f   theCreateNickNameDlg.obj
 0001:000fb9a0       _$E5                       004fc9a0 f   theCreateNickNameDlg.obj
 0001:000fb9d0       _$E7                       004fc9d0 f   theCreateNickNameDlg.obj
 0001:000fba00       _$E9                       004fca00 f   theCreateNickNameDlg.obj
 0001:000fba20       _$E11                      004fca20 f   theCreateNickNameDlg.obj
 0001:000fba40       _$E13                      004fca40 f   theCreateNickNameDlg.obj
 0001:000fba60       _$E15                      004fca60 f   theCreateNickNameDlg.obj
 0001:000fba80       _$E17                      004fca80 f   theCreateNickNameDlg.obj
 0001:000fbab0       _$E19                      004fcab0 f   theCreateNickNameDlg.obj
 0001:000fbaf0       _$E21                      004fcaf0 f   theCreateNickNameDlg.obj
 0001:000fbb10       _$E23                      004fcb10 f   theCreateNickNameDlg.obj
 0001:000fbb30       _$E25                      004fcb30 f   theCreateNickNameDlg.obj
 0001:000fbb50       _$E27                      004fcb50 f   theCreateNickNameDlg.obj
 0001:000fbb70       _$E29                      004fcb70 f   theCreateNickNameDlg.obj
 0001:000fbb90       _$E31                      004fcb90 f   theCreateNickNameDlg.obj
 0001:000fbbb0       _$E33                      004fcbb0 f   theCreateNickNameDlg.obj
 0001:000fbbd0       _$E35                      004fcbd0 f   theCreateNickNameDlg.obj
 0001:000fbbf0       _$E37                      004fcbf0 f   theCreateNickNameDlg.obj
 0001:000fbc10       _$E39                      004fcc10 f   theCreateNickNameDlg.obj
 0001:000fbc30       _$E41                      004fcc30 f   theCreateNickNameDlg.obj
 0001:000fbc50       _$E43                      004fcc50 f   theCreateNickNameDlg.obj
 0001:000fbc70       _$E1                       004fcc70 f   theFernsaceDialog.obj
 0001:000fbc90       _$E3                       004fcc90 f   theFernsaceDialog.obj
 0001:000fbca0       _$E5                       004fcca0 f   theFernsaceDialog.obj
 0001:000fbcd0       _$E7                       004fccd0 f   theFernsaceDialog.obj
 0001:000fbd00       _$E9                       004fcd00 f   theFernsaceDialog.obj
 0001:000fbd20       _$E11                      004fcd20 f   theFernsaceDialog.obj
 0001:000fbd40       _$E13                      004fcd40 f   theFernsaceDialog.obj
 0001:000fbd60       _$E15                      004fcd60 f   theFernsaceDialog.obj
 0001:000fbd80       _$E17                      004fcd80 f   theFernsaceDialog.obj
 0001:000fbdb0       _$E19                      004fcdb0 f   theFernsaceDialog.obj
 0001:000fbdf0       _$E21                      004fcdf0 f   theFernsaceDialog.obj
 0001:000fbe10       _$E23                      004fce10 f   theFernsaceDialog.obj
 0001:000fbe30       _$E25                      004fce30 f   theFernsaceDialog.obj
 0001:000fbe50       _$E27                      004fce50 f   theFernsaceDialog.obj
 0001:000fbe70       _$E29                      004fce70 f   theFernsaceDialog.obj
 0001:000fbe90       _$E31                      004fce90 f   theFernsaceDialog.obj
 0001:000fbeb0       _$E33                      004fceb0 f   theFernsaceDialog.obj
 0001:000fbed0       _$E35                      004fced0 f   theFernsaceDialog.obj
 0001:000fbef0       _$E37                      004fcef0 f   theFernsaceDialog.obj
 0001:000fbf10       _$E39                      004fcf10 f   theFernsaceDialog.obj
 0001:000fbf30       _$E41                      004fcf30 f   theFernsaceDialog.obj
 0001:000fbf50       _$E43                      004fcf50 f   theFernsaceDialog.obj
 0001:000fbf70       _$E1                       004fcf70 f   theMessageBoxDlg.obj
 0001:000fbf90       _$E3                       004fcf90 f   theMessageBoxDlg.obj
 0001:000fbfa0       _$E5                       004fcfa0 f   theMessageBoxDlg.obj
 0001:000fbfd0       _$E7                       004fcfd0 f   theMessageBoxDlg.obj
 0001:000fc000       _$E9                       004fd000 f   theMessageBoxDlg.obj
 0001:000fc020       _$E11                      004fd020 f   theMessageBoxDlg.obj
 0001:000fc040       _$E13                      004fd040 f   theMessageBoxDlg.obj
 0001:000fc060       _$E15                      004fd060 f   theMessageBoxDlg.obj
 0001:000fc080       _$E17                      004fd080 f   theMessageBoxDlg.obj
 0001:000fc0b0       _$E19                      004fd0b0 f   theMessageBoxDlg.obj
 0001:000fc0f0       _$E21                      004fd0f0 f   theMessageBoxDlg.obj
 0001:000fc110       _$E23                      004fd110 f   theMessageBoxDlg.obj
 0001:000fc130       _$E25                      004fd130 f   theMessageBoxDlg.obj
 0001:000fc150       _$E27                      004fd150 f   theMessageBoxDlg.obj
 0001:000fc170       _$E29                      004fd170 f   theMessageBoxDlg.obj
 0001:000fc190       _$E31                      004fd190 f   theMessageBoxDlg.obj
 0001:000fc1b0       _$E33                      004fd1b0 f   theMessageBoxDlg.obj
 0001:000fc1d0       _$E35                      004fd1d0 f   theMessageBoxDlg.obj
 0001:000fc1f0       _$E37                      004fd1f0 f   theMessageBoxDlg.obj
 0001:000fc210       _$E39                      004fd210 f   theMessageBoxDlg.obj
 0001:000fc230       _$E41                      004fd230 f   theMessageBoxDlg.obj
 0001:000fc250       _$E43                      004fd250 f   theMessageBoxDlg.obj
 0001:000fc270       _$E1                       004fd270 f   theOptionsDialog.obj
 0001:000fc290       _$E3                       004fd290 f   theOptionsDialog.obj
 0001:000fc2a0       _$E5                       004fd2a0 f   theOptionsDialog.obj
 0001:000fc2d0       _$E7                       004fd2d0 f   theOptionsDialog.obj
 0001:000fc300       _$E9                       004fd300 f   theOptionsDialog.obj
 0001:000fc320       _$E11                      004fd320 f   theOptionsDialog.obj
 0001:000fc340       _$E13                      004fd340 f   theOptionsDialog.obj
 0001:000fc360       _$E15                      004fd360 f   theOptionsDialog.obj
 0001:000fc380       _$E17                      004fd380 f   theOptionsDialog.obj
 0001:000fc3a0       _$E19                      004fd3a0 f   theOptionsDialog.obj
 0001:000fc3c0       _$E21                      004fd3c0 f   theOptionsDialog.obj
 0001:000fc3e0       _$E23                      004fd3e0 f   theOptionsDialog.obj
 0001:000fc400       _$E25                      004fd400 f   theOptionsDialog.obj
 0001:000fc420       _$E27                      004fd420 f   theOptionsDialog.obj
 0001:000fc450       _$E29                      004fd450 f   theOptionsDialog.obj
 0001:000fc490       _$E31                      004fd490 f   theOptionsDialog.obj
 0001:000fc4b0       _$E33                      004fd4b0 f   theOptionsDialog.obj
 0001:000fc4d0       _$E35                      004fd4d0 f   theOptionsDialog.obj
 0001:000fc4f0       _$E37                      004fd4f0 f   theOptionsDialog.obj
 0001:000fc510       _$E39                      004fd510 f   theOptionsDialog.obj
 0001:000fc530       _$E41                      004fd530 f   theOptionsDialog.obj
 0001:000fc550       _$E43                      004fd550 f   theOptionsDialog.obj
 0001:000fc570       _$E1                       004fd570 f   theTipDialog.obj
 0001:000fc590       _$E3                       004fd590 f   theTipDialog.obj
 0001:000fc5a0       _$E5                       004fd5a0 f   theTipDialog.obj
 0001:000fc5d0       _$E7                       004fd5d0 f   theTipDialog.obj
 0001:000fc600       _$E9                       004fd600 f   theTipDialog.obj
 0001:000fc620       _$E11                      004fd620 f   theTipDialog.obj
 0001:000fc640       _$E13                      004fd640 f   theTipDialog.obj
 0001:000fc660       _$E15                      004fd660 f   theTipDialog.obj
 0001:000fc680       _$E17                      004fd680 f   theTipDialog.obj
 0001:000fc6a0       _$E19                      004fd6a0 f   theTipDialog.obj
 0001:000fc6d0       _$E21                      004fd6d0 f   theTipDialog.obj
 0001:000fc710       _$E23                      004fd710 f   theTipDialog.obj
 0001:000fc730       _$E25                      004fd730 f   theTipDialog.obj
 0001:000fc750       _$E27                      004fd750 f   theTipDialog.obj
 0001:000fc770       _$E29                      004fd770 f   theTipDialog.obj
 0001:000fc790       _$E31                      004fd790 f   theTipDialog.obj
 0001:000fc7b0       _$E33                      004fd7b0 f   theTipDialog.obj
 0001:000fc7d0       _$E35                      004fd7d0 f   theTipDialog.obj
 0001:000fc7f0       _$E37                      004fd7f0 f   theTipDialog.obj
 0001:000fc810       _$E39                      004fd810 f   theTipDialog.obj
 0001:000fc830       _$E41                      004fd830 f   theTipDialog.obj
 0001:000fc850       _$E43                      004fd850 f   theTipDialog.obj
 0001:000fc870       _$E1                       004fd870 f   theTombStoneDialog.obj
 0001:000fc890       _$E3                       004fd890 f   theTombStoneDialog.obj
 0001:000fc8a0       _$E5                       004fd8a0 f   theTombStoneDialog.obj
 0001:000fc8d0       _$E7                       004fd8d0 f   theTombStoneDialog.obj
 0001:000fc900       _$E9                       004fd900 f   theTombStoneDialog.obj
 0001:000fc920       _$E11                      004fd920 f   theTombStoneDialog.obj
 0001:000fc940       _$E13                      004fd940 f   theTombStoneDialog.obj
 0001:000fc960       _$E15                      004fd960 f   theTombStoneDialog.obj
 0001:000fc980       _$E17                      004fd980 f   theTombStoneDialog.obj
 0001:000fc9b0       _$E19                      004fd9b0 f   theTombStoneDialog.obj
 0001:000fc9f0       _$E21                      004fd9f0 f   theTombStoneDialog.obj
 0001:000fca10       _$E23                      004fda10 f   theTombStoneDialog.obj
 0001:000fca30       _$E25                      004fda30 f   theTombStoneDialog.obj
 0001:000fca50       _$E27                      004fda50 f   theTombStoneDialog.obj
 0001:000fca70       _$E29                      004fda70 f   theTombStoneDialog.obj
 0001:000fca90       _$E31                      004fda90 f   theTombStoneDialog.obj
 0001:000fcab0       _$E33                      004fdab0 f   theTombStoneDialog.obj
 0001:000fcad0       _$E35                      004fdad0 f   theTombStoneDialog.obj
 0001:000fcaf0       _$E37                      004fdaf0 f   theTombStoneDialog.obj
 0001:000fcb10       _$E39                      004fdb10 f   theTombStoneDialog.obj
 0001:000fcb30       _$E41                      004fdb30 f   theTombStoneDialog.obj
 0001:000fcb50       _$E43                      004fdb50 f   theTombStoneDialog.obj
 0001:000fcb70       _$E1                       004fdb70 f   Fog.obj
 0001:000fcb90       _$E3                       004fdb90 f   Fog.obj
 0001:000fcba0       _$E5                       004fdba0 f   Fog.obj
 0001:000fcbd0       _$E7                       004fdbd0 f   Fog.obj
 0001:000fcc00       _$E9                       004fdc00 f   Fog.obj
 0001:000fcc20       _$E11                      004fdc20 f   Fog.obj
 0001:000fcc40       _$E13                      004fdc40 f   Fog.obj
 0001:000fcc60       _$E15                      004fdc60 f   Fog.obj
 0001:000fcc80       _$E17                      004fdc80 f   Fog.obj
 0001:000fcca0       _$E19                      004fdca0 f   Fog.obj
 0001:000fccc0       _$E21                      004fdcc0 f   Fog.obj
 0001:000fcce0       _$E23                      004fdce0 f   Fog.obj
 0001:000fcd00       _$E25                      004fdd00 f   Fog.obj
 0001:000fcd20       _$E1                       004fdd20 f   Lightning.obj
 0001:000fcd40       _$E3                       004fdd40 f   Lightning.obj
 0001:000fcd50       _$E5                       004fdd50 f   Lightning.obj
 0001:000fcd80       _$E7                       004fdd80 f   Lightning.obj
 0001:000fcdb0       _$E9                       004fddb0 f   Lightning.obj
 0001:000fcdd0       _$E11                      004fddd0 f   Lightning.obj
 0001:000fcdf0       _$E13                      004fddf0 f   Lightning.obj
 0001:000fce10       _$E15                      004fde10 f   Lightning.obj
 0001:000fce30       _$E17                      004fde30 f   Lightning.obj
 0001:000fce50       _$E1                       004fde50 f   Rain.obj
 0001:000fce70       _$E3                       004fde70 f   Rain.obj
 0001:000fce80       _$E5                       004fde80 f   Rain.obj
 0001:000fceb0       _$E7                       004fdeb0 f   Rain.obj
 0001:000fcee0       _$E9                       004fdee0 f   Rain.obj
 0001:000fcf00       _$E11                      004fdf00 f   Rain.obj
 0001:000fcf20       _$E13                      004fdf20 f   Rain.obj
 0001:000fcf40       _$E15                      004fdf40 f   Rain.obj
 0001:000fcf60       _$E17                      004fdf60 f   Rain.obj
 0001:000fcf80       _$E19                      004fdf80 f   Rain.obj
 0001:000fcfa0       _$E21                      004fdfa0 f   Rain.obj
 0001:000fcfc0       _$E23                      004fdfc0 f   Rain.obj
 0001:000fcfe0       _$E25                      004fdfe0 f   Rain.obj
 0001:000fd000       _$E27                      004fe000 f   Rain.obj
 0001:000fd020       _$E1                       004fe020 f   SunBeam.obj
 0001:000fd040       _$E3                       004fe040 f   SunBeam.obj
 0001:000fd050       _$E5                       004fe050 f   SunBeam.obj
 0001:000fd080       _$E7                       004fe080 f   SunBeam.obj
 0001:000fd0b0       _$E9                       004fe0b0 f   SunBeam.obj
 0001:000fd0d0       _$E11                      004fe0d0 f   SunBeam.obj
 0001:000fd0f0       _$E13                      004fe0f0 f   SunBeam.obj
 0001:000fd110       _$E15                      004fe110 f   SunBeam.obj
 0001:000fd130       _$E17                      004fe130 f   SunBeam.obj
 0001:000fd150       _$E19                      004fe150 f   SunBeam.obj
 0001:000fd170       _$E21                      004fe170 f   SunBeam.obj
 0001:000fd190       _$E23                      004fe190 f   SunBeam.obj
 0001:000fd1b0       _$E25                      004fe1b0 f   SunBeam.obj
 0001:000fd1d0       _$E1                       004fe1d0 f   Weather.obj
 0001:000fd1f0       _$E3                       004fe1f0 f   Weather.obj
 0001:000fd200       _$E5                       004fe200 f   Weather.obj
 0001:000fd230       _$E7                       004fe230 f   Weather.obj
 0001:000fd260       _$E9                       004fe260 f   Weather.obj
 0001:000fd280       _$E11                      004fe280 f   Weather.obj
 0001:000fd2a0       _$E13                      004fe2a0 f   Weather.obj
 0001:000fd2c0       _$E15                      004fe2c0 f   Weather.obj
 0001:000fd2e0       _$E17                      004fe2e0 f   Weather.obj
 0001:000fd300       _$E19                      004fe300 f   Weather.obj
 0001:000fd330       _$E21                      004fe330 f   Weather.obj
 0001:000fd370       _$E23                      004fe370 f   Weather.obj
 0001:000fd390       _$E25                      004fe390 f   Weather.obj
 0001:000fd3b0       _$E27                      004fe3b0 f   Weather.obj
 0001:000fd3d0       _$E29                      004fe3d0 f   Weather.obj
 0001:000fd3f0       _$E31                      004fe3f0 f   Weather.obj
 0001:000fd410       _$E33                      004fe410 f   Weather.obj
 0001:000fd430       _$E1                       004fe430 f   ContentMap.obj
 0001:000fd450       _$E3                       004fe450 f   ContentMap.obj
 0001:000fd460       _$E5                       004fe460 f   ContentMap.obj
 0001:000fd490       _$E7                       004fe490 f   ContentMap.obj
 0001:000fd4c0       _$E9                       004fe4c0 f   ContentMap.obj
 0001:000fd4e0       _$E11                      004fe4e0 f   ContentMap.obj
 0001:000fd500       _$E13                      004fe500 f   ContentMap.obj
 0001:000fd520       _$E15                      004fe520 f   ContentMap.obj
 0001:000fd540       _$E17                      004fe540 f   ContentMap.obj
 0001:000fd570       _$E19                      004fe570 f   ContentMap.obj
 0001:000fd5b0       _$E21                      004fe5b0 f   ContentMap.obj
 0001:000fd5d0       _$E23                      004fe5d0 f   ContentMap.obj
 0001:000fd5f0       _$E25                      004fe5f0 f   ContentMap.obj
 0001:000fd610       _$E27                      004fe610 f   ContentMap.obj
 0001:000fd630       _$E29                      004fe630 f   ContentMap.obj
 0001:000fd650       _$E31                      004fe650 f   ContentMap.obj
 0001:000fd670       _$E33                      004fe670 f   ContentMap.obj
 0001:000fd690       _$E35                      004fe690 f   ContentMap.obj
 0001:000fd6b0       _$E37                      004fe6b0 f   ContentMap.obj
 0001:000fd6d0       _$E39                      004fe6d0 f   ContentMap.obj
 0001:000fd6f0       _$E41                      004fe6f0 f   ContentMap.obj
 0001:000fd710       _$E43                      004fe710 f   ContentMap.obj
 0001:000fd720       _$E1                       004fe720 f   Environment.obj
 0001:000fd740       _$E3                       004fe740 f   Environment.obj
 0001:000fd750       _$E5                       004fe750 f   Environment.obj
 0001:000fd780       _$E7                       004fe780 f   Environment.obj
 0001:000fd7b0       _$E9                       004fe7b0 f   Environment.obj
 0001:000fd7d0       _$E11                      004fe7d0 f   Environment.obj
 0001:000fd7f0       _$E13                      004fe7f0 f   Environment.obj
 0001:000fd810       _$E15                      004fe810 f   Environment.obj
 0001:000fd830       _$E17                      004fe830 f   Environment.obj
 0001:000fd850       _$E19                      004fe850 f   Environment.obj
 0001:000fd870       _$E21                      004fe870 f   Environment.obj
 0001:000fd890       _$E23                      004fe890 f   Environment.obj
 0001:000fd8b0       _$E25                      004fe8b0 f   Environment.obj
 0001:000fd8d0       _$E27                      004fe8d0 f   Environment.obj
 0001:000fd8f0       _$E29                      004fe8f0 f   Environment.obj
 0001:000fd910       _$E31                      004fe910 f   Environment.obj
 0001:000fd940       _$E33                      004fe940 f   Environment.obj
 0001:000fd980       _$E35                      004fe980 f   Environment.obj
 0001:000fd9a0       _$E37                      004fe9a0 f   Environment.obj
 0001:000fd9c0       _$E39                      004fe9c0 f   Environment.obj
 0001:000fd9e0       _$E41                      004fe9e0 f   Environment.obj
 0001:000fda00       _$E43                      004fea00 f   Environment.obj
 0001:000fda20       _$E45                      004fea20 f   Environment.obj
 0001:000fda40       _$E47                      004fea40 f   Environment.obj
 0001:000fda50       _$E1                       004fea50 f   HotSpot.obj
 0001:000fda70       _$E3                       004fea70 f   HotSpot.obj
 0001:000fda80       _$E5                       004fea80 f   HotSpot.obj
 0001:000fdab0       _$E7                       004feab0 f   HotSpot.obj
 0001:000fdae0       _$E9                       004feae0 f   HotSpot.obj
 0001:000fdb00       _$E11                      004feb00 f   HotSpot.obj
 0001:000fdb20       _$E13                      004feb20 f   HotSpot.obj
 0001:000fdb40       _$E15                      004feb40 f   HotSpot.obj
 0001:000fdb60       _$E17                      004feb60 f   HotSpot.obj
 0001:000fdb90       _$E19                      004feb90 f   HotSpot.obj
 0001:000fdbd0       _$E21                      004febd0 f   HotSpot.obj
 0001:000fdbf0       _$E23                      004febf0 f   HotSpot.obj
 0001:000fdc10       _$E25                      004fec10 f   HotSpot.obj
 0001:000fdc30       _$E27                      004fec30 f   HotSpot.obj
 0001:000fdc50       _$E29                      004fec50 f   HotSpot.obj
 0001:000fdc70       _$E31                      004fec70 f   HotSpot.obj
 0001:000fdc90       _$E33                      004fec90 f   HotSpot.obj
 0001:000fdcb0       _$E35                      004fecb0 f   HotSpot.obj
 0001:000fdcd0       _$E37                      004fecd0 f   HotSpot.obj
 0001:000fdcf0       _$E39                      004fecf0 f   HotSpot.obj
 0001:000fdd10       _$E41                      004fed10 f   HotSpot.obj
 0001:000fdd30       _$E43                      004fed30 f   HotSpot.obj
 0001:000fdd50       _$E45                      004fed50 f   HotSpot.obj
 0001:000fdd70       _$E47                      004fed70 f   HotSpot.obj
 0001:000fdd90       _$E49                      004fed90 f   HotSpot.obj
 0001:000fddb0       _$E51                      004fedb0 f   HotSpot.obj
 0001:000fddd0       _$E53                      004fedd0 f   HotSpot.obj
 0001:000fddf0       _$E55                      004fedf0 f   HotSpot.obj
 0001:000fde10       _$E57                      004fee10 f   HotSpot.obj
 0001:000fde30       _$E59                      004fee30 f   HotSpot.obj
 0001:000fde80       _$E61                      004fee80 f   HotSpot.obj
 0001:000fdea0       _$E63                      004feea0 f   HotSpot.obj
 0001:000fdec0       _$E65                      004feec0 f   HotSpot.obj
 0001:000fdee0       _$E67                      004feee0 f   HotSpot.obj
 0001:000fdf00       _$E69                      004fef00 f   HotSpot.obj
 0001:000fdf30       _$E71                      004fef30 f   HotSpot.obj
 0001:000fdf50       _$E73                      004fef50 f   HotSpot.obj
 0001:000fdf80       _$E75                      004fef80 f   HotSpot.obj
 0001:000fdfa0       _$E77                      004fefa0 f   HotSpot.obj
 0001:000fdfb0       _$E1                       004fefb0 f   Redirect.obj
 0001:000fdfd0       _$E3                       004fefd0 f   Redirect.obj
 0001:000fdfe0       _$E5                       004fefe0 f   Redirect.obj
 0001:000fe010       _$E7                       004ff010 f   Redirect.obj
 0001:000fe040       _$E9                       004ff040 f   Redirect.obj
 0001:000fe060       _$E11                      004ff060 f   Redirect.obj
 0001:000fe080       _$E13                      004ff080 f   Redirect.obj
 0001:000fe0a0       _$E15                      004ff0a0 f   Redirect.obj
 0001:000fe0c0       _$E17                      004ff0c0 f   Redirect.obj
 0001:000fe0f0       _$E19                      004ff0f0 f   Redirect.obj
 0001:000fe130       _$E21                      004ff130 f   Redirect.obj
 0001:000fe150       _$E23                      004ff150 f   Redirect.obj
 0001:000fe170       _$E25                      004ff170 f   Redirect.obj
 0001:000fe190       _$E27                      004ff190 f   Redirect.obj
 0001:000fe1b0       _$E29                      004ff1b0 f   Redirect.obj
 0001:000fe1d0       _$E31                      004ff1d0 f   Redirect.obj
 0001:000fe1e0       _$E1                       004ff1e0 f   Waypoint.obj
 0001:000fe200       _$E3                       004ff200 f   Waypoint.obj
 0001:000fe210       _$E5                       004ff210 f   Waypoint.obj
 0001:000fe240       _$E7                       004ff240 f   Waypoint.obj
 0001:000fe270       _$E9                       004ff270 f   Waypoint.obj
 0001:000fe290       _$E11                      004ff290 f   Waypoint.obj
 0001:000fe2b0       _$E13                      004ff2b0 f   Waypoint.obj
 0001:000fe2d0       _$E15                      004ff2d0 f   Waypoint.obj
 0001:000fe2e0       _$E1                       004ff2e0 f   WorldMap.obj
 0001:000fe300       _$E3                       004ff300 f   WorldMap.obj
 0001:000fe310       _$E5                       004ff310 f   WorldMap.obj
 0001:000fe340       _$E7                       004ff340 f   WorldMap.obj
 0001:000fe370       _$E9                       004ff370 f   WorldMap.obj
 0001:000fe390       _$E11                      004ff390 f   WorldMap.obj
 0001:000fe3b0       _$E13                      004ff3b0 f   WorldMap.obj
 0001:000fe3d0       _$E15                      004ff3d0 f   WorldMap.obj
 0001:000fe3f0       _$E1                       004ff3f0 f   WorldPath.obj
 0001:000fe410       _$E3                       004ff410 f   WorldPath.obj
 0001:000fe420       _$E5                       004ff420 f   WorldPath.obj
 0001:000fe450       _$E7                       004ff450 f   WorldPath.obj
 0001:000fe480       _$E9                       004ff480 f   WorldPath.obj
 0001:000fe4a0       _$E11                      004ff4a0 f   WorldPath.obj
 0001:000fe4c0       _$E13                      004ff4c0 f   WorldPath.obj
 0001:000fe4e0       _$E15                      004ff4e0 f   WorldPath.obj
 0001:000fe500       _$E17                      004ff500 f   WorldPath.obj
 0001:000fe510       _$E1                       004ff510 f   WorldView.obj
 0001:000fe530       _$E3                       004ff530 f   WorldView.obj
 0001:000fe540       _$E5                       004ff540 f   WorldView.obj
 0001:000fe570       _$E7                       004ff570 f   WorldView.obj
 0001:000fe5a0       _$E9                       004ff5a0 f   WorldView.obj
 0001:000fe5c0       _$E11                      004ff5c0 f   WorldView.obj
 0001:000fe5e0       _$E13                      004ff5e0 f   WorldView.obj
 0001:000fe600       _$E15                      004ff600 f   WorldView.obj
 0001:000fe620       _$E17                      004ff620 f   WorldView.obj
 0001:000fe630       _$E1                       004ff630 f   EnvironmentalSound.obj
 0001:000fe650       _$E3                       004ff650 f   EnvironmentalSound.obj
 0001:000fe660       _$E5                       004ff660 f   EnvironmentalSound.obj
 0001:000fe690       _$E7                       004ff690 f   EnvironmentalSound.obj
 0001:000fe6c0       _$E9                       004ff6c0 f   EnvironmentalSound.obj
 0001:000fe6e0       _$E11                      004ff6e0 f   EnvironmentalSound.obj
 0001:000fe700       _$E13                      004ff700 f   EnvironmentalSound.obj
 0001:000fe720       _$E15                      004ff720 f   EnvironmentalSound.obj
 0001:000fe740       _$E17                      004ff740 f   EnvironmentalSound.obj
 0001:000fe770       _$E19                      004ff770 f   EnvironmentalSound.obj
 0001:000fe7b0       _$E21                      004ff7b0 f   EnvironmentalSound.obj
 0001:000fe7d0       _$E23                      004ff7d0 f   EnvironmentalSound.obj
 0001:000fe7f0       _$E25                      004ff7f0 f   EnvironmentalSound.obj
 0001:000fe810       _$E27                      004ff810 f   EnvironmentalSound.obj
 0001:000fe830       _$E29                      004ff830 f   EnvironmentalSound.obj
 0001:000fe850       _$E31                      004ff850 f   EnvironmentalSound.obj
 0001:000fe870       _$E33                      004ff870 f   EnvironmentalSound.obj
 0001:000fe890       _$E35                      004ff890 f   EnvironmentalSound.obj
 0001:000fe8b0       _$E37                      004ff8b0 f   EnvironmentalSound.obj
 0001:000fe8d0       _$E39                      004ff8d0 f   EnvironmentalSound.obj
 0001:000fe8f0       _$E41                      004ff8f0 f   EnvironmentalSound.obj
 0001:000fe910       _$E43                      004ff910 f   EnvironmentalSound.obj
 0001:000fe930       _$E1                       004ff930 f   Sound.obj
 0001:000fe950       _$E3                       004ff950 f   Sound.obj
 0001:000fe960       _$E5                       004ff960 f   Sound.obj
 0001:000fe990       _$E7                       004ff990 f   Sound.obj
 0001:000fe9c0       _$E9                       004ff9c0 f   Sound.obj
 0001:000fe9e0       _$E11                      004ff9e0 f   Sound.obj
 0001:000fea00       _$E13                      004ffa00 f   Sound.obj
 0001:000fea20       _$E15                      004ffa20 f   Sound.obj
 0001:000fea40       _$E17                      004ffa40 f   Sound.obj
 0001:000fea70       _$E19                      004ffa70 f   Sound.obj
 0001:000feab0       _$E21                      004ffab0 f   Sound.obj
 0001:000fead0       _$E23                      004ffad0 f   Sound.obj
 0001:000feaf0       _$E25                      004ffaf0 f   Sound.obj
 0001:000feb10       _$E27                      004ffb10 f   Sound.obj
 0001:000feb30       _$E29                      004ffb30 f   Sound.obj
 0001:000feb50       _$E31                      004ffb50 f   Sound.obj
 0001:000feb70       _$E33                      004ffb70 f   Sound.obj
 0001:000feb90       _$E35                      004ffb90 f   Sound.obj
 0001:000febb0       _$E37                      004ffbb0 f   Sound.obj
 0001:000febd0       _$E39                      004ffbd0 f   Sound.obj
 0001:000febf0       _$E41                      004ffbf0 f   Sound.obj
 0001:000fec10       _$E43                      004ffc10 f   Sound.obj
 0001:000fec30       _$E1                       004ffc30 f   SoundTrack.obj
 0001:000fec50       _$E3                       004ffc50 f   SoundTrack.obj
 0001:000fec60       _$E5                       004ffc60 f   SoundTrack.obj
 0001:000fec90       _$E7                       004ffc90 f   SoundTrack.obj
 0001:000fecc0       _$E9                       004ffcc0 f   SoundTrack.obj
 0001:000fece0       _$E11                      004ffce0 f   SoundTrack.obj
 0001:000fed00       _$E13                      004ffd00 f   SoundTrack.obj
 0001:000fed20       _$E15                      004ffd20 f   SoundTrack.obj
 0001:000fed40       _$E17                      004ffd40 f   SoundTrack.obj
 0001:000fed70       _$E19                      004ffd70 f   SoundTrack.obj
 0001:000fedb0       _$E21                      004ffdb0 f   SoundTrack.obj
 0001:000fedd0       _$E23                      004ffdd0 f   SoundTrack.obj
 0001:000fedf0       _$E25                      004ffdf0 f   SoundTrack.obj
 0001:000fee10       _$E27                      004ffe10 f   SoundTrack.obj
 0001:000fee30       _$E29                      004ffe30 f   SoundTrack.obj
 0001:000fee50       _$E31                      004ffe50 f   SoundTrack.obj
 0001:000fee70       _$E33                      004ffe70 f   SoundTrack.obj
 0001:000fee90       _$E35                      004ffe90 f   SoundTrack.obj
 0001:000feeb0       _$E37                      004ffeb0 f   SoundTrack.obj
 0001:000feed0       _$E39                      004ffed0 f   SoundTrack.obj
 0001:000feef0       _$E41                      004ffef0 f   SoundTrack.obj
 0001:000fef10       _$E43                      004fff10 f   SoundTrack.obj
 0001:000fef30       _$E1                       004fff30 f   ldwarialbold.obj
 0001:000fef50       _$E3                       004fff50 f   ldwarialbold.obj
 0001:000fef60       _$E5                       004fff60 f   ldwarialbold.obj
 0001:000fef90       _$E7                       004fff90 f   ldwarialbold.obj
 0001:000fefc0       _$E9                       004fffc0 f   ldwarialbold.obj
 0001:000fefe0       _$E11                      004fffe0 f   ldwarialbold.obj
 0001:000ff000       _$E13                      00500000 f   ldwarialbold.obj
 0001:000ff020       _$E1                       00500020 f   ldwBurweed27.obj
 0001:000ff040       _$E3                       00500040 f   ldwBurweed27.obj
 0001:000ff050       _$E5                       00500050 f   ldwBurweed27.obj
 0001:000ff080       _$E7                       00500080 f   ldwBurweed27.obj
 0001:000ff0b0       _$E9                       005000b0 f   ldwBurweed27.obj
 0001:000ff0d0       _$E11                      005000d0 f   ldwBurweed27.obj
 0001:000ff0f0       _$E13                      005000f0 f   ldwBurweed27.obj
 0001:000ff110       _$E1                       00500110 f   highscore.obj
 0001:000ff130       _$E3                       00500130 f   highscore.obj
 0001:000ff140       _$E5                       00500140 f   highscore.obj
 0001:000ff170       _$E7                       00500170 f   highscore.obj
 0001:000ff1a0       _$E9                       005001a0 f   highscore.obj
 0001:000ff1c0       _$E11                      005001c0 f   highscore.obj
 0001:000ff1e0       _$E13                      005001e0 f   highscore.obj
 0001:000ff200       _$E1                       00500200 f   Bird.obj
 0001:000ff220       _$E3                       00500220 f   Bird.obj
 0001:000ff230       _$E5                       00500230 f   Bird.obj
 0001:000ff260       _$E7                       00500260 f   Bird.obj
 0001:000ff290       _$E9                       00500290 f   Bird.obj
 0001:000ff2b0       _$E11                      005002b0 f   Bird.obj
 0001:000ff2d0       _$E13                      005002d0 f   Bird.obj
 0001:000ff2f0       _$E15                      005002f0 f   Bird.obj
 0001:000ff310       _$E17                      00500310 f   Bird.obj
 0001:000ff330       _$E19                      00500330 f   Bird.obj
 0001:000ff350       _$E21                      00500350 f   Bird.obj
 0001:000ff370       _$E23                      00500370 f   Bird.obj
 0001:000ff390       _$E25                      00500390 f   Bird.obj
 0001:000ff3b0       _$E27                      005003b0 f   Bird.obj
 0001:000ff3d0       _$E1                       005003d0 f   HummingbirdClass.obj
 0001:000ff3f0       _$E3                       005003f0 f   HummingbirdClass.obj
 0001:000ff400       _$E5                       00500400 f   HummingbirdClass.obj
 0001:000ff430       _$E7                       00500430 f   HummingbirdClass.obj
 0001:000ff460       _$E9                       00500460 f   HummingbirdClass.obj
 0001:000ff480       _$E11                      00500480 f   HummingbirdClass.obj
 0001:000ff4a0       _$E13                      005004a0 f   HummingbirdClass.obj
 0001:000ff4c0       _$E15                      005004c0 f   HummingbirdClass.obj
 0001:000ff4e0       _$E17                      005004e0 f   HummingbirdClass.obj
 0001:000ff510       _$E19                      00500510 f   HummingbirdClass.obj
 0001:000ff550       _$E21                      00500550 f   HummingbirdClass.obj
 0001:000ff570       _$E23                      00500570 f   HummingbirdClass.obj
 0001:000ff590       _$E25                      00500590 f   HummingbirdClass.obj
 0001:000ff5b0       _$E27                      005005b0 f   HummingbirdClass.obj
 0001:000ff5d0       _$E29                      005005d0 f   HummingbirdClass.obj
 0001:000ff5f0       _$E31                      005005f0 f   HummingbirdClass.obj
 0001:000ff610       _$E33                      00500610 f   HummingbirdClass.obj
 0001:000ff630       _$E35                      00500630 f   HummingbirdClass.obj
 0001:000ff650       _$E37                      00500650 f   HummingbirdClass.obj
 0001:000ff670       _$E39                      00500670 f   HummingbirdClass.obj
 0001:000ff690       _$E41                      00500690 f   HummingbirdClass.obj
 0001:000ff6b0       _$E1                       005006b0 f   Shark.obj
 0001:000ff6d0       _$E3                       005006d0 f   Shark.obj
 0001:000ff6e0       _$E5                       005006e0 f   Shark.obj
 0001:000ff710       _$E7                       00500710 f   Shark.obj
 0001:000ff740       _$E9                       00500740 f   Shark.obj
 0001:000ff760       _$E11                      00500760 f   Shark.obj
 0001:000ff780       _$E13                      00500780 f   Shark.obj
 0001:000ff7a0       _$E15                      005007a0 f   Shark.obj
 0001:000ff7c0       _$E17                      005007c0 f   Shark.obj
 0001:000ff7e0       _$E19                      005007e0 f   Shark.obj
 0001:000ff800       _$E21                      00500800 f   Shark.obj
 0001:000ff820       _$E23                      00500820 f   Shark.obj
 0001:000ff840       _$E25                      00500840 f   Shark.obj
 0001:000ff860       _$E27                      00500860 f   Shark.obj
 0001:000ff880       _$E29                      00500880 f   Shark.obj
 0001:000ff890       _$E1                       00500890 f   theButterflyClass.obj
 0001:000ff8b0       _$E3                       005008b0 f   theButterflyClass.obj
 0001:000ff8c0       _$E5                       005008c0 f   theButterflyClass.obj
 0001:000ff8f0       _$E7                       005008f0 f   theButterflyClass.obj
 0001:000ff920       _$E9                       00500920 f   theButterflyClass.obj
 0001:000ff940       _$E11                      00500940 f   theButterflyClass.obj
 0001:000ff960       _$E13                      00500960 f   theButterflyClass.obj
 0001:000ff980       _$E15                      00500980 f   theButterflyClass.obj
 0001:000ff9a0       _$E17                      005009a0 f   theButterflyClass.obj
 0001:000ff9d0       _$E19                      005009d0 f   theButterflyClass.obj
 0001:000ffa10       _$E21                      00500a10 f   theButterflyClass.obj
 0001:000ffa30       _$E23                      00500a30 f   theButterflyClass.obj
 0001:000ffa50       _$E25                      00500a50 f   theButterflyClass.obj
 0001:000ffa70       _$E27                      00500a70 f   theButterflyClass.obj
 0001:000ffa90       _$E29                      00500a90 f   theButterflyClass.obj
 0001:000ffab0       _$E31                      00500ab0 f   theButterflyClass.obj
 0001:000ffad0       _$E33                      00500ad0 f   theButterflyClass.obj
 0001:000ffaf0       _$E35                      00500af0 f   theButterflyClass.obj
 0001:000ffb10       _$E37                      00500b10 f   theButterflyClass.obj
 0001:000ffb30       _$E39                      00500b30 f   theButterflyClass.obj
 0001:000ffb50       _$E41                      00500b50 f   theButterflyClass.obj
 0001:000ffb70       _$E1                       00500b70 f   BFGProtection.obj
 0001:000ffb80       _$E1                       00500b80 f   Distributor.obj
 0001:000ffba0       _$E3                       00500ba0 f   Distributor.obj
 0001:000ffbb0       _$E5                       00500bb0 f   Distributor.obj
 0001:000ffbe0       _$E7                       00500be0 f   Distributor.obj
 0001:000ffc10       _$E9                       00500c10 f   Distributor.obj
 0001:000ffc30       _$E11                      00500c30 f   Distributor.obj
 0001:000ffc50       _$E13                      00500c50 f   Distributor.obj
 0001:000ffc70       _$E15                      00500c70 f   Distributor.obj
 0001:000ffc90       _$E17                      00500c90 f   Distributor.obj
 0001:000ffcb0       _$E19                      00500cb0 f   Distributor.obj
 0001:000ffcd0       _$E21                      00500cd0 f   Distributor.obj
 0001:000ffcf0       _$E23                      00500cf0 f   Distributor.obj
 0001:000ffd10       _$E25                      00500d10 f   Distributor.obj
 0001:000ffd20       _$E1                       00500d20 f   Expiration.obj
 0001:000ffd40       _$E3                       00500d40 f   Expiration.obj
 0001:000ffd50       _$E5                       00500d50 f   Expiration.obj
 0001:000ffd80       _$E7                       00500d80 f   Expiration.obj
 0001:000ffdb0       _$E9                       00500db0 f   Expiration.obj
 0001:000ffdd0       _$E11                      00500dd0 f   Expiration.obj
 0001:000ffdf0       _$E13                      00500df0 f   Expiration.obj
 0001:000ffe10       _$E15                      00500e10 f   Expiration.obj
 0001:000ffe20       _$E1                       00500e20 f   main.obj
 0001:000ffe40       _$E3                       00500e40 f   main.obj
 0001:000ffe50       _$E5                       00500e50 f   main.obj
 0001:000ffe80       _$E7                       00500e80 f   main.obj
 0001:000ffeb0       _$E9                       00500eb0 f   main.obj
 0001:000ffed0       _$E11                      00500ed0 f   main.obj
 0001:000ffef0       _$E13                      00500ef0 f   main.obj
 0001:000fff10       _$E15                      00500f10 f   main.obj
 0001:000fff30       _$E17                      00500f30 f   main.obj
 0001:000fff60       _$E19                      00500f60 f   main.obj
 0001:000fffa0       _$E21                      00500fa0 f   main.obj
 0001:000fffc0       _$E23                      00500fc0 f   main.obj
 0001:000fffe0       _$E25                      00500fe0 f   main.obj
 0001:00100000       _$E27                      00501000 f   main.obj
 0001:00100020       _$E29                      00501020 f   main.obj
 0001:00100040       _$E31                      00501040 f   main.obj
 0001:00100060       _$E33                      00501060 f   main.obj
 0001:00100080       _$E35                      00501080 f   main.obj
 0001:001000a0       _$E37                      005010a0 f   main.obj
 0001:001000c0       _$E39                      005010c0 f   main.obj
 0001:001000e0       _$E41                      005010e0 f   main.obj
 0001:00100100       _$E1                       00501100 f   FoodStore.obj
 0001:00100120       _$E3                       00501120 f   FoodStore.obj
 0001:00100130       _$E5                       00501130 f   FoodStore.obj
 0001:00100160       _$E7                       00501160 f   FoodStore.obj
 0001:00100190       _$E9                       00501190 f   FoodStore.obj
 0001:001001b0       _$E11                      005011b0 f   FoodStore.obj
 0001:001001d0       _$E13                      005011d0 f   FoodStore.obj
 0001:001001f0       _$E15                      005011f0 f   FoodStore.obj
 0001:00100200       _$E1                       00501200 f   GameStats.obj
 0001:00100220       _$E3                       00501220 f   GameStats.obj
 0001:00100230       _$E5                       00501230 f   GameStats.obj
 0001:00100260       _$E7                       00501260 f   GameStats.obj
 0001:00100290       _$E9                       00501290 f   GameStats.obj
 0001:001002b0       _$E11                      005012b0 f   GameStats.obj
 0001:001002d0       _$E13                      005012d0 f   GameStats.obj
 0001:001002f0       _$E15                      005012f0 f   GameStats.obj
 0001:00100310       _$E17                      00501310 f   GameStats.obj
 0001:00100340       _$E19                      00501340 f   GameStats.obj
 0001:00100380       _$E21                      00501380 f   GameStats.obj
 0001:001003a0       _$E23                      005013a0 f   GameStats.obj
 0001:001003c0       _$E25                      005013c0 f   GameStats.obj
 0001:001003e0       _$E27                      005013e0 f   GameStats.obj
 0001:00100400       _$E29                      00501400 f   GameStats.obj
 0001:00100420       _$E31                      00501420 f   GameStats.obj
 0001:00100440       _$E33                      00501440 f   GameStats.obj
 0001:00100460       _$E35                      00501460 f   GameStats.obj
 0001:00100480       _$E37                      00501480 f   GameStats.obj
 0001:001004a0       _$E39                      005014a0 f   GameStats.obj
 0001:001004c0       _$E41                      005014c0 f   GameStats.obj
 0001:001004e0       _$E43                      005014e0 f   GameStats.obj
 0001:001004f0       _$E1                       005014f0 f   GameTime.obj
 0001:00100510       _$E3                       00501510 f   GameTime.obj
 0001:00100520       _$E5                       00501520 f   GameTime.obj
 0001:00100550       _$E7                       00501550 f   GameTime.obj
 0001:00100580       _$E9                       00501580 f   GameTime.obj
 0001:001005a0       _$E11                      005015a0 f   GameTime.obj
 0001:001005c0       _$E13                      005015c0 f   GameTime.obj
 0001:001005e0       _$E15                      005015e0 f   GameTime.obj
 0001:00100600       _$E17                      00501600 f   GameTime.obj
 0001:00100630       _$E19                      00501630 f   GameTime.obj
 0001:00100670       _$E21                      00501670 f   GameTime.obj
 0001:00100690       _$E23                      00501690 f   GameTime.obj
 0001:001006b0       _$E25                      005016b0 f   GameTime.obj
 0001:001006d0       _$E27                      005016d0 f   GameTime.obj
 0001:001006f0       _$E29                      005016f0 f   GameTime.obj
 0001:00100710       _$E31                      00501710 f   GameTime.obj
 0001:00100730       _$E33                      00501730 f   GameTime.obj
 0001:00100750       _$E35                      00501750 f   GameTime.obj
 0001:00100770       _$E37                      00501770 f   GameTime.obj
 0001:00100790       _$E39                      00501790 f   GameTime.obj
 0001:001007b0       _$E41                      005017b0 f   GameTime.obj
 0001:001007d0       _$E43                      005017d0 f   GameTime.obj
 0001:001007e0       _$E1                       005017e0 f   GameTimer.obj
 0001:00100800       _$E3                       00501800 f   GameTimer.obj
 0001:00100810       _$E5                       00501810 f   GameTimer.obj
 0001:00100840       _$E7                       00501840 f   GameTimer.obj
 0001:00100870       _$E9                       00501870 f   GameTimer.obj
 0001:00100890       _$E11                      00501890 f   GameTimer.obj
 0001:001008b0       _$E13                      005018b0 f   GameTimer.obj
 0001:001008d0       _$E15                      005018d0 f   GameTimer.obj
 0001:001008f0       _$E17                      005018f0 f   GameTimer.obj
 0001:00100920       _$E19                      00501920 f   GameTimer.obj
 0001:00100960       _$E21                      00501960 f   GameTimer.obj
 0001:00100980       _$E23                      00501980 f   GameTimer.obj
 0001:001009a0       _$E25                      005019a0 f   GameTimer.obj
 0001:001009c0       _$E27                      005019c0 f   GameTimer.obj
 0001:001009e0       _$E29                      005019e0 f   GameTimer.obj
 0001:00100a00       _$E31                      00501a00 f   GameTimer.obj
 0001:00100a20       _$E33                      00501a20 f   GameTimer.obj
 0001:00100a40       _$E35                      00501a40 f   GameTimer.obj
 0001:00100a60       _$E37                      00501a60 f   GameTimer.obj
 0001:00100a80       _$E39                      00501a80 f   GameTimer.obj
 0001:00100aa0       _$E41                      00501aa0 f   GameTimer.obj
 0001:00100ac0       _$E1                       00501ac0 f   Potion.obj
 0001:00100ae0       _$E3                       00501ae0 f   Potion.obj
 0001:00100af0       _$E5                       00501af0 f   Potion.obj
 0001:00100b20       _$E7                       00501b20 f   Potion.obj
 0001:00100b50       _$E9                       00501b50 f   Potion.obj
 0001:00100b70       _$E11                      00501b70 f   Potion.obj
 0001:00100b90       _$E13                      00501b90 f   Potion.obj
 0001:00100bb0       _$E15                      00501bb0 f   Potion.obj
 0001:00100bd0       _$E17                      00501bd0 f   Potion.obj
 0001:00100bf0       _$E19                      00501bf0 f   Potion.obj
 0001:00100c10       _$E21                      00501c10 f   Potion.obj
 0001:00100c30       _$E23                      00501c30 f   Potion.obj
 0001:00100c50       _$E25                      00501c50 f   Potion.obj
 0001:00100c70       _$E27                      00501c70 f   Potion.obj
 0001:00100ca0       _$E29                      00501ca0 f   Potion.obj
 0001:00100ce0       _$E31                      00501ce0 f   Potion.obj
 0001:00100cf0       _$E1                       00501cf0 f   Tech.obj
 0001:00100d00       _$E1                       00501d00 f   TechPoints.obj
 0001:00100d20       _$E3                       00501d20 f   TechPoints.obj
 0001:00100d30       _$E5                       00501d30 f   TechPoints.obj
 0001:00100d60       _$E7                       00501d60 f   TechPoints.obj
 0001:00100d90       _$E9                       00501d90 f   TechPoints.obj
 0001:00100db0       _$E11                      00501db0 f   TechPoints.obj
 0001:00100dd0       _$E13                      00501dd0 f   TechPoints.obj
 0001:00100df0       _$E15                      00501df0 f   TechPoints.obj
 0001:00100e00       _$E1                       00501e00 f   theGame.obj
 0001:00100e20       _$E3                       00501e20 f   theGame.obj
 0001:00100e30       _$E5                       00501e30 f   theGame.obj
 0001:00100e60       _$E7                       00501e60 f   theGame.obj
 0001:00100e90       _$E9                       00501e90 f   theGame.obj
 0001:00100eb0       _$E11                      00501eb0 f   theGame.obj
 0001:00100ed0       _$E13                      00501ed0 f   theGame.obj
 0001:00100ef0       _$E15                      00501ef0 f   theGame.obj
 0001:00100f10       _$E17                      00501f10 f   theGame.obj
 0001:00100f40       _$E19                      00501f40 f   theGame.obj
 0001:00100f80       _$E21                      00501f80 f   theGame.obj
 0001:00100fa0       _$E23                      00501fa0 f   theGame.obj
 0001:00100fc0       _$E25                      00501fc0 f   theGame.obj
 0001:00100fe0       _$E27                      00501fe0 f   theGame.obj
 0001:00101000       _$E29                      00502000 f   theGame.obj
 0001:00101020       _$E31                      00502020 f   theGame.obj
 0001:00101040       _$E33                      00502040 f   theGame.obj
 0001:00101060       _$E35                      00502060 f   theGame.obj
 0001:00101080       _$E37                      00502080 f   theGame.obj
 0001:001010a0       _$E39                      005020a0 f   theGame.obj
 0001:001010c0       _$E41                      005020c0 f   theGame.obj
 0001:001010e0       _$E43                      005020e0 f   theGame.obj
 0001:00101100       _$E45                      00502100 f   theGame.obj
 0001:00101120       _$E47                      00502120 f   theGame.obj
 0001:00101140       _$E49                      00502140 f   theGame.obj
 0001:00101160       _$E1                       00502160 f   theGameState.obj
 0001:00101180       _$E3                       00502180 f   theGameState.obj
 0001:00101190       _$E5                       00502190 f   theGameState.obj
 0001:001011c0       _$E7                       005021c0 f   theGameState.obj
 0001:001011f0       _$E9                       005021f0 f   theGameState.obj
 0001:00101210       _$E11                      00502210 f   theGameState.obj
 0001:00101230       _$E13                      00502230 f   theGameState.obj
 0001:00101250       _$E15                      00502250 f   theGameState.obj
 0001:00101270       _$E17                      00502270 f   theGameState.obj
 0001:001012a0       _$E19                      005022a0 f   theGameState.obj
 0001:001012e0       _$E21                      005022e0 f   theGameState.obj
 0001:00101300       _$E23                      00502300 f   theGameState.obj
 0001:00101320       _$E25                      00502320 f   theGameState.obj
 0001:00101340       _$E27                      00502340 f   theGameState.obj
 0001:00101360       _$E29                      00502360 f   theGameState.obj
 0001:00101380       _$E31                      00502380 f   theGameState.obj
 0001:001013a0       _$E33                      005023a0 f   theGameState.obj
 0001:001013c0       _$E35                      005023c0 f   theGameState.obj
 0001:001013e0       _$E37                      005023e0 f   theGameState.obj
 0001:00101400       _$E39                      00502400 f   theGameState.obj
 0001:00101420       _$E41                      00502420 f   theGameState.obj
 0001:00101440       _$E43                      00502440 f   theGameState.obj
 0001:00101460       _$E45                      00502460 f   theGameState.obj
 0001:00101480       _$E1                       00502480 f   theRealtimeManager.obj
 0001:001014a0       _$E3                       005024a0 f   theRealtimeManager.obj
 0001:001014b0       _$E5                       005024b0 f   theRealtimeManager.obj
 0001:001014e0       _$E7                       005024e0 f   theRealtimeManager.obj
 0001:00101510       _$E9                       00502510 f   theRealtimeManager.obj
 0001:00101530       _$E11                      00502530 f   theRealtimeManager.obj
 0001:00101550       _$E13                      00502550 f   theRealtimeManager.obj
 0001:00101570       _$E15                      00502570 f   theRealtimeManager.obj
 0001:00101590       _$E17                      00502590 f   theRealtimeManager.obj
 0001:001015c0       _$E19                      005025c0 f   theRealtimeManager.obj
 0001:00101600       _$E21                      00502600 f   theRealtimeManager.obj
 0001:00101620       _$E23                      00502620 f   theRealtimeManager.obj
 0001:00101640       _$E25                      00502640 f   theRealtimeManager.obj
 0001:00101660       _$E27                      00502660 f   theRealtimeManager.obj
 0001:00101680       _$E29                      00502680 f   theRealtimeManager.obj
 0001:001016a0       _$E31                      005026a0 f   theRealtimeManager.obj
 0001:001016c0       _$E33                      005026c0 f   theRealtimeManager.obj
 0001:001016e0       _$E35                      005026e0 f   theRealtimeManager.obj
 0001:00101700       _$E37                      00502700 f   theRealtimeManager.obj
 0001:00101720       _$E39                      00502720 f   theRealtimeManager.obj
 0001:00101740       _$E41                      00502740 f   theRealtimeManager.obj
 0001:00101760       _$E1                       00502760 f   Decal.obj
 0001:00101780       _$E3                       00502780 f   Decal.obj
 0001:00101790       _$E5                       00502790 f   Decal.obj
 0001:001017c0       _$E7                       005027c0 f   Decal.obj
 0001:001017f0       _$E9                       005027f0 f   Decal.obj
 0001:00101810       _$E11                      00502810 f   Decal.obj
 0001:00101830       _$E13                      00502830 f   Decal.obj
 0001:00101850       _$E15                      00502850 f   Decal.obj
 0001:00101870       _$E17                      00502870 f   Decal.obj
 0001:001018a0       _$E19                      005028a0 f   Decal.obj
 0001:001018e0       _$E21                      005028e0 f   Decal.obj
 0001:00101900       _$E23                      00502900 f   Decal.obj
 0001:00101920       _$E25                      00502920 f   Decal.obj
 0001:00101940       _$E27                      00502940 f   Decal.obj
 0001:00101960       _$E29                      00502960 f   Decal.obj
 0001:00101980       _$E31                      00502980 f   Decal.obj
 0001:001019a0       _$E33                      005029a0 f   Decal.obj
 0001:001019c0       _$E35                      005029c0 f   Decal.obj
 0001:001019e0       _$E37                      005029e0 f   Decal.obj
 0001:00101a00       _$E39                      00502a00 f   Decal.obj
 0001:00101a20       _$E41                      00502a20 f   Decal.obj
 0001:00101a40       _$E43                      00502a40 f   Decal.obj
 0001:00101a50       _$E1                       00502a50 f   FloatingAnim.obj
 0001:00101a70       _$E3                       00502a70 f   FloatingAnim.obj
 0001:00101a80       _$E5                       00502a80 f   FloatingAnim.obj
 0001:00101ab0       _$E7                       00502ab0 f   FloatingAnim.obj
 0001:00101ae0       _$E9                       00502ae0 f   FloatingAnim.obj
 0001:00101b00       _$E11                      00502b00 f   FloatingAnim.obj
 0001:00101b20       _$E13                      00502b20 f   FloatingAnim.obj
 0001:00101b40       _$E15                      00502b40 f   FloatingAnim.obj
 0001:00101b60       _$E17                      00502b60 f   FloatingAnim.obj
 0001:00101b80       _$E19                      00502b80 f   FloatingAnim.obj
 0001:00101ba0       _$E21                      00502ba0 f   FloatingAnim.obj
 0001:00101bc0       _$E23                      00502bc0 f   FloatingAnim.obj
 0001:00101be0       _$E25                      00502be0 f   FloatingAnim.obj
 0001:00101c00       _$E27                      00502c00 f   FloatingAnim.obj
 0001:00101c30       _$E29                      00502c30 f   FloatingAnim.obj
 0001:00101c70       _$E31                      00502c70 f   FloatingAnim.obj
 0001:00101c90       _$E33                      00502c90 f   FloatingAnim.obj
 0001:00101cb0       _$E35                      00502cb0 f   FloatingAnim.obj
 0001:00101cd0       _$E37                      00502cd0 f   FloatingAnim.obj
 0001:00101cf0       _$E39                      00502cf0 f   FloatingAnim.obj
 0001:00101d10       _$E41                      00502d10 f   FloatingAnim.obj
 0001:00101d30       _$E43                      00502d30 f   FloatingAnim.obj
 0001:00101d50       _$E1                       00502d50 f   Smoke.obj
 0001:00101d70       _$E3                       00502d70 f   Smoke.obj
 0001:00101d80       _$E5                       00502d80 f   Smoke.obj
 0001:00101db0       _$E7                       00502db0 f   Smoke.obj
 0001:00101de0       _$E9                       00502de0 f   Smoke.obj
 0001:00101e00       _$E11                      00502e00 f   Smoke.obj
 0001:00101e20       _$E13                      00502e20 f   Smoke.obj
 0001:00101e40       _$E15                      00502e40 f   Smoke.obj
 0001:00101e60       _$E17                      00502e60 f   Smoke.obj
 0001:00101e80       _$E19                      00502e80 f   Smoke.obj
 0001:00101ea0       _$E21                      00502ea0 f   Smoke.obj
 0001:00101ec0       _$E23                      00502ec0 f   Smoke.obj
 0001:00101ee0       _$E25                      00502ee0 f   Smoke.obj
 0001:00101ef0       _$E1                       00502ef0 f   BehaviorEditor.obj
 0001:00101f10       _$E3                       00502f10 f   BehaviorEditor.obj
 0001:00101f20       _$E5                       00502f20 f   BehaviorEditor.obj
 0001:00101f50       _$E7                       00502f50 f   BehaviorEditor.obj
 0001:00101f80       _$E9                       00502f80 f   BehaviorEditor.obj
 0001:00101fa0       _$E11                      00502fa0 f   BehaviorEditor.obj
 0001:00101fc0       _$E13                      00502fc0 f   BehaviorEditor.obj
 0001:00101fe0       _$E15                      00502fe0 f   BehaviorEditor.obj
 0001:00102000       _$E17                      00503000 f   BehaviorEditor.obj
 0001:00102030       _$E19                      00503030 f   BehaviorEditor.obj
 0001:00102070       _$E21                      00503070 f   BehaviorEditor.obj
 0001:00102090       _$E23                      00503090 f   BehaviorEditor.obj
 0001:001020b0       _$E25                      005030b0 f   BehaviorEditor.obj
 0001:001020d0       _$E27                      005030d0 f   BehaviorEditor.obj
 0001:001020f0       _$E29                      005030f0 f   BehaviorEditor.obj
 0001:00102110       _$E31                      00503110 f   BehaviorEditor.obj
 0001:00102120       _$E1                       00503120 f   ContentMapEditor.obj
 0001:00102140       _$E3                       00503140 f   ContentMapEditor.obj
 0001:00102150       _$E5                       00503150 f   ContentMapEditor.obj
 0001:00102180       _$E7                       00503180 f   ContentMapEditor.obj
 0001:001021b0       _$E9                       005031b0 f   ContentMapEditor.obj
 0001:001021d0       _$E11                      005031d0 f   ContentMapEditor.obj
 0001:001021f0       _$E13                      005031f0 f   ContentMapEditor.obj
 0001:00102210       _$E15                      00503210 f   ContentMapEditor.obj
 0001:00102230       _$E17                      00503230 f   ContentMapEditor.obj
 0001:00102240       _$E1                       00503240 f   Debugger.obj
 0001:00102260       _$E3                       00503260 f   Debugger.obj
 0001:00102270       _$E5                       00503270 f   Debugger.obj
 0001:001022a0       _$E7                       005032a0 f   Debugger.obj
 0001:001022d0       _$E9                       005032d0 f   Debugger.obj
 0001:001022f0       _$E11                      005032f0 f   Debugger.obj
 0001:00102310       _$E13                      00503310 f   Debugger.obj
 0001:00102330       _$E15                      00503330 f   Debugger.obj
 0001:00102340       _$E1                       00503340 f   Editor.obj
 0001:00102360       _$E3                       00503360 f   Editor.obj
 0001:00102370       _$E5                       00503370 f   Editor.obj
 0001:001023a0       _$E7                       005033a0 f   Editor.obj
 0001:001023d0       _$E9                       005033d0 f   Editor.obj
 0001:001023f0       _$E11                      005033f0 f   Editor.obj
 0001:00102410       _$E13                      00503410 f   Editor.obj
 0001:00102430       _$E15                      00503430 f   Editor.obj
 0001:00102450       _$E17                      00503450 f   Editor.obj
 0001:00102480       _$E19                      00503480 f   Editor.obj
 0001:001024c0       _$E21                      005034c0 f   Editor.obj
 0001:001024e0       _$E23                      005034e0 f   Editor.obj
 0001:00102500       _$E25                      00503500 f   Editor.obj
 0001:00102520       _$E27                      00503520 f   Editor.obj
 0001:00102540       _$E29                      00503540 f   Editor.obj
 0001:00102560       _$E31                      00503560 f   Editor.obj
 0001:00102570       _$E1                       00503570 f   WaypointEditor.obj
 0001:00102590       _$E3                       00503590 f   WaypointEditor.obj
 0001:001025a0       _$E5                       005035a0 f   WaypointEditor.obj
 0001:001025d0       _$E7                       005035d0 f   WaypointEditor.obj
 0001:00102600       _$E9                       00503600 f   WaypointEditor.obj
 0001:00102620       _$E11                      00503620 f   WaypointEditor.obj
 0001:00102640       _$E13                      00503640 f   WaypointEditor.obj
 0001:00102660       _$E15                      00503660 f   WaypointEditor.obj
 0001:00102680       _$E17                      00503680 f   WaypointEditor.obj
 0001:001026a0       _$E19                      005036a0 f   WaypointEditor.obj
 0001:001026c0       _$E21                      005036c0 f   WaypointEditor.obj
 0001:001026e0       _$E23                      005036e0 f   WaypointEditor.obj
 0001:00102700       _$E25                      00503700 f   WaypointEditor.obj
 0001:00102710       _$E1                       00503710 f   Collectable.obj
 0001:00102730       _$E3                       00503730 f   Collectable.obj
 0001:00102740       _$E5                       00503740 f   Collectable.obj
 0001:00102770       _$E7                       00503770 f   Collectable.obj
 0001:001027a0       _$E9                       005037a0 f   Collectable.obj
 0001:001027c0       _$E11                      005037c0 f   Collectable.obj
 0001:001027e0       _$E13                      005037e0 f   Collectable.obj
 0001:00102800       _$E15                      00503800 f   Collectable.obj
 0001:00102820       _$E17                      00503820 f   Collectable.obj
 0001:00102840       _$E19                      00503840 f   Collectable.obj
 0001:00102860       _$E21                      00503860 f   Collectable.obj
 0001:00102880       _$E23                      00503880 f   Collectable.obj
 0001:001028a0       _$E25                      005038a0 f   Collectable.obj
 0001:001028c0       _$E27                      005038c0 f   Collectable.obj
 0001:001028e0       _$E29                      005038e0 f   Collectable.obj
 0001:00102900       _$E31                      00503900 f   Collectable.obj
 0001:00102930       _$E33                      00503930 f   Collectable.obj
 0001:00102950       _$E35                      00503950 f   Collectable.obj
 0001:00102980       _$E37                      00503980 f   Collectable.obj
 0001:001029c0       _$E39                      005039c0 f   Collectable.obj
 0001:001029e0       _$E41                      005039e0 f   Collectable.obj
 0001:00102a00       _$E43                      00503a00 f   Collectable.obj
 0001:00102a20       _$E45                      00503a20 f   Collectable.obj
 0001:00102a40       _$E47                      00503a40 f   Collectable.obj
 0001:00102a60       _$E49                      00503a60 f   Collectable.obj
 0001:00102a70       _$E1                       00503a70 f   CollectableItem.obj
 0001:00102a90       _$E3                       00503a90 f   CollectableItem.obj
 0001:00102aa0       _$E5                       00503aa0 f   CollectableItem.obj
 0001:00102ad0       _$E7                       00503ad0 f   CollectableItem.obj
 0001:00102b00       _$E9                       00503b00 f   CollectableItem.obj
 0001:00102b20       _$E11                      00503b20 f   CollectableItem.obj
 0001:00102b40       _$E13                      00503b40 f   CollectableItem.obj
 0001:00102b60       _$E15                      00503b60 f   CollectableItem.obj
 0001:00102b80       _$E17                      00503b80 f   CollectableItem.obj
 0001:00102bb0       _$E19                      00503bb0 f   CollectableItem.obj
 0001:00102bf0       _$E21                      00503bf0 f   CollectableItem.obj
 0001:00102c10       _$E23                      00503c10 f   CollectableItem.obj
 0001:00102c30       _$E25                      00503c30 f   CollectableItem.obj
 0001:00102c50       _$E27                      00503c50 f   CollectableItem.obj
 0001:00102c70       _$E29                      00503c70 f   CollectableItem.obj
 0001:00102c90       _$E31                      00503c90 f   CollectableItem.obj
 0001:00102cb0       _$E33                      00503cb0 f   CollectableItem.obj
 0001:00102cd0       _$E35                      00503cd0 f   CollectableItem.obj
 0001:00102cf0       _$E37                      00503cf0 f   CollectableItem.obj
 0001:00102d10       _$E39                      00503d10 f   CollectableItem.obj
 0001:00102d30       _$E41                      00503d30 f   CollectableItem.obj
 0001:00102d50       _$E43                      00503d50 f   CollectableItem.obj
 0001:00102d60       _$E1                       00503d60 f   DealerSay.obj
 0001:00102d80       _$E3                       00503d80 f   DealerSay.obj
 0001:00102d90       _$E5                       00503d90 f   DealerSay.obj
 0001:00102dc0       _$E7                       00503dc0 f   DealerSay.obj
 0001:00102df0       _$E9                       00503df0 f   DealerSay.obj
 0001:00102e10       _$E11                      00503e10 f   DealerSay.obj
 0001:00102e30       _$E13                      00503e30 f   DealerSay.obj
 0001:00102e50       _$E15                      00503e50 f   DealerSay.obj
 0001:00102e70       _$E17                      00503e70 f   DealerSay.obj
 0001:00102ea0       _$E19                      00503ea0 f   DealerSay.obj
 0001:00102ee0       _$E21                      00503ee0 f   DealerSay.obj
 0001:00102f00       _$E23                      00503f00 f   DealerSay.obj
 0001:00102f20       _$E25                      00503f20 f   DealerSay.obj
 0001:00102f40       _$E27                      00503f40 f   DealerSay.obj
 0001:00102f60       _$E29                      00503f60 f   DealerSay.obj
 0001:00102f80       _$E31                      00503f80 f   DealerSay.obj
 0001:00102fa0       _$E33                      00503fa0 f   DealerSay.obj
 0001:00102fc0       _$E35                      00503fc0 f   DealerSay.obj
 0001:00102fe0       _$E37                      00503fe0 f   DealerSay.obj
 0001:00103000       _$E39                      00504000 f   DealerSay.obj
 0001:00103020       _$E41                      00504020 f   DealerSay.obj
 0001:00103040       _$E43                      00504040 f   DealerSay.obj
 0001:00103050       _$E1                       00504050 f   SceneManager.obj
 0001:00103070       _$E3                       00504070 f   SceneManager.obj
 0001:00103080       _$E5                       00504080 f   SceneManager.obj
 0001:001030b0       _$E7                       005040b0 f   SceneManager.obj
 0001:001030e0       _$E9                       005040e0 f   SceneManager.obj
 0001:00103100       _$E11                      00504100 f   SceneManager.obj
 0001:00103120       _$E13                      00504120 f   SceneManager.obj
 0001:00103140       _$E15                      00504140 f   SceneManager.obj
 0001:00103160       _$E17                      00504160 f   SceneManager.obj
 0001:00103180       _$E19                      00504180 f   SceneManager.obj
 0001:001031a0       _$E21                      005041a0 f   SceneManager.obj
 0001:001031c0       _$E23                      005041c0 f   SceneManager.obj
 0001:001031e0       _$E25                      005041e0 f   SceneManager.obj
 0001:00103200       _$E27                      00504200 f   SceneManager.obj
 0001:00103230       _$E29                      00504230 f   SceneManager.obj
 0001:00103270       _$E31                      00504270 f   SceneManager.obj
 0001:00103290       _$E33                      00504290 f   SceneManager.obj
 0001:001032b0       _$E35                      005042b0 f   SceneManager.obj
 0001:001032d0       _$E37                      005042d0 f   SceneManager.obj
 0001:001032f0       _$E39                      005042f0 f   SceneManager.obj
 0001:00103310       _$E41                      00504310 f   SceneManager.obj
 0001:00103330       _$E43                      00504330 f   SceneManager.obj
 0001:00103350       _$E45                      00504350 f   SceneManager.obj
 0001:00103370       _$E47                      00504370 f   SceneManager.obj
 0001:00103380       _$E1                       00504380 f   theDealerSay.obj
 0001:001033a0       _$E3                       005043a0 f   theDealerSay.obj
 0001:001033b0       _$E5                       005043b0 f   theDealerSay.obj
 0001:001033e0       _$E7                       005043e0 f   theDealerSay.obj
 0001:00103410       _$E9                       00504410 f   theDealerSay.obj
 0001:00103430       _$E11                      00504430 f   theDealerSay.obj
 0001:00103450       _$E13                      00504450 f   theDealerSay.obj
 0001:00103470       _$E15                      00504470 f   theDealerSay.obj
 0001:00103490       _$E17                      00504490 f   theDealerSay.obj
 0001:001034c0       _$E19                      005044c0 f   theDealerSay.obj
 0001:00103500       _$E21                      00504500 f   theDealerSay.obj
 0001:00103520       _$E23                      00504520 f   theDealerSay.obj
 0001:00103540       _$E25                      00504540 f   theDealerSay.obj
 0001:00103560       _$E27                      00504560 f   theDealerSay.obj
 0001:00103580       _$E29                      00504580 f   theDealerSay.obj
 0001:001035a0       _$E31                      005045a0 f   theDealerSay.obj
 0001:001035c0       _$E33                      005045c0 f   theDealerSay.obj
 0001:001035e0       _$E35                      005045e0 f   theDealerSay.obj
 0001:00103600       _$E37                      00504600 f   theDealerSay.obj
 0001:00103620       _$E39                      00504620 f   theDealerSay.obj
 0001:00103640       _$E41                      00504640 f   theDealerSay.obj
 0001:00103660       _$E1                       00504660 f   theGraphicsManager.obj
 0001:00103680       _$E3                       00504680 f   theGraphicsManager.obj
 0001:00103690       _$E5                       00504690 f   theGraphicsManager.obj
 0001:001036c0       _$E7                       005046c0 f   theGraphicsManager.obj
 0001:001036f0       _$E9                       005046f0 f   theGraphicsManager.obj
 0001:00103710       _$E11                      00504710 f   theGraphicsManager.obj
 0001:00103730       _$E13                      00504730 f   theGraphicsManager.obj
 0001:00103750       _$E15                      00504750 f   theGraphicsManager.obj
 0001:00103770       _$E17                      00504770 f   theGraphicsManager.obj
 0001:00103790       _$E19                      00504790 f   theGraphicsManager.obj
 0001:001037b0       _$E21                      005047b0 f   theGraphicsManager.obj
 0001:001037d0       _$E23                      005047d0 f   theGraphicsManager.obj
 0001:001037f0       _$E25                      005047f0 f   theGraphicsManager.obj
 0001:00103810       _$E27                      00504810 f   theGraphicsManager.obj
 0001:00103840       _$E29                      00504840 f   theGraphicsManager.obj
 0001:00103880       _$E31                      00504880 f   theGraphicsManager.obj
 0001:001038a0       _$E33                      005048a0 f   theGraphicsManager.obj
 0001:001038c0       _$E35                      005048c0 f   theGraphicsManager.obj
 0001:001038e0       _$E37                      005048e0 f   theGraphicsManager.obj
 0001:00103900       _$E39                      00504900 f   theGraphicsManager.obj
 0001:00103920       _$E41                      00504920 f   theGraphicsManager.obj
 0001:00103940       _$E43                      00504940 f   theGraphicsManager.obj
 0001:00103960       _$E45                      00504960 f   theGraphicsManager.obj
 0001:00103980       _$E47                      00504980 f   theGraphicsManager.obj
 0001:001039a0       _$E1                       005049a0 f   thePrizeMsgAssembler.obj
 0001:001039c0       _$E3                       005049c0 f   thePrizeMsgAssembler.obj
 0001:001039d0       _$E5                       005049d0 f   thePrizeMsgAssembler.obj
 0001:00103a00       _$E7                       00504a00 f   thePrizeMsgAssembler.obj
 0001:00103a30       _$E9                       00504a30 f   thePrizeMsgAssembler.obj
 0001:00103a50       _$E11                      00504a50 f   thePrizeMsgAssembler.obj
 0001:00103a70       _$E13                      00504a70 f   thePrizeMsgAssembler.obj
 0001:00103a90       _$E15                      00504a90 f   thePrizeMsgAssembler.obj
 0001:00103ab0       _$E17                      00504ab0 f   thePrizeMsgAssembler.obj
 0001:00103ae0       _$E19                      00504ae0 f   thePrizeMsgAssembler.obj
 0001:00103b20       _$E21                      00504b20 f   thePrizeMsgAssembler.obj
 0001:00103b40       _$E23                      00504b40 f   thePrizeMsgAssembler.obj
 0001:00103b60       _$E25                      00504b60 f   thePrizeMsgAssembler.obj
 0001:00103b80       _$E27                      00504b80 f   thePrizeMsgAssembler.obj
 0001:00103ba0       _$E29                      00504ba0 f   thePrizeMsgAssembler.obj
 0001:00103bc0       _$E31                      00504bc0 f   thePrizeMsgAssembler.obj
 0001:00103be0       _$E33                      00504be0 f   thePrizeMsgAssembler.obj
 0001:00103c00       _$E35                      00504c00 f   thePrizeMsgAssembler.obj
 0001:00103c20       _$E37                      00504c20 f   thePrizeMsgAssembler.obj
 0001:00103c40       _$E39                      00504c40 f   thePrizeMsgAssembler.obj
 0001:00103c60       _$E41                      00504c60 f   thePrizeMsgAssembler.obj
 0001:00103c80       _$E43                      00504c80 f   thePrizeMsgAssembler.obj
 0001:00103ca0       _$E1                       00504ca0 f   theSlicedVariableMeter.obj
 0001:00103cc0       _$E3                       00504cc0 f   theSlicedVariableMeter.obj
 0001:00103cd0       _$E5                       00504cd0 f   theSlicedVariableMeter.obj
 0001:00103d00       _$E7                       00504d00 f   theSlicedVariableMeter.obj
 0001:00103d30       _$E9                       00504d30 f   theSlicedVariableMeter.obj
 0001:00103d50       _$E11                      00504d50 f   theSlicedVariableMeter.obj
 0001:00103d70       _$E13                      00504d70 f   theSlicedVariableMeter.obj
 0001:00103d90       _$E15                      00504d90 f   theSlicedVariableMeter.obj
 0001:00103db0       _$E17                      00504db0 f   theSlicedVariableMeter.obj
 0001:00103de0       _$E19                      00504de0 f   theSlicedVariableMeter.obj
 0001:00103e20       _$E21                      00504e20 f   theSlicedVariableMeter.obj
 0001:00103e40       _$E23                      00504e40 f   theSlicedVariableMeter.obj
 0001:00103e60       _$E25                      00504e60 f   theSlicedVariableMeter.obj
 0001:00103e80       _$E27                      00504e80 f   theSlicedVariableMeter.obj
 0001:00103ea0       _$E29                      00504ea0 f   theSlicedVariableMeter.obj
 0001:00103ec0       _$E31                      00504ec0 f   theSlicedVariableMeter.obj
 0001:00103ee0       _$E33                      00504ee0 f   theSlicedVariableMeter.obj
 0001:00103f00       _$E35                      00504f00 f   theSlicedVariableMeter.obj
 0001:00103f20       _$E37                      00504f20 f   theSlicedVariableMeter.obj
 0001:00103f40       _$E39                      00504f40 f   theSlicedVariableMeter.obj
 0001:00103f60       _$E41                      00504f60 f   theSlicedVariableMeter.obj
 0001:00103f80       _$E43                      00504f80 f   theSlicedVariableMeter.obj
 0001:00103fa0       _$E1                       00504fa0 f   theStringManager.obj
 0001:00103fc0       _$E3                       00504fc0 f   theStringManager.obj
 0001:00103fd0       _$E5                       00504fd0 f   theStringManager.obj
 0001:00104000       _$E7                       00505000 f   theStringManager.obj
 0001:00104030       _$E9                       00505030 f   theStringManager.obj
 0001:00104050       _$E11                      00505050 f   theStringManager.obj
 0001:00104070       _$E13                      00505070 f   theStringManager.obj
 0001:00104090       _$E1                       00505090 f   theVariableMeter.obj
 0001:001040b0       _$E3                       005050b0 f   theVariableMeter.obj
 0001:001040c0       _$E5                       005050c0 f   theVariableMeter.obj
 0001:001040f0       _$E7                       005050f0 f   theVariableMeter.obj
 0001:00104120       _$E9                       00505120 f   theVariableMeter.obj
 0001:00104140       _$E11                      00505140 f   theVariableMeter.obj
 0001:00104160       _$E13                      00505160 f   theVariableMeter.obj
 0001:00104180       _$E15                      00505180 f   theVariableMeter.obj
 0001:001041a0       _$E17                      005051a0 f   theVariableMeter.obj
 0001:001041c0       _$E19                      005051c0 f   theVariableMeter.obj
 0001:001041e0       _$E21                      005051e0 f   theVariableMeter.obj
 0001:00104200       _$E23                      00505200 f   theVariableMeter.obj
 0001:00104220       _$E1                       00505220 f   AlchemyLab.obj
 0001:00104240       _$E3                       00505240 f   AlchemyLab.obj
 0001:00104250       _$E5                       00505250 f   AlchemyLab.obj
 0001:00104280       _$E7                       00505280 f   AlchemyLab.obj
 0001:001042b0       _$E9                       005052b0 f   AlchemyLab.obj
 0001:001042d0       _$E11                      005052d0 f   AlchemyLab.obj
 0001:001042f0       _$E13                      005052f0 f   AlchemyLab.obj
 0001:00104310       _$E15                      00505310 f   AlchemyLab.obj
 0001:00104330       _$E17                      00505330 f   AlchemyLab.obj
 0001:00104350       _$E19                      00505350 f   AlchemyLab.obj
 0001:00104370       _$E21                      00505370 f   AlchemyLab.obj
 0001:00104390       _$E23                      00505390 f   AlchemyLab.obj
 0001:001043b0       _$E25                      005053b0 f   AlchemyLab.obj
 0001:001043d0       _$E27                      005053d0 f   AlchemyLab.obj
 0001:00104400       _$E29                      00505400 f   AlchemyLab.obj
 0001:00104440       _$E33                      00505440 f   AlchemyLab.obj
 0001:00104450       _$E1                       00505450 f   AlchemyPot.obj
 0001:00104470       _$E3                       00505470 f   AlchemyPot.obj
 0001:00104480       _$E5                       00505480 f   AlchemyPot.obj
 0001:001044b0       _$E7                       005054b0 f   AlchemyPot.obj
 0001:001044e0       _$E9                       005054e0 f   AlchemyPot.obj
 0001:00104500       _$E11                      00505500 f   AlchemyPot.obj
 0001:00104520       _$E13                      00505520 f   AlchemyPot.obj
 0001:00104540       _$E15                      00505540 f   AlchemyPot.obj
 0001:00104560       _$E17                      00505560 f   AlchemyPot.obj
 0001:00104580       _$E19                      00505580 f   AlchemyPot.obj
 0001:001045a0       _$E21                      005055a0 f   AlchemyPot.obj
 0001:001045c0       _$E23                      005055c0 f   AlchemyPot.obj
 0001:001045e0       _$E25                      005055e0 f   AlchemyPot.obj
 0001:00104600       _$E27                      00505600 f   AlchemyPot.obj
 0001:00104630       _$E29                      00505630 f   AlchemyPot.obj
 0001:00104670       _$E31                      00505670 f   AlchemyPot.obj
 0001:00104680       _$E1                       00505680 f   AlchemyTable.obj
 0001:001046a0       _$E3                       005056a0 f   AlchemyTable.obj
 0001:001046b0       _$E5                       005056b0 f   AlchemyTable.obj
 0001:001046e0       _$E7                       005056e0 f   AlchemyTable.obj
 0001:00104710       _$E9                       00505710 f   AlchemyTable.obj
 0001:00104730       _$E11                      00505730 f   AlchemyTable.obj
 0001:00104750       _$E13                      00505750 f   AlchemyTable.obj
 0001:00104770       _$E15                      00505770 f   AlchemyTable.obj
 0001:00104790       _$E17                      00505790 f   AlchemyTable.obj
 0001:001047b0       _$E19                      005057b0 f   AlchemyTable.obj
 0001:001047d0       _$E21                      005057d0 f   AlchemyTable.obj
 0001:001047f0       _$E23                      005057f0 f   AlchemyTable.obj
 0001:00104810       _$E25                      00505810 f   AlchemyTable.obj
 0001:00104830       _$E27                      00505830 f   AlchemyTable.obj
 0001:00104860       _$E29                      00505860 f   AlchemyTable.obj
 0001:001048a0       _$E32                      005058a0 f   AlchemyTable.obj
 0001:001048b0       _$E1                       005058b0 f   Aromatherapy.obj
 0001:001048d0       _$E3                       005058d0 f   Aromatherapy.obj
 0001:001048e0       _$E5                       005058e0 f   Aromatherapy.obj
 0001:00104910       _$E7                       00505910 f   Aromatherapy.obj
 0001:00104940       _$E9                       00505940 f   Aromatherapy.obj
 0001:00104960       _$E11                      00505960 f   Aromatherapy.obj
 0001:00104980       _$E13                      00505980 f   Aromatherapy.obj
 0001:001049a0       _$E15                      005059a0 f   Aromatherapy.obj
 0001:001049c0       _$E17                      005059c0 f   Aromatherapy.obj
 0001:001049e0       _$E19                      005059e0 f   Aromatherapy.obj
 0001:00104a00       _$E21                      00505a00 f   Aromatherapy.obj
 0001:00104a20       _$E23                      00505a20 f   Aromatherapy.obj
 0001:00104a40       _$E25                      00505a40 f   Aromatherapy.obj
 0001:00104a60       _$E27                      00505a60 f   Aromatherapy.obj
 0001:00104a90       _$E29                      00505a90 f   Aromatherapy.obj
 0001:00104ad0       _$E31                      00505ad0 f   Aromatherapy.obj
 0001:00104b50       _$E34                      00505b50 f   Aromatherapy.obj
 0001:00104b60       _$E1                       00505b60 f   Bath.obj
 0001:00104b80       _$E3                       00505b80 f   Bath.obj
 0001:00104b90       _$E5                       00505b90 f   Bath.obj
 0001:00104bc0       _$E7                       00505bc0 f   Bath.obj
 0001:00104bf0       _$E9                       00505bf0 f   Bath.obj
 0001:00104c10       _$E11                      00505c10 f   Bath.obj
 0001:00104c30       _$E13                      00505c30 f   Bath.obj
 0001:00104c50       _$E15                      00505c50 f   Bath.obj
 0001:00104c70       _$E17                      00505c70 f   Bath.obj
 0001:00104c90       _$E19                      00505c90 f   Bath.obj
 0001:00104cb0       _$E21                      00505cb0 f   Bath.obj
 0001:00104cd0       _$E23                      00505cd0 f   Bath.obj
 0001:00104cf0       _$E25                      00505cf0 f   Bath.obj
 0001:00104d10       _$E27                      00505d10 f   Bath.obj
 0001:00104d30       _$E29                      00505d30 f   Bath.obj
 0001:00104d60       _$E31                      00505d60 f   Bath.obj
 0001:00104da0       _$E33                      00505da0 f   Bath.obj
 0001:00104dc0       _$E35                      00505dc0 f   Bath.obj
 0001:00104de0       _$E37                      00505de0 f   Bath.obj
 0001:00104df0       _$E1                       00505df0 f   BeeHive.obj
 0001:00104e10       _$E3                       00505e10 f   BeeHive.obj
 0001:00104e20       _$E5                       00505e20 f   BeeHive.obj
 0001:00104e50       _$E7                       00505e50 f   BeeHive.obj
 0001:00104e80       _$E9                       00505e80 f   BeeHive.obj
 0001:00104ea0       _$E11                      00505ea0 f   BeeHive.obj
 0001:00104ec0       _$E13                      00505ec0 f   BeeHive.obj
 0001:00104ee0       _$E15                      00505ee0 f   BeeHive.obj
 0001:00104f00       _$E17                      00505f00 f   BeeHive.obj
 0001:00104f20       _$E19                      00505f20 f   BeeHive.obj
 0001:00104f50       _$E21                      00505f50 f   BeeHive.obj
 0001:00104f90       _$E23                      00505f90 f   BeeHive.obj
 0001:00104fb0       _$E25                      00505fb0 f   BeeHive.obj
 0001:00104fd0       _$E27                      00505fd0 f   BeeHive.obj
 0001:00104ff0       _$E29                      00505ff0 f   BeeHive.obj
 0001:00105010       _$E31                      00506010 f   BeeHive.obj
 0001:00105030       _$E33                      00506030 f   BeeHive.obj
 0001:00105050       _$E35                      00506050 f   BeeHive.obj
 0001:00105070       _$E37                      00506070 f   BeeHive.obj
 0001:00105090       _$E39                      00506090 f   BeeHive.obj
 0001:001050b0       _$E41                      005060b0 f   BeeHive.obj
 0001:001050d0       _$E43                      005060d0 f   BeeHive.obj
 0001:001050f0       _$E45                      005060f0 f   BeeHive.obj
 0001:00105100       _$E1                       00506100 f   ChalkBoard.obj
 0001:00105120       _$E3                       00506120 f   ChalkBoard.obj
 0001:00105130       _$E5                       00506130 f   ChalkBoard.obj
 0001:00105160       _$E7                       00506160 f   ChalkBoard.obj
 0001:00105190       _$E9                       00506190 f   ChalkBoard.obj
 0001:001051b0       _$E11                      005061b0 f   ChalkBoard.obj
 0001:001051d0       _$E13                      005061d0 f   ChalkBoard.obj
 0001:001051f0       _$E15                      005061f0 f   ChalkBoard.obj
 0001:00105210       _$E17                      00506210 f   ChalkBoard.obj
 0001:00105230       _$E19                      00506230 f   ChalkBoard.obj
 0001:00105250       _$E21                      00506250 f   ChalkBoard.obj
 0001:00105270       _$E23                      00506270 f   ChalkBoard.obj
 0001:00105290       _$E25                      00506290 f   ChalkBoard.obj
 0001:001052b0       _$E27                      005062b0 f   ChalkBoard.obj
 0001:001052c0       _$E1                       005062c0 f   Chief.obj
 0001:001052e0       _$E3                       005062e0 f   Chief.obj
 0001:001052f0       _$E5                       005062f0 f   Chief.obj
 0001:00105320       _$E7                       00506320 f   Chief.obj
 0001:00105350       _$E9                       00506350 f   Chief.obj
 0001:00105370       _$E11                      00506370 f   Chief.obj
 0001:00105390       _$E13                      00506390 f   Chief.obj
 0001:001053b0       _$E15                      005063b0 f   Chief.obj
 0001:001053d0       _$E17                      005063d0 f   Chief.obj
 0001:00105400       _$E19                      00506400 f   Chief.obj
 0001:00105440       _$E21                      00506440 f   Chief.obj
 0001:00105460       _$E23                      00506460 f   Chief.obj
 0001:00105480       _$E25                      00506480 f   Chief.obj
 0001:001054a0       _$E27                      005064a0 f   Chief.obj
 0001:001054c0       _$E29                      005064c0 f   Chief.obj
 0001:001054e0       _$E31                      005064e0 f   Chief.obj
 0001:00105500       _$E33                      00506500 f   Chief.obj
 0001:00105520       _$E35                      00506520 f   Chief.obj
 0001:00105540       _$E37                      00506540 f   Chief.obj
 0001:00105560       _$E39                      00506560 f   Chief.obj
 0001:00105580       _$E41                      00506580 f   Chief.obj
 0001:001055a0       _$E43                      005065a0 f   Chief.obj
 0001:001055c0       _$E45                      005065c0 f   Chief.obj
 0001:001055e0       _$E47                      005065e0 f   Chief.obj
 0001:001055f0       _$E1                       005065f0 f   Construction.obj
 0001:00105610       _$E3                       00506610 f   Construction.obj
 0001:00105620       _$E5                       00506620 f   Construction.obj
 0001:00105650       _$E7                       00506650 f   Construction.obj
 0001:00105680       _$E9                       00506680 f   Construction.obj
 0001:001056a0       _$E11                      005066a0 f   Construction.obj
 0001:001056c0       _$E13                      005066c0 f   Construction.obj
 0001:001056e0       _$E15                      005066e0 f   Construction.obj
 0001:00105700       _$E17                      00506700 f   Construction.obj
 0001:00105730       _$E19                      00506730 f   Construction.obj
 0001:00105770       _$E21                      00506770 f   Construction.obj
 0001:00105790       _$E23                      00506790 f   Construction.obj
 0001:001057b0       _$E25                      005067b0 f   Construction.obj
 0001:001057d0       _$E27                      005067d0 f   Construction.obj
 0001:001057f0       _$E29                      005067f0 f   Construction.obj
 0001:00105810       _$E31                      00506810 f   Construction.obj
 0001:00105870       _$E33                      00506870 f   Construction.obj
 0001:00105880       _$E1                       00506880 f   DoorKey.obj
 0001:001058a0       _$E3                       005068a0 f   DoorKey.obj
 0001:001058b0       _$E5                       005068b0 f   DoorKey.obj
 0001:001058e0       _$E7                       005068e0 f   DoorKey.obj
 0001:00105910       _$E9                       00506910 f   DoorKey.obj
 0001:00105930       _$E11                      00506930 f   DoorKey.obj
 0001:00105950       _$E13                      00506950 f   DoorKey.obj
 0001:00105970       _$E15                      00506970 f   DoorKey.obj
 0001:00105990       _$E17                      00506990 f   DoorKey.obj
 0001:001059b0       _$E19                      005069b0 f   DoorKey.obj
 0001:001059d0       _$E21                      005069d0 f   DoorKey.obj
 0001:001059f0       _$E23                      005069f0 f   DoorKey.obj
 0001:00105a10       _$E25                      00506a10 f   DoorKey.obj
 0001:00105a30       _$E27                      00506a30 f   DoorKey.obj
 0001:00105a60       _$E29                      00506a60 f   DoorKey.obj
 0001:00105aa0       _$E31                      00506aa0 f   DoorKey.obj
 0001:00105ac0       _$E33                      00506ac0 f   DoorKey.obj
 0001:00105ae0       _$E35                      00506ae0 f   DoorKey.obj
 0001:00105b00       _$E37                      00506b00 f   DoorKey.obj
 0001:00105b20       _$E39                      00506b20 f   DoorKey.obj
 0001:00105b40       _$E41                      00506b40 f   DoorKey.obj
 0001:00105c80       _$E43                      00506c80 f   DoorKey.obj
 0001:00105c90       _$E1                       00506c90 f   FirePit.obj
 0001:00105cb0       _$E3                       00506cb0 f   FirePit.obj
 0001:00105cc0       _$E5                       00506cc0 f   FirePit.obj
 0001:00105cf0       _$E7                       00506cf0 f   FirePit.obj
 0001:00105d20       _$E9                       00506d20 f   FirePit.obj
 0001:00105d40       _$E11                      00506d40 f   FirePit.obj
 0001:00105d60       _$E13                      00506d60 f   FirePit.obj
 0001:00105d80       _$E15                      00506d80 f   FirePit.obj
 0001:00105da0       _$E17                      00506da0 f   FirePit.obj
 0001:00105dc0       _$E19                      00506dc0 f   FirePit.obj
 0001:00105de0       _$E21                      00506de0 f   FirePit.obj
 0001:00105e00       _$E23                      00506e00 f   FirePit.obj
 0001:00105e20       _$E25                      00506e20 f   FirePit.obj
 0001:00105e40       _$E27                      00506e40 f   FirePit.obj
 0001:00105e60       _$E29                      00506e60 f   FirePit.obj
 0001:00105e90       _$E31                      00506e90 f   FirePit.obj
 0001:00105ed0       _$E33                      00506ed0 f   FirePit.obj
 0001:00105ee0       _$E1                       00506ee0 f   Orchard.obj
 0001:00105f00       _$E3                       00506f00 f   Orchard.obj
 0001:00105f10       _$E5                       00506f10 f   Orchard.obj
 0001:00105f40       _$E7                       00506f40 f   Orchard.obj
 0001:00105f70       _$E9                       00506f70 f   Orchard.obj
 0001:00105f90       _$E11                      00506f90 f   Orchard.obj
 0001:00105fb0       _$E13                      00506fb0 f   Orchard.obj
 0001:00105fd0       _$E15                      00506fd0 f   Orchard.obj
 0001:00105ff0       _$E17                      00506ff0 f   Orchard.obj
 0001:00106020       _$E19                      00507020 f   Orchard.obj
 0001:00106060       _$E21                      00507060 f   Orchard.obj
 0001:00106080       _$E23                      00507080 f   Orchard.obj
 0001:001060a0       _$E25                      005070a0 f   Orchard.obj
 0001:001060c0       _$E27                      005070c0 f   Orchard.obj
 0001:001060e0       _$E29                      005070e0 f   Orchard.obj
 0001:00106100       _$E31                      00507100 f   Orchard.obj
 0001:00106120       _$E33                      00507120 f   Orchard.obj
 0001:00106140       _$E35                      00507140 f   Orchard.obj
 0001:00106160       _$E37                      00507160 f   Orchard.obj
 0001:00106180       _$E39                      00507180 f   Orchard.obj
 0001:001061a0       _$E41                      005071a0 f   Orchard.obj
 0001:001061c0       _$E44                      005071c0 f   Orchard.obj
 0001:001061d0       _$E1                       005071d0 f   PrincessStatue.obj
 0001:001061f0       _$E3                       005071f0 f   PrincessStatue.obj
 0001:00106200       _$E5                       00507200 f   PrincessStatue.obj
 0001:00106230       _$E7                       00507230 f   PrincessStatue.obj
 0001:00106260       _$E9                       00507260 f   PrincessStatue.obj
 0001:00106280       _$E11                      00507280 f   PrincessStatue.obj
 0001:001062a0       _$E13                      005072a0 f   PrincessStatue.obj
 0001:001062c0       _$E15                      005072c0 f   PrincessStatue.obj
 0001:001062e0       _$E17                      005072e0 f   PrincessStatue.obj
 0001:00106330       _$E19                      00507330 f   PrincessStatue.obj
 0001:00106350       _$E21                      00507350 f   PrincessStatue.obj
 0001:00106370       _$E23                      00507370 f   PrincessStatue.obj
 0001:001063a0       _$E25                      005073a0 f   PrincessStatue.obj
 0001:001063e0       _$E27                      005073e0 f   PrincessStatue.obj
 0001:00106400       _$E29                      00507400 f   PrincessStatue.obj
 0001:00106420       _$E31                      00507420 f   PrincessStatue.obj
 0001:00106440       _$E33                      00507440 f   PrincessStatue.obj
 0001:00106460       _$E35                      00507460 f   PrincessStatue.obj
 0001:00106480       _$E37                      00507480 f   PrincessStatue.obj
 0001:001065e0       _$E39                      005075e0 f   PrincessStatue.obj
 0001:001065f0       _$E1                       005075f0 f   Puzzle.obj
 0001:00106610       _$E3                       00507610 f   Puzzle.obj
 0001:00106620       _$E5                       00507620 f   Puzzle.obj
 0001:00106650       _$E7                       00507650 f   Puzzle.obj
 0001:00106680       _$E9                       00507680 f   Puzzle.obj
 0001:001066a0       _$E11                      005076a0 f   Puzzle.obj
 0001:001066c0       _$E13                      005076c0 f   Puzzle.obj
 0001:001066e0       _$E15                      005076e0 f   Puzzle.obj
 0001:00106700       _$E17                      00507700 f   Puzzle.obj
 0001:00106730       _$E19                      00507730 f   Puzzle.obj
 0001:00106770       _$E21                      00507770 f   Puzzle.obj
 0001:00106790       _$E23                      00507790 f   Puzzle.obj
 0001:001067b0       _$E25                      005077b0 f   Puzzle.obj
 0001:001067d0       _$E27                      005077d0 f   Puzzle.obj
 0001:001067f0       _$E29                      005077f0 f   Puzzle.obj
 0001:00106810       _$E31                      00507810 f   Puzzle.obj
 0001:00106830       _$E33                      00507830 f   Puzzle.obj
 0001:00106850       _$E35                      00507850 f   Puzzle.obj
 0001:00106870       _$E37                      00507870 f   Puzzle.obj
 0001:00106890       _$E39                      00507890 f   Puzzle.obj
 0001:001068b0       _$E41                      005078b0 f   Puzzle.obj
 0001:001068d0       _$E43                      005078d0 f   Puzzle.obj
 0001:001068f0       _$E45                      005078f0 f   Puzzle.obj
 0001:00106910       _$E47                      00507910 f   Puzzle.obj
 0001:00106930       _$E49                      00507930 f   Puzzle.obj
 0001:00106950       _$E51                      00507950 f   Puzzle.obj
 0001:00106970       _$E53                      00507970 f   Puzzle.obj
 0001:00106990       _$E55                      00507990 f   Puzzle.obj
 0001:001069b0       _$E57                      005079b0 f   Puzzle.obj
 0001:001069d0       _$E59                      005079d0 f   Puzzle.obj
 0001:00106a20       _$E61                      00507a20 f   Puzzle.obj
 0001:00106a40       _$E63                      00507a40 f   Puzzle.obj
 0001:00106a60       _$E65                      00507a60 f   Puzzle.obj
 0001:00106a80       _$E67                      00507a80 f   Puzzle.obj
 0001:00106aa0       _$E69                      00507aa0 f   Puzzle.obj
 0001:00106ad0       _$E71                      00507ad0 f   Puzzle.obj
 0001:00106af0       _$E73                      00507af0 f   Puzzle.obj
 0001:00106b10       _$E75                      00507b10 f   Puzzle.obj
 0001:00106b40       _$E77                      00507b40 f   Puzzle.obj
 0001:00106b60       _$E79                      00507b60 f   Puzzle.obj
 0001:00106b70       _$E1                       00507b70 f   RainLift.obj
 0001:00106b90       _$E3                       00507b90 f   RainLift.obj
 0001:00106ba0       _$E5                       00507ba0 f   RainLift.obj
 0001:00106bd0       _$E7                       00507bd0 f   RainLift.obj
 0001:00106c00       _$E9                       00507c00 f   RainLift.obj
 0001:00106c20       _$E11                      00507c20 f   RainLift.obj
 0001:00106c40       _$E13                      00507c40 f   RainLift.obj
 0001:00106c60       _$E15                      00507c60 f   RainLift.obj
 0001:00106c80       _$E17                      00507c80 f   RainLift.obj
 0001:00106ca0       _$E19                      00507ca0 f   RainLift.obj
 0001:00106cc0       _$E21                      00507cc0 f   RainLift.obj
 0001:00106ce0       _$E23                      00507ce0 f   RainLift.obj
 0001:00106d00       _$E25                      00507d00 f   RainLift.obj
 0001:00106d20       _$E27                      00507d20 f   RainLift.obj
 0001:00106d40       _$E29                      00507d40 f   RainLift.obj
 0001:00106d60       _$E31                      00507d60 f   RainLift.obj
 0001:00106d80       _$E33                      00507d80 f   RainLift.obj
 0001:00106db0       _$E35                      00507db0 f   RainLift.obj
 0001:00106df0       _$E37                      00507df0 f   RainLift.obj
 0001:00106e00       _$E1                       00507e00 f   RosterOfTheDead.obj
 0001:00106e20       _$E3                       00507e20 f   RosterOfTheDead.obj
 0001:00106e30       _$E5                       00507e30 f   RosterOfTheDead.obj
 0001:00106e60       _$E7                       00507e60 f   RosterOfTheDead.obj
 0001:00106e90       _$E9                       00507e90 f   RosterOfTheDead.obj
 0001:00106eb0       _$E11                      00507eb0 f   RosterOfTheDead.obj
 0001:00106ed0       _$E13                      00507ed0 f   RosterOfTheDead.obj
 0001:00106ef0       _$E15                      00507ef0 f   RosterOfTheDead.obj
 0001:00106f10       _$E17                      00507f10 f   RosterOfTheDead.obj
 0001:00106f30       _$E19                      00507f30 f   RosterOfTheDead.obj
 0001:00106f50       _$E21                      00507f50 f   RosterOfTheDead.obj
 0001:00106f70       _$E23                      00507f70 f   RosterOfTheDead.obj
 0001:00106f90       _$E25                      00507f90 f   RosterOfTheDead.obj
 0001:00106fb0       _$E27                      00507fb0 f   RosterOfTheDead.obj
 0001:00106fd0       _$E29                      00507fd0 f   RosterOfTheDead.obj
 0001:00107000       _$E31                      00508000 f   RosterOfTheDead.obj
 0001:00107040       _$E34                      00508040 f   RosterOfTheDead.obj
 0001:00107050       _$E1                       00508050 f   Ruins.obj
 0001:00107070       _$E3                       00508070 f   Ruins.obj
 0001:00107080       _$E5                       00508080 f   Ruins.obj
 0001:001070b0       _$E7                       005080b0 f   Ruins.obj
 0001:001070e0       _$E9                       005080e0 f   Ruins.obj
 0001:00107100       _$E11                      00508100 f   Ruins.obj
 0001:00107120       _$E13                      00508120 f   Ruins.obj
 0001:00107140       _$E15                      00508140 f   Ruins.obj
 0001:00107170       _$E17                      00508170 f   Ruins.obj
 0001:00107190       _$E19                      00508190 f   Ruins.obj
 0001:001071b0       _$E21                      005081b0 f   Ruins.obj
 0001:001071d0       _$E23                      005081d0 f   Ruins.obj
 0001:001071f0       _$E25                      005081f0 f   Ruins.obj
 0001:00107210       _$E27                      00508210 f   Ruins.obj
 0001:00107230       _$E29                      00508230 f   Ruins.obj
 0001:00107260       _$E31                      00508260 f   Ruins.obj
 0001:001072a0       _$E34                      005082a0 f   Ruins.obj
 0001:001072b0       _$E1                       005082b0 f   SharkCharmer.obj
 0001:001072d0       _$E3                       005082d0 f   SharkCharmer.obj
 0001:001072e0       _$E5                       005082e0 f   SharkCharmer.obj
 0001:00107310       _$E7                       00508310 f   SharkCharmer.obj
 0001:00107340       _$E9                       00508340 f   SharkCharmer.obj
 0001:00107360       _$E11                      00508360 f   SharkCharmer.obj
 0001:00107380       _$E13                      00508380 f   SharkCharmer.obj
 0001:001073a0       _$E15                      005083a0 f   SharkCharmer.obj
 0001:001073c0       _$E17                      005083c0 f   SharkCharmer.obj
 0001:001073e0       _$E19                      005083e0 f   SharkCharmer.obj
 0001:00107410       _$E21                      00508410 f   SharkCharmer.obj
 0001:00107450       _$E23                      00508450 f   SharkCharmer.obj
 0001:00107470       _$E25                      00508470 f   SharkCharmer.obj
 0001:00107490       _$E27                      00508490 f   SharkCharmer.obj
 0001:001074b0       _$E29                      005084b0 f   SharkCharmer.obj
 0001:001074d0       _$E31                      005084d0 f   SharkCharmer.obj
 0001:001074f0       _$E33                      005084f0 f   SharkCharmer.obj
 0001:00107500       _$E1                       00508500 f   SunDisk.obj
 0001:00107520       _$E3                       00508520 f   SunDisk.obj
 0001:00107530       _$E5                       00508530 f   SunDisk.obj
 0001:00107560       _$E7                       00508560 f   SunDisk.obj
 0001:00107590       _$E9                       00508590 f   SunDisk.obj
 0001:001075b0       _$E11                      005085b0 f   SunDisk.obj
 0001:001075d0       _$E13                      005085d0 f   SunDisk.obj
 0001:001075f0       _$E15                      005085f0 f   SunDisk.obj
 0001:00107610       _$E17                      00508610 f   SunDisk.obj
 0001:00107640       _$E19                      00508640 f   SunDisk.obj
 0001:00107660       _$E21                      00508660 f   SunDisk.obj
 0001:00107680       _$E23                      00508680 f   SunDisk.obj
 0001:001076a0       _$E25                      005086a0 f   SunDisk.obj
 0001:001076c0       _$E27                      005086c0 f   SunDisk.obj
 0001:001076e0       _$E29                      005086e0 f   SunDisk.obj
 0001:00107700       _$E31                      00508700 f   SunDisk.obj
 0001:00107720       _$E33                      00508720 f   SunDisk.obj
 0001:00107750       _$E35                      00508750 f   SunDisk.obj
 0001:00107790       _$E37                      00508790 f   SunDisk.obj
 0001:001077a0       _$E1                       005087a0 f   WeatherDance.obj
 0001:001077c0       _$E3                       005087c0 f   WeatherDance.obj
 0001:001077d0       _$E5                       005087d0 f   WeatherDance.obj
 0001:00107800       _$E7                       00508800 f   WeatherDance.obj
 0001:00107830       _$E9                       00508830 f   WeatherDance.obj
 0001:00107850       _$E11                      00508850 f   WeatherDance.obj
 0001:00107870       _$E13                      00508870 f   WeatherDance.obj
 0001:00107890       _$E15                      00508890 f   WeatherDance.obj
 0001:001078b0       _$E17                      005088b0 f   WeatherDance.obj
 0001:001078e0       _$E19                      005088e0 f   WeatherDance.obj
 0001:00107920       _$E21                      00508920 f   WeatherDance.obj
 0001:00107940       _$E23                      00508940 f   WeatherDance.obj
 0001:00107960       _$E25                      00508960 f   WeatherDance.obj
 0001:00107980       _$E27                      00508980 f   WeatherDance.obj
 0001:001079a0       _$E29                      005089a0 f   WeatherDance.obj
 0001:001079c0       _$E31                      005089c0 f   WeatherDance.obj
 0001:001079d0       _$E1                       005089d0 f   MoviePlayer.obj
 0001:001079f0       _$E3                       005089f0 f   MoviePlayer.obj
 0001:00107a00       _$E5                       00508a00 f   MoviePlayer.obj
 0001:00107a30       _$E7                       00508a30 f   MoviePlayer.obj
 0001:00107a60       _$E9                       00508a60 f   MoviePlayer.obj
 0001:00107a80       _$E11                      00508a80 f   MoviePlayer.obj
 0001:00107aa0       _$E13                      00508aa0 f   MoviePlayer.obj
 0001:00107ac0       _$E15                      00508ac0 f   MoviePlayer.obj
 0001:00107ae0       _$E1                       00508ae0 f   FlashPlayer.obj
 0001:00107b00       _$E5                       00508b00 f   FlashPlayer.obj
 0001:00107b20       _$E1                       00508b20 f   Achievement.obj
 0001:00107b40       _$E3                       00508b40 f   Achievement.obj
 0001:00107b50       _$E5                       00508b50 f   Achievement.obj
 0001:00107b80       _$E7                       00508b80 f   Achievement.obj
 0001:00107bb0       _$E9                       00508bb0 f   Achievement.obj
 0001:00107bd0       _$E11                      00508bd0 f   Achievement.obj
 0001:00107bf0       _$E13                      00508bf0 f   Achievement.obj
 0001:00107c10       _$E15                      00508c10 f   Achievement.obj
 0001:00107c30       _$E17                      00508c30 f   Achievement.obj
 0001:00107c60       _$E19                      00508c60 f   Achievement.obj
 0001:00107ca0       _$E21                      00508ca0 f   Achievement.obj
 0001:00107cc0       _$E23                      00508cc0 f   Achievement.obj
 0001:00107ce0       _$E25                      00508ce0 f   Achievement.obj
 0001:00107d00       _$E27                      00508d00 f   Achievement.obj
 0001:00107d20       _$E29                      00508d20 f   Achievement.obj
 0001:00107d40       _$E31                      00508d40 f   Achievement.obj
 0001:00107d60       _$E33                      00508d60 f   Achievement.obj
 0001:00107d80       _$E35                      00508d80 f   Achievement.obj
 0001:00107da0       _$E37                      00508da0 f   Achievement.obj
 0001:00107dc0       _$E39                      00508dc0 f   Achievement.obj
 0001:00107de0       _$E41                      00508de0 f   Achievement.obj
 0001:00107e00       _$E43                      00508e00 f   Achievement.obj
 0001:00107e10       _$E1                       00508e10 f   TutorialTip.obj
 0001:00107e30       _$E3                       00508e30 f   TutorialTip.obj
 0001:00107e40       _$E5                       00508e40 f   TutorialTip.obj
 0001:00107e70       _$E7                       00508e70 f   TutorialTip.obj
 0001:00107ea0       _$E9                       00508ea0 f   TutorialTip.obj
 0001:00107ec0       _$E11                      00508ec0 f   TutorialTip.obj
 0001:00107ee0       _$E13                      00508ee0 f   TutorialTip.obj
 0001:00107f00       _$E15                      00508f00 f   TutorialTip.obj
 0001:00107f20       _$E17                      00508f20 f   TutorialTip.obj
 0001:00107f50       _$E19                      00508f50 f   TutorialTip.obj
 0001:00107f90       _$E21                      00508f90 f   TutorialTip.obj
 0001:00107fb0       _$E23                      00508fb0 f   TutorialTip.obj
 0001:00107fd0       _$E25                      00508fd0 f   TutorialTip.obj
 0001:00107ff0       _$E27                      00508ff0 f   TutorialTip.obj
 0001:00108010       _$E29                      00509010 f   TutorialTip.obj
 0001:00108030       _$E31                      00509030 f   TutorialTip.obj
 0001:00108050       _$E33                      00509050 f   TutorialTip.obj
 0001:00108070       _$E35                      00509070 f   TutorialTip.obj
 0001:00108090       _$E37                      00509090 f   TutorialTip.obj
 0001:001080b0       _$E39                      005090b0 f   TutorialTip.obj
 0001:001080d0       _$E41                      005090d0 f   TutorialTip.obj
 0001:001080f0       _$E43                      005090f0 f   TutorialTip.obj
 0001:00108100       _$E1                       00509100 f   Pages.obj
 0001:00108120       _$E3                       00509120 f   Pages.obj
 0001:00108130       _$E5                       00509130 f   Pages.obj
 0001:00108160       _$E7                       00509160 f   Pages.obj
 0001:00108190       _$E9                       00509190 f   Pages.obj
 0001:001081b0       _$E11                      005091b0 f   Pages.obj
 0001:001081d0       _$E13                      005091d0 f   Pages.obj
 0001:001081f0       _$E15                      005091f0 f   Pages.obj
 0001:00108210       _$E17                      00509210 f   Pages.obj
 0001:00108230       _$E19                      00509230 f   Pages.obj
 0001:00108250       _$E21                      00509250 f   Pages.obj
 0001:00108270       _$E23                      00509270 f   Pages.obj
 0001:00108290       _$E25                      00509290 f   Pages.obj
 0001:001082a0       _$E27                      005092a0 f   Pages.obj
 0001:001082b0       _$E29                      005092b0 f   Pages.obj
 0001:001082c0       _$E31                      005092c0 f   Pages.obj
 0001:001082d0       _$E33                      005092d0 f   Pages.obj
 0001:001082e0       _$E35                      005092e0 f   Pages.obj
 0001:001082f0       _$E37                      005092f0 f   Pages.obj
 0001:00108300       _$E39                      00509300 f   Pages.obj
 0001:00108310       _$E41                      00509310 f   Pages.obj
 0001:00108320       _$E43                      00509320 f   Pages.obj
 0001:00108330       _$E45                      00509330 f   Pages.obj
 0001:00108340       _$E47                      00509340 f   Pages.obj
 0001:00108350       _$E1                       00509350 f   Story.obj
 0001:00108370       _$E3                       00509370 f   Story.obj
 0001:00108380       _$E5                       00509380 f   Story.obj
 0001:001083b0       _$E7                       005093b0 f   Story.obj
 0001:001083e0       _$E9                       005093e0 f   Story.obj
 0001:00108400       _$E11                      00509400 f   Story.obj
 0001:00108420       _$E13                      00509420 f   Story.obj
 0001:00108440       _$E15                      00509440 f   Story.obj
 0001:00108460       _$E17                      00509460 f   Story.obj
 0001:00108480       _$E19                      00509480 f   Story.obj
 0001:001084a0       _$E21                      005094a0 f   Story.obj
 0001:001084c0       _$E23                      005094c0 f   Story.obj
 0001:001084e0       _$E25                      005094e0 f   Story.obj
 0001:00108500       _$E27                      00509500 f   Story.obj
 0001:00108530       _$E29                      00509530 f   Story.obj
 0001:00108570       _$E31                      00509570 f   Story.obj
 0001:00108590       _$E33                      00509590 f   Story.obj
 0001:001085b0       _$E35                      005095b0 f   Story.obj
 0001:001085d0       _$E37                      005095d0 f   Story.obj
 0001:001085f0       _$E39                      005095f0 f   Story.obj
 0001:00108610       _$E41                      00509610 f   Story.obj
 0001:00108630       _$E43                      00509630 f   Story.obj
 0001:00108650       _$E45                      00509650 f   Story.obj
 0001:0010865f       _$E5                       0050965f f   atls:atlbase.obj
 0001:00108680       _$E26                      00509680 f   Fog.obj
 0001:00108690       _$E18                      00509690 f   Lightning.obj
 0001:001086a0       _$E28                      005096a0 f   Rain.obj
 0001:001086b0       _$E26                      005096b0 f   SunBeam.obj
 0001:001086c0       _$E34                      005096c0 f   Weather.obj
 0001:001086d0       _$E16                      005096d0 f   WorldMap.obj
 0001:001086e0       _$E44                      005096e0 f   EnvironmentalSound.obj
 0001:001086f0       _$E44                      005096f0 f   Sound.obj
 0001:00108700       _$E44                      00509700 f   SoundTrack.obj
 0001:00108710       _$E28                      00509710 f   Bird.obj
 0001:00108720       _$E44                      00509720 f   FloatingAnim.obj
 0001:00108730       _$E16                      00509730 f   MoviePlayer.obj
 0001:00108740       _$E6                       00509740 f   FlashPlayer.obj
 0001:00108750       _$E2                       00509750 f   FlashPlayer.obj
 0001:0010875f       _$E6                       0050975f f   atls:atlbase.obj
